 wzSound_d

 Timestamp is 56cd519b (Wed Feb 24 15:45:47 2016)

 Preferred load address is 10000000

 Start         Length     Name                   Class
 0001:00000000 000705b5H .textbss                DATA
 0002:00000000 00101e43H .text                   CODE
 0002:00101e50 000040eaH .text$x                 CODE
 0002:00105f40 000012fdH .text$yc                CODE
 0002:00107240 00001268H .text$yd                CODE
 0003:00000000 00000104H .CRT$XCA                DATA
 0003:00000104 00000104H .CRT$XCC                DATA
 0003:00000208 0000013eH .CRT$XCU                DATA
 0003:00000348 00000104H .CRT$XCZ                DATA
 0003:0000044c 00000104H .CRT$XIA                DATA
 0003:00000550 00000118H .CRT$XIC                DATA
 0003:00000668 00000104H .CRT$XIZ                DATA
 0003:0000076c 00000104H .CRT$XPA                DATA
 0003:00000870 00000109H .CRT$XPX                DATA
 0003:0000097c 00000104H .CRT$XPXA               DATA
 0003:00000a80 00000104H .CRT$XPZ                DATA
 0003:00000b84 00000104H .CRT$XTA                DATA
 0003:00000c88 00000104H .CRT$XTZ                DATA
 0003:00000d90 0011b832H .rdata                  DATA
 0003:0011c5c4 00000173H .rdata$debug            DATA
 0003:0011c738 00000502H .rdata$r                DATA
 0003:0011cc3c 00000104H .rtc$IAA                DATA
 0003:0011cd40 0000019eH .rtc$IMZ                DATA
 0003:0011cee0 00000104H .rtc$IZZ                DATA
 0003:0011cfe4 00000104H .rtc$TAA                DATA
 0003:0011d0e8 0000019eH .rtc$TMZ                DATA
 0003:0011d288 00000104H .rtc$TZZ                DATA
 0003:0011d390 00004337H .xdata$x                DATA
 0003:001216d0 00000d3eH .edata                  DATA
 0004:00000000 00014ffbH .data                   DATA
 0004:00015000 0010f028H .bss                    DATA
 0005:00000000 00000064H .idata$2                DATA
 0005:00000064 00000014H .idata$3                DATA
 0005:00000078 00000380H .idata$4                DATA
 0005:000003f8 00000380H .idata$5                DATA
 0005:00000778 00000c60H .idata$6                DATA
 0006:00000000 000001c0H .rsrc$01                DATA
 0006:000001c0 00000e29H .rsrc$02                DATA

  Address         Publics by Value              Rva+Base       Lib:Object

 0000:00000000       __except_list              00000000     <absolute>
 0000:00000000       ___safe_se_handler_count   00000000     <absolute>
 0000:00000000       ___safe_se_handler_table   00000000     <absolute>
 0000:00000000       ___ImageBase               10000000     <linker-defined>
 0001:00000000       __enc$textbss$begin        10001000     <linker-defined>
 0001:000705b5       __enc$textbss$end          100715b5     <linker-defined>
 0002:000079e0       ?Constructor@AudioStreamServices@@QAEXXZ 100799e0 f   audiostr.obj
 0002:00007a00       ?Initialize@AudioStreamServices@@QAEHXZ 10079a00 f   audiostr.obj
 0002:00007a40       ??0AudioStream@@QAE@XZ     10079a40 f   audiostr.obj
 0002:00007a80       ??1AudioStream@@QAE@XZ     10079a80 f   audiostr.obj
 0002:00007ac0       ?Init_Data@AudioStream@@QAEXXZ 10079ac0 f   audiostr.obj
 0002:00007bd0       ?Create@AudioStream@@QAEHPADHPAVAudioStreamServices@@@Z 10079bd0 f   audiostr.obj
 0002:00007e10       ?Destroy@AudioStream@@QAEHXZ 10079e10 f   audiostr.obj
 0002:00007f10       ?WriteWaveData@AudioStream@@IAEHIPAIH@Z 10079f10 f   audiostr.obj
 0002:000081e0       ?WriteSilence@AudioStream@@IAEHI@Z 1007a1e0 f   audiostr.obj
 0002:000083a0       ?GetMaxWriteSize@AudioStream@@IAEKXZ 1007a3a0 f   audiostr.obj
 0002:00008490       ?ServiceBuffer@AudioStream@@IAEHXZ 1007a490 f   audiostr.obj
 0002:00008920       ?Cue@AudioStream@@IAEXXZ   1007a920 f   audiostr.obj
 0002:00008a40       ?Play@AudioStream@@QAEXJH@Z 1007aa40 f   audiostr.obj
 0002:00008bf0       ?TimerCallback@AudioStream@@KAHK@Z 1007abf0 f   audiostr.obj
 0002:00008c20       ?Set_Sample_Cutoff@AudioStream@@QAEXI@Z 1007ac20 f   audiostr.obj
 0002:00008c60       ?Get_Samples_Committed@AudioStream@@QAEIXZ 1007ac60 f   audiostr.obj
 0002:00008ca0       ?Fade_and_Destroy@AudioStream@@QAEXXZ 1007aca0 f   audiostr.obj
 0002:00008cd0       ?Fade_and_Stop@AudioStream@@QAEXXZ 1007acd0 f   audiostr.obj
 0002:00008d00       ?Stop@AudioStream@@QAEXH@Z 1007ad00 f   audiostr.obj
 0002:00008d70       ?Stop_and_Rewind@AudioStream@@QAEXXZ 1007ad70 f   audiostr.obj
 0002:00008de0       ?Set_Volume@AudioStream@@QAEXJ@Z 1007ade0 f   audiostr.obj
 0002:00008ea0       ?Get_Volume@AudioStream@@QAEJXZ 1007aea0 f   audiostr.obj
 0002:00008ec0       ?constructor@Timer@@QAEXXZ 1007aec0 f   audiostr.obj
 0002:00008ee0       ?destructor@Timer@@QAEXXZ  1007aee0 f   audiostr.obj
 0002:00008f30       ?Create@Timer@@QAEHIIKP6AHK@Z@Z 1007af30 f   audiostr.obj
 0002:00008fd0       ?TimeProc@Timer@@KGXIIKKK@Z 1007afd0 f   audiostr.obj
 0002:00009010       ?Init@WaveFile@@QAEXXZ     1007b010 f   audiostr.obj
 0002:000090b0       ?Close@WaveFile@@QAEXXZ    1007b0b0 f   audiostr.obj
 0002:00009170       ?Open@WaveFile@@QAEHPAD@Z  1007b170 f   audiostr.obj
 0002:00009680       ?Cue@WaveFile@@QAEHXZ      1007b680 f   audiostr.obj
 0002:00009740       ?Read@WaveFile@@QAEHPAEIH@Z 1007b740 f   audiostr.obj
 0002:000099f0       ?GetSilenceData@WaveFile@@QAEEXZ 1007b9f0 f   audiostr.obj
 0002:00009a50       ?audiostream_init@@YAXXZ   1007ba50 f   audiostr.obj
 0002:00009b10       ?audiostream_close@@YAXXZ  1007bb10 f   audiostr.obj
 0002:00009bb0       ?audiostream_open@@YAHPADHMH@Z 1007bbb0 f   audiostr.obj
 0002:00009cc0       ?audiostream_close_file@@YAXHH@Z 1007bcc0 f   audiostr.obj
 0002:00009d30       ?audiostream_close_all@@YAXHH@Z 1007bd30 f   audiostr.obj
 0002:00009db0       ?audiostream_play@@YAXHMHH@Z 1007bdb0 f   audiostr.obj
 0002:00009e60       ?audiostream_stop@@YAXHHH@Z 1007be60 f   audiostr.obj
 0002:00009ec0       ?audiostream_is_playing@@YAHH@Z 1007bec0 f   audiostr.obj
 0002:00009f10       ?audiostream_set_volume_all@@YAXMH@Z 1007bf10 f   audiostr.obj
 0002:00009fd0       ?audiostream_set_volume@@YAXHM@Z 1007bfd0 f   audiostr.obj
 0002:0000a060       ?audiostream_is_paused@@YAHH@Z 1007c060 f   audiostr.obj
 0002:0000a0c0       ?audiostream_set_looping@@YAXHH@Z 1007c0c0 f   audiostr.obj
 0002:0000a110       ?audiostream_set_sample_cutoff@@YAXHI@Z 1007c110 f   audiostr.obj
 0002:0000a160       ?audiostream_get_samples_committed@@YAIH@Z 1007c160 f   audiostr.obj
 0002:0000a1b0       ?audiostream_done_reading@@YAHH@Z 1007c1b0 f   audiostr.obj
 0002:0000a210       ?audiostream_is_inited@@YAHXZ 1007c210 f   audiostr.obj
 0002:0000a220       ?audiostream_pause@@YAXH@Z 1007c220 f   audiostr.obj
 0002:0000a270       ?audiostream_pause_all@@YAXH@Z 1007c270 f   audiostr.obj
 0002:0000a2e0       ?audiostream_unpause@@YAXH@Z 1007c2e0 f   audiostr.obj
 0002:0000a360       ?audiostream_unpause_all@@YAXH@Z 1007c360 f   audiostr.obj
 0002:0000ae50       ?GetUncompressedAvgDataRate@WaveFile@@QAEIXZ 1007ce50 f i audiostr.obj
 0002:0000ae70       ?GetPDS@AudioStreamServices@@QAEPAUIDirectSound8@@XZ 1007ce70 f i audiostr.obj
 0002:0000ae90       ?Set_Base_Volume@AudioStream@@QAEXM@Z 1007ce90 f i audiostr.obj
 0002:0000aec0       ?Set_Default_Volume@AudioStream@@QAEXJ@Z 1007cec0 f i audiostr.obj
 0002:0000aef0       ?Get_Default_Volume@AudioStream@@QAEJXZ 1007cef0 f i audiostr.obj
 0002:0000af20       ?Is_Playing@AudioStream@@QAEHXZ 1007cf20 f i audiostr.obj
 0002:0000af40       ?Get_Base_Volume@AudioStream@@QAEMXZ 1007cf40 f i audiostr.obj
 0002:0000af70       ?Is_Paused@AudioStream@@QAEHXZ 1007cf70 f i audiostr.obj
 0002:0000afa0       ?Set_looping@AudioStream@@QAEXH@Z 1007cfa0 f i audiostr.obj
 0002:0000afd0       ?Is_Past_Limit@AudioStream@@QAEHXZ 1007cfd0 f i audiostr.obj
 0002:0000b000       ?Is_looping@AudioStream@@QAEHXZ 1007d000 f i audiostr.obj
 0002:0000b020       ?ds_is_3d_buffer@@YAHPAUIDirectSoundBuffer@@@Z 1007d020 f   ds.obj
 0002:0000b0d0       ?ds_is_3d_buffer@@YAHHH@Z  1007d0d0 f   ds.obj
 0002:0000b100       ?ds_build_vol_lookup@@YAXXZ 1007d100 f   ds.obj
 0002:0000b190       ?ds_convert_volume@@YAHM@Z 1007d190 f   ds.obj
 0002:0000b1e0       ?ds_get_percentage_vol@@YAMH@Z 1007d1e0 f   ds.obj
 0002:0000b240       ?ds_parse_sound@@YAHPAUCFILE@@PAPAEPAIPAPAUtWAVEFORMATEX@@PAUOggVorbis_File@@@Z 1007d240 f   ds.obj
 0002:0000b4d0       ?ds_get_sid@@YAHXZ         1007d4d0 f   ds.obj
 0002:0000b540       ?ds_get_hid@@YAHXZ         1007d540 f   ds.obj
 0002:0000b5b0       ?ds_load_buffer@@YAHPAH00PAXPAUsound_info@@H@Z 1007d5b0 f   ds.obj
 0002:0000bc20       ?ds_init_channels@@YAXXZ   1007dc20 f   ds.obj
 0002:0000bdb0       ?ds_init_software_buffers@@YAXXZ 1007ddb0 f   ds.obj
 0002:0000bdf0       ?ds_init_hardware_buffers@@YAXXZ 1007ddf0 f   ds.obj
 0002:0000be30       ?ds_init_buffers@@YAXXZ    1007de30 f   ds.obj
 0002:0000be50       ?ds_get_soundcard_caps@@YAXPAU_DSCAPS@@@Z 1007de50 f   ds.obj
 0002:0000bef0       ?ds_show_caps@@YAXPAU_DSCAPS@@@Z 1007def0 f   ds.obj
 0002:0000c0b0       ?ds_get_primary_format@@YAXPAUtWAVEFORMATEX@@KG@Z 1007e0b0 f   ds.obj
 0002:0000c120       ?ds_dll_get_functions@@YAXXZ 1007e120 f   ds.obj
 0002:0000c150       ?ds_dll_load@@YAHXZ        1007e150 f   ds.obj
 0002:0000c1a0       ?ds_init_property_set@@YAHKG@Z 1007e1a0 f   ds.obj
 0002:0000c350       ?ds_init@@YAHHIG@Z         1007e350 f   ds.obj
 0002:0000c780       ?get_DSERR_text@@YAPADH@Z  1007e780 f   ds.obj
 0002:0000c990       ?ds_close_channel@@YAXH@Z  1007e990 f   ds.obj
 0002:0000cb50       ?ds_close_all_channels@@YAXXZ 1007eb50 f   ds.obj
 0002:0000cba0       ?ds_unload_buffer@@YAXHH@Z 1007eba0 f   ds.obj
 0002:0000ccb0       ?ds_close_software_buffers@@YAXXZ 1007ecb0 f   ds.obj
 0002:0000cd70       ?ds_close_hardware_buffers@@YAXXZ 1007ed70 f   ds.obj
 0002:0000ce30       ?ds_close_buffers@@YAXXZ   1007ee30 f   ds.obj
 0002:0000ce50       ?ds_close@@YAXXZ           1007ee50 f   ds.obj
 0002:0000cfa0       ?ds_get_3d_interface@@YAXPAUIDirectSoundBuffer@@PAPAUIDirectSound3DBuffer@@@Z 1007efa0 f   ds.obj
 0002:0000d080       ?ds_get_free_channel@@YAHHHH@Z 1007f080 f   ds.obj
 0002:0000d320       ?ds_channel_dup@@YAHPAUIDirectSoundBuffer@@HH@Z 1007f320 f   ds.obj
 0002:0000d400       ?ds_restore_buffer@@YAXPAUIDirectSoundBuffer@@@Z 1007f400 f   ds.obj
 0002:0000d460       ?ds_create_buffer@@YAHHHHH@Z 1007f460 f   ds.obj
 0002:0000d600       ?ds_lock_data@@YAHHPAEH@Z  1007f600 f   ds.obj
 0002:0000d7c0       ?ds_stop_easy@@YAXH@Z      1007f7c0 f   ds.obj
 0002:0000d820       ?ds_play_easy@@YAHHH@Z     1007f820 f   ds.obj
 0002:0000d8a0       ?ds_play@@YAHHHHHHHH_NH@Z  1007f8a0 f   ds.obj
 0002:0000dbc0       ?ds_get_channel@@YAHH@Z    1007fbc0 f   ds.obj
 0002:0000dc50       ?ds_find_channel@@YAPAUchannel@@HPAH@Z 1007fc50 f   ds.obj
 0002:0000dd10       ?ds_is_channel_playing@@YAHH@Z 1007fd10 f   ds.obj
 0002:0000ddf0       ?ds_stop_channel@@YAXH@Z   1007fdf0 f   ds.obj
 0002:0000de10       ?ds_stop_channel_all@@YAXXZ 1007fe10 f   ds.obj
 0002:0000de70       ?ds_pause_channel@@YAXH@Z  1007fe70 f   ds.obj
 0002:0000e000       ?ds_pause_channel_all@@YAXXZ 10080000 f   ds.obj
 0002:0000e060       ?ds_unpause_channel@@YAXH@Z 10080060 f   ds.obj
 0002:0000e1f0       ?ds_unpause_channel_all@@YAXXZ 100801f0 f   ds.obj
 0002:0000e250       ?ds_set_volume@@YAXHH@Z    10080250 f   ds.obj
 0002:0000e460       ?ds_set_volume_all@@YAXH@Z 10080460 f   ds.obj
 0002:0000e4c0       ?ds_set_pan@@YAXHH@Z       100804c0 f   ds.obj
 0002:0000e5b0       ?ds_get_pitch@@YAHH@Z      100805b0 f   ds.obj
 0002:0000e700       ?ds_set_pitch@@YAXHH@Z     10080700 f   ds.obj
 0002:0000e810       ?ds_chg_loop_status@@YAXHH@Z 10080810 f   ds.obj
 0002:0000e970       ?ds3d_play@@YAHPAUgame_snd@@HHHPAUvector@@1HHHHHHHPAUSND_DIRECTION@@@Z 10080970 f   ds.obj
 0002:0000ed40       ?ds_set_position@@YAXHK@Z  10080d40 f   ds.obj
 0002:0000ed90       ?ds_get_play_position@@YAKH@Z 10080d90 f   ds.obj
 0002:0000ee60       ?ds_get_write_position@@YAKH@Z 10080e60 f   ds.obj
 0002:0000ef30       ?ds_get_channel_size@@YAHH@Z 10080f30 f   ds.obj
 0002:0000f020       ?ds_get_number_channels@@YAHXZ 10081020 f   ds.obj
 0002:0000f0a0       ?ds_get_data@@YAHHPAD@Z    100810a0 f   ds.obj
 0002:0000f200       ?ds_get_size@@YAHHPAH@Z    10081200 f   ds.obj
 0002:0000f2c0       ?ds_using_ds3d@@YAHXZ      100812c0 f   ds.obj
 0002:0000f2d0       ?ds_get_primary_buffer_interface@@YAIXZ 100812d0 f   ds.obj
 0002:0000f2e0       ?ds_get_dsound_interface@@YAIXZ 100812e0 f   ds.obj
 0002:0000f2f0       ?ds_get_property_set_interface@@YAIXZ 100812f0 f   ds.obj
 0002:0000f300       ?ds_eax_set_volume@@YAHM@Z 10081300 f   ds.obj
 0002:0000f390       ?ds_eax_set_decay_time@@YAHM@Z 10081390 f   ds.obj
 0002:0000f420       ?ds_eax_set_damping@@YAHM@Z 10081420 f   ds.obj
 0002:0000f4b0       ?ds_eax_set_environment@@YAHK@Z 100814b0 f   ds.obj
 0002:0000f520       ?ds_eax_set_preset@@YAHK@Z 10081520 f   ds.obj
 0002:0000f5a0       ?ds_eax_set_all@@YAHKMMM@Z 100815a0 f   ds.obj
 0002:0000f670       ?ds_eax_get_all@@YAHPAUEAX_REVERBPROPERTIES@@@Z 10081670 f   ds.obj
 0002:0000f720       ?ds_eax_close@@YAXXZ       10081720 f   ds.obj
 0002:0000f740       ?ds_eax_init@@YAHXZ        10081740 f   ds.obj
 0002:0000f890       ?ds_eax_is_inited@@YAHXZ   10081890 f   ds.obj
 0002:0000f8a0       ?ds_do_frame@@YAXXZ        100818a0 f   ds.obj
 0002:00010ba0       ?log@@YAMM@Z               10082ba0 f i ds.obj
 0002:00010bd0       _logf                      10082bd0 f i ds.obj
 0002:00010c10       ??1iterator@?$_Tree@V?$_Tmap_traits@HUgame_snd@@U?$less@H@std@@V?$allocator@U?$pair@$$CBHUgame_snd@@@std@@@3@$0A@@std@@@std@@QAE@XZ 10082c10 f i ds.obj
 0002:00010c40       ??1const_iterator@?$_Tree@V?$_Tmap_traits@HUgame_snd@@U?$less@H@std@@V?$allocator@U?$pair@$$CBHUgame_snd@@@std@@@3@$0A@@std@@@std@@QAE@XZ 10082c40 f i ds.obj
 0002:00010c70       ??1?$_Bidit@U?$pair@$$CBHUgame_snd@@@std@@HPBU12@ABU12@@std@@QAE@XZ 10082c70 f i ds.obj
 0002:00010ca0       ??1?$_Iterator_with_base@Ubidirectional_iterator_tag@std@@U?$pair@$$CBHUgame_snd@@@2@HPBU32@ABU32@V_Iterator_base@2@@std@@QAE@XZ 10082ca0 f i ds.obj
 0002:00010cd0       ??1_Iterator_base@std@@QAE@XZ 10082cd0 f i ds.obj
 0002:00010da0       ?_Orphan_me@_Iterator_base@std@@QAEXXZ 10082da0 f i ds.obj
 0002:00010e60       ?end@?$_Tree@V?$_Tmap_traits@HUgame_snd@@U?$less@H@std@@V?$allocator@U?$pair@$$CBHUgame_snd@@@std@@@3@$0A@@std@@@std@@QAE?AViterator@12@XZ 10082e60 f i ds.obj
 0002:00010ec0       ?find@?$_Tree@V?$_Tmap_traits@HUgame_snd@@U?$less@H@std@@V?$allocator@U?$pair@$$CBHUgame_snd@@@std@@@3@$0A@@std@@@std@@QAE?AViterator@12@ABH@Z 10082ec0 f i ds.obj
 0002:000110d0       ??Citerator@?$_Tree@V?$_Tmap_traits@HUgame_snd@@U?$less@H@std@@V?$allocator@U?$pair@$$CBHUgame_snd@@@std@@@3@$0A@@std@@@std@@QBEPAU?$pair@$$CBHUgame_snd@@@2@XZ 100830d0 f i ds.obj
 0002:00011100       ??8const_iterator@?$_Tree@V?$_Tmap_traits@HUgame_snd@@U?$less@H@std@@V?$allocator@U?$pair@$$CBHUgame_snd@@@std@@@3@$0A@@std@@@std@@QBE_NABV012@@Z 10083100 f i ds.obj
 0002:000111d0       ??0iterator@?$_Tree@V?$_Tmap_traits@HUgame_snd@@U?$less@H@std@@V?$allocator@U?$pair@$$CBHUgame_snd@@@std@@@3@$0A@@std@@@std@@QAE@ABV012@@Z 100831d0 f i ds.obj
 0002:00011210       ??0const_iterator@?$_Tree@V?$_Tmap_traits@HUgame_snd@@U?$less@H@std@@V?$allocator@U?$pair@$$CBHUgame_snd@@@std@@@3@$0A@@std@@@std@@QAE@ABV012@@Z 10083210 f i ds.obj
 0002:00011260       ??0?$_Bidit@U?$pair@$$CBHUgame_snd@@@std@@HPBU12@ABU12@@std@@QAE@ABU01@@Z 10083260 f i ds.obj
 0002:000112a0       ??0?$_Iterator_with_base@Ubidirectional_iterator_tag@std@@U?$pair@$$CBHUgame_snd@@@2@HPBU32@ABU32@V_Iterator_base@2@@std@@QAE@ABU01@@Z 100832a0 f i ds.obj
 0002:000112e0       ??0_Iterator_base@std@@QAE@ABV01@@Z 100832e0 f i ds.obj
 0002:00011330       ??4_Iterator_base@std@@QAEAAV01@ABV01@@Z 10083330 f i ds.obj
 0002:00011430       ?_Adopt@_Iterator_base@std@@QAEXPBV_Container_base_secure@2@@Z 10083430 f i ds.obj
 0002:00011540       ?_Key@?$_Tree@V?$_Tmap_traits@HUgame_snd@@U?$less@H@std@@V?$allocator@U?$pair@$$CBHUgame_snd@@@std@@@3@$0A@@std@@@std@@KAABHPAU_Node@?$_Tree_nod@V?$_Tmap_traits@HUgame_snd@@U?$less@H@std@@V?$allocator@U?$pair@$$CBHUgame_snd@@@std@@@3@$0A@@std@@@2@@Z 10083540 f i ds.obj
 0002:00011570       ?lower_bound@?$_Tree@V?$_Tmap_traits@HUgame_snd@@U?$less@H@std@@V?$allocator@U?$pair@$$CBHUgame_snd@@@std@@@3@$0A@@std@@@std@@QAE?AViterator@12@ABH@Z 10083570 f i ds.obj
 0002:000115e0       ??0iterator@?$_Tree@V?$_Tmap_traits@HUgame_snd@@U?$less@H@std@@V?$allocator@U?$pair@$$CBHUgame_snd@@@std@@@3@$0A@@std@@@std@@QAE@PAU_Node@?$_Tree_nod@V?$_Tmap_traits@HUgame_snd@@U?$less@H@std@@V?$allocator@U?$pair@$$CBHUgame_snd@@@std@@@3@$0A@@std@@@2@PBV12@@Z 100835e0 f i ds.obj
 0002:00011620       ??Diterator@?$_Tree@V?$_Tmap_traits@HUgame_snd@@U?$less@H@std@@V?$allocator@U?$pair@$$CBHUgame_snd@@@std@@@3@$0A@@std@@@std@@QBEAAU?$pair@$$CBHUgame_snd@@@2@XZ 10083620 f i ds.obj
 0002:00011650       ?_Mynode@const_iterator@?$_Tree@V?$_Tmap_traits@HUgame_snd@@U?$less@H@std@@V?$allocator@U?$pair@$$CBHUgame_snd@@@std@@@3@$0A@@std@@@std@@QBEPAU_Node@?$_Tree_nod@V?$_Tmap_traits@HUgame_snd@@U?$less@H@std@@V?$allocator@U?$pair@$$CBHUgame_snd@@@std@@@3@$0A@@std@@@3@XZ 10083650 f i ds.obj
 0002:00011670       ?_Myval@?$_Tree@V?$_Tmap_traits@HUgame_snd@@U?$less@H@std@@V?$allocator@U?$pair@$$CBHUgame_snd@@@std@@@3@$0A@@std@@@std@@KAAAU?$pair@$$CBHUgame_snd@@@2@PAU_Node@?$_Tree_nod@V?$_Tmap_traits@HUgame_snd@@U?$less@H@std@@V?$allocator@U?$pair@$$CBHUgame_snd@@@std@@@3@$0A@@std@@@2@@Z 10083670 f i ds.obj
 0002:00011680       ?_Lbound@?$_Tree@V?$_Tmap_traits@HUgame_snd@@U?$less@H@std@@V?$allocator@U?$pair@$$CBHUgame_snd@@@std@@@3@$0A@@std@@@std@@IBEPAU_Node@?$_Tree_nod@V?$_Tmap_traits@HUgame_snd@@U?$less@H@std@@V?$allocator@U?$pair@$$CBHUgame_snd@@@std@@@3@$0A@@std@@@2@ABH@Z 10083680 f i ds.obj
 0002:00011770       ?_Kfn@?$_Tmap_traits@HUgame_snd@@U?$less@H@std@@V?$allocator@U?$pair@$$CBHUgame_snd@@@std@@@3@$0A@@std@@SAABHABU?$pair@$$CBHUgame_snd@@@2@@Z 10083770 f i ds.obj
 0002:00011780       ??0const_iterator@?$_Tree@V?$_Tmap_traits@HUgame_snd@@U?$less@H@std@@V?$allocator@U?$pair@$$CBHUgame_snd@@@std@@@3@$0A@@std@@@std@@QAE@PAU_Node@?$_Tree_nod@V?$_Tmap_traits@HUgame_snd@@U?$less@H@std@@V?$allocator@U?$pair@$$CBHUgame_snd@@@std@@@3@$0A@@std@@@2@PBV12@@Z 10083780 f i ds.obj
 0002:00011820       ??Dconst_iterator@?$_Tree@V?$_Tmap_traits@HUgame_snd@@U?$less@H@std@@V?$allocator@U?$pair@$$CBHUgame_snd@@@std@@@3@$0A@@std@@@std@@QBEABU?$pair@$$CBHUgame_snd@@@2@XZ 10083820 f i ds.obj
 0002:000118f0       ??0?$_Bidit@U?$pair@$$CBHUgame_snd@@@std@@HPBU12@ABU12@@std@@QAE@XZ 100838f0 f i ds.obj
 0002:00011920       ??0?$_Iterator_with_base@Ubidirectional_iterator_tag@std@@U?$pair@$$CBHUgame_snd@@@2@HPBU32@ABU32@V_Iterator_base@2@@std@@QAE@XZ 10083920 f i ds.obj
 0002:00011950       ??0_Iterator_base@std@@QAE@XZ 10083950 f i ds.obj
 0002:00011990       ?_Isnil@?$_Tree@V?$_Tmap_traits@HUgame_snd@@U?$less@H@std@@V?$allocator@U?$pair@$$CBHUgame_snd@@@std@@@3@$0A@@std@@@std@@KAAADPAU_Node@?$_Tree_nod@V?$_Tmap_traits@HUgame_snd@@U?$less@H@std@@V?$allocator@U?$pair@$$CBHUgame_snd@@@std@@@3@$0A@@std@@@2@@Z 10083990 f i ds.obj
 0002:000119a0       ?_Left@?$_Tree@V?$_Tmap_traits@HUgame_snd@@U?$less@H@std@@V?$allocator@U?$pair@$$CBHUgame_snd@@@std@@@3@$0A@@std@@@std@@KAAAPAU_Node@?$_Tree_nod@V?$_Tmap_traits@HUgame_snd@@U?$less@H@std@@V?$allocator@U?$pair@$$CBHUgame_snd@@@std@@@3@$0A@@std@@@2@PAU342@@Z 100839a0 f i ds.obj
 0002:000119b0       ?_Right@?$_Tree@V?$_Tmap_traits@HUgame_snd@@U?$less@H@std@@V?$allocator@U?$pair@$$CBHUgame_snd@@@std@@@3@$0A@@std@@@std@@KAAAPAU_Node@?$_Tree_nod@V?$_Tmap_traits@HUgame_snd@@U?$less@H@std@@V?$allocator@U?$pair@$$CBHUgame_snd@@@std@@@3@$0A@@std@@@2@PAU342@@Z 100839b0 f i ds.obj
 0002:000119c0       ?_Root@?$_Tree@V?$_Tmap_traits@HUgame_snd@@U?$less@H@std@@V?$allocator@U?$pair@$$CBHUgame_snd@@@std@@@3@$0A@@std@@@std@@IBEAAPAU_Node@?$_Tree_nod@V?$_Tmap_traits@HUgame_snd@@U?$less@H@std@@V?$allocator@U?$pair@$$CBHUgame_snd@@@std@@@3@$0A@@std@@@2@XZ 100839c0 f i ds.obj
 0002:00011a00       ?_Parent@?$_Tree@V?$_Tmap_traits@HUgame_snd@@U?$less@H@std@@V?$allocator@U?$pair@$$CBHUgame_snd@@@std@@@3@$0A@@std@@@std@@KAAAPAU_Node@?$_Tree_nod@V?$_Tmap_traits@HUgame_snd@@U?$less@H@std@@V?$allocator@U?$pair@$$CBHUgame_snd@@@std@@@3@$0A@@std@@@2@PAU342@@Z 10083a00 f i ds.obj
 0002:00011a10       ??$CAP@M@@YAXAAMMM@Z       10083a10 f i ds.obj
 0002:00011a60       ??$_Debug_lt_pred@U?$less@H@std@@HH@std@@YA_NU?$less@H@0@ABH1PB_WI@Z 10083a60 f i ds.obj
 0002:00011ad0       ??R?$less@H@std@@QBE_NABH0@Z 10083ad0 f i ds.obj
 0002:00011b00       ?ds3d_update_buffer@@YAHHPAUgame_snd@@MMPAUvector@@1@Z 10083b00 f   ds3d.obj
 0002:00011da0       ?ds3d_set_sound_cone@@YAHHPAUvector@@HHH@Z 10083da0 f   ds3d.obj
 0002:00011f00       ?ds3d_update_listener@@YAHPAUvector@@0PAUmatrix@@MMM@Z 10083f00 f   ds3d.obj
 0002:00012110       ?ds3d_init_listener@@YAHXZ 10084110 f   ds3d.obj
 0002:00012190       ?ds3d_close_listener@@YAXXZ 10084190 f   ds3d.obj
 0002:000121d0       ?ds3d_init@@YAHH@Z         100841d0 f   ds3d.obj
 0002:00012370       ?ds3d_close@@YAXXZ         10084370 f   ds3d.obj
 0002:000125c0       ?sound_size@@YAHXZ         100845c0 f   sound.obj
 0002:000125e0       ?sound_get@@YAPAUsound@@H@Z 100845e0 f   sound.obj
 0002:000126f0       ?sound_cache_reset@@YAXXZ  100846f0 f   sound.obj
 0002:00012710       ?sound_cache_maintain_milliseconds_set@@YAXH@Z 10084710 f   sound.obj
 0002:00012720       ?sound_cache_maintain_milliseconds_get@@YAHXZ 10084720 f   sound.obj
 0002:00012730       ?sound_cache_on@@YAXXZ     10084730 f   sound.obj
 0002:00012740       ?sound_cache_off@@YAXXZ    10084740 f   sound.obj
 0002:00012750       ?sound_cache_is@@YA_NXZ    10084750 f   sound.obj
 0002:00012760       ?ds_priority@@YAHH@Z       10084760 f   sound.obj
 0002:000127b0       ?snd_clear@@YAXXZ          100847b0 f   sound.obj
 0002:000127d0       ?snd_init@@YAHHIG@Z        100847d0 f   sound.obj
 0002:00012920       ?snd_load@@YAPAUsound@@PAUgame_snd@@H@Z 10084920 f   sound.obj
 0002:00012ce0       ?snd_unload@@YAHH@Z        10084ce0 f   sound.obj
 0002:00012d40       ?snd_unload@@YAXPAUsound@@@Z 10084d40 f   sound.obj
 0002:00012da0       ?snd_unload_all@@YAXXZ     10084da0 f   sound.obj
 0002:00012eb0       ?snd_close@@YAXXZ          10084eb0 f   sound.obj
 0002:00012ef0       ?snd_play@@YAHPAUgame_snd@@MMH_NHH@Z 10084ef0 f   sound.obj
 0002:00013080       ?snd_play_3d@@YAHPAUgame_snd@@PAUvector@@1M1HMH1MHHPAUSND_DIRECTION@@MM@Z 10085080 f   sound.obj
 0002:00013400       ?snd_update_3d_pos@@YAXHPAUgame_snd@@PAUvector@@@Z 10085400 f   sound.obj
 0002:000134b0       ?snd_update_3d_source_position@@YAXHPAUvector@@0MM@Z 100854b0 f   sound.obj
 0002:00013620       ?snd_update_3d_source_orientation@@YAXHPAUvector@@HHM@Z 10085620 f   sound.obj
 0002:00013690       ?snd_get_3d_vol_and_pan@@YAHPAUgame_snd@@PAUvector@@PAM2M@Z 10085690 f   sound.obj
 0002:00013830       ?snd_play_looping@@YAHPAUgame_snd@@MHHMHH@Z 10085830 f   sound.obj
 0002:00013990       ?snd_stop@@YAXH@Z          10085990 f   sound.obj
 0002:000139e0       ?snd_pause@@YAXH@Z         100859e0 f   sound.obj
 0002:00013a30       ?snd_pause_all@@YAXXZ      10085a30 f   sound.obj
 0002:00013a50       ?snd_unpause@@YAXH@Z       10085a50 f   sound.obj
 0002:00013aa0       ?snd_unpause_all@@YAXXZ    10085aa0 f   sound.obj
 0002:00013ac0       ?snd_set_volume@@YAXHM@Z   10085ac0 f   sound.obj
 0002:00013b50       ?snd_set_volume_all@@YAXM@Z 10085b50 f   sound.obj
 0002:00013ba0       ?snd_set_pan@@YAXHM@Z      10085ba0 f   sound.obj
 0002:00013c10       ?snd_get_pitch@@YAHH@Z     10085c10 f   sound.obj
 0002:00013c90       ?snd_set_pitch@@YAXHH@Z    10085c90 f   sound.obj
 0002:00013d00       ?snd_is_playing@@YAHH@Z    10085d00 f   sound.obj
 0002:00013d70       ?snd_chg_loop_status@@YAXHH@Z 10085d70 f   sound.obj
 0002:00013de0       ?snd_stop_all@@YAXXZ       10085de0 f   sound.obj
 0002:00013e00       ?sound_get_ds@@YAIXZ       10085e00 f   sound.obj
 0002:00013e10       ?snd_is_inited@@YAHXZ      10085e10 f   sound.obj
 0002:00013e30       ?snd_update_listener@@YAXPAUvector@@0PAUmatrix@@MMM@Z 10085e30 f   sound.obj
 0002:00013e70       ?snd_num_playing@@YAHXZ    10085e70 f   sound.obj
 0002:00013e90       ?snd_stop_any_sound@@YAXXZ 10085e90 f   sound.obj
 0002:00013ef0       ?sound_env_set@@YAHPAUsound_env@@@Z 10085ef0 f   sound.obj
 0002:00013f70       ?sound_env_set_preset@@YAHK@Z 10085f70 f   sound.obj
 0002:00013f90       ?sound_env_get@@YAHPAUsound_env@@@Z 10085f90 f   sound.obj
 0002:00014020       ?sound_env_disable@@YAHXZ  10086020 f   sound.obj
 0002:000140a0       ?sound_env_supported@@YAHXZ 100860a0 f   sound.obj
 0002:000140c0       ?sound_check_channel@@YAXXZ 100860c0 f   sound.obj
 0002:000140e0       ?sound_update_cache@@YAXXZ 100860e0 f   sound.obj
 0002:00014a80       ??1iterator@?$_Tree@V?$_Tmap_traits@HUsound@@U?$less@H@std@@V?$allocator@U?$pair@$$CBHUsound@@@std@@@3@$0A@@std@@@std@@QAE@XZ 10086a80 f i sound.obj
 0002:00014ab0       ??1const_iterator@?$_Tree@V?$_Tmap_traits@HUsound@@U?$less@H@std@@V?$allocator@U?$pair@$$CBHUsound@@@std@@@3@$0A@@std@@@std@@QAE@XZ 10086ab0 f i sound.obj
 0002:00014ae0       ??1?$_Bidit@U?$pair@$$CBHUsound@@@std@@HPBU12@ABU12@@std@@QAE@XZ 10086ae0 f i sound.obj
 0002:00014b10       ??1?$_Iterator_with_base@Ubidirectional_iterator_tag@std@@U?$pair@$$CBHUsound@@@2@HPBU32@ABU32@V_Iterator_base@2@@std@@QAE@XZ 10086b10 f i sound.obj
 0002:00014b40       ??0const_iterator@?$_Tree@V?$_Tmap_traits@HUsound@@U?$less@H@std@@V?$allocator@U?$pair@$$CBHUsound@@@std@@@3@$0A@@std@@@std@@QAE@ABV012@@Z 10086b40 f i sound.obj
 0002:00014b90       ??4iterator@?$_Tree@V?$_Tmap_traits@HUsound@@U?$less@H@std@@V?$allocator@U?$pair@$$CBHUsound@@@std@@@3@$0A@@std@@@std@@QAEAAV012@ABV012@@Z 10086b90 f i sound.obj
 0002:00014bd0       ??0?$_Bidit@U?$pair@$$CBHUsound@@@std@@HPBU12@ABU12@@std@@QAE@ABU01@@Z 10086bd0 f i sound.obj
 0002:00014c10       ??4const_iterator@?$_Tree@V?$_Tmap_traits@HUsound@@U?$less@H@std@@V?$allocator@U?$pair@$$CBHUsound@@@std@@@3@$0A@@std@@@std@@QAEAAV012@ABV012@@Z 10086c10 f i sound.obj
 0002:00014c60       ??0?$_Iterator_with_base@Ubidirectional_iterator_tag@std@@U?$pair@$$CBHUsound@@@2@HPBU32@ABU32@V_Iterator_base@2@@std@@QAE@ABU01@@Z 10086c60 f i sound.obj
 0002:00014ca0       ??4?$_Bidit@U?$pair@$$CBHUsound@@@std@@HPBU12@ABU12@@std@@QAEAAU01@ABU01@@Z 10086ca0 f i sound.obj
 0002:00014ce0       ??4?$_Iterator_with_base@Ubidirectional_iterator_tag@std@@U?$pair@$$CBHUsound@@@2@HPBU32@ABU32@V_Iterator_base@2@@std@@QAEAAU01@ABU01@@Z 10086ce0 f i sound.obj
 0002:00014d20       ??A?$map@HUsound@@U?$less@H@std@@V?$allocator@U?$pair@$$CBHUsound@@@std@@@3@@std@@QAEAAUsound@@ABH@Z 10086d20 f i sound.obj
 0002:00014fb0       ??0sound@@QAE@XZ           10086fb0 f i sound.obj
 0002:00015030       ?begin@?$_Tree@V?$_Tmap_traits@HUsound@@U?$less@H@std@@V?$allocator@U?$pair@$$CBHUsound@@@std@@@3@$0A@@std@@@std@@QAE?AViterator@12@XZ 10087030 f i sound.obj
 0002:000150a0       ?end@?$_Tree@V?$_Tmap_traits@HUsound@@U?$less@H@std@@V?$allocator@U?$pair@$$CBHUsound@@@std@@@3@$0A@@std@@@std@@QAE?AViterator@12@XZ 100870a0 f i sound.obj
 0002:00015100       ?size@?$_Tree@V?$_Tmap_traits@HUsound@@U?$less@H@std@@V?$allocator@U?$pair@$$CBHUsound@@@std@@@3@$0A@@std@@@std@@QBEIXZ 10087100 f i sound.obj
 0002:00015120       ?erase@?$_Tree@V?$_Tmap_traits@HUsound@@U?$less@H@std@@V?$allocator@U?$pair@$$CBHUsound@@@std@@@3@$0A@@std@@@std@@QAE?AViterator@12@Vconst_iterator@12@@Z 10087120 f i sound.obj
 0002:00015b40       ?erase@?$_Tree@V?$_Tmap_traits@HUsound@@U?$less@H@std@@V?$allocator@U?$pair@$$CBHUsound@@@std@@@3@$0A@@std@@@std@@QAEIABH@Z 10087b40 f i sound.obj
 0002:00015cf0       ?clear@?$_Tree@V?$_Tmap_traits@HUsound@@U?$less@H@std@@V?$allocator@U?$pair@$$CBHUsound@@@std@@@3@$0A@@std@@@std@@QAEXXZ 10087cf0 f i sound.obj
 0002:00015d90       ?find@?$_Tree@V?$_Tmap_traits@HUsound@@U?$less@H@std@@V?$allocator@U?$pair@$$CBHUsound@@@std@@@3@$0A@@std@@@std@@QAE?AViterator@12@ABH@Z 10087d90 f i sound.obj
 0002:00015fa0       ??Citerator@?$_Tree@V?$_Tmap_traits@HUsound@@U?$less@H@std@@V?$allocator@U?$pair@$$CBHUsound@@@std@@@3@$0A@@std@@@std@@QBEPAU?$pair@$$CBHUsound@@@2@XZ 10087fa0 f i sound.obj
 0002:00015fd0       ??Eiterator@?$_Tree@V?$_Tmap_traits@HUsound@@U?$less@H@std@@V?$allocator@U?$pair@$$CBHUsound@@@std@@@3@$0A@@std@@@std@@QAEAAV012@XZ 10087fd0 f i sound.obj
 0002:00016000       ??9const_iterator@?$_Tree@V?$_Tmap_traits@HUsound@@U?$less@H@std@@V?$allocator@U?$pair@$$CBHUsound@@@std@@@3@$0A@@std@@@std@@QBE_NABV012@@Z 10088000 f i sound.obj
 0002:00016050       ??9const_iterator@?$_Tree@V?$_Tmap_traits@HUgame_snd@@U?$less@H@std@@V?$allocator@U?$pair@$$CBHUgame_snd@@@std@@@3@$0A@@std@@@std@@QBE_NABV012@@Z 10088050 f i sound.obj
 0002:000160a0       ??1?$pair@Viterator@?$_Tree@V?$_Tmap_traits@HUsound@@U?$less@H@std@@V?$allocator@U?$pair@$$CBHUsound@@@std@@@3@$0A@@std@@@std@@V123@@std@@QAE@XZ 100880a0 f i sound.obj
 0002:00016120       ??0iterator@?$_Tree@V?$_Tmap_traits@HUsound@@U?$less@H@std@@V?$allocator@U?$pair@$$CBHUsound@@@std@@@3@$0A@@std@@@std@@QAE@ABV012@@Z 10088120 f i sound.obj
 0002:00016160       ?_Color@?$_Tree@V?$_Tmap_traits@HUsound@@U?$less@H@std@@V?$allocator@U?$pair@$$CBHUsound@@@std@@@3@$0A@@std@@@std@@KAAADPAU_Node@?$_Tree_nod@V?$_Tmap_traits@HUsound@@U?$less@H@std@@V?$allocator@U?$pair@$$CBHUsound@@@std@@@3@$0A@@std@@@2@@Z 10088160 f i sound.obj
 0002:00016170       ?_Isnil@?$_Tree@V?$_Tmap_traits@HUsound@@U?$less@H@std@@V?$allocator@U?$pair@$$CBHUsound@@@std@@@3@$0A@@std@@@std@@KAAADPAU_Node@?$_Tree_nod@V?$_Tmap_traits@HUsound@@U?$less@H@std@@V?$allocator@U?$pair@$$CBHUsound@@@std@@@3@$0A@@std@@@2@@Z 10088170 f i sound.obj
 0002:00016180       ?_Key@?$_Tree@V?$_Tmap_traits@HUsound@@U?$less@H@std@@V?$allocator@U?$pair@$$CBHUsound@@@std@@@3@$0A@@std@@@std@@KAABHPAU_Node@?$_Tree_nod@V?$_Tmap_traits@HUsound@@U?$less@H@std@@V?$allocator@U?$pair@$$CBHUsound@@@std@@@3@$0A@@std@@@2@@Z 10088180 f i sound.obj
 0002:000161b0       ?_Left@?$_Tree@V?$_Tmap_traits@HUsound@@U?$less@H@std@@V?$allocator@U?$pair@$$CBHUsound@@@std@@@3@$0A@@std@@@std@@KAAAPAU_Node@?$_Tree_nod@V?$_Tmap_traits@HUsound@@U?$less@H@std@@V?$allocator@U?$pair@$$CBHUsound@@@std@@@3@$0A@@std@@@2@PAU342@@Z 100881b0 f i sound.obj
 0002:000161c0       ?_Parent@?$_Tree@V?$_Tmap_traits@HUsound@@U?$less@H@std@@V?$allocator@U?$pair@$$CBHUsound@@@std@@@3@$0A@@std@@@std@@KAAAPAU_Node@?$_Tree_nod@V?$_Tmap_traits@HUsound@@U?$less@H@std@@V?$allocator@U?$pair@$$CBHUsound@@@std@@@3@$0A@@std@@@2@PAU342@@Z 100881c0 f i sound.obj
 0002:000161d0       ?_Right@?$_Tree@V?$_Tmap_traits@HUsound@@U?$less@H@std@@V?$allocator@U?$pair@$$CBHUsound@@@std@@@3@$0A@@std@@@std@@KAAAPAU_Node@?$_Tree_nod@V?$_Tmap_traits@HUsound@@U?$less@H@std@@V?$allocator@U?$pair@$$CBHUsound@@@std@@@3@$0A@@std@@@2@PAU342@@Z 100881d0 f i sound.obj
 0002:000161e0       ?_Make_iter@?$_Tree@V?$_Tmap_traits@HUsound@@U?$less@H@std@@V?$allocator@U?$pair@$$CBHUsound@@@std@@@3@$0A@@std@@@std@@QBE?AViterator@12@Vconst_iterator@12@@Z 100881e0 f i sound.obj
 0002:000162d0       ?insert@?$_Tree@V?$_Tmap_traits@HUsound@@U?$less@H@std@@V?$allocator@U?$pair@$$CBHUsound@@@std@@@3@$0A@@std@@@std@@QAE?AViterator@12@Vconst_iterator@12@ABU?$pair@$$CBHUsound@@@2@@Z 100882d0 f i sound.obj
 0002:00017140       ?erase@?$_Tree@V?$_Tmap_traits@HUsound@@U?$less@H@std@@V?$allocator@U?$pair@$$CBHUsound@@@std@@@3@$0A@@std@@@std@@QAE?AViterator@12@Vconst_iterator@12@0@Z 10089140 f i sound.obj
 0002:000173d0       ?lower_bound@?$_Tree@V?$_Tmap_traits@HUsound@@U?$less@H@std@@V?$allocator@U?$pair@$$CBHUsound@@@std@@@3@$0A@@std@@@std@@QAE?AViterator@12@ABH@Z 100893d0 f i sound.obj
 0002:00017440       ?equal_range@?$_Tree@V?$_Tmap_traits@HUsound@@U?$less@H@std@@V?$allocator@U?$pair@$$CBHUsound@@@std@@@3@$0A@@std@@@std@@QAE?AU?$pair@Viterator@?$_Tree@V?$_Tmap_traits@HUsound@@U?$less@H@std@@V?$allocator@U?$pair@$$CBHUsound@@@std@@@3@$0A@@std@@@std@@V123@@2@ABH@Z 10089440 f i sound.obj
 0002:000174a0       ?_Erase@?$_Tree@V?$_Tmap_traits@HUsound@@U?$less@H@std@@V?$allocator@U?$pair@$$CBHUsound@@@std@@@3@$0A@@std@@@std@@IAEXPAU_Node@?$_Tree_nod@V?$_Tmap_traits@HUsound@@U?$less@H@std@@V?$allocator@U?$pair@$$CBHUsound@@@std@@@3@$0A@@std@@@2@@Z 100894a0 f i sound.obj
 0002:00017560       ?_Lmost@?$_Tree@V?$_Tmap_traits@HUsound@@U?$less@H@std@@V?$allocator@U?$pair@$$CBHUsound@@@std@@@3@$0A@@std@@@std@@IBEAAPAU_Node@?$_Tree_nod@V?$_Tmap_traits@HUsound@@U?$less@H@std@@V?$allocator@U?$pair@$$CBHUsound@@@std@@@3@$0A@@std@@@2@XZ 10089560 f i sound.obj
 0002:000175a0       ?_Lrotate@?$_Tree@V?$_Tmap_traits@HUsound@@U?$less@H@std@@V?$allocator@U?$pair@$$CBHUsound@@@std@@@3@$0A@@std@@@std@@IAEXPAU_Node@?$_Tree_nod@V?$_Tmap_traits@HUsound@@U?$less@H@std@@V?$allocator@U?$pair@$$CBHUsound@@@std@@@3@$0A@@std@@@2@@Z 100895a0 f i sound.obj
 0002:00017740       ?_Max@?$_Tree@V?$_Tmap_traits@HUsound@@U?$less@H@std@@V?$allocator@U?$pair@$$CBHUsound@@@std@@@3@$0A@@std@@@std@@KAPAU_Node@?$_Tree_nod@V?$_Tmap_traits@HUsound@@U?$less@H@std@@V?$allocator@U?$pair@$$CBHUsound@@@std@@@3@$0A@@std@@@2@PAU342@@Z 10089740 f i sound.obj
 0002:00017790       ?_Min@?$_Tree@V?$_Tmap_traits@HUsound@@U?$less@H@std@@V?$allocator@U?$pair@$$CBHUsound@@@std@@@3@$0A@@std@@@std@@KAPAU_Node@?$_Tree_nod@V?$_Tmap_traits@HUsound@@U?$less@H@std@@V?$allocator@U?$pair@$$CBHUsound@@@std@@@3@$0A@@std@@@2@PAU342@@Z 10089790 f i sound.obj
 0002:000177e0       ?_Rmost@?$_Tree@V?$_Tmap_traits@HUsound@@U?$less@H@std@@V?$allocator@U?$pair@$$CBHUsound@@@std@@@3@$0A@@std@@@std@@IBEAAPAU_Node@?$_Tree_nod@V?$_Tmap_traits@HUsound@@U?$less@H@std@@V?$allocator@U?$pair@$$CBHUsound@@@std@@@3@$0A@@std@@@2@XZ 100897e0 f i sound.obj
 0002:00017820       ?_Root@?$_Tree@V?$_Tmap_traits@HUsound@@U?$less@H@std@@V?$allocator@U?$pair@$$CBHUsound@@@std@@@3@$0A@@std@@@std@@IBEAAPAU_Node@?$_Tree_nod@V?$_Tmap_traits@HUsound@@U?$less@H@std@@V?$allocator@U?$pair@$$CBHUsound@@@std@@@3@$0A@@std@@@2@XZ 10089820 f i sound.obj
 0002:00017860       ?_Rrotate@?$_Tree@V?$_Tmap_traits@HUsound@@U?$less@H@std@@V?$allocator@U?$pair@$$CBHUsound@@@std@@@3@$0A@@std@@@std@@IAEXPAU_Node@?$_Tree_nod@V?$_Tmap_traits@HUsound@@U?$less@H@std@@V?$allocator@U?$pair@$$CBHUsound@@@std@@@3@$0A@@std@@@2@@Z 10089860 f i sound.obj
 0002:00017a00       ?_Orphan_ptr@?$_Tree@V?$_Tmap_traits@HUsound@@U?$less@H@std@@V?$allocator@U?$pair@$$CBHUsound@@@std@@@3@$0A@@std@@@std@@IBEXAAV12@PAU_Node@?$_Tree_nod@V?$_Tmap_traits@HUsound@@U?$less@H@std@@V?$allocator@U?$pair@$$CBHUsound@@@std@@@3@$0A@@std@@@2@@Z 10089a00 f i sound.obj
 0002:00017b00       ?deallocate@?$allocator@U_Node@?$_Tree_nod@V?$_Tmap_traits@HUsound@@U?$less@H@std@@V?$allocator@U?$pair@$$CBHUsound@@@std@@@3@$0A@@std@@@std@@@std@@QAEXPAU_Node@?$_Tree_nod@V?$_Tmap_traits@HUsound@@U?$less@H@std@@V?$allocator@U?$pair@$$CBHUsound@@@std@@@3@$0A@@std@@@2@I@Z 10089b00 f i sound.obj
 0002:00017b40       ?destroy@?$allocator@U_Node@?$_Tree_nod@V?$_Tmap_traits@HUsound@@U?$less@H@std@@V?$allocator@U?$pair@$$CBHUsound@@@std@@@3@$0A@@std@@@std@@@std@@QAEXPAU_Node@?$_Tree_nod@V?$_Tmap_traits@HUsound@@U?$less@H@std@@V?$allocator@U?$pair@$$CBHUsound@@@std@@@3@$0A@@std@@@2@@Z 10089b40 f i sound.obj
 0002:00017b80       ??0iterator@?$_Tree@V?$_Tmap_traits@HUsound@@U?$less@H@std@@V?$allocator@U?$pair@$$CBHUsound@@@std@@@3@$0A@@std@@@std@@QAE@PAU_Node@?$_Tree_nod@V?$_Tmap_traits@HUsound@@U?$less@H@std@@V?$allocator@U?$pair@$$CBHUsound@@@std@@@3@$0A@@std@@@2@PBV12@@Z 10089b80 f i sound.obj
 0002:00017bc0       ??Diterator@?$_Tree@V?$_Tmap_traits@HUsound@@U?$less@H@std@@V?$allocator@U?$pair@$$CBHUsound@@@std@@@3@$0A@@std@@@std@@QBEAAU?$pair@$$CBHUsound@@@2@XZ 10089bc0 f i sound.obj
 0002:00017bf0       ??Econst_iterator@?$_Tree@V?$_Tmap_traits@HUsound@@U?$less@H@std@@V?$allocator@U?$pair@$$CBHUsound@@@std@@@3@$0A@@std@@@std@@QAEAAV012@XZ 10089bf0 f i sound.obj
 0002:00017c20       ??8const_iterator@?$_Tree@V?$_Tmap_traits@HUsound@@U?$less@H@std@@V?$allocator@U?$pair@$$CBHUsound@@@std@@@3@$0A@@std@@@std@@QBE_NABV012@@Z 10089c20 f i sound.obj
 0002:00017cf0       ?_Mynode@const_iterator@?$_Tree@V?$_Tmap_traits@HUsound@@U?$less@H@std@@V?$allocator@U?$pair@$$CBHUsound@@@std@@@3@$0A@@std@@@std@@QBEPAU_Node@?$_Tree_nod@V?$_Tmap_traits@HUsound@@U?$less@H@std@@V?$allocator@U?$pair@$$CBHUsound@@@std@@@3@$0A@@std@@@3@XZ 10089cf0 f i sound.obj
 0002:00017d10       ??0?$pair@$$CBHUsound@@@std@@QAE@ABHABUsound@@@Z 10089d10 f i sound.obj
 0002:00017d60       ??1?$pair@Viterator@?$_Tree@V?$_Tmap_traits@HUsound@@U?$less@H@std@@V?$allocator@U?$pair@$$CBHUsound@@@std@@@3@$0A@@std@@@std@@_N@std@@QAE@XZ 10089d60 f i sound.obj
 0002:00017d90       ?_Myval@?$_Tree@V?$_Tmap_traits@HUsound@@U?$less@H@std@@V?$allocator@U?$pair@$$CBHUsound@@@std@@@3@$0A@@std@@@std@@KAAAU?$pair@$$CBHUsound@@@2@PAU_Node@?$_Tree_nod@V?$_Tmap_traits@HUsound@@U?$less@H@std@@V?$allocator@U?$pair@$$CBHUsound@@@std@@@3@$0A@@std@@@2@@Z 10089d90 f i sound.obj
 0002:00017da0       ?insert@?$_Tree@V?$_Tmap_traits@HUsound@@U?$less@H@std@@V?$allocator@U?$pair@$$CBHUsound@@@std@@@3@$0A@@std@@@std@@QAE?AU?$pair@Viterator@?$_Tree@V?$_Tmap_traits@HUsound@@U?$less@H@std@@V?$allocator@U?$pair@$$CBHUsound@@@std@@@3@$0A@@std@@@std@@_N@2@ABU?$pair@$$CBHUsound@@@2@@Z 10089da0 f i sound.obj
 0002:000181e0       ?_Eqrange@?$_Tree@V?$_Tmap_traits@HUsound@@U?$less@H@std@@V?$allocator@U?$pair@$$CBHUsound@@@std@@@3@$0A@@std@@@std@@IAE?AU?$pair@Viterator@?$_Tree@V?$_Tmap_traits@HUsound@@U?$less@H@std@@V?$allocator@U?$pair@$$CBHUsound@@@std@@@3@$0A@@std@@@std@@V123@@2@ABH@Z 1008a1e0 f i sound.obj
 0002:00018510       ?_Insert@?$_Tree@V?$_Tmap_traits@HUsound@@U?$less@H@std@@V?$allocator@U?$pair@$$CBHUsound@@@std@@@3@$0A@@std@@@std@@IAE?AViterator@12@_NPAU_Node@?$_Tree_nod@V?$_Tmap_traits@HUsound@@U?$less@H@std@@V?$allocator@U?$pair@$$CBHUsound@@@std@@@3@$0A@@std@@@2@ABU?$pair@$$CBHUsound@@@2@@Z 1008a510 f i sound.obj
 0002:00018ae0       ??0length_error@std@@QAE@ABV?$basic_string@DU?$char_traits@D@std@@V?$allocator@D@2@@1@@Z 1008aae0 f i sound.obj
 0002:00018b30       ??0logic_error@std@@QAE@ABV?$basic_string@DU?$char_traits@D@std@@V?$allocator@D@2@@1@@Z 1008ab30 f i sound.obj
 0002:00018bd0       ?what@logic_error@std@@UBEPBDXZ 1008abd0 f i sound.obj
 0002:00018c00       ??_Elogic_error@std@@UAEPAXI@Z 1008ac00 f i sound.obj
 0002:00018c00       ??_Glogic_error@std@@UAEPAXI@Z 1008ac00 f i sound.obj
 0002:00018c50       ??1logic_error@std@@UAE@XZ 1008ac50 f i sound.obj
 0002:00018ca0       ??1length_error@std@@UAE@XZ 1008aca0 f i sound.obj
 0002:00018ce0       ??_Elength_error@std@@UAEPAXI@Z 1008ace0 f i sound.obj
 0002:00018ce0       ??_Glength_error@std@@UAEPAXI@Z 1008ace0 f i sound.obj
 0002:00018d30       ??0?$basic_string@DU?$char_traits@D@std@@V?$allocator@D@2@@std@@QAE@ABV01@@Z 1008ad30 f i sound.obj
 0002:00018de0       ??1?$basic_string@DU?$char_traits@D@std@@V?$allocator@D@2@@std@@QAE@XZ 1008ade0 f i sound.obj
 0002:00018e70       ?c_str@?$basic_string@DU?$char_traits@D@std@@V?$allocator@D@2@@std@@QBEPBDXZ 1008ae70 f i sound.obj
 0002:00018ea0       ??1?$_String_val@DV?$allocator@D@std@@@std@@QAE@XZ 1008aea0 f i sound.obj
 0002:00018ed0       ??1_String_base@std@@QAE@XZ 1008aed0 f i sound.obj
 0002:00018f00       ??1_Container_base_secure@std@@QAE@XZ 1008af00 f i sound.obj
 0002:00018f30       ?_Orphan_all@_Container_base_secure@std@@QBEXXZ 1008af30 f i sound.obj
 0002:00019000       ?assign@?$basic_string@DU?$char_traits@D@std@@V?$allocator@D@2@@std@@QAEAAV12@ABV12@II@Z 1008b000 f i sound.obj
 0002:00019110       ?size@?$basic_string@DU?$char_traits@D@std@@V?$allocator@D@2@@std@@QBEIXZ 1008b110 f i sound.obj
 0002:00019130       ?_Tidy@?$basic_string@DU?$char_traits@D@std@@V?$allocator@D@2@@std@@IAEX_NI@Z 1008b130 f i sound.obj
 0002:000191f0       ?_Myptr@?$basic_string@DU?$char_traits@D@std@@V?$allocator@D@2@@std@@IBEPBDXZ 1008b1f0 f i sound.obj
 0002:00019240       ??0?$_String_val@DV?$allocator@D@std@@@std@@QAE@ABV01@@Z 1008b240 f i sound.obj
 0002:000192a0       ??0_String_base@std@@QAE@XZ 1008b2a0 f i sound.obj
 0002:000192d0       ??0_Container_base_secure@std@@QAE@XZ 1008b2d0 f i sound.obj
 0002:00019300       ?erase@?$basic_string@DU?$char_traits@D@std@@V?$allocator@D@2@@std@@QAEAAV12@II@Z 1008b300 f i sound.obj
 0002:000193e0       ?_Eos@?$basic_string@DU?$char_traits@D@std@@V?$allocator@D@2@@std@@IAEXI@Z 1008b3e0 f i sound.obj
 0002:00019440       ?assign@?$char_traits@D@std@@SAXAADABD@Z 1008b440 f i sound.obj
 0002:00019460       ?_Grow@?$basic_string@DU?$char_traits@D@std@@V?$allocator@D@2@@std@@IAE_NI_N@Z 1008b460 f i sound.obj
 0002:00019540       ?_Myptr@?$basic_string@DU?$char_traits@D@std@@V?$allocator@D@2@@std@@IAEPADXZ 1008b540 f i sound.obj
 0002:00019590       ??0?$allocator@D@std@@QAE@ABV01@@Z 1008b590 f i sound.obj
 0002:000195b0       ?deallocate@?$allocator@D@std@@QAEXPADI@Z 1008b5b0 f i sound.obj
 0002:000195f0       ?_Lbound@?$_Tree@V?$_Tmap_traits@HUsound@@U?$less@H@std@@V?$allocator@U?$pair@$$CBHUsound@@@std@@@3@$0A@@std@@@std@@IBEPAU_Node@?$_Tree_nod@V?$_Tmap_traits@HUsound@@U?$less@H@std@@V?$allocator@U?$pair@$$CBHUsound@@@std@@@3@$0A@@std@@@2@ABH@Z 1008b5f0 f i sound.obj
 0002:000196e0       ?_Kfn@?$_Tmap_traits@HUsound@@U?$less@H@std@@V?$allocator@U?$pair@$$CBHUsound@@@std@@@3@$0A@@std@@SAABHABU?$pair@$$CBHUsound@@@2@@Z 1008b6e0 f i sound.obj
 0002:000196f0       ??0const_iterator@?$_Tree@V?$_Tmap_traits@HUsound@@U?$less@H@std@@V?$allocator@U?$pair@$$CBHUsound@@@std@@@3@$0A@@std@@@std@@QAE@XZ 1008b6f0 f i sound.obj
 0002:00019730       ??0const_iterator@?$_Tree@V?$_Tmap_traits@HUsound@@U?$less@H@std@@V?$allocator@U?$pair@$$CBHUsound@@@std@@@3@$0A@@std@@@std@@QAE@PAU_Node@?$_Tree_nod@V?$_Tmap_traits@HUsound@@U?$less@H@std@@V?$allocator@U?$pair@$$CBHUsound@@@std@@@3@$0A@@std@@@2@PBV12@@Z 1008b730 f i sound.obj
 0002:000197d0       ??Dconst_iterator@?$_Tree@V?$_Tmap_traits@HUsound@@U?$less@H@std@@V?$allocator@U?$pair@$$CBHUsound@@@std@@@3@$0A@@std@@@std@@QBEABU?$pair@$$CBHUsound@@@2@XZ 1008b7d0 f i sound.obj
 0002:000198a0       ??Econst_iterator@?$_Tree@V?$_Tmap_traits@HUsound@@U?$less@H@std@@V?$allocator@U?$pair@$$CBHUsound@@@std@@@3@$0A@@std@@@std@@QAE?AV012@H@Z 1008b8a0 f i sound.obj
 0002:000199a0       ??Fconst_iterator@?$_Tree@V?$_Tmap_traits@HUsound@@U?$less@H@std@@V?$allocator@U?$pair@$$CBHUsound@@@std@@@3@$0A@@std@@@std@@QAEAAV012@XZ 1008b9a0 f i sound.obj
 0002:000199d0       ?_Inc@const_iterator@?$_Tree@V?$_Tmap_traits@HUsound@@U?$less@H@std@@V?$allocator@U?$pair@$$CBHUsound@@@std@@@3@$0A@@std@@@std@@QAEXXZ 1008b9d0 f i sound.obj
 0002:00019b60       ??0length_error@std@@QAE@ABV01@@Z 1008bb60 f i sound.obj
 0002:00019bb0       ??0logic_error@std@@QAE@ABV01@@Z 1008bbb0 f i sound.obj
 0002:00019c50       ??0?$_Bidit@U?$pair@$$CBHUsound@@@std@@HPBU12@ABU12@@std@@QAE@XZ 1008bc50 f i sound.obj
 0002:00019c80       ??0?$_Iterator_with_base@Ubidirectional_iterator_tag@std@@U?$pair@$$CBHUsound@@@2@HPBU32@ABU32@V_Iterator_base@2@@std@@QAE@XZ 1008bc80 f i sound.obj
 0002:00019cb0       ??0?$basic_string@DU?$char_traits@D@std@@V?$allocator@D@2@@std@@QAE@PBD@Z 1008bcb0 f i sound.obj
 0002:00019d60       ?max_size@?$basic_string@DU?$char_traits@D@std@@V?$allocator@D@2@@std@@QBEIXZ 1008bd60 f i sound.obj
 0002:00019dd0       ?_Copy@?$basic_string@DU?$char_traits@D@std@@V?$allocator@D@2@@std@@IAEXII@Z 1008bdd0 f i sound.obj
 0002:00019fe0       ?max_size@?$_Tree@V?$_Tmap_traits@HUsound@@U?$less@H@std@@V?$allocator@U?$pair@$$CBHUsound@@@std@@@3@$0A@@std@@@std@@QBEIXZ 1008bfe0 f i sound.obj
 0002:0001a010       ?_Buynode@?$_Tree@V?$_Tmap_traits@HUsound@@U?$less@H@std@@V?$allocator@U?$pair@$$CBHUsound@@@std@@@3@$0A@@std@@@std@@IAEPAU_Node@?$_Tree_nod@V?$_Tmap_traits@HUsound@@U?$less@H@std@@V?$allocator@U?$pair@$$CBHUsound@@@std@@@3@$0A@@std@@@2@PAU342@00ABU?$pair@$$CBHUsound@@@2@D@Z 1008c010 f i sound.obj
 0002:0001a160       ??2@YAPAXIPAX@Z            1008c160 f i sound.obj
 0002:0001a170       ??3@YAXPAX0@Z              1008c170 f i sound.obj
 0002:0001a180       ??Fiterator@?$_Tree@V?$_Tmap_traits@HUsound@@U?$less@H@std@@V?$allocator@U?$pair@$$CBHUsound@@@std@@@3@$0A@@std@@@std@@QAEAAV012@XZ 1008c180 f i sound.obj
 0002:0001a1b0       ?_Dec@const_iterator@?$_Tree@V?$_Tmap_traits@HUsound@@U?$less@H@std@@V?$allocator@U?$pair@$$CBHUsound@@@std@@@3@$0A@@std@@@std@@QAEXXZ 1008c1b0 f i sound.obj
 0002:0001a480       ??0?$pair@Viterator@?$_Tree@V?$_Tmap_traits@HUsound@@U?$less@H@std@@V?$allocator@U?$pair@$$CBHUsound@@@std@@@3@$0A@@std@@@std@@V123@@std@@QAE@ABViterator@?$_Tree@V?$_Tmap_traits@HUsound@@U?$less@H@std@@V?$allocator@U?$pair@$$CBHUsound@@@std@@@3@$0A@@std@@@1@0@Z 1008c480 f i sound.obj
 0002:0001a520       ??0?$pair@Viterator@?$_Tree@V?$_Tmap_traits@HUsound@@U?$less@H@std@@V?$allocator@U?$pair@$$CBHUsound@@@std@@@3@$0A@@std@@@std@@_N@std@@QAE@ABViterator@?$_Tree@V?$_Tmap_traits@HUsound@@U?$less@H@std@@V?$allocator@U?$pair@$$CBHUsound@@@std@@@3@$0A@@std@@@1@AB_N@Z 1008c520 f i sound.obj
 0002:0001a570       ?assign@?$basic_string@DU?$char_traits@D@std@@V?$allocator@D@2@@std@@QAEAAV12@PBD@Z 1008c570 f i sound.obj
 0002:0001a5d0       ?length@?$char_traits@D@std@@SAIPBD@Z 1008c5d0 f i sound.obj
 0002:0001a5f0       ??0?$_String_val@DV?$allocator@D@std@@@std@@IAE@V?$allocator@D@1@@Z 1008c5f0 f i sound.obj
 0002:0001a640       ??0?$allocator@D@std@@QAE@XZ 1008c640 f i sound.obj
 0002:0001a660       ?allocate@?$allocator@D@std@@QAEPADI@Z 1008c660 f i sound.obj
 0002:0001a6a0       ?max_size@?$allocator@D@std@@QBEIXZ 1008c6a0 f i sound.obj
 0002:0001a700       ?max_size@?$allocator@U?$pair@$$CBHUsound@@@std@@@std@@QBEIXZ 1008c700 f i sound.obj
 0002:0001a760       ?allocate@?$allocator@U_Node@?$_Tree_nod@V?$_Tmap_traits@HUsound@@U?$less@H@std@@V?$allocator@U?$pair@$$CBHUsound@@@std@@@3@$0A@@std@@@std@@@std@@QAEPAU_Node@?$_Tree_nod@V?$_Tmap_traits@HUsound@@U?$less@H@std@@V?$allocator@U?$pair@$$CBHUsound@@@std@@@3@$0A@@std@@@2@I@Z 1008c760 f i sound.obj
 0002:0001a7a0       ??0_Node@?$_Tree_nod@V?$_Tmap_traits@HUsound@@U?$less@H@std@@V?$allocator@U?$pair@$$CBHUsound@@@std@@@3@$0A@@std@@@std@@QAE@PAU012@00ABU?$pair@$$CBHUsound@@@2@D@Z 1008c7a0 f i sound.obj
 0002:0001a820       ?assign@?$basic_string@DU?$char_traits@D@std@@V?$allocator@D@2@@std@@QAEAAV12@PBDI@Z 1008c820 f i sound.obj
 0002:0001a900       ?_Inside@?$basic_string@DU?$char_traits@D@std@@V?$allocator@D@2@@std@@IAE_NPBD@Z 1008c900 f i sound.obj
 0002:0001a960       ??$_Debug_pointer@D@std@@YAXPBDPB_WI@Z 1008c960 f i sound.obj
 0002:0001a990       ??$swap@D@std@@YAXAAD0@Z   1008c990 f i sound.obj
 0002:0001a9d0       ??$_Distance@Viterator@?$_Tree@V?$_Tmap_traits@HUsound@@U?$less@H@std@@V?$allocator@U?$pair@$$CBHUsound@@@std@@@3@$0A@@std@@@std@@I@std@@YAXViterator@?$_Tree@V?$_Tmap_traits@HUsound@@U?$less@H@std@@V?$allocator@U?$pair@$$CBHUsound@@@std@@@3@$0A@@std@@@0@0AAI@Z 1008c9d0 f i sound.obj
 0002:0001aad0       ??$copy_s@U?$char_traits@D@std@@@_Traits_helper@std@@YAPADPADIPBDI@Z 1008cad0 f i sound.obj
 0002:0001ab20       ??$_Destroy@U_Node@?$_Tree_nod@V?$_Tmap_traits@HUsound@@U?$less@H@std@@V?$allocator@U?$pair@$$CBHUsound@@@std@@@3@$0A@@std@@@std@@@std@@YAXPAU_Node@?$_Tree_nod@V?$_Tmap_traits@HUsound@@U?$less@H@std@@V?$allocator@U?$pair@$$CBHUsound@@@std@@@3@$0A@@std@@@0@@Z 1008cb20 f i sound.obj
 0002:0001ab30       ??$move_s@U?$char_traits@D@std@@@_Traits_helper@std@@YAPADPADIPBDI@Z 1008cb30 f i sound.obj
 0002:0001ab80       ??$_Allocate@D@std@@YAPADIPAD@Z 1008cb80 f i sound.obj
 0002:0001ac10       ??0bad_alloc@std@@QAE@PBD@Z 1008cc10 f i sound.obj
 0002:0001ac60       ??1bad_alloc@std@@UAE@XZ   1008cc60 f i sound.obj
 0002:0001aca0       ??_Ebad_alloc@std@@UAEPAXI@Z 1008cca0 f i sound.obj
 0002:0001aca0       ??_Gbad_alloc@std@@UAEPAXI@Z 1008cca0 f i sound.obj
 0002:0001acf0       ??$_Allocate@U_Node@?$_Tree_nod@V?$_Tmap_traits@HUsound@@U?$less@H@std@@V?$allocator@U?$pair@$$CBHUsound@@@std@@@3@$0A@@std@@@std@@@std@@YAPAU_Node@?$_Tree_nod@V?$_Tmap_traits@HUsound@@U?$less@H@std@@V?$allocator@U?$pair@$$CBHUsound@@@std@@@3@$0A@@std@@@0@IPAU120@@Z 1008ccf0 f i sound.obj
 0002:0001ad80       ??0bad_alloc@std@@QAE@ABV01@@Z 1008cd80 f i sound.obj
 0002:0001add0       ??$_Iter_cat@Viterator@?$_Tree@V?$_Tmap_traits@HUsound@@U?$less@H@std@@V?$allocator@U?$pair@$$CBHUsound@@@std@@@3@$0A@@std@@@std@@@std@@YA?AUbidirectional_iterator_tag@0@ABViterator@?$_Tree@V?$_Tmap_traits@HUsound@@U?$less@H@std@@V?$allocator@U?$pair@$$CBHUsound@@@std@@@3@$0A@@std@@@0@@Z 1008cdd0 f i sound.obj
 0002:0001ae30       ??$_Distance2@Viterator@?$_Tree@V?$_Tmap_traits@HUsound@@U?$less@H@std@@V?$allocator@U?$pair@$$CBHUsound@@@std@@@3@$0A@@std@@@std@@I@std@@YAXViterator@?$_Tree@V?$_Tmap_traits@HUsound@@U?$less@H@std@@V?$allocator@U?$pair@$$CBHUsound@@@std@@@3@$0A@@std@@@0@0AAIUbidirectional_iterator_tag@0@@Z 1008ce30 f i sound.obj
 0002:0001aee0       ??$_Char_traits_cat@U?$char_traits@D@std@@@std@@YA?AU_Secure_char_traits_tag@0@XZ 1008cee0 f i sound.obj
 0002:0001af50       ??$copy_s@U?$char_traits@D@std@@@_Traits_helper@std@@YAPADPADIPBDIU_Secure_char_traits_tag@1@@Z 1008cf50 f i sound.obj
 0002:0001af80       ?_Copy_s@?$char_traits@D@std@@SAPADPADIPBDI@Z 1008cf80 f i sound.obj
 0002:0001afb0       ??$move_s@U?$char_traits@D@std@@@_Traits_helper@std@@YAPADPADIPBDIU_Secure_char_traits_tag@1@@Z 1008cfb0 f i sound.obj
 0002:0001afe0       ?_Move_s@?$char_traits@D@std@@SAPADPADIPBDI@Z 1008cfe0 f i sound.obj
 0002:0001b010       ??0?$map@HUsound@@U?$less@H@std@@V?$allocator@U?$pair@$$CBHUsound@@@std@@@3@@std@@QAE@XZ 1008d010 f i sound.obj
 0002:0001b060       ??0?$_Tree@V?$_Tmap_traits@HUsound@@U?$less@H@std@@V?$allocator@U?$pair@$$CBHUsound@@@std@@@3@$0A@@std@@@std@@QAE@ABU?$less@H@1@ABV?$allocator@U?$pair@$$CBHUsound@@@std@@@1@@Z 1008d060 f i sound.obj
 0002:0001b110       ??1?$_Tree_val@V?$_Tmap_traits@HUsound@@U?$less@H@std@@V?$allocator@U?$pair@$$CBHUsound@@@std@@@3@$0A@@std@@@std@@QAE@XZ 1008d110 f i sound.obj
 0002:0001b140       ??1?$_Tree_ptr@V?$_Tmap_traits@HUsound@@U?$less@H@std@@V?$allocator@U?$pair@$$CBHUsound@@@std@@@3@$0A@@std@@@std@@QAE@XZ 1008d140 f i sound.obj
 0002:0001b170       ??1?$_Tree_nod@V?$_Tmap_traits@HUsound@@U?$less@H@std@@V?$allocator@U?$pair@$$CBHUsound@@@std@@@3@$0A@@std@@@std@@QAE@XZ 1008d170 f i sound.obj
 0002:0001b1a0       ??1?$_Tmap_traits@HUsound@@U?$less@H@std@@V?$allocator@U?$pair@$$CBHUsound@@@std@@@3@$0A@@std@@QAE@XZ 1008d1a0 f i sound.obj
 0002:0001b1d0       ??1?$_Container_base_aux_alloc_empty@V?$allocator@U?$pair@$$CBHUsound@@@std@@@std@@@std@@IAE@XZ 1008d1d0 f i sound.obj
 0002:0001b200       ??0?$allocator@U?$pair@$$CBHUsound@@@std@@@std@@QAE@XZ 1008d200 f i sound.obj
 0002:0001b220       ?_Init@?$_Tree@V?$_Tmap_traits@HUsound@@U?$less@H@std@@V?$allocator@U?$pair@$$CBHUsound@@@std@@@3@$0A@@std@@@std@@IAEXXZ 1008d220 f i sound.obj
 0002:0001b2c0       ??0?$_Tree_val@V?$_Tmap_traits@HUsound@@U?$less@H@std@@V?$allocator@U?$pair@$$CBHUsound@@@std@@@3@$0A@@std@@@std@@IAE@ABU?$less@H@1@V?$allocator@U?$pair@$$CBHUsound@@@std@@@1@@Z 1008d2c0 f i sound.obj
 0002:0001b330       ??0?$allocator@U?$pair@$$CBHUsound@@@std@@@std@@QAE@ABV01@@Z 1008d330 f i sound.obj
 0002:0001b350       ?_Buynode@?$_Tree@V?$_Tmap_traits@HUsound@@U?$less@H@std@@V?$allocator@U?$pair@$$CBHUsound@@@std@@@3@$0A@@std@@@std@@IAEPAU_Node@?$_Tree_nod@V?$_Tmap_traits@HUsound@@U?$less@H@std@@V?$allocator@U?$pair@$$CBHUsound@@@std@@@3@$0A@@std@@@2@XZ 1008d350 f i sound.obj
 0002:0001b560       ?destroy@?$allocator@PAU_Node@?$_Tree_nod@V?$_Tmap_traits@HUsound@@U?$less@H@std@@V?$allocator@U?$pair@$$CBHUsound@@@std@@@3@$0A@@std@@@std@@@std@@QAEXPAPAU_Node@?$_Tree_nod@V?$_Tmap_traits@HUsound@@U?$less@H@std@@V?$allocator@U?$pair@$$CBHUsound@@@std@@@3@$0A@@std@@@2@@Z 1008d560 f i sound.obj
 0002:0001b5a0       ??0?$_Tree_ptr@V?$_Tmap_traits@HUsound@@U?$less@H@std@@V?$allocator@U?$pair@$$CBHUsound@@@std@@@3@$0A@@std@@@std@@QAE@ABU?$less@H@1@V?$allocator@U?$pair@$$CBHUsound@@@std@@@1@@Z 1008d5a0 f i sound.obj
 0002:0001b610       ??0?$_Tree_nod@V?$_Tmap_traits@HUsound@@U?$less@H@std@@V?$allocator@U?$pair@$$CBHUsound@@@std@@@3@$0A@@std@@@std@@IAE@ABU?$less@H@1@V?$allocator@U?$pair@$$CBHUsound@@@std@@@1@@Z 1008d610 f i sound.obj
 0002:0001b680       ?construct@?$allocator@PAU_Node@?$_Tree_nod@V?$_Tmap_traits@HUsound@@U?$less@H@std@@V?$allocator@U?$pair@$$CBHUsound@@@std@@@3@$0A@@std@@@std@@@std@@QAEXPAPAU_Node@?$_Tree_nod@V?$_Tmap_traits@HUsound@@U?$less@H@std@@V?$allocator@U?$pair@$$CBHUsound@@@std@@@3@$0A@@std@@@2@ABQAU342@@Z 1008d680 f i sound.obj
 0002:0001b6c0       ??0?$_Tmap_traits@HUsound@@U?$less@H@std@@V?$allocator@U?$pair@$$CBHUsound@@@std@@@3@$0A@@std@@QAE@U?$less@H@1@V?$allocator@U?$pair@$$CBHUsound@@@std@@@1@@Z 1008d6c0 f i sound.obj
 0002:0001b720       ??0?$_Container_base_aux_alloc_empty@V?$allocator@U?$pair@$$CBHUsound@@@std@@@std@@@std@@IAE@V?$allocator@U?$pair@$$CBHUsound@@@std@@@1@@Z 1008d720 f i sound.obj
 0002:0001b760       ??$_Destroy@PAU_Node@?$_Tree_nod@V?$_Tmap_traits@HUsound@@U?$less@H@std@@V?$allocator@U?$pair@$$CBHUsound@@@std@@@3@$0A@@std@@@std@@@std@@YAXPAPAU_Node@?$_Tree_nod@V?$_Tmap_traits@HUsound@@U?$less@H@std@@V?$allocator@U?$pair@$$CBHUsound@@@std@@@3@$0A@@std@@@0@@Z 1008d760 f i sound.obj
 0002:0001b770       ??$?0U?$pair@$$CBHUsound@@@std@@@?$allocator@PAU_Node@?$_Tree_nod@V?$_Tmap_traits@HUsound@@U?$less@H@std@@V?$allocator@U?$pair@$$CBHUsound@@@std@@@3@$0A@@std@@@std@@@std@@QAE@ABV?$allocator@U?$pair@$$CBHUsound@@@std@@@1@@Z 1008d770 f i sound.obj
 0002:0001b790       ??$?0U?$pair@$$CBHUsound@@@std@@@?$allocator@U_Node@?$_Tree_nod@V?$_Tmap_traits@HUsound@@U?$less@H@std@@V?$allocator@U?$pair@$$CBHUsound@@@std@@@3@$0A@@std@@@std@@@std@@QAE@ABV?$allocator@U?$pair@$$CBHUsound@@@std@@@1@@Z 1008d790 f i sound.obj
 0002:0001b7b0       ??$_Construct@PAU_Node@?$_Tree_nod@V?$_Tmap_traits@HUsound@@U?$less@H@std@@V?$allocator@U?$pair@$$CBHUsound@@@std@@@3@$0A@@std@@@std@@PAU123@@std@@YAXPAPAU_Node@?$_Tree_nod@V?$_Tmap_traits@HUsound@@U?$less@H@std@@V?$allocator@U?$pair@$$CBHUsound@@@std@@@3@$0A@@std@@@0@ABQAU120@@Z 1008d7b0 f i sound.obj
 0002:0001b830       ??1?$map@HUsound@@U?$less@H@std@@V?$allocator@U?$pair@$$CBHUsound@@@std@@@3@@std@@QAE@XZ 1008d830 f i sound.obj
 0002:0001b860       ??1?$_Tree@V?$_Tmap_traits@HUsound@@U?$less@H@std@@V?$allocator@U?$pair@$$CBHUsound@@@std@@@3@$0A@@std@@@std@@QAE@XZ 1008d860 f i sound.obj
 0002:0001b8e0       ?_Tidy@?$_Tree@V?$_Tmap_traits@HUsound@@U?$less@H@std@@V?$allocator@U?$pair@$$CBHUsound@@@std@@@3@$0A@@std@@@std@@IAEXXZ 1008d8e0 f i sound.obj
 0002:0001bab0       ?ogg_cfread@@YAIPAXII0@Z   1008dab0 f   ogg.obj
 0002:0001baf0       ?ogg_cfseek@@YAHPAX_JH@Z   1008daf0 f   ogg.obj
 0002:0001bb30       ?ogg_cfclose@@YAHPAX@Z     1008db30 f   ogg.obj
 0002:0001bb60       ?ogg_cftell@@YAJPAX@Z      1008db60 f   ogg.obj
 0002:0001bb90       ?ogg_mmio_read@@YAIPAXII0@Z 1008db90 f   ogg.obj
 0002:0001bbe0       ?ogg_mmio_seek@@YAHPAX_JH@Z 1008dbe0 f   ogg.obj
 0002:0001bc20       ?ogg_mmio_close@@YAHPAX@Z  1008dc20 f   ogg.obj
 0002:0001bc60       ?ogg_mmio_tell@@YAJPAX@Z   1008dc60 f   ogg.obj
 0002:0001bca0       ?OGG_init@@YAHXZ           1008dca0 f   ogg.obj
 0002:0001bd60       ?ambi_init@@YAXXZ          1008dd60 f   ambientsnd.obj
 0002:0001bd70       ?ambi_close@@YAXXZ         1008dd70 f   ambientsnd.obj
 0002:0001bd80       ?ambi_start@@YAHHHHMHH@Z   1008dd80 f   ambientsnd.obj
 0002:0001bfa0       ?ambi_stop@@YAXHH@Z        1008dfa0 f   ambientsnd.obj
 0002:0001c180       ?ambi_stop_all@@YAXH@Z     1008e180 f   ambientsnd.obj
 0002:0001c1a0       ?ambi_pause@@YAXH@Z        1008e1a0 f   ambientsnd.obj
 0002:0001c1e0       ?ambi_pause_all@@YAXXZ     1008e1e0 f   ambientsnd.obj
 0002:0001c200       ?ambi_unpause@@YAXH@Z      1008e200 f   ambientsnd.obj
 0002:0001c240       ?ambi_unpause_all@@YAXXZ   1008e240 f   ambientsnd.obj
 0002:0001c260       ?ambi_set_volume@@YAXHM@Z  1008e260 f   ambientsnd.obj
 0002:0001c3b0       ?ambi_set_volume_all@@YAXM@Z 1008e3b0 f   ambientsnd.obj
 0002:0001c3d0       ?ambi_set_loop@@YAXHH@Z    1008e3d0 f   ambientsnd.obj
 0002:0001c410       ?ambi_state@@YAHH@Z        1008e410 f   ambientsnd.obj
 0002:0001c640       ??1iterator@?$_Tree@V?$_Tmap_traits@HUAmbientSnd@@U?$less@H@std@@V?$allocator@U?$pair@$$CBHUAmbientSnd@@@std@@@3@$0A@@std@@@std@@QAE@XZ 1008e640 f i ambientsnd.obj
 0002:0001c670       ??1const_iterator@?$_Tree@V?$_Tmap_traits@HUAmbientSnd@@U?$less@H@std@@V?$allocator@U?$pair@$$CBHUAmbientSnd@@@std@@@3@$0A@@std@@@std@@QAE@XZ 1008e670 f i ambientsnd.obj
 0002:0001c6a0       ??1?$_Bidit@U?$pair@$$CBHUAmbientSnd@@@std@@HPBU12@ABU12@@std@@QAE@XZ 1008e6a0 f i ambientsnd.obj
 0002:0001c6d0       ??1?$_Iterator_with_base@Ubidirectional_iterator_tag@std@@U?$pair@$$CBHUAmbientSnd@@@2@HPBU32@ABU32@V_Iterator_base@2@@std@@QAE@XZ 1008e6d0 f i ambientsnd.obj
 0002:0001c700       ??1iterator@?$_Tree@V?$_Tmap_traits@HHU?$less@H@std@@V?$allocator@U?$pair@$$CBHH@std@@@2@$0A@@std@@@std@@QAE@XZ 1008e700 f i ambientsnd.obj
 0002:0001c730       ??1const_iterator@?$_Tree@V?$_Tmap_traits@HHU?$less@H@std@@V?$allocator@U?$pair@$$CBHH@std@@@2@$0A@@std@@@std@@QAE@XZ 1008e730 f i ambientsnd.obj
 0002:0001c760       ??1?$_Bidit@U?$pair@$$CBHH@std@@HPBU12@ABU12@@std@@QAE@XZ 1008e760 f i ambientsnd.obj
 0002:0001c790       ??1?$_Iterator_with_base@Ubidirectional_iterator_tag@std@@U?$pair@$$CBHH@2@HPBU32@ABU32@V_Iterator_base@2@@std@@QAE@XZ 1008e790 f i ambientsnd.obj
 0002:0001c7c0       ??A?$map@HHU?$less@H@std@@V?$allocator@U?$pair@$$CBHH@std@@@2@@std@@QAEAAHABH@Z 1008e7c0 f i ambientsnd.obj
 0002:0001c9e0       ?end@?$_Tree@V?$_Tmap_traits@HHU?$less@H@std@@V?$allocator@U?$pair@$$CBHH@std@@@2@$0A@@std@@@std@@QAE?AViterator@12@XZ 1008e9e0 f i ambientsnd.obj
 0002:0001ca40       ?find@?$_Tree@V?$_Tmap_traits@HHU?$less@H@std@@V?$allocator@U?$pair@$$CBHH@std@@@2@$0A@@std@@@std@@QAE?AViterator@12@ABH@Z 1008ea40 f i ambientsnd.obj
 0002:0001cc50       ??A?$map@HUAmbientSnd@@U?$less@H@std@@V?$allocator@U?$pair@$$CBHUAmbientSnd@@@std@@@3@@std@@QAEAAUAmbientSnd@@ABH@Z 1008ec50 f i ambientsnd.obj
 0002:0001cef0       ?end@?$_Tree@V?$_Tmap_traits@HUAmbientSnd@@U?$less@H@std@@V?$allocator@U?$pair@$$CBHUAmbientSnd@@@std@@@3@$0A@@std@@@std@@QAE?AViterator@12@XZ 1008eef0 f i ambientsnd.obj
 0002:0001cf50       ?find@?$_Tree@V?$_Tmap_traits@HUAmbientSnd@@U?$less@H@std@@V?$allocator@U?$pair@$$CBHUAmbientSnd@@@std@@@3@$0A@@std@@@std@@QAE?AViterator@12@ABH@Z 1008ef50 f i ambientsnd.obj
 0002:0001d160       ??Citerator@?$_Tree@V?$_Tmap_traits@HHU?$less@H@std@@V?$allocator@U?$pair@$$CBHH@std@@@2@$0A@@std@@@std@@QBEPAU?$pair@$$CBHH@2@XZ 1008f160 f i ambientsnd.obj
 0002:0001d190       ??8const_iterator@?$_Tree@V?$_Tmap_traits@HHU?$less@H@std@@V?$allocator@U?$pair@$$CBHH@std@@@2@$0A@@std@@@std@@QBE_NABV012@@Z 1008f190 f i ambientsnd.obj
 0002:0001d260       ??Citerator@?$_Tree@V?$_Tmap_traits@HUAmbientSnd@@U?$less@H@std@@V?$allocator@U?$pair@$$CBHUAmbientSnd@@@std@@@3@$0A@@std@@@std@@QBEPAU?$pair@$$CBHUAmbientSnd@@@2@XZ 1008f260 f i ambientsnd.obj
 0002:0001d290       ??8const_iterator@?$_Tree@V?$_Tmap_traits@HUAmbientSnd@@U?$less@H@std@@V?$allocator@U?$pair@$$CBHUAmbientSnd@@@std@@@3@$0A@@std@@@std@@QBE_NABV012@@Z 1008f290 f i ambientsnd.obj
 0002:0001d360       ??0const_iterator@?$_Tree@V?$_Tmap_traits@HHU?$less@H@std@@V?$allocator@U?$pair@$$CBHH@std@@@2@$0A@@std@@@std@@QAE@ABV012@@Z 1008f360 f i ambientsnd.obj
 0002:0001d3b0       ??4iterator@?$_Tree@V?$_Tmap_traits@HHU?$less@H@std@@V?$allocator@U?$pair@$$CBHH@std@@@2@$0A@@std@@@std@@QAEAAV012@ABV012@@Z 1008f3b0 f i ambientsnd.obj
 0002:0001d3f0       ??0iterator@?$_Tree@V?$_Tmap_traits@HHU?$less@H@std@@V?$allocator@U?$pair@$$CBHH@std@@@2@$0A@@std@@@std@@QAE@ABV012@@Z 1008f3f0 f i ambientsnd.obj
 0002:0001d430       ??0const_iterator@?$_Tree@V?$_Tmap_traits@HUAmbientSnd@@U?$less@H@std@@V?$allocator@U?$pair@$$CBHUAmbientSnd@@@std@@@3@$0A@@std@@@std@@QAE@ABV012@@Z 1008f430 f i ambientsnd.obj
 0002:0001d480       ??4iterator@?$_Tree@V?$_Tmap_traits@HUAmbientSnd@@U?$less@H@std@@V?$allocator@U?$pair@$$CBHUAmbientSnd@@@std@@@3@$0A@@std@@@std@@QAEAAV012@ABV012@@Z 1008f480 f i ambientsnd.obj
 0002:0001d4c0       ??0iterator@?$_Tree@V?$_Tmap_traits@HUAmbientSnd@@U?$less@H@std@@V?$allocator@U?$pair@$$CBHUAmbientSnd@@@std@@@3@$0A@@std@@@std@@QAE@ABV012@@Z 1008f4c0 f i ambientsnd.obj
 0002:0001d500       ??0?$_Bidit@U?$pair@$$CBHH@std@@HPBU12@ABU12@@std@@QAE@ABU01@@Z 1008f500 f i ambientsnd.obj
 0002:0001d540       ??4const_iterator@?$_Tree@V?$_Tmap_traits@HHU?$less@H@std@@V?$allocator@U?$pair@$$CBHH@std@@@2@$0A@@std@@@std@@QAEAAV012@ABV012@@Z 1008f540 f i ambientsnd.obj
 0002:0001d590       ??0?$_Bidit@U?$pair@$$CBHUAmbientSnd@@@std@@HPBU12@ABU12@@std@@QAE@ABU01@@Z 1008f590 f i ambientsnd.obj
 0002:0001d5d0       ??4const_iterator@?$_Tree@V?$_Tmap_traits@HUAmbientSnd@@U?$less@H@std@@V?$allocator@U?$pair@$$CBHUAmbientSnd@@@std@@@3@$0A@@std@@@std@@QAEAAV012@ABV012@@Z 1008f5d0 f i ambientsnd.obj
 0002:0001d620       ??0?$_Iterator_with_base@Ubidirectional_iterator_tag@std@@U?$pair@$$CBHH@2@HPBU32@ABU32@V_Iterator_base@2@@std@@QAE@ABU01@@Z 1008f620 f i ambientsnd.obj
 0002:0001d660       ??4?$_Bidit@U?$pair@$$CBHH@std@@HPBU12@ABU12@@std@@QAEAAU01@ABU01@@Z 1008f660 f i ambientsnd.obj
 0002:0001d6a0       ??0?$_Iterator_with_base@Ubidirectional_iterator_tag@std@@U?$pair@$$CBHUAmbientSnd@@@2@HPBU32@ABU32@V_Iterator_base@2@@std@@QAE@ABU01@@Z 1008f6a0 f i ambientsnd.obj
 0002:0001d6e0       ??4?$_Bidit@U?$pair@$$CBHUAmbientSnd@@@std@@HPBU12@ABU12@@std@@QAEAAU01@ABU01@@Z 1008f6e0 f i ambientsnd.obj
 0002:0001d720       ??4?$_Iterator_with_base@Ubidirectional_iterator_tag@std@@U?$pair@$$CBHH@2@HPBU32@ABU32@V_Iterator_base@2@@std@@QAEAAU01@ABU01@@Z 1008f720 f i ambientsnd.obj
 0002:0001d760       ??4?$_Iterator_with_base@Ubidirectional_iterator_tag@std@@U?$pair@$$CBHUAmbientSnd@@@2@HPBU32@ABU32@V_Iterator_base@2@@std@@QAEAAU01@ABU01@@Z 1008f760 f i ambientsnd.obj
 0002:0001d7a0       ?_Key@?$_Tree@V?$_Tmap_traits@HHU?$less@H@std@@V?$allocator@U?$pair@$$CBHH@std@@@2@$0A@@std@@@std@@KAABHPAU_Node@?$_Tree_nod@V?$_Tmap_traits@HHU?$less@H@std@@V?$allocator@U?$pair@$$CBHH@std@@@2@$0A@@std@@@2@@Z 1008f7a0 f i ambientsnd.obj
 0002:0001d7d0       ?insert@?$_Tree@V?$_Tmap_traits@HHU?$less@H@std@@V?$allocator@U?$pair@$$CBHH@std@@@2@$0A@@std@@@std@@QAE?AViterator@12@Vconst_iterator@12@ABU?$pair@$$CBHH@2@@Z 1008f7d0 f i ambientsnd.obj
 0002:0001e640       ?lower_bound@?$_Tree@V?$_Tmap_traits@HHU?$less@H@std@@V?$allocator@U?$pair@$$CBHH@std@@@2@$0A@@std@@@std@@QAE?AViterator@12@ABH@Z 10090640 f i ambientsnd.obj
 0002:0001e6b0       ?_Key@?$_Tree@V?$_Tmap_traits@HUAmbientSnd@@U?$less@H@std@@V?$allocator@U?$pair@$$CBHUAmbientSnd@@@std@@@3@$0A@@std@@@std@@KAABHPAU_Node@?$_Tree_nod@V?$_Tmap_traits@HUAmbientSnd@@U?$less@H@std@@V?$allocator@U?$pair@$$CBHUAmbientSnd@@@std@@@3@$0A@@std@@@2@@Z 100906b0 f i ambientsnd.obj
 0002:0001e6e0       ?insert@?$_Tree@V?$_Tmap_traits@HUAmbientSnd@@U?$less@H@std@@V?$allocator@U?$pair@$$CBHUAmbientSnd@@@std@@@3@$0A@@std@@@std@@QAE?AViterator@12@Vconst_iterator@12@ABU?$pair@$$CBHUAmbientSnd@@@2@@Z 100906e0 f i ambientsnd.obj
 0002:0001f550       ?lower_bound@?$_Tree@V?$_Tmap_traits@HUAmbientSnd@@U?$less@H@std@@V?$allocator@U?$pair@$$CBHUAmbientSnd@@@std@@@3@$0A@@std@@@std@@QAE?AViterator@12@ABH@Z 10091550 f i ambientsnd.obj
 0002:0001f5c0       ??0iterator@?$_Tree@V?$_Tmap_traits@HHU?$less@H@std@@V?$allocator@U?$pair@$$CBHH@std@@@2@$0A@@std@@@std@@QAE@PAU_Node@?$_Tree_nod@V?$_Tmap_traits@HHU?$less@H@std@@V?$allocator@U?$pair@$$CBHH@std@@@2@$0A@@std@@@2@PBV12@@Z 100915c0 f i ambientsnd.obj
 0002:0001f600       ??Diterator@?$_Tree@V?$_Tmap_traits@HHU?$less@H@std@@V?$allocator@U?$pair@$$CBHH@std@@@2@$0A@@std@@@std@@QBEAAU?$pair@$$CBHH@2@XZ 10091600 f i ambientsnd.obj
 0002:0001f630       ?_Mynode@const_iterator@?$_Tree@V?$_Tmap_traits@HHU?$less@H@std@@V?$allocator@U?$pair@$$CBHH@std@@@2@$0A@@std@@@std@@QBEPAU_Node@?$_Tree_nod@V?$_Tmap_traits@HHU?$less@H@std@@V?$allocator@U?$pair@$$CBHH@std@@@2@$0A@@std@@@3@XZ 10091630 f i ambientsnd.obj
 0002:0001f650       ??0?$pair@$$CBHH@std@@QAE@ABH0@Z 10091650 f i ambientsnd.obj
 0002:0001f690       ??0iterator@?$_Tree@V?$_Tmap_traits@HUAmbientSnd@@U?$less@H@std@@V?$allocator@U?$pair@$$CBHUAmbientSnd@@@std@@@3@$0A@@std@@@std@@QAE@PAU_Node@?$_Tree_nod@V?$_Tmap_traits@HUAmbientSnd@@U?$less@H@std@@V?$allocator@U?$pair@$$CBHUAmbientSnd@@@std@@@3@$0A@@std@@@2@PBV12@@Z 10091690 f i ambientsnd.obj
 0002:0001f6d0       ??Diterator@?$_Tree@V?$_Tmap_traits@HUAmbientSnd@@U?$less@H@std@@V?$allocator@U?$pair@$$CBHUAmbientSnd@@@std@@@3@$0A@@std@@@std@@QBEAAU?$pair@$$CBHUAmbientSnd@@@2@XZ 100916d0 f i ambientsnd.obj
 0002:0001f700       ?_Mynode@const_iterator@?$_Tree@V?$_Tmap_traits@HUAmbientSnd@@U?$less@H@std@@V?$allocator@U?$pair@$$CBHUAmbientSnd@@@std@@@3@$0A@@std@@@std@@QBEPAU_Node@?$_Tree_nod@V?$_Tmap_traits@HUAmbientSnd@@U?$less@H@std@@V?$allocator@U?$pair@$$CBHUAmbientSnd@@@std@@@3@$0A@@std@@@3@XZ 10091700 f i ambientsnd.obj
 0002:0001f720       ??0?$pair@$$CBHUAmbientSnd@@@std@@QAE@ABHABUAmbientSnd@@@Z 10091720 f i ambientsnd.obj
 0002:0001f770       ??1?$pair@Viterator@?$_Tree@V?$_Tmap_traits@HHU?$less@H@std@@V?$allocator@U?$pair@$$CBHH@std@@@2@$0A@@std@@@std@@_N@std@@QAE@XZ 10091770 f i ambientsnd.obj
 0002:0001f7a0       ??1?$pair@Viterator@?$_Tree@V?$_Tmap_traits@HUAmbientSnd@@U?$less@H@std@@V?$allocator@U?$pair@$$CBHUAmbientSnd@@@std@@@3@$0A@@std@@@std@@_N@std@@QAE@XZ 100917a0 f i ambientsnd.obj
 0002:0001f7d0       ?_Isnil@?$_Tree@V?$_Tmap_traits@HHU?$less@H@std@@V?$allocator@U?$pair@$$CBHH@std@@@2@$0A@@std@@@std@@KAAADPAU_Node@?$_Tree_nod@V?$_Tmap_traits@HHU?$less@H@std@@V?$allocator@U?$pair@$$CBHH@std@@@2@$0A@@std@@@2@@Z 100917d0 f i ambientsnd.obj
 0002:0001f7e0       ?_Right@?$_Tree@V?$_Tmap_traits@HHU?$less@H@std@@V?$allocator@U?$pair@$$CBHH@std@@@2@$0A@@std@@@std@@KAAAPAU_Node@?$_Tree_nod@V?$_Tmap_traits@HHU?$less@H@std@@V?$allocator@U?$pair@$$CBHH@std@@@2@$0A@@std@@@2@PAU342@@Z 100917e0 f i ambientsnd.obj
 0002:0001f7f0       ?_Myval@?$_Tree@V?$_Tmap_traits@HHU?$less@H@std@@V?$allocator@U?$pair@$$CBHH@std@@@2@$0A@@std@@@std@@KAAAU?$pair@$$CBHH@2@PAU_Node@?$_Tree_nod@V?$_Tmap_traits@HHU?$less@H@std@@V?$allocator@U?$pair@$$CBHH@std@@@2@$0A@@std@@@2@@Z 100917f0 f i ambientsnd.obj
 0002:0001f800       ?begin@?$_Tree@V?$_Tmap_traits@HHU?$less@H@std@@V?$allocator@U?$pair@$$CBHH@std@@@2@$0A@@std@@@std@@QAE?AViterator@12@XZ 10091800 f i ambientsnd.obj
 0002:0001f870       ?size@?$_Tree@V?$_Tmap_traits@HHU?$less@H@std@@V?$allocator@U?$pair@$$CBHH@std@@@2@$0A@@std@@@std@@QBEIXZ 10091870 f i ambientsnd.obj
 0002:0001f890       ?insert@?$_Tree@V?$_Tmap_traits@HHU?$less@H@std@@V?$allocator@U?$pair@$$CBHH@std@@@2@$0A@@std@@@std@@QAE?AU?$pair@Viterator@?$_Tree@V?$_Tmap_traits@HHU?$less@H@std@@V?$allocator@U?$pair@$$CBHH@std@@@2@$0A@@std@@@std@@_N@2@ABU?$pair@$$CBHH@2@@Z 10091890 f i ambientsnd.obj
 0002:0001fcd0       ?_Left@?$_Tree@V?$_Tmap_traits@HHU?$less@H@std@@V?$allocator@U?$pair@$$CBHH@std@@@2@$0A@@std@@@std@@KAAAPAU_Node@?$_Tree_nod@V?$_Tmap_traits@HHU?$less@H@std@@V?$allocator@U?$pair@$$CBHH@std@@@2@$0A@@std@@@2@PAU342@@Z 10091cd0 f i ambientsnd.obj
 0002:0001fce0       ?_Insert@?$_Tree@V?$_Tmap_traits@HHU?$less@H@std@@V?$allocator@U?$pair@$$CBHH@std@@@2@$0A@@std@@@std@@IAE?AViterator@12@_NPAU_Node@?$_Tree_nod@V?$_Tmap_traits@HHU?$less@H@std@@V?$allocator@U?$pair@$$CBHH@std@@@2@$0A@@std@@@2@ABU?$pair@$$CBHH@2@@Z 10091ce0 f i ambientsnd.obj
 0002:000202b0       ?_Parent@?$_Tree@V?$_Tmap_traits@HHU?$less@H@std@@V?$allocator@U?$pair@$$CBHH@std@@@2@$0A@@std@@@std@@KAAAPAU_Node@?$_Tree_nod@V?$_Tmap_traits@HHU?$less@H@std@@V?$allocator@U?$pair@$$CBHH@std@@@2@$0A@@std@@@2@PAU342@@Z 100922b0 f i ambientsnd.obj
 0002:000202c0       ?_Lbound@?$_Tree@V?$_Tmap_traits@HHU?$less@H@std@@V?$allocator@U?$pair@$$CBHH@std@@@2@$0A@@std@@@std@@IBEPAU_Node@?$_Tree_nod@V?$_Tmap_traits@HHU?$less@H@std@@V?$allocator@U?$pair@$$CBHH@std@@@2@$0A@@std@@@2@ABH@Z 100922c0 f i ambientsnd.obj
 0002:000203b0       ?_Rmost@?$_Tree@V?$_Tmap_traits@HHU?$less@H@std@@V?$allocator@U?$pair@$$CBHH@std@@@2@$0A@@std@@@std@@IBEAAPAU_Node@?$_Tree_nod@V?$_Tmap_traits@HHU?$less@H@std@@V?$allocator@U?$pair@$$CBHH@std@@@2@$0A@@std@@@2@XZ 100923b0 f i ambientsnd.obj
 0002:000203f0       ?_Kfn@?$_Tmap_traits@HHU?$less@H@std@@V?$allocator@U?$pair@$$CBHH@std@@@2@$0A@@std@@SAABHABU?$pair@$$CBHH@2@@Z 100923f0 f i ambientsnd.obj
 0002:00020400       ?_Isnil@?$_Tree@V?$_Tmap_traits@HUAmbientSnd@@U?$less@H@std@@V?$allocator@U?$pair@$$CBHUAmbientSnd@@@std@@@3@$0A@@std@@@std@@KAAADPAU_Node@?$_Tree_nod@V?$_Tmap_traits@HUAmbientSnd@@U?$less@H@std@@V?$allocator@U?$pair@$$CBHUAmbientSnd@@@std@@@3@$0A@@std@@@2@@Z 10092400 f i ambientsnd.obj
 0002:00020410       ?_Right@?$_Tree@V?$_Tmap_traits@HUAmbientSnd@@U?$less@H@std@@V?$allocator@U?$pair@$$CBHUAmbientSnd@@@std@@@3@$0A@@std@@@std@@KAAAPAU_Node@?$_Tree_nod@V?$_Tmap_traits@HUAmbientSnd@@U?$less@H@std@@V?$allocator@U?$pair@$$CBHUAmbientSnd@@@std@@@3@$0A@@std@@@2@PAU342@@Z 10092410 f i ambientsnd.obj
 0002:00020420       ?_Myval@?$_Tree@V?$_Tmap_traits@HUAmbientSnd@@U?$less@H@std@@V?$allocator@U?$pair@$$CBHUAmbientSnd@@@std@@@3@$0A@@std@@@std@@KAAAU?$pair@$$CBHUAmbientSnd@@@2@PAU_Node@?$_Tree_nod@V?$_Tmap_traits@HUAmbientSnd@@U?$less@H@std@@V?$allocator@U?$pair@$$CBHUAmbientSnd@@@std@@@3@$0A@@std@@@2@@Z 10092420 f i ambientsnd.obj
 0002:00020430       ?begin@?$_Tree@V?$_Tmap_traits@HUAmbientSnd@@U?$less@H@std@@V?$allocator@U?$pair@$$CBHUAmbientSnd@@@std@@@3@$0A@@std@@@std@@QAE?AViterator@12@XZ 10092430 f i ambientsnd.obj
 0002:000204a0       ?size@?$_Tree@V?$_Tmap_traits@HUAmbientSnd@@U?$less@H@std@@V?$allocator@U?$pair@$$CBHUAmbientSnd@@@std@@@3@$0A@@std@@@std@@QBEIXZ 100924a0 f i ambientsnd.obj
 0002:000204c0       ?insert@?$_Tree@V?$_Tmap_traits@HUAmbientSnd@@U?$less@H@std@@V?$allocator@U?$pair@$$CBHUAmbientSnd@@@std@@@3@$0A@@std@@@std@@QAE?AU?$pair@Viterator@?$_Tree@V?$_Tmap_traits@HUAmbientSnd@@U?$less@H@std@@V?$allocator@U?$pair@$$CBHUAmbientSnd@@@std@@@3@$0A@@std@@@std@@_N@2@ABU?$pair@$$CBHUAmbientSnd@@@2@@Z 100924c0 f i ambientsnd.obj
 0002:00020900       ?_Insert@?$_Tree@V?$_Tmap_traits@HUAmbientSnd@@U?$less@H@std@@V?$allocator@U?$pair@$$CBHUAmbientSnd@@@std@@@3@$0A@@std@@@std@@IAE?AViterator@12@_NPAU_Node@?$_Tree_nod@V?$_Tmap_traits@HUAmbientSnd@@U?$less@H@std@@V?$allocator@U?$pair@$$CBHUAmbientSnd@@@std@@@3@$0A@@std@@@2@ABU?$pair@$$CBHUAmbientSnd@@@2@@Z 10092900 f i ambientsnd.obj
 0002:00020ed0       ?_Lbound@?$_Tree@V?$_Tmap_traits@HUAmbientSnd@@U?$less@H@std@@V?$allocator@U?$pair@$$CBHUAmbientSnd@@@std@@@3@$0A@@std@@@std@@IBEPAU_Node@?$_Tree_nod@V?$_Tmap_traits@HUAmbientSnd@@U?$less@H@std@@V?$allocator@U?$pair@$$CBHUAmbientSnd@@@std@@@3@$0A@@std@@@2@ABH@Z 10092ed0 f i ambientsnd.obj
 0002:00020fc0       ?_Rmost@?$_Tree@V?$_Tmap_traits@HUAmbientSnd@@U?$less@H@std@@V?$allocator@U?$pair@$$CBHUAmbientSnd@@@std@@@3@$0A@@std@@@std@@IBEAAPAU_Node@?$_Tree_nod@V?$_Tmap_traits@HUAmbientSnd@@U?$less@H@std@@V?$allocator@U?$pair@$$CBHUAmbientSnd@@@std@@@3@$0A@@std@@@2@XZ 10092fc0 f i ambientsnd.obj
 0002:00021000       ?_Kfn@?$_Tmap_traits@HUAmbientSnd@@U?$less@H@std@@V?$allocator@U?$pair@$$CBHUAmbientSnd@@@std@@@3@$0A@@std@@SAABHABU?$pair@$$CBHUAmbientSnd@@@2@@Z 10093000 f i ambientsnd.obj
 0002:00021010       ??0const_iterator@?$_Tree@V?$_Tmap_traits@HHU?$less@H@std@@V?$allocator@U?$pair@$$CBHH@std@@@2@$0A@@std@@@std@@QAE@XZ 10093010 f i ambientsnd.obj
 0002:00021050       ??0const_iterator@?$_Tree@V?$_Tmap_traits@HHU?$less@H@std@@V?$allocator@U?$pair@$$CBHH@std@@@2@$0A@@std@@@std@@QAE@PAU_Node@?$_Tree_nod@V?$_Tmap_traits@HHU?$less@H@std@@V?$allocator@U?$pair@$$CBHH@std@@@2@$0A@@std@@@2@PBV12@@Z 10093050 f i ambientsnd.obj
 0002:000210f0       ??Dconst_iterator@?$_Tree@V?$_Tmap_traits@HHU?$less@H@std@@V?$allocator@U?$pair@$$CBHH@std@@@2@$0A@@std@@@std@@QBEABU?$pair@$$CBHH@2@XZ 100930f0 f i ambientsnd.obj
 0002:000211c0       ??Econst_iterator@?$_Tree@V?$_Tmap_traits@HHU?$less@H@std@@V?$allocator@U?$pair@$$CBHH@std@@@2@$0A@@std@@@std@@QAEAAV012@XZ 100931c0 f i ambientsnd.obj
 0002:000211f0       ??Fconst_iterator@?$_Tree@V?$_Tmap_traits@HHU?$less@H@std@@V?$allocator@U?$pair@$$CBHH@std@@@2@$0A@@std@@@std@@QAEAAV012@XZ 100931f0 f i ambientsnd.obj
 0002:00021220       ??0const_iterator@?$_Tree@V?$_Tmap_traits@HUAmbientSnd@@U?$less@H@std@@V?$allocator@U?$pair@$$CBHUAmbientSnd@@@std@@@3@$0A@@std@@@std@@QAE@XZ 10093220 f i ambientsnd.obj
 0002:00021260       ??0const_iterator@?$_Tree@V?$_Tmap_traits@HUAmbientSnd@@U?$less@H@std@@V?$allocator@U?$pair@$$CBHUAmbientSnd@@@std@@@3@$0A@@std@@@std@@QAE@PAU_Node@?$_Tree_nod@V?$_Tmap_traits@HUAmbientSnd@@U?$less@H@std@@V?$allocator@U?$pair@$$CBHUAmbientSnd@@@std@@@3@$0A@@std@@@2@PBV12@@Z 10093260 f i ambientsnd.obj
 0002:00021300       ??Dconst_iterator@?$_Tree@V?$_Tmap_traits@HUAmbientSnd@@U?$less@H@std@@V?$allocator@U?$pair@$$CBHUAmbientSnd@@@std@@@3@$0A@@std@@@std@@QBEABU?$pair@$$CBHUAmbientSnd@@@2@XZ 10093300 f i ambientsnd.obj
 0002:000213d0       ??Econst_iterator@?$_Tree@V?$_Tmap_traits@HUAmbientSnd@@U?$less@H@std@@V?$allocator@U?$pair@$$CBHUAmbientSnd@@@std@@@3@$0A@@std@@@std@@QAEAAV012@XZ 100933d0 f i ambientsnd.obj
 0002:00021400       ??Fconst_iterator@?$_Tree@V?$_Tmap_traits@HUAmbientSnd@@U?$less@H@std@@V?$allocator@U?$pair@$$CBHUAmbientSnd@@@std@@@3@$0A@@std@@@std@@QAEAAV012@XZ 10093400 f i ambientsnd.obj
 0002:00021430       ??0?$_Bidit@U?$pair@$$CBHH@std@@HPBU12@ABU12@@std@@QAE@XZ 10093430 f i ambientsnd.obj
 0002:00021460       ??0?$_Bidit@U?$pair@$$CBHUAmbientSnd@@@std@@HPBU12@ABU12@@std@@QAE@XZ 10093460 f i ambientsnd.obj
 0002:00021490       ??0?$_Iterator_with_base@Ubidirectional_iterator_tag@std@@U?$pair@$$CBHH@2@HPBU32@ABU32@V_Iterator_base@2@@std@@QAE@XZ 10093490 f i ambientsnd.obj
 0002:000214c0       ??0?$_Iterator_with_base@Ubidirectional_iterator_tag@std@@U?$pair@$$CBHUAmbientSnd@@@2@HPBU32@ABU32@V_Iterator_base@2@@std@@QAE@XZ 100934c0 f i ambientsnd.obj
 0002:000214f0       ?_Color@?$_Tree@V?$_Tmap_traits@HHU?$less@H@std@@V?$allocator@U?$pair@$$CBHH@std@@@2@$0A@@std@@@std@@KAAADPAU_Node@?$_Tree_nod@V?$_Tmap_traits@HHU?$less@H@std@@V?$allocator@U?$pair@$$CBHH@std@@@2@$0A@@std@@@2@@Z 100934f0 f i ambientsnd.obj
 0002:00021500       ?max_size@?$_Tree@V?$_Tmap_traits@HHU?$less@H@std@@V?$allocator@U?$pair@$$CBHH@std@@@2@$0A@@std@@@std@@QBEIXZ 10093500 f i ambientsnd.obj
 0002:00021530       ?_Lmost@?$_Tree@V?$_Tmap_traits@HHU?$less@H@std@@V?$allocator@U?$pair@$$CBHH@std@@@2@$0A@@std@@@std@@IBEAAPAU_Node@?$_Tree_nod@V?$_Tmap_traits@HHU?$less@H@std@@V?$allocator@U?$pair@$$CBHH@std@@@2@$0A@@std@@@2@XZ 10093530 f i ambientsnd.obj
 0002:00021570       ?_Lrotate@?$_Tree@V?$_Tmap_traits@HHU?$less@H@std@@V?$allocator@U?$pair@$$CBHH@std@@@2@$0A@@std@@@std@@IAEXPAU_Node@?$_Tree_nod@V?$_Tmap_traits@HHU?$less@H@std@@V?$allocator@U?$pair@$$CBHH@std@@@2@$0A@@std@@@2@@Z 10093570 f i ambientsnd.obj
 0002:00021710       ?_Root@?$_Tree@V?$_Tmap_traits@HHU?$less@H@std@@V?$allocator@U?$pair@$$CBHH@std@@@2@$0A@@std@@@std@@IBEAAPAU_Node@?$_Tree_nod@V?$_Tmap_traits@HHU?$less@H@std@@V?$allocator@U?$pair@$$CBHH@std@@@2@$0A@@std@@@2@XZ 10093710 f i ambientsnd.obj
 0002:00021750       ?_Rrotate@?$_Tree@V?$_Tmap_traits@HHU?$less@H@std@@V?$allocator@U?$pair@$$CBHH@std@@@2@$0A@@std@@@std@@IAEXPAU_Node@?$_Tree_nod@V?$_Tmap_traits@HHU?$less@H@std@@V?$allocator@U?$pair@$$CBHH@std@@@2@$0A@@std@@@2@@Z 10093750 f i ambientsnd.obj
 0002:000218f0       ?_Buynode@?$_Tree@V?$_Tmap_traits@HHU?$less@H@std@@V?$allocator@U?$pair@$$CBHH@std@@@2@$0A@@std@@@std@@IAEPAU_Node@?$_Tree_nod@V?$_Tmap_traits@HHU?$less@H@std@@V?$allocator@U?$pair@$$CBHH@std@@@2@$0A@@std@@@2@PAU342@00ABU?$pair@$$CBHH@2@D@Z 100938f0 f i ambientsnd.obj
 0002:00021a40       ?deallocate@?$allocator@U_Node@?$_Tree_nod@V?$_Tmap_traits@HHU?$less@H@std@@V?$allocator@U?$pair@$$CBHH@std@@@2@$0A@@std@@@std@@@std@@QAEXPAU_Node@?$_Tree_nod@V?$_Tmap_traits@HHU?$less@H@std@@V?$allocator@U?$pair@$$CBHH@std@@@2@$0A@@std@@@2@I@Z 10093a40 f i ambientsnd.obj
 0002:00021a80       ?_Color@?$_Tree@V?$_Tmap_traits@HUAmbientSnd@@U?$less@H@std@@V?$allocator@U?$pair@$$CBHUAmbientSnd@@@std@@@3@$0A@@std@@@std@@KAAADPAU_Node@?$_Tree_nod@V?$_Tmap_traits@HUAmbientSnd@@U?$less@H@std@@V?$allocator@U?$pair@$$CBHUAmbientSnd@@@std@@@3@$0A@@std@@@2@@Z 10093a80 f i ambientsnd.obj
 0002:00021a90       ?_Left@?$_Tree@V?$_Tmap_traits@HUAmbientSnd@@U?$less@H@std@@V?$allocator@U?$pair@$$CBHUAmbientSnd@@@std@@@3@$0A@@std@@@std@@KAAAPAU_Node@?$_Tree_nod@V?$_Tmap_traits@HUAmbientSnd@@U?$less@H@std@@V?$allocator@U?$pair@$$CBHUAmbientSnd@@@std@@@3@$0A@@std@@@2@PAU342@@Z 10093a90 f i ambientsnd.obj
 0002:00021aa0       ?_Parent@?$_Tree@V?$_Tmap_traits@HUAmbientSnd@@U?$less@H@std@@V?$allocator@U?$pair@$$CBHUAmbientSnd@@@std@@@3@$0A@@std@@@std@@KAAAPAU_Node@?$_Tree_nod@V?$_Tmap_traits@HUAmbientSnd@@U?$less@H@std@@V?$allocator@U?$pair@$$CBHUAmbientSnd@@@std@@@3@$0A@@std@@@2@PAU342@@Z 10093aa0 f i ambientsnd.obj
 0002:00021ab0       ?max_size@?$_Tree@V?$_Tmap_traits@HUAmbientSnd@@U?$less@H@std@@V?$allocator@U?$pair@$$CBHUAmbientSnd@@@std@@@3@$0A@@std@@@std@@QBEIXZ 10093ab0 f i ambientsnd.obj
 0002:00021ae0       ?_Lmost@?$_Tree@V?$_Tmap_traits@HUAmbientSnd@@U?$less@H@std@@V?$allocator@U?$pair@$$CBHUAmbientSnd@@@std@@@3@$0A@@std@@@std@@IBEAAPAU_Node@?$_Tree_nod@V?$_Tmap_traits@HUAmbientSnd@@U?$less@H@std@@V?$allocator@U?$pair@$$CBHUAmbientSnd@@@std@@@3@$0A@@std@@@2@XZ 10093ae0 f i ambientsnd.obj
 0002:00021b20       ?_Lrotate@?$_Tree@V?$_Tmap_traits@HUAmbientSnd@@U?$less@H@std@@V?$allocator@U?$pair@$$CBHUAmbientSnd@@@std@@@3@$0A@@std@@@std@@IAEXPAU_Node@?$_Tree_nod@V?$_Tmap_traits@HUAmbientSnd@@U?$less@H@std@@V?$allocator@U?$pair@$$CBHUAmbientSnd@@@std@@@3@$0A@@std@@@2@@Z 10093b20 f i ambientsnd.obj
 0002:00021cc0       ?_Root@?$_Tree@V?$_Tmap_traits@HUAmbientSnd@@U?$less@H@std@@V?$allocator@U?$pair@$$CBHUAmbientSnd@@@std@@@3@$0A@@std@@@std@@IBEAAPAU_Node@?$_Tree_nod@V?$_Tmap_traits@HUAmbientSnd@@U?$less@H@std@@V?$allocator@U?$pair@$$CBHUAmbientSnd@@@std@@@3@$0A@@std@@@2@XZ 10093cc0 f i ambientsnd.obj
 0002:00021d00       ?_Rrotate@?$_Tree@V?$_Tmap_traits@HUAmbientSnd@@U?$less@H@std@@V?$allocator@U?$pair@$$CBHUAmbientSnd@@@std@@@3@$0A@@std@@@std@@IAEXPAU_Node@?$_Tree_nod@V?$_Tmap_traits@HUAmbientSnd@@U?$less@H@std@@V?$allocator@U?$pair@$$CBHUAmbientSnd@@@std@@@3@$0A@@std@@@2@@Z 10093d00 f i ambientsnd.obj
 0002:00021ea0       ?_Buynode@?$_Tree@V?$_Tmap_traits@HUAmbientSnd@@U?$less@H@std@@V?$allocator@U?$pair@$$CBHUAmbientSnd@@@std@@@3@$0A@@std@@@std@@IAEPAU_Node@?$_Tree_nod@V?$_Tmap_traits@HUAmbientSnd@@U?$less@H@std@@V?$allocator@U?$pair@$$CBHUAmbientSnd@@@std@@@3@$0A@@std@@@2@PAU342@00ABU?$pair@$$CBHUAmbientSnd@@@2@D@Z 10093ea0 f i ambientsnd.obj
 0002:00021ff0       ??Fiterator@?$_Tree@V?$_Tmap_traits@HHU?$less@H@std@@V?$allocator@U?$pair@$$CBHH@std@@@2@$0A@@std@@@std@@QAEAAV012@XZ 10093ff0 f i ambientsnd.obj
 0002:00022020       ?_Dec@const_iterator@?$_Tree@V?$_Tmap_traits@HHU?$less@H@std@@V?$allocator@U?$pair@$$CBHH@std@@@2@$0A@@std@@@std@@QAEXXZ 10094020 f i ambientsnd.obj
 0002:000222f0       ?_Inc@const_iterator@?$_Tree@V?$_Tmap_traits@HHU?$less@H@std@@V?$allocator@U?$pair@$$CBHH@std@@@2@$0A@@std@@@std@@QAEXXZ 100942f0 f i ambientsnd.obj
 0002:00022480       ??Fiterator@?$_Tree@V?$_Tmap_traits@HUAmbientSnd@@U?$less@H@std@@V?$allocator@U?$pair@$$CBHUAmbientSnd@@@std@@@3@$0A@@std@@@std@@QAEAAV012@XZ 10094480 f i ambientsnd.obj
 0002:000224b0       ?_Dec@const_iterator@?$_Tree@V?$_Tmap_traits@HUAmbientSnd@@U?$less@H@std@@V?$allocator@U?$pair@$$CBHUAmbientSnd@@@std@@@3@$0A@@std@@@std@@QAEXXZ 100944b0 f i ambientsnd.obj
 0002:00022780       ?_Inc@const_iterator@?$_Tree@V?$_Tmap_traits@HUAmbientSnd@@U?$less@H@std@@V?$allocator@U?$pair@$$CBHUAmbientSnd@@@std@@@3@$0A@@std@@@std@@QAEXXZ 10094780 f i ambientsnd.obj
 0002:00022910       ??0?$pair@Viterator@?$_Tree@V?$_Tmap_traits@HHU?$less@H@std@@V?$allocator@U?$pair@$$CBHH@std@@@2@$0A@@std@@@std@@_N@std@@QAE@ABViterator@?$_Tree@V?$_Tmap_traits@HHU?$less@H@std@@V?$allocator@U?$pair@$$CBHH@std@@@2@$0A@@std@@@1@AB_N@Z 10094910 f i ambientsnd.obj
 0002:00022960       ??0?$pair@Viterator@?$_Tree@V?$_Tmap_traits@HUAmbientSnd@@U?$less@H@std@@V?$allocator@U?$pair@$$CBHUAmbientSnd@@@std@@@3@$0A@@std@@@std@@_N@std@@QAE@ABViterator@?$_Tree@V?$_Tmap_traits@HUAmbientSnd@@U?$less@H@std@@V?$allocator@U?$pair@$$CBHUAmbientSnd@@@std@@@3@$0A@@std@@@1@AB_N@Z 10094960 f i ambientsnd.obj
 0002:000229b0       ?_Max@?$_Tree@V?$_Tmap_traits@HHU?$less@H@std@@V?$allocator@U?$pair@$$CBHH@std@@@2@$0A@@std@@@std@@KAPAU_Node@?$_Tree_nod@V?$_Tmap_traits@HHU?$less@H@std@@V?$allocator@U?$pair@$$CBHH@std@@@2@$0A@@std@@@2@PAU342@@Z 100949b0 f i ambientsnd.obj
 0002:00022a00       ?_Min@?$_Tree@V?$_Tmap_traits@HHU?$less@H@std@@V?$allocator@U?$pair@$$CBHH@std@@@2@$0A@@std@@@std@@KAPAU_Node@?$_Tree_nod@V?$_Tmap_traits@HHU?$less@H@std@@V?$allocator@U?$pair@$$CBHH@std@@@2@$0A@@std@@@2@PAU342@@Z 10094a00 f i ambientsnd.obj
 0002:00022a50       ?max_size@?$allocator@U?$pair@$$CBHH@std@@@std@@QBEIXZ 10094a50 f i ambientsnd.obj
 0002:00022ab0       ?allocate@?$allocator@U_Node@?$_Tree_nod@V?$_Tmap_traits@HHU?$less@H@std@@V?$allocator@U?$pair@$$CBHH@std@@@2@$0A@@std@@@std@@@std@@QAEPAU_Node@?$_Tree_nod@V?$_Tmap_traits@HHU?$less@H@std@@V?$allocator@U?$pair@$$CBHH@std@@@2@$0A@@std@@@2@I@Z 10094ab0 f i ambientsnd.obj
 0002:00022af0       ?_Max@?$_Tree@V?$_Tmap_traits@HUAmbientSnd@@U?$less@H@std@@V?$allocator@U?$pair@$$CBHUAmbientSnd@@@std@@@3@$0A@@std@@@std@@KAPAU_Node@?$_Tree_nod@V?$_Tmap_traits@HUAmbientSnd@@U?$less@H@std@@V?$allocator@U?$pair@$$CBHUAmbientSnd@@@std@@@3@$0A@@std@@@2@PAU342@@Z 10094af0 f i ambientsnd.obj
 0002:00022b40       ?_Min@?$_Tree@V?$_Tmap_traits@HUAmbientSnd@@U?$less@H@std@@V?$allocator@U?$pair@$$CBHUAmbientSnd@@@std@@@3@$0A@@std@@@std@@KAPAU_Node@?$_Tree_nod@V?$_Tmap_traits@HUAmbientSnd@@U?$less@H@std@@V?$allocator@U?$pair@$$CBHUAmbientSnd@@@std@@@3@$0A@@std@@@2@PAU342@@Z 10094b40 f i ambientsnd.obj
 0002:00022b90       ?max_size@?$allocator@U?$pair@$$CBHUAmbientSnd@@@std@@@std@@QBEIXZ 10094b90 f i ambientsnd.obj
 0002:00022bf0       ?deallocate@?$allocator@U_Node@?$_Tree_nod@V?$_Tmap_traits@HUAmbientSnd@@U?$less@H@std@@V?$allocator@U?$pair@$$CBHUAmbientSnd@@@std@@@3@$0A@@std@@@std@@@std@@QAEXPAU_Node@?$_Tree_nod@V?$_Tmap_traits@HUAmbientSnd@@U?$less@H@std@@V?$allocator@U?$pair@$$CBHUAmbientSnd@@@std@@@3@$0A@@std@@@2@I@Z 10094bf0 f i ambientsnd.obj
 0002:00022c30       ?allocate@?$allocator@U_Node@?$_Tree_nod@V?$_Tmap_traits@HUAmbientSnd@@U?$less@H@std@@V?$allocator@U?$pair@$$CBHUAmbientSnd@@@std@@@3@$0A@@std@@@std@@@std@@QAEPAU_Node@?$_Tree_nod@V?$_Tmap_traits@HUAmbientSnd@@U?$less@H@std@@V?$allocator@U?$pair@$$CBHUAmbientSnd@@@std@@@3@$0A@@std@@@2@I@Z 10094c30 f i ambientsnd.obj
 0002:00022c70       ??0_Node@?$_Tree_nod@V?$_Tmap_traits@HHU?$less@H@std@@V?$allocator@U?$pair@$$CBHH@std@@@2@$0A@@std@@@std@@QAE@PAU012@00ABU?$pair@$$CBHH@2@D@Z 10094c70 f i ambientsnd.obj
 0002:00022ce0       ??0_Node@?$_Tree_nod@V?$_Tmap_traits@HUAmbientSnd@@U?$less@H@std@@V?$allocator@U?$pair@$$CBHUAmbientSnd@@@std@@@3@$0A@@std@@@std@@QAE@PAU012@00ABU?$pair@$$CBHUAmbientSnd@@@2@D@Z 10094ce0 f i ambientsnd.obj
 0002:00022d60       ??$_Allocate@U_Node@?$_Tree_nod@V?$_Tmap_traits@HHU?$less@H@std@@V?$allocator@U?$pair@$$CBHH@std@@@2@$0A@@std@@@std@@@std@@YAPAU_Node@?$_Tree_nod@V?$_Tmap_traits@HHU?$less@H@std@@V?$allocator@U?$pair@$$CBHH@std@@@2@$0A@@std@@@0@IPAU120@@Z 10094d60 f i ambientsnd.obj
 0002:00022df0       ??$_Allocate@U_Node@?$_Tree_nod@V?$_Tmap_traits@HUAmbientSnd@@U?$less@H@std@@V?$allocator@U?$pair@$$CBHUAmbientSnd@@@std@@@3@$0A@@std@@@std@@@std@@YAPAU_Node@?$_Tree_nod@V?$_Tmap_traits@HUAmbientSnd@@U?$less@H@std@@V?$allocator@U?$pair@$$CBHUAmbientSnd@@@std@@@3@$0A@@std@@@0@IPAU120@@Z 10094df0 f i ambientsnd.obj
 0002:00022e80       ??0?$map@HHU?$less@H@std@@V?$allocator@U?$pair@$$CBHH@std@@@2@@std@@QAE@XZ 10094e80 f i ambientsnd.obj
 0002:00022ed0       ??0?$_Tree@V?$_Tmap_traits@HHU?$less@H@std@@V?$allocator@U?$pair@$$CBHH@std@@@2@$0A@@std@@@std@@QAE@ABU?$less@H@1@ABV?$allocator@U?$pair@$$CBHH@std@@@1@@Z 10094ed0 f i ambientsnd.obj
 0002:00022f80       ??1?$_Tree_val@V?$_Tmap_traits@HHU?$less@H@std@@V?$allocator@U?$pair@$$CBHH@std@@@2@$0A@@std@@@std@@QAE@XZ 10094f80 f i ambientsnd.obj
 0002:00022fb0       ??1?$_Tree_ptr@V?$_Tmap_traits@HHU?$less@H@std@@V?$allocator@U?$pair@$$CBHH@std@@@2@$0A@@std@@@std@@QAE@XZ 10094fb0 f i ambientsnd.obj
 0002:00022fe0       ??1?$_Tree_nod@V?$_Tmap_traits@HHU?$less@H@std@@V?$allocator@U?$pair@$$CBHH@std@@@2@$0A@@std@@@std@@QAE@XZ 10094fe0 f i ambientsnd.obj
 0002:00023010       ??1?$_Tmap_traits@HHU?$less@H@std@@V?$allocator@U?$pair@$$CBHH@std@@@2@$0A@@std@@QAE@XZ 10095010 f i ambientsnd.obj
 0002:00023040       ??1?$_Container_base_aux_alloc_empty@V?$allocator@U?$pair@$$CBHH@std@@@std@@@std@@IAE@XZ 10095040 f i ambientsnd.obj
 0002:00023070       ??0?$allocator@U?$pair@$$CBHH@std@@@std@@QAE@XZ 10095070 f i ambientsnd.obj
 0002:00023090       ?_Init@?$_Tree@V?$_Tmap_traits@HHU?$less@H@std@@V?$allocator@U?$pair@$$CBHH@std@@@2@$0A@@std@@@std@@IAEXXZ 10095090 f i ambientsnd.obj
 0002:00023130       ??0?$_Tree_val@V?$_Tmap_traits@HHU?$less@H@std@@V?$allocator@U?$pair@$$CBHH@std@@@2@$0A@@std@@@std@@IAE@ABU?$less@H@1@V?$allocator@U?$pair@$$CBHH@std@@@1@@Z 10095130 f i ambientsnd.obj
 0002:000231a0       ??0?$allocator@U?$pair@$$CBHH@std@@@std@@QAE@ABV01@@Z 100951a0 f i ambientsnd.obj
 0002:000231c0       ?_Buynode@?$_Tree@V?$_Tmap_traits@HHU?$less@H@std@@V?$allocator@U?$pair@$$CBHH@std@@@2@$0A@@std@@@std@@IAEPAU_Node@?$_Tree_nod@V?$_Tmap_traits@HHU?$less@H@std@@V?$allocator@U?$pair@$$CBHH@std@@@2@$0A@@std@@@2@XZ 100951c0 f i ambientsnd.obj
 0002:000233d0       ?destroy@?$allocator@PAU_Node@?$_Tree_nod@V?$_Tmap_traits@HHU?$less@H@std@@V?$allocator@U?$pair@$$CBHH@std@@@2@$0A@@std@@@std@@@std@@QAEXPAPAU_Node@?$_Tree_nod@V?$_Tmap_traits@HHU?$less@H@std@@V?$allocator@U?$pair@$$CBHH@std@@@2@$0A@@std@@@2@@Z 100953d0 f i ambientsnd.obj
 0002:00023410       ??0?$_Tree_ptr@V?$_Tmap_traits@HHU?$less@H@std@@V?$allocator@U?$pair@$$CBHH@std@@@2@$0A@@std@@@std@@QAE@ABU?$less@H@1@V?$allocator@U?$pair@$$CBHH@std@@@1@@Z 10095410 f i ambientsnd.obj
 0002:00023480       ??0?$_Tree_nod@V?$_Tmap_traits@HHU?$less@H@std@@V?$allocator@U?$pair@$$CBHH@std@@@2@$0A@@std@@@std@@IAE@ABU?$less@H@1@V?$allocator@U?$pair@$$CBHH@std@@@1@@Z 10095480 f i ambientsnd.obj
 0002:000234f0       ?construct@?$allocator@PAU_Node@?$_Tree_nod@V?$_Tmap_traits@HHU?$less@H@std@@V?$allocator@U?$pair@$$CBHH@std@@@2@$0A@@std@@@std@@@std@@QAEXPAPAU_Node@?$_Tree_nod@V?$_Tmap_traits@HHU?$less@H@std@@V?$allocator@U?$pair@$$CBHH@std@@@2@$0A@@std@@@2@ABQAU342@@Z 100954f0 f i ambientsnd.obj
 0002:00023530       ??0?$_Tmap_traits@HHU?$less@H@std@@V?$allocator@U?$pair@$$CBHH@std@@@2@$0A@@std@@QAE@U?$less@H@1@V?$allocator@U?$pair@$$CBHH@std@@@1@@Z 10095530 f i ambientsnd.obj
 0002:00023590       ??0?$_Container_base_aux_alloc_empty@V?$allocator@U?$pair@$$CBHH@std@@@std@@@std@@IAE@V?$allocator@U?$pair@$$CBHH@std@@@1@@Z 10095590 f i ambientsnd.obj
 0002:000235d0       ??$_Destroy@PAU_Node@?$_Tree_nod@V?$_Tmap_traits@HHU?$less@H@std@@V?$allocator@U?$pair@$$CBHH@std@@@2@$0A@@std@@@std@@@std@@YAXPAPAU_Node@?$_Tree_nod@V?$_Tmap_traits@HHU?$less@H@std@@V?$allocator@U?$pair@$$CBHH@std@@@2@$0A@@std@@@0@@Z 100955d0 f i ambientsnd.obj
 0002:000235e0       ??$?0U?$pair@$$CBHH@std@@@?$allocator@PAU_Node@?$_Tree_nod@V?$_Tmap_traits@HHU?$less@H@std@@V?$allocator@U?$pair@$$CBHH@std@@@2@$0A@@std@@@std@@@std@@QAE@ABV?$allocator@U?$pair@$$CBHH@std@@@1@@Z 100955e0 f i ambientsnd.obj
 0002:00023600       ??$?0U?$pair@$$CBHH@std@@@?$allocator@U_Node@?$_Tree_nod@V?$_Tmap_traits@HHU?$less@H@std@@V?$allocator@U?$pair@$$CBHH@std@@@2@$0A@@std@@@std@@@std@@QAE@ABV?$allocator@U?$pair@$$CBHH@std@@@1@@Z 10095600 f i ambientsnd.obj
 0002:00023620       ??$_Construct@PAU_Node@?$_Tree_nod@V?$_Tmap_traits@HHU?$less@H@std@@V?$allocator@U?$pair@$$CBHH@std@@@2@$0A@@std@@@std@@PAU123@@std@@YAXPAPAU_Node@?$_Tree_nod@V?$_Tmap_traits@HHU?$less@H@std@@V?$allocator@U?$pair@$$CBHH@std@@@2@$0A@@std@@@0@ABQAU120@@Z 10095620 f i ambientsnd.obj
 0002:000236a0       ??1?$map@HHU?$less@H@std@@V?$allocator@U?$pair@$$CBHH@std@@@2@@std@@QAE@XZ 100956a0 f i ambientsnd.obj
 0002:000236d0       ??1?$_Tree@V?$_Tmap_traits@HHU?$less@H@std@@V?$allocator@U?$pair@$$CBHH@std@@@2@$0A@@std@@@std@@QAE@XZ 100956d0 f i ambientsnd.obj
 0002:00023750       ?_Tidy@?$_Tree@V?$_Tmap_traits@HHU?$less@H@std@@V?$allocator@U?$pair@$$CBHH@std@@@2@$0A@@std@@@std@@IAEXXZ 10095750 f i ambientsnd.obj
 0002:00023920       ?erase@?$_Tree@V?$_Tmap_traits@HHU?$less@H@std@@V?$allocator@U?$pair@$$CBHH@std@@@2@$0A@@std@@@std@@QAE?AViterator@12@Vconst_iterator@12@0@Z 10095920 f i ambientsnd.obj
 0002:00023bb0       ?_Make_iter@?$_Tree@V?$_Tmap_traits@HHU?$less@H@std@@V?$allocator@U?$pair@$$CBHH@std@@@2@$0A@@std@@@std@@QBE?AViterator@12@Vconst_iterator@12@@Z 10095bb0 f i ambientsnd.obj
 0002:00023ca0       ?erase@?$_Tree@V?$_Tmap_traits@HHU?$less@H@std@@V?$allocator@U?$pair@$$CBHH@std@@@2@$0A@@std@@@std@@QAE?AViterator@12@Vconst_iterator@12@@Z 10095ca0 f i ambientsnd.obj
 0002:000246c0       ?clear@?$_Tree@V?$_Tmap_traits@HHU?$less@H@std@@V?$allocator@U?$pair@$$CBHH@std@@@2@$0A@@std@@@std@@QAEXXZ 100966c0 f i ambientsnd.obj
 0002:00024760       ??Econst_iterator@?$_Tree@V?$_Tmap_traits@HHU?$less@H@std@@V?$allocator@U?$pair@$$CBHH@std@@@2@$0A@@std@@@std@@QAE?AV012@H@Z 10096760 f i ambientsnd.obj
 0002:00024860       ??9const_iterator@?$_Tree@V?$_Tmap_traits@HHU?$less@H@std@@V?$allocator@U?$pair@$$CBHH@std@@@2@$0A@@std@@@std@@QBE_NABV012@@Z 10096860 f i ambientsnd.obj
 0002:000248b0       ?_Erase@?$_Tree@V?$_Tmap_traits@HHU?$less@H@std@@V?$allocator@U?$pair@$$CBHH@std@@@2@$0A@@std@@@std@@IAEXPAU_Node@?$_Tree_nod@V?$_Tmap_traits@HHU?$less@H@std@@V?$allocator@U?$pair@$$CBHH@std@@@2@$0A@@std@@@2@@Z 100968b0 f i ambientsnd.obj
 0002:00024970       ?_Orphan_ptr@?$_Tree@V?$_Tmap_traits@HHU?$less@H@std@@V?$allocator@U?$pair@$$CBHH@std@@@2@$0A@@std@@@std@@IBEXAAV12@PAU_Node@?$_Tree_nod@V?$_Tmap_traits@HHU?$less@H@std@@V?$allocator@U?$pair@$$CBHH@std@@@2@$0A@@std@@@2@@Z 10096970 f i ambientsnd.obj
 0002:00024a70       ?destroy@?$allocator@U_Node@?$_Tree_nod@V?$_Tmap_traits@HHU?$less@H@std@@V?$allocator@U?$pair@$$CBHH@std@@@2@$0A@@std@@@std@@@std@@QAEXPAU_Node@?$_Tree_nod@V?$_Tmap_traits@HHU?$less@H@std@@V?$allocator@U?$pair@$$CBHH@std@@@2@$0A@@std@@@2@@Z 10096a70 f i ambientsnd.obj
 0002:00024ab0       ??$_Destroy@U_Node@?$_Tree_nod@V?$_Tmap_traits@HHU?$less@H@std@@V?$allocator@U?$pair@$$CBHH@std@@@2@$0A@@std@@@std@@@std@@YAXPAU_Node@?$_Tree_nod@V?$_Tmap_traits@HHU?$less@H@std@@V?$allocator@U?$pair@$$CBHH@std@@@2@$0A@@std@@@0@@Z 10096ab0 f i ambientsnd.obj
 0002:00024ac0       ?event_music_init@@YAHXZ   10096ac0 f   eventmusic.obj
 0002:00024ad0       ?event_music_close@@YAXXZ  10096ad0 f   eventmusic.obj
 0002:00024ae0       ?event_music_start@@YAHHMH@Z 10096ae0 f   eventmusic.obj
 0002:00024c40       ?event_music_stop@@YAXHH@Z 10096c40 f   eventmusic.obj
 0002:00024df0       ?event_music_stop_all@@YAXH@Z 10096df0 f   eventmusic.obj
 0002:00024e10       ?event_music_pause@@YAXH@Z 10096e10 f   eventmusic.obj
 0002:00024e50       ?event_music_pause_all@@YAXXZ 10096e50 f   eventmusic.obj
 0002:00024e70       ?event_music_unpause@@YAXH@Z 10096e70 f   eventmusic.obj
 0002:00024eb0       ?event_music_unpause_all@@YAXXZ 10096eb0 f   eventmusic.obj
 0002:00024ed0       ?event_music_set_volume@@YAXHM@Z 10096ed0 f   eventmusic.obj
 0002:00024f20       ?event_music_set_volume_all@@YAXM@Z 10096f20 f   eventmusic.obj
 0002:00024f40       ?event_music_set_loop@@YAXHH@Z 10096f40 f   eventmusic.obj
 0002:00024f80       ?event_music_state@@YAHH@Z 10096f80 f   eventmusic.obj
 0002:00025130       ?gamesnd_init_sounds@@YAXXZ 10097130 f   gamesnd.obj
 0002:00025160       ?gamesnd_close@@YAXXZ      10097160 f   gamesnd.obj
 0002:00025180       ?gamesnd_stop_iface@@YAXH@Z 10097180 f   gamesnd.obj
 0002:000251a0       ?gamesnd_play_iface@@YAHHM@Z 100971a0 f   gamesnd.obj
 0002:000252e0       ?gamesnd_load_gameplay_sounds@@YAXXZ 100972e0 f   gamesnd.obj
 0002:00025410       ?gamesnd_unload_gameplay_sounds@@YAXXZ 10097410 f   gamesnd.obj
 0002:00025540       ?gamesnd_load_interface_sounds@@YAXXZ 10097540 f   gamesnd.obj
 0002:00025680       ?gamesnd_unload_interface_sounds@@YAXXZ 10097680 f   gamesnd.obj
 0002:00025940       ?begin@?$_Tree@V?$_Tmap_traits@HUgame_snd@@U?$less@H@std@@V?$allocator@U?$pair@$$CBHUgame_snd@@@std@@@3@$0A@@std@@@std@@QAE?AViterator@12@XZ 10097940 f i gamesnd.obj
 0002:000259b0       ?clear@?$_Tree@V?$_Tmap_traits@HUgame_snd@@U?$less@H@std@@V?$allocator@U?$pair@$$CBHUgame_snd@@@std@@@3@$0A@@std@@@std@@QAEXXZ 100979b0 f i gamesnd.obj
 0002:00025a50       ??Eiterator@?$_Tree@V?$_Tmap_traits@HUgame_snd@@U?$less@H@std@@V?$allocator@U?$pair@$$CBHUgame_snd@@@std@@@3@$0A@@std@@@std@@QAEAAV012@XZ 10097a50 f i gamesnd.obj
 0002:00025a80       ?_Erase@?$_Tree@V?$_Tmap_traits@HUgame_snd@@U?$less@H@std@@V?$allocator@U?$pair@$$CBHUgame_snd@@@std@@@3@$0A@@std@@@std@@IAEXPAU_Node@?$_Tree_nod@V?$_Tmap_traits@HUgame_snd@@U?$less@H@std@@V?$allocator@U?$pair@$$CBHUgame_snd@@@std@@@3@$0A@@std@@@2@@Z 10097a80 f i gamesnd.obj
 0002:00025b40       ?_Lmost@?$_Tree@V?$_Tmap_traits@HUgame_snd@@U?$less@H@std@@V?$allocator@U?$pair@$$CBHUgame_snd@@@std@@@3@$0A@@std@@@std@@IBEAAPAU_Node@?$_Tree_nod@V?$_Tmap_traits@HUgame_snd@@U?$less@H@std@@V?$allocator@U?$pair@$$CBHUgame_snd@@@std@@@3@$0A@@std@@@2@XZ 10097b40 f i gamesnd.obj
 0002:00025b80       ?_Rmost@?$_Tree@V?$_Tmap_traits@HUgame_snd@@U?$less@H@std@@V?$allocator@U?$pair@$$CBHUgame_snd@@@std@@@3@$0A@@std@@@std@@IBEAAPAU_Node@?$_Tree_nod@V?$_Tmap_traits@HUgame_snd@@U?$less@H@std@@V?$allocator@U?$pair@$$CBHUgame_snd@@@std@@@3@$0A@@std@@@2@XZ 10097b80 f i gamesnd.obj
 0002:00025bc0       ?_Orphan_ptr@?$_Tree@V?$_Tmap_traits@HUgame_snd@@U?$less@H@std@@V?$allocator@U?$pair@$$CBHUgame_snd@@@std@@@3@$0A@@std@@@std@@IBEXAAV12@PAU_Node@?$_Tree_nod@V?$_Tmap_traits@HUgame_snd@@U?$less@H@std@@V?$allocator@U?$pair@$$CBHUgame_snd@@@std@@@3@$0A@@std@@@2@@Z 10097bc0 f i gamesnd.obj
 0002:00025cc0       ??Econst_iterator@?$_Tree@V?$_Tmap_traits@HUgame_snd@@U?$less@H@std@@V?$allocator@U?$pair@$$CBHUgame_snd@@@std@@@3@$0A@@std@@@std@@QAEAAV012@XZ 10097cc0 f i gamesnd.obj
 0002:00025cf0       ?deallocate@?$allocator@U_Node@?$_Tree_nod@V?$_Tmap_traits@HUgame_snd@@U?$less@H@std@@V?$allocator@U?$pair@$$CBHUgame_snd@@@std@@@3@$0A@@std@@@std@@@std@@QAEXPAU_Node@?$_Tree_nod@V?$_Tmap_traits@HUgame_snd@@U?$less@H@std@@V?$allocator@U?$pair@$$CBHUgame_snd@@@std@@@3@$0A@@std@@@2@I@Z 10097cf0 f i gamesnd.obj
 0002:00025d30       ?destroy@?$allocator@U_Node@?$_Tree_nod@V?$_Tmap_traits@HUgame_snd@@U?$less@H@std@@V?$allocator@U?$pair@$$CBHUgame_snd@@@std@@@3@$0A@@std@@@std@@@std@@QAEXPAU_Node@?$_Tree_nod@V?$_Tmap_traits@HUgame_snd@@U?$less@H@std@@V?$allocator@U?$pair@$$CBHUgame_snd@@@std@@@3@$0A@@std@@@2@@Z 10097d30 f i gamesnd.obj
 0002:00025d70       ?_Inc@const_iterator@?$_Tree@V?$_Tmap_traits@HUgame_snd@@U?$less@H@std@@V?$allocator@U?$pair@$$CBHUgame_snd@@@std@@@3@$0A@@std@@@std@@QAEXXZ 10097d70 f i gamesnd.obj
 0002:00025f00       ?_Min@?$_Tree@V?$_Tmap_traits@HUgame_snd@@U?$less@H@std@@V?$allocator@U?$pair@$$CBHUgame_snd@@@std@@@3@$0A@@std@@@std@@KAPAU_Node@?$_Tree_nod@V?$_Tmap_traits@HUgame_snd@@U?$less@H@std@@V?$allocator@U?$pair@$$CBHUgame_snd@@@std@@@3@$0A@@std@@@2@PAU342@@Z 10097f00 f i gamesnd.obj
 0002:00025f50       ??$_Destroy@U_Node@?$_Tree_nod@V?$_Tmap_traits@HUgame_snd@@U?$less@H@std@@V?$allocator@U?$pair@$$CBHUgame_snd@@@std@@@3@$0A@@std@@@std@@@std@@YAXPAU_Node@?$_Tree_nod@V?$_Tmap_traits@HUgame_snd@@U?$less@H@std@@V?$allocator@U?$pair@$$CBHUgame_snd@@@std@@@3@$0A@@std@@@0@@Z 10097f50 f i gamesnd.obj
 0002:00025f60       ?gamesnd_parse_soundtbl@@YAXPAD@Z 10097f60 f   scriptparser.obj
 0002:00026a20       ?gamesnd_parse_musictbl@@YAXPAD@Z 10098a20 f   scriptparser.obj
 0002:00026e50       ?gamesnd_parse_voicetbl@@YAXPAD@Z 10098e50 f   scriptparser.obj
 0002:00027260       ?gamesnd_parse_configtbl@@YAXPAD@Z 10099260 f   scriptparser.obj
 0002:00027520       ?gamesnd_parse_soundtxt@@YAXPAD@Z 10099520 f   scriptparser.obj
 0002:00028170       ?gamesnd_parse_musictxt@@YAXPAD@Z 1009a170 f   scriptparser.obj
 0002:00028670       ?gamesnd_parse_voicetxt@@YAXPAD@Z 1009a670 f   scriptparser.obj
 0002:00028b30       ?gamesnd_parse_configtxt@@YAXPAD@Z 1009ab30 f   scriptparser.obj
 0002:00028e80       ?gamesnd_parse_config@@YAXPAD_N@Z 1009ae80 f   scriptparser.obj
 0002:00028eb0       ?gamesnd_parse_music@@YAXPAD_N@Z 1009aeb0 f   scriptparser.obj
 0002:00028ee0       ?gamesnd_parse_sound@@YAXPAD_N@Z 1009aee0 f   scriptparser.obj
 0002:00028f10       ?gamesnd_parse_voice@@YAXPAD_N@Z 1009af10 f   scriptparser.obj
 0002:00029b40       ??1?$pair@Viterator@?$_Tree@V?$_Tmap_traits@HUgame_snd@@U?$less@H@std@@V?$allocator@U?$pair@$$CBHUgame_snd@@@std@@@3@$0A@@std@@@std@@_N@std@@QAE@XZ 1009bb40 f i scriptparser.obj
 0002:00029b70       ??0ST_ROWS@@QAE@XZ         1009bb70 f i scriptparser.obj
 0002:00029ba0       ??1ST_ROWS@@QAE@XZ         1009bba0 f i scriptparser.obj
 0002:00029bd0       ??4?$basic_string@DU?$char_traits@D@std@@V?$allocator@D@2@@std@@QAEAAV01@ABV01@@Z 1009bbd0 f i scriptparser.obj
 0002:00029c10       ?empty@?$basic_string@DU?$char_traits@D@std@@V?$allocator@D@2@@std@@QBE_NXZ 1009bc10 f i scriptparser.obj
 0002:00029c40       ??A?$map@HUgame_snd@@U?$less@H@std@@V?$allocator@U?$pair@$$CBHUgame_snd@@@std@@@3@@std@@QAEAAUgame_snd@@ABH@Z 1009bc40 f i scriptparser.obj
 0002:00029ee0       ?insert@?$_Tree@V?$_Tmap_traits@HUgame_snd@@U?$less@H@std@@V?$allocator@U?$pair@$$CBHUgame_snd@@@std@@@3@$0A@@std@@@std@@QAE?AU?$pair@Viterator@?$_Tree@V?$_Tmap_traits@HUgame_snd@@U?$less@H@std@@V?$allocator@U?$pair@$$CBHUgame_snd@@@std@@@3@$0A@@std@@@std@@_N@2@ABU?$pair@$$CBHUgame_snd@@@2@@Z 1009bee0 f i scriptparser.obj
 0002:0002a320       ?allocate@?$_DebugHeapAllocator@D@std@@QAAPADIPBX@Z 1009c320 f i scriptparser.obj
 0002:0002a3c0       ?allocate@?$_DebugHeapAllocator@D@std@@QAEPADI@Z 1009c3c0 f i scriptparser.obj
 0002:0002a460       ?deallocate@?$_DebugHeapAllocator@D@std@@QAEXPADI@Z 1009c460 f i scriptparser.obj
 0002:0002a4a0       ?size@?$vector@V?$basic_string@DU?$char_traits@D@std@@V?$allocator@D@2@@std@@V?$allocator@V?$basic_string@DU?$char_traits@D@std@@V?$allocator@D@2@@std@@@2@@std@@QBEIXZ 1009c4a0 f i scriptparser.obj
 0002:0002a4d0       ??A?$vector@V?$basic_string@DU?$char_traits@D@std@@V?$allocator@D@2@@std@@V?$allocator@V?$basic_string@DU?$char_traits@D@std@@V?$allocator@D@2@@std@@@2@@std@@QAEAAV?$basic_string@DU?$char_traits@D@std@@V?$allocator@D@2@@1@I@Z 1009c4d0 f i scriptparser.obj
 0002:0002a5f0       ??0?$vector@UST_CELLS@@V?$allocator@UST_CELLS@@@std@@@std@@QAE@XZ 1009c5f0 f i scriptparser.obj
 0002:0002a690       ??1?$vector@UST_CELLS@@V?$allocator@UST_CELLS@@@std@@@std@@QAE@XZ 1009c690 f i scriptparser.obj
 0002:0002a710       ?size@?$vector@UST_CELLS@@V?$allocator@UST_CELLS@@@std@@@std@@QBEIXZ 1009c710 f i scriptparser.obj
 0002:0002a740       ??A?$vector@UST_CELLS@@V?$allocator@UST_CELLS@@@std@@@std@@QAEAAUST_CELLS@@I@Z 1009c740 f i scriptparser.obj
 0002:0002a860       ??0?$pair@$$CBHUgame_snd@@@std@@QAE@ABHABUgame_snd@@@Z 1009c860 f i scriptparser.obj
 0002:0002a8b0       ??4iterator@?$_Tree@V?$_Tmap_traits@HUgame_snd@@U?$less@H@std@@V?$allocator@U?$pair@$$CBHUgame_snd@@@std@@@3@$0A@@std@@@std@@QAEAAV012@ABV012@@Z 1009c8b0 f i scriptparser.obj
 0002:0002a8f0       ??0?$_DebugHeapAllocator@D@std@@QAE@XZ 1009c8f0 f i scriptparser.obj
 0002:0002a920       ??1?$_Vector_val@UST_CELLS@@V?$allocator@UST_CELLS@@@std@@@std@@QAE@XZ 1009c920 f i scriptparser.obj
 0002:0002a950       ??4const_iterator@?$_Tree@V?$_Tmap_traits@HUgame_snd@@U?$less@H@std@@V?$allocator@U?$pair@$$CBHUgame_snd@@@std@@@3@$0A@@std@@@std@@QAEAAV012@ABV012@@Z 1009c950 f i scriptparser.obj
 0002:0002a9a0       ??4?$_Bidit@U?$pair@$$CBHUgame_snd@@@std@@HPBU12@ABU12@@std@@QAEAAU01@ABU01@@Z 1009c9a0 f i scriptparser.obj
 0002:0002a9e0       ??4?$_Iterator_with_base@Ubidirectional_iterator_tag@std@@U?$pair@$$CBHUgame_snd@@@2@HPBU32@ABU32@V_Iterator_base@2@@std@@QAEAAU01@ABU01@@Z 1009c9e0 f i scriptparser.obj
 0002:0002aa20       ?assign@?$basic_string@DU?$char_traits@D@std@@V?$allocator@D@2@@std@@QAEAAV12@ABV12@@Z 1009ca20 f i scriptparser.obj
 0002:0002aa60       ?insert@?$_Tree@V?$_Tmap_traits@HUgame_snd@@U?$less@H@std@@V?$allocator@U?$pair@$$CBHUgame_snd@@@std@@@3@$0A@@std@@@std@@QAE?AViterator@12@Vconst_iterator@12@ABU?$pair@$$CBHUgame_snd@@@2@@Z 1009ca60 f i scriptparser.obj
 0002:0002b8d0       ?_Insert@?$_Tree@V?$_Tmap_traits@HUgame_snd@@U?$less@H@std@@V?$allocator@U?$pair@$$CBHUgame_snd@@@std@@@3@$0A@@std@@@std@@IAE?AViterator@12@_NPAU_Node@?$_Tree_nod@V?$_Tmap_traits@HUgame_snd@@U?$less@H@std@@V?$allocator@U?$pair@$$CBHUgame_snd@@@std@@@3@$0A@@std@@@2@ABU?$pair@$$CBHUgame_snd@@@2@@Z 1009d8d0 f i scriptparser.obj
 0002:0002bea0       ?_Buy@?$vector@UST_CELLS@@V?$allocator@UST_CELLS@@@std@@@std@@IAE_NI@Z 1009dea0 f i scriptparser.obj
 0002:0002bf60       ?_Tidy@?$vector@UST_CELLS@@V?$allocator@UST_CELLS@@@std@@@std@@IAEXXZ 1009df60 f i scriptparser.obj
 0002:0002c010       ??0?$_Vector_val@UST_CELLS@@V?$allocator@UST_CELLS@@@std@@@std@@IAE@V?$allocator@UST_CELLS@@@1@@Z 1009e010 f i scriptparser.obj
 0002:0002c080       ??1?$_Container_base_aux_alloc_empty@V?$allocator@UST_CELLS@@@std@@@std@@IAE@XZ 1009e080 f i scriptparser.obj
 0002:0002c0b0       ??0?$allocator@UST_CELLS@@@std@@QAE@XZ 1009e0b0 f i scriptparser.obj
 0002:0002c0d0       ??0?$pair@Viterator@?$_Tree@V?$_Tmap_traits@HUgame_snd@@U?$less@H@std@@V?$allocator@U?$pair@$$CBHUgame_snd@@@std@@@3@$0A@@std@@@std@@_N@std@@QAE@ABViterator@?$_Tree@V?$_Tmap_traits@HUgame_snd@@U?$less@H@std@@V?$allocator@U?$pair@$$CBHUgame_snd@@@std@@@3@$0A@@std@@@1@AB_N@Z 1009e0d0 f i scriptparser.obj
 0002:0002c120       ??Fiterator@?$_Tree@V?$_Tmap_traits@HUgame_snd@@U?$less@H@std@@V?$allocator@U?$pair@$$CBHUgame_snd@@@std@@@3@$0A@@std@@@std@@QAEAAV012@XZ 1009e120 f i scriptparser.obj
 0002:0002c150       ??0?$_DebugHeapAllocator@D@std@@QAE@ABV01@@Z 1009e150 f i scriptparser.obj
 0002:0002c190       ?_Color@?$_Tree@V?$_Tmap_traits@HUgame_snd@@U?$less@H@std@@V?$allocator@U?$pair@$$CBHUgame_snd@@@std@@@3@$0A@@std@@@std@@KAAADPAU_Node@?$_Tree_nod@V?$_Tmap_traits@HUgame_snd@@U?$less@H@std@@V?$allocator@U?$pair@$$CBHUgame_snd@@@std@@@3@$0A@@std@@@2@@Z 1009e190 f i scriptparser.obj
 0002:0002c1a0       ?size@?$_Tree@V?$_Tmap_traits@HUgame_snd@@U?$less@H@std@@V?$allocator@U?$pair@$$CBHUgame_snd@@@std@@@3@$0A@@std@@@std@@QBEIXZ 1009e1a0 f i scriptparser.obj
 0002:0002c1c0       ?max_size@?$_Tree@V?$_Tmap_traits@HUgame_snd@@U?$less@H@std@@V?$allocator@U?$pair@$$CBHUgame_snd@@@std@@@3@$0A@@std@@@std@@QBEIXZ 1009e1c0 f i scriptparser.obj
 0002:0002c1f0       ?_Lrotate@?$_Tree@V?$_Tmap_traits@HUgame_snd@@U?$less@H@std@@V?$allocator@U?$pair@$$CBHUgame_snd@@@std@@@3@$0A@@std@@@std@@IAEXPAU_Node@?$_Tree_nod@V?$_Tmap_traits@HUgame_snd@@U?$less@H@std@@V?$allocator@U?$pair@$$CBHUgame_snd@@@std@@@3@$0A@@std@@@2@@Z 1009e1f0 f i scriptparser.obj
 0002:0002c390       ?_Rrotate@?$_Tree@V?$_Tmap_traits@HUgame_snd@@U?$less@H@std@@V?$allocator@U?$pair@$$CBHUgame_snd@@@std@@@3@$0A@@std@@@std@@IAEXPAU_Node@?$_Tree_nod@V?$_Tmap_traits@HUgame_snd@@U?$less@H@std@@V?$allocator@U?$pair@$$CBHUgame_snd@@@std@@@3@$0A@@std@@@2@@Z 1009e390 f i scriptparser.obj
 0002:0002c530       ?_Buynode@?$_Tree@V?$_Tmap_traits@HUgame_snd@@U?$less@H@std@@V?$allocator@U?$pair@$$CBHUgame_snd@@@std@@@3@$0A@@std@@@std@@IAEPAU_Node@?$_Tree_nod@V?$_Tmap_traits@HUgame_snd@@U?$less@H@std@@V?$allocator@U?$pair@$$CBHUgame_snd@@@std@@@3@$0A@@std@@@2@PAU342@00ABU?$pair@$$CBHUgame_snd@@@2@D@Z 1009e530 f i scriptparser.obj
 0002:0002c680       ?max_size@?$vector@UST_CELLS@@V?$allocator@UST_CELLS@@@std@@@std@@QBEIXZ 1009e680 f i scriptparser.obj
 0002:0002c6b0       ?_Destroy@?$vector@UST_CELLS@@V?$allocator@UST_CELLS@@@std@@@std@@IAEXPAUST_CELLS@@0@Z 1009e6b0 f i scriptparser.obj
 0002:0002c700       ?_Xlen@?$vector@UST_CELLS@@V?$allocator@UST_CELLS@@@std@@@std@@KAXXZ 1009e700 f i scriptparser.obj
 0002:0002c7b0       ??0?$_Container_base_aux_alloc_empty@V?$allocator@UST_CELLS@@@std@@@std@@IAE@V?$allocator@UST_CELLS@@@1@@Z 1009e7b0 f i scriptparser.obj
 0002:0002c7f0       ??0?$allocator@UST_CELLS@@@std@@QAE@ABV01@@Z 1009e7f0 f i scriptparser.obj
 0002:0002c810       ?deallocate@?$allocator@UST_CELLS@@@std@@QAEXPAUST_CELLS@@I@Z 1009e810 f i scriptparser.obj
 0002:0002c850       ?allocate@?$allocator@UST_CELLS@@@std@@QAEPAUST_CELLS@@I@Z 1009e850 f i scriptparser.obj
 0002:0002c890       ??0const_iterator@?$_Tree@V?$_Tmap_traits@HUgame_snd@@U?$less@H@std@@V?$allocator@U?$pair@$$CBHUgame_snd@@@std@@@3@$0A@@std@@@std@@QAE@XZ 1009e890 f i scriptparser.obj
 0002:0002c8d0       ??Fconst_iterator@?$_Tree@V?$_Tmap_traits@HUgame_snd@@U?$less@H@std@@V?$allocator@U?$pair@$$CBHUgame_snd@@@std@@@3@$0A@@std@@@std@@QAEAAV012@XZ 1009e8d0 f i scriptparser.obj
 0002:0002c900       ?max_size@?$allocator@U?$pair@$$CBHUgame_snd@@@std@@@std@@QBEIXZ 1009e900 f i scriptparser.obj
 0002:0002c960       ?allocate@?$allocator@U_Node@?$_Tree_nod@V?$_Tmap_traits@HUgame_snd@@U?$less@H@std@@V?$allocator@U?$pair@$$CBHUgame_snd@@@std@@@3@$0A@@std@@@std@@@std@@QAEPAU_Node@?$_Tree_nod@V?$_Tmap_traits@HUgame_snd@@U?$less@H@std@@V?$allocator@U?$pair@$$CBHUgame_snd@@@std@@@3@$0A@@std@@@2@I@Z 1009e960 f i scriptparser.obj
 0002:0002c9a0       ?max_size@?$allocator@UST_CELLS@@@std@@QBEIXZ 1009e9a0 f i scriptparser.obj
 0002:0002ca00       ?_Dec@const_iterator@?$_Tree@V?$_Tmap_traits@HUgame_snd@@U?$less@H@std@@V?$allocator@U?$pair@$$CBHUgame_snd@@@std@@@3@$0A@@std@@@std@@QAEXXZ 1009ea00 f i scriptparser.obj
 0002:0002ccd0       ??0_Node@?$_Tree_nod@V?$_Tmap_traits@HUgame_snd@@U?$less@H@std@@V?$allocator@U?$pair@$$CBHUgame_snd@@@std@@@3@$0A@@std@@@std@@QAE@PAU012@00ABU?$pair@$$CBHUgame_snd@@@2@D@Z 1009ecd0 f i scriptparser.obj
 0002:0002cd50       ?_Max@?$_Tree@V?$_Tmap_traits@HUgame_snd@@U?$less@H@std@@V?$allocator@U?$pair@$$CBHUgame_snd@@@std@@@3@$0A@@std@@@std@@KAPAU_Node@?$_Tree_nod@V?$_Tmap_traits@HUgame_snd@@U?$less@H@std@@V?$allocator@U?$pair@$$CBHUgame_snd@@@std@@@3@$0A@@std@@@2@PAU342@@Z 1009ed50 f i scriptparser.obj
 0002:0002cda0       ??$?8DU?$char_traits@D@std@@V?$allocator@D@1@@std@@YA_NPBDABV?$basic_string@DU?$char_traits@D@std@@V?$allocator@D@2@@0@@Z 1009eda0 f i scriptparser.obj
 0002:0002cdd0       ?compare@?$basic_string@DU?$char_traits@D@std@@V?$allocator@D@2@@std@@QBEHPBD@Z 1009edd0 f i scriptparser.obj
 0002:0002ce40       ?compare@?$basic_string@DU?$char_traits@D@std@@V?$allocator@D@2@@std@@QBEHIIPBDI@Z 1009ee40 f i scriptparser.obj
 0002:0002cf60       ?compare@?$char_traits@D@std@@SAHPBD0I@Z 1009ef60 f i scriptparser.obj
 0002:0002cf90       ??$_DebugHeapDelete@X@std@@YAXPAX@Z 1009ef90 f i scriptparser.obj
 0002:0002cfc0       ??$_Destroy_range@V?$allocator@UST_CELLS@@@std@@@std@@YAXPAUST_CELLS@@0AAV?$allocator@UST_CELLS@@@0@@Z 1009efc0 f i scriptparser.obj
 0002:0002d020       ??$_Allocate@UST_CELLS@@@std@@YAPAUST_CELLS@@IPAU1@@Z 1009f020 f i scriptparser.obj
 0002:0002d0b0       ??$_Allocate@U_Node@?$_Tree_nod@V?$_Tmap_traits@HUgame_snd@@U?$less@H@std@@V?$allocator@U?$pair@$$CBHUgame_snd@@@std@@@3@$0A@@std@@@std@@@std@@YAPAU_Node@?$_Tree_nod@V?$_Tmap_traits@HUgame_snd@@U?$less@H@std@@V?$allocator@U?$pair@$$CBHUgame_snd@@@std@@@3@$0A@@std@@@0@IPAU120@@Z 1009f0b0 f i scriptparser.obj
 0002:0002d140       ??$_Ptr_cat@PAUST_CELLS@@PAU1@@std@@YA?AU_Nonscalar_ptr_iterator_tag@0@AAPAUST_CELLS@@0@Z 1009f140 f i scriptparser.obj
 0002:0002d1a0       ??$_Destroy_range@V?$allocator@UST_CELLS@@@std@@@std@@YAXPAUST_CELLS@@0AAV?$allocator@UST_CELLS@@@0@U_Nonscalar_ptr_iterator_tag@0@@Z 1009f1a0 f i scriptparser.obj
 0002:0002d1e0       ?destroy@?$allocator@UST_CELLS@@@std@@QAEXPAUST_CELLS@@@Z 1009f1e0 f i scriptparser.obj
 0002:0002d220       ??$_Destroy@UST_CELLS@@@std@@YAXPAUST_CELLS@@@Z 1009f220 f i scriptparser.obj
 0002:0002d240       ??_GST_CELLS@@QAEPAXI@Z    1009f240 f i scriptparser.obj
 0002:0002d290       ??1ST_CELLS@@QAE@XZ        1009f290 f i scriptparser.obj
 0002:0002d2c0       ??1?$vector@V?$basic_string@DU?$char_traits@D@std@@V?$allocator@D@2@@std@@V?$allocator@V?$basic_string@DU?$char_traits@D@std@@V?$allocator@D@2@@std@@@2@@std@@QAE@XZ 1009f2c0 f i scriptparser.obj
 0002:0002d340       ??1?$_Vector_val@V?$basic_string@DU?$char_traits@D@std@@V?$allocator@D@2@@std@@V?$allocator@V?$basic_string@DU?$char_traits@D@std@@V?$allocator@D@2@@std@@@2@@std@@QAE@XZ 1009f340 f i scriptparser.obj
 0002:0002d370       ?_Tidy@?$vector@V?$basic_string@DU?$char_traits@D@std@@V?$allocator@D@2@@std@@V?$allocator@V?$basic_string@DU?$char_traits@D@std@@V?$allocator@D@2@@std@@@2@@std@@IAEXXZ 1009f370 f i scriptparser.obj
 0002:0002d420       ??1?$_Container_base_aux_alloc_empty@V?$allocator@V?$basic_string@DU?$char_traits@D@std@@V?$allocator@D@2@@std@@@std@@@std@@IAE@XZ 1009f420 f i scriptparser.obj
 0002:0002d450       ?_Destroy@?$vector@V?$basic_string@DU?$char_traits@D@std@@V?$allocator@D@2@@std@@V?$allocator@V?$basic_string@DU?$char_traits@D@std@@V?$allocator@D@2@@std@@@2@@std@@IAEXPAV?$basic_string@DU?$char_traits@D@std@@V?$allocator@D@2@@2@0@Z 1009f450 f i scriptparser.obj
 0002:0002d4a0       ?deallocate@?$allocator@V?$basic_string@DU?$char_traits@D@std@@V?$allocator@D@2@@std@@@std@@QAEXPAV?$basic_string@DU?$char_traits@D@std@@V?$allocator@D@2@@2@I@Z 1009f4a0 f i scriptparser.obj
 0002:0002d4e0       ??$_Destroy_range@V?$allocator@V?$basic_string@DU?$char_traits@D@std@@V?$allocator@D@2@@std@@@std@@@std@@YAXPAV?$basic_string@DU?$char_traits@D@std@@V?$allocator@D@2@@0@0AAV?$allocator@V?$basic_string@DU?$char_traits@D@std@@V?$allocator@D@2@@std@@@0@@Z 1009f4e0 f i scriptparser.obj
 0002:0002d540       ??$_Ptr_cat@PAV?$basic_string@DU?$char_traits@D@std@@V?$allocator@D@2@@std@@PAV12@@std@@YA?AU_Nonscalar_ptr_iterator_tag@0@AAPAV?$basic_string@DU?$char_traits@D@std@@V?$allocator@D@2@@0@0@Z 1009f540 f i scriptparser.obj
 0002:0002d5a0       ??$_Destroy_range@V?$allocator@V?$basic_string@DU?$char_traits@D@std@@V?$allocator@D@2@@std@@@std@@@std@@YAXPAV?$basic_string@DU?$char_traits@D@std@@V?$allocator@D@2@@0@0AAV?$allocator@V?$basic_string@DU?$char_traits@D@std@@V?$allocator@D@2@@std@@@0@U_Nonscalar_ptr_iterator_tag@0@@Z 1009f5a0 f i scriptparser.obj
 0002:0002d5e0       ?destroy@?$allocator@V?$basic_string@DU?$char_traits@D@std@@V?$allocator@D@2@@std@@@std@@QAEXPAV?$basic_string@DU?$char_traits@D@std@@V?$allocator@D@2@@2@@Z 1009f5e0 f i scriptparser.obj
 0002:0002d620       ??$_Destroy@V?$basic_string@DU?$char_traits@D@std@@V?$allocator@D@2@@std@@@std@@YAXPAV?$basic_string@DU?$char_traits@D@std@@V?$allocator@D@2@@0@@Z 1009f620 f i scriptparser.obj
 0002:0002d640       ??_G?$basic_string@DU?$char_traits@D@std@@V?$allocator@D@2@@std@@QAEPAXI@Z 1009f640 f i scriptparser.obj
 0002:0002d690       ??0?$map@HUgame_snd@@U?$less@H@std@@V?$allocator@U?$pair@$$CBHUgame_snd@@@std@@@3@@std@@QAE@XZ 1009f690 f i scriptparser.obj
 0002:0002d6e0       ??0?$_Tree@V?$_Tmap_traits@HUgame_snd@@U?$less@H@std@@V?$allocator@U?$pair@$$CBHUgame_snd@@@std@@@3@$0A@@std@@@std@@QAE@ABU?$less@H@1@ABV?$allocator@U?$pair@$$CBHUgame_snd@@@std@@@1@@Z 1009f6e0 f i scriptparser.obj
 0002:0002d790       ??1?$_Tree_val@V?$_Tmap_traits@HUgame_snd@@U?$less@H@std@@V?$allocator@U?$pair@$$CBHUgame_snd@@@std@@@3@$0A@@std@@@std@@QAE@XZ 1009f790 f i scriptparser.obj
 0002:0002d7c0       ??1?$_Tree_ptr@V?$_Tmap_traits@HUgame_snd@@U?$less@H@std@@V?$allocator@U?$pair@$$CBHUgame_snd@@@std@@@3@$0A@@std@@@std@@QAE@XZ 1009f7c0 f i scriptparser.obj
 0002:0002d7f0       ??1?$_Tree_nod@V?$_Tmap_traits@HUgame_snd@@U?$less@H@std@@V?$allocator@U?$pair@$$CBHUgame_snd@@@std@@@3@$0A@@std@@@std@@QAE@XZ 1009f7f0 f i scriptparser.obj
 0002:0002d820       ??1?$_Tmap_traits@HUgame_snd@@U?$less@H@std@@V?$allocator@U?$pair@$$CBHUgame_snd@@@std@@@3@$0A@@std@@QAE@XZ 1009f820 f i scriptparser.obj
 0002:0002d850       ??1?$_Container_base_aux_alloc_empty@V?$allocator@U?$pair@$$CBHUgame_snd@@@std@@@std@@@std@@IAE@XZ 1009f850 f i scriptparser.obj
 0002:0002d880       ??0?$allocator@U?$pair@$$CBHUgame_snd@@@std@@@std@@QAE@XZ 1009f880 f i scriptparser.obj
 0002:0002d8a0       ?_Init@?$_Tree@V?$_Tmap_traits@HUgame_snd@@U?$less@H@std@@V?$allocator@U?$pair@$$CBHUgame_snd@@@std@@@3@$0A@@std@@@std@@IAEXXZ 1009f8a0 f i scriptparser.obj
 0002:0002d940       ??0?$_Tree_val@V?$_Tmap_traits@HUgame_snd@@U?$less@H@std@@V?$allocator@U?$pair@$$CBHUgame_snd@@@std@@@3@$0A@@std@@@std@@IAE@ABU?$less@H@1@V?$allocator@U?$pair@$$CBHUgame_snd@@@std@@@1@@Z 1009f940 f i scriptparser.obj
 0002:0002d9b0       ??0?$allocator@U?$pair@$$CBHUgame_snd@@@std@@@std@@QAE@ABV01@@Z 1009f9b0 f i scriptparser.obj
 0002:0002d9d0       ?_Buynode@?$_Tree@V?$_Tmap_traits@HUgame_snd@@U?$less@H@std@@V?$allocator@U?$pair@$$CBHUgame_snd@@@std@@@3@$0A@@std@@@std@@IAEPAU_Node@?$_Tree_nod@V?$_Tmap_traits@HUgame_snd@@U?$less@H@std@@V?$allocator@U?$pair@$$CBHUgame_snd@@@std@@@3@$0A@@std@@@2@XZ 1009f9d0 f i scriptparser.obj
 0002:0002dbe0       ?destroy@?$allocator@PAU_Node@?$_Tree_nod@V?$_Tmap_traits@HUgame_snd@@U?$less@H@std@@V?$allocator@U?$pair@$$CBHUgame_snd@@@std@@@3@$0A@@std@@@std@@@std@@QAEXPAPAU_Node@?$_Tree_nod@V?$_Tmap_traits@HUgame_snd@@U?$less@H@std@@V?$allocator@U?$pair@$$CBHUgame_snd@@@std@@@3@$0A@@std@@@2@@Z 1009fbe0 f i scriptparser.obj
 0002:0002dc20       ??0?$_Tree_ptr@V?$_Tmap_traits@HUgame_snd@@U?$less@H@std@@V?$allocator@U?$pair@$$CBHUgame_snd@@@std@@@3@$0A@@std@@@std@@QAE@ABU?$less@H@1@V?$allocator@U?$pair@$$CBHUgame_snd@@@std@@@1@@Z 1009fc20 f i scriptparser.obj
 0002:0002dc90       ??0?$_Tree_nod@V?$_Tmap_traits@HUgame_snd@@U?$less@H@std@@V?$allocator@U?$pair@$$CBHUgame_snd@@@std@@@3@$0A@@std@@@std@@IAE@ABU?$less@H@1@V?$allocator@U?$pair@$$CBHUgame_snd@@@std@@@1@@Z 1009fc90 f i scriptparser.obj
 0002:0002dd00       ?construct@?$allocator@PAU_Node@?$_Tree_nod@V?$_Tmap_traits@HUgame_snd@@U?$less@H@std@@V?$allocator@U?$pair@$$CBHUgame_snd@@@std@@@3@$0A@@std@@@std@@@std@@QAEXPAPAU_Node@?$_Tree_nod@V?$_Tmap_traits@HUgame_snd@@U?$less@H@std@@V?$allocator@U?$pair@$$CBHUgame_snd@@@std@@@3@$0A@@std@@@2@ABQAU342@@Z 1009fd00 f i scriptparser.obj
 0002:0002dd40       ??0?$_Tmap_traits@HUgame_snd@@U?$less@H@std@@V?$allocator@U?$pair@$$CBHUgame_snd@@@std@@@3@$0A@@std@@QAE@U?$less@H@1@V?$allocator@U?$pair@$$CBHUgame_snd@@@std@@@1@@Z 1009fd40 f i scriptparser.obj
 0002:0002dda0       ??0?$_Container_base_aux_alloc_empty@V?$allocator@U?$pair@$$CBHUgame_snd@@@std@@@std@@@std@@IAE@V?$allocator@U?$pair@$$CBHUgame_snd@@@std@@@1@@Z 1009fda0 f i scriptparser.obj
 0002:0002dde0       ??$_Destroy@PAU_Node@?$_Tree_nod@V?$_Tmap_traits@HUgame_snd@@U?$less@H@std@@V?$allocator@U?$pair@$$CBHUgame_snd@@@std@@@3@$0A@@std@@@std@@@std@@YAXPAPAU_Node@?$_Tree_nod@V?$_Tmap_traits@HUgame_snd@@U?$less@H@std@@V?$allocator@U?$pair@$$CBHUgame_snd@@@std@@@3@$0A@@std@@@0@@Z 1009fde0 f i scriptparser.obj
 0002:0002ddf0       ??$?0U?$pair@$$CBHUgame_snd@@@std@@@?$allocator@PAU_Node@?$_Tree_nod@V?$_Tmap_traits@HUgame_snd@@U?$less@H@std@@V?$allocator@U?$pair@$$CBHUgame_snd@@@std@@@3@$0A@@std@@@std@@@std@@QAE@ABV?$allocator@U?$pair@$$CBHUgame_snd@@@std@@@1@@Z 1009fdf0 f i scriptparser.obj
 0002:0002de10       ??$?0U?$pair@$$CBHUgame_snd@@@std@@@?$allocator@U_Node@?$_Tree_nod@V?$_Tmap_traits@HUgame_snd@@U?$less@H@std@@V?$allocator@U?$pair@$$CBHUgame_snd@@@std@@@3@$0A@@std@@@std@@@std@@QAE@ABV?$allocator@U?$pair@$$CBHUgame_snd@@@std@@@1@@Z 1009fe10 f i scriptparser.obj
 0002:0002de30       ??$_Construct@PAU_Node@?$_Tree_nod@V?$_Tmap_traits@HUgame_snd@@U?$less@H@std@@V?$allocator@U?$pair@$$CBHUgame_snd@@@std@@@3@$0A@@std@@@std@@PAU123@@std@@YAXPAPAU_Node@?$_Tree_nod@V?$_Tmap_traits@HUgame_snd@@U?$less@H@std@@V?$allocator@U?$pair@$$CBHUgame_snd@@@std@@@3@$0A@@std@@@0@ABQAU120@@Z 1009fe30 f i scriptparser.obj
 0002:0002deb0       ??0?$map@HUAmbientSnd@@U?$less@H@std@@V?$allocator@U?$pair@$$CBHUAmbientSnd@@@std@@@3@@std@@QAE@XZ 1009feb0 f i scriptparser.obj
 0002:0002df00       ??0?$_Tree@V?$_Tmap_traits@HUAmbientSnd@@U?$less@H@std@@V?$allocator@U?$pair@$$CBHUAmbientSnd@@@std@@@3@$0A@@std@@@std@@QAE@ABU?$less@H@1@ABV?$allocator@U?$pair@$$CBHUAmbientSnd@@@std@@@1@@Z 1009ff00 f i scriptparser.obj
 0002:0002dfb0       ??1?$_Tree_val@V?$_Tmap_traits@HUAmbientSnd@@U?$less@H@std@@V?$allocator@U?$pair@$$CBHUAmbientSnd@@@std@@@3@$0A@@std@@@std@@QAE@XZ 1009ffb0 f i scriptparser.obj
 0002:0002dfe0       ??1?$_Tree_ptr@V?$_Tmap_traits@HUAmbientSnd@@U?$less@H@std@@V?$allocator@U?$pair@$$CBHUAmbientSnd@@@std@@@3@$0A@@std@@@std@@QAE@XZ 1009ffe0 f i scriptparser.obj
 0002:0002e010       ??1?$_Tree_nod@V?$_Tmap_traits@HUAmbientSnd@@U?$less@H@std@@V?$allocator@U?$pair@$$CBHUAmbientSnd@@@std@@@3@$0A@@std@@@std@@QAE@XZ 100a0010 f i scriptparser.obj
 0002:0002e040       ??1?$_Tmap_traits@HUAmbientSnd@@U?$less@H@std@@V?$allocator@U?$pair@$$CBHUAmbientSnd@@@std@@@3@$0A@@std@@QAE@XZ 100a0040 f i scriptparser.obj
 0002:0002e070       ??1?$_Container_base_aux_alloc_empty@V?$allocator@U?$pair@$$CBHUAmbientSnd@@@std@@@std@@@std@@IAE@XZ 100a0070 f i scriptparser.obj
 0002:0002e0a0       ??0?$allocator@U?$pair@$$CBHUAmbientSnd@@@std@@@std@@QAE@XZ 100a00a0 f i scriptparser.obj
 0002:0002e0c0       ?_Init@?$_Tree@V?$_Tmap_traits@HUAmbientSnd@@U?$less@H@std@@V?$allocator@U?$pair@$$CBHUAmbientSnd@@@std@@@3@$0A@@std@@@std@@IAEXXZ 100a00c0 f i scriptparser.obj
 0002:0002e160       ??0?$_Tree_val@V?$_Tmap_traits@HUAmbientSnd@@U?$less@H@std@@V?$allocator@U?$pair@$$CBHUAmbientSnd@@@std@@@3@$0A@@std@@@std@@IAE@ABU?$less@H@1@V?$allocator@U?$pair@$$CBHUAmbientSnd@@@std@@@1@@Z 100a0160 f i scriptparser.obj
 0002:0002e1d0       ??0?$allocator@U?$pair@$$CBHUAmbientSnd@@@std@@@std@@QAE@ABV01@@Z 100a01d0 f i scriptparser.obj
 0002:0002e1f0       ?_Buynode@?$_Tree@V?$_Tmap_traits@HUAmbientSnd@@U?$less@H@std@@V?$allocator@U?$pair@$$CBHUAmbientSnd@@@std@@@3@$0A@@std@@@std@@IAEPAU_Node@?$_Tree_nod@V?$_Tmap_traits@HUAmbientSnd@@U?$less@H@std@@V?$allocator@U?$pair@$$CBHUAmbientSnd@@@std@@@3@$0A@@std@@@2@XZ 100a01f0 f i scriptparser.obj
 0002:0002e400       ?destroy@?$allocator@PAU_Node@?$_Tree_nod@V?$_Tmap_traits@HUAmbientSnd@@U?$less@H@std@@V?$allocator@U?$pair@$$CBHUAmbientSnd@@@std@@@3@$0A@@std@@@std@@@std@@QAEXPAPAU_Node@?$_Tree_nod@V?$_Tmap_traits@HUAmbientSnd@@U?$less@H@std@@V?$allocator@U?$pair@$$CBHUAmbientSnd@@@std@@@3@$0A@@std@@@2@@Z 100a0400 f i scriptparser.obj
 0002:0002e440       ??0?$_Tree_ptr@V?$_Tmap_traits@HUAmbientSnd@@U?$less@H@std@@V?$allocator@U?$pair@$$CBHUAmbientSnd@@@std@@@3@$0A@@std@@@std@@QAE@ABU?$less@H@1@V?$allocator@U?$pair@$$CBHUAmbientSnd@@@std@@@1@@Z 100a0440 f i scriptparser.obj
 0002:0002e4b0       ??0?$_Tree_nod@V?$_Tmap_traits@HUAmbientSnd@@U?$less@H@std@@V?$allocator@U?$pair@$$CBHUAmbientSnd@@@std@@@3@$0A@@std@@@std@@IAE@ABU?$less@H@1@V?$allocator@U?$pair@$$CBHUAmbientSnd@@@std@@@1@@Z 100a04b0 f i scriptparser.obj
 0002:0002e520       ?construct@?$allocator@PAU_Node@?$_Tree_nod@V?$_Tmap_traits@HUAmbientSnd@@U?$less@H@std@@V?$allocator@U?$pair@$$CBHUAmbientSnd@@@std@@@3@$0A@@std@@@std@@@std@@QAEXPAPAU_Node@?$_Tree_nod@V?$_Tmap_traits@HUAmbientSnd@@U?$less@H@std@@V?$allocator@U?$pair@$$CBHUAmbientSnd@@@std@@@3@$0A@@std@@@2@ABQAU342@@Z 100a0520 f i scriptparser.obj
 0002:0002e560       ??0?$_Tmap_traits@HUAmbientSnd@@U?$less@H@std@@V?$allocator@U?$pair@$$CBHUAmbientSnd@@@std@@@3@$0A@@std@@QAE@U?$less@H@1@V?$allocator@U?$pair@$$CBHUAmbientSnd@@@std@@@1@@Z 100a0560 f i scriptparser.obj
 0002:0002e5c0       ??0?$_Container_base_aux_alloc_empty@V?$allocator@U?$pair@$$CBHUAmbientSnd@@@std@@@std@@@std@@IAE@V?$allocator@U?$pair@$$CBHUAmbientSnd@@@std@@@1@@Z 100a05c0 f i scriptparser.obj
 0002:0002e600       ??$_Destroy@PAU_Node@?$_Tree_nod@V?$_Tmap_traits@HUAmbientSnd@@U?$less@H@std@@V?$allocator@U?$pair@$$CBHUAmbientSnd@@@std@@@3@$0A@@std@@@std@@@std@@YAXPAPAU_Node@?$_Tree_nod@V?$_Tmap_traits@HUAmbientSnd@@U?$less@H@std@@V?$allocator@U?$pair@$$CBHUAmbientSnd@@@std@@@3@$0A@@std@@@0@@Z 100a0600 f i scriptparser.obj
 0002:0002e610       ??$?0U?$pair@$$CBHUAmbientSnd@@@std@@@?$allocator@PAU_Node@?$_Tree_nod@V?$_Tmap_traits@HUAmbientSnd@@U?$less@H@std@@V?$allocator@U?$pair@$$CBHUAmbientSnd@@@std@@@3@$0A@@std@@@std@@@std@@QAE@ABV?$allocator@U?$pair@$$CBHUAmbientSnd@@@std@@@1@@Z 100a0610 f i scriptparser.obj
 0002:0002e630       ??$?0U?$pair@$$CBHUAmbientSnd@@@std@@@?$allocator@U_Node@?$_Tree_nod@V?$_Tmap_traits@HUAmbientSnd@@U?$less@H@std@@V?$allocator@U?$pair@$$CBHUAmbientSnd@@@std@@@3@$0A@@std@@@std@@@std@@QAE@ABV?$allocator@U?$pair@$$CBHUAmbientSnd@@@std@@@1@@Z 100a0630 f i scriptparser.obj
 0002:0002e650       ??$_Construct@PAU_Node@?$_Tree_nod@V?$_Tmap_traits@HUAmbientSnd@@U?$less@H@std@@V?$allocator@U?$pair@$$CBHUAmbientSnd@@@std@@@3@$0A@@std@@@std@@PAU123@@std@@YAXPAPAU_Node@?$_Tree_nod@V?$_Tmap_traits@HUAmbientSnd@@U?$less@H@std@@V?$allocator@U?$pair@$$CBHUAmbientSnd@@@std@@@3@$0A@@std@@@0@ABQAU120@@Z 100a0650 f i scriptparser.obj
 0002:0002e6d0       ??0?$map@HUVoiceSnd@@U?$less@H@std@@V?$allocator@U?$pair@$$CBHUVoiceSnd@@@std@@@3@@std@@QAE@XZ 100a06d0 f i scriptparser.obj
 0002:0002e720       ??0?$_Tree@V?$_Tmap_traits@HUVoiceSnd@@U?$less@H@std@@V?$allocator@U?$pair@$$CBHUVoiceSnd@@@std@@@3@$0A@@std@@@std@@QAE@ABU?$less@H@1@ABV?$allocator@U?$pair@$$CBHUVoiceSnd@@@std@@@1@@Z 100a0720 f i scriptparser.obj
 0002:0002e7d0       ??1?$_Tree_val@V?$_Tmap_traits@HUVoiceSnd@@U?$less@H@std@@V?$allocator@U?$pair@$$CBHUVoiceSnd@@@std@@@3@$0A@@std@@@std@@QAE@XZ 100a07d0 f i scriptparser.obj
 0002:0002e800       ??1?$_Tree_ptr@V?$_Tmap_traits@HUVoiceSnd@@U?$less@H@std@@V?$allocator@U?$pair@$$CBHUVoiceSnd@@@std@@@3@$0A@@std@@@std@@QAE@XZ 100a0800 f i scriptparser.obj
 0002:0002e830       ??1?$_Tree_nod@V?$_Tmap_traits@HUVoiceSnd@@U?$less@H@std@@V?$allocator@U?$pair@$$CBHUVoiceSnd@@@std@@@3@$0A@@std@@@std@@QAE@XZ 100a0830 f i scriptparser.obj
 0002:0002e860       ??1?$_Tmap_traits@HUVoiceSnd@@U?$less@H@std@@V?$allocator@U?$pair@$$CBHUVoiceSnd@@@std@@@3@$0A@@std@@QAE@XZ 100a0860 f i scriptparser.obj
 0002:0002e890       ??1?$_Container_base_aux_alloc_empty@V?$allocator@U?$pair@$$CBHUVoiceSnd@@@std@@@std@@@std@@IAE@XZ 100a0890 f i scriptparser.obj
 0002:0002e8c0       ??0?$allocator@U?$pair@$$CBHUVoiceSnd@@@std@@@std@@QAE@XZ 100a08c0 f i scriptparser.obj
 0002:0002e8e0       ?_Init@?$_Tree@V?$_Tmap_traits@HUVoiceSnd@@U?$less@H@std@@V?$allocator@U?$pair@$$CBHUVoiceSnd@@@std@@@3@$0A@@std@@@std@@IAEXXZ 100a08e0 f i scriptparser.obj
 0002:0002e980       ??0?$_Tree_val@V?$_Tmap_traits@HUVoiceSnd@@U?$less@H@std@@V?$allocator@U?$pair@$$CBHUVoiceSnd@@@std@@@3@$0A@@std@@@std@@IAE@ABU?$less@H@1@V?$allocator@U?$pair@$$CBHUVoiceSnd@@@std@@@1@@Z 100a0980 f i scriptparser.obj
 0002:0002e9f0       ??0?$allocator@U?$pair@$$CBHUVoiceSnd@@@std@@@std@@QAE@ABV01@@Z 100a09f0 f i scriptparser.obj
 0002:0002ea10       ?_Isnil@?$_Tree@V?$_Tmap_traits@HUVoiceSnd@@U?$less@H@std@@V?$allocator@U?$pair@$$CBHUVoiceSnd@@@std@@@3@$0A@@std@@@std@@KAAADPAU_Node@?$_Tree_nod@V?$_Tmap_traits@HUVoiceSnd@@U?$less@H@std@@V?$allocator@U?$pair@$$CBHUVoiceSnd@@@std@@@3@$0A@@std@@@2@@Z 100a0a10 f i scriptparser.obj
 0002:0002ea20       ?_Lmost@?$_Tree@V?$_Tmap_traits@HUVoiceSnd@@U?$less@H@std@@V?$allocator@U?$pair@$$CBHUVoiceSnd@@@std@@@3@$0A@@std@@@std@@IBEAAPAU_Node@?$_Tree_nod@V?$_Tmap_traits@HUVoiceSnd@@U?$less@H@std@@V?$allocator@U?$pair@$$CBHUVoiceSnd@@@std@@@3@$0A@@std@@@2@XZ 100a0a20 f i scriptparser.obj
 0002:0002ea60       ?_Left@?$_Tree@V?$_Tmap_traits@HUVoiceSnd@@U?$less@H@std@@V?$allocator@U?$pair@$$CBHUVoiceSnd@@@std@@@3@$0A@@std@@@std@@KAAAPAU_Node@?$_Tree_nod@V?$_Tmap_traits@HUVoiceSnd@@U?$less@H@std@@V?$allocator@U?$pair@$$CBHUVoiceSnd@@@std@@@3@$0A@@std@@@2@PAU342@@Z 100a0a60 f i scriptparser.obj
 0002:0002ea70       ?_Rmost@?$_Tree@V?$_Tmap_traits@HUVoiceSnd@@U?$less@H@std@@V?$allocator@U?$pair@$$CBHUVoiceSnd@@@std@@@3@$0A@@std@@@std@@IBEAAPAU_Node@?$_Tree_nod@V?$_Tmap_traits@HUVoiceSnd@@U?$less@H@std@@V?$allocator@U?$pair@$$CBHUVoiceSnd@@@std@@@3@$0A@@std@@@2@XZ 100a0a70 f i scriptparser.obj
 0002:0002eab0       ?_Right@?$_Tree@V?$_Tmap_traits@HUVoiceSnd@@U?$less@H@std@@V?$allocator@U?$pair@$$CBHUVoiceSnd@@@std@@@3@$0A@@std@@@std@@KAAAPAU_Node@?$_Tree_nod@V?$_Tmap_traits@HUVoiceSnd@@U?$less@H@std@@V?$allocator@U?$pair@$$CBHUVoiceSnd@@@std@@@3@$0A@@std@@@2@PAU342@@Z 100a0ab0 f i scriptparser.obj
 0002:0002eac0       ?_Root@?$_Tree@V?$_Tmap_traits@HUVoiceSnd@@U?$less@H@std@@V?$allocator@U?$pair@$$CBHUVoiceSnd@@@std@@@3@$0A@@std@@@std@@IBEAAPAU_Node@?$_Tree_nod@V?$_Tmap_traits@HUVoiceSnd@@U?$less@H@std@@V?$allocator@U?$pair@$$CBHUVoiceSnd@@@std@@@3@$0A@@std@@@2@XZ 100a0ac0 f i scriptparser.obj
 0002:0002eb00       ?_Parent@?$_Tree@V?$_Tmap_traits@HUVoiceSnd@@U?$less@H@std@@V?$allocator@U?$pair@$$CBHUVoiceSnd@@@std@@@3@$0A@@std@@@std@@KAAAPAU_Node@?$_Tree_nod@V?$_Tmap_traits@HUVoiceSnd@@U?$less@H@std@@V?$allocator@U?$pair@$$CBHUVoiceSnd@@@std@@@3@$0A@@std@@@2@PAU342@@Z 100a0b00 f i scriptparser.obj
 0002:0002eb10       ?_Buynode@?$_Tree@V?$_Tmap_traits@HUVoiceSnd@@U?$less@H@std@@V?$allocator@U?$pair@$$CBHUVoiceSnd@@@std@@@3@$0A@@std@@@std@@IAEPAU_Node@?$_Tree_nod@V?$_Tmap_traits@HUVoiceSnd@@U?$less@H@std@@V?$allocator@U?$pair@$$CBHUVoiceSnd@@@std@@@3@$0A@@std@@@2@XZ 100a0b10 f i scriptparser.obj
 0002:0002ed20       ?deallocate@?$allocator@U_Node@?$_Tree_nod@V?$_Tmap_traits@HUVoiceSnd@@U?$less@H@std@@V?$allocator@U?$pair@$$CBHUVoiceSnd@@@std@@@3@$0A@@std@@@std@@@std@@QAEXPAU_Node@?$_Tree_nod@V?$_Tmap_traits@HUVoiceSnd@@U?$less@H@std@@V?$allocator@U?$pair@$$CBHUVoiceSnd@@@std@@@3@$0A@@std@@@2@I@Z 100a0d20 f i scriptparser.obj
 0002:0002ed60       ?destroy@?$allocator@PAU_Node@?$_Tree_nod@V?$_Tmap_traits@HUVoiceSnd@@U?$less@H@std@@V?$allocator@U?$pair@$$CBHUVoiceSnd@@@std@@@3@$0A@@std@@@std@@@std@@QAEXPAPAU_Node@?$_Tree_nod@V?$_Tmap_traits@HUVoiceSnd@@U?$less@H@std@@V?$allocator@U?$pair@$$CBHUVoiceSnd@@@std@@@3@$0A@@std@@@2@@Z 100a0d60 f i scriptparser.obj
 0002:0002eda0       ??0?$_Tree_ptr@V?$_Tmap_traits@HUVoiceSnd@@U?$less@H@std@@V?$allocator@U?$pair@$$CBHUVoiceSnd@@@std@@@3@$0A@@std@@@std@@QAE@ABU?$less@H@1@V?$allocator@U?$pair@$$CBHUVoiceSnd@@@std@@@1@@Z 100a0da0 f i scriptparser.obj
 0002:0002ee10       ?_Color@?$_Tree@V?$_Tmap_traits@HUVoiceSnd@@U?$less@H@std@@V?$allocator@U?$pair@$$CBHUVoiceSnd@@@std@@@3@$0A@@std@@@std@@KAAADPAU_Node@?$_Tree_nod@V?$_Tmap_traits@HUVoiceSnd@@U?$less@H@std@@V?$allocator@U?$pair@$$CBHUVoiceSnd@@@std@@@3@$0A@@std@@@2@@Z 100a0e10 f i scriptparser.obj
 0002:0002ee20       ??0?$_Tree_nod@V?$_Tmap_traits@HUVoiceSnd@@U?$less@H@std@@V?$allocator@U?$pair@$$CBHUVoiceSnd@@@std@@@3@$0A@@std@@@std@@IAE@ABU?$less@H@1@V?$allocator@U?$pair@$$CBHUVoiceSnd@@@std@@@1@@Z 100a0e20 f i scriptparser.obj
 0002:0002ee90       ?allocate@?$allocator@U_Node@?$_Tree_nod@V?$_Tmap_traits@HUVoiceSnd@@U?$less@H@std@@V?$allocator@U?$pair@$$CBHUVoiceSnd@@@std@@@3@$0A@@std@@@std@@@std@@QAEPAU_Node@?$_Tree_nod@V?$_Tmap_traits@HUVoiceSnd@@U?$less@H@std@@V?$allocator@U?$pair@$$CBHUVoiceSnd@@@std@@@3@$0A@@std@@@2@I@Z 100a0e90 f i scriptparser.obj
 0002:0002eed0       ?construct@?$allocator@PAU_Node@?$_Tree_nod@V?$_Tmap_traits@HUVoiceSnd@@U?$less@H@std@@V?$allocator@U?$pair@$$CBHUVoiceSnd@@@std@@@3@$0A@@std@@@std@@@std@@QAEXPAPAU_Node@?$_Tree_nod@V?$_Tmap_traits@HUVoiceSnd@@U?$less@H@std@@V?$allocator@U?$pair@$$CBHUVoiceSnd@@@std@@@3@$0A@@std@@@2@ABQAU342@@Z 100a0ed0 f i scriptparser.obj
 0002:0002ef10       ??0?$_Tmap_traits@HUVoiceSnd@@U?$less@H@std@@V?$allocator@U?$pair@$$CBHUVoiceSnd@@@std@@@3@$0A@@std@@QAE@U?$less@H@1@V?$allocator@U?$pair@$$CBHUVoiceSnd@@@std@@@1@@Z 100a0f10 f i scriptparser.obj
 0002:0002ef70       ??0?$_Container_base_aux_alloc_empty@V?$allocator@U?$pair@$$CBHUVoiceSnd@@@std@@@std@@@std@@IAE@V?$allocator@U?$pair@$$CBHUVoiceSnd@@@std@@@1@@Z 100a0f70 f i scriptparser.obj
 0002:0002efb0       ??$_Destroy@PAU_Node@?$_Tree_nod@V?$_Tmap_traits@HUVoiceSnd@@U?$less@H@std@@V?$allocator@U?$pair@$$CBHUVoiceSnd@@@std@@@3@$0A@@std@@@std@@@std@@YAXPAPAU_Node@?$_Tree_nod@V?$_Tmap_traits@HUVoiceSnd@@U?$less@H@std@@V?$allocator@U?$pair@$$CBHUVoiceSnd@@@std@@@3@$0A@@std@@@0@@Z 100a0fb0 f i scriptparser.obj
 0002:0002efc0       ??$?0U?$pair@$$CBHUVoiceSnd@@@std@@@?$allocator@PAU_Node@?$_Tree_nod@V?$_Tmap_traits@HUVoiceSnd@@U?$less@H@std@@V?$allocator@U?$pair@$$CBHUVoiceSnd@@@std@@@3@$0A@@std@@@std@@@std@@QAE@ABV?$allocator@U?$pair@$$CBHUVoiceSnd@@@std@@@1@@Z 100a0fc0 f i scriptparser.obj
 0002:0002efe0       ??$?0U?$pair@$$CBHUVoiceSnd@@@std@@@?$allocator@U_Node@?$_Tree_nod@V?$_Tmap_traits@HUVoiceSnd@@U?$less@H@std@@V?$allocator@U?$pair@$$CBHUVoiceSnd@@@std@@@3@$0A@@std@@@std@@@std@@QAE@ABV?$allocator@U?$pair@$$CBHUVoiceSnd@@@std@@@1@@Z 100a0fe0 f i scriptparser.obj
 0002:0002f000       ??$_Allocate@U_Node@?$_Tree_nod@V?$_Tmap_traits@HUVoiceSnd@@U?$less@H@std@@V?$allocator@U?$pair@$$CBHUVoiceSnd@@@std@@@3@$0A@@std@@@std@@@std@@YAPAU_Node@?$_Tree_nod@V?$_Tmap_traits@HUVoiceSnd@@U?$less@H@std@@V?$allocator@U?$pair@$$CBHUVoiceSnd@@@std@@@3@$0A@@std@@@0@IPAU120@@Z 100a1000 f i scriptparser.obj
 0002:0002f090       ??$_Construct@PAU_Node@?$_Tree_nod@V?$_Tmap_traits@HUVoiceSnd@@U?$less@H@std@@V?$allocator@U?$pair@$$CBHUVoiceSnd@@@std@@@3@$0A@@std@@@std@@PAU123@@std@@YAXPAPAU_Node@?$_Tree_nod@V?$_Tmap_traits@HUVoiceSnd@@U?$less@H@std@@V?$allocator@U?$pair@$$CBHUVoiceSnd@@@std@@@3@$0A@@std@@@0@ABQAU120@@Z 100a1090 f i scriptparser.obj
 0002:0002f110       ??1?$map@HUgame_snd@@U?$less@H@std@@V?$allocator@U?$pair@$$CBHUgame_snd@@@std@@@3@@std@@QAE@XZ 100a1110 f i scriptparser.obj
 0002:0002f140       ??1?$_Tree@V?$_Tmap_traits@HUgame_snd@@U?$less@H@std@@V?$allocator@U?$pair@$$CBHUgame_snd@@@std@@@3@$0A@@std@@@std@@QAE@XZ 100a1140 f i scriptparser.obj
 0002:0002f1c0       ?_Tidy@?$_Tree@V?$_Tmap_traits@HUgame_snd@@U?$less@H@std@@V?$allocator@U?$pair@$$CBHUgame_snd@@@std@@@3@$0A@@std@@@std@@IAEXXZ 100a11c0 f i scriptparser.obj
 0002:0002f390       ?erase@?$_Tree@V?$_Tmap_traits@HUgame_snd@@U?$less@H@std@@V?$allocator@U?$pair@$$CBHUgame_snd@@@std@@@3@$0A@@std@@@std@@QAE?AViterator@12@Vconst_iterator@12@0@Z 100a1390 f i scriptparser.obj
 0002:0002f620       ?_Make_iter@?$_Tree@V?$_Tmap_traits@HUgame_snd@@U?$less@H@std@@V?$allocator@U?$pair@$$CBHUgame_snd@@@std@@@3@$0A@@std@@@std@@QBE?AViterator@12@Vconst_iterator@12@@Z 100a1620 f i scriptparser.obj
 0002:0002f710       ?erase@?$_Tree@V?$_Tmap_traits@HUgame_snd@@U?$less@H@std@@V?$allocator@U?$pair@$$CBHUgame_snd@@@std@@@3@$0A@@std@@@std@@QAE?AViterator@12@Vconst_iterator@12@@Z 100a1710 f i scriptparser.obj
 0002:00030130       ??Econst_iterator@?$_Tree@V?$_Tmap_traits@HUgame_snd@@U?$less@H@std@@V?$allocator@U?$pair@$$CBHUgame_snd@@@std@@@3@$0A@@std@@@std@@QAE?AV012@H@Z 100a2130 f i scriptparser.obj
 0002:00030230       ??1?$map@HUAmbientSnd@@U?$less@H@std@@V?$allocator@U?$pair@$$CBHUAmbientSnd@@@std@@@3@@std@@QAE@XZ 100a2230 f i scriptparser.obj
 0002:00030260       ??1?$_Tree@V?$_Tmap_traits@HUAmbientSnd@@U?$less@H@std@@V?$allocator@U?$pair@$$CBHUAmbientSnd@@@std@@@3@$0A@@std@@@std@@QAE@XZ 100a2260 f i scriptparser.obj
 0002:000302e0       ?_Tidy@?$_Tree@V?$_Tmap_traits@HUAmbientSnd@@U?$less@H@std@@V?$allocator@U?$pair@$$CBHUAmbientSnd@@@std@@@3@$0A@@std@@@std@@IAEXXZ 100a22e0 f i scriptparser.obj
 0002:000304b0       ?erase@?$_Tree@V?$_Tmap_traits@HUAmbientSnd@@U?$less@H@std@@V?$allocator@U?$pair@$$CBHUAmbientSnd@@@std@@@3@$0A@@std@@@std@@QAE?AViterator@12@Vconst_iterator@12@0@Z 100a24b0 f i scriptparser.obj
 0002:00030740       ?_Make_iter@?$_Tree@V?$_Tmap_traits@HUAmbientSnd@@U?$less@H@std@@V?$allocator@U?$pair@$$CBHUAmbientSnd@@@std@@@3@$0A@@std@@@std@@QBE?AViterator@12@Vconst_iterator@12@@Z 100a2740 f i scriptparser.obj
 0002:00030830       ?erase@?$_Tree@V?$_Tmap_traits@HUAmbientSnd@@U?$less@H@std@@V?$allocator@U?$pair@$$CBHUAmbientSnd@@@std@@@3@$0A@@std@@@std@@QAE?AViterator@12@Vconst_iterator@12@@Z 100a2830 f i scriptparser.obj
 0002:00031250       ?clear@?$_Tree@V?$_Tmap_traits@HUAmbientSnd@@U?$less@H@std@@V?$allocator@U?$pair@$$CBHUAmbientSnd@@@std@@@3@$0A@@std@@@std@@QAEXXZ 100a3250 f i scriptparser.obj
 0002:000312f0       ??Econst_iterator@?$_Tree@V?$_Tmap_traits@HUAmbientSnd@@U?$less@H@std@@V?$allocator@U?$pair@$$CBHUAmbientSnd@@@std@@@3@$0A@@std@@@std@@QAE?AV012@H@Z 100a32f0 f i scriptparser.obj
 0002:000313f0       ??9const_iterator@?$_Tree@V?$_Tmap_traits@HUAmbientSnd@@U?$less@H@std@@V?$allocator@U?$pair@$$CBHUAmbientSnd@@@std@@@3@$0A@@std@@@std@@QBE_NABV012@@Z 100a33f0 f i scriptparser.obj
 0002:00031440       ?_Erase@?$_Tree@V?$_Tmap_traits@HUAmbientSnd@@U?$less@H@std@@V?$allocator@U?$pair@$$CBHUAmbientSnd@@@std@@@3@$0A@@std@@@std@@IAEXPAU_Node@?$_Tree_nod@V?$_Tmap_traits@HUAmbientSnd@@U?$less@H@std@@V?$allocator@U?$pair@$$CBHUAmbientSnd@@@std@@@3@$0A@@std@@@2@@Z 100a3440 f i scriptparser.obj
 0002:00031500       ?_Orphan_ptr@?$_Tree@V?$_Tmap_traits@HUAmbientSnd@@U?$less@H@std@@V?$allocator@U?$pair@$$CBHUAmbientSnd@@@std@@@3@$0A@@std@@@std@@IBEXAAV12@PAU_Node@?$_Tree_nod@V?$_Tmap_traits@HUAmbientSnd@@U?$less@H@std@@V?$allocator@U?$pair@$$CBHUAmbientSnd@@@std@@@3@$0A@@std@@@2@@Z 100a3500 f i scriptparser.obj
 0002:00031600       ?destroy@?$allocator@U_Node@?$_Tree_nod@V?$_Tmap_traits@HUAmbientSnd@@U?$less@H@std@@V?$allocator@U?$pair@$$CBHUAmbientSnd@@@std@@@3@$0A@@std@@@std@@@std@@QAEXPAU_Node@?$_Tree_nod@V?$_Tmap_traits@HUAmbientSnd@@U?$less@H@std@@V?$allocator@U?$pair@$$CBHUAmbientSnd@@@std@@@3@$0A@@std@@@2@@Z 100a3600 f i scriptparser.obj
 0002:00031640       ??$_Destroy@U_Node@?$_Tree_nod@V?$_Tmap_traits@HUAmbientSnd@@U?$less@H@std@@V?$allocator@U?$pair@$$CBHUAmbientSnd@@@std@@@3@$0A@@std@@@std@@@std@@YAXPAU_Node@?$_Tree_nod@V?$_Tmap_traits@HUAmbientSnd@@U?$less@H@std@@V?$allocator@U?$pair@$$CBHUAmbientSnd@@@std@@@3@$0A@@std@@@0@@Z 100a3640 f i scriptparser.obj
 0002:00031650       ??1?$map@HUVoiceSnd@@U?$less@H@std@@V?$allocator@U?$pair@$$CBHUVoiceSnd@@@std@@@3@@std@@QAE@XZ 100a3650 f i scriptparser.obj
 0002:00031680       ??1?$_Tree@V?$_Tmap_traits@HUVoiceSnd@@U?$less@H@std@@V?$allocator@U?$pair@$$CBHUVoiceSnd@@@std@@@3@$0A@@std@@@std@@QAE@XZ 100a3680 f i scriptparser.obj
 0002:00031700       ?_Tidy@?$_Tree@V?$_Tmap_traits@HUVoiceSnd@@U?$less@H@std@@V?$allocator@U?$pair@$$CBHUVoiceSnd@@@std@@@3@$0A@@std@@@std@@IAEXXZ 100a3700 f i scriptparser.obj
 0002:000318d0       ??1iterator@?$_Tree@V?$_Tmap_traits@HUVoiceSnd@@U?$less@H@std@@V?$allocator@U?$pair@$$CBHUVoiceSnd@@@std@@@3@$0A@@std@@@std@@QAE@XZ 100a38d0 f i scriptparser.obj
 0002:00031900       ??0const_iterator@?$_Tree@V?$_Tmap_traits@HUVoiceSnd@@U?$less@H@std@@V?$allocator@U?$pair@$$CBHUVoiceSnd@@@std@@@3@$0A@@std@@@std@@QAE@ABV012@@Z 100a3900 f i scriptparser.obj
 0002:00031950       ??1const_iterator@?$_Tree@V?$_Tmap_traits@HUVoiceSnd@@U?$less@H@std@@V?$allocator@U?$pair@$$CBHUVoiceSnd@@@std@@@3@$0A@@std@@@std@@QAE@XZ 100a3950 f i scriptparser.obj
 0002:00031980       ??0?$_Bidit@U?$pair@$$CBHUVoiceSnd@@@std@@HPBU12@ABU12@@std@@QAE@ABU01@@Z 100a3980 f i scriptparser.obj
 0002:000319c0       ??1?$_Bidit@U?$pair@$$CBHUVoiceSnd@@@std@@HPBU12@ABU12@@std@@QAE@XZ 100a39c0 f i scriptparser.obj
 0002:000319f0       ??0?$_Iterator_with_base@Ubidirectional_iterator_tag@std@@U?$pair@$$CBHUVoiceSnd@@@2@HPBU32@ABU32@V_Iterator_base@2@@std@@QAE@ABU01@@Z 100a39f0 f i scriptparser.obj
 0002:00031a30       ??1?$_Iterator_with_base@Ubidirectional_iterator_tag@std@@U?$pair@$$CBHUVoiceSnd@@@2@HPBU32@ABU32@V_Iterator_base@2@@std@@QAE@XZ 100a3a30 f i scriptparser.obj
 0002:00031a60       ?begin@?$_Tree@V?$_Tmap_traits@HUVoiceSnd@@U?$less@H@std@@V?$allocator@U?$pair@$$CBHUVoiceSnd@@@std@@@3@$0A@@std@@@std@@QAE?AViterator@12@XZ 100a3a60 f i scriptparser.obj
 0002:00031ad0       ?end@?$_Tree@V?$_Tmap_traits@HUVoiceSnd@@U?$less@H@std@@V?$allocator@U?$pair@$$CBHUVoiceSnd@@@std@@@3@$0A@@std@@@std@@QAE?AViterator@12@XZ 100a3ad0 f i scriptparser.obj
 0002:00031b30       ?erase@?$_Tree@V?$_Tmap_traits@HUVoiceSnd@@U?$less@H@std@@V?$allocator@U?$pair@$$CBHUVoiceSnd@@@std@@@3@$0A@@std@@@std@@QAE?AViterator@12@Vconst_iterator@12@0@Z 100a3b30 f i scriptparser.obj
 0002:00031dc0       ?_Make_iter@?$_Tree@V?$_Tmap_traits@HUVoiceSnd@@U?$less@H@std@@V?$allocator@U?$pair@$$CBHUVoiceSnd@@@std@@@3@$0A@@std@@@std@@QBE?AViterator@12@Vconst_iterator@12@@Z 100a3dc0 f i scriptparser.obj
 0002:00031eb0       ?erase@?$_Tree@V?$_Tmap_traits@HUVoiceSnd@@U?$less@H@std@@V?$allocator@U?$pair@$$CBHUVoiceSnd@@@std@@@3@$0A@@std@@@std@@QAE?AViterator@12@Vconst_iterator@12@@Z 100a3eb0 f i scriptparser.obj
 0002:000328d0       ?clear@?$_Tree@V?$_Tmap_traits@HUVoiceSnd@@U?$less@H@std@@V?$allocator@U?$pair@$$CBHUVoiceSnd@@@std@@@3@$0A@@std@@@std@@QAEXXZ 100a48d0 f i scriptparser.obj
 0002:00032970       ??0iterator@?$_Tree@V?$_Tmap_traits@HUVoiceSnd@@U?$less@H@std@@V?$allocator@U?$pair@$$CBHUVoiceSnd@@@std@@@3@$0A@@std@@@std@@QAE@PAU_Node@?$_Tree_nod@V?$_Tmap_traits@HUVoiceSnd@@U?$less@H@std@@V?$allocator@U?$pair@$$CBHUVoiceSnd@@@std@@@3@$0A@@std@@@2@PBV12@@Z 100a4970 f i scriptparser.obj
 0002:000329b0       ??Econst_iterator@?$_Tree@V?$_Tmap_traits@HUVoiceSnd@@U?$less@H@std@@V?$allocator@U?$pair@$$CBHUVoiceSnd@@@std@@@3@$0A@@std@@@std@@QAE?AV012@H@Z 100a49b0 f i scriptparser.obj
 0002:00032ab0       ??8const_iterator@?$_Tree@V?$_Tmap_traits@HUVoiceSnd@@U?$less@H@std@@V?$allocator@U?$pair@$$CBHUVoiceSnd@@@std@@@3@$0A@@std@@@std@@QBE_NABV012@@Z 100a4ab0 f i scriptparser.obj
 0002:00032b80       ??9const_iterator@?$_Tree@V?$_Tmap_traits@HUVoiceSnd@@U?$less@H@std@@V?$allocator@U?$pair@$$CBHUVoiceSnd@@@std@@@3@$0A@@std@@@std@@QBE_NABV012@@Z 100a4b80 f i scriptparser.obj
 0002:00032bd0       ??0iterator@?$_Tree@V?$_Tmap_traits@HUVoiceSnd@@U?$less@H@std@@V?$allocator@U?$pair@$$CBHUVoiceSnd@@@std@@@3@$0A@@std@@@std@@QAE@ABV012@@Z 100a4bd0 f i scriptparser.obj
 0002:00032c10       ?_Erase@?$_Tree@V?$_Tmap_traits@HUVoiceSnd@@U?$less@H@std@@V?$allocator@U?$pair@$$CBHUVoiceSnd@@@std@@@3@$0A@@std@@@std@@IAEXPAU_Node@?$_Tree_nod@V?$_Tmap_traits@HUVoiceSnd@@U?$less@H@std@@V?$allocator@U?$pair@$$CBHUVoiceSnd@@@std@@@3@$0A@@std@@@2@@Z 100a4c10 f i scriptparser.obj
 0002:00032cd0       ?_Lrotate@?$_Tree@V?$_Tmap_traits@HUVoiceSnd@@U?$less@H@std@@V?$allocator@U?$pair@$$CBHUVoiceSnd@@@std@@@3@$0A@@std@@@std@@IAEXPAU_Node@?$_Tree_nod@V?$_Tmap_traits@HUVoiceSnd@@U?$less@H@std@@V?$allocator@U?$pair@$$CBHUVoiceSnd@@@std@@@3@$0A@@std@@@2@@Z 100a4cd0 f i scriptparser.obj
 0002:00032e70       ?_Max@?$_Tree@V?$_Tmap_traits@HUVoiceSnd@@U?$less@H@std@@V?$allocator@U?$pair@$$CBHUVoiceSnd@@@std@@@3@$0A@@std@@@std@@KAPAU_Node@?$_Tree_nod@V?$_Tmap_traits@HUVoiceSnd@@U?$less@H@std@@V?$allocator@U?$pair@$$CBHUVoiceSnd@@@std@@@3@$0A@@std@@@2@PAU342@@Z 100a4e70 f i scriptparser.obj
 0002:00032ec0       ?_Min@?$_Tree@V?$_Tmap_traits@HUVoiceSnd@@U?$less@H@std@@V?$allocator@U?$pair@$$CBHUVoiceSnd@@@std@@@3@$0A@@std@@@std@@KAPAU_Node@?$_Tree_nod@V?$_Tmap_traits@HUVoiceSnd@@U?$less@H@std@@V?$allocator@U?$pair@$$CBHUVoiceSnd@@@std@@@3@$0A@@std@@@2@PAU342@@Z 100a4ec0 f i scriptparser.obj
 0002:00032f10       ?_Rrotate@?$_Tree@V?$_Tmap_traits@HUVoiceSnd@@U?$less@H@std@@V?$allocator@U?$pair@$$CBHUVoiceSnd@@@std@@@3@$0A@@std@@@std@@IAEXPAU_Node@?$_Tree_nod@V?$_Tmap_traits@HUVoiceSnd@@U?$less@H@std@@V?$allocator@U?$pair@$$CBHUVoiceSnd@@@std@@@3@$0A@@std@@@2@@Z 100a4f10 f i scriptparser.obj
 0002:000330b0       ?_Orphan_ptr@?$_Tree@V?$_Tmap_traits@HUVoiceSnd@@U?$less@H@std@@V?$allocator@U?$pair@$$CBHUVoiceSnd@@@std@@@3@$0A@@std@@@std@@IBEXAAV12@PAU_Node@?$_Tree_nod@V?$_Tmap_traits@HUVoiceSnd@@U?$less@H@std@@V?$allocator@U?$pair@$$CBHUVoiceSnd@@@std@@@3@$0A@@std@@@2@@Z 100a50b0 f i scriptparser.obj
 0002:000331b0       ?destroy@?$allocator@U_Node@?$_Tree_nod@V?$_Tmap_traits@HUVoiceSnd@@U?$less@H@std@@V?$allocator@U?$pair@$$CBHUVoiceSnd@@@std@@@3@$0A@@std@@@std@@@std@@QAEXPAU_Node@?$_Tree_nod@V?$_Tmap_traits@HUVoiceSnd@@U?$less@H@std@@V?$allocator@U?$pair@$$CBHUVoiceSnd@@@std@@@3@$0A@@std@@@2@@Z 100a51b0 f i scriptparser.obj
 0002:000331f0       ??0const_iterator@?$_Tree@V?$_Tmap_traits@HUVoiceSnd@@U?$less@H@std@@V?$allocator@U?$pair@$$CBHUVoiceSnd@@@std@@@3@$0A@@std@@@std@@QAE@PAU_Node@?$_Tree_nod@V?$_Tmap_traits@HUVoiceSnd@@U?$less@H@std@@V?$allocator@U?$pair@$$CBHUVoiceSnd@@@std@@@3@$0A@@std@@@2@PBV12@@Z 100a51f0 f i scriptparser.obj
 0002:00033290       ??Econst_iterator@?$_Tree@V?$_Tmap_traits@HUVoiceSnd@@U?$less@H@std@@V?$allocator@U?$pair@$$CBHUVoiceSnd@@@std@@@3@$0A@@std@@@std@@QAEAAV012@XZ 100a5290 f i scriptparser.obj
 0002:000332c0       ?_Mynode@const_iterator@?$_Tree@V?$_Tmap_traits@HUVoiceSnd@@U?$less@H@std@@V?$allocator@U?$pair@$$CBHUVoiceSnd@@@std@@@3@$0A@@std@@@std@@QBEPAU_Node@?$_Tree_nod@V?$_Tmap_traits@HUVoiceSnd@@U?$less@H@std@@V?$allocator@U?$pair@$$CBHUVoiceSnd@@@std@@@3@$0A@@std@@@3@XZ 100a52c0 f i scriptparser.obj
 0002:000332e0       ??0?$_Bidit@U?$pair@$$CBHUVoiceSnd@@@std@@HPBU12@ABU12@@std@@QAE@XZ 100a52e0 f i scriptparser.obj
 0002:00033310       ??0?$_Iterator_with_base@Ubidirectional_iterator_tag@std@@U?$pair@$$CBHUVoiceSnd@@@2@HPBU32@ABU32@V_Iterator_base@2@@std@@QAE@XZ 100a5310 f i scriptparser.obj
 0002:00033340       ?_Inc@const_iterator@?$_Tree@V?$_Tmap_traits@HUVoiceSnd@@U?$less@H@std@@V?$allocator@U?$pair@$$CBHUVoiceSnd@@@std@@@3@$0A@@std@@@std@@QAEXXZ 100a5340 f i scriptparser.obj
 0002:000334d0       ??$_Destroy@U_Node@?$_Tree_nod@V?$_Tmap_traits@HUVoiceSnd@@U?$less@H@std@@V?$allocator@U?$pair@$$CBHUVoiceSnd@@@std@@@3@$0A@@std@@@std@@@std@@YAXPAU_Node@?$_Tree_nod@V?$_Tmap_traits@HUVoiceSnd@@U?$less@H@std@@V?$allocator@U?$pair@$$CBHUVoiceSnd@@@std@@@3@$0A@@std@@@0@@Z 100a54d0 f i scriptparser.obj
 0002:000334e0       ?voice_init@@YAXXZ         100a54e0 f   voicesnd.obj
 0002:000334f0       ?voice_close@@YAXXZ        100a54f0 f   voicesnd.obj
 0002:00033500       ?voice_start@@YAHHMH@Z     100a5500 f   voicesnd.obj
 0002:00033670       ?voice_stop@@YAXHH@Z       100a5670 f   voicesnd.obj
 0002:00033820       ?voice_stop_all@@YAXH@Z    100a5820 f   voicesnd.obj
 0002:00033840       ?voice_pause@@YAXH@Z       100a5840 f   voicesnd.obj
 0002:00033880       ?voice_pause_all@@YAXXZ    100a5880 f   voicesnd.obj
 0002:000338a0       ?voice_unpause@@YAXH@Z     100a58a0 f   voicesnd.obj
 0002:000338e0       ?voice_unpause_all@@YAXXZ  100a58e0 f   voicesnd.obj
 0002:00033900       ?voice_set_volume@@YAXHM@Z 100a5900 f   voicesnd.obj
 0002:00033950       ?voice_set_volume_all@@YAXM@Z 100a5950 f   voicesnd.obj
 0002:00033970       ?voice_set_loop@@YAXHH@Z   100a5970 f   voicesnd.obj
 0002:000339b0       ?voice_state@@YAHH@Z       100a59b0 f   voicesnd.obj
 0002:00033b70       ?timer_close@@YAXXZ        100a5b70 f   timer.obj
 0002:00033bc0       ?timer_init@@YAXXZ         100a5bc0 f   timer.obj
 0002:00033c40       ?timer_get_fixed_seconds@@YAJXZ 100a5c40 f   timer.obj
 0002:00033d50       ?timer_get_fixed_secondsX@@YAJXZ 100a5d50 f   timer.obj
 0002:00033d70       ?timer_get_approx_seconds@@YAJXZ 100a5d70 f   timer.obj
 0002:00033d90       ?timer_get_milliseconds@@YAHXZ 100a5d90 f   timer.obj
 0002:00033db0       ?timer_get_microseconds@@YAHXZ 100a5db0 f   timer.obj
 0002:00033de0       ?timestamp_reset@@YAXXZ    100a5de0 f   timer.obj
 0002:00033df0       ?timestamp_inc@@YAXM@Z     100a5df0 f   timer.obj
 0002:00033e50       ?timestamp@@YAHH@Z         100a5e50 f   timer.obj
 0002:00033eb0       ?timestamp_until@@YAHH@Z   100a5eb0 f   timer.obj
 0002:00033ec0       ?timestamp@@YAHXZ          100a5ec0 f   timer.obj
 0002:00033ed0       ?timestamp_has_time_elapsed@@YAHHH@Z 100a5ed0 f   timer.obj
 0002:00033f10       ?timing_event_lookup@@YAHPAD@Z 100a5f10 f   timer.obj
 0002:00033f80       ?timing_frame_start@@YAXXZ 100a5f80 f   timer.obj
 0002:00034010       ?timing_frame_stop@@YAXXZ  100a6010 f   timer.obj
 0002:00034040       ?timing_frame_total@@YAHXZ 100a6040 f   timer.obj
 0002:00034050       ?timing_event_start@@YAXPAD@Z 100a6050 f   timer.obj
 0002:00034130       ?timing_event_stop@@YAXPAD@Z 100a6130 f   timer.obj
 0002:000341b0       ?timing_event_total@@YAHPAD@Z 100a61b0 f   timer.obj
 0002:00034200       ?timing_event_pct@@YAMPAD@Z 100a6200 f   timer.obj
 0002:00034430       ?amdInitialize@@YAHPAPAUHMIXER__@@0@Z 100a6430 f   util_audiomixer.obj
 0002:00034820       ?amdUninitialize@@YAHPAUHMIXER__@@@Z 100a6820 f   util_audiomixer.obj
 0002:00034870       ?amdGetMasterVolumeControl@@YAHPAUHMIXER__@@PAHPAK2@Z 100a6870 f   util_audiomixer.obj
 0002:000349e0       ?amdGetMasterVolumeValue@@YAHPAUHMIXER__@@HPAK@Z 100a69e0 f   util_audiomixer.obj
 0002:00034ac0       ?amdSetMasterVolumeValue@@YAHPAUHMIXER__@@HK@Z 100a6ac0 f   util_audiomixer.obj
 0002:00034b90       ?amdGetMasterPanControl@@YAHPAUHMIXER__@@PAHPAJ2@Z 100a6b90 f   util_audiomixer.obj
 0002:00034d10       ?amdGetMasterPanValue@@YAHPAUHMIXER__@@HPAJ@Z 100a6d10 f   util_audiomixer.obj
 0002:00034df0       ?amdSetMasterPanValue@@YAHPAUHMIXER__@@HJ@Z 100a6df0 f   util_audiomixer.obj
 0002:00034ec0       ?amdGetMasterMuteControl@@YAHPAUHMIXER__@@PAH@Z 100a6ec0 f   util_audiomixer.obj
 0002:00035010       ?amdGetMasterMuteValue@@YAHPAUHMIXER__@@HPAJ@Z 100a7010 f   util_audiomixer.obj
 0002:000350f0       ?amdSetMasterMuteValue@@YAHPAUHMIXER__@@HJ@Z 100a70f0 f   util_audiomixer.obj
 0002:000351c0       ?amdGetVolume@@YAXPAUHMIXER__@@HKKPAH1@Z 100a71c0 f   util_audiomixer.obj
 0002:000352f0       ?amdSetVolume@@YAXPAUHMIXER__@@HKKHH@Z 100a72f0 f   util_audiomixer.obj
 0002:00035420       ?amdGetWavVolumeControl@@YAHPAUHMIXER__@@PAHPAK2@Z 100a7420 f   util_audiomixer.obj
 0002:00035590       ?amdGetWavVolumeValue@@YAHPAUHMIXER__@@HPAK@Z 100a7590 f   util_audiomixer.obj
 0002:00035670       ?amdSetWavVolumeValue@@YAHPAUHMIXER__@@HK@Z 100a7670 f   util_audiomixer.obj
 0002:00035740       ?amdGetWavPanControl@@YAHPAUHMIXER__@@PAHPAJ2@Z 100a7740 f   util_audiomixer.obj
 0002:000358c0       ?amdGetWavPanValue@@YAHPAUHMIXER__@@HPAJ@Z 100a78c0 f   util_audiomixer.obj
 0002:000359a0       ?amdSetWavPanValue@@YAHPAUHMIXER__@@HJ@Z 100a79a0 f   util_audiomixer.obj
 0002:00035a70       ?amdGetWavMuteControl@@YAHPAUHMIXER__@@PAH@Z 100a7a70 f   util_audiomixer.obj
 0002:00035bc0       ?amdGetWavMuteValue@@YAHPAUHMIXER__@@HPAJ@Z 100a7bc0 f   util_audiomixer.obj
 0002:00035ca0       ?amdSetWavMuteValue@@YAHPAUHMIXER__@@HJ@Z 100a7ca0 f   util_audiomixer.obj
 0002:00035d70       ?amdGetMicInputVolumeControl@@YAHPAUHMIXER__@@PAHPAK22@Z 100a7d70 f   util_audiomixer.obj
 0002:00036200       ?amdGetMicInputVolumeValue@@YAHPAUHMIXER__@@HPAKK@Z 100a8200 f   util_audiomixer.obj
 0002:000362e0       ?amdSetMicInputVolumeValue@@YAHPAUHMIXER__@@PAHKK@Z 100a82e0 f   util_audiomixer.obj
 0002:000363e0       ?amdGetMicOutputVolumeControl@@YAHPAUHMIXER__@@PAHPAK2@Z 100a83e0 f   util_audiomixer.obj
 0002:00036640       ?amdGetMicOutputVolumeValue@@YAHPAUHMIXER__@@HPAK@Z 100a8640 f   util_audiomixer.obj
 0002:00036720       ?amdSetMicOutputVolumeValue@@YAHPAUHMIXER__@@HK@Z 100a8720 f   util_audiomixer.obj
 0002:000367f0       ?amdGetMicPanControl@@YAHPAUHMIXER__@@PAHPAJ2@Z 100a87f0 f   util_audiomixer.obj
 0002:00036970       ?amdGetMicPanValue@@YAHPAUHMIXER__@@HPAJ@Z 100a8970 f   util_audiomixer.obj
 0002:00036a50       ?amdSetMicPanValue@@YAHPAUHMIXER__@@HJ@Z 100a8a50 f   util_audiomixer.obj
 0002:00036b20       ?amdGetMicOutputMuteControl@@YAHPAUHMIXER__@@PAH@Z 100a8b20 f   util_audiomixer.obj
 0002:00036d60       ?amdGetMicOutputMuteValue@@YAHPAUHMIXER__@@HPAJ@Z 100a8d60 f   util_audiomixer.obj
 0002:00036e40       ?amdSetMicOutputMuteValue@@YAHPAUHMIXER__@@HJ@Z 100a8e40 f   util_audiomixer.obj
 0002:00036f10       ?SelectMic@@YAXPAUHMIXER__@@@Z 100a8f10 f   util_audiomixer.obj
 0002:00037f30       __LOG                      100a9f30 f   util_debug.obj
 0002:00038010       __LOG2                     100aa010 f   util_debug.obj
 0002:000381f0       _path_is_directory         100aa1f0 f   util_shwapi.obj
 0002:00038240       _get_program_path          100aa240 f   util_shwapi.obj
 0002:000382c0       _path_add_backslash        100aa2c0 f   util_shwapi.obj
 0002:00038300       _path_is_relative          100aa300 f   util_shwapi.obj
 0002:000384a0       _path_remove_filespec      100aa4a0 f   util_shwapi.obj
 0002:00038590       _path_unquote              100aa590 f   util_shwapi.obj
 0002:00038660       __offset                   100aa660 f   util_shwapi.obj
 0002:00038730       __getat                    100aa730 f   util_shwapi.obj
 0002:00038770       __strsize                  100aa770 f   util_shwapi.obj
 0002:000387c0       __strsizez                 100aa7c0 f   util_shwapi.obj
 0002:00038800       __strzcpy                  100aa800 f   util_shwapi.obj
 0002:000388d0       __strzcat                  100aa8d0 f   util_shwapi.obj
 0002:00038980       __strzncpy                 100aa980 f   util_shwapi.obj
 0002:00038a90       __strzncat                 100aaa90 f   util_shwapi.obj
 0002:00038b60       __setat                    100aab60 f   util_shwapi.obj
 0002:00038c10       __insert                   100aac10 f   util_shwapi.obj
 0002:00038c90       __remove                   100aac90 f   util_shwapi.obj
 0002:00038d00       _replace_filename          100aad00 f   util_shwapi.obj
 0002:00038e30       _replace_extension         100aae30 f   util_shwapi.obj
 0002:00038fc0       _append_filename           100aafc0 f   util_shwapi.obj
 0002:00039180       _get_filename              100ab180 f   util_shwapi.obj
 0002:00039210       _get_extension             100ab210 f   util_shwapi.obj
 0002:000392d0       _put_backslash             100ab2d0 f   util_shwapi.obj
 0002:000397c0       _str_trim                  100ab7c0 f   util_string.obj
 0002:00039830       _str_delete_substr         100ab830 f   util_string.obj
 0002:000398a0       _STR_AllocSetString        100ab8a0 f   util_string.obj
 0002:00039920       _hexVal                    100ab920 f   util_string.obj
 0002:00039980       _trimLeft                  100ab980 f   util_string.obj
 0002:00039a10       _trimInet                  100aba10 f   util_string.obj
 0002:00039a90       _trimRight                 100aba90 f   util_string.obj
 0002:00039b00       _trimDirSeparator          100abb00 f   util_string.obj
 0002:00039b60       _trim                      100abb60 f   util_string.obj
 0002:00039b90       _splitPath                 100abb90 f   util_string.obj
 0002:00039ca0       _getExtension              100abca0 f   util_string.obj
 0002:00039d20       _translateEscapeString     100abd20 f   util_string.obj
 0002:00039e00       _translateFilepath         100abe00 f   util_string.obj
 0002:0003a000       ?cfopen@@YAPAUCFILE@@PAD0H@Z 100ac000 f   cfile.obj
 0002:0003a0d0       ?cfclose@@YAHPAUCFILE@@@Z  100ac0d0 f   cfile.obj
 0002:0003a150       ?cf_open_file_cfblock@@YAPAUCFILE@@PAU_iobuf@@H@Z 100ac150 f   cfile.obj
 0002:0003a1a0       ?cf_open_vfs_cfblock@@YAPAUCFILE@@PAXH@Z 100ac1a0 f   cfile.obj
 0002:0003a250       ?cf_init_lowlevel_read_code@@YAXPAUCFILE@@HH@Z 100ac250 f   cfile.obj
 0002:0003a380       ?cfeof@@YAHPAUCFILE@@@Z    100ac380 f   cfile.obj
 0002:0003a470       ?cftell@@YAHPAUCFILE@@@Z   100ac470 f   cfile.obj
 0002:0003a540       ?cfseek@@YAHPAUCFILE@@HH@Z 100ac540 f   cfile.obj
 0002:0003a6c0       ?cfread@@YAHPAXHHPAUCFILE@@@Z 100ac6c0 f   cfile.obj
 0002:0003a8c0       ?cfread_float@@YAMPAUCFILE@@M@Z 100ac8c0 f   cfile.obj
 0002:0003a940       ?cfread_int@@YAHPAUCFILE@@H@Z 100ac940 f   cfile.obj
 0002:0003a9c0       ?cfread_uint@@YAIPAUCFILE@@I@Z 100ac9c0 f   cfile.obj
 0002:0003aa40       ?cfread_short@@YAFPAUCFILE@@F@Z 100aca40 f   cfile.obj
 0002:0003aac0       ?cfread_ushort@@YAGPAUCFILE@@G@Z 100acac0 f   cfile.obj
 0002:0003ab40       ?cfread_ubyte@@YAEPAUCFILE@@E@Z 100acb40 f   cfile.obj
 0002:0003abc0       ?cfread_char@@YADPAUCFILE@@D@Z 100acbc0 f   cfile.obj
 0002:0003ac40       ?cfread_string@@YAXPADHPAUCFILE@@@Z 100acc40 f   cfile.obj
 0002:0003aca0       ?cfread_string_len@@YAXPADHPAUCFILE@@@Z 100acca0 f   cfile.obj
 0002:0003ad00       ?cfget_cfile_block@@YAPAUCFILE@@XZ 100acd00 f   cfile.obj
 0002:0003adb0       ?cffree_cfile_block@@YAXPAUCFILE@@@Z 100acdb0 f   cfile.obj
 0002:0003ae60       ?cfilelength@@YAHPAUCFILE@@@Z 100ace60 f   cfile.obj
 0002:0003b210       ?fixmul@@YAJJJ@Z           100ad210 f   fix.obj
 0002:0003b260       ?fixdiv@@YAJJJ@Z           100ad260 f   fix.obj
 0002:0003b290       ?fixmuldiv@@YAJJJJ@Z       100ad290 f   fix.obj
 0002:0003b2f0       ?fl_isqrt_c@@YAMM@Z        100ad2f0 f   floating.obj
 0002:0003b360       ?fl_roundoff@@YAMMH@Z      100ad360 f   floating.obj
 0002:0003b3d0       ?frand@@YAMXZ              100ad3d0 f   floating.obj
 0002:0003b420       ?frand_range@@YAMMM@Z      100ad420 f   floating.obj
 0002:0003b460       ?rand_chance@@YAHMM@Z      100ad460 f   floating.obj
 0002:0003b560       ?atan2_safe@@YAMMM@Z       100ad560 f   vecmat.obj
 0002:0003b610       ?vm_vec_projection_parallel@@YAMPAUvector@@00@Z 100ad610 f   vecmat.obj
 0002:0003b660       ?vm_vec_projection_onto_plane@@YAXPAUvector@@00@Z 100ad660 f   vecmat.obj
 0002:0003b6c0       ?vm_project_point_onto_plane@@YAXPAUvector@@000@Z 100ad6c0 f   vecmat.obj
 0002:0003b740       ?asqrt@@YAMM@Z             100ad740 f   vecmat.obj
 0002:0003b780       ?vm_set_identity@@YAXPAUmatrix@@@Z 100ad780 f   vecmat.obj
 0002:0003b7d0       ?vm_vec_add@@YAXPAUvector@@00@Z 100ad7d0 f   vecmat.obj
 0002:0003b810       ?vm_vec_sub@@YAXPAUvector@@00@Z 100ad810 f   vecmat.obj
 0002:0003b850       ?vm_vec_add2@@YAXPAUvector@@0@Z 100ad850 f   vecmat.obj
 0002:0003b890       ?vm_vec_sub2@@YAXPAUvector@@0@Z 100ad890 f   vecmat.obj
 0002:0003b8d0       ?vm_vert2vec@@YAXPAUvertex@@PAUvector@@@Z 100ad8d0 f   vecmat.obj
 0002:0003b900       ?vm_vec2vert@@YAXPAUvector@@PAUvertex@@@Z 100ad900 f   vecmat.obj
 0002:0003b930       ?vm_vec_avg_n@@YAPAUvector@@PAU1@HQAU1@@Z 100ad930 f   vecmat.obj
 0002:0003b9e0       ?vm_vec_avg@@YAPAUvector@@PAU1@00@Z 100ad9e0 f   vecmat.obj
 0002:0003ba30       ?vm_vec_avg3@@YAPAUvector@@PAU1@000@Z 100ada30 f   vecmat.obj
 0002:0003ba90       ?vm_vec_avg4@@YAPAUvector@@PAU1@0000@Z 100ada90 f   vecmat.obj
 0002:0003bb00       ?vm_vec_scale@@YAXPAUvector@@M@Z 100adb00 f   vecmat.obj
 0002:0003bb30       ?vm_vec_copy_scale@@YAXPAUvector@@0M@Z 100adb30 f   vecmat.obj
 0002:0003bb60       ?vm_vec_scale_add@@YAXPAUvector@@00M@Z 100adb60 f   vecmat.obj
 0002:0003bbb0       ?vm_vec_scale_add2@@YAXPAUvector@@0M@Z 100adbb0 f   vecmat.obj
 0002:0003bc00       ?vm_vec_scale_sub2@@YAXPAUvector@@0M@Z 100adc00 f   vecmat.obj
 0002:0003bc50       ?vm_vec_scale2@@YAXPAUvector@@MM@Z 100adc50 f   vecmat.obj
 0002:0003bca0       ?vm_vec_dotprod@@YAMPAUvector@@0@Z 100adca0 f   vecmat.obj
 0002:0003bce0       ?vm_vec_dot3@@YAMMMMPAUvector@@@Z 100adce0 f   vecmat.obj
 0002:0003bd20       ?vm_vec_mag@@YAMPAUvector@@@Z 100add20 f   vecmat.obj
 0002:0003bdb0       ?vm_vec_mag_squared@@YAMPAUvector@@@Z 100addb0 f   vecmat.obj
 0002:0003be10       ?vm_vec_dist_squared@@YAMPAUvector@@0@Z 100ade10 f   vecmat.obj
 0002:0003be80       ?vm_vec_dist@@YAMPAUvector@@0@Z 100ade80 f   vecmat.obj
 0002:0003bf00       ?vm_vec_mag_quick@@YAMPAUvector@@@Z 100adf00 f   vecmat.obj
 0002:0003c030       ?vm_vec_dist_quick@@YAMPAUvector@@0@Z 100ae030 f   vecmat.obj
 0002:0003c0b0       ?vm_vec_copy_normalize@@YAMPAUvector@@0@Z 100ae0b0 f   vecmat.obj
 0002:0003c160       ?vm_vec_normalize@@YAMPAUvector@@@Z 100ae160 f   vecmat.obj
 0002:0003c190       ?vm_vec_normalize_safe@@YAMPAUvector@@@Z 100ae190 f   vecmat.obj
 0002:0003c230       ?vm_vec_imag@@YAMPAUvector@@@Z 100ae230 f   vecmat.obj
 0002:0003c2a0       ?vm_vec_copy_normalize_quick@@YAMPAUvector@@0@Z 100ae2a0 f   vecmat.obj
 0002:0003c310       ?vm_vec_normalize_quick@@YAMPAUvector@@@Z 100ae310 f   vecmat.obj
 0002:0003c380       ?vm_vec_copy_normalize_quick_mag@@YAMPAUvector@@0@Z 100ae380 f   vecmat.obj
 0002:0003c3f0       ?vm_vec_normalize_quick_mag@@YAMPAUvector@@@Z 100ae3f0 f   vecmat.obj
 0002:0003c450       ?vm_vec_normalized_dir@@YAMPAUvector@@00@Z 100ae450 f   vecmat.obj
 0002:0003c490       ?vm_vec_normalized_dir_quick@@YAMPAUvector@@00@Z 100ae490 f   vecmat.obj
 0002:0003c4c0       ?vm_vec_normalized_dir_quick_mag@@YAMPAUvector@@00@Z 100ae4c0 f   vecmat.obj
 0002:0003c500       ?vm_vec_normal@@YAPAUvector@@PAU1@000@Z 100ae500 f   vecmat.obj
 0002:0003c540       ?vm_vec_crossprod@@YAPAUvector@@PAU1@00@Z 100ae540 f   vecmat.obj
 0002:0003c5b0       ?vm_test_parallel@@YAHPAUvector@@0@Z 100ae5b0 f   vecmat.obj
 0002:0003c670       ?vm_vec_perp@@YAPAUvector@@PAU1@000@Z 100ae670 f   vecmat.obj
 0002:0003c710       ?vm_vec_delta_ang@@YAMPAUvector@@00@Z 100ae710 f   vecmat.obj
 0002:0003c7d0       ?vm_vec_delta_ang_norm@@YAMPAUvector@@00@Z 100ae7d0 f   vecmat.obj
 0002:0003c890       ?sincos_2_matrix@@YAPAUmatrix@@PAU1@MMMMMM@Z 100ae890 f   vecmat.obj
 0002:0003c950       ?vm_angles_2_matrix@@YAPAUmatrix@@PAU1@PAUangles@@@Z 100ae950 f   vecmat.obj
 0002:0003ca40       ?vm_angle_2_matrix@@YAPAUmatrix@@PAU1@MH@Z 100aea40 f   vecmat.obj
 0002:0003cba0       ?vm_vec_ang_2_matrix@@YAPAUmatrix@@PAU1@PAUvector@@M@Z 100aeba0 f   vecmat.obj
 0002:0003cc80       ?vm_vector_2_matrix@@YAPAUmatrix@@PAU1@PAUvector@@11@Z 100aec80 f   vecmat.obj
 0002:0003cea0       ?vm_vector_2_matrix_norm@@YAPAUmatrix@@PAU1@PAUvector@@11@Z 100aeea0 f   vecmat.obj
 0002:0003d060       ?vm_vec_rotate@@YAPAUvector@@PAU1@0PAUmatrix@@@Z 100af060 f   vecmat.obj
 0002:0003d0f0       ?vm_vec_unrotate@@YAPAUvector@@PAU1@0PAUmatrix@@@Z 100af0f0 f   vecmat.obj
 0002:0003d180       ?vm_transpose_matrix@@YAPAUmatrix@@PAU1@@Z 100af180 f   vecmat.obj
 0002:0003d1f0       ?vm_copy_transpose_matrix@@YAPAUmatrix@@PAU1@0@Z 100af1f0 f   vecmat.obj
 0002:0003d270       ?vm_matrix_x_matrix@@YAPAUmatrix@@PAU1@00@Z 100af270 f   vecmat.obj
 0002:0003d450       ?vm_extract_angles_matrix@@YAPAUangles@@PAU1@PAUmatrix@@@Z 100af450 f   vecmat.obj
 0002:0003d620       ?vm_extract_angles_vector_normalized@@YAPAUangles@@PAU1@PAUvector@@@Z 100af620 f   vecmat.obj
 0002:0003d6a0       ?vm_extract_angles_vector@@YAPAUangles@@PAU1@PAUvector@@@Z 100af6a0 f   vecmat.obj
 0002:0003d730       ?vm_dist_to_plane@@YAMPAUvector@@00@Z 100af730 f   vecmat.obj
 0002:0003d7b0       ?vm_trackball@@YAXHHPAUmatrix@@@Z 100af7b0 f   vecmat.obj
 0002:0003d8f0       ?vm_vec_outer_product@@YAXPAUmatrix@@PAUvector@@@Z 100af8f0 f   vecmat.obj
 0002:0003d990       ?find_nearest_point_on_line@@YAMPAUvector@@000@Z 100af990 f   vecmat.obj
 0002:0003db40       ?vm_orthogonalize_matrix@@YAXPAUmatrix@@@Z 100afb40 f   vecmat.obj
 0002:0003dd10       ?vm_fix_matrix@@YAXPAUmatrix@@@Z 100afd10 f   vecmat.obj
 0002:0003dfc0       ?vm_rotate_matrix_by_angles@@YAXPAUmatrix@@PAUangles@@@Z 100affc0 f   vecmat.obj
 0002:0003e070       ?vm_vec_dot_to_point@@YAMPAUvector@@00@Z 100b0070 f   vecmat.obj
 0002:0003e100       ?compute_point_on_plane@@YAXPAUvector@@PAUplane@@0@Z 100b0100 f   vecmat.obj
 0002:0003e200       ?vm_vec_rand_vec_quick@@YAXPAUvector@@@Z 100b0200 f   vecmat.obj
 0002:0003e2a0       ?vm_rot_point_around_line@@YAXPAUvector@@0M00@Z 100b02a0 f   vecmat.obj
 0002:0003e3e0       ?vm_vec_cmp@@YAHPAUvector@@0@Z 100b03e0 f   vecmat.obj
 0002:0003e430       ?vm_matrix_cmp@@YAHPAUmatrix@@0@Z 100b0430 f   vecmat.obj
 0002:0003e530       ?vm_interp_angle@@YAXPAMMM@Z 100b0530 f   vecmat.obj
 0002:0003e670       ?vm_check_matrix_for_zeros@@YAHPAUmatrix@@@Z 100b0670 f   vecmat.obj
 0002:0003e810       ?vm_vec_same@@YAHPAUvector@@0@Z 100b0810 f   vecmat.obj
 0002:0003e860       ?vm_quaternion_rotate@@YAXPAUmatrix@@MPAUvector@@@Z 100b0860 f   vecmat.obj
 0002:0003ea40       ?rotate_z@@YAXPAUmatrix@@M@Z 100b0a40 f   vecmat.obj
 0002:0003eac0       ?vm_matrix_to_rot_axis_and_angle@@YAXPAUmatrix@@PAMPAUvector@@@Z 100b0ac0 f   vecmat.obj
 0002:0003ed40       ?approach@@YAMMMMMMPAMH@Z  100b0d40 f   vecmat.obj
 0002:0003f180       ?away@@YAMMMMMMPAMH@Z      100b1180 f   vecmat.obj
 0002:0003f2b0       ?vm_matrix_interpolate@@YAXPAUmatrix@@0PAUvector@@M0111H@Z 100b12b0 f   vecmat.obj
 0002:0003fc80       ?get_camera_limits@@YAXPAUmatrix@@0MPAUvector@@1@Z 100b1c80 f   vecmat.obj
 0002:0003feb0       ?vm_fvec_matrix_interpolate@@YAXPAUmatrix@@0PAUvector@@M0111H@Z 100b1eb0 f   vecmat.obj
 0002:00040c00       ?vm_forward_interpolate@@YAXPAUvector@@PAUmatrix@@0MM1000H@Z 100b2c00 f   vecmat.obj
 0002:00041710       ?vm_find_bounding_sphere@@YAXPAUvector@@H0PAM@Z 100b3710 f   vecmat.obj
 0002:00041d50       ?vm_rotate_vec_to_body@@YAPAUvector@@PAU1@0PAUmatrix@@@Z 100b3d50 f   vecmat.obj
 0002:00041d70       ?vm_rotate_vec_to_world@@YAPAUvector@@PAU1@0PAUmatrix@@@Z 100b3d70 f   vecmat.obj
 0002:00041d90       ?vm_estimate_next_orientation@@YAXPAUmatrix@@00@Z 100b3d90 f   vecmat.obj
 0002:00041e40       ?is_valid_vec@@YAHPAUvector@@@Z 100b3e40 f   vecmat.obj
 0002:00041ec0       ?is_valid_matrix@@YAHPAUmatrix@@@Z 100b3ec0 f   vecmat.obj
 0002:00041f30       ?vm_vec_interp_constant@@YAXPAUvector@@00M@Z 100b3f30 f   vecmat.obj
 0002:00042000       ?vm_vec_random_cone@@YAXPAUvector@@0MPAUmatrix@@@Z 100b4000 f   vecmat.obj
 0002:00042170       ?vm_vec_random_in_circle@@YAXPAUvector@@0PAUmatrix@@MH@Z 100b4170 f   vecmat.obj
 0002:00042260       ?vm_vec_dist_to_line@@YAHPAUvector@@000PAM@Z 100b4260 f   vecmat.obj
 0002:000423c0       ?vm_vec_dist_squared_to_line@@YAXPAUvector@@000PAM@Z 100b43c0 f   vecmat.obj
 0002:000440c0       ?atan@@YAMM@Z              100b60c0 f i vecmat.obj
 0002:000440f0       _atanf                     100b60f0 f i vecmat.obj
 0002:00044130       ?sqrt@@YAMM@Z              100b6130 f i vecmat.obj
 0002:00044160       _sqrtf                     100b6160 f i vecmat.obj
 0002:000441a0       ?acos@@YAMM@Z              100b61a0 f i vecmat.obj
 0002:000441d0       _acosf                     100b61d0 f i vecmat.obj
 0002:00044210       ?cos@@YAMM@Z               100b6210 f i vecmat.obj
 0002:00044240       _cosf                      100b6240 f i vecmat.obj
 0002:00044280       ?sin@@YAMM@Z               100b6280 f i vecmat.obj
 0002:000442b0       _sinf                      100b62b0 f i vecmat.obj
 0002:000442f0       ?asin@@YAMM@Z              100b62f0 f i vecmat.obj
 0002:00044320       _asinf                     100b6320 f i vecmat.obj
 0002:00044360       ?myrand@@YAHXZ             100b6360 f   systemvars.obj
 0002:000443a0       ?ole2_bufread@@YAXPAUOLE2Stream@@@Z 100b63a0 f   ole.obj
 0002:00044490       ?ole2_read@@YAHPAXJJPAUOLE2Stream@@@Z 100b6490 f   ole.obj
 0002:00044630       ?ole2_sopen@@YAPAUOLE2Stream@@PAUOLE2@@K@Z 100b6630 f   ole.obj
 0002:000446d0       ?ole2_seek@@YAXPAUOLE2Stream@@K@Z 100b66d0 f   ole.obj
 0002:000447c0       ?ole2_fopen@@YAPAUOLE2Stream@@PAUOLE2@@PAD@Z 100b67c0 f   ole.obj
 0002:00044860       ?ole2_open@@YAPAUOLE2@@PAD@Z 100b6860 f   ole.obj
 0002:00044f10       ?ole2_close@@YAXPAUOLE2@@@Z 100b6f10 f   ole.obj
 0002:00044f60       ?ole2_fclose@@YAXPAUOLE2Stream@@@Z 100b6f60 f   ole.obj
 0002:00045270       ?xls@@YAHXZ                100b7270 f   xls.obj
 0002:00045280       ?xls_addSST@@YAXPAUxlsWorkBook@@PAUSST@@K@Z 100b7280 f   xls.obj
 0002:000452f0       ?xls_appendSST@@YAXPAUxlsWorkBook@@PAEK@Z 100b72f0 f   xls.obj
 0002:000456e0       ?NumFromRk@@YANPAE@Z       100b76e0 f   xls.obj
 0002:00045750       ?xls_addSheet@@YAXPAUxlsWorkBook@@PAE@Z 100b7750 f   xls.obj
 0002:00045840       ?xls_addRow@@YAXPAUxlsWorkSheet@@PAUROW@@@Z 100b7840 f   xls.obj
 0002:000458e0       ?xls_makeTable@@YAXPAUxlsWorkSheet@@@Z 100b78e0 f   xls.obj
 0002:00045ae0       ?xls_addCell@@YAXPAUxlsWorkSheet@@PAUBOF@@PAE@Z 100b7ae0 f   xls.obj
 0002:00045dd0       ?xls_addFont@@YAXPAUxlsWorkBook@@PAUFONT@@@Z 100b7dd0 f   xls.obj
 0002:00045ee0       ?xls_addXF@@YAXPAUxlsWorkBook@@PAUXF@@@Z 100b7ee0 f   xls.obj
 0002:00045ff0       ?xls_addColinfo@@YAXPAUxlsWorkSheet@@PAUCOLINFO@@@Z 100b7ff0 f   xls.obj
 0002:000460c0       ?xls_mergedCells@@YAXPAUxlsWorkSheet@@PAUBOF@@PAE@Z 100b80c0 f   xls.obj
 0002:00046220       ?xls_parseWorkBook@@YAXPAUxlsWorkBook@@@Z 100b8220 f   xls.obj
 0002:00046520       ?xls_preparseWorkSheet@@YAXPAUxlsWorkSheet@@@Z 100b8520 f   xls.obj
 0002:00046690       ?xls_formatColumn@@YAXPAUxlsWorkSheet@@@Z 100b8690 f   xls.obj
 0002:000467f0       ?xls_parseWorkSheet@@YAXPAUxlsWorkSheet@@@Z 100b87f0 f   xls.obj
 0002:00046aa0       ?xls_getWorkSheet@@YAPAUxlsWorkSheet@@PAUxlsWorkBook@@H@Z 100b8aa0 f   xls.obj
 0002:00046b10       ?xls_open@@YAPAUxlsWorkBook@@PAD0@Z 100b8b10 f   xls.obj
 0002:00046c10       ?xls_close@@YAXPAUxlsWorkBook@@@Z 100b8c10 f   xls.obj
 0002:00046c70       ?GetTxtFile@@YAHPADPAUST_ROWS@@@Z 100b8c70 f   xls.obj
 0002:00046fa0       ?SetRows@@YAXAAV?$basic_string@DU?$char_traits@D@std@@V?$allocator@D@2@@std@@PAUST_ROWS@@@Z 100b8fa0 f   xls.obj
 0002:00047120       ?IsRows@@YAHV?$basic_string@DU?$char_traits@D@std@@V?$allocator@D@2@@std@@@Z 100b9120 f   xls.obj
 0002:00047220       ?SetRow@@YAXV?$basic_string@DU?$char_traits@D@std@@V?$allocator@D@2@@std@@PAUST_ROWS@@@Z 100b9220 f   xls.obj
 0002:00047c10       ??0ST_CELLS@@QAE@XZ        100b9c10 f i xls.obj
 0002:00047c40       ??0?$basic_string@DU?$char_traits@D@std@@V?$allocator@D@2@@std@@QAE@XZ 100b9c40 f i xls.obj
 0002:00047ce0       ??4?$basic_string@DU?$char_traits@D@std@@V?$allocator@D@2@@std@@QAEAAV01@PBD@Z 100b9ce0 f i xls.obj
 0002:00047d20       ??Y?$basic_string@DU?$char_traits@D@std@@V?$allocator@D@2@@std@@QAEAAV01@ABV01@@Z 100b9d20 f i xls.obj
 0002:00047d60       ??Y?$basic_string@DU?$char_traits@D@std@@V?$allocator@D@2@@std@@QAEAAV01@PBD@Z 100b9d60 f i xls.obj
 0002:00047da0       ?find@?$basic_string@DU?$char_traits@D@std@@V?$allocator@D@2@@std@@QBEIPBDI@Z 100b9da0 f i xls.obj
 0002:00047e10       ?substr@?$basic_string@DU?$char_traits@D@std@@V?$allocator@D@2@@std@@QBE?AV12@II@Z 100b9e10 f i xls.obj
 0002:00047e90       ??0?$vector@V?$basic_string@DU?$char_traits@D@std@@V?$allocator@D@2@@std@@V?$allocator@V?$basic_string@DU?$char_traits@D@std@@V?$allocator@D@2@@std@@@2@@std@@QAE@XZ 100b9e90 f i xls.obj
 0002:00047f30       ?push_back@?$vector@V?$basic_string@DU?$char_traits@D@std@@V?$allocator@D@2@@std@@V?$allocator@V?$basic_string@DU?$char_traits@D@std@@V?$allocator@D@2@@std@@@2@@std@@QAEXABV?$basic_string@DU?$char_traits@D@std@@V?$allocator@D@2@@2@@Z 100b9f30 f i xls.obj
 0002:00048070       ?push_back@?$vector@UST_CELLS@@V?$allocator@UST_CELLS@@@std@@@std@@QAEXABUST_CELLS@@@Z 100ba070 f i xls.obj
 0002:000481b0       ??1?$_Vector_iterator@V?$basic_string@DU?$char_traits@D@std@@V?$allocator@D@2@@std@@V?$allocator@V?$basic_string@DU?$char_traits@D@std@@V?$allocator@D@2@@std@@@2@@std@@QAE@XZ 100ba1b0 f i xls.obj
 0002:000481e0       ??0?$_Vector_const_iterator@V?$basic_string@DU?$char_traits@D@std@@V?$allocator@D@2@@std@@V?$allocator@V?$basic_string@DU?$char_traits@D@std@@V?$allocator@D@2@@std@@@2@@std@@QAE@ABV01@@Z 100ba1e0 f i xls.obj
 0002:00048230       ??1?$_Vector_const_iterator@V?$basic_string@DU?$char_traits@D@std@@V?$allocator@D@2@@std@@V?$allocator@V?$basic_string@DU?$char_traits@D@std@@V?$allocator@D@2@@std@@@2@@std@@QAE@XZ 100ba230 f i xls.obj
 0002:00048260       ??1?$_Vector_iterator@UST_CELLS@@V?$allocator@UST_CELLS@@@std@@@std@@QAE@XZ 100ba260 f i xls.obj
 0002:00048290       ??0?$_Vector_const_iterator@UST_CELLS@@V?$allocator@UST_CELLS@@@std@@@std@@QAE@ABV01@@Z 100ba290 f i xls.obj
 0002:000482e0       ??1?$_Vector_const_iterator@UST_CELLS@@V?$allocator@UST_CELLS@@@std@@@std@@QAE@XZ 100ba2e0 f i xls.obj
 0002:00048310       ??0?$_Ranit@V?$basic_string@DU?$char_traits@D@std@@V?$allocator@D@2@@std@@HPBV12@ABV12@@std@@QAE@ABU01@@Z 100ba310 f i xls.obj
 0002:00048350       ??1?$_Ranit@V?$basic_string@DU?$char_traits@D@std@@V?$allocator@D@2@@std@@HPBV12@ABV12@@std@@QAE@XZ 100ba350 f i xls.obj
 0002:00048380       ??0?$_Ranit@UST_CELLS@@HPBU1@ABU1@@std@@QAE@ABU01@@Z 100ba380 f i xls.obj
 0002:000483c0       ??1?$_Ranit@UST_CELLS@@HPBU1@ABU1@@std@@QAE@XZ 100ba3c0 f i xls.obj
 0002:000483f0       ??0?$_Iterator_with_base@Urandom_access_iterator_tag@std@@V?$basic_string@DU?$char_traits@D@std@@V?$allocator@D@2@@2@HPBV32@ABV32@V_Iterator_base@2@@std@@QAE@ABU01@@Z 100ba3f0 f i xls.obj
 0002:00048430       ??1?$_Iterator_with_base@Urandom_access_iterator_tag@std@@V?$basic_string@DU?$char_traits@D@std@@V?$allocator@D@2@@2@HPBV32@ABV32@V_Iterator_base@2@@std@@QAE@XZ 100ba430 f i xls.obj
 0002:00048460       ??0?$_Iterator_with_base@Urandom_access_iterator_tag@std@@UST_CELLS@@HPBU3@ABU3@V_Iterator_base@2@@std@@QAE@ABU01@@Z 100ba460 f i xls.obj
 0002:000484a0       ??1?$_Iterator_with_base@Urandom_access_iterator_tag@std@@UST_CELLS@@HPBU3@ABU3@V_Iterator_base@2@@std@@QAE@XZ 100ba4a0 f i xls.obj
 0002:000484d0       ??0?$basic_string@DU?$char_traits@D@std@@V?$allocator@D@2@@std@@QAE@ABV01@IIABV?$allocator@D@1@@Z 100ba4d0 f i xls.obj
 0002:000485b0       ?append@?$basic_string@DU?$char_traits@D@std@@V?$allocator@D@2@@std@@QAEAAV12@ABV12@@Z 100ba5b0 f i xls.obj
 0002:000485f0       ?append@?$basic_string@DU?$char_traits@D@std@@V?$allocator@D@2@@std@@QAEAAV12@PBD@Z 100ba5f0 f i xls.obj
 0002:00048650       ?find@?$basic_string@DU?$char_traits@D@std@@V?$allocator@D@2@@std@@QBEIPBDII@Z 100ba650 f i xls.obj
 0002:000487a0       ?find@?$char_traits@D@std@@SAPBDPBDIABD@Z 100ba7a0 f i xls.obj
 0002:000487d0       ?get_allocator@?$basic_string@DU?$char_traits@D@std@@V?$allocator@D@2@@std@@QBE?AV?$allocator@D@2@XZ 100ba7d0 f i xls.obj
 0002:00048810       ?capacity@?$vector@V?$basic_string@DU?$char_traits@D@std@@V?$allocator@D@2@@std@@V?$allocator@V?$basic_string@DU?$char_traits@D@std@@V?$allocator@D@2@@std@@@2@@std@@QBEIXZ 100ba810 f i xls.obj
 0002:00048870       ?end@?$vector@V?$basic_string@DU?$char_traits@D@std@@V?$allocator@D@2@@std@@V?$allocator@V?$basic_string@DU?$char_traits@D@std@@V?$allocator@D@2@@std@@@2@@std@@QAE?AV?$_Vector_iterator@V?$basic_string@DU?$char_traits@D@std@@V?$allocator@D@2@@std@@V?$allocator@V?$basic_string@DU?$char_traits@D@std@@V?$allocator@D@2@@std@@@2@@2@XZ 100ba870 f i xls.obj
 0002:000488d0       ?insert@?$vector@V?$basic_string@DU?$char_traits@D@std@@V?$allocator@D@2@@std@@V?$allocator@V?$basic_string@DU?$char_traits@D@std@@V?$allocator@D@2@@std@@@2@@std@@QAE?AV?$_Vector_iterator@V?$basic_string@DU?$char_traits@D@std@@V?$allocator@D@2@@std@@V?$allocator@V?$basic_string@DU?$char_traits@D@std@@V?$allocator@D@2@@std@@@2@@2@V?$_Vector_const_iterator@V?$basic_string@DU?$char_traits@D@std@@V?$allocator@D@2@@std@@V?$allocator@V?$basic_string@DU?$char_traits@D@std@@V?$allocator@D@2@@std@@@2@@2@ABV?$basic_string@DU?$char_traits@D@std@@V?$allocator@D@2@@2@@Z 100ba8d0 f i xls.obj
 0002:00048a60       ?_Buy@?$vector@V?$basic_string@DU?$char_traits@D@std@@V?$allocator@D@2@@std@@V?$allocator@V?$basic_string@DU?$char_traits@D@std@@V?$allocator@D@2@@std@@@2@@std@@IAE_NI@Z 100baa60 f i xls.obj
 0002:00048b20       ?_Ufill@?$vector@V?$basic_string@DU?$char_traits@D@std@@V?$allocator@D@2@@std@@V?$allocator@V?$basic_string@DU?$char_traits@D@std@@V?$allocator@D@2@@std@@@2@@std@@IAEPAV?$basic_string@DU?$char_traits@D@std@@V?$allocator@D@2@@2@PAV32@IABV32@@Z 100bab20 f i xls.obj
 0002:00048b80       ?_Orphan_range@?$vector@V?$basic_string@DU?$char_traits@D@std@@V?$allocator@D@2@@std@@V?$allocator@V?$basic_string@DU?$char_traits@D@std@@V?$allocator@D@2@@std@@@2@@std@@IBEXPAV?$basic_string@DU?$char_traits@D@std@@V?$allocator@D@2@@2@0@Z 100bab80 f i xls.obj
 0002:00048c70       ??0?$_Vector_val@V?$basic_string@DU?$char_traits@D@std@@V?$allocator@D@2@@std@@V?$allocator@V?$basic_string@DU?$char_traits@D@std@@V?$allocator@D@2@@std@@@2@@std@@IAE@V?$allocator@V?$basic_string@DU?$char_traits@D@std@@V?$allocator@D@2@@std@@@1@@Z 100bac70 f i xls.obj
 0002:00048ce0       ??0?$allocator@V?$basic_string@DU?$char_traits@D@std@@V?$allocator@D@2@@std@@@std@@QAE@XZ 100bace0 f i xls.obj
 0002:00048d00       ?capacity@?$vector@UST_CELLS@@V?$allocator@UST_CELLS@@@std@@@std@@QBEIXZ 100bad00 f i xls.obj
 0002:00048d60       ?end@?$vector@UST_CELLS@@V?$allocator@UST_CELLS@@@std@@@std@@QAE?AV?$_Vector_iterator@UST_CELLS@@V?$allocator@UST_CELLS@@@std@@@2@XZ 100bad60 f i xls.obj
 0002:00048dc0       ?insert@?$vector@UST_CELLS@@V?$allocator@UST_CELLS@@@std@@@std@@QAE?AV?$_Vector_iterator@UST_CELLS@@V?$allocator@UST_CELLS@@@std@@@2@V?$_Vector_const_iterator@UST_CELLS@@V?$allocator@UST_CELLS@@@std@@@2@ABUST_CELLS@@@Z 100badc0 f i xls.obj
 0002:00048f50       ?_Ufill@?$vector@UST_CELLS@@V?$allocator@UST_CELLS@@@std@@@std@@IAEPAUST_CELLS@@PAU3@IABU3@@Z 100baf50 f i xls.obj
 0002:00048fb0       ?_Orphan_range@?$vector@UST_CELLS@@V?$allocator@UST_CELLS@@@std@@@std@@IBEXPAUST_CELLS@@0@Z 100bafb0 f i xls.obj
 0002:000490a0       ?append@?$basic_string@DU?$char_traits@D@std@@V?$allocator@D@2@@std@@QAEAAV12@ABV12@II@Z 100bb0a0 f i xls.obj
 0002:000491c0       ?append@?$basic_string@DU?$char_traits@D@std@@V?$allocator@D@2@@std@@QAEAAV12@PBDI@Z 100bb1c0 f i xls.obj
 0002:00049310       ?begin@?$vector@V?$basic_string@DU?$char_traits@D@std@@V?$allocator@D@2@@std@@V?$allocator@V?$basic_string@DU?$char_traits@D@std@@V?$allocator@D@2@@std@@@2@@std@@QAE?AV?$_Vector_iterator@V?$basic_string@DU?$char_traits@D@std@@V?$allocator@D@2@@std@@V?$allocator@V?$basic_string@DU?$char_traits@D@std@@V?$allocator@D@2@@std@@@2@@2@XZ 100bb310 f i xls.obj
 0002:00049370       ?max_size@?$vector@V?$basic_string@DU?$char_traits@D@std@@V?$allocator@D@2@@std@@V?$allocator@V?$basic_string@DU?$char_traits@D@std@@V?$allocator@D@2@@std@@@2@@std@@QBEIXZ 100bb370 f i xls.obj
 0002:000493a0       ?_Insert_n@?$vector@V?$basic_string@DU?$char_traits@D@std@@V?$allocator@D@2@@std@@V?$allocator@V?$basic_string@DU?$char_traits@D@std@@V?$allocator@D@2@@std@@@2@@std@@IAEXV?$_Vector_const_iterator@V?$basic_string@DU?$char_traits@D@std@@V?$allocator@D@2@@std@@V?$allocator@V?$basic_string@DU?$char_traits@D@std@@V?$allocator@D@2@@std@@@2@@2@IABV?$basic_string@DU?$char_traits@D@std@@V?$allocator@D@2@@2@@Z 100bb3a0 f i xls.obj
 0002:00049980       ?_Xlen@?$vector@V?$basic_string@DU?$char_traits@D@std@@V?$allocator@D@2@@std@@V?$allocator@V?$basic_string@DU?$char_traits@D@std@@V?$allocator@D@2@@std@@@2@@std@@KAXXZ 100bb980 f i xls.obj
 0002:00049a30       ??0?$_Container_base_aux_alloc_empty@V?$allocator@V?$basic_string@DU?$char_traits@D@std@@V?$allocator@D@2@@std@@@std@@@std@@IAE@V?$allocator@V?$basic_string@DU?$char_traits@D@std@@V?$allocator@D@2@@std@@@1@@Z 100bba30 f i xls.obj
 0002:00049a70       ??0?$allocator@V?$basic_string@DU?$char_traits@D@std@@V?$allocator@D@2@@std@@@std@@QAE@ABV01@@Z 100bba70 f i xls.obj
 0002:00049a90       ?allocate@?$allocator@V?$basic_string@DU?$char_traits@D@std@@V?$allocator@D@2@@std@@@std@@QAEPAV?$basic_string@DU?$char_traits@D@std@@V?$allocator@D@2@@2@I@Z 100bba90 f i xls.obj
 0002:00049ad0       ?begin@?$vector@UST_CELLS@@V?$allocator@UST_CELLS@@@std@@@std@@QAE?AV?$_Vector_iterator@UST_CELLS@@V?$allocator@UST_CELLS@@@std@@@2@XZ 100bbad0 f i xls.obj
 0002:00049b30       ?_Insert_n@?$vector@UST_CELLS@@V?$allocator@UST_CELLS@@@std@@@std@@IAEXV?$_Vector_const_iterator@UST_CELLS@@V?$allocator@UST_CELLS@@@std@@@2@IABUST_CELLS@@@Z 100bbb30 f i xls.obj
 0002:0004a110       ??0?$_Vector_iterator@V?$basic_string@DU?$char_traits@D@std@@V?$allocator@D@2@@std@@V?$allocator@V?$basic_string@DU?$char_traits@D@std@@V?$allocator@D@2@@std@@@2@@std@@QAE@PAV?$basic_string@DU?$char_traits@D@std@@V?$allocator@D@2@@1@PBV_Container_base_secure@1@@Z 100bc110 f i xls.obj
 0002:0004a150       ??H?$_Vector_iterator@V?$basic_string@DU?$char_traits@D@std@@V?$allocator@D@2@@std@@V?$allocator@V?$basic_string@DU?$char_traits@D@std@@V?$allocator@D@2@@std@@@2@@std@@QBE?AV01@H@Z 100bc150 f i xls.obj
 0002:0004a260       ??G?$_Vector_const_iterator@V?$basic_string@DU?$char_traits@D@std@@V?$allocator@D@2@@std@@V?$allocator@V?$basic_string@DU?$char_traits@D@std@@V?$allocator@D@2@@std@@@2@@std@@QBEHABV01@@Z 100bc260 f i xls.obj
 0002:0004a2b0       ??0?$_Vector_iterator@UST_CELLS@@V?$allocator@UST_CELLS@@@std@@@std@@QAE@PAUST_CELLS@@PBV_Container_base_secure@1@@Z 100bc2b0 f i xls.obj
 0002:0004a2f0       ??H?$_Vector_iterator@UST_CELLS@@V?$allocator@UST_CELLS@@@std@@@std@@QBE?AV01@H@Z 100bc2f0 f i xls.obj
 0002:0004a400       ??G?$_Vector_const_iterator@UST_CELLS@@V?$allocator@UST_CELLS@@@std@@@std@@QBEHABV01@@Z 100bc400 f i xls.obj
 0002:0004a450       ??0ST_CELLS@@QAE@ABU0@@Z   100bc450 f i xls.obj
 0002:0004a490       ??0?$_Vector_iterator@V?$basic_string@DU?$char_traits@D@std@@V?$allocator@D@2@@std@@V?$allocator@V?$basic_string@DU?$char_traits@D@std@@V?$allocator@D@2@@std@@@2@@std@@QAE@ABV01@@Z 100bc490 f i xls.obj
 0002:0004a4d0       ??0?$_Vector_iterator@UST_CELLS@@V?$allocator@UST_CELLS@@@std@@@std@@QAE@ABV01@@Z 100bc4d0 f i xls.obj
 0002:0004a510       ??0?$vector@V?$basic_string@DU?$char_traits@D@std@@V?$allocator@D@2@@std@@V?$allocator@V?$basic_string@DU?$char_traits@D@std@@V?$allocator@D@2@@std@@@2@@std@@QAE@ABV01@@Z 100bc510 f i xls.obj
 0002:0004a690       ?max_size@?$allocator@V?$basic_string@DU?$char_traits@D@std@@V?$allocator@D@2@@std@@@std@@QBEIXZ 100bc690 f i xls.obj
 0002:0004a6f0       ??Y?$_Vector_iterator@V?$basic_string@DU?$char_traits@D@std@@V?$allocator@D@2@@std@@V?$allocator@V?$basic_string@DU?$char_traits@D@std@@V?$allocator@D@2@@std@@@2@@std@@QAEAAV01@H@Z 100bc6f0 f i xls.obj
 0002:0004a730       ??0?$_Vector_const_iterator@V?$basic_string@DU?$char_traits@D@std@@V?$allocator@D@2@@std@@V?$allocator@V?$basic_string@DU?$char_traits@D@std@@V?$allocator@D@2@@std@@@2@@std@@QAE@PAV?$basic_string@DU?$char_traits@D@std@@V?$allocator@D@2@@1@PBV_Container_base_secure@1@@Z 100bc730 f i xls.obj
 0002:0004a840       ?_Compat@?$_Vector_const_iterator@V?$basic_string@DU?$char_traits@D@std@@V?$allocator@D@2@@std@@V?$allocator@V?$basic_string@DU?$char_traits@D@std@@V?$allocator@D@2@@std@@@2@@std@@QBEXABV12@@Z 100bc840 f i xls.obj
 0002:0004a8f0       ??Y?$_Vector_iterator@UST_CELLS@@V?$allocator@UST_CELLS@@@std@@@std@@QAEAAV01@H@Z 100bc8f0 f i xls.obj
 0002:0004a930       ??0?$_Vector_const_iterator@UST_CELLS@@V?$allocator@UST_CELLS@@@std@@@std@@QAE@PAUST_CELLS@@PBV_Container_base_secure@1@@Z 100bc930 f i xls.obj
 0002:0004aa40       ?_Compat@?$_Vector_const_iterator@UST_CELLS@@V?$allocator@UST_CELLS@@@std@@@std@@QBEXABV12@@Z 100bca40 f i xls.obj
 0002:0004aaf0       ??0?$_Ranit@V?$basic_string@DU?$char_traits@D@std@@V?$allocator@D@2@@std@@HPBV12@ABV12@@std@@QAE@XZ 100bcaf0 f i xls.obj
 0002:0004ab20       ??0?$_Ranit@UST_CELLS@@HPBU1@ABU1@@std@@QAE@XZ 100bcb20 f i xls.obj
 0002:0004ab50       ??0?$_Iterator_with_base@Urandom_access_iterator_tag@std@@V?$basic_string@DU?$char_traits@D@std@@V?$allocator@D@2@@2@HPBV32@ABV32@V_Iterator_base@2@@std@@QAE@XZ 100bcb50 f i xls.obj
 0002:0004ab80       ??0?$_Iterator_with_base@Urandom_access_iterator_tag@std@@UST_CELLS@@HPBU3@ABU3@V_Iterator_base@2@@std@@QAE@XZ 100bcb80 f i xls.obj
 0002:0004abb0       ?begin@?$vector@V?$basic_string@DU?$char_traits@D@std@@V?$allocator@D@2@@std@@V?$allocator@V?$basic_string@DU?$char_traits@D@std@@V?$allocator@D@2@@std@@@2@@std@@QBE?AV?$_Vector_const_iterator@V?$basic_string@DU?$char_traits@D@std@@V?$allocator@D@2@@std@@V?$allocator@V?$basic_string@DU?$char_traits@D@std@@V?$allocator@D@2@@std@@@2@@2@XZ 100bcbb0 f i xls.obj
 0002:0004ac10       ?end@?$vector@V?$basic_string@DU?$char_traits@D@std@@V?$allocator@D@2@@std@@V?$allocator@V?$basic_string@DU?$char_traits@D@std@@V?$allocator@D@2@@std@@@2@@std@@QBE?AV?$_Vector_const_iterator@V?$basic_string@DU?$char_traits@D@std@@V?$allocator@D@2@@std@@V?$allocator@V?$basic_string@DU?$char_traits@D@std@@V?$allocator@D@2@@std@@@2@@2@XZ 100bcc10 f i xls.obj
 0002:0004ac70       ??Y?$_Vector_const_iterator@V?$basic_string@DU?$char_traits@D@std@@V?$allocator@D@2@@std@@V?$allocator@V?$basic_string@DU?$char_traits@D@std@@V?$allocator@D@2@@std@@@2@@std@@QAEAAV01@H@Z 100bcc70 f i xls.obj
 0002:0004adc0       ?_Getmycont@_Iterator_base@std@@QBEPBV_Container_base_secure@2@XZ 100bcdc0 f i xls.obj
 0002:0004ade0       ?_Has_container@_Iterator_base@std@@QBE_NXZ 100bcde0 f i xls.obj
 0002:0004ae10       ??Y?$_Vector_const_iterator@UST_CELLS@@V?$allocator@UST_CELLS@@@std@@@std@@QAEAAV01@H@Z 100bce10 f i xls.obj
 0002:0004af60       ??$unchecked_uninitialized_fill_n@PAV?$basic_string@DU?$char_traits@D@std@@V?$allocator@D@2@@std@@IV12@V?$allocator@V?$basic_string@DU?$char_traits@D@std@@V?$allocator@D@2@@std@@@2@@stdext@@YAXPAV?$basic_string@DU?$char_traits@D@std@@V?$allocator@D@2@@std@@IABV12@AAV?$allocator@V?$basic_string@DU?$char_traits@D@std@@V?$allocator@D@2@@std@@@2@@Z 100bcf60 f i xls.obj
 0002:0004afd0       ??$unchecked_uninitialized_fill_n@PAUST_CELLS@@IU1@V?$allocator@UST_CELLS@@@std@@@stdext@@YAXPAUST_CELLS@@IABU1@AAV?$allocator@UST_CELLS@@@std@@@Z 100bcfd0 f i xls.obj
 0002:0004b040       ??$_Umove@PAV?$basic_string@DU?$char_traits@D@std@@V?$allocator@D@2@@std@@@?$vector@V?$basic_string@DU?$char_traits@D@std@@V?$allocator@D@2@@std@@V?$allocator@V?$basic_string@DU?$char_traits@D@std@@V?$allocator@D@2@@std@@@2@@std@@IAEPAV?$basic_string@DU?$char_traits@D@std@@V?$allocator@D@2@@1@PAV21@00@Z 100bd040 f i xls.obj
 0002:0004b090       ??$fill@PAV?$basic_string@DU?$char_traits@D@std@@V?$allocator@D@2@@std@@V12@@std@@YAXPAV?$basic_string@DU?$char_traits@D@std@@V?$allocator@D@2@@0@0ABV10@@Z 100bd090 f i xls.obj
 0002:0004b0d0       ??$_Unchecked_move_backward@PAV?$basic_string@DU?$char_traits@D@std@@V?$allocator@D@2@@std@@PAV12@@stdext@@YAPAV?$basic_string@DU?$char_traits@D@std@@V?$allocator@D@2@@std@@PAV12@00@Z 100bd0d0 f i xls.obj
 0002:0004b170       ??$_Allocate@V?$basic_string@DU?$char_traits@D@std@@V?$allocator@D@2@@std@@@std@@YAPAV?$basic_string@DU?$char_traits@D@std@@V?$allocator@D@2@@0@IPAV10@@Z 100bd170 f i xls.obj
 0002:0004b200       ??$_Umove@PAUST_CELLS@@@?$vector@UST_CELLS@@V?$allocator@UST_CELLS@@@std@@@std@@IAEPAUST_CELLS@@PAU2@00@Z 100bd200 f i xls.obj
 0002:0004b250       ??$fill@PAUST_CELLS@@U1@@std@@YAXPAUST_CELLS@@0ABU1@@Z 100bd250 f i xls.obj
 0002:0004b290       ??$_Unchecked_move_backward@PAUST_CELLS@@PAU1@@stdext@@YAPAUST_CELLS@@PAU1@00@Z 100bd290 f i xls.obj
 0002:0004b330       ??$_Ucopy@V?$_Vector_const_iterator@V?$basic_string@DU?$char_traits@D@std@@V?$allocator@D@2@@std@@V?$allocator@V?$basic_string@DU?$char_traits@D@std@@V?$allocator@D@2@@std@@@2@@std@@@?$vector@V?$basic_string@DU?$char_traits@D@std@@V?$allocator@D@2@@std@@V?$allocator@V?$basic_string@DU?$char_traits@D@std@@V?$allocator@D@2@@std@@@2@@std@@IAEPAV?$basic_string@DU?$char_traits@D@std@@V?$allocator@D@2@@1@V?$_Vector_const_iterator@V?$basic_string@DU?$char_traits@D@std@@V?$allocator@D@2@@std@@V?$allocator@V?$basic_string@DU?$char_traits@D@std@@V?$allocator@D@2@@std@@@2@@1@0PAV21@@Z 100bd330 f i xls.obj
 0002:0004b440       ??$_Uninit_fill_n@PAV?$basic_string@DU?$char_traits@D@std@@V?$allocator@D@2@@std@@IV12@V?$allocator@V?$basic_string@DU?$char_traits@D@std@@V?$allocator@D@2@@std@@@2@@std@@YAXPAV?$basic_string@DU?$char_traits@D@std@@V?$allocator@D@2@@0@IABV10@AAV?$allocator@V?$basic_string@DU?$char_traits@D@std@@V?$allocator@D@2@@std@@@0@U_Nonscalar_ptr_iterator_tag@0@U_Range_checked_iterator_tag@0@@Z 100bd440 f i xls.obj
 0002:0004b540       ??$_Uninit_fill_n@PAUST_CELLS@@IU1@V?$allocator@UST_CELLS@@@std@@@std@@YAXPAUST_CELLS@@IABU1@AAV?$allocator@UST_CELLS@@@0@U_Nonscalar_ptr_iterator_tag@0@U_Range_checked_iterator_tag@0@@Z 100bd540 f i xls.obj
 0002:0004b640       ??$_Unchecked_uninitialized_move@PAV?$basic_string@DU?$char_traits@D@std@@V?$allocator@D@2@@std@@PAV12@V?$allocator@V?$basic_string@DU?$char_traits@D@std@@V?$allocator@D@2@@std@@@2@@stdext@@YAPAV?$basic_string@DU?$char_traits@D@std@@V?$allocator@D@2@@std@@PAV12@00AAV?$allocator@V?$basic_string@DU?$char_traits@D@std@@V?$allocator@D@2@@std@@@2@@Z 100bd640 f i xls.obj
 0002:0004b6c0       ??$_Checked_base@PAV?$basic_string@DU?$char_traits@D@std@@V?$allocator@D@2@@std@@@std@@YAPAV?$basic_string@DU?$char_traits@D@std@@V?$allocator@D@2@@0@AAPAV10@@Z 100bd6c0 f i xls.obj
 0002:0004b750       ??$_Fill@PAV?$basic_string@DU?$char_traits@D@std@@V?$allocator@D@2@@std@@V12@@std@@YAXPAV?$basic_string@DU?$char_traits@D@std@@V?$allocator@D@2@@0@0ABV10@@Z 100bd750 f i xls.obj
 0002:0004b7b0       ??$_Iter_random@PAV?$basic_string@DU?$char_traits@D@std@@V?$allocator@D@2@@std@@PAV12@@std@@YA?AUrandom_access_iterator_tag@0@ABQAV?$basic_string@DU?$char_traits@D@std@@V?$allocator@D@2@@0@0@Z 100bd7b0 f i xls.obj
 0002:0004b810       ??$_Move_cat@PAV?$basic_string@DU?$char_traits@D@std@@V?$allocator@D@2@@std@@@std@@YA?AU_Swap_move_tag@0@ABQAV?$basic_string@DU?$char_traits@D@std@@V?$allocator@D@2@@0@@Z 100bd810 f i xls.obj
 0002:0004b870       ??$_Move_backward_opt@PAV?$basic_string@DU?$char_traits@D@std@@V?$allocator@D@2@@std@@PAV12@@std@@YAPAV?$basic_string@DU?$char_traits@D@std@@V?$allocator@D@2@@0@PAV10@00Urandom_access_iterator_tag@0@U_Swap_move_tag@0@U_Range_checked_iterator_tag@0@@Z 100bd870 f i xls.obj
 0002:0004b900       ??$_Unchecked_uninitialized_move@PAUST_CELLS@@PAU1@V?$allocator@UST_CELLS@@@std@@@stdext@@YAPAUST_CELLS@@PAU1@00AAV?$allocator@UST_CELLS@@@std@@@Z 100bd900 f i xls.obj
 0002:0004b980       ??$_Checked_base@PAUST_CELLS@@@std@@YAPAUST_CELLS@@AAPAU1@@Z 100bd980 f i xls.obj
 0002:0004ba10       ??$_Fill@PAUST_CELLS@@U1@@std@@YAXPAUST_CELLS@@0ABU1@@Z 100bda10 f i xls.obj
 0002:0004ba70       ??$_Iter_random@PAUST_CELLS@@PAU1@@std@@YA?AUrandom_access_iterator_tag@0@ABQAUST_CELLS@@0@Z 100bda70 f i xls.obj
 0002:0004bad0       ??$_Move_cat@PAUST_CELLS@@@std@@YA?AU_Undefined_move_tag@0@ABQAUST_CELLS@@@Z 100bdad0 f i xls.obj
 0002:0004bb30       ??$_Move_backward_opt@PAUST_CELLS@@PAU1@Urandom_access_iterator_tag@std@@U_Undefined_move_tag@3@@std@@YAPAUST_CELLS@@PAU1@00Urandom_access_iterator_tag@0@U_Undefined_move_tag@0@U_Range_checked_iterator_tag@0@@Z 100bdb30 f i xls.obj
 0002:0004bba0       ??$unchecked_uninitialized_copy@V?$_Vector_const_iterator@V?$basic_string@DU?$char_traits@D@std@@V?$allocator@D@2@@std@@V?$allocator@V?$basic_string@DU?$char_traits@D@std@@V?$allocator@D@2@@std@@@2@@std@@PAV?$basic_string@DU?$char_traits@D@std@@V?$allocator@D@2@@2@V?$allocator@V?$basic_string@DU?$char_traits@D@std@@V?$allocator@D@2@@std@@@2@@stdext@@YAPAV?$basic_string@DU?$char_traits@D@std@@V?$allocator@D@2@@std@@V?$_Vector_const_iterator@V?$basic_string@DU?$char_traits@D@std@@V?$allocator@D@2@@std@@V?$allocator@V?$basic_string@DU?$char_traits@D@std@@V?$allocator@D@2@@std@@@2@@2@0PAV12@AAV?$allocator@V?$basic_string@DU?$char_traits@D@std@@V?$allocator@D@2@@std@@@2@@Z 100bdba0 f i xls.obj
 0002:0004bce0       ??4ST_CELLS@@QAEAAU0@ABU0@@Z 100bdce0 f i xls.obj
 0002:0004bd20       ??4?$vector@V?$basic_string@DU?$char_traits@D@std@@V?$allocator@D@2@@std@@V?$allocator@V?$basic_string@DU?$char_traits@D@std@@V?$allocator@D@2@@std@@@2@@std@@QAEAAV01@ABV01@@Z 100bdd20 f i xls.obj
 0002:0004bf30       ?construct@?$allocator@V?$basic_string@DU?$char_traits@D@std@@V?$allocator@D@2@@std@@@std@@QAEXPAV?$basic_string@DU?$char_traits@D@std@@V?$allocator@D@2@@2@ABV32@@Z 100bdf30 f i xls.obj
 0002:0004bf70       ?construct@?$allocator@UST_CELLS@@@std@@QAEXPAUST_CELLS@@ABU3@@Z 100bdf70 f i xls.obj
 0002:0004bfb0       ?clear@?$vector@V?$basic_string@DU?$char_traits@D@std@@V?$allocator@D@2@@std@@V?$allocator@V?$basic_string@DU?$char_traits@D@std@@V?$allocator@D@2@@std@@@2@@std@@QAEXXZ 100bdfb0 f i xls.obj
 0002:0004c0e0       ?erase@?$vector@V?$basic_string@DU?$char_traits@D@std@@V?$allocator@D@2@@std@@V?$allocator@V?$basic_string@DU?$char_traits@D@std@@V?$allocator@D@2@@std@@@2@@std@@QAE?AV?$_Vector_iterator@V?$basic_string@DU?$char_traits@D@std@@V?$allocator@D@2@@std@@V?$allocator@V?$basic_string@DU?$char_traits@D@std@@V?$allocator@D@2@@std@@@2@@2@V?$_Vector_const_iterator@V?$basic_string@DU?$char_traits@D@std@@V?$allocator@D@2@@std@@V?$allocator@V?$basic_string@DU?$char_traits@D@std@@V?$allocator@D@2@@std@@@2@@2@0@Z 100be0e0 f i xls.obj
 0002:0004c340       ?_Make_iter@?$vector@V?$basic_string@DU?$char_traits@D@std@@V?$allocator@D@2@@std@@V?$allocator@V?$basic_string@DU?$char_traits@D@std@@V?$allocator@D@2@@std@@@2@@std@@QBE?AV?$_Vector_iterator@V?$basic_string@DU?$char_traits@D@std@@V?$allocator@D@2@@std@@V?$allocator@V?$basic_string@DU?$char_traits@D@std@@V?$allocator@D@2@@std@@@2@@2@V?$_Vector_const_iterator@V?$basic_string@DU?$char_traits@D@std@@V?$allocator@D@2@@std@@V?$allocator@V?$basic_string@DU?$char_traits@D@std@@V?$allocator@D@2@@std@@@2@@2@@Z 100be340 f i xls.obj
 0002:0004c3f0       ??9?$_Vector_const_iterator@V?$basic_string@DU?$char_traits@D@std@@V?$allocator@D@2@@std@@V?$allocator@V?$basic_string@DU?$char_traits@D@std@@V?$allocator@D@2@@std@@@2@@std@@QBE_NABV01@@Z 100be3f0 f i xls.obj
 0002:0004c440       ??M?$_Vector_const_iterator@V?$basic_string@DU?$char_traits@D@std@@V?$allocator@D@2@@std@@V?$allocator@V?$basic_string@DU?$char_traits@D@std@@V?$allocator@D@2@@std@@@2@@std@@QBE_NABV01@@Z 100be440 f i xls.obj
 0002:0004c490       ??8?$_Vector_const_iterator@V?$basic_string@DU?$char_traits@D@std@@V?$allocator@D@2@@std@@V?$allocator@V?$basic_string@DU?$char_traits@D@std@@V?$allocator@D@2@@std@@@2@@std@@QBE_NABV01@@Z 100be490 f i xls.obj
 0002:0004c4e0       ??$_Uninit_move@PAV?$basic_string@DU?$char_traits@D@std@@V?$allocator@D@2@@std@@PAV12@V?$allocator@V?$basic_string@DU?$char_traits@D@std@@V?$allocator@D@2@@std@@@2@@std@@YAPAV?$basic_string@DU?$char_traits@D@std@@V?$allocator@D@2@@0@PAV10@00AAV?$allocator@V?$basic_string@DU?$char_traits@D@std@@V?$allocator@D@2@@std@@@0@U_Swap_move_tag@0@U_Range_checked_iterator_tag@0@@Z 100be4e0 f i xls.obj
 0002:0004c6b0       ??$_Checked_base@PAV?$basic_string@DU?$char_traits@D@std@@V?$allocator@D@2@@std@@@std@@YAPAV?$basic_string@DU?$char_traits@D@std@@V?$allocator@D@2@@0@AAPAV10@U_Unchanged_checked_iterator_base_type_tag@0@@Z 100be6b0 f i xls.obj
 0002:0004c6c0       ??$_Debug_range@PAV?$basic_string@DU?$char_traits@D@std@@V?$allocator@D@2@@std@@@std@@YAXPAV?$basic_string@DU?$char_traits@D@std@@V?$allocator@D@2@@0@0PB_WI@Z 100be6c0 f i xls.obj
 0002:0004c720       ??$_Move_backward_opt@PAV?$basic_string@DU?$char_traits@D@std@@V?$allocator@D@2@@std@@PAV12@Uforward_iterator_tag@2@@std@@YAPAV?$basic_string@DU?$char_traits@D@std@@V?$allocator@D@2@@0@PAV10@00Uforward_iterator_tag@0@U_Swap_move_tag@0@U_Range_checked_iterator_tag@0@@Z 100be720 f i xls.obj
 0002:0004c790       ??$_Uninit_move@PAUST_CELLS@@PAU1@V?$allocator@UST_CELLS@@@std@@U_Undefined_move_tag@3@@std@@YAPAUST_CELLS@@PAU1@00AAV?$allocator@UST_CELLS@@@0@U_Undefined_move_tag@0@U_Range_checked_iterator_tag@0@@Z 100be790 f i xls.obj
 0002:0004c7c0       ??$_Checked_base@PAUST_CELLS@@@std@@YAPAUST_CELLS@@AAPAU1@U_Unchanged_checked_iterator_base_type_tag@0@@Z 100be7c0 f i xls.obj
 0002:0004c7d0       ??$_Debug_range@PAUST_CELLS@@@std@@YAXPAUST_CELLS@@0PB_WI@Z 100be7d0 f i xls.obj
 0002:0004c830       ??$_Copy_backward_opt@PAUST_CELLS@@PAU1@@std@@YAPAUST_CELLS@@PAU1@00Urandom_access_iterator_tag@0@U_Nonscalar_ptr_iterator_tag@0@U_Range_checked_iterator_tag@0@@Z 100be830 f i xls.obj
 0002:0004c8d0       ??$_Checked_base@V?$_Vector_const_iterator@V?$basic_string@DU?$char_traits@D@std@@V?$allocator@D@2@@std@@V?$allocator@V?$basic_string@DU?$char_traits@D@std@@V?$allocator@D@2@@std@@@2@@std@@@std@@YA?AV?$_Vector_const_iterator@V?$basic_string@DU?$char_traits@D@std@@V?$allocator@D@2@@std@@V?$allocator@V?$basic_string@DU?$char_traits@D@std@@V?$allocator@D@2@@std@@@2@@0@AAV10@@Z 100be8d0 f i xls.obj
 0002:0004c970       ??$_Ptr_cat@V?$_Vector_const_iterator@V?$basic_string@DU?$char_traits@D@std@@V?$allocator@D@2@@std@@V?$allocator@V?$basic_string@DU?$char_traits@D@std@@V?$allocator@D@2@@std@@@2@@std@@PAV?$basic_string@DU?$char_traits@D@std@@V?$allocator@D@2@@2@@std@@YA?AU_Nonscalar_ptr_iterator_tag@0@AAV?$_Vector_const_iterator@V?$basic_string@DU?$char_traits@D@std@@V?$allocator@D@2@@std@@V?$allocator@V?$basic_string@DU?$char_traits@D@std@@V?$allocator@D@2@@std@@@2@@0@AAPAV?$basic_string@DU?$char_traits@D@std@@V?$allocator@D@2@@0@@Z 100be970 f i xls.obj
 0002:0004c9d0       ??$_Uninit_copy@V?$_Vector_const_iterator@V?$basic_string@DU?$char_traits@D@std@@V?$allocator@D@2@@std@@V?$allocator@V?$basic_string@DU?$char_traits@D@std@@V?$allocator@D@2@@std@@@2@@std@@PAV?$basic_string@DU?$char_traits@D@std@@V?$allocator@D@2@@2@V?$allocator@V?$basic_string@DU?$char_traits@D@std@@V?$allocator@D@2@@std@@@2@@std@@YAPAV?$basic_string@DU?$char_traits@D@std@@V?$allocator@D@2@@0@V?$_Vector_const_iterator@V?$basic_string@DU?$char_traits@D@std@@V?$allocator@D@2@@std@@V?$allocator@V?$basic_string@DU?$char_traits@D@std@@V?$allocator@D@2@@std@@@2@@0@0PAV10@AAV?$allocator@V?$basic_string@DU?$char_traits@D@std@@V?$allocator@D@2@@std@@@0@U_Nonscalar_ptr_iterator_tag@0@U_Range_checked_iterator_tag@0@@Z 100be9d0 f i xls.obj
 0002:0004cbb0       ??$unchecked_copy@PAV?$basic_string@DU?$char_traits@D@std@@V?$allocator@D@2@@std@@PAV12@@stdext@@YAPAV?$basic_string@DU?$char_traits@D@std@@V?$allocator@D@2@@std@@PAV12@00@Z 100bebb0 f i xls.obj
 0002:0004cc50       ??$_Ucopy@PAV?$basic_string@DU?$char_traits@D@std@@V?$allocator@D@2@@std@@@?$vector@V?$basic_string@DU?$char_traits@D@std@@V?$allocator@D@2@@std@@V?$allocator@V?$basic_string@DU?$char_traits@D@std@@V?$allocator@D@2@@std@@@2@@std@@IAEPAV?$basic_string@DU?$char_traits@D@std@@V?$allocator@D@2@@1@PAV21@00@Z 100bec50 f i xls.obj
 0002:0004cca0       ??$_Construct@V?$basic_string@DU?$char_traits@D@std@@V?$allocator@D@2@@std@@V12@@std@@YAXPAV?$basic_string@DU?$char_traits@D@std@@V?$allocator@D@2@@0@ABV10@@Z 100beca0 f i xls.obj
 0002:0004cd60       ??$_Construct@UST_CELLS@@U1@@std@@YAXPAUST_CELLS@@ABU1@@Z 100bed60 f i xls.obj
 0002:0004ce20       ??D?$_Vector_const_iterator@V?$basic_string@DU?$char_traits@D@std@@V?$allocator@D@2@@std@@V?$allocator@V?$basic_string@DU?$char_traits@D@std@@V?$allocator@D@2@@std@@@2@@std@@QBEABV?$basic_string@DU?$char_traits@D@std@@V?$allocator@D@2@@1@XZ 100bee20 f i xls.obj
 0002:0004cef0       ??E?$_Vector_const_iterator@V?$basic_string@DU?$char_traits@D@std@@V?$allocator@D@2@@std@@V?$allocator@V?$basic_string@DU?$char_traits@D@std@@V?$allocator@D@2@@std@@@2@@std@@QAEAAV01@XZ 100beef0 f i xls.obj
 0002:0004d030       ??$_Debug_pointer@V?$basic_string@DU?$char_traits@D@std@@V?$allocator@D@2@@std@@@std@@YAXPAV?$basic_string@DU?$char_traits@D@std@@V?$allocator@D@2@@0@PB_WI@Z 100bf030 f i xls.obj
 0002:0004d060       ??$_Swap_adl@V?$basic_string@DU?$char_traits@D@std@@V?$allocator@D@2@@std@@@std@@YAXAAV?$basic_string@DU?$char_traits@D@std@@V?$allocator@D@2@@0@0@Z 100bf060 f i xls.obj
 0002:0004d090       ??$_Iter_cat@PAV?$basic_string@DU?$char_traits@D@std@@V?$allocator@D@2@@std@@@std@@YA?AUrandom_access_iterator_tag@0@ABQAV?$basic_string@DU?$char_traits@D@std@@V?$allocator@D@2@@0@@Z 100bf090 f i xls.obj
 0002:0004d0f0       ??$_Debug_range2@PAV?$basic_string@DU?$char_traits@D@std@@V?$allocator@D@2@@std@@@std@@YAXPAV?$basic_string@DU?$char_traits@D@std@@V?$allocator@D@2@@0@0PB_WIUrandom_access_iterator_tag@0@@Z 100bf0f0 f i xls.obj
 0002:0004d160       ??$unchecked_uninitialized_copy@PAUST_CELLS@@PAU1@V?$allocator@UST_CELLS@@@std@@@stdext@@YAPAUST_CELLS@@PAU1@00AAV?$allocator@UST_CELLS@@@std@@@Z 100bf160 f i xls.obj
 0002:0004d1e0       ??$_Iter_cat@PAUST_CELLS@@@std@@YA?AUrandom_access_iterator_tag@0@ABQAUST_CELLS@@@Z 100bf1e0 f i xls.obj
 0002:0004d240       ??$_Debug_range2@PAUST_CELLS@@@std@@YAXPAUST_CELLS@@0PB_WIUrandom_access_iterator_tag@0@@Z 100bf240 f i xls.obj
 0002:0004d2b0       ??$_Copy_backward_opt@PAUST_CELLS@@PAU1@Uforward_iterator_tag@std@@@std@@YAPAUST_CELLS@@PAU1@00Uforward_iterator_tag@0@U_Nonscalar_ptr_iterator_tag@0@U_Range_checked_iterator_tag@0@@Z 100bf2b0 f i xls.obj
 0002:0004d320       ??$_Checked_base@V?$_Vector_const_iterator@V?$basic_string@DU?$char_traits@D@std@@V?$allocator@D@2@@std@@V?$allocator@V?$basic_string@DU?$char_traits@D@std@@V?$allocator@D@2@@std@@@2@@std@@@std@@YA?AV?$_Vector_const_iterator@V?$basic_string@DU?$char_traits@D@std@@V?$allocator@D@2@@std@@V?$allocator@V?$basic_string@DU?$char_traits@D@std@@V?$allocator@D@2@@std@@@2@@0@AAV10@U_Unchanged_checked_iterator_base_type_tag@0@@Z 100bf320 f i xls.obj
 0002:0004d370       ??$_Debug_range@V?$_Vector_const_iterator@V?$basic_string@DU?$char_traits@D@std@@V?$allocator@D@2@@std@@V?$allocator@V?$basic_string@DU?$char_traits@D@std@@V?$allocator@D@2@@std@@@2@@std@@@std@@YAXV?$_Vector_const_iterator@V?$basic_string@DU?$char_traits@D@std@@V?$allocator@D@2@@std@@V?$allocator@V?$basic_string@DU?$char_traits@D@std@@V?$allocator@D@2@@std@@@2@@0@0PB_WI@Z 100bf370 f i xls.obj
 0002:0004d480       ??$_Copy_opt@PAV?$basic_string@DU?$char_traits@D@std@@V?$allocator@D@2@@std@@PAV12@@std@@YAPAV?$basic_string@DU?$char_traits@D@std@@V?$allocator@D@2@@0@PAV10@00Urandom_access_iterator_tag@0@U_Nonscalar_ptr_iterator_tag@0@U_Range_checked_iterator_tag@0@@Z 100bf480 f i xls.obj
 0002:0004d510       ??$unchecked_uninitialized_copy@PAV?$basic_string@DU?$char_traits@D@std@@V?$allocator@D@2@@std@@PAV12@V?$allocator@V?$basic_string@DU?$char_traits@D@std@@V?$allocator@D@2@@std@@@2@@stdext@@YAPAV?$basic_string@DU?$char_traits@D@std@@V?$allocator@D@2@@std@@PAV12@00AAV?$allocator@V?$basic_string@DU?$char_traits@D@std@@V?$allocator@D@2@@std@@@2@@Z 100bf510 f i xls.obj
 0002:0004d590       ??$swap@DU?$char_traits@D@std@@V?$allocator@D@2@@std@@YAXAAV?$basic_string@DU?$char_traits@D@std@@V?$allocator@D@2@@0@0@Z 100bf590 f i xls.obj
 0002:0004d5b0       ??$_Uninit_copy@PAUST_CELLS@@PAU1@V?$allocator@UST_CELLS@@@std@@@std@@YAPAUST_CELLS@@PAU1@00AAV?$allocator@UST_CELLS@@@0@U_Nonscalar_ptr_iterator_tag@0@U_Range_checked_iterator_tag@0@@Z 100bf5b0 f i xls.obj
 0002:0004d6f0       ??$_Debug_pointer@UST_CELLS@@@std@@YAXPAUST_CELLS@@PB_WI@Z 100bf6f0 f i xls.obj
 0002:0004d720       ??$_Iter_cat@V?$_Vector_const_iterator@V?$basic_string@DU?$char_traits@D@std@@V?$allocator@D@2@@std@@V?$allocator@V?$basic_string@DU?$char_traits@D@std@@V?$allocator@D@2@@std@@@2@@std@@@std@@YA?AUrandom_access_iterator_tag@0@ABV?$_Vector_const_iterator@V?$basic_string@DU?$char_traits@D@std@@V?$allocator@D@2@@std@@V?$allocator@V?$basic_string@DU?$char_traits@D@std@@V?$allocator@D@2@@std@@@2@@0@@Z 100bf720 f i xls.obj
 0002:0004d780       ??$_Debug_range2@V?$_Vector_const_iterator@V?$basic_string@DU?$char_traits@D@std@@V?$allocator@D@2@@std@@V?$allocator@V?$basic_string@DU?$char_traits@D@std@@V?$allocator@D@2@@std@@@2@@std@@@std@@YAXV?$_Vector_const_iterator@V?$basic_string@DU?$char_traits@D@std@@V?$allocator@D@2@@std@@V?$allocator@V?$basic_string@DU?$char_traits@D@std@@V?$allocator@D@2@@std@@@2@@0@0PB_WIUrandom_access_iterator_tag@0@@Z 100bf780 f i xls.obj
 0002:0004d870       ??$_Copy_opt@PAV?$basic_string@DU?$char_traits@D@std@@V?$allocator@D@2@@std@@PAV12@Uforward_iterator_tag@2@@std@@YAPAV?$basic_string@DU?$char_traits@D@std@@V?$allocator@D@2@@0@PAV10@00Uforward_iterator_tag@0@U_Nonscalar_ptr_iterator_tag@0@U_Range_checked_iterator_tag@0@@Z 100bf870 f i xls.obj
 0002:0004d8e0       ??$_Uninit_copy@PAV?$basic_string@DU?$char_traits@D@std@@V?$allocator@D@2@@std@@PAV12@V?$allocator@V?$basic_string@DU?$char_traits@D@std@@V?$allocator@D@2@@std@@@2@@std@@YAPAV?$basic_string@DU?$char_traits@D@std@@V?$allocator@D@2@@0@PAV10@00AAV?$allocator@V?$basic_string@DU?$char_traits@D@std@@V?$allocator@D@2@@std@@@0@U_Nonscalar_ptr_iterator_tag@0@U_Range_checked_iterator_tag@0@@Z 100bf8e0 f i xls.obj
 0002:0004da20       ?swap@?$basic_string@DU?$char_traits@D@std@@V?$allocator@D@2@@std@@QAEXAAV12@@Z 100bfa20 f i xls.obj
 0002:0004dc40       ?_Swap_all@_Container_base_secure@std@@QBEXAAV12@@Z 100bfc40 f i xls.obj
 0002:0004dd60       ??$_Debug_pointer@V?$_Vector_const_iterator@V?$basic_string@DU?$char_traits@D@std@@V?$allocator@D@2@@std@@V?$allocator@V?$basic_string@DU?$char_traits@D@std@@V?$allocator@D@2@@std@@@2@@std@@@std@@YAXAAV?$_Vector_const_iterator@V?$basic_string@DU?$char_traits@D@std@@V?$allocator@D@2@@std@@V?$allocator@V?$basic_string@DU?$char_traits@D@std@@V?$allocator@D@2@@std@@@2@@0@PB_WI@Z 100bfd60 f i xls.obj
 0002:0004dd70       ??$?8DD@std@@YA_NABV?$allocator@D@0@0@Z 100bfd70 f i xls.obj
 0002:0004dd80       ?dumpbuf@@YAXPADJPAE@Z     100bfd80 f   xlstool.obj
 0002:0004ddd0       ?verbose@@YAXPAD@Z         100bfdd0 f   xlstool.obj
 0002:0004de00       ?utf8_decode@@YAPADPBDHPAH0@Z 100bfe00 f   xlstool.obj
 0002:0004e040       ?get_unicode@@YAPADPAEE@Z  100c0040 f   xlstool.obj
 0002:0004e210       ?xls_getColor@@YAKGG@Z     100c0210 f   xlstool.obj
 0002:0004e290       ?xls_showBookInfo@@YAXPAUxlsWorkBook@@@Z 100c0290 f   xlstool.obj
 0002:0004e4a0       ?xls_showBOF@@YAXPAUBOF@@@Z 100c04a0 f   xlstool.obj
 0002:0004e580       ?xls_showBOUNDSHEET@@YAXPAUBOUNDSHEET@@@Z 100c0580 f   xlstool.obj
 0002:0004e640       ?xls_showROW@@YAXPAUst_row_data@@@Z 100c0640 f   xlstool.obj
 0002:0004e6f0       ?xls_showColinfo@@YAXPAUst_colinfo_data@@@Z 100c06f0 f   xlstool.obj
 0002:0004e7e0       ?xls_showCell@@YAXPAUst_cell_data@@@Z 100c07e0 f   xlstool.obj
 0002:0004e8c0       ?xls_showFont@@YAXPAUst_font_data@@@Z 100c08c0 f   xlstool.obj
 0002:0004e990       ?xls_showXF@@YAXPAUst_xf_data@@@Z 100c0990 f   xlstool.obj
 0002:0004ea70       ?xls_getfcell@@YAPADPAUxlsWorkBook@@PAUst_cell_data@@@Z 100c0a70 f   xlstool.obj
 0002:0004ed50       ?xls_getCSS@@YAPADPAUxlsWorkBook@@@Z 100c0d50 f   xlstool.obj
 0002:0004f940       _DllMain@12                100c1940 f   wzSound.obj
 0002:0004f980       ?wzsnd_init@@YAHPAUWZSNDINFO@@@Z 100c1980 f   wzSound.obj
 0002:0004ff00       ?wzsnd_reload_soundtable@@YAXXZ 100c1f00 f   wzSound.obj
 0002:0004ff40       ?wzsnd_reload_musictable@@YAXXZ 100c1f40 f   wzSound.obj
 0002:0004ff80       ?wzsnd_reload_voicetable@@YAXXZ 100c1f80 f   wzSound.obj
 0002:0004ffc0       ?wzsnd_uninit@@YAXXZ       100c1fc0 f   wzSound.obj
 0002:000500d0       ?wzsnd_load_gameplay@@YAXXZ 100c20d0 f   wzSound.obj
 0002:00050100       ?wzsnd_unload_gameplay@@YAXXZ 100c2100 f   wzSound.obj
 0002:00050130       ?wzsnd_play@@YAHHHHMH@Z    100c2130 f   wzSound.obj
 0002:000502a0       ?wzsnd_play_3d@@YAHHPAU_D3DVECTOR@@00HHPAUSND_SOURCEDESC@@@Z 100c22a0 f   wzSound.obj
 0002:00050530       ?wzsnd_update_3d_source@@YAXHPAU_D3DVECTOR@@0PAUSND_SOURCEDESC@@@Z 100c2530 f   wzSound.obj
 0002:00050610       ?wzsnd_update_listener@@YAXPAU_D3DVECTOR@@000@Z 100c2610 f   wzSound.obj
 0002:000506d0       ?wzsnd_getState_sound@@YAHH@Z 100c26d0 f   wzSound.obj
 0002:00050710       ?wzsnd_stop@@YAXH@Z        100c2710 f   wzSound.obj
 0002:00050740       ?wzsnd_stop_all@@YAXXZ     100c2740 f   wzSound.obj
 0002:00050770       ?wzsnd_pause@@YAXH@Z       100c2770 f   wzSound.obj
 0002:000507a0       ?wzsnd_pause_all@@YAXXZ    100c27a0 f   wzSound.obj
 0002:000507d0       ?wzsnd_unpause@@YAXH@Z     100c27d0 f   wzSound.obj
 0002:00050800       ?wzsnd_unpause_all@@YAXXZ  100c2800 f   wzSound.obj
 0002:00050830       ?wzsnd_set_volume@@YAXHM@Z 100c2830 f   wzSound.obj
 0002:00050870       ?wzsnd_set_volume_all@@YAXM@Z 100c2870 f   wzSound.obj
 0002:000508b0       ?wzsnd_set_loop@@YAXHH@Z   100c28b0 f   wzSound.obj
 0002:000508f0       ?wzsnd_load_ui@@YAXXZ      100c28f0 f   wzSound.obj
 0002:00050920       ?wzsnd_unload_ui@@YAXXZ    100c2920 f   wzSound.obj
 0002:00050950       ?wzsnd_play_ui@@YAHHM@Z    100c2950 f   wzSound.obj
 0002:00050990       ?wzsnd_stop_ui@@YAXH@Z     100c2990 f   wzSound.obj
 0002:000509b0       ?wzsnd_play_ambi@@YAHHHHMHH@Z 100c29b0 f   wzSound.obj
 0002:00050a00       ?wzsnd_stop_ambi@@YAXHH@Z  100c2a00 f   wzSound.obj
 0002:00050a40       ?wzsnd_stop_all_ambi@@YAXH@Z 100c2a40 f   wzSound.obj
 0002:00050a70       ?wzsnd_pause_ambi@@YAXH@Z  100c2a70 f   wzSound.obj
 0002:00050aa0       ?wzsnd_pause_all_ambi@@YAXXZ 100c2aa0 f   wzSound.obj
 0002:00050ad0       ?wzsnd_unpause_ambi@@YAXH@Z 100c2ad0 f   wzSound.obj
 0002:00050b00       ?wzsnd_unpause_all_ambi@@YAXXZ 100c2b00 f   wzSound.obj
 0002:00050b30       ?wzsnd_set_volume_ambi@@YAXHM@Z 100c2b30 f   wzSound.obj
 0002:00050b70       ?wzsnd_set_volume_all_ambi@@YAXM@Z 100c2b70 f   wzSound.obj
 0002:00050bb0       ?wzsnd_set_loop_ambi@@YAXHH@Z 100c2bb0 f   wzSound.obj
 0002:00050bf0       ?wzsnd_getState_ambi@@YAHH@Z 100c2bf0 f   wzSound.obj
 0002:00050c10       ?wzsnd_play_voice@@YAHHHMH@Z 100c2c10 f   wzSound.obj
 0002:00050c70       ?wzsnd_stop_voice@@YAXHH@Z 100c2c70 f   wzSound.obj
 0002:00050cb0       ?wzsnd_stop_all_voice@@YAXH@Z 100c2cb0 f   wzSound.obj
 0002:00050ce0       ?wzsnd_pause_voice@@YAXH@Z 100c2ce0 f   wzSound.obj
 0002:00050d10       ?wzsnd_pause_all_voice@@YAXXZ 100c2d10 f   wzSound.obj
 0002:00050d40       ?wzsnd_unpause_voice@@YAXH@Z 100c2d40 f   wzSound.obj
 0002:00050d70       ?wzsnd_unpause_all_voice@@YAXXZ 100c2d70 f   wzSound.obj
 0002:00050da0       ?wzsnd_set_volume_voice@@YAXHM@Z 100c2da0 f   wzSound.obj
 0002:00050de0       ?wzsnd_set_volume_all_voice@@YAXM@Z 100c2de0 f   wzSound.obj
 0002:00050e20       ?wzsnd_set_loop_voice@@YAXHH@Z 100c2e20 f   wzSound.obj
 0002:00050e60       ?wzsnd_getState_voice@@YAHH@Z 100c2e60 f   wzSound.obj
 0002:00050ea0       ?wzsnd_getState_bgm@@YAHH@Z 100c2ea0 f   wzSound.obj
 0002:00050ee0       ?wzsnd_play_bgm@@YAHHHMH@Z 100c2ee0 f   wzSound.obj
 0002:00050f40       ?wzsnd_stop_bgm@@YAXHH@Z   100c2f40 f   wzSound.obj
 0002:00050f80       ?wzsnd_stop_all_bgm@@YAXH@Z 100c2f80 f   wzSound.obj
 0002:00050fb0       ?wzsnd_pause_bgm@@YAXH@Z   100c2fb0 f   wzSound.obj
 0002:00050fe0       ?wzsnd_pause_all_bgm@@YAXXZ 100c2fe0 f   wzSound.obj
 0002:00051010       ?wzsnd_unpause_bgm@@YAXH@Z 100c3010 f   wzSound.obj
 0002:00051040       ?wzsnd_unpause_all_bgm@@YAXXZ 100c3040 f   wzSound.obj
 0002:00051070       ?wzsnd_set_volume_bgm@@YAXHM@Z 100c3070 f   wzSound.obj
 0002:000510b0       ?wzsnd_set_volume_all_bgm@@YAXM@Z 100c30b0 f   wzSound.obj
 0002:000510f0       ?wzsnd_set_loop_bgm@@YAXHH@Z 100c30f0 f   wzSound.obj
 0002:00051130       ?wzsnd_get_interfacesoundtable@@YAHPAUsoundEntry@@@Z 100c3130 f   wzSound.obj
 0002:000512d0       ?wzsnd_get_soundtable@@YAHPAUsoundEntry@@@Z 100c32d0 f   wzSound.obj
 0002:00051440       ?wzsnd_get_soundtableArray@@YAHPAUsoundEntry@@@Z 100c3440 f   wzSound.obj
 0002:000515b0       ?wzsnd_get_ambienttable@@YAHPAUsoundEntry@@@Z 100c35b0 f   wzSound.obj
 0002:00051750       ?wzsnd_set_master_vol@@YAXHH@Z 100c3750 f   wzSound.obj
 0002:000517a0       ?wzsnd_get_master_vol@@YAXPAH0@Z 100c37a0 f   wzSound.obj
 0002:000517f0       ?wzsnd_set_master_mute@@YAX_N@Z 100c37f0 f   wzSound.obj
 0002:00051830       ?wzsnd_get_master_mute@@YA_NXZ 100c3830 f   wzSound.obj
 0002:000518d0       ?wzsnd_set_wav_vol@@YAXHH@Z 100c38d0 f   wzSound.obj
 0002:00051920       ?wzsnd_get_wav_vol@@YAXPAH0@Z 100c3920 f   wzSound.obj
 0002:00051970       ?wzsnd_set_wav_mute@@YAX_N@Z 100c3970 f   wzSound.obj
 0002:000519b0       ?wzsnd_get_wav_mute@@YA_NXZ 100c39b0 f   wzSound.obj
 0002:00051a50       ?wzsnd_set_mic_input_vol@@YAXK@Z 100c3a50 f   wzSound.obj
 0002:00051ab0       ?wzsnd_get_mic_input_vol@@YAXPAK@Z 100c3ab0 f   wzSound.obj
 0002:00051b60       ?wzsnd_set_mic_output_vol@@YAXK@Z 100c3b60 f   wzSound.obj
 0002:00051bc0       ?wzsnd_get_mic_output_vol@@YAXPAK@Z 100c3bc0 f   wzSound.obj
 0002:00051c60       ?wzsnd_set_mic_output_mute@@YAX_N@Z 100c3c60 f   wzSound.obj
 0002:00051ca0       ?wzsnd_get_mic_output_mute@@YA_NXZ 100c3ca0 f   wzSound.obj
 0002:00051d40       ?wzsnd_env_set@@YAXPAUsound_env@@@Z 100c3d40 f   wzSound.obj
 0002:00051d70       ?wzsnd_env_set_preset@@YAXK@Z 100c3d70 f   wzSound.obj
 0002:00051da0       ?wzsnd_env_get@@YAXPAUsound_env@@@Z 100c3da0 f   wzSound.obj
 0002:00051dd0       ?wzsnd_env_disable@@YAXXZ  100c3dd0 f   wzSound.obj
 0002:00051e00       ?wzsnd_env_supported@@YAHXZ 100c3e00 f   wzSound.obj
 0002:00051e30       ?wzsnd_check_channel@@YAXXZ 100c3e30 f   wzSound.obj
 0002:00051e50       ?wzsnd_update_cache@@YAXXZ 100c3e50 f   wzSound.obj
 0002:00051e70       ?wzsnd_cache_maintain_milliseconds_set@@YAXH@Z 100c3e70 f   wzSound.obj
 0002:00051e90       ?wzsnd_cache_maintain_milliseconds_get@@YAHXZ 100c3e90 f   wzSound.obj
 0002:00051eb0       ?wzsnd_cache_on@@YAXXZ     100c3eb0 f   wzSound.obj
 0002:00051ed0       ?wzsnd_cache_off@@YAXXZ    100c3ed0 f   wzSound.obj
 0002:00051ef0       ?wzsnd_cache_is@@YA_NXZ    100c3ef0 f   wzSound.obj
 0002:00051f10       ?wzsnd_cache_size@@YAHXZ   100c3f10 f   wzSound.obj
 0002:000528a0       ??0SND_SOURCEDESC@@QAE@XZ  100c48a0 f i wzSound.obj
 0002:00052910       ??Eiterator@?$_Tree@V?$_Tmap_traits@HUAmbientSnd@@U?$less@H@std@@V?$allocator@U?$pair@$$CBHUAmbientSnd@@@std@@@3@$0A@@std@@@std@@QAEAAV012@XZ 100c4910 f i wzSound.obj
 0002:00052940       _InitializeCriticalSection@4 100c4940 f   kernel32:KERNEL32.dll
 0002:00052946       _DeleteCriticalSection@4   100c4946 f   kernel32:KERNEL32.dll
 0002:0005294c       _LeaveCriticalSection@4    100c494c f   kernel32:KERNEL32.dll
 0002:00052952       _EnterCriticalSection@4    100c4952 f   kernel32:KERNEL32.dll
 0002:00052958       _InterlockedExchange@8     100c4958 f   kernel32:KERNEL32.dll
 0002:0005295e       _GetCurrentDirectoryA@8    100c495e f   kernel32:KERNEL32.dll
 0002:00052964       _GetProcAddress@8          100c4964 f   kernel32:KERNEL32.dll
 0002:0005296a       _LoadLibraryA@4            100c496a f   kernel32:KERNEL32.dll
 0002:00052970       _FreeLibrary@4             100c4970 f   kernel32:KERNEL32.dll
 0002:00052976       _Sleep@4                   100c4976 f   kernel32:KERNEL32.dll
 0002:0005297c       _GetLastError@0            100c497c f   kernel32:KERNEL32.dll
 0002:00052982       _LocalFree@4               100c4982 f   kernel32:KERNEL32.dll
 0002:00052988       _LocalAlloc@8              100c4988 f   kernel32:KERNEL32.dll
 0002:0005298e       _OutputDebugStringA@4      100c498e f   kernel32:KERNEL32.dll
 0002:00052994       _GetFileAttributesA@4      100c4994 f   kernel32:KERNEL32.dll
 0002:0005299a       _GetModuleFileNameA@12     100c499a f   kernel32:KERNEL32.dll
 0002:000529a0       _GetDriveTypeA@4           100c49a0 f   kernel32:KERNEL32.dll
 0002:000529a6       _MulDiv@12                 100c49a6 f   kernel32:KERNEL32.dll
 0002:000529ac       _GetDesktopWindow@0        100c49ac f   user32:USER32.dll
 0002:000529b2       _CoUninitialize@0          100c49b2 f   ole32:ole32.dll
 0002:000529b8       _CoInitialize@4            100c49b8 f   ole32:ole32.dll
 0002:000529c0       ??0_Init_locks@std@@QAE@XZ 100c49c0 f   libcpmtd:xlock.obj
 0002:00052a10       ??1_Init_locks@std@@QAE@XZ 100c4a10 f   libcpmtd:xlock.obj
 0002:00052a60       ?_Init_locks_ctor@_Init_locks@std@@CAXPAV12@@Z 100c4a60 f   libcpmtd:xlock.obj
 0002:00052ab0       ?_Init_locks_dtor@_Init_locks@std@@CAXPAV12@@Z 100c4ab0 f   libcpmtd:xlock.obj
 0002:00052b00       ??0_Lockit@std@@QAE@XZ     100c4b00 f   libcpmtd:xlock.obj
 0002:00052b30       ??0_Lockit@std@@QAE@H@Z    100c4b30 f   libcpmtd:xlock.obj
 0002:00052b70       ??1_Lockit@std@@QAE@XZ     100c4b70 f   libcpmtd:xlock.obj
 0002:00052ba0       ?_Lockit_ctor@_Lockit@std@@CAXPAV12@@Z 100c4ba0 f   libcpmtd:xlock.obj
 0002:00052bc0       ?_Lockit_ctor@_Lockit@std@@CAXPAV12@H@Z 100c4bc0 f   libcpmtd:xlock.obj
 0002:00052bf0       ?_Lockit_dtor@_Lockit@std@@CAXPAV12@@Z 100c4bf0 f   libcpmtd:xlock.obj
 0002:00052c10       ?_Lockit_ctor@_Lockit@std@@SAXH@Z 100c4c10 f   libcpmtd:xlock.obj
 0002:00052c30       ?_Lockit_dtor@_Lockit@std@@SAXH@Z 100c4c30 f   libcpmtd:xlock.obj
 0002:00052c50       ?_Debug_message@std@@YAXPBD0@Z 100c4c50 f   libcpmtd:stdthrow.obj
 0002:00052cc0       ?_Debug_message@std@@YAXPB_W0I@Z 100c4cc0 f   libcpmtd:stdthrow.obj
 0002:00052cf0       ?_Debug_message@std@@YAXPBG0I@Z 100c4cf0 f   libcpmtd:stdthrow.obj
 0002:00052d10       ?_Throw@std@@YAXABVexception@stdext@@@Z 100c4d10 f   libcpmtd:stdthrow.obj
 0002:00052d40       ?_Xlen@_String_base@std@@SAXXZ 100c4d40 f   libcpmtd:string.obj
 0002:00052dc0       ?_Xran@_String_base@std@@SAXXZ 100c4dc0 f   libcpmtd:string.obj
 0002:00052e40       ??0out_of_range@std@@QAE@ABV?$basic_string@DU?$char_traits@D@std@@V?$allocator@D@2@@1@@Z 100c4e40 f i libcpmtd:string.obj
 0002:00052e70       ??1out_of_range@std@@UAE@XZ 100c4e70 f i libcpmtd:string.obj
 0002:00052e90       ??_Eout_of_range@std@@UAEPAXI@Z 100c4e90 f i libcpmtd:string.obj
 0002:00052e90       ??_Gout_of_range@std@@UAEPAXI@Z 100c4e90 f i libcpmtd:string.obj
 0002:00052ec0       ??0out_of_range@std@@QAE@ABV01@@Z 100c4ec0 f i libcpmtd:string.obj
 0002:00052ef0       ?_Xinvarg@_String_base@std@@SAXXZ 100c4ef0 f   libcpmtd:string.obj
 0002:00052f70       ??0invalid_argument@std@@QAE@ABV?$basic_string@DU?$char_traits@D@std@@V?$allocator@D@2@@1@@Z 100c4f70 f i libcpmtd:string.obj
 0002:00052fa0       ??1invalid_argument@std@@UAE@XZ 100c4fa0 f i libcpmtd:string.obj
 0002:00052fc0       ??_Ginvalid_argument@std@@UAEPAXI@Z 100c4fc0 f i libcpmtd:string.obj
 0002:00052fc0       ??_Einvalid_argument@std@@UAEPAXI@Z 100c4fc0 f i libcpmtd:string.obj
 0002:00052ff0       ??0invalid_argument@std@@QAE@ABV01@@Z 100c4ff0 f i libcpmtd:string.obj
 0002:00053020       ??2@YAPAXIABU_DebugHeapTag_t@std@@PADH@Z 100c5020 f   libcpmtd:xdebug.obj
 0002:000530a0       ??0bad_alloc@std@@QAE@XZ   100c50a0 f i libcpmtd:xdebug.obj
 0002:000530d0       ??_U@YAPAXIABU_DebugHeapTag_t@std@@PADH@Z 100c50d0 f   libcpmtd:xdebug.obj
 0002:000530f0       ??3@YAXPAXABU_DebugHeapTag_t@std@@PADH@Z 100c50f0 f   libcpmtd:xdebug.obj
 0002:00053110       ??_V@YAXPAXABU_DebugHeapTag_t@std@@PADH@Z 100c5110 f   libcpmtd:xdebug.obj
 0002:00053130       ?_DebugHeapTag_func@std@@YAABU_DebugHeapTag_t@1@XZ 100c5130 f   libcpmtd:xdebug.obj
 0002:00053140       __Once                     100c5140 f   libcpmtd:xmtx.obj
 0002:000531a0       __Mtxinit                  100c51a0 f   libcpmtd:xmtx.obj
 0002:000531c0       __Mtxdst                   100c51c0 f   libcpmtd:xmtx.obj
 0002:000531e0       __Mtxlock                  100c51e0 f   libcpmtd:xmtx.obj
 0002:00053200       __Mtxunlock                100c5200 f   libcpmtd:xmtx.obj
 0002:00053220       _ov_clear                  100c5220 f   vorbisfile_static:vorbisfile.obj
 0002:00053320       _ov_open_callbacks         100c5320 f   vorbisfile_static:vorbisfile.obj
 0002:00053ec0       _ov_open                   100c5ec0 f   vorbisfile_static:vorbisfile.obj
 0002:00053f30       _ov_halfrate               100c5f30 f   vorbisfile_static:vorbisfile.obj
 0002:00053ff0       _ov_halfrate_p             100c5ff0 f   vorbisfile_static:vorbisfile.obj
 0002:00054010       _ov_test_callbacks         100c6010 f   vorbisfile_static:vorbisfile.obj
 0002:00054050       _ov_test                   100c6050 f   vorbisfile_static:vorbisfile.obj
 0002:000540a0       _ov_test_open              100c60a0 f   vorbisfile_static:vorbisfile.obj
 0002:000540c0       _ov_streams                100c60c0 f   vorbisfile_static:vorbisfile.obj
 0002:000540d0       _ov_seekable               100c60d0 f   vorbisfile_static:vorbisfile.obj
 0002:000540e0       _ov_bitrate                100c60e0 f   vorbisfile_static:vorbisfile.obj
 0002:00054240       _ov_bitrate_instant        100c6240 f   vorbisfile_static:vorbisfile.obj
 0002:000542b0       _ov_serialnumber           100c62b0 f   vorbisfile_static:vorbisfile.obj
 0002:000542f0       _ov_raw_total              100c62f0 f   vorbisfile_static:vorbisfile.obj
 0002:00054370       _ov_pcm_total              100c6370 f   vorbisfile_static:vorbisfile.obj
 0002:000543e0       _ov_time_total             100c63e0 f   vorbisfile_static:vorbisfile.obj
 0002:00054470       _ov_raw_seek               100c6470 f   vorbisfile_static:vorbisfile.obj
 0002:00054790       _ov_pcm_seek_page          100c6790 f   vorbisfile_static:vorbisfile.obj
 0002:00054d80       _ov_pcm_seek               100c6d80 f   vorbisfile_static:vorbisfile.obj
 0002:000553d0       _ov_time_seek              100c73d0 f   vorbisfile_static:vorbisfile.obj
 0002:000554d0       _ov_time_seek_page         100c74d0 f   vorbisfile_static:vorbisfile.obj
 0002:000555d0       _ov_raw_tell               100c75d0 f   vorbisfile_static:vorbisfile.obj
 0002:000555f0       _ov_pcm_tell               100c75f0 f   vorbisfile_static:vorbisfile.obj
 0002:00055610       _ov_time_tell              100c7610 f   vorbisfile_static:vorbisfile.obj
 0002:00055700       _ov_info                   100c7700 f   vorbisfile_static:vorbisfile.obj
 0002:00055740       _ov_comment                100c7740 f   vorbisfile_static:vorbisfile.obj
 0002:00055780       _ov_read                   100c7780 f   vorbisfile_static:vorbisfile.obj
 0002:00055af0       _ov_read_float             100c7af0 f   vorbisfile_static:vorbisfile.obj
 0002:00055b90       _ov_crosslap               100c7b90 f   vorbisfile_static:vorbisfile.obj
 0002:00056060       _ov_raw_seek_lap           100c8060 f   vorbisfile_static:vorbisfile.obj
 0002:000561d0       _ov_pcm_seek_lap           100c81d0 f   vorbisfile_static:vorbisfile.obj
 0002:000561f0       _ov_pcm_seek_page_lap      100c81f0 f   vorbisfile_static:vorbisfile.obj
 0002:00056210       _ov_time_seek_lap          100c8210 f   vorbisfile_static:vorbisfile.obj
 0002:00056380       _ov_time_seek_page_lap     100c8380 f   vorbisfile_static:vorbisfile.obj
 0002:000563a0       _vorbis_comment_init       100c83a0 f   vorbisfile_static:info.obj
 0002:000563c0       _vorbis_comment_add        100c83c0 f   vorbisfile_static:info.obj
 0002:00056470       _vorbis_comment_add_tag    100c8470 f   vorbisfile_static:info.obj
 0002:00056530       _vorbis_comment_query      100c8530 f   vorbisfile_static:info.obj
 0002:00056660       _vorbis_comment_query_count 100c8660 f   vorbisfile_static:info.obj
 0002:00056720       _vorbis_comment_clear      100c8720 f   vorbisfile_static:info.obj
 0002:00056790       _vorbis_info_blocksize     100c8790 f   vorbisfile_static:info.obj
 0002:000567b0       _vorbis_info_init          100c87b0 f   vorbisfile_static:info.obj
 0002:000567e0       _vorbis_info_clear         100c87e0 f   vorbisfile_static:info.obj
 0002:00056950       _vorbis_synthesis_headerin 100c8950 f   vorbisfile_static:info.obj
 0002:00056ec0       _vorbis_commentheader_out  100c8ec0 f   vorbisfile_static:info.obj
 0002:00057050       _vorbis_analysis_headerout 100c9050 f   vorbisfile_static:info.obj
 0002:00057590       _vorbis_granule_time       100c9590 f   vorbisfile_static:info.obj
 0002:000575c0       _vorbis_block_init         100c95c0 f   vorbisfile_static:block.obj
 0002:00057610       __vorbis_block_alloc       100c9610 f   vorbisfile_static:block.obj
 0002:00057680       __vorbis_block_ripcord     100c9680 f   vorbisfile_static:block.obj
 0002:000576f0       _vorbis_block_clear        100c96f0 f   vorbisfile_static:block.obj
 0002:00057750       _vorbis_analysis_init      100c9750 f   vorbisfile_static:block.obj
 0002:00057b70       _vorbis_dsp_clear          100c9b70 f   vorbisfile_static:block.obj
 0002:00057da0       _vorbis_analysis_buffer    100c9da0 f   vorbisfile_static:block.obj
 0002:00057e70       _vorbis_analysis_wrote     100c9e70 f   vorbisfile_static:block.obj
 0002:000580d0       _vorbis_analysis_blockout  100ca0d0 f   vorbisfile_static:block.obj
 0002:00058400       _vorbis_synthesis_restart  100ca400 f   vorbisfile_static:block.obj
 0002:00058470       _vorbis_synthesis_init     100ca470 f   vorbisfile_static:block.obj
 0002:000584a0       _vorbis_synthesis_blockin  100ca4a0 f   vorbisfile_static:block.obj
 0002:00058af0       _vorbis_synthesis_pcmout   100caaf0 f   vorbisfile_static:block.obj
 0002:00058b50       _vorbis_synthesis_read     100cab50 f   vorbisfile_static:block.obj
 0002:00058b80       _vorbis_synthesis_lapout   100cab80 f   vorbisfile_static:block.obj
 0002:00058d80       _vorbis_window             100cad80 f   vorbisfile_static:block.obj
 0002:00058dc0       _vorbis_synthesis          100cadc0 f   vorbisfile_static:synthesis.obj
 0002:00058f10       _vorbis_synthesis_trackonly 100caf10 f   vorbisfile_static:synthesis.obj
 0002:00058ff0       _vorbis_packet_blocksize   100caff0 f   vorbisfile_static:synthesis.obj
 0002:00059070       _vorbis_synthesis_halfrate 100cb070 f   vorbisfile_static:synthesis.obj
 0002:000590a0       _vorbis_synthesis_halfrate_p 100cb0a0 f   vorbisfile_static:synthesis.obj
 0002:000590b0       _vorbis_analysis           100cb0b0 f   vorbisfile_static:analysis.obj
 0002:00059140       __analysis_output_always   100cb140 f   vorbisfile_static:analysis.obj
 0002:00059290       __analysis_output          100cb290 f   vorbisfile_static:analysis.obj
 0002:00059300       __vp_global_look           100cb300 f   vorbisfile_static:psy.obj
 0002:00059330       __vp_global_free           100cb330 f   vorbisfile_static:psy.obj
 0002:00059350       __vi_gpsy_free             100cb350 f   vorbisfile_static:psy.obj
 0002:00059370       __vi_psy_free              100cb370 f   vorbisfile_static:psy.obj
 0002:00059390       __vp_psy_init              100cb390 f   vorbisfile_static:psy.obj
 0002:0005a0e0       __vp_psy_clear             100cc0e0 f   vorbisfile_static:psy.obj
 0002:0005a1a0       __vp_remove_floor          100cc1a0 f   vorbisfile_static:psy.obj
 0002:0005a200       __vp_noisemask             100cc200 f   vorbisfile_static:psy.obj
 0002:0005a8c0       __vp_tonemask              100cc8c0 f   vorbisfile_static:psy.obj
 0002:0005adb0       __vp_offset_and_mix        100ccdb0 f   vorbisfile_static:psy.obj
 0002:0005ae40       __vp_ampmax_decay          100cce40 f   vorbisfile_static:psy.obj
 0002:0005ae90       __vp_quantize_couple_memo  100cce90 f   vorbisfile_static:psy.obj
 0002:0005b140       __vp_quantize_couple_sort  100cd140 f   vorbisfile_static:psy.obj
 0002:0005b2f0       __vp_noise_normalize_sort  100cd2f0 f   vorbisfile_static:psy.obj
 0002:0005b3c0       __vp_noise_normalize       100cd3c0 f   vorbisfile_static:psy.obj
 0002:0005b630       __vp_couple                100cd630 f   vorbisfile_static:psy.obj
 0002:0005bb60       __ilog                     100cdb60 f   vorbisfile_static:sharedbook.obj
 0002:0005bb70       __float32_pack             100cdb70 f   vorbisfile_static:sharedbook.obj
 0002:0005bc00       __float32_unpack           100cdc00 f   vorbisfile_static:sharedbook.obj
 0002:0005bc50       __make_words               100cdc50 f   vorbisfile_static:sharedbook.obj
 0002:0005bdd0       __book_maptype1_quantvals  100cddd0 f   vorbisfile_static:sharedbook.obj
 0002:0005be40       __book_unquantize          100cde40 f   vorbisfile_static:sharedbook.obj
 0002:0005c030       _vorbis_staticbook_clear   100ce030 f   vorbisfile_static:sharedbook.obj
 0002:0005c100       _vorbis_staticbook_destroy 100ce100 f   vorbisfile_static:sharedbook.obj
 0002:0005c120       _vorbis_book_clear         100ce120 f   vorbisfile_static:sharedbook.obj
 0002:0005c180       _vorbis_book_init_encode   100ce180 f   vorbisfile_static:sharedbook.obj
 0002:0005c1e0       _vorbis_book_init_decode   100ce1e0 f   vorbisfile_static:sharedbook.obj
 0002:0005c630       __best                     100ce630 f   vorbisfile_static:sharedbook.obj
 0002:0005c7e0       _vorbis_book_codeword      100ce7e0 f   vorbisfile_static:sharedbook.obj
 0002:0005c800       _vorbis_book_codelen       100ce800 f   vorbisfile_static:sharedbook.obj
 0002:0005c820       _vorbis_staticbook_pack    100ce820 f   vorbisfile_static:codebook.obj
 0002:0005ca70       _vorbis_staticbook_unpack  100cea70 f   vorbisfile_static:codebook.obj
 0002:0005ccb0       _vorbis_book_encode        100cecb0 f   vorbisfile_static:codebook.obj
 0002:0005ccf0       _vorbis_book_errorv        100cecf0 f   vorbisfile_static:codebook.obj
 0002:0005cd30       _vorbis_book_encodev       100ced30 f   vorbisfile_static:codebook.obj
 0002:0005cd80       _vorbis_book_decode        100ced80 f   vorbisfile_static:codebook.obj
 0002:0005cf10       _vorbis_book_decodevs_add  100cef10 f   vorbisfile_static:codebook.obj
 0002:0005d110       _vorbis_book_decodev_add   100cf110 f   vorbisfile_static:codebook.obj
 0002:0005d4a0       _vorbis_book_decodev_set   100cf4a0 f   vorbisfile_static:codebook.obj
 0002:0005d620       _vorbis_book_decodevv_add  100cf620 f   vorbisfile_static:codebook.obj
 0002:0005d7e0       _vorbis_bitrate_init       100cf7e0 f   vorbisfile_static:bitrate.obj
 0002:0005d9e0       _vorbis_bitrate_clear      100cf9e0 f   vorbisfile_static:bitrate.obj
 0002:0005dac0       _vorbis_bitrate_managed    100cfac0 f   vorbisfile_static:bitrate.obj
 0002:0005dae0       _vorbis_bitrate_addblock   100cfae0 f   vorbisfile_static:bitrate.obj
 0002:0005e780       _vorbis_bitrate_flushpacket 100d0780 f   vorbisfile_static:bitrate.obj
 0002:0005e840       __ve_envelope_init         100d0840 f   vorbisfile_static:envelope.obj
 0002:0005e9e0       __ve_envelope_clear        100d09e0 f   vorbisfile_static:envelope.obj
 0002:0005ea40       __ve_envelope_search       100d0a40 f   vorbisfile_static:envelope.obj
 0002:0005f000       __ve_envelope_mark         100d1000 f   vorbisfile_static:envelope.obj
 0002:0005f0c0       __ve_envelope_shift        100d10c0 f   vorbisfile_static:envelope.obj
 0002:0005f140       _drft_forward              100d1140 f   vorbisfile_static:smallft.obj
 0002:00060500       _drft_backward             100d2500 f   vorbisfile_static:smallft.obj
 0002:00061b10       _drft_init                 100d3b10 f   vorbisfile_static:smallft.obj
 0002:00061d00       _drft_clear                100d3d00 f   vorbisfile_static:smallft.obj
 0002:00061d40       _mdct_init                 100d3d40 f   vorbisfile_static:mdct.obj
 0002:00061f20       _mdct_clear                100d3f20 f   vorbisfile_static:mdct.obj
 0002:00061f60       _mdct_backward             100d3f60 f   vorbisfile_static:mdct.obj
 0002:00062b20       _mdct_forward              100d4b20 f   vorbisfile_static:mdct.obj
 0002:00062fa0       _vorbis_lpc_from_data      100d4fa0 f   vorbisfile_static:lpc.obj
 0002:00063150       _vorbis_lpc_predict        100d5150 f   vorbisfile_static:lpc.obj
 0002:00063220       __vorbis_window_get        100d5220 f   vorbisfile_static:window.obj
 0002:00063230       __vorbis_apply_window      100d5230 f   vorbisfile_static:window.obj
 0002:000643e0       _res0_free_info            100d63e0 f   vorbisfile_static:res0.obj
 0002:00064400       _res0_free_look            100d6400 f   vorbisfile_static:res0.obj
 0002:00064480       _res0_pack                 100d6480 f   vorbisfile_static:res0.obj
 0002:000645a0       _res0_unpack               100d65a0 f   vorbisfile_static:res0.obj
 0002:000646e0       _res0_look                 100d66e0 f   vorbisfile_static:res0.obj
 0002:000648c0       _res0_inverse              100d68c0 f   vorbisfile_static:res0.obj
 0002:00064b40       _res1_forward              100d6b40 f   vorbisfile_static:res0.obj
 0002:000650f0       _res1_class                100d70f0 f   vorbisfile_static:res0.obj
 0002:00065380       _res1_inverse              100d7380 f   vorbisfile_static:res0.obj
 0002:000653e0       _res2_class                100d73e0 f   vorbisfile_static:res0.obj
 0002:000655c0       _res2_forward              100d75c0 f   vorbisfile_static:res0.obj
 0002:00065720       _res2_inverse              100d7720 f   vorbisfile_static:res0.obj
 0002:00065f50       _floor1_fit                100d7f50 f   vorbisfile_static:floor1.obj
 0002:00066af0       _floor1_interpolate_fit    100d8af0 f   vorbisfile_static:floor1.obj
 0002:00066ba0       _floor1_encode             100d8ba0 f   vorbisfile_static:floor1.obj
 0002:00067b80       _vorbis_lsp_to_curve       100d9b80 f   vorbisfile_static:lsp.obj
 0002:00067d00       _vorbis_coslook            100d9d00 f   vorbisfile_static:lsp.obj
 0002:00067d50       _vorbis_invsqlook          100d9d50 f   vorbisfile_static:lsp.obj
 0002:00067da0       _vorbis_invsq2explook      100d9da0 f   vorbisfile_static:lsp.obj
 0002:00067db0       _vorbis_fromdBlook         100d9db0 f   vorbisfile_static:lsp.obj
 0002:00067e10       _vorbis_lpc_to_lsp         100d9e10 f   vorbisfile_static:lsp.obj
 0002:00068330       __RTC_InitBase             100da330 f   LIBCMTD:_init_.obj
 0002:00068360       __RTC_Shutdown             100da360 f   LIBCMTD:_init_.obj
 0002:00068380       __RTC_CheckEsp             100da380 f   LIBCMTD:_stack_.obj
 0002:000683b0       @_RTC_CheckStackVars@8     100da3b0 f   LIBCMTD:_stack_.obj
 0002:00068410       @_RTC_AllocaHelper@12      100da410 f   LIBCMTD:_stack_.obj
 0002:00068450       @_RTC_CheckStackVars2@12   100da450 f   LIBCMTD:_stack_.obj
 0002:00068530       _free                      100da530 f   LIBCMTD:dbgfree.obj
 0002:00068550       _memset                    100da550 f   LIBCMTD:memset.obj
 0002:000685d0       _malloc                    100da5d0 f   LIBCMTD:dbgmalloc.obj
 0002:00068600       _memcpy                    100da600 f   LIBCMTD:memcpy.obj
 0002:00068970       _strcpy                    100da970 f   LIBCMTD:strcat.obj
 0002:00068980       _strcat                    100da980 f   LIBCMTD:strcat.obj
 0002:00068a70       __stricmp_l                100daa70 f   LIBCMTD:stricmp.obj
 0002:00068c20       ??0_LocaleUpdate@@QAE@PAUlocaleinfo_struct@@@Z 100dac20 f i LIBCMTD:stricmp.obj
 0002:00068d00       ??1_LocaleUpdate@@QAE@XZ   100dad00 f i LIBCMTD:stricmp.obj
 0002:00068d30       ?GetLocaleT@_LocaleUpdate@@QAEPAUlocaleinfo_struct@@XZ 100dad30 f i LIBCMTD:stricmp.obj
 0002:00068d40       ___ascii_stricmp           100dad40 f   LIBCMTD:stricmp.obj
 0002:00068dc0       _stricmp                   100dadc0 f   LIBCMTD:stricmp.obj
 0002:00068dc0       __stricmp                  100dadc0 f   LIBCMTD:stricmp.obj
 0002:00068ed0       @__security_check_cookie@4 100daed0 f   LIBCMTD:secchk.obj
 0002:00068ee0       __fpmath                   100daee0 f   LIBCMTD:_fpinit_.obj
 0002:00068f10       __fpclear                  100daf10 f   LIBCMTD:_fpinit_.obj
 0002:00068f20       __cfltcvt_init             100daf20 f   LIBCMTD:_fpinit_.obj
 0002:00068f90       ___setfflag                100daf90 f   LIBCMTD:_fpinit_.obj
 0002:00068fb0       __onexit                   100dafb0 f   LIBCMTD:onexit.obj
 0002:00069180       _atexit                    100db180 f   LIBCMTD:onexit.obj
 0002:000691a0       ___onexitinit              100db1a0 f   LIBCMTD:onexit.obj
 0002:00069200       ??_L@YGXPAXIHP6EX0@Z1@Z    100db200 f   LIBCMTD:ehvecctr.obj
 0002:000692b0       ??_M@YGXPAXIHP6EX0@Z@Z     100db2b0 f   LIBCMTD:ehvecdtr.obj
 0002:00069360       ?__ArrayUnwind@@YGXPAXIHP6EX0@Z@Z 100db360 f   LIBCMTD:ehvecdtr.obj
 0002:00069420       __ftol2_sse                100db420 f   LIBCMTD:ftol2.obj
 0002:00069429       __ftol2_pentium4           100db429 f   LIBCMTD:ftol2.obj
 0002:0006943c       __ftol2_sse_excpt          100db43c f   LIBCMTD:ftol2.obj
 0002:00069456       __ftol2                    100db456 f   LIBCMTD:ftol2.obj
 0002:000694d0       _log                       100db4d0 f   LIBCMTD:_log_.obj
 0002:00069510       __CIlog                    100db510 f   LIBCMTD:_log_.obj
 0002:0006954b       __CIlog_default            100db54b f   LIBCMTD:_log_.obj
 0002:0006955f       __log_default              100db55f     LIBCMTD:_log_.obj
 0002:00069620       _pow                       100db620 f   LIBCMTD:_pow_.obj
 0002:00069660       __CIpow                    100db660 f   LIBCMTD:_pow_.obj
 0002:0006969b       __CIpow_default            100db69b f   LIBCMTD:_pow_.obj
 0002:000696b4       __pow_default              100db6b4     LIBCMTD:_pow_.obj
 0002:000698b0       ?_JumpToContinuation@@YGXPAXPAUEHRegistrationNode@@@Z 100db8b0 f   LIBCMTD:_trnsctrl_.obj
 0002:000698f0       ?_CallMemberFunction0@@YGXPAX0@Z 100db8f0 f   LIBCMTD:_trnsctrl_.obj
 0002:00069900       ?_CallMemberFunction1@@YGXPAX00@Z 100db900 f   LIBCMTD:_trnsctrl_.obj
 0002:00069910       ?_CallMemberFunction2@@YGXPAX00H@Z 100db910 f   LIBCMTD:_trnsctrl_.obj
 0002:00069920       ?_UnwindNestedFrames@@YGXPAUEHRegistrationNode@@PAUEHExceptionRecord@@@Z 100db920 f   LIBCMTD:_trnsctrl_.obj
 0002:00069980       ___CxxFrameHandler         100db980 f   LIBCMTD:_trnsctrl_.obj
 0002:000699c0       ___CxxFrameHandler3        100db9c0 f   LIBCMTD:_trnsctrl_.obj
 0002:00069a00       ___CxxFrameHandler2        100dba00 f   LIBCMTD:_trnsctrl_.obj
 0002:00069a40       ___CxxLongjmpUnwind@4      100dba40 f   LIBCMTD:_trnsctrl_.obj
 0002:00069a70       ?_CallCatchBlock2@@YAPAXPAUEHRegistrationNode@@PBU_s_FuncInfo@@PAXHK@Z 100dba70 f   LIBCMTD:_trnsctrl_.obj
 0002:00069b30       ?_CallSETranslator@@YAHPAUEHExceptionRecord@@PAUEHRegistrationNode@@PAX2PBU_s_FuncInfo@@H1@Z 100dbb30 f   LIBCMTD:_trnsctrl_.obj
 0002:00069cd0       ?_GetRangeOfTrysToCheck@@YAPBU_s_TryBlockMapEntry@@PBU_s_FuncInfo@@HHPAI1@Z 100dbcd0 f   LIBCMTD:_trnsctrl_.obj
 0002:00069d50       __CreateFrameInfo          100dbd50 f   LIBCMTD:_trnsctrl_.obj
 0002:00069d80       __IsExceptionObjectToBeDestroyed 100dbd80 f   LIBCMTD:_trnsctrl_.obj
 0002:00069db0       __FindAndUnlinkFrame       100dbdb0 f   LIBCMTD:_trnsctrl_.obj
 0002:00069e10       __initp_misc_invarg        100dbe10 f   LIBCMTD:invarg.obj
 0002:00069e20       __invalid_parameter        100dbe20 f   LIBCMTD:invarg.obj
 0002:00069e90       __invoke_watson            100dbe90 f   LIBCMTD:invarg.obj
 0002:00069fe0       __set_invalid_parameter_handler 100dbfe0 f   LIBCMTD:invarg.obj
 0002:0006a030       __get_invalid_parameter_handler 100dc030 f   LIBCMTD:invarg.obj
 0002:0006a060       ?_invalid_parameter@@YAXPBG00II@Z 100dc060 f   LIBCMTD:invarg.obj
 0002:0006a090       ?_invoke_watson@@YAXPBG00II@Z 100dc090 f   LIBCMTD:invarg.obj
 0002:0006a0c0       __CrtSetReportHookW2       100dc0c0 f   LIBCMTD:dbgrptw.obj
 0002:0006a3e0       __CrtDbgReportW            100dc3e0 f   LIBCMTD:dbgrptw.obj
 0002:0006a420       __CrtDbgReportWV           100dc420 f i LIBCMTD:dbgrptw.obj
 0002:0006a450       ___crtMessageWindowW       100dc450 f   LIBCMTD:dbgrptw.obj
 0002:0006a850       __invoke_watson_if_error   100dc850 f i LIBCMTD:dbgrptw.obj
 0002:0006a880       __invoke_watson_if_oneof   100dc880 f i LIBCMTD:dbgrptw.obj
 0002:0006a8d0       ?_CrtDbgReportW@@YAHHPBGH00ZZ 100dc8d0 f   LIBCMTD:dbgrptw.obj
 0002:0006a910       _strncpy                   100dc910 f   LIBCMTD:strncpy.obj
 0002:0006aa40       _strlen                    100dca40 f   LIBCMTD:strlen.obj
 0002:0006aad0       ??3@YAXPAX@Z               100dcad0 f   LIBCMTD:dbgdel.obj
 0002:0006abc0       __CxxThrowException@8      100dcbc0 f   LIBCMTD:throw.obj
 0002:0006ac20       ?name@type_info@@QBEPBDPAU__type_info_node@@@Z 100dcc20 f   LIBCMTD:typinfo.obj
 0002:0006ac40       ??1type_info@@UAE@XZ       100dcc40 f   LIBCMTD:typinfo.obj
 0002:0006ac70       ??_Etype_info@@UAEPAXI@Z   100dcc70 f i LIBCMTD:typinfo.obj
 0002:0006ac70       ??_Gtype_info@@UAEPAXI@Z   100dcc70 f i LIBCMTD:typinfo.obj
 0002:0006aca0       ?_name_internal_method@type_info@@QBEPBDPAU__type_info_node@@@Z 100dcca0 f   LIBCMTD:typinfo.obj
 0002:0006acc0       ?_type_info_dtor_internal_method@type_info@@QAEXXZ 100dccc0 f   LIBCMTD:typinfo.obj
 0002:0006ace0       ??8type_info@@QBE_NABV0@@Z 100dcce0 f   LIBCMTD:typinfo.obj
 0002:0006ad10       ??9type_info@@QBE_NABV0@@Z 100dcd10 f   LIBCMTD:typinfo.obj
 0002:0006ad40       ?before@type_info@@QBEHABV1@@Z 100dcd40 f   LIBCMTD:typinfo.obj
 0002:0006ad70       ?raw_name@type_info@@QBEPBDXZ 100dcd70 f   LIBCMTD:typinfo.obj
 0002:0006ad90       ??0type_info@@AAE@ABV0@@Z  100dcd90 f   LIBCMTD:typinfo.obj
 0002:0006adb0       ??4type_info@@AAEAAV0@ABV0@@Z 100dcdb0 f   LIBCMTD:typinfo.obj
 0002:0006add0       ??0exception@std@@QAE@XZ   100dcdd0 f   LIBCMTD:stdexcpt.obj
 0002:0006ae00       ??_Eexception@std@@UAEPAXI@Z 100dce00 f i LIBCMTD:stdexcpt.obj
 0002:0006ae00       ??_Gexception@std@@UAEPAXI@Z 100dce00 f i LIBCMTD:stdexcpt.obj
 0002:0006ae30       ??0exception@std@@QAE@ABQBD@Z 100dce30 f   LIBCMTD:stdexcpt.obj
 0002:0006aec0       ??0exception@std@@QAE@ABQBDH@Z 100dcec0 f   LIBCMTD:stdexcpt.obj
 0002:0006aef0       ??0exception@std@@QAE@ABV01@@Z 100dcef0 f   LIBCMTD:stdexcpt.obj
 0002:0006af90       ??4exception@std@@QAEAAV01@ABV01@@Z 100dcf90 f   LIBCMTD:stdexcpt.obj
 0002:0006b040       ??1exception@std@@UAE@XZ   100dd040 f   LIBCMTD:stdexcpt.obj
 0002:0006b070       ?what@exception@std@@UBEPBDXZ 100dd070 f   LIBCMTD:stdexcpt.obj
 0002:0006b0a0       ??0bad_cast@std@@QAE@PBD@Z 100dd0a0 f   LIBCMTD:stdexcpt.obj
 0002:0006b0d0       ??_Ebad_cast@std@@UAEPAXI@Z 100dd0d0 f i LIBCMTD:stdexcpt.obj
 0002:0006b0d0       ??_Gbad_cast@std@@UAEPAXI@Z 100dd0d0 f i LIBCMTD:stdexcpt.obj
 0002:0006b100       ??0bad_cast@std@@QAE@ABV01@@Z 100dd100 f   LIBCMTD:stdexcpt.obj
 0002:0006b130       ??1bad_cast@std@@UAE@XZ    100dd130 f   LIBCMTD:stdexcpt.obj
 0002:0006b150       ??0bad_typeid@std@@QAE@PBD@Z 100dd150 f   LIBCMTD:stdexcpt.obj
 0002:0006b180       ??_Ebad_typeid@std@@UAEPAXI@Z 100dd180 f i LIBCMTD:stdexcpt.obj
 0002:0006b180       ??_Gbad_typeid@std@@UAEPAXI@Z 100dd180 f i LIBCMTD:stdexcpt.obj
 0002:0006b1b0       ??0bad_typeid@std@@QAE@ABV01@@Z 100dd1b0 f   LIBCMTD:stdexcpt.obj
 0002:0006b1e0       ??1bad_typeid@std@@UAE@XZ  100dd1e0 f   LIBCMTD:stdexcpt.obj
 0002:0006b200       ??0__non_rtti_object@std@@QAE@PBD@Z 100dd200 f   LIBCMTD:stdexcpt.obj
 0002:0006b230       ??_G__non_rtti_object@std@@UAEPAXI@Z 100dd230 f i LIBCMTD:stdexcpt.obj
 0002:0006b230       ??_E__non_rtti_object@std@@UAEPAXI@Z 100dd230 f i LIBCMTD:stdexcpt.obj
 0002:0006b260       ??0__non_rtti_object@std@@QAE@ABV01@@Z 100dd260 f   LIBCMTD:stdexcpt.obj
 0002:0006b290       ??1__non_rtti_object@std@@UAE@XZ 100dd290 f   LIBCMTD:stdexcpt.obj
 0002:0006b2b0       ??2@YAPAXI@Z               100dd2b0 f   LIBCMTD:new.obj
 0002:0006b330       _memcpy_s                  100dd330 f   LIBCMTD:memcpy_s.obj
 0002:0006b4c0       _memmove_s                 100dd4c0 f   LIBCMTD:memmove_s.obj
 0002:0006b620       _sprintf                   100dd620 f   LIBCMTD:sprintf.obj
 0002:0006b7a0       __sprintf_l                100dd7a0 f   LIBCMTD:sprintf.obj
 0002:0006b7d0       _sprintf_s                 100dd7d0 f   LIBCMTD:sprintf.obj
 0002:0006b800       __sprintf_s_l              100dd800 f   LIBCMTD:sprintf.obj
 0002:0006b830       __snprintf_s               100dd830 f   LIBCMTD:sprintf.obj
 0002:0006b860       __snprintf_s_l             100dd860 f   LIBCMTD:sprintf.obj
 0002:0006b890       __sprintf_p                100dd890 f   LIBCMTD:sprintf.obj
 0002:0006b8c0       __sprintf_p_l              100dd8c0 f   LIBCMTD:sprintf.obj
 0002:0006b8f0       __scprintf                 100dd8f0 f   LIBCMTD:sprintf.obj
 0002:0006b910       __scprintf_p               100dd910 f   LIBCMTD:sprintf.obj
 0002:0006b930       __scprintf_l               100dd930 f   LIBCMTD:sprintf.obj
 0002:0006b960       __scprintf_p_l             100dd960 f   LIBCMTD:sprintf.obj
 0002:0006b990       _atol                      100dd990 f   LIBCMTD:atox.obj
 0002:0006b9b0       __atol_l                   100dd9b0 f   LIBCMTD:atox.obj
 0002:0006b9d0       _atoi                      100dd9d0 f   LIBCMTD:atox.obj
 0002:0006b9f0       __atoi_l                   100dd9f0 f   LIBCMTD:atox.obj
 0002:0006ba10       __atoi64                   100dda10 f   LIBCMTD:atox.obj
 0002:0006ba30       __atoi64_l                 100dda30 f   LIBCMTD:atox.obj
 0002:0006ba50       _DebuggerKnownHandle       100dda50 f   LIBCMTD:_error_.obj
 0002:0006bb10       ?_RTC_Failure@@YAXPAXH@Z   100ddb10 f   LIBCMTD:_error_.obj
 0002:0006be20       ?_RTC_StackFailure@@YAXPAXPBD@Z 100dde20 f   LIBCMTD:_error_.obj
 0002:0006bf20       ?_RTC_AllocaFailure@@YAXPAXPAU_RTC_ALLOCA_NODE@@H@Z 100ddf20 f   LIBCMTD:_error_.obj
 0002:0006c0d0       __RTC_UninitUse            100de0d0 f   LIBCMTD:_error_.obj
 0002:0006c1c0       __atof_l                   100de1c0 f   LIBCMTD:atof.obj
 0002:0006c2f0       _atof                      100de2f0 f   LIBCMTD:atof.obj
 0002:0006c310       ___strgtold12              100de310 f   LIBCMTD:atof.obj
 0002:0006c370       ___STRINGTOLD              100de370 f   LIBCMTD:atof.obj
 0002:0006c3c0       _memcmp                    100de3c0 f   LIBCMTD:memcmp.obj
 0002:0006ce30       __alldiv                   100dee30 f   LIBCMTD:lldiv.obj
 0002:0006cee0       __allmul                   100deee0 f   LIBCMTD:llmul.obj
 0002:0006cf20       _strcmp                    100def20 f   LIBCMTD:strcmp.obj
 0002:0006cfb0       __vsprintf_l               100defb0 f   LIBCMTD:vsprintf.obj
 0002:0006d130       _vsprintf                  100df130 f   LIBCMTD:vsprintf.obj
 0002:0006d150       __vscprintf_helper         100df150 f   LIBCMTD:vsprintf.obj
 0002:0006d210       __vscprintf                100df210 f   LIBCMTD:vsprintf.obj
 0002:0006d230       __vscprintf_l              100df230 f   LIBCMTD:vsprintf.obj
 0002:0006d250       __vscprintf_p              100df250 f   LIBCMTD:vsprintf.obj
 0002:0006d270       __vscprintf_p_l            100df270 f   LIBCMTD:vsprintf.obj
 0002:0006d290       __chkstk                   100df290 f   LIBCMTD:chkstk.obj
 0002:0006d290       __alloca_probe             100df290     LIBCMTD:chkstk.obj
 0002:0006d2d0       _strchr                    100df2d0 f   LIBCMTD:strchr.obj
 0002:0006d2d6       ___from_strstr_to_strchr   100df2d6     LIBCMTD:strchr.obj
 0002:0006d390       __splitpath                100df390 f   LIBCMTD:splitpat.obj
 0002:0006d7d0       __makepath                 100df7d0 f   LIBCMTD:makepath.obj
 0002:0006d800       _memmove                   100df800 f   LIBCMTD:memmove.obj
 0002:0006db70       _strstr                    100dfb70 f   LIBCMTD:strstr.obj
 0002:0006dc00       __fsopen                   100dfc00 f   LIBCMTD:fopen.obj
 0002:0006de10       _fopen                     100dfe10 f   LIBCMTD:fopen.obj
 0002:0006de30       _fopen_s                   100dfe30 f   LIBCMTD:fopen.obj
 0002:0006ded0       _fclose                    100dfed0 f   LIBCMTD:fclose.obj
 0002:0006dfe0       __fclose_nolock            100dffe0 f   LIBCMTD:fclose.obj
 0002:0006e0e0       _ftell                     100e00e0 f   LIBCMTD:ftell.obj
 0002:0006e1d0       __ftell_nolock             100e01d0 f   LIBCMTD:ftell.obj
 0002:0006e4a0       _fseek                     100e04a0 f   LIBCMTD:fseek.obj
 0002:0006e610       __fseek_nolock             100e0610 f   LIBCMTD:fseek.obj
 0002:0006e6f0       _fread_s                   100e06f0 f   LIBCMTD:fread.obj
 0002:0006e820       __fread_nolock_s           100e0820 f   LIBCMTD:fread.obj
 0002:0006ee00       _fread                     100e0e00 f   LIBCMTD:fread.obj
 0002:0006ee30       __fread_nolock             100e0e30 f   LIBCMTD:fread.obj
 0002:0006ee60       __allshr                   100e0e60 f   LIBCMTD:llshr.obj
 0002:0006ee90       __CIsqrt                   100e0e90 f   LIBCMTD:_sqrt_.obj
 0002:0006eea4       _sqrt                      100e0ea4     LIBCMTD:_sqrt_.obj
 0002:0006ef50       _atan                      100e0f50 f   LIBCMTD:_atan_.obj
 0002:0006ef90       __CIatan                   100e0f90 f   LIBCMTD:_atan_.obj
 0002:0006efcb       __CIatan_default           100e0fcb f   LIBCMTD:_atan_.obj
 0002:0006efdf       __atan_default             100e0fdf     LIBCMTD:_atan_.obj
 0002:0006f070       _fabs                      100e1070 f   LIBCMTD:_fabs_.obj
 0002:0006f170       _acos                      100e1170 f   LIBCMTD:_acos_.obj
 0002:0006f1b0       __CIacos                   100e11b0 f   LIBCMTD:_acos_.obj
 0002:0006f1eb       __CIacos_default           100e11eb f   LIBCMTD:_acos_.obj
 0002:0006f1ff       __acos_default             100e11ff     LIBCMTD:_acos_.obj
 0002:0006f2c0       _cos                       100e12c0 f   LIBCMTD:_cos_.obj
 0002:0006f300       __CIcos                    100e1300 f   LIBCMTD:_cos_.obj
 0002:0006f33b       __CIcos_default            100e133b f   LIBCMTD:_cos_.obj
 0002:0006f34f       __cos_default              100e134f     LIBCMTD:_cos_.obj
 0002:0006f3f0       _sin                       100e13f0 f   LIBCMTD:_sin_.obj
 0002:0006f430       __CIsin                    100e1430 f   LIBCMTD:_sin_.obj
 0002:0006f46b       __CIsin_default            100e146b f   LIBCMTD:_sin_.obj
 0002:0006f47f       __sin_default              100e147f     LIBCMTD:_sin_.obj
 0002:0006f520       _asin                      100e1520 f   LIBCMTD:_asin_.obj
 0002:0006f560       __CIasin                   100e1560 f   LIBCMTD:_asin_.obj
 0002:0006f59b       __CIasin_default           100e159b f   LIBCMTD:_asin_.obj
 0002:0006f5af       __asin_default             100e15af     LIBCMTD:_asin_.obj
 0002:0006f670       __copysign                 100e1670 f   LIBCMTD:_ieeemisc_.obj
 0002:0006f6b0       __chgsign                  100e16b0 f   LIBCMTD:_ieeemisc_.obj
 0002:0006f6f0       __scalb                    100e16f0 f   LIBCMTD:_ieeemisc_.obj
 0002:0006f710       __logb                     100e1710 f   LIBCMTD:_ieeemisc_.obj
 0002:0006f840       __nextafter                100e1840 f   LIBCMTD:_ieeemisc_.obj
 0002:0006fb60       __finite                   100e1b60 f   LIBCMTD:_ieeemisc_.obj
 0002:0006fb80       __isnan                    100e1b80 f   LIBCMTD:_ieeemisc_.obj
 0002:0006fbd0       __fpclass                  100e1bd0 f   LIBCMTD:_ieeemisc_.obj
 0002:0006fca0       _srand                     100e1ca0 f   LIBCMTD:rand.obj
 0002:0006fcc0       _rand                      100e1cc0 f   LIBCMTD:rand.obj
 0002:0006fd00       _ldiv                      100e1d00 f   LIBCMTD:ldiv.obj
 0002:0006fd30       _realloc                   100e1d30 f   LIBCMTD:dbgrealloc.obj
 0002:0006fd60       _printf                    100e1d60 f   LIBCMTD:printf.obj
 0002:0006fea0       __printf_l                 100e1ea0 f   LIBCMTD:printf.obj
 0002:0006fed0       __printf_s_l               100e1ed0 f   LIBCMTD:printf.obj
 0002:0006ff00       _printf_s                  100e1f00 f   LIBCMTD:printf.obj
 0002:0006ff30       __printf_p_l               100e1f30 f   LIBCMTD:printf.obj
 0002:0006ff60       __printf_p                 100e1f60 f   LIBCMTD:printf.obj
 0002:0006ff90       __set_printf_count_output  100e1f90 f   LIBCMTD:printf.obj
 0002:0006ffe0       __get_printf_count_output  100e1fe0 f   LIBCMTD:printf.obj
 0002:00070000       _memchr                    100e2000 f   LIBCMTD:memchr.obj
 0002:000700b0       _fwrite                    100e20b0 f   LIBCMTD:fwrite.obj
 0002:000701c0       __fwrite_nolock            100e21c0 f   LIBCMTD:fwrite.obj
 0002:00070590       __dosmaperr                100e2590 f   LIBCMTD:dosmap.obj
 0002:000705c0       __get_errno_from_oserr     100e25c0 f   LIBCMTD:dosmap.obj
 0002:00070640       __set_errno                100e2640 f   LIBCMTD:dosmap.obj
 0002:00070670       __get_errno                100e2670 f   LIBCMTD:dosmap.obj
 0002:000706f0       __set_doserrno             100e26f0 f   LIBCMTD:dosmap.obj
 0002:00070720       __get_doserrno             100e2720 f   LIBCMTD:dosmap.obj
 0002:000707a0       __errno                    100e27a0 f   LIBCMTD:dosmap.obj
 0002:000707d0       ___doserrno                100e27d0 f   LIBCMTD:dosmap.obj
 0002:00070800       __malloc_dbg               100e2800 f   LIBCMTD:dbgheap.obj
 0002:00070830       __nh_malloc                100e2830 f   LIBCMTD:dbgheap.obj
 0002:00070850       __nh_malloc_dbg            100e2850 f   LIBCMTD:dbgheap.obj
 0002:00070920       __heap_alloc               100e2920 f   LIBCMTD:dbgheap.obj
 0002:00070cf0       __heap_alloc_dbg           100e2cf0 f   LIBCMTD:dbgheap.obj
 0002:00070d50       __calloc_dbg_impl          100e2d50 f   LIBCMTD:dbgheap.obj
 0002:00070e20       __calloc_dbg               100e2e20 f   LIBCMTD:dbgheap.obj
 0002:00070e80       __recalloc                 100e2e80 f   LIBCMTD:dbgheap.obj
 0002:00070eb0       __realloc_dbg              100e2eb0 f   LIBCMTD:dbgheap.obj
 0002:00071550       __recalloc_dbg             100e3550 f   LIBCMTD:dbgheap.obj
 0002:00071650       __expand                   100e3650 f   LIBCMTD:dbgheap.obj
 0002:00071680       __expand_dbg               100e3680 f   LIBCMTD:dbgheap.obj
 0002:00071790       __free_nolock              100e3790 f   LIBCMTD:dbgheap.obj
 0002:000717b0       __free_dbg                 100e37b0 f   LIBCMTD:dbgheap.obj
 0002:00071830       __free_dbg_nolock          100e3830 f   LIBCMTD:dbgheap.obj
 0002:00071d10       __msize                    100e3d10 f   LIBCMTD:dbgheap.obj
 0002:00071d30       __msize_dbg                100e3d30 f   LIBCMTD:dbgheap.obj
 0002:00071f20       __CrtSetBreakAlloc         100e3f20 f   LIBCMTD:dbgheap.obj
 0002:00071f40       __CrtSetDbgBlockType       100e3f40 f   LIBCMTD:dbgheap.obj
 0002:00072030       __CrtSetAllocHook          100e4030 f   LIBCMTD:dbgheap.obj
 0002:00072050       __CrtGetAllocHook          100e4050 f   LIBCMTD:dbgheap.obj
 0002:000720b0       __CrtCheckMemory           100e40b0 f   LIBCMTD:dbgheap.obj
 0002:00072510       __CrtSetDbgFlag            100e4510 f   LIBCMTD:dbgheap.obj
 0002:00072660       __CrtDoForAllClientObjects 100e4660 f   LIBCMTD:dbgheap.obj
 0002:00072780       __CrtIsValidPointer        100e4780 f   LIBCMTD:dbgheap.obj
 0002:00072790       __CrtIsValidHeapPointer    100e4790 f   LIBCMTD:dbgheap.obj
 0002:00072830       __CrtIsMemoryBlock         100e4830 f   LIBCMTD:dbgheap.obj
 0002:000729a0       __CrtReportBlockType       100e49a0 f   LIBCMTD:dbgheap.obj
 0002:000729d0       __CrtSetDumpClient         100e49d0 f   LIBCMTD:dbgheap.obj
 0002:000729f0       __CrtGetDumpClient         100e49f0 f   LIBCMTD:dbgheap.obj
 0002:00072a00       __CrtMemCheckpoint         100e4a00 f   LIBCMTD:dbgheap.obj
 0002:00072c20       __CrtMemDifference         100e4c20 f   LIBCMTD:dbgheap.obj
 0002:00072e40       __CrtMemDumpAllObjectsSince 100e4e40 f   LIBCMTD:dbgheap.obj
 0002:00073330       __CrtDumpMemoryLeaks       100e5330 f   LIBCMTD:dbgheap.obj
 0002:000733a0       __CrtMemDumpStatistics     100e53a0 f   LIBCMTD:dbgheap.obj
 0002:000734b0       __aligned_malloc           100e54b0 f   LIBCMTD:dbgheap.obj
 0002:000734d0       __aligned_malloc_dbg       100e54d0 f   LIBCMTD:dbgheap.obj
 0002:00073500       __aligned_realloc          100e5500 f   LIBCMTD:dbgheap.obj
 0002:00073530       __aligned_recalloc         100e5530 f   LIBCMTD:dbgheap.obj
 0002:00073560       __aligned_realloc_dbg      100e5560 f   LIBCMTD:dbgheap.obj
 0002:00073590       __aligned_recalloc_dbg     100e5590 f   LIBCMTD:dbgheap.obj
 0002:000735c0       __aligned_offset_malloc    100e55c0 f   LIBCMTD:dbgheap.obj
 0002:000735e0       __aligned_offset_malloc_dbg 100e55e0 f   LIBCMTD:dbgheap.obj
 0002:00073780       __aligned_offset_realloc   100e5780 f   LIBCMTD:dbgheap.obj
 0002:000737b0       __aligned_offset_recalloc  100e57b0 f   LIBCMTD:dbgheap.obj
 0002:000737e0       __aligned_offset_realloc_dbg 100e57e0 f   LIBCMTD:dbgheap.obj
 0002:00073ab0       __aligned_offset_recalloc_dbg 100e5ab0 f   LIBCMTD:dbgheap.obj
 0002:00073bc0       __aligned_free             100e5bc0 f   LIBCMTD:dbgheap.obj
 0002:00073be0       __aligned_free_dbg         100e5be0 f   LIBCMTD:dbgheap.obj
 0002:00073c90       __CrtSetDebugFillThreshold 100e5c90 f   LIBCMTD:dbgheap.obj
 0002:00073cb0       __CrtSetCheckCount         100e5cb0 f   LIBCMTD:dbgheap.obj
 0002:00073cd0       __CrtGetCheckCount         100e5cd0 f   LIBCMTD:dbgheap.obj
 0002:00073ce0       __aligned_msize            100e5ce0 f   LIBCMTD:dbgheap.obj
 0002:00073d00       __aligned_msize_dbg        100e5d00 f   LIBCMTD:dbgheap.obj
 0002:00073e10       __CRT_INIT@12              100e5e10 f   LIBCMTD:dllcrt0.obj
 0002:00073fe0       __DllMainCRTStartup@12     100e5fe0 f   LIBCMTD:dllcrt0.obj
 0002:000741d0       _abort                     100e61d0 f   LIBCMTD:abort.obj
 0002:00074310       __set_abort_behavior       100e6310 f   LIBCMTD:abort.obj
 0002:00074340       _fputs                     100e6340 f   LIBCMTD:fputs.obj
 0002:000745e0       ___iob_func                100e65e0 f   LIBCMTD:_file.obj
 0002:000745f0       ___initstdio               100e65f0 f   LIBCMTD:_file.obj
 0002:00074740       ___endstdio                100e6740 f   LIBCMTD:_file.obj
 0002:00074770       __lock_file                100e6770 f   LIBCMTD:_file.obj
 0002:000747d0       __lock_file2               100e67d0 f   LIBCMTD:_file.obj
 0002:00074810       __unlock_file              100e6810 f   LIBCMTD:_file.obj
 0002:00074870       __unlock_file2             100e6870 f   LIBCMTD:_file.obj
 0002:000748b0       _fflush                    100e68b0 f   LIBCMTD:fflush.obj
 0002:00074950       __fflush_nolock            100e6950 f   LIBCMTD:fflush.obj
 0002:000749b0       __flush                    100e69b0 f   LIBCMTD:fflush.obj
 0002:00074a70       __flushall                 100e6a70 f   LIBCMTD:fflush.obj
 0002:00074c40       _calloc                    100e6c40 f   LIBCMTD:dbgcalloc.obj
 0002:00074c70       _floor                     100e6c70 f   LIBCMTD:_floor_pentium4_.obj
 0002:00074cb0       __floor_pentium4           100e6cb0 f   LIBCMTD:_floor_pentium4_.obj
 0002:00074da0       __ftol                     100e6da0 f   LIBCMTD:_ftol_.obj
 0002:00074dd0       __toupper                  100e6dd0 f   LIBCMTD:toupper.obj
 0002:00074de0       __toupper_l                100e6de0 f   LIBCMTD:toupper.obj
 0002:00074fc0       _toupper                   100e6fc0 f   LIBCMTD:toupper.obj
 0002:00075010       _fprintf                   100e7010 f   LIBCMTD:fprintf.obj
 0002:000752b0       __fprintf_l                100e72b0 f   LIBCMTD:fprintf.obj
 0002:000752e0       __fprintf_s_l              100e72e0 f   LIBCMTD:fprintf.obj
 0002:00075310       _fprintf_s                 100e7310 f   LIBCMTD:fprintf.obj
 0002:00075340       __fprintf_p_l              100e7340 f   LIBCMTD:fprintf.obj
 0002:00075370       __fprintf_p                100e7370 f   LIBCMTD:fprintf.obj
 0002:000753a0       _perror                    100e73a0 f   LIBCMTD:perror.obj
 0002:000754a0       __get_sys_err_msg          100e74a0 f i LIBCMTD:perror.obj
 0002:000754e0       _ceil                      100e74e0 f   LIBCMTD:_ceil_pentium4_.obj
 0002:00075520       __ceil_pentium4            100e7520 f   LIBCMTD:_ceil_pentium4_.obj
 0002:00075600       _qsort                     100e7600 f   LIBCMTD:qsort.obj
 0002:00075bb0       _ldexp                     100e7bb0 f   LIBCMTD:_ldexp_.obj
 0002:00075e70       __crt_waiting_on_module_handle 100e7e70 f   LIBCMTD:crt0dat.obj
 0002:00075ed0       __cinit                    100e7ed0 f   LIBCMTD:crt0dat.obj
 0002:00075f70       _exit                      100e7f70 f   LIBCMTD:crt0dat.obj
 0002:00075f90       __exit                     100e7f90 f   LIBCMTD:crt0dat.obj
 0002:00075fb0       __cexit                    100e7fb0 f   LIBCMTD:crt0dat.obj
 0002:00075fd0       __c_exit                   100e7fd0 f   LIBCMTD:crt0dat.obj
 0002:00075ff0       __amsg_exit                100e7ff0 f   LIBCMTD:crt0dat.obj
 0002:00076030       ___freeCrtMemory           100e8030 f   LIBCMTD:crt0dat.obj
 0002:00076380       ___crtCorExitProcess       100e8380 f   LIBCMTD:crt0dat.obj
 0002:000763c0       ___crtExitProcess          100e83c0 f   LIBCMTD:crt0dat.obj
 0002:000763e0       __lockexit                 100e83e0 f   LIBCMTD:crt0dat.obj
 0002:00076400       __unlockexit               100e8400 f   LIBCMTD:crt0dat.obj
 0002:00076420       __init_pointers            100e8420 f   LIBCMTD:crt0dat.obj
 0002:000764e0       __initterm_e               100e84e0 f   LIBCMTD:crt0dat.obj
 0002:00076520       __get_wpgmptr              100e8520 f   LIBCMTD:crt0dat.obj
 0002:00076610       __get_pgmptr               100e8610 f   LIBCMTD:crt0dat.obj
 0002:00076700       _frexp                     100e8700 f   LIBCMTD:_frexp_.obj
 0002:00076870       __RTC_NumErrors            100e8870 f   LIBCMTD:_userapi_.obj
 0002:00076880       __RTC_GetErrDesc           100e8880 f   LIBCMTD:_userapi_.obj
 0002:000768a0       __RTC_SetErrorType         100e88a0 f   LIBCMTD:_userapi_.obj
 0002:000768d0       __RTC_SetErrorFunc         100e88d0 f   LIBCMTD:_userapi_.obj
 0002:000768f0       __RTC_SetErrorFuncW        100e88f0 f   LIBCMTD:_userapi_.obj
 0002:00076910       ?_RTC_GetErrorFunc@@YAP6AHHPBDH00ZZPBX@Z 100e8910 f   LIBCMTD:_userapi_.obj
 0002:00076920       ?_RTC_GetErrorFuncW@@YAP6AHHPB_WH00ZZPBX@Z 100e8920 f   LIBCMTD:_userapi_.obj
 0002:00076930       __chkesp                   100e8930 f   LIBCMTD:chkesp.obj
 0002:00076970       __CRT_RTC_INIT             100e8970 f   LIBCMTD:chkesp.obj
 0002:00076980       __CRT_RTC_INITW            100e8980 f   LIBCMTD:chkesp.obj
 0002:00076990       __VEC_memzero              100e8990 f   LIBCMTD:p4_memset.obj
 0002:00076a80       __get_sse2_info            100e8a80 f   LIBCMTD:cpu_disp.obj
 0002:00076bb0       ___sse2_available_init     100e8bb0 f   LIBCMTD:cpu_disp.obj
 0002:00076bd0       __VEC_memcpy               100e8bd0 f   LIBCMTD:p4_memcpy.obj
 0002:00076d50       __tolower                  100e8d50 f   LIBCMTD:tolower.obj
 0002:00076d60       __tolower_l                100e8d60 f   LIBCMTD:tolower.obj
 0002:00076f40       _tolower                   100e8f40 f   LIBCMTD:tolower.obj
 0002:00076f90       ___updatetmbcinfo          100e8f90 f   LIBCMTD:mbctype.obj
 0002:000770a0       __setmbcp                  100e90a0 f   LIBCMTD:mbctype.obj
 0002:00077450       __setmbcp_nolock           100e9450 f   LIBCMTD:mbctype.obj
 0002:00077c40       __getmbcp                  100e9c40 f   LIBCMTD:mbctype.obj
 0002:00077cb0       ___initmbctable            100e9cb0 f   LIBCMTD:mbctype.obj
 0002:00077ce0       ____setlc_active_func      100e9ce0 f   LIBCMTD:setlocal.obj
 0002:00077cf0       ____unguarded_readlc_active_add_func 100e9cf0 f   LIBCMTD:setlocal.obj
 0002:00077d00       ___freetlocinfo            100e9d00 f   LIBCMTD:setlocal.obj
 0002:00077fe0       ___addlocaleref            100e9fe0 f   LIBCMTD:setlocal.obj
 0002:00078100       ___removelocaleref         100ea100 f   LIBCMTD:setlocal.obj
 0002:00078230       ___updatetlocinfo          100ea230 f   LIBCMTD:setlocal.obj
 0002:00078380       __configthreadlocale       100ea380 f   LIBCMTD:setlocal.obj
 0002:00078490       __locterm                  100ea490 f   LIBCMTD:setlocal.obj
 0002:00078530       __free_locale              100ea530 f   LIBCMTD:setlocal.obj
 0002:00078670       ___free_locale             100ea670 f   LIBCMTD:setlocal.obj
 0002:00078690       __create_locale            100ea690 f   LIBCMTD:setlocal.obj
 0002:000788c0       ___create_locale           100ea8c0 f   LIBCMTD:setlocal.obj
 0002:000788e0       __get_current_locale       100ea8e0 f   LIBCMTD:setlocal.obj
 0002:00078a00       ___get_current_locale      100eaa00 f   LIBCMTD:setlocal.obj
 0002:00078a10       _setlocale                 100eaa10 f   LIBCMTD:setlocal.obj
 0002:00079920       __expandlocale             100eb920 f   LIBCMTD:setlocal.obj
 0002:00079bd0       ___init_dummy              100ebbd0 f   LIBCMTD:setlocal.obj
 0002:00079be0       __strcats                  100ebbe0 f   LIBCMTD:setlocal.obj
 0002:00079c60       ___lc_strtolc              100ebc60 f   LIBCMTD:setlocal.obj
 0002:00079e60       ___lc_lctostr              100ebe60 f   LIBCMTD:setlocal.obj
 0002:00079f00       __encode_pointer           100ebf00 f   LIBCMTD:tidtable.obj
 0002:00079fa0       __crt_wait_module_handle   100ebfa0 f i LIBCMTD:tidtable.obj
 0002:00079fd0       __encoded_null             100ebfd0 f   LIBCMTD:tidtable.obj
 0002:00079ff0       __decode_pointer           100ebff0 f   LIBCMTD:tidtable.obj
 0002:0007a090       ___crtTlsAlloc@4           100ec090 f   LIBCMTD:tidtable.obj
 0002:0007a0a0       ___fls_getvalue@4          100ec0a0 f   LIBCMTD:tidtable.obj
 0002:0007a0c0       ___get_flsindex            100ec0c0 f   LIBCMTD:tidtable.obj
 0002:0007a0d0       ___set_flsgetvalue         100ec0d0 f   LIBCMTD:tidtable.obj
 0002:0007a120       ___fls_setvalue@8          100ec120 f   LIBCMTD:tidtable.obj
 0002:0007a150       __mtinit                   100ec150 f   LIBCMTD:tidtable.obj
 0002:0007a360       __mtterm                   100ec360 f   LIBCMTD:tidtable.obj
 0002:0007a3c0       __initptd                  100ec3c0 f   LIBCMTD:tidtable.obj
 0002:0007a520       __getptd_noexit            100ec520 f   LIBCMTD:tidtable.obj
 0002:0007a5e0       __getptd                   100ec5e0 f   LIBCMTD:tidtable.obj
 0002:0007a610       __freefls@4                100ec610 f   LIBCMTD:tidtable.obj
 0002:0007a820       __freeptd                  100ec820 f   LIBCMTD:tidtable.obj
 0002:0007a8a0       ___threadid                100ec8a0 f   LIBCMTD:tidtable.obj
 0002:0007a8b0       ___threadhandle            100ec8b0 f   LIBCMTD:tidtable.obj
 0002:0007a8c0       ___report_gsfailure        100ec8c0 f   LIBCMTD:gs_report.obj
 0002:0007a9d0       __setdefaultprecision      100ec9d0 f   LIBCMTD:fp8.obj
 0002:0007aa10       __ms_p5_test_fdiv          100eca10 f   LIBCMTD:_testfdiv_.obj
 0002:0007aa60       __ms_p5_mp_test_fdiv       100eca60 f   LIBCMTD:_testfdiv_.obj
 0002:0007aab0       __forcdecpt                100ecab0 f   LIBCMTD:cvt.obj
 0002:0007aad0       __forcdecpt_l              100ecad0 f   LIBCMTD:cvt.obj
 0002:0007ab90       __cropzeros                100ecb90 f   LIBCMTD:cvt.obj
 0002:0007abb0       __cropzeros_l              100ecbb0 f   LIBCMTD:cvt.obj
 0002:0007acc0       __positive                 100eccc0 f   LIBCMTD:cvt.obj
 0002:0007acf0       __fassign_l                100eccf0 f   LIBCMTD:cvt.obj
 0002:0007ad50       __fassign                  100ecd50 f   LIBCMTD:cvt.obj
 0002:0007ad70       __cftoe_l                  100ecd70 f   LIBCMTD:cvt.obj
 0002:0007b2c0       __cftoe                    100ed2c0 f   LIBCMTD:cvt.obj
 0002:0007b2f0       __cftoa_l                  100ed2f0 f   LIBCMTD:cvt.obj
 0002:0007bad0       ?strrchr@@YAPADPADH@Z      100edad0 f i LIBCMTD:cvt.obj
 0002:0007baf0       __cftoa                    100edaf0 f   LIBCMTD:cvt.obj
 0002:0007bb20       __cftof_l                  100edb20 f   LIBCMTD:cvt.obj
 0002:0007bf30       __cftof                    100edf30 f   LIBCMTD:cvt.obj
 0002:0007bf60       __cftog_l                  100edf60 f   LIBCMTD:cvt.obj
 0002:0007c190       __cftog                    100ee190 f   LIBCMTD:cvt.obj
 0002:0007c1c0       __cfltcvt_l                100ee1c0 f   LIBCMTD:cvt.obj
 0002:0007c280       __cfltcvt                  100ee280 f   LIBCMTD:cvt.obj
 0002:0007c2e0       __initp_misc_cfltcvt_tab   100ee2e0 f   LIBCMTD:cmiscdat.obj
 0002:0007c330       __except_handler4          100ee330 f   LIBCMTD:chandler4.obj
 0002:0007c550       __initp_eh_hooks           100ee550 f   LIBCMTD:hooks.obj
 0002:0007c570       ?terminate@@YAXXZ          100ee570 f   LIBCMTD:hooks.obj
 0002:0007c5f0       ?unexpected@@YAXXZ         100ee5f0 f   LIBCMTD:hooks.obj
 0002:0007c620       ?_inconsistency@@YAXXZ     100ee620 f   LIBCMTD:hooks.obj
 0002:0007c6b0       __sse2_mathfcns_init       100ee6b0 f   LIBCMTD:_mathfcns_.obj
 0002:0007c6d0       __set_SSE2_enable          100ee6d0 f   LIBCMTD:_mathfcns_.obj
 0002:0007c6f0       __CIlog_pentium4           100ee6f0 f   LIBCMTD:_log_pentium4_.obj
 0002:0007c708       __log_pentium4             100ee708     LIBCMTD:_log_pentium4_.obj
 0002:0007c971       __fFEXP                    100ee971     LIBCMTD:_87tran_.obj
 0002:0007c9d8       __rtinfpopse               100ee9d8     LIBCMTD:_87tran_.obj
 0002:0007c9da       __rtinfnpopse              100ee9da     LIBCMTD:_87tran_.obj
 0002:0007c9ea       __fFLN                     100ee9ea     LIBCMTD:_87tran_.obj
 0002:0007ca9f       __rtinfpop                 100eea9f     LIBCMTD:_87tran_.obj
 0002:0007caa1       __rtinfnpop                100eeaa1     LIBCMTD:_87tran_.obj
 0002:0007cabe       __ffexpm1                  100eeabe     LIBCMTD:_87tran_.obj
 0002:0007cb70       __trandisp1                100eeb70 f   LIBCMTD:_87disp_.obj
 0002:0007cbd7       __trandisp2                100eebd7 f   LIBCMTD:_87disp_.obj
 0002:0007cc63       __rttospopde               100eec63     LIBCMTD:_87disp_.obj
 0002:0007cc68       __rttospop                 100eec68     LIBCMTD:_87disp_.obj
 0002:0007cc6a       __rtnospop                 100eec6a     LIBCMTD:_87disp_.obj
 0002:0007cc6c       __rttosnpop                100eec6c     LIBCMTD:_87disp_.obj
 0002:0007cc6d       __rtnospopde               100eec6d     LIBCMTD:_87disp_.obj
 0002:0007cc74       __rtzeropop                100eec74     LIBCMTD:_87disp_.obj
 0002:0007cc76       __rtzeronpop               100eec76     LIBCMTD:_87disp_.obj
 0002:0007cc7b       __rtonepop                 100eec7b     LIBCMTD:_87disp_.obj
 0002:0007cc7d       __rtonenpop                100eec7d     LIBCMTD:_87disp_.obj
 0002:0007cc82       __tosnan1                  100eec82     LIBCMTD:_87disp_.obj
 0002:0007ccad       __nosnan2                  100eecad     LIBCMTD:_87disp_.obj
 0002:0007ccaf       __tosnan2                  100eecaf     LIBCMTD:_87disp_.obj
 0002:0007ccd7       __nan2                     100eecd7     LIBCMTD:_87disp_.obj
 0002:0007cd16       __rtindfpop                100eed16     LIBCMTD:_87disp_.obj
 0002:0007cd18       __rtindfnpop               100eed18     LIBCMTD:_87disp_.obj
 0002:0007cd29       __rttosnpopde              100eed29     LIBCMTD:_87disp_.obj
 0002:0007cd33       __rtchsifneg               100eed33     LIBCMTD:_87disp_.obj
 0002:0007cd40       __twoToTOS                 100eed40 f   LIBCMTD:_common_.obj
 0002:0007cd55       __load_CW                  100eed55 f   LIBCMTD:_common_.obj
 0002:0007cd6c       __convertTOStoQNaN         100eed6c f   LIBCMTD:_common_.obj
 0002:0007cd85       __fload_withFB             100eed85 f   LIBCMTD:_common_.obj
 0002:0007cdc8       __checkTOS_withFB          100eedc8 f   LIBCMTD:_common_.obj
 0002:0007cdde       __fast_exit                100eedde f   LIBCMTD:_common_.obj
 0002:0007cdeb       __math_exit                100eedeb f   LIBCMTD:_common_.obj
 0002:0007ce15       __check_overflow_exit      100eee15 f   LIBCMTD:_common_.obj
 0002:0007ce29       __check_range_exit         100eee29 f   LIBCMTD:_common_.obj
 0002:0007ced0       __startTwoArgErrorHandling 100eeed0 f   LIBCMTD:_genexcep_.obj
 0002:0007cee7       __startOneArgErrorHandling 100eeee7 f   LIBCMTD:_genexcep_.obj
 0002:0007cf30       __CIpow_pentium4           100eef30 f   LIBCMTD:_pow_pentium4_.obj
 0002:0007cf49       __pow_pentium4             100eef49     LIBCMTD:_pow_pentium4_.obj
 0002:0007da90       __powhlp                   100efa90 f   LIBCMTD:_powhlp_.obj
 0002:0007dc40       __d_inttype                100efc40 f   LIBCMTD:_powhlp_.obj
 0002:0007dcd0       ___InternalCxxFrameHandler 100efcd0 f   LIBCMTD:frame.obj
 0002:0007e2d0       ??0bad_exception@std@@QAE@PBD@Z 100f02d0 f i LIBCMTD:frame.obj
 0002:0007e300       ??1bad_exception@std@@UAE@XZ 100f0300 f i LIBCMTD:frame.obj
 0002:0007e320       ??_Ebad_exception@std@@UAEPAXI@Z 100f0320 f i LIBCMTD:frame.obj
 0002:0007e320       ??_Gbad_exception@std@@UAEPAXI@Z 100f0320 f i LIBCMTD:frame.obj
 0002:0007e350       ??0bad_exception@std@@QAE@ABV01@@Z 100f0350 f i LIBCMTD:frame.obj
 0002:0007e500       ___TypeMatch               100f0500 f   LIBCMTD:frame.obj
 0002:0007e5b0       ___FrameUnwindFilter       100f05b0 f   LIBCMTD:frame.obj
 0002:0007e630       ___FrameUnwindToState      100f0630 f   LIBCMTD:frame.obj
 0002:0007eb70       ___BuildCatchObjectHelper  100f0b70 f   LIBCMTD:frame.obj
 0002:0007ede0       ___BuildCatchObject        100f0de0 f   LIBCMTD:frame.obj
 0002:0007eef0       ___DestructExceptionObject 100f0ef0 f   LIBCMTD:frame.obj
 0002:0007efa0       ___AdjustPointer           100f0fa0 f   LIBCMTD:frame.obj
 0002:0007eff0       ?__uncaught_exception@@YA_NXZ 100f0ff0 f   LIBCMTD:frame.obj
 0002:0007f010       ___CxxExceptionFilter      100f1010 f   LIBCMTD:frame.obj
 0002:0007f200       ___CxxRegisterExceptionObject 100f1200 f   LIBCMTD:frame.obj
 0002:0007f330       ___CxxDetectRethrow        100f1330 f   LIBCMTD:frame.obj
 0002:0007f3c0       ___CxxUnregisterExceptionObject 100f13c0 f   LIBCMTD:frame.obj
 0002:0007f540       ___CxxQueryExceptionSize   100f1540 f   LIBCMTD:frame.obj
 0002:0007f550       ___CxxCallUnwindDtor       100f1550 f   LIBCMTD:frame.obj
 0002:0007f5d0       ___CxxCallUnwindDelDtor    100f15d0 f   LIBCMTD:frame.obj
 0002:0007f650       ___CxxCallUnwindStdDelDtor 100f1650 f   LIBCMTD:frame.obj
 0002:0007f6d0       ___CxxCallUnwindVecDtor    100f16d0 f   LIBCMTD:frame.obj
 0002:0007f900       ?_is_exception_typeof@@YAHABVtype_info@@PAU_EXCEPTION_POINTERS@@@Z 100f1900 f   LIBCMTD:frame.obj
 0002:0007f9e0       __CallSettingFrame@12      100f19e0 f   LIBCMTD:lowhelpr.obj
 0002:0007fa07       __NLG_Return               100f1a07     LIBCMTD:lowhelpr.obj
 0002:0007fa30       __CrtDefaultAllocHook      100f1a30 f   LIBCMTD:dbghook.obj
 0002:0007fa40       __crt_debugger_hook        100f1a40 f   LIBCMTD:dbghook.obj
 0002:0007fa60       __mtinitlocks              100f1a60 f   LIBCMTD:mlock.obj
 0002:0007faf0       __mtdeletelocks            100f1af0 f   LIBCMTD:mlock.obj
 0002:0007fbb0       __mtinitlocknum            100f1bb0 f   LIBCMTD:mlock.obj
 0002:0007fd00       __lock                     100f1d00 f   LIBCMTD:mlock.obj
 0002:0007fd40       __unlock                   100f1d40 f   LIBCMTD:mlock.obj
 0002:0007fd60       __lockerr_exit             100f1d60 f   LIBCMTD:mlock.obj
 0002:0007fd80       __CrtDbgBreak              100f1d80 f   LIBCMTD:dbgrptt.obj
 0002:0007fd90       __CrtSetReportMode         100f1d90 f   LIBCMTD:dbgrptt.obj
 0002:0007fed0       __CrtSetReportFile         100f1ed0 f   LIBCMTD:dbgrptt.obj
 0002:0007ffd0       __CrtSetReportHook         100f1fd0 f   LIBCMTD:dbgrptt.obj
 0002:0007fff0       __CrtGetReportHook         100f1ff0 f   LIBCMTD:dbgrptt.obj
 0002:00080000       __VCrtDbgReportA           100f2000 f   LIBCMTD:dbgrptt.obj
 0002:00080830       __VCrtDbgReportW           100f2830 f   LIBCMTD:dbgrptt.obj
 0002:00081160       __initp_misc_winsig        100f3160 f   LIBCMTD:winsig.obj
 0002:00081190       _signal                    100f3190 f   LIBCMTD:winsig.obj
 0002:00081630       _raise                     100f3630 f   LIBCMTD:winsig.obj
 0002:000819a0       ___get_sigabrt             100f39a0 f   LIBCMTD:winsig.obj
 0002:000819c0       ___fpecode                 100f39c0 f   LIBCMTD:winsig.obj
 0002:000819d0       ___pxcptinfoptrs           100f39d0 f   LIBCMTD:winsig.obj
 0002:000819e0       ___crtMessageBoxW          100f39e0 f   LIBCMTD:crtmboxw.obj
 0002:00081c00       __swprintf                 100f3c00 f   LIBCMTD:swprintf.obj
 0002:00081dd0       ___swprintf_l              100f3dd0 f   LIBCMTD:swprintf.obj
 0002:00081e00       _swprintf_s                100f3e00 f   LIBCMTD:swprintf.obj
 0002:00081e30       __snwprintf_s              100f3e30 f   LIBCMTD:swprintf.obj
 0002:00081e60       __swprintf_p               100f3e60 f   LIBCMTD:swprintf.obj
 0002:00081e90       __swprintf_s_l             100f3e90 f   LIBCMTD:swprintf.obj
 0002:00081ec0       __snwprintf_s_l            100f3ec0 f   LIBCMTD:swprintf.obj
 0002:00081ef0       __swprintf_p_l             100f3ef0 f   LIBCMTD:swprintf.obj
 0002:00081f20       __scwprintf                100f3f20 f   LIBCMTD:swprintf.obj
 0002:00081f40       __scwprintf_p              100f3f40 f   LIBCMTD:swprintf.obj
 0002:00081f60       __scwprintf_l              100f3f60 f   LIBCMTD:swprintf.obj
 0002:00081f90       __scwprintf_p_l            100f3f90 f   LIBCMTD:swprintf.obj
 0002:00081fc0       _wcslen                    100f3fc0 f   LIBCMTD:wcslen.obj
 0002:00081ff0       _wcscpy_s                  100f3ff0 f   LIBCMTD:wcscpy_s.obj
 0002:000822d0       ?_Type_info_dtor@type_info@@CAXPAV1@@Z 100f42d0 f   LIBCMTD:typname.obj
 0002:000823e0       ?_Name_base@type_info@@CAPBDPBV1@PAU__type_info_node@@@Z 100f43e0 f   LIBCMTD:typname.obj
 0002:00082580       ?_Type_info_dtor_internal@type_info@@CAXPAV1@@Z 100f4580 f   LIBCMTD:typname.obj
 0002:00082690       ___unDNameHelper           100f4690 f   LIBCMTD:typname.obj
 0002:000826d0       ?_Name_base_internal@type_info@@CAPBDPBV1@PAU__type_info_node@@@Z 100f46d0 f   LIBCMTD:typname.obj
 0002:00082890       ___clean_type_info_names_internal 100f4890 f   LIBCMTD:typname.obj
 0002:00082950       _strcpy_s                  100f4950 f   LIBCMTD:strcpy_s.obj
 0002:00082c30       __initp_heap_handler       100f4c30 f   LIBCMTD:handler.obj
 0002:00082c40       ?_set_new_handler@@YAP6AHI@ZP6AHI@Z@Z 100f4c40 f   LIBCMTD:handler.obj
 0002:00082c90       ?_set_new_handler@@YAP6AHI@ZH@Z 100f4c90 f   LIBCMTD:handler.obj
 0002:00082cd0       ?_query_new_handler@@YAP6AHI@ZXZ 100f4cd0 f   LIBCMTD:handler.obj
 0002:00082cf0       __callnewh                 100f4cf0 f   LIBCMTD:handler.obj
 0002:00082d30       __flsbuf                   100f4d30 f   LIBCMTD:_flsbuf.obj
 0002:00082ff0       __output_l                 100f4ff0 f   LIBCMTD:output.obj
 0002:00084420       _get_int_arg               100f6420 f i LIBCMTD:output.obj
 0002:00084440       _get_int64_arg             100f6440 f i LIBCMTD:output.obj
 0002:00084460       _get_short_arg             100f6460 f i LIBCMTD:output.obj
 0002:00084480       __vsnprintf_helper         100f6480 f   LIBCMTD:vsnprnc.obj
 0002:00084650       __vsnprintf_c              100f6650 f   LIBCMTD:vsnprnc.obj
 0002:000846a0       __vsnprintf_c_l            100f66a0 f   LIBCMTD:vsnprnc.obj
 0002:000846f0       __vsprintf_s_l             100f66f0 f   LIBCMTD:vsnprnc.obj
 0002:00084960       _vsprintf_s                100f6960 f   LIBCMTD:vsnprnc.obj
 0002:00084990       __vsnprintf_s_l            100f6990 f   LIBCMTD:vsnprnc.obj
 0002:00084d30       __vsnprintf_s              100f6d30 f   LIBCMTD:vsnprnc.obj
 0002:00084d60       __vsprintf_p               100f6d60 f   LIBCMTD:vsnprnc.obj
 0002:00084db0       __vsprintf_p_l             100f6db0 f   LIBCMTD:vsnprnc.obj
 0002:00084e00       _strtol                    100f6e00 f   LIBCMTD:strtol.obj
 0002:00085330       __strtol_l                 100f7330 f   LIBCMTD:strtol.obj
 0002:00085360       _strtoul                   100f7360 f   LIBCMTD:strtol.obj
 0002:000853b0       __strtoul_l                100f73b0 f   LIBCMTD:strtol.obj
 0002:000853e0       __strtoi64                 100f73e0 f   LIBCMTD:strtoq.obj
 0002:00085950       __strtoi64_l               100f7950 f   LIBCMTD:strtoq.obj
 0002:00085980       __strtoui64                100f7980 f   LIBCMTD:strtoq.obj
 0002:000859d0       __strtoui64_l              100f79d0 f   LIBCMTD:strtoq.obj
 0002:00085a00       ?_RTC_GetSrcLine@@YAHPAEPA_WKPAH1K@Z 100f7a00 f   LIBCMTD:_pdblkup_.obj
 0002:00085ea0       __fltin2                   100f7ea0 f   LIBCMTD:_cfin_.obj
 0002:00085f80       __chvalidator              100f7f80 f   LIBCMTD:isctype.obj
 0002:00085fd0       __chvalidator_l            100f7fd0 f   LIBCMTD:isctype.obj
 0002:00086080       __isctype_l                100f8080 f   LIBCMTD:isctype.obj
 0002:000861a0       __isctype                  100f81a0 f   LIBCMTD:isctype.obj
 0002:000861e0       ___strgtold12_l            100f81e0 f   LIBCMTD:_strgtold_.obj
 0002:00086c90       ___multtenpow12            100f8c90 f i LIBCMTD:_strgtold_.obj
 0002:00086d70       ___ld12mul                 100f8d70 f i LIBCMTD:_strgtold_.obj
 0002:00087170       ___addl                    100f9170 f i LIBCMTD:_strgtold_.obj
 0002:000871b0       ___shl_12                  100f91b0 f i LIBCMTD:_strgtold_.obj
 0002:00087220       ___shr_12                  100f9220 f i LIBCMTD:_strgtold_.obj
 0002:00087290       ___STRINGTOLD_L            100f9290 f   LIBCMTD:_strgtold_.obj
 0002:00087300       __validate_param_reuseA    100f9300 f   LIBCMTD:outputp.obj
 0002:00087570       __output_p_l               100f9570 f   LIBCMTD:outputp.obj
 0002:0008b130       _get_crtdouble_arg         100fd130 f i LIBCMTD:outputp.obj
 0002:0008b150       __ismbbkalnum_l            100fd150 f   LIBCMTD:ismbbyte.obj
 0002:0008b170       __ismbbkalnum              100fd170 f   LIBCMTD:ismbbyte.obj
 0002:0008b190       __ismbbkprint_l            100fd190 f   LIBCMTD:ismbbyte.obj
 0002:0008b1b0       __ismbbkprint              100fd1b0 f   LIBCMTD:ismbbyte.obj
 0002:0008b1d0       __ismbbkpunct_l            100fd1d0 f   LIBCMTD:ismbbyte.obj
 0002:0008b1f0       __ismbbkpunct              100fd1f0 f   LIBCMTD:ismbbyte.obj
 0002:0008b210       __ismbbalnum_l             100fd210 f   LIBCMTD:ismbbyte.obj
 0002:0008b230       __ismbbalnum               100fd230 f   LIBCMTD:ismbbyte.obj
 0002:0008b250       __ismbbalpha_l             100fd250 f   LIBCMTD:ismbbyte.obj
 0002:0008b270       __ismbbalpha               100fd270 f   LIBCMTD:ismbbyte.obj
 0002:0008b290       __ismbbgraph_l             100fd290 f   LIBCMTD:ismbbyte.obj
 0002:0008b2b0       __ismbbgraph               100fd2b0 f   LIBCMTD:ismbbyte.obj
 0002:0008b2d0       __ismbbprint_l             100fd2d0 f   LIBCMTD:ismbbyte.obj
 0002:0008b2f0       __ismbbprint               100fd2f0 f   LIBCMTD:ismbbyte.obj
 0002:0008b310       __ismbbpunct_l             100fd310 f   LIBCMTD:ismbbyte.obj
 0002:0008b330       __ismbbpunct               100fd330 f   LIBCMTD:ismbbyte.obj
 0002:0008b350       __ismbblead_l              100fd350 f   LIBCMTD:ismbbyte.obj
 0002:0008b370       __ismbblead                100fd370 f   LIBCMTD:ismbbyte.obj
 0002:0008b390       __ismbbtrail_l             100fd390 f   LIBCMTD:ismbbyte.obj
 0002:0008b3b0       __ismbbtrail               100fd3b0 f   LIBCMTD:ismbbyte.obj
 0002:0008b3d0       __ismbbkana_l              100fd3d0 f   LIBCMTD:ismbbyte.obj
 0002:0008b440       __ismbbkana                100fd440 f   LIBCMTD:ismbbyte.obj
 0002:0008b530       __mbsnbcpy_s               100fd530 f   LIBCMTD:mbsnbcpy_s.obj
 0002:0008b560       __makepath_s               100fd560 f   LIBCMTD:makepath_s.obj
 0002:0008b900       __openfile                 100fd900 f   LIBCMTD:_open.obj
 0002:0008c0c0       __getstream                100fe0c0 f   LIBCMTD:stream.obj
 0002:0008c320       __local_unwind4            100fe320 f   LIBCMTD:exsup4.obj
 0002:0008c3f6       __seh_longjmp_unwind4@4    100fe3f6 f   LIBCMTD:exsup4.obj
 0002:0008c412       @_EH4_CallFilterFunc@8     100fe412 f   LIBCMTD:exsup4.obj
 0002:0008c429       @_EH4_TransferToHandler@8  100fe429 f   LIBCMTD:exsup4.obj
 0002:0008c442       @_EH4_GlobalUnwind@4       100fe442 f   LIBCMTD:exsup4.obj
 0002:0008c45c       @_EH4_LocalUnwind@16       100fe45c f   LIBCMTD:exsup4.obj
 0002:0008c480       __close                    100fe480 f   LIBCMTD:close.obj
 0002:0008c690       __close_nolock             100fe690 f   LIBCMTD:close.obj
 0002:0008c760       __fileno                   100fe760 f   LIBCMTD:fileno.obj
 0002:0008c760       _fileno                    100fe760 f   LIBCMTD:fileno.obj
 0002:0008c7e0       __freebuf                  100fe7e0 f   LIBCMTD:_freebuf.obj
 0002:0008c870       __ioinit                   100fe870 f   LIBCMTD:ioinit.obj
 0002:0008cd10       __ioterm                   100fed10 f   LIBCMTD:ioinit.obj
 0002:0008cdb0       __lseek                    100fedb0 f   LIBCMTD:lseek.obj
 0002:0008cfe0       __lseek_nolock             100fefe0 f   LIBCMTD:lseek.obj
 0002:0008d0c0       __filbuf                   100ff0c0 f   LIBCMTD:_filbuf.obj
 0002:0008d310       __read                     100ff310 f   LIBCMTD:read.obj
 0002:0008d5a0       __read_nolock              100ff5a0 f   LIBCMTD:read.obj
 0002:0008e4f0       __CIatan_pentium4          101004f0 f   LIBCMTD:_atan_pentium4_.obj
 0002:0008e508       __atan_pentium4            10100508     LIBCMTD:_atan_pentium4_.obj
 0002:0008e7e0       __handle_qnan1             101007e0 f   LIBCMTD:_fpexcept_.obj
 0002:0008e840       __handle_qnan2             10100840 f   LIBCMTD:_fpexcept_.obj
 0002:0008e8b0       __except1                  101008b0 f   LIBCMTD:_fpexcept_.obj
 0002:0008e9b0       __except2                  101009b0 f   LIBCMTD:_fpexcept_.obj
 0002:0008eac0       __raise_exc_ex             10100ac0 f   LIBCMTD:_fpexcept_.obj
 0002:0008eff0       __raise_exc                10100ff0 f   LIBCMTD:_fpexcept_.obj
 0002:0008f020       __raise_excf               10101020 f   LIBCMTD:_fpexcept_.obj
 0002:0008f050       __handle_exc               10101050 f   LIBCMTD:_fpexcept_.obj
 0002:0008f360       __umatherr                 10101360 f   LIBCMTD:_fpexcept_.obj
 0002:0008f400       __set_errno_from_matherr   10101400 f   LIBCMTD:_fpexcept_.obj
 0002:0008f490       __errcode                  10101490 f   LIBCMTD:_fpexcept_.obj
 0002:0008f500       __set_exp                  10101500 f   LIBCMTD:_util_.obj
 0002:0008f540       __get_exp                  10101540 f   LIBCMTD:_util_.obj
 0002:0008f570       __add_exp                  10101570 f   LIBCMTD:_util_.obj
 0002:0008f5b0       __set_bexp                 101015b0 f   LIBCMTD:_util_.obj
 0002:0008f5e0       __sptype                   101015e0 f   LIBCMTD:_util_.obj
 0002:0008f660       __decomp                   10101660 f   LIBCMTD:_util_.obj
 0002:0008f780       __statfp                   10101780 f   LIBCMTD:_fpctrl_.obj
 0002:0008f7a0       __clrfp                    101017a0 f   LIBCMTD:_fpctrl_.obj
 0002:0008f7c0       __ctrlfp                   101017c0 f   LIBCMTD:_fpctrl_.obj
 0002:0008f7f0       __set_statfp               101017f0 f   LIBCMTD:_fpctrl_.obj
 0002:0008f860       ___get_fpsr_sse2           10101860 f   LIBCMTD:_fpctrl_.obj
 0002:0008f890       ___set_fpsr_sse2           10101890 f   LIBCMTD:_fpctrl_.obj
 0002:0008f970       ___fclrf_sse2              10101970 f   LIBCMTD:_fpctrl_.obj
 0002:0008f990       ___statfp_sse2             10101990 f   LIBCMTD:_fpctrl_.obj
 0002:0008f9c0       ___clrfp_sse2              101019c0 f   LIBCMTD:_fpctrl_.obj
 0002:0008fa00       ___ctrlfp_sse2             10101a00 f   LIBCMTD:_fpctrl_.obj
 0002:0008fa60       ___set_statfp_sse2         10101a60 f   LIBCMTD:_fpctrl_.obj
 0002:0008fa90       __CIacos_pentium4          10101a90 f   LIBCMTD:_acos_pentium4_.obj
 0002:0008faa8       __acos_pentium4            10101aa8     LIBCMTD:_acos_pentium4_.obj
 0002:0008fff0       __CIcos_pentium4           10101ff0 f   LIBCMTD:_cos_pentium4_.obj
 0002:00090008       __cos_pentium4             10102008     LIBCMTD:_cos_pentium4_.obj
 0002:000901a0       __CIsin_pentium4           101021a0 f   LIBCMTD:_sin_pentium4_.obj
 0002:000901b8       __sin_pentium4             101021b8     LIBCMTD:_sin_pentium4_.obj
 0002:00090370       __CIasin_pentium4          10102370 f   LIBCMTD:_asin_pentium4_.obj
 0002:00090388       __asin_pentium4            10102388     LIBCMTD:_asin_pentium4_.obj
 0002:000908f0       __stbuf                    101028f0 f   LIBCMTD:_sftbuf.obj
 0002:00090a50       __ftbuf                    10102a50 f   LIBCMTD:_sftbuf.obj
 0002:00090ae0       _vprintf_helper            10102ae0 f   LIBCMTD:vprintf.obj
 0002:00090c00       __vprintf_l                10102c00 f   LIBCMTD:vprintf.obj
 0002:00090c20       __vprintf_s_l              10102c20 f   LIBCMTD:vprintf.obj
 0002:00090c40       __vprintf_p_l              10102c40 f   LIBCMTD:vprintf.obj
 0002:00090c60       _vprintf                   10102c60 f   LIBCMTD:vprintf.obj
 0002:00090c80       _vprintf_s                 10102c80 f   LIBCMTD:vprintf.obj
 0002:00090ca0       __vprintf_p                10102ca0 f   LIBCMTD:vprintf.obj
 0002:00090cc0       __write                    10102cc0 f   LIBCMTD:write.obj
 0002:00090ef0       __write_nolock             10102ef0 f   LIBCMTD:write.obj
 0002:00091a30       _V6_HeapAlloc              10103a30 f   LIBCMTD:malloc.obj
 0002:00091ad0       __malloc_base              10103ad0 f   LIBCMTD:malloc.obj
 0002:00091b60       __heap_alloc_base          10103b60 f i LIBCMTD:malloc.obj
 0002:00091c20       __CrtSetReportHook2        10103c20 f   LIBCMTD:dbgrpt.obj
 0002:00091f40       __CrtDbgReport             10103f40 f   LIBCMTD:dbgrpt.obj
 0002:00091f80       __CrtDbgReportV            10103f80 f i LIBCMTD:dbgrpt.obj
 0002:00091fb0       ___crtMessageWindowA       10103fb0 f   LIBCMTD:dbgrpt.obj
 0002:000923b0       __expand_base              101043b0 f   LIBCMTD:expand.obj
 0002:00092680       __realloc_base             10104680 f   LIBCMTD:realloc.obj
 0002:00092a20       __free_base                10104a20 f   LIBCMTD:free.obj
 0002:00092b50       __heapchk                  10104b50 f   LIBCMTD:heapchk.obj
 0002:00092c20       __heapset                  10104c20 f   LIBCMTD:heapchk.obj
 0002:00092c30       ___heap_select             10104c30 f   LIBCMTD:heapinit.obj
 0002:00092c50       __heap_init                10104c50 f   LIBCMTD:heapinit.obj
 0002:00092cd0       __heap_term                10104cd0 f   LIBCMTD:heapinit.obj
 0002:00092d70       __get_heap_handle          10104d70 f   LIBCMTD:heapinit.obj
 0002:00092db0       __get_sbh_threshold        10104db0 f   LIBCMTD:sbheap.obj
 0002:00092e00       __set_sbh_threshold        10104e00 f   LIBCMTD:sbheap.obj
 0002:00092f90       __set_amblksiz             10104f90 f   LIBCMTD:sbheap.obj
 0002:000930a0       __get_amblksiz             101050a0 f   LIBCMTD:sbheap.obj
 0002:00093190       ___sbh_heap_init           10105190 f   LIBCMTD:sbheap.obj
 0002:00093200       ___sbh_find_block          10105200 f   LIBCMTD:sbheap.obj
 0002:00093260       ___sbh_verify_block        10105260 f   LIBCMTD:sbheap.obj
 0002:000932c0       ___sbh_free_block          101052c0 f   LIBCMTD:sbheap.obj
 0002:00093880       ___sbh_alloc_block         10105880 f   LIBCMTD:sbheap.obj
 0002:00093da0       ___sbh_alloc_new_region    10105da0 f   LIBCMTD:sbheap.obj
 0002:00093eb0       ___sbh_alloc_new_group     10105eb0 f   LIBCMTD:sbheap.obj
 0002:000940a0       ___sbh_resize_block        101060a0 f   LIBCMTD:sbheap.obj
 0002:00094670       ___sbh_heapmin             10106670 f   LIBCMTD:sbheap.obj
 0002:000947a0       ___sbh_heap_check          101067a0 f   LIBCMTD:sbheap.obj
 0002:00094c90       __setenvp                  10106c90 f   LIBCMTD:stdenvp.obj
 0002:00094e30       __setargv                  10106e30 f   LIBCMTD:stdargv.obj
 0002:00094f50       __set_pgmptr               10106f50 f i LIBCMTD:stdargv.obj
 0002:000952c0       ___crtGetEnvironmentStringsA 101072c0 f   LIBCMTD:a_env.obj
 0002:000954e0       __RTC_Initialize           101074e0 f   LIBCMTD:_initsect_.obj
 0002:00095510       __RTC_Terminate            10107510 f   LIBCMTD:_initsect_.obj
 0002:00095540       ___security_init_cookie    10107540 f   LIBCMTD:gs_support.obj
 0002:00095620       __initp_misc_winxfltr      10107620 f   LIBCMTD:winxfltr.obj
 0002:00095630       ___CppXcptFilter           10107630 f   LIBCMTD:winxfltr.obj
 0002:00095660       __XcptFilter               10107660 f   LIBCMTD:winxfltr.obj
 0002:00095890       __FF_MSGBANNER             10107890 f   LIBCMTD:crt0msg.obj
 0002:000958e0       __NMSG_WRITE               101078e0 f   LIBCMTD:crt0msg.obj
 0002:00095b80       __GET_RTERRMSG             10107b80 f   LIBCMTD:crt0msg.obj
 0002:00095bd0       __fcloseall                10107bd0 f   LIBCMTD:closeall.obj
 0002:00095d00       __commit                   10107d00 f   LIBCMTD:commit.obj
 0002:00095f20       ___libm_setusermatherr     10107f20 f   LIBCMTD:_libm_error_.obj
 0002:00095f60       ___libm_error_support      10107f60 f   LIBCMTD:_libm_error_.obj
 0002:00096aa0       __floor_default            10108aa0 f   LIBCMTD:_floor_.obj
 0002:00096be0       ___crtLCMapStringA         10108be0 f   LIBCMTD:a_map.obj
 0002:00097140       __MarkAllocaS              10109140 f i LIBCMTD:a_map.obj
 0002:00097170       __freea                    10109170 f i LIBCMTD:a_map.obj
 0002:00097230       __isleadbyte_l             10109230 f i LIBCMTD:_wctype.obj
 0002:00097280       _isleadbyte                10109280 f i LIBCMTD:_wctype.obj
 0002:000972a0       __iswalpha_l               101092a0 f i LIBCMTD:_wctype.obj
 0002:000972c0       _iswalpha                  101092c0 f i LIBCMTD:_wctype.obj
 0002:000972e0       __iswupper_l               101092e0 f i LIBCMTD:_wctype.obj
 0002:00097300       _iswupper                  10109300 f i LIBCMTD:_wctype.obj
 0002:00097320       __iswlower_l               10109320 f i LIBCMTD:_wctype.obj
 0002:00097340       _iswlower                  10109340 f i LIBCMTD:_wctype.obj
 0002:00097360       __iswdigit_l               10109360 f i LIBCMTD:_wctype.obj
 0002:00097380       _iswdigit                  10109380 f i LIBCMTD:_wctype.obj
 0002:000973a0       __iswxdigit_l              101093a0 f i LIBCMTD:_wctype.obj
 0002:000973c0       _iswxdigit                 101093c0 f i LIBCMTD:_wctype.obj
 0002:000973e0       __iswspace_l               101093e0 f i LIBCMTD:_wctype.obj
 0002:00097400       _iswspace                  10109400 f i LIBCMTD:_wctype.obj
 0002:00097420       __iswpunct_l               10109420 f i LIBCMTD:_wctype.obj
 0002:00097440       _iswpunct                  10109440 f i LIBCMTD:_wctype.obj
 0002:00097460       __iswalnum_l               10109460 f i LIBCMTD:_wctype.obj
 0002:00097480       _iswalnum                  10109480 f i LIBCMTD:_wctype.obj
 0002:000974a0       __iswprint_l               101094a0 f i LIBCMTD:_wctype.obj
 0002:000974c0       _iswprint                  101094c0 f i LIBCMTD:_wctype.obj
 0002:000974e0       __iswgraph_l               101094e0 f i LIBCMTD:_wctype.obj
 0002:00097500       _iswgraph                  10109500 f i LIBCMTD:_wctype.obj
 0002:00097520       __iswcntrl_l               10109520 f i LIBCMTD:_wctype.obj
 0002:00097540       _iswcntrl                  10109540 f i LIBCMTD:_wctype.obj
 0002:00097560       _iswascii                  10109560 f i LIBCMTD:_wctype.obj
 0002:00097580       __iswcsym_l                10109580 f i LIBCMTD:_wctype.obj
 0002:000975c0       ___iswcsym                 101095c0 f i LIBCMTD:_wctype.obj
 0002:00097600       __iswcsymf_l               10109600 f i LIBCMTD:_wctype.obj
 0002:00097640       ___iswcsymf                10109640 f i LIBCMTD:_wctype.obj
 0002:00097680       _vfprintf_helper           10109680 f   LIBCMTD:vfprintf.obj
 0002:00097920       __vfprintf_l               10109920 f   LIBCMTD:vfprintf.obj
 0002:00097950       __vfprintf_s_l             10109950 f   LIBCMTD:vfprintf.obj
 0002:00097980       __vfprintf_p_l             10109980 f   LIBCMTD:vfprintf.obj
 0002:000979b0       _vfprintf                  101099b0 f   LIBCMTD:vfprintf.obj
 0002:000979e0       _vfprintf_s                101099e0 f   LIBCMTD:vfprintf.obj
 0002:00097a10       __vfprintf_p               10109a10 f   LIBCMTD:vfprintf.obj
 0002:00097a40       __alloc_osfhnd             10109a40 f   LIBCMTD:osfinfo.obj
 0002:00097cf0       __set_osfhnd               10109cf0 f   LIBCMTD:osfinfo.obj
 0002:00097dc0       __free_osfhnd              10109dc0 f   LIBCMTD:osfinfo.obj
 0002:00097eb0       __get_osfhandle            10109eb0 f   LIBCMTD:osfinfo.obj
 0002:00098020       __open_osfhandle           1010a020 f   LIBCMTD:osfinfo.obj
 0002:00098250       ___lock_fhandle            1010a250 f   LIBCMTD:osfinfo.obj
 0002:00098350       __unlock_fhandle           1010a350 f   LIBCMTD:osfinfo.obj
 0002:00098380       ___sys_nerr                1010a380 f   LIBCMTD:syserr.obj
 0002:00098390       ___sys_errlist             1010a390 f   LIBCMTD:syserr.obj
 0002:000983a0       __ceil_default             1010a3a0 f   LIBCMTD:_ceil_.obj
 0002:000984e0       __ValidateImageBase        1010a4e0 f   LIBCMTD:pesect.obj
 0002:00098540       __FindPESection            1010a540 f   LIBCMTD:pesect.obj
 0002:000985c0       __IsNonwritableInCurrentImage 1010a5c0 f   LIBCMTD:pesect.obj
 0002:000986e0       __initp_misc_rand_s        1010a6e0 f   LIBCMTD:rand_s.obj
 0002:000986f0       _rand_s                    1010a6f0 f   LIBCMTD:rand_s.obj
 0002:00098910       ___getlocaleinfo           1010a910 f   LIBCMTD:inithelp.obj
 0002:00098bb0       __initp_misc_purevirt      1010abb0 f   LIBCMTD:inithelp.obj
 0002:00098bc0       __initp_misc_initcrit      1010abc0 f   LIBCMTD:initcrit.obj
 0002:00098bd0       ___crtInitCritSecAndSpinCount 1010abd0 f   LIBCMTD:initcrit.obj
 0002:00098c80       ___crtGetStringTypeA       1010ac80 f   LIBCMTD:a_str.obj
 0002:00098f10       ___pwctype_func            1010af10 f   LIBCMTD:ctype.obj
 0002:00098f20       ___pctype_func             1010af20 f   LIBCMTD:ctype.obj
 0002:00098f70       ___init_time               1010af70 f   LIBCMTD:inittime.obj
 0002:00099690       ___free_lc_time            1010b690 f   LIBCMTD:inittime.obj
 0002:000999a0       ___init_numeric            1010b9a0 f   LIBCMTD:initnum.obj
 0002:00099d00       ___free_lconv_num          1010bd00 f   LIBCMTD:initnum.obj
 0002:00099d70       ___init_monetary           1010bd70 f   LIBCMTD:initmon.obj
 0002:0009a270       ___free_lconv_mon          1010c270 f   LIBCMTD:initmon.obj
 0002:0009a360       ___init_ctype              1010c360 f   LIBCMTD:initctyp.obj
 0002:0009a910       ____mb_cur_max_func        1010c910 f   LIBCMTD:initctyp.obj
 0002:0009a960       ____mb_cur_max_l_func      1010c960 f   LIBCMTD:initctyp.obj
 0002:0009a990       ____lc_codepage_func       1010c990 f   LIBCMTD:initctyp.obj
 0002:0009a9e0       ____lc_collate_cp_func     1010c9e0 f   LIBCMTD:initctyp.obj
 0002:0009aa30       ____lc_handle_func         1010ca30 f   LIBCMTD:initctyp.obj
 0002:0009aa80       ___init_collate            1010ca80 f   LIBCMTD:initcoll.obj
 0002:0009aa90       __Getdays_l                1010ca90 f   LIBCMTD:strftime.obj
 0002:0009ac50       __Getdays                  1010cc50 f   LIBCMTD:strftime.obj
 0002:0009ac70       __Getmonths_l              1010cc70 f   LIBCMTD:strftime.obj
 0002:0009ae30       __Getmonths                1010ce30 f   LIBCMTD:strftime.obj
 0002:0009ae50       __Gettnames_l              1010ce50 f   LIBCMTD:strftime.obj
 0002:0009b3c0       __Gettnames                1010d3c0 f   LIBCMTD:strftime.obj
 0002:0009b3e0       __strftime_l               1010d3e0 f   LIBCMTD:strftime.obj
 0002:0009b410       _strftime                  1010d410 f   LIBCMTD:strftime.obj
 0002:0009b440       __Strftime                 1010d440 f   LIBCMTD:strftime.obj
 0002:0009b470       __Strftime_l               1010d470 f   LIBCMTD:strftime.obj
 0002:0009d280       _localeconv                1010f280 f   LIBCMTD:lconv.obj
 0002:0009d2d0       _strncpy_s                 1010f2d0 f   LIBCMTD:strncpy_s.obj
 0002:0009d6c0       _strcspn                   1010f6c0 f   LIBCMTD:strcspn.obj
 0002:0009d710       _strncmp                   1010f710 f   LIBCMTD:strncmp.obj
 0002:0009d890       _strpbrk                   1010f890 f   LIBCMTD:strpbrk.obj
 0002:0009d8d0       _strcat_s                  1010f8d0 f   LIBCMTD:strcat_s.obj
 0002:0009dcb0       ___get_qualified_locale    1010fcb0 f   LIBCMTD:getqloc.obj
 0002:0009eb50       __controlfp_s              10110b50 f   LIBCMTD:_contrlfp_.obj
 0002:0009ec30       __isalpha_l                10110c30 f i LIBCMTD:_ctype.obj
 0002:0009ecc0       _isalpha                   10110cc0 f i LIBCMTD:_ctype.obj
 0002:0009ed00       __isupper_l                10110d00 f i LIBCMTD:_ctype.obj
 0002:0009ed80       _isupper                   10110d80 f i LIBCMTD:_ctype.obj
 0002:0009edb0       __islower_l                10110db0 f i LIBCMTD:_ctype.obj
 0002:0009ee30       _islower                   10110e30 f i LIBCMTD:_ctype.obj
 0002:0009ee60       __isdigit_l                10110e60 f i LIBCMTD:_ctype.obj
 0002:0009eee0       _isdigit                   10110ee0 f i LIBCMTD:_ctype.obj
 0002:0009ef10       __isxdigit_l               10110f10 f i LIBCMTD:_ctype.obj
 0002:0009efa0       _isxdigit                  10110fa0 f i LIBCMTD:_ctype.obj
 0002:0009efe0       __isspace_l                10110fe0 f i LIBCMTD:_ctype.obj
 0002:0009f060       _isspace                   10111060 f i LIBCMTD:_ctype.obj
 0002:0009f090       __ispunct_l                10111090 f i LIBCMTD:_ctype.obj
 0002:0009f110       _ispunct                   10111110 f i LIBCMTD:_ctype.obj
 0002:0009f140       __isalnum_l                10111140 f i LIBCMTD:_ctype.obj
 0002:0009f1d0       _isalnum                   101111d0 f i LIBCMTD:_ctype.obj
 0002:0009f210       __isprint_l                10111210 f i LIBCMTD:_ctype.obj
 0002:0009f2a0       _isprint                   101112a0 f i LIBCMTD:_ctype.obj
 0002:0009f2e0       __isgraph_l                101112e0 f i LIBCMTD:_ctype.obj
 0002:0009f370       _isgraph                   10111370 f i LIBCMTD:_ctype.obj
 0002:0009f3b0       __iscntrl_l                101113b0 f i LIBCMTD:_ctype.obj
 0002:0009f430       _iscntrl                   10111430 f i LIBCMTD:_ctype.obj
 0002:0009f460       ___isascii                 10111460 f i LIBCMTD:_ctype.obj
 0002:0009f480       ___toascii                 10111480 f i LIBCMTD:_ctype.obj
 0002:0009f490       __iscsymf_l                10111490 f i LIBCMTD:_ctype.obj
 0002:0009f4d0       ___iscsymf                 101114d0 f i LIBCMTD:_ctype.obj
 0002:0009f510       __iscsym_l                 10111510 f i LIBCMTD:_ctype.obj
 0002:0009f550       ___iscsym                  10111550 f i LIBCMTD:_ctype.obj
 0002:0009f590       __atodbl_l                 10111590 f   LIBCMTD:atodbl.obj
 0002:0009f6a0       __atodbl                   101116a0 f   LIBCMTD:atodbl.obj
 0002:0009f6c0       __atoldbl_l                101116c0 f   LIBCMTD:atodbl.obj
 0002:0009f7d0       __atoldbl                  101117d0 f   LIBCMTD:atodbl.obj
 0002:0009f7f0       __atoflt_l                 101117f0 f   LIBCMTD:atodbl.obj
 0002:0009f900       __atoflt                   10111900 f   LIBCMTD:atodbl.obj
 0002:0009f920       __fptostr                  10111920 f   LIBCMTD:_fptostr.obj
 0002:0009fbd0       __fltout2                  10111bd0 f   LIBCMTD:_cfout_.obj
 0002:0009fc80       ___dtold                   10111c80 f   LIBCMTD:_cfout_.obj
 0002:0009fde0       __set_output_format        10111de0 f   LIBCMTD:outputformat.obj
 0002:0009fe60       __get_output_format        10111e60 f   LIBCMTD:outputformat.obj
 0002:0009fe70       __allrem                   10111e70 f   LIBCMTD:llrem.obj
 0002:0009ff30       __allshl                   10111f30 f   LIBCMTD:llshl.obj
 0002:0009ff50       __aullshr                  10111f50 f   LIBCMTD:ullshr.obj
 0002:0009ff70       _strrchr                   10111f70 f   LIBCMTD:strrchr.obj
 0002:0009ffa0       __fptrap                   10111fa0 f   LIBCMTD:crt0fp.obj
 0002:0009ffc0       _fdiv_main_routine         10111fc0 f   LIBCMTD:_adj_fdiv_.obj
 0002:000a00d7       __adj_fdiv_r               101120d7 f   LIBCMTD:_adj_fdiv_.obj
 0002:000a0576       __fdivp_sti_st             10112576 f   LIBCMTD:_adj_fdiv_.obj
 0002:000a0589       __fdivrp_sti_st            10112589 f   LIBCMTD:_adj_fdiv_.obj
 0002:000a059c       __adj_fdiv_m32             1011259c f   LIBCMTD:_adj_fdiv_.obj
 0002:000a05e8       __adj_fdiv_m64             101125e8 f   LIBCMTD:_adj_fdiv_.obj
 0002:000a0634       __adj_fdiv_m16i            10112634 f   LIBCMTD:_adj_fdiv_.obj
 0002:000a0668       __adj_fdiv_m32i            10112668 f   LIBCMTD:_adj_fdiv_.obj
 0002:000a069c       __adj_fdivr_m32            1011269c f   LIBCMTD:_adj_fdiv_.obj
 0002:000a06e8       __adj_fdivr_m64            101126e8 f   LIBCMTD:_adj_fdiv_.obj
 0002:000a0734       __adj_fdivr_m16i           10112734 f   LIBCMTD:_adj_fdiv_.obj
 0002:000a0768       __adj_fdivr_m32i           10112768 f   LIBCMTD:_adj_fdiv_.obj
 0002:000a079c       __safe_fdiv                1011279c f   LIBCMTD:_adj_fdiv_.obj
 0002:000a07b1       __safe_fdivr               101127b1 f   LIBCMTD:_adj_fdiv_.obj
 0002:000a07c6       __fprem_common             101127c6 f   LIBCMTD:_adj_fdiv_.obj
 0002:000a09cc       __adj_fprem                101129cc f   LIBCMTD:_adj_fdiv_.obj
 0002:000a0a7e       __fprem1_common            10112a7e f   LIBCMTD:_adj_fdiv_.obj
 0002:000a0c84       __adj_fprem1               10112c84 f   LIBCMTD:_adj_fdiv_.obj
 0002:000a0d39       __safe_fprem               10112d39 f   LIBCMTD:_adj_fdiv_.obj
 0002:000a0d3f       __safe_fprem1              10112d3f f   LIBCMTD:_adj_fdiv_.obj
 0002:000a0d45       __adj_fpatan               10112d45 f   LIBCMTD:_adj_fdiv_.obj
 0002:000a0d48       __adj_fptan                10112d48 f   LIBCMTD:_adj_fdiv_.obj
 0002:000a0d50       __87except                 10112d50 f   LIBCMTD:_87except_.obj
 0002:000a0f00       __frnd                     10112f00 f   LIBCMTD:_frnd_.obj
 0002:000a0f20       ?_ValidateRead@@YAHPBXI@Z  10112f20 f   LIBCMTD:validate.obj
 0002:000a0f50       ?_ValidateWrite@@YAHPAXI@Z 10112f50 f   LIBCMTD:validate.obj
 0002:000a0f80       ?_ValidateExecute@@YAHP6GHXZ@Z 10112f80 f   LIBCMTD:validate.obj
 0002:000a0fa4       __global_unwind2           10112fa4 f   LIBCMTD:exsup.obj
 0002:000a1009       __local_unwind2            10113009 f   LIBCMTD:exsup.obj
 0002:000a108d       __abnormal_termination     1011308d f   LIBCMTD:exsup.obj
 0002:000a10b0       __NLG_Notify1              101130b0 f   LIBCMTD:exsup.obj
 0002:000a10b9       __NLG_Notify               101130b9 f   LIBCMTD:exsup.obj
 0002:000a10d0       __NLG_Dispatch2            101130d0     LIBCMTD:exsup.obj
 0002:000a10d0       __NLG_Dispatch             101130d0     LIBCMTD:exsup.obj
 0002:000a10d8       __NLG_Call                 101130d8 f   LIBCMTD:exsup.obj
 0002:000a10da       __NLG_Return2              101130da     LIBCMTD:exsup.obj
 0002:000a10e0       __mbstowcs_l_helper        101130e0 f   LIBCMTD:mbstowcs.obj
 0002:000a1430       __mbstowcs_l               10113430 f   LIBCMTD:mbstowcs.obj
 0002:000a1450       _mbstowcs                  10113450 f   LIBCMTD:mbstowcs.obj
 0002:000a14a0       __mbstowcs_s_l             101134a0 f   LIBCMTD:mbstowcs.obj
 0002:000a1820       _mbstowcs_s                10113820 f   LIBCMTD:mbstowcs.obj
 0002:000a1850       __itoa_s                   10113850 f   LIBCMTD:xtoas.obj
 0002:000a1c20       __ltoa_s                   10113c20 f   LIBCMTD:xtoas.obj
 0002:000a1c60       __ultoa_s                  10113c60 f   LIBCMTD:xtoas.obj
 0002:000a1c80       __i64toa_s                 10113c80 f   LIBCMTD:xtoas.obj
 0002:000a2080       __ui64toa_s                10114080 f   LIBCMTD:xtoas.obj
 0002:000a20a0       __wcstombs_l_helper        101140a0 f   LIBCMTD:wcstombs.obj
 0002:000a2590       __wcstombs_l               10114590 f   LIBCMTD:wcstombs.obj
 0002:000a25b0       _wcstombs                  101145b0 f   LIBCMTD:wcstombs.obj
 0002:000a25d0       __wcstombs_s_l             101145d0 f   LIBCMTD:wcstombs.obj
 0002:000a2900       _wcstombs_s                10114900 f   LIBCMTD:wcstombs.obj
 0002:000a2930       _wcscat_s                  10114930 f   LIBCMTD:wcscat_s.obj
 0002:000a2d20       __vswprintf_helper         10114d20 f   LIBCMTD:vswprnc.obj
 0002:000a2f50       __vswprintf_c              10114f50 f   LIBCMTD:vswprnc.obj
 0002:000a2fa0       __vswprintf_c_l            10114fa0 f   LIBCMTD:vswprnc.obj
 0002:000a2ff0       __vswprintf_s_l            10114ff0 f   LIBCMTD:vswprnc.obj
 0002:000a3260       _vswprintf_s               10115260 f   LIBCMTD:vswprnc.obj
 0002:000a3290       __vsnwprintf_s_l           10115290 f   LIBCMTD:vswprnc.obj
 0002:000a3640       __vsnwprintf_s             10115640 f   LIBCMTD:vswprnc.obj
 0002:000a3670       __vswprintf_p              10115670 f   LIBCMTD:vswprnc.obj
 0002:000a36c0       __vswprintf_p_l            101156c0 f   LIBCMTD:vswprnc.obj
 0002:000a3710       __itow_s                   10115710 f   LIBCMTD:xtows.obj
 0002:000a3af0       __ltow_s                   10115af0 f   LIBCMTD:xtows.obj
 0002:000a3b30       __ultow_s                  10115b30 f   LIBCMTD:xtows.obj
 0002:000a3b50       __i64tow_s                 10115b50 f   LIBCMTD:xtows.obj
 0002:000a3f70       __ui64tow_s                10115f70 f   LIBCMTD:xtows.obj
 0002:000a3f90       __woutput_l                10115f90 f   LIBCMTD:woutput.obj
 0002:000a5160       __vswprintf_l              10117160 f   LIBCMTD:vswprint.obj
 0002:000a5330       __vswprintf                10117330 f   LIBCMTD:vswprint.obj
 0002:000a5350       ___vswprintf_l             10117350 f   LIBCMTD:vswprint.obj
 0002:000a5370       __vscwprintf_helper        10117370 f   LIBCMTD:vswprint.obj
 0002:000a5430       __vscwprintf               10117430 f   LIBCMTD:vswprint.obj
 0002:000a5450       __vscwprintf_l             10117450 f   LIBCMTD:vswprint.obj
 0002:000a5470       __vscwprintf_p             10117470 f   LIBCMTD:vswprint.obj
 0002:000a5490       __vscwprintf_p_l           10117490 f   LIBCMTD:vswprint.obj
 0002:000a54b0       ___unDName                 101174b0 f   LIBCMTD:undname.obj
 0002:000a5590       ?Constructor@HeapManager@@QAEXP6APAXI@ZP6AXPAX@Z@Z 10117590 f i LIBCMTD:undname.obj
 0002:000a55d0       ?Destructor@HeapManager@@QAEXXZ 101175d0 f i LIBCMTD:undname.obj
 0002:000a5620       ___unDNameEx               10117620 f   LIBCMTD:undname.obj
 0002:000a5700       ??0UnDecorator@@QAE@PADPBDHP6APADJ@ZK@Z 10117700 f i LIBCMTD:undname.obj
 0002:000a57a0       ??BUnDecorator@@QAEPADXZ   101177a0 f i LIBCMTD:undname.obj
 0002:000a59d0       ?dbGetString@DName@@QBEPADXZ 101179d0 f   LIBCMTD:undname.obj
 0002:000a5a00       ?getDecoratedName@UnDecorator@@CA?AVDName@@XZ 10117a00 f   LIBCMTD:undname.obj
 0002:000a5d10       ?getSymbolName@UnDecorator@@CA?AVDName@@XZ 10117d10 f i LIBCMTD:undname.obj
 0002:000a5d90       ?getZName@UnDecorator@@CA?AVDName@@_N0@Z 10117d90 f   LIBCMTD:undname.obj
 0002:000a6030       ?getOperatorName@UnDecorator@@CA?AVDName@@_NPA_N@Z 10118030 f i LIBCMTD:undname.obj
 0002:000a69a0       ?getStringEncoding@UnDecorator@@CA?AVDName@@PADH@Z 101189a0 f   LIBCMTD:undname.obj
 0002:000a6aa0       ?getScope@UnDecorator@@CA?AVDName@@XZ 10118aa0 f   LIBCMTD:undname.obj
 0002:000a6e80       ?getSignedDimension@UnDecorator@@CA?AVDName@@XZ 10118e80 f   LIBCMTD:undname.obj
 0002:000a6f00       ?getDimension@UnDecorator@@CA?AVDName@@_N@Z 10118f00 f   LIBCMTD:undname.obj
 0002:000a71b0       ?getNumberOfDimensions@UnDecorator@@CAHXZ 101191b0 f   LIBCMTD:undname.obj
 0002:000a72b0       ?getTemplateName@UnDecorator@@CA?AVDName@@_N@Z 101192b0 f   LIBCMTD:undname.obj
 0002:000a7470       ?getTemplateArgumentList@UnDecorator@@CA?AVDName@@XZ 10119470 f   LIBCMTD:undname.obj
 0002:000a76f0       ?getTemplateConstant@UnDecorator@@CA?AVDName@@XZ 101196f0 f   LIBCMTD:undname.obj
 0002:000a7b80       ?composeDeclaration@UnDecorator@@CA?AVDName@@ABV2@@Z 10119b80 f i LIBCMTD:undname.obj
 0002:000a9180       ?getTypeEncoding@UnDecorator@@CAHXZ 1011b180 f i LIBCMTD:undname.obj
 0002:000a9bc0       ?getBasedType@UnDecorator@@CA?AVDName@@XZ 1011bbc0 f   LIBCMTD:undname.obj
 0002:000a9c80       ?getScopedName@UnDecorator@@CA?AVDName@@XZ 1011bc80 f   LIBCMTD:undname.obj
 0002:000a9da0       ?getCallingConvention@UnDecorator@@CA?AVDName@@XZ 1011bda0 f   LIBCMTD:undname.obj
 0002:000a9f00       ?getReturnType@UnDecorator@@CA?AVDName@@PAV2@@Z 1011bf00 f   LIBCMTD:undname.obj
 0002:000a9f50       ?getDataType@UnDecorator@@CA?AVDName@@PAV2@@Z 1011bf50 f   LIBCMTD:undname.obj
 0002:000aa060       ?getPrimaryDataType@UnDecorator@@CA?AVDName@@ABV2@@Z 1011c060 f   LIBCMTD:undname.obj
 0002:000aa310       ?getArgumentTypes@UnDecorator@@CA?AVDName@@XZ 1011c310 f   LIBCMTD:undname.obj
 0002:000aa470       ?getArgumentList@UnDecorator@@CA?AVDName@@XZ 1011c470 f   LIBCMTD:undname.obj
 0002:000aa5c0       ?getThrowTypes@UnDecorator@@CA?AVDName@@XZ 1011c5c0 f   LIBCMTD:undname.obj
 0002:000aa670       ?getBasicDataType@UnDecorator@@CA?AVDName@@ABV2@@Z 1011c670 f   LIBCMTD:undname.obj
 0002:000aac20       ?getECSUDataType@UnDecorator@@CA?AVDName@@XZ 1011cc20 f   LIBCMTD:undname.obj
 0002:000aadf0       ?getECSUName@UnDecorator@@CA?AVDName@@XZ 1011cdf0 f i LIBCMTD:undname.obj
 0002:000aae10       ?getEnumType@UnDecorator@@CA?AVDName@@XZ 1011ce10 f i LIBCMTD:undname.obj
 0002:000aaf60       ?getFunctionIndirectType@UnDecorator@@CA?AVDName@@ABV2@@Z 1011cf60 f   LIBCMTD:undname.obj
 0002:000ab3a0       ?getPtrRefType@UnDecorator@@CA?AVDName@@ABV2@0D@Z 1011d3a0 f   LIBCMTD:undname.obj
 0002:000ab500       ?getExtendedDataIndirectType@UnDecorator@@CA?AVDName@@AADAA_NH@Z 1011d500 f   LIBCMTD:undname.obj
 0002:000ab710       ?getDataIndirectType@UnDecorator@@CA?AVDName@@ABV2@D0H@Z 1011d710 f   LIBCMTD:undname.obj
 0002:000abe10       ?getPtrRefDataType@UnDecorator@@CA?AVDName@@ABV2@H@Z 1011de10 f i LIBCMTD:undname.obj
 0002:000abf50       ?getArrayType@UnDecorator@@CA?AVDName@@ABV2@@Z 1011df50 f i LIBCMTD:undname.obj
 0002:000ac180       ?getLexicalFrame@UnDecorator@@CA?AVDName@@XZ 1011e180 f i LIBCMTD:undname.obj
 0002:000ac1c0       ?getThisType@UnDecorator@@CA?AVDName@@XZ 1011e1c0 f i LIBCMTD:undname.obj
 0002:000ac200       ?getPointerType@UnDecorator@@CA?AVDName@@ABV2@0@Z 1011e200 f i LIBCMTD:undname.obj
 0002:000ac220       ?getPointerTypeArray@UnDecorator@@CA?AVDName@@ABV2@0@Z 1011e220 f i LIBCMTD:undname.obj
 0002:000ac240       ?getReferenceType@UnDecorator@@CA?AVDName@@ABV2@0@Z 1011e240 f i LIBCMTD:undname.obj
 0002:000ac260       ?getDisplacement@UnDecorator@@CA?AVDName@@XZ 1011e260 f i LIBCMTD:undname.obj
 0002:000ac280       ?getCallIndex@UnDecorator@@CA?AVDName@@XZ 1011e280 f i LIBCMTD:undname.obj
 0002:000ac2a0       ?getGuardNumber@UnDecorator@@CA?AVDName@@XZ 1011e2a0 f i LIBCMTD:undname.obj
 0002:000ac2c0       ?getVbTableType@UnDecorator@@CA?AVDName@@ABV2@@Z 1011e2c0 f i LIBCMTD:undname.obj
 0002:000ac2e0       ?getVCallThunkType@UnDecorator@@CA?AVDName@@XZ 1011e2e0 f i LIBCMTD:undname.obj
 0002:000ac340       ?getVfTableType@UnDecorator@@CA?AVDName@@ABV2@@Z 1011e340 f i LIBCMTD:undname.obj
 0002:000ac500       ?getStorageConvention@UnDecorator@@CA?AVDName@@XZ 1011e500 f i LIBCMTD:undname.obj
 0002:000ac520       ?getDataIndirectType@UnDecorator@@CA?AVDName@@XZ 1011e520 f i LIBCMTD:undname.obj
 0002:000ac560       ?getVdispMapType@UnDecorator@@CA?AVDName@@ABV2@@Z 1011e560 f i LIBCMTD:undname.obj
 0002:000ac5d0       ?getExternalDataType@UnDecorator@@CA?AVDName@@ABV2@@Z 1011e5d0 f i LIBCMTD:undname.obj
 0002:000ac660       ?doMSKeywords@UnDecorator@@SAHXZ 1011e660 f i LIBCMTD:undname.obj
 0002:000ac680       ?doPtr64@UnDecorator@@SAHXZ 1011e680 f i LIBCMTD:undname.obj
 0002:000ac6a0       ?doFunctionReturns@UnDecorator@@SAHXZ 1011e6a0 f i LIBCMTD:undname.obj
 0002:000ac6c0       ?doAllocationModel@UnDecorator@@SAHXZ 1011e6c0 f i LIBCMTD:undname.obj
 0002:000ac6e0       ?doAllocationLanguage@UnDecorator@@SAHXZ 1011e6e0 f i LIBCMTD:undname.obj
 0002:000ac700       ?doThisTypes@UnDecorator@@SAHXZ 1011e700 f i LIBCMTD:undname.obj
 0002:000ac720       ?doAccessSpecifiers@UnDecorator@@SAHXZ 1011e720 f i LIBCMTD:undname.obj
 0002:000ac740       ?doThrowTypes@UnDecorator@@SAHXZ 1011e740 f i LIBCMTD:undname.obj
 0002:000ac760       ?doMemberTypes@UnDecorator@@SAHXZ 1011e760 f i LIBCMTD:undname.obj
 0002:000ac780       ?doNameOnly@UnDecorator@@SAHXZ 1011e780 f i LIBCMTD:undname.obj
 0002:000ac7a0       ?doTypeOnly@UnDecorator@@SAHXZ 1011e7a0 f i LIBCMTD:undname.obj
 0002:000ac7c0       ?haveTemplateParameters@UnDecorator@@SAHXZ 1011e7c0 f i LIBCMTD:undname.obj
 0002:000ac7e0       ?doEcsu@UnDecorator@@SAHXZ 1011e7e0 f i LIBCMTD:undname.obj
 0002:000ac800       ?doEllipsis@UnDecorator@@SAHXZ 1011e800 f i LIBCMTD:undname.obj
 0002:000ac820       ?UScore@UnDecorator@@SAPBDW4Tokens@@@Z 1011e820 f   LIBCMTD:undname.obj
 0002:000ac850       ?doUnderScore@UnDecorator@@SAHXZ 1011e850 f i LIBCMTD:undname.obj
 0002:000ac870       ??2@YAPAXIAAVHeapManager@@H@Z 1011e870 f i LIBCMTD:undname.obj
 0002:000ac890       ?getMemory@HeapManager@@QAEPAXIH@Z 1011e890 f   LIBCMTD:undname.obj
 0002:000ac9a0       ??0Block@HeapManager@@QAE@XZ 1011e9a0 f i LIBCMTD:undname.obj
 0002:000ac9c0       ??H@YA?AVDName@@DABV0@@Z   1011e9c0 f i LIBCMTD:undname.obj
 0002:000ac9f0       ??H@YA?AVDName@@W4DNameStatus@@ABV0@@Z 1011e9f0 f i LIBCMTD:undname.obj
 0002:000aca20       ??H@YA?AVDName@@PBDABV0@@Z 1011ea20 f i LIBCMTD:undname.obj
 0002:000aca50       ??0DName@@QAE@XZ           1011ea50 f i LIBCMTD:undname.obj
 0002:000acb10       ??0DName@@QAE@D@Z          1011eb10 f   LIBCMTD:undname.obj
 0002:000acbf0       ??0DName@@QAE@ABV0@@Z      1011ebf0 f i LIBCMTD:undname.obj
 0002:000acc20       ??0DName@@QAE@PAV0@@Z      1011ec20 f   LIBCMTD:undname.obj
 0002:000acd50       ??0DName@@QAE@PBD@Z        1011ed50 f   LIBCMTD:undname.obj
 0002:000ace30       ??0DName@@QAE@AAPBDD@Z     1011ee30 f   LIBCMTD:undname.obj
 0002:000ad0f0       ?doNoIdentCharCheck@UnDecorator@@SAHXZ 1011f0f0 f i LIBCMTD:undname.obj
 0002:000ad110       ??0DName@@QAE@_K@Z         1011f110 f   LIBCMTD:undname.obj
 0002:000ad250       ??0DName@@QAE@_J@Z         1011f250 f   LIBCMTD:undname.obj
 0002:000ad3d0       ??0DName@@QAE@W4DNameStatus@@@Z 1011f3d0 f   LIBCMTD:undname.obj
 0002:000ad4f0       ?isValid@DName@@QBEHXZ     1011f4f0 f i LIBCMTD:undname.obj
 0002:000ad520       ?isEmpty@DName@@QBEHXZ     1011f520 f i LIBCMTD:undname.obj
 0002:000ad540       ?status@DName@@QBE?AW4DNameStatus@@XZ 1011f540 f i LIBCMTD:undname.obj
 0002:000ad560       ?setPtrRef@DName@@QAEAAV1@XZ 1011f560 f i LIBCMTD:undname.obj
 0002:000ad590       ?isPtrRef@DName@@QBEHXZ    1011f590 f i LIBCMTD:undname.obj
 0002:000ad5b0       ?isUDC@DName@@QBEHXZ       1011f5b0 f i LIBCMTD:undname.obj
 0002:000ad5f0       ?setIsUDC@DName@@QAEXXZ    1011f5f0 f i LIBCMTD:undname.obj
 0002:000ad620       ?isUDTThunk@DName@@QBEHXZ  1011f620 f i LIBCMTD:undname.obj
 0002:000ad660       ?setIsArray@DName@@QAEXXZ  1011f660 f i LIBCMTD:undname.obj
 0002:000ad680       ?isArray@DName@@QBEHXZ     1011f680 f i LIBCMTD:undname.obj
 0002:000ad6a0       ?isNoTE@DName@@QBEHXZ      1011f6a0 f i LIBCMTD:undname.obj
 0002:000ad6c0       ?setIsNoTE@DName@@QAEXXZ   1011f6c0 f i LIBCMTD:undname.obj
 0002:000ad6e0       ?isPinPtr@DName@@QBEHXZ    1011f6e0 f i LIBCMTD:undname.obj
 0002:000ad700       ?setIsPinPtr@DName@@QAEXXZ 1011f700 f i LIBCMTD:undname.obj
 0002:000ad720       ?isComArray@DName@@QBEHXZ  1011f720 f i LIBCMTD:undname.obj
 0002:000ad740       ?setIsComArray@DName@@QAEXXZ 1011f740 f i LIBCMTD:undname.obj
 0002:000ad760       ?isVCallThunk@DName@@QBEHXZ 1011f760 f i LIBCMTD:undname.obj
 0002:000ad780       ?setIsVCallThunk@DName@@QAEXXZ 1011f780 f i LIBCMTD:undname.obj
 0002:000ad7a0       ?length@DName@@QBEHXZ      1011f7a0 f i LIBCMTD:undname.obj
 0002:000ad7d0       ?getLastChar@DName@@QBEDXZ 1011f7d0 f i LIBCMTD:undname.obj
 0002:000ad800       ?getString@DName@@QBEPADPADH@Z 1011f800 f i LIBCMTD:undname.obj
 0002:000ad890       ?getString@DName@@QBEPADPAD0@Z 1011f890 f i LIBCMTD:undname.obj
 0002:000ad8d0       ??HDName@@QBE?AV0@D@Z      1011f8d0 f   LIBCMTD:undname.obj
 0002:000ad910       ??HDName@@QBE?AV0@PBD@Z    1011f910 f   LIBCMTD:undname.obj
 0002:000ad950       ??HDName@@QBE?AV0@ABV0@@Z  1011f950 f   LIBCMTD:undname.obj
 0002:000ad990       ??HDName@@QBE?AV0@PAV0@@Z  1011f990 f   LIBCMTD:undname.obj
 0002:000ad9d0       ??HDName@@QBE?AV0@W4DNameStatus@@@Z 1011f9d0 f   LIBCMTD:undname.obj
 0002:000ada10       ?append@DName@@AAEXPAVDNameNode@@@Z 1011fa10 f   LIBCMTD:undname.obj
 0002:000adaa0       ??YDName@@QAEAAV0@D@Z      1011faa0 f   LIBCMTD:undname.obj
 0002:000adb30       ??YDName@@QAEAAV0@PBD@Z    1011fb30 f   LIBCMTD:undname.obj
 0002:000adbd0       ??YDName@@QAEAAV0@ABV0@@Z  1011fbd0 f   LIBCMTD:undname.obj
 0002:000adc40       ??YDName@@QAEAAV0@PAV0@@Z  1011fc40 f   LIBCMTD:undname.obj
 0002:000add00       ??YDName@@QAEAAV0@W4DNameStatus@@@Z 1011fd00 f   LIBCMTD:undname.obj
 0002:000add70       ??_5DName@@QAEAAV0@ABV0@@Z 1011fd70 f   LIBCMTD:undname.obj
 0002:000addd0       ??4DName@@QAEAAV0@D@Z      1011fdd0 f i LIBCMTD:undname.obj
 0002:000adeb0       ??4DName@@QAEAAV0@PBD@Z    1011feb0 f   LIBCMTD:undname.obj
 0002:000adf90       ??4DName@@QAEAAV0@ABV0@@Z  1011ff90 f   LIBCMTD:undname.obj
 0002:000adfc0       ??4DName@@QAEAAV0@PAV0@@Z  1011ffc0 f   LIBCMTD:undname.obj
 0002:000ae100       ??4DName@@QAEAAV0@W4DNameStatus@@@Z 10120100 f   LIBCMTD:undname.obj
 0002:000ae200       ?doPchar@DName@@AAEXPBDH@Z 10120200 f   LIBCMTD:undname.obj
 0002:000ae340       ?isFull@Replicator@@QBEHXZ 10120340 f i LIBCMTD:undname.obj
 0002:000ae360       ??0Replicator@@QAE@XZ      10120360 f i LIBCMTD:undname.obj
 0002:000ae380       ??YReplicator@@QAEAAV0@ABVDName@@@Z 10120380 f   LIBCMTD:undname.obj
 0002:000ae410       ??AReplicator@@QBE?AVDName@@H@Z 10120410 f   LIBCMTD:undname.obj
 0002:000ae480       ??0DNameNode@@IAE@XZ       10120480 f   LIBCMTD:undname.obj
 0002:000ae4a0       ??0charNode@@QAE@D@Z       101204a0 f   LIBCMTD:undname.obj
 0002:000ae4d0       ?length@charNode@@UBEHXZ   101204d0 f i LIBCMTD:undname.obj
 0002:000ae4f0       ?getLastChar@charNode@@UBEDXZ 101204f0 f i LIBCMTD:undname.obj
 0002:000ae510       ?getString@charNode@@UBEPADPAD0@Z 10120510 f i LIBCMTD:undname.obj
 0002:000ae540       ??0pcharNode@@QAE@PBDH@Z   10120540 f   LIBCMTD:undname.obj
 0002:000ae5d0       ?length@pcharNode@@UBEHXZ  101205d0 f i LIBCMTD:undname.obj
 0002:000ae5f0       ?getLastChar@pcharNode@@UBEDXZ 101205f0 f i LIBCMTD:undname.obj
 0002:000ae630       ?getString@pcharNode@@UBEPADPAD0@Z 10120630 f i LIBCMTD:undname.obj
 0002:000ae660       ?getStringHelper@@YAPADPAD00H@Z 10120660 f i LIBCMTD:undname.obj
 0002:000ae6a0       ??0pDNameNode@@QAE@PAVDName@@@Z 101206a0 f   LIBCMTD:undname.obj
 0002:000ae700       ?length@pDNameNode@@UBEHXZ 10120700 f i LIBCMTD:undname.obj
 0002:000ae740       ?getLastChar@pDNameNode@@UBEDXZ 10120740 f i LIBCMTD:undname.obj
 0002:000ae770       ?getString@pDNameNode@@UBEPADPAD0@Z 10120770 f i LIBCMTD:undname.obj
 0002:000ae7b0       ??0DNameStatusNode@@AAE@W4DNameStatus@@@Z 101207b0 f   LIBCMTD:undname.obj
 0002:000ae800       ?length@DNameStatusNode@@UBEHXZ 10120800 f i LIBCMTD:undname.obj
 0002:000ae820       ?getLastChar@DNameStatusNode@@UBEDXZ 10120820 f i LIBCMTD:undname.obj
 0002:000ae840       ?getString@DNameStatusNode@@UBEPADPAD0@Z 10120840 f i LIBCMTD:undname.obj
 0002:000ae880       ?make@DNameStatusNode@@SAPAV1@W4DNameStatus@@@Z 10120880 f i LIBCMTD:undname.obj
 0002:000ae930       ??0pairNode@@QAE@PAVDNameNode@@0@Z 10120930 f   LIBCMTD:undname.obj
 0002:000ae970       ?length@pairNode@@UBEHXZ   10120970 f i LIBCMTD:undname.obj
 0002:000ae9c0       ?getLastChar@pairNode@@UBEDXZ 101209c0 f i LIBCMTD:undname.obj
 0002:000aea10       ?getString@pairNode@@UBEPADPAD0@Z 10120a10 f i LIBCMTD:undname.obj
 0002:000aeb50       __lseeki64                 10120b50 f   LIBCMTD:lseeki64.obj
 0002:000aeda0       __lseeki64_nolock          10120da0 f   LIBCMTD:lseeki64.obj
 0002:000aee90       __getbuf                   10120e90 f   LIBCMTD:_getbuf.obj
 0002:000aef50       __isatty                   10120f50 f   LIBCMTD:isatty.obj
 0002:000af030       __wctomb_s_l               10121030 f   LIBCMTD:wctomb.obj
 0002:000af330       _wctomb_s                  10121330 f   LIBCMTD:wctomb.obj
 0002:000af360       __wctomb_l                 10121360 f   LIBCMTD:wctomb.obj
 0002:000af3e0       _wctomb                    101213e0 f   LIBCMTD:wctomb.obj
 0002:000af430       __aulldiv                  10121430 f   LIBCMTD:ulldiv.obj
 0002:000af4a0       __aullrem                  101214a0 f   LIBCMTD:ullrem.obj
 0002:000af520       __output_s_l               10121520 f   LIBCMTD:outputs.obj
 0002:000b0ab0       __ld12tod                  10122ab0 f   LIBCMTD:_intrncvt_.obj
 0002:000b0ad0       __ld12cvt                  10122ad0 f i LIBCMTD:_intrncvt_.obj
 0002:000b0d20       __RoundMan                 10122d20 f i LIBCMTD:_intrncvt_.obj
 0002:000b0e00       __ZeroTail                 10122e00 f i LIBCMTD:_intrncvt_.obj
 0002:000b0e90       __IncMan                   10122e90 f i LIBCMTD:_intrncvt_.obj
 0002:000b0f40       __CopyMan                  10122f40 f i LIBCMTD:_intrncvt_.obj
 0002:000b0f90       __FillZeroMan              10122f90 f i LIBCMTD:_intrncvt_.obj
 0002:000b0fd0       __IsZeroMan                10122fd0 f i LIBCMTD:_intrncvt_.obj
 0002:000b1010       __ShrMan                   10123010 f i LIBCMTD:_intrncvt_.obj
 0002:000b1100       __ld12tof                  10123100 f   LIBCMTD:_intrncvt_.obj
 0002:000b1120       __ld12told                 10123120 f   LIBCMTD:_intrncvt_.obj
 0002:000b11d0       ___mtold12                 101231d0 f   LIBCMTD:_mantold_.obj
 0002:000b1330       ___add_12                  10123330 f i LIBCMTD:_mantold_.obj
 0002:000b13e0       __mbsnbcpy_s_l             101233e0 f   LIBCMTD:mbsnbcpy_s_l.obj
 0002:000b1a60       __mbsdec_l                 10123a60 f   LIBCMTD:mbsdec.obj
 0002:000b1bd0       __mbsdec                   10123bd0 f   LIBCMTD:mbsdec.obj
 0002:000b1bf0       __open                     10123bf0 f   LIBCMTD:open.obj
 0002:000b1d70       __sopen_helper             10123d70 f   LIBCMTD:open.obj
 0002:000b2fd0       __sopen                    10124fd0 f   LIBCMTD:open.obj
 0002:000b3050       __sopen_s                  10125050 f   LIBCMTD:open.obj
 0002:000b3080       __mbsnbicmp_l              10125080 f   LIBCMTD:mbsnbicm.obj
 0002:000b3520       __mbsnbicmp                10125520 f   LIBCMTD:mbsnbicm.obj
 0002:000b3540       __mbsnbcmp_l               10125540 f   LIBCMTD:mbsnbcmp.obj
 0002:000b3820       __mbsnbcmp                 10125820 f   LIBCMTD:mbsnbcmp.obj
 0002:000b3840       __matherr                  10125840 f   LIBCMTD:_matherr_.obj
 0002:000b3850       __putwch                   10125850 f   LIBCMTD:putwch.obj
 0002:000b38e0       __putwch_nolock            101258e0 f   LIBCMTD:putwch.obj
 0002:000b39e0       __cputws                   101259e0 f   LIBCMTD:putwch.obj
 0002:000b3b30       __mbtowc_l                 10125b30 f   LIBCMTD:mbtowc.obj
 0002:000b3d50       _mbtowc                    10125d50 f   LIBCMTD:mbtowc.obj
 0002:000b3d70       ___crtMessageBoxA          10125d70 f   LIBCMTD:crtmbox.obj
 0002:000b3f90       __set_error_mode           10125f90 f   LIBCMTD:errmode.obj
 0002:000b4050       ___set_app_type            10126050 f   LIBCMTD:errmode.obj
 0002:000b4060       ___get_app_type            10126060 f   LIBCMTD:errmode.obj
 0002:000b4070       ___ansicp                  10126070 f   LIBCMTD:convrtcp.obj
 0002:000b40d0       ___convertcp               101260d0 f   LIBCMTD:convrtcp.obj
 0002:000b4320       __iswctype_l               10126320 f   LIBCMTD:iswctype.obj
 0002:000b43d0       _iswctype                  101263d0 f   LIBCMTD:iswctype.obj
 0002:000b4460       _is_wctype                 10126460 f   LIBCMTD:iswctype.obj
 0002:000b4480       ___crtGetLocaleInfoW       10126480 f   LIBCMTD:w_loc.obj
 0002:000b44f0       ___crtGetLocaleInfoA       101264f0 f   LIBCMTD:a_loc.obj
 0002:000b46d0       __get_daylight             101266d0 f   LIBCMTD:timeset.obj
 0002:000b4750       __get_dstbias              10126750 f   LIBCMTD:timeset.obj
 0002:000b47d0       __get_timezone             101267d0 f   LIBCMTD:timeset.obj
 0002:000b4850       __get_tzname               10126850 f   LIBCMTD:timeset.obj
 0002:000b4a20       ___daylight                10126a20 f   LIBCMTD:timeset.obj
 0002:000b4a30       ___dstbias                 10126a30 f   LIBCMTD:timeset.obj
 0002:000b4a40       ___timezone                10126a40 f   LIBCMTD:timeset.obj
 0002:000b4a50       ___tzname                  10126a50 f   LIBCMTD:timeset.obj
 0002:000b4a60       ___tzset                   10126a60 f   LIBCMTD:tzset.obj
 0002:000b4b00       __tzset                    10126b00 f   LIBCMTD:tzset.obj
 0002:000b50b0       __set_daylight             101270b0 f i LIBCMTD:tzset.obj
 0002:000b50d0       __set_dstbias              101270d0 f i LIBCMTD:tzset.obj
 0002:000b50f0       __set_timezone             101270f0 f i LIBCMTD:tzset.obj
 0002:000b5110       __isindst                  10127110 f   LIBCMTD:tzset.obj
 0002:000b57c0       __strnicmp_l               101277c0 f   LIBCMTD:strnicmp.obj
 0002:000b5a00       __strnicmp                 10127a00 f   LIBCMTD:strnicmp.obj
 0002:000b5b90       __statusfp2                10127b90 f   LIBCMTD:_ieee87_.obj
 0002:000b5bd0       __statusfp                 10127bd0 f   LIBCMTD:_ieee87_.obj
 0002:000b5c20       __clearfp                  10127c20 f   LIBCMTD:_ieee87_.obj
 0002:000b5c70       ___control87_2             10127c70 f   LIBCMTD:_ieee87_.obj
 0002:000b5d20       __controlfp                10127d20 f   LIBCMTD:_ieee87_.obj
 0002:000b5d40       __control87                10127d40 f i LIBCMTD:_ieee87_.obj
 0002:000b5df0       __set_controlfp            10127df0 f   LIBCMTD:_ieee87_.obj
 0002:000b5e80       __fpreset                  10127e80 f   LIBCMTD:_ieee87_.obj
 0002:000b6640       _$I10_OUTPUT               10128640 f   LIBCMTD:_x10fout_.obj
 0002:000b6bf0       __woutput_s_l              10128bf0 f   LIBCMTD:woutputs.obj
 0002:000b7f20       __validate_param_reuseW    10129f20 f   LIBCMTD:woutputp.obj
 0002:000b8190       __woutput_p_l              1012a190 f   LIBCMTD:woutputp.obj
 0002:000bb8f0       _fputwc                    1012d8f0 f   LIBCMTD:fputwc.obj
 0002:000bb9f0       __fputwc_nolock            1012d9f0 f   LIBCMTD:fputwc.obj
 0002:000bbce0       _putwc                     1012dce0 f   LIBCMTD:fputwc.obj
 0002:000bbd00       __purecall                 1012dd00 f   LIBCMTD:purevirt.obj
 0002:000bbd40       __set_purecall_handler     1012dd40 f   LIBCMTD:purevirt.obj
 0002:000bbd80       __get_purecall_handler     1012dd80 f   LIBCMTD:purevirt.obj
 0002:000bbda0       __chsize_s                 1012dda0 f   LIBCMTD:chsize.obj
 0002:000bc040       __chsize_nolock            1012e040 f   LIBCMTD:chsize.obj
 0002:000bc2e0       __chsize                   1012e2e0 f   LIBCMTD:chsize.obj
 0002:000bc310       __setmode                  1012e310 f   LIBCMTD:setmode.obj
 0002:000bc5a0       __setmode_nolock           1012e5a0 f   LIBCMTD:setmode.obj
 0002:000bc810       __set_fmode                1012e810 f   LIBCMTD:setmode.obj
 0002:000bc8c0       __get_fmode                1012e8c0 f   LIBCMTD:setmode.obj
 0002:000bc940       ___initconin               1012e940 f   LIBCMTD:initcon.obj
 0002:000bc970       ___initconout              1012e970 f   LIBCMTD:initcon.obj
 0002:000bc9a0       ___termcon                 1012e9a0 f   LIBCMTD:initcon.obj
 0002:000bc9f0       ___crtGetStringTypeW       1012e9f0 f   LIBCMTD:w_str.obj
 0002:000bca70       _getenv                    1012ea70 f   LIBCMTD:getenv.obj
 0002:000bcbc0       __getenv_helper_nolock     1012ebc0 f   LIBCMTD:getenv.obj
 0002:000bcce0       _getenv_s                  1012ece0 f   LIBCMTD:getenv.obj
 0002:000bcf10       __dupenv_s                 1012ef10 f   LIBCMTD:getenv.obj
 0002:000bcf40       __dupenv_s_dbg             1012ef40 f   LIBCMTD:getenv.obj
 0002:000bd190       ___ascii_strnicmp          1012f190 f   LIBCMTD:_strnicm.obj
 0002:000bd200       _wcstol                    1012f200 f   LIBCMTD:wcstol.obj
 0002:000bd680       __wcstol_l                 1012f680 f   LIBCMTD:wcstol.obj
 0002:000bd6b0       _wcstoul                   1012f6b0 f   LIBCMTD:wcstol.obj
 0002:000bd700       __wcstoul_l                1012f700 f   LIBCMTD:wcstol.obj
 0002:000bd730       __flswbuf                  1012f730 f   LIBCMTD:_flswbuf.obj
 0002:000bda10       _strnlen                   1012fa10 f   LIBCMTD:strlen_s.obj
 0002:000bda50       __mbsnbicoll_l             1012fa50 f   LIBCMTD:mbsnbico.obj
 0002:000bdc90       __mbsnbicoll               1012fc90 f   LIBCMTD:mbsnbico.obj
 0002:000bdcb0       ___wtomb_environ           1012fcb0 f   LIBCMTD:wtombenv.obj
 0002:000bdda0       __wchartodigit             1012fda0 f   LIBCMTD:wchtodig.obj
 0002:000be0d0       ___crtCompareStringA       101300d0 f   LIBCMTD:a_cmp.obj
 0002:000be690       __strnicoll_l              10130690 f   LIBCMTD:strnicol.obj
 0002:000be8e0       __strnicoll                101308e0 f   LIBCMTD:strnicol.obj
 0002:000be920       ___crtsetenv               10130920 f   LIBCMTD:setenv.obj
 0002:000befa0       __mbschr_l                 10130fa0 f   LIBCMTD:mbschr.obj
 0002:000bf130       __mbschr                   10131130 f   LIBCMTD:mbschr.obj
 0002:000c9f55       _aliases_lookup            1013bf55 f   iconv:iconv.obj
 0002:000ca094       _aliases2_lookup           1013c094 f   iconv:iconv.obj
 0002:000ca0c4       _libiconv_open             1013c0c4 f   iconv:iconv.obj
 0002:000cad34       _libiconv                  1013cd34 f   iconv:iconv.obj
 0002:000cad6a       _libiconv_close            1013cd6a f   iconv:iconv.obj
 0002:000cad77       _libiconvctl               1013cd77 f   iconv:iconv.obj
 0002:000cae5a       _libiconvlist              1013ce5a f   iconv:iconv.obj
 0002:000cafba       _locale_charset            1013cfba f   iconv:localcharset.obj
 0002:000cb050       ??1CAutoFree@@QAE@XZ       1013d050 f   wzFilePacker_static_d:wzFilePacker.obj
 0002:000cb0a0       ??0CPackFile@@QAE@XZ       1013d0a0 f   wzFilePacker_static_d:wzFilePacker.obj
 0002:000cb120       ??1CPackFile@@QAE@XZ       1013d120 f   wzFilePacker_static_d:wzFilePacker.obj
 0002:000cb170       ?Open@CPackFile@@QAEPAXPBD0K@Z 1013d170 f   wzFilePacker_static_d:wzFilePacker.obj
 0002:000cb320       ?CONVERT_PATHCHAR@CPackFile@@CAXPAD@Z 1013d320 f i wzFilePacker_static_d:wzFilePacker.obj
 0002:000cb3d0       ?_tcsstr@@YAPADPADPBD@Z    1013d3d0 f i wzFilePacker_static_d:wzFilePacker.obj
 0002:000cb430       __tcsstr                   1013d430 f i wzFilePacker_static_d:wzFilePacker.obj
 0002:000cb490       ?Close@CPackFile@@QAEXXZ   1013d490 f   wzFilePacker_static_d:wzFilePacker.obj
 0002:000cb510       ?CreateFinder@CPackFile@@AAEPAXPAXPBD@Z 1013d510 f   wzFilePacker_static_d:wzFilePacker.obj
 0002:000cb570       ?DestroyFinder@CPackFile@@AAEXPAX@Z 1013d570 f   wzFilePacker_static_d:wzFilePacker.obj
 0002:000cb5d0       ?FinderGetNextFile@CPackFile@@AAEHPAX@Z 1013d5d0 f   wzFilePacker_static_d:wzFilePacker.obj
 0002:000cb630       ?FinderGetProperties@CPackFile@@AAEHPAXPAUFileProperties@@@Z 1013d630 f   wzFilePacker_static_d:wzFilePacker.obj
 0002:000cb790       ?FindFile@CPackFile@@QAEHPAXPBDAAV?$vector@V?$basic_string@DU?$char_traits@D@std@@V?$allocator@D@2@@std@@V?$allocator@V?$basic_string@DU?$char_traits@D@std@@V?$allocator@D@2@@std@@@2@@std@@2H@Z 1013d790 f   wzFilePacker_static_d:wzFilePacker.obj
 0002:000cbb70       ?CreateFileA@CPackFile@@QAEPAXPBD_K@Z 1013db70 f   wzFilePacker_static_d:wzFilePacker.obj
 0002:000cbbf0       ?OpenFile@CPackFile@@QAEPAXPBDK@Z 1013dbf0 f   wzFilePacker_static_d:wzFilePacker.obj
 0002:000cbc60       ?DeleteFileA@CPackFile@@QAEHPBD@Z 1013dc60 f   wzFilePacker_static_d:wzFilePacker.obj
 0002:000cbcd0       ?FileExists@CPackFile@@QAEHPBD@Z 1013dcd0 f   wzFilePacker_static_d:wzFilePacker.obj
 0002:000cbd40       ?RenameFile@CPackFile@@QAEHPBD0@Z 1013dd40 f   wzFilePacker_static_d:wzFilePacker.obj
 0002:000cbdd0       ?RemoveDirectoryA@CPackFile@@QAEHPBD@Z 1013ddd0 f   wzFilePacker_static_d:wzFilePacker.obj
 0002:000cbe40       ?CreateDirectoryA@CPackFile@@QAEHPBD@Z 1013de40 f   wzFilePacker_static_d:wzFilePacker.obj
 0002:000cbec0       ?CloseFile@CPackFile@@QAEXPAX@Z 1013dec0 f   wzFilePacker_static_d:wzFilePacker.obj
 0002:000cbf20       ?GetFileProperties@CPackFile@@QAEHPAXPAUFileProperties@@@Z 1013df20 f   wzFilePacker_static_d:wzFilePacker.obj
 0002:000cc080       ?ReadFile@CPackFile@@QAEHPAX0K@Z 1013e080 f   wzFilePacker_static_d:wzFilePacker.obj
 0002:000cc0e0       ?WriteFile@CPackFile@@QAEHPAXPBXK@Z 1013e0e0 f   wzFilePacker_static_d:wzFilePacker.obj
 0002:000cc140       ?GetFileSize@CPackFile@@QAEHPAXPA_K@Z 1013e140 f   wzFilePacker_static_d:wzFilePacker.obj
 0002:000cc1a0       ?GetFilePointer@CPackFile@@QAEHPAXPA_K@Z 1013e1a0 f   wzFilePacker_static_d:wzFilePacker.obj
 0002:000cc200       ?SetFilePointer@CPackFile@@QAEHPAX_KK@Z 1013e200 f   wzFilePacker_static_d:wzFilePacker.obj
 0002:000cc260       ?IsEOF@CPackFile@@QAEHPAX@Z 1013e260 f   wzFilePacker_static_d:wzFilePacker.obj
 0002:000cc2c0       ?AddFile@CPackFile@@QAEHPBD0@Z 1013e2c0 f   wzFilePacker_static_d:wzFilePacker.obj
 0002:000cc540       ?SetHwnd@CPackFile@@QAEXPAUHWND__@@@Z 1013e540 f   wzFilePacker_static_d:wzFilePacker.obj
 0002:000cc590       ?GetFindFileNameInPackFile@CPackFile@@SAHPBDPAD@Z 1013e590 f   wzFilePacker_static_d:wzFilePacker.obj
 0002:000cc830       ?ExtractFile@CPackFile@@QAEHPAXPBD1@Z 1013e830 f   wzFilePacker_static_d:wzFilePacker.obj
 0002:000cca20       ?ExtractAll@CPackFile@@QAEHPAXPBD@Z 1013ea20 f   wzFilePacker_static_d:wzFilePacker.obj
 0002:000cd260       ?EncryptHdr@CPackFile@@SAHPAD@Z 1013f260 f   wzFilePacker_static_d:wzFilePacker.obj
 0002:000cd500       ?WriteHeader@CPackFile@@QAEXPADHH@Z 1013f500 f   wzFilePacker_static_d:wzFilePacker.obj
 0002:000cd860       ?MurgeFile@CPackFile@@QAEHPAXH@Z 1013f860 f   wzFilePacker_static_d:wzFilePacker.obj
 0002:000ce360       ?length@?$basic_string@DU?$char_traits@D@std@@V?$allocator@D@2@@std@@QBEIXZ 10140360 f i wzFilePacker_static_d:wzFilePacker.obj
 0002:000ce3a0       ?find_last_of@?$basic_string@DU?$char_traits@D@std@@V?$allocator@D@2@@std@@QBEIPBDI@Z 101403a0 f i wzFilePacker_static_d:wzFilePacker.obj
 0002:000ce430       ??D?$_Vector_iterator@V?$basic_string@DU?$char_traits@D@std@@V?$allocator@D@2@@std@@V?$allocator@V?$basic_string@DU?$char_traits@D@std@@V?$allocator@D@2@@std@@@2@@std@@QBEAAV?$basic_string@DU?$char_traits@D@std@@V?$allocator@D@2@@1@XZ 10140430 f i wzFilePacker_static_d:wzFilePacker.obj
 0002:000ce480       ??E?$_Vector_iterator@V?$basic_string@DU?$char_traits@D@std@@V?$allocator@D@2@@std@@V?$allocator@V?$basic_string@DU?$char_traits@D@std@@V?$allocator@D@2@@std@@@2@@std@@QAE?AV01@H@Z 10140480 f i wzFilePacker_static_d:wzFilePacker.obj
 0002:000ce5a0       ?find_last_of@?$basic_string@DU?$char_traits@D@std@@V?$allocator@D@2@@std@@QBEIPBDII@Z 101405a0 f i wzFilePacker_static_d:wzFilePacker.obj
 0002:000ce6d0       ??E?$_Vector_iterator@V?$basic_string@DU?$char_traits@D@std@@V?$allocator@D@2@@std@@V?$allocator@V?$basic_string@DU?$char_traits@D@std@@V?$allocator@D@2@@std@@@2@@std@@QAEAAV01@XZ 101406d0 f i wzFilePacker_static_d:wzFilePacker.obj
 0002:000ce730       ??0CAutoFree@@QAE@XZ       10140730 f i wzFilePacker_static_d:wzFilePacker.obj
 0002:000ce770       @geVFile_CloseAPI@0        10140770 f   wzFilePacker_static_d:vfile.obj
 0002:000ce7e0       @geVFile_RegisterFileSystem@8 101407e0 f   wzFilePacker_static_d:vfile.obj
 0002:000cea90       @geVFile_OpenNewSystem@20  10140a90 f   wzFilePacker_static_d:vfile.obj
 0002:000cee20       @geVFile_UpdateSystem@4    10140e20 f   wzFilePacker_static_d:vfile.obj
 0002:000cf210       @geVFile_UpdateContext@12  10141210 f   wzFilePacker_static_d:vfile.obj
 0002:000cf2e0       @geVFile_Open_Detail@20    101412e0 f   wzFilePacker_static_d:vfile.obj
 0002:000cf5e0       @geVFile_Open@12           101415e0 f   wzFilePacker_static_d:vfile.obj
 0002:000cf8e0       @geVFile_GetContext@4      101418e0 f   wzFilePacker_static_d:vfile.obj
 0002:000cf960       @geVFile_AddPath@12        10141960 f   wzFilePacker_static_d:vfile.obj
 0002:000cfc60       @geVFile_DeleteFile@8      10141c60 f   wzFilePacker_static_d:vfile.obj
 0002:000cfd40       @geVFile_RenameFile@12     10141d40 f   wzFilePacker_static_d:vfile.obj
 0002:000cfe40       @geVFile_FileExists@8      10141e40 f   wzFilePacker_static_d:vfile.obj
 0002:000cfec0       @geVFile_Close@4           10141ec0 f   wzFilePacker_static_d:vfile.obj
 0002:000cffc0       @geVFile_GetS@12           10141fc0 f   wzFilePacker_static_d:vfile.obj
 0002:000d00a0       @geVFile_Read@12           101420a0 f   wzFilePacker_static_d:vfile.obj
 0002:000d0180       @geVFile_Write@12          10142180 f   wzFilePacker_static_d:vfile.obj
 0002:000d0260       @geVFile_Seek@16           10142260 f   wzFilePacker_static_d:vfile.obj
 0002:000d0310       _geVFile_Printf            10142310 f   wzFilePacker_static_d:vfile.obj
 0002:000d0470       @geVFile_EOF@4             10142470 f   wzFilePacker_static_d:vfile.obj
 0002:000d0500       @geVFile_Tell@8            10142500 f   wzFilePacker_static_d:vfile.obj
 0002:000d05a0       @geVFile_Size@8            101425a0 f   wzFilePacker_static_d:vfile.obj
 0002:000d0640       @geVFile_GetProperties@8   10142640 f   wzFilePacker_static_d:vfile.obj
 0002:000d06e0       @geVFile_SetSize@12        101426e0 f   wzFilePacker_static_d:vfile.obj
 0002:000d0780       @geVFile_SetAttributes@8   10142780 f   wzFilePacker_static_d:vfile.obj
 0002:000d0820       @geVFile_SetTime@8         10142820 f   wzFilePacker_static_d:vfile.obj
 0002:000d08c0       @geVFile_SetHints@8        101428c0 f   wzFilePacker_static_d:vfile.obj
 0002:000d0960       @geVFile_EnlargeDirectorySize@8 10142960 f   wzFilePacker_static_d:vfile.obj
 0002:000d0a00       @geVFile_CreateFinder@8    10142a00 f   wzFilePacker_static_d:vfile.obj
 0002:000d0b40       @geVFile_DestroyFinder@4   10142b40 f   wzFilePacker_static_d:vfile.obj
 0002:000d0c20       @geVFile_FinderGetNextFile@4 10142c20 f   wzFilePacker_static_d:vfile.obj
 0002:000d0d10       @geVFile_FinderGetProperties@8 10142d10 f   wzFilePacker_static_d:vfile.obj
 0002:000d0e00       @geVFile_TimeToWin32FileTime@8 10142e00 f   wzFilePacker_static_d:vfile.obj
 0002:000d0e50       @geVFile_SetVersion@8      10142e50 f   wzFilePacker_static_d:vfile.obj
 0002:000d0ea0       @geVFile_IsPrevVersion@4   10142ea0 f   wzFilePacker_static_d:vfile.obj
 0002:000d0ee0       _EmptyDirectory            10142ee0 f   wzFilePacker_static_d:vFile_util.obj
 0002:000d11a0       _SetupDirectory            101431a0 f   wzFilePacker_static_d:vFile_util.obj
 0002:000d1200       _ExtractVFS                10143200 f   wzFilePacker_static_d:vFile_util.obj
 0002:000d1540       _ExplorerVFS               10143540 f   wzFilePacker_static_d:vFile_util.obj
 0002:000d1840       _CopyVFile                 10143840 f   wzFilePacker_static_d:vFile_util.obj
 0002:000d1b20       _CopyOneFile               10143b20 f   wzFilePacker_static_d:vFile_util.obj
 0002:000d1c30       _GetDir                    10143c30 f   wzFilePacker_static_d:vFile_util.obj
 0002:000d1fa0       _GetFiles                  10143fa0 f   wzFilePacker_static_d:vFile_util.obj
 0002:000d2480       _MakeDirectory             10144480 f   wzFilePacker_static_d:vFile_util.obj
 0002:000d2630       _geRam_EnableCriticalCallback 10144630 f   wzFilePacker_static_d:Ram.obj
 0002:000d2680       _geRam_SetCriticalCallback 10144680 f   wzFilePacker_static_d:Ram.obj
 0002:000d26d0       _geRam_AllocateClear       101446d0 f   wzFilePacker_static_d:Ram.obj
 0002:000d2770       __geRam_DebugAllocate      10144770 f   wzFilePacker_static_d:Ram.obj
 0002:000d2a00       _geRam_Free_               10144a00 f   wzFilePacker_static_d:Ram.obj
 0002:000d2cc0       __geRam_DebugRealloc       10144cc0 f   wzFilePacker_static_d:Ram.obj
 0002:000d2e90       _geRam_ReportAllocations   10144e90 f   wzFilePacker_static_d:Ram.obj
 0002:000d2ee0       _geRam_AddAllocation       10144ee0 f   wzFilePacker_static_d:Ram.obj
 0002:000d2f70       _geRam_IsValidPtr          10144f70 f   wzFilePacker_static_d:Ram.obj
 0002:000d3070       _Encrypt                   10145070 f   wzFilePacker_static_d:fsvfs.obj
 0002:000d3100       _Decrypt                   10145100 f   wzFilePacker_static_d:fsvfs.obj
 0002:000d9010       @FSVFS_GetAPIs@0           1014b010 f   wzFilePacker_static_d:fsvfs.obj
 0002:000daaa0       @FSMemory_GetAPIs@0        1014caa0 f   wzFilePacker_static_d:FSMEMORY.obj
 0002:000dd870       @FSDos_GetAPIs@0           1014f870 f   wzFilePacker_static_d:fsdos.obj
 0002:000dd8b0       _DirTree_Create            1014f8b0 f   wzFilePacker_static_d:dirtree.obj
 0002:000dd9a0       _DirTree_Destroy           1014f9a0 f   wzFilePacker_static_d:dirtree.obj
 0002:000ddac0       _DirTree_SetAllFileOffset  1014fac0 f   wzFilePacker_static_d:dirtree.obj
 0002:000ddc60       _DirTree_SetFileSize       1014fc60 f   wzFilePacker_static_d:dirtree.obj
 0002:000ddce0       _DirTree_GetFileSize       1014fce0 f   wzFilePacker_static_d:dirtree.obj
 0002:000ddd60       _DirTree_WriteToFile       1014fd60 f   wzFilePacker_static_d:dirtree.obj
 0002:000de2d0       _DirTree_GetSize           101502d0 f   wzFilePacker_static_d:dirtree.obj
 0002:000de3d0       _DirTree_CreateFromFile    101503d0 f   wzFilePacker_static_d:dirtree.obj
 0002:000df2d0       _DirTree_FindExact         101512d0 f   wzFilePacker_static_d:dirtree.obj
 0002:000df410       _DirTree_FindPartial       10151410 f   wzFilePacker_static_d:dirtree.obj
 0002:000df570       _DirTree_AddFile           10151570 f   wzFilePacker_static_d:dirtree.obj
 0002:000df800       _DirTree_Remove            10151800 f   wzFilePacker_static_d:dirtree.obj
 0002:000dfa20       _DirTree_SetFileAttributes 10151a20 f   wzFilePacker_static_d:dirtree.obj
 0002:000dfb30       _DirTree_GetFileAttributes 10151b30 f   wzFilePacker_static_d:dirtree.obj
 0002:000dfbd0       _DirTree_SetFileOffset     10151bd0 f   wzFilePacker_static_d:dirtree.obj
 0002:000dfc80       _DirTree_GetFileOffset     10151c80 f   wzFilePacker_static_d:dirtree.obj
 0002:000dfd30       _DirTree_SetFileTime       10151d30 f   wzFilePacker_static_d:dirtree.obj
 0002:000dfdb0       _DirTree_GetFileTime       10151db0 f   wzFilePacker_static_d:dirtree.obj
 0002:000dfe30       _DirTree_SetFileHints      10151e30 f   wzFilePacker_static_d:dirtree.obj
 0002:000dff30       _DirTree_GetFileHints      10151f30 f   wzFilePacker_static_d:dirtree.obj
 0002:000dff80       _DirTree_GetName           10151f80 f   wzFilePacker_static_d:dirtree.obj
 0002:000e0090       _DirTree_FileExists        10152090 f   wzFilePacker_static_d:dirtree.obj
 0002:000e0100       _DirTree_CreateFinder      10152100 f   wzFilePacker_static_d:dirtree.obj
 0002:000e0370       _DirTree_DestroyFinder     10152370 f   wzFilePacker_static_d:dirtree.obj
 0002:000e04b0       _DirTree_FinderGetNextFile 101524b0 f   wzFilePacker_static_d:dirtree.obj
 0002:000e0650       _DuplicateString           10152650 f   wzFilePacker_static_d:dirtree-common.obj
 0002:000e06f0       _GetNextDir                101526f0 f   wzFilePacker_static_d:dirtree-common.obj
 0002:000e0790       _MatchPattern              10152790 f   wzFilePacker_static_d:dirtree-common.obj
 0002:000e0930       _PathHasDir                10152930 f   wzFilePacker_static_d:dirtree-common.obj
 0002:000e0990       _timeKillEvent@4           10152990 f   winmm:WINMM.dll
 0002:000e0996       _timeSetEvent@20           10152996 f   winmm:WINMM.dll
 0002:000e099c       _mmioClose@8               1015299c f   winmm:WINMM.dll
 0002:000e09a2       _mmioSeek@12               101529a2 f   winmm:WINMM.dll
 0002:000e09a8       _mmioRead@12               101529a8 f   winmm:WINMM.dll
 0002:000e09ae       _timeEndPeriod@4           101529ae f   winmm:WINMM.dll
 0002:000e09b4       _timeGetTime@0             101529b4 f   winmm:WINMM.dll
 0002:000e09ba       _timeBeginPeriod@4         101529ba f   winmm:WINMM.dll
 0002:000e09c0       _mixerClose@4              101529c0 f   winmm:WINMM.dll
 0002:000e09c6       _mixerGetDevCapsA@12       101529c6 f   winmm:WINMM.dll
 0002:000e09cc       _mixerOpen@20              101529cc f   winmm:WINMM.dll
 0002:000e09d2       _mixerGetNumDevs@0         101529d2 f   winmm:WINMM.dll
 0002:000e09d8       _mixerGetLineInfoA@12      101529d8 f   winmm:WINMM.dll
 0002:000e09de       _mixerGetLineControlsA@12  101529de f   winmm:WINMM.dll
 0002:000e09e4       _mixerGetControlDetailsA@12 101529e4 f   winmm:WINMM.dll
 0002:000e09ea       _mixerSetControlDetails@12 101529ea f   winmm:WINMM.dll
 0002:000e09f0       _filelength                101529f0 f   libcmt:flength.obj
 0002:000e09f0       __filelength               101529f0 f   libcmt:flength.obj
 0002:000e0b2e       __mbsstr_l                 10152b2e f   libcmt:mbsstr.obj
 0002:000e0cbf       __mbsstr                   10152cbf f   libcmt:mbsstr.obj
 0002:000e0d00       __wassert                  10152d00 f   libcmt:wassert.obj
 0002:000e1626       _remove                    10153626 f   libcmt:unlink.obj
 0002:000e1662       __unlink                   10153662 f   libcmt:unlink.obj
 0002:000e166f       __findclose                1015366f f   libcmt:findfile.obj
 0002:000e169e       ___timet_from_ft           1015369e f   libcmt:findfile.obj
 0002:000e171d       __findfirst32              1015371d f   libcmt:findfile.obj
 0002:000e188d       __findnext32               1015388d f   libcmt:findfile.obj
 0002:000e19fc       ___time64_t_from_ft        101539fc f   libcmt:findfi32.obj
 0002:000e1a7e       __findfirst64i32           10153a7e f   libcmt:findfi32.obj
 0002:000e1bfa       __findnext64i32            10153bfa f   libcmt:findfi32.obj
 0002:000e1d74       __SEH_prolog4              10153d74 f   libcmt:sehprolg4.obj
 0002:000e1db9       __SEH_epilog4              10153db9 f   libcmt:sehprolg4.obj
 0002:000e1de3       _fwprintf                  10153de3 f   libcmt:fwprintf.obj
 0002:000e1e9c       __fwprintf_l               10153e9c f   libcmt:fwprintf.obj
 0002:000e1ebf       __fwprintf_s_l             10153ebf f   libcmt:fwprintf.obj
 0002:000e1ee2       _fwprintf_s                10153ee2 f   libcmt:fwprintf.obj
 0002:000e1f03       __fwprintf_p_l             10153f03 f   libcmt:fwprintf.obj
 0002:000e1f26       __fwprintf_p               10153f26 f   libcmt:fwprintf.obj
 0002:000e1f47       _setvbuf                   10153f47 f   libcmt:setvbuf.obj
 0002:000e2084       _wcsncat_s                 10154084 f   libcmt:wcsncat_s.obj
 0002:000e21ad       _wcsncpy_s                 101541ad f   libcmt:wcsncpy_s.obj
 0002:000e22b4       ___loctotime32_t           101542b4 f   libcmt:dtoxtime.obj
 0002:000e253b       ___loctotime64_t           1015453b f   libcmt:dtoxtm64.obj
 0002:000e2840       _vfwprintf_helper          10154840 f   libcmt:vfwprint.obj
 0002:000e28f7       __vfwprintf_l              101548f7 f   libcmt:vfwprint.obj
 0002:000e291f       __vfwprintf_s_l            1015491f f   libcmt:vfwprint.obj
 0002:000e2947       __vfwprintf_p_l            10154947 f   libcmt:vfwprint.obj
 0002:000e296f       _vfwprintf                 1015496f f   libcmt:vfwprint.obj
 0002:000e2995       _vfwprintf_s               10154995 f   libcmt:vfwprint.obj
 0002:000e29bb       __vfwprintf_p              101549bb f   libcmt:vfwprint.obj
 0002:000e29e1       _wait_a_bit                101549e1 f i libcmt:crtheap.obj
 0002:000e2a10       __set_malloc_crt_max_wait  10154a10 f   libcmt:crtheap.obj
 0002:000e2a2a       __malloc_crt               10154a2a f   libcmt:crtheap.obj
 0002:000e2a80       __calloc_crt               10154a80 f   libcmt:crtheap.obj
 0002:000e2adf       __realloc_crt              10154adf f   libcmt:crtheap.obj
 0002:000e2b40       __recalloc_crt             10154b40 f   libcmt:crtheap.obj
 0002:000e2ba6       __calloc_impl              10154ba6 f   libcmt:calloc_impl.obj
 0002:000e2d0c       _MakeSureDirectoryPathExists@4 10154d0c f   Dbghelp:dbghelp.dll
 0002:000e2d12       _InterlockedIncrement@4    10154d12 f   kernel32:KERNEL32.dll
 0002:000e2d18       _InterlockedDecrement@4    10154d18 f   kernel32:KERNEL32.dll
 0002:000e2d1e       _RtlUnwind@16              10154d1e f   kernel32:KERNEL32.dll
 0002:000e2d24       _TerminateProcess@8        10154d24 f   kernel32:KERNEL32.dll
 0002:000e2d2a       _GetCurrentProcess@0       10154d2a f   kernel32:KERNEL32.dll
 0002:000e2d30       _UnhandledExceptionFilter@4 10154d30 f   kernel32:KERNEL32.dll
 0002:000e2d36       _SetUnhandledExceptionFilter@4 10154d36 f   kernel32:KERNEL32.dll
 0002:000e2d3c       _IsDebuggerPresent@0       10154d3c f   kernel32:KERNEL32.dll
 0002:000e2d42       _GetModuleFileNameW@12     10154d42 f   kernel32:KERNEL32.dll
 0002:000e2d48       _RaiseException@16         10154d48 f   kernel32:KERNEL32.dll
 0002:000e2d4e       _DebugBreak@0              10154d4e f   kernel32:KERNEL32.dll
 0002:000e2d54       _WideCharToMultiByte@32    10154d54 f   kernel32:KERNEL32.dll
 0002:000e2d5a       _MultiByteToWideChar@24    10154d5a f   kernel32:KERNEL32.dll
 0002:000e2d60       _lstrlenA@4                10154d60 f   kernel32:KERNEL32.dll
 0002:000e2d66       _HeapValidate@12           10154d66 f   kernel32:KERNEL32.dll
 0002:000e2d6c       _IsBadReadPtr@8            10154d6c f   kernel32:KERNEL32.dll
 0002:000e2d72       _GetCurrentThreadId@0      10154d72 f   kernel32:KERNEL32.dll
 0002:000e2d78       _GetCommandLineA@0         10154d78 f   kernel32:KERNEL32.dll
 0002:000e2d7e       _GetModuleHandleW@4        10154d7e f   kernel32:KERNEL32.dll
 0002:000e2d84       _ExitProcess@4             10154d84 f   kernel32:KERNEL32.dll
 0002:000e2d8a       _GetACP@0                  10154d8a f   kernel32:KERNEL32.dll
 0002:000e2d90       _GetOEMCP@0                10154d90 f   kernel32:KERNEL32.dll
 0002:000e2d96       _GetCPInfo@8               10154d96 f   kernel32:KERNEL32.dll
 0002:000e2d9c       _IsValidCodePage@4         10154d9c f   kernel32:KERNEL32.dll
 0002:000e2da2       _TlsGetValue@4             10154da2 f   kernel32:KERNEL32.dll
 0002:000e2da8       _TlsAlloc@0                10154da8 f   kernel32:KERNEL32.dll
 0002:000e2dae       _TlsSetValue@8             10154dae f   kernel32:KERNEL32.dll
 0002:000e2db4       _TlsFree@4                 10154db4 f   kernel32:KERNEL32.dll
 0002:000e2dba       _SetLastError@4            10154dba f   kernel32:KERNEL32.dll
 0002:000e2dc0       _GetCurrentThread@0        10154dc0 f   kernel32:KERNEL32.dll
 0002:000e2dc6       _GetModuleHandleA@4        10154dc6 f   kernel32:KERNEL32.dll
 0002:000e2dcc       _FatalAppExitA@8           10154dcc f   kernel32:KERNEL32.dll
 0002:000e2dd2       _GetStdHandle@4            10154dd2 f   kernel32:KERNEL32.dll
 0002:000e2dd8       _WriteFile@20              10154dd8 f   kernel32:KERNEL32.dll
 0002:000e2dde       _WriteConsoleW@20          10154dde f   kernel32:KERNEL32.dll
 0002:000e2de4       _GetFileType@4             10154de4 f   kernel32:KERNEL32.dll
 0002:000e2dea       _OutputDebugStringW@4      10154dea f   kernel32:KERNEL32.dll
 0002:000e2df0       _SetConsoleCtrlHandler@8   10154df0 f   kernel32:KERNEL32.dll
 0002:000e2df6       _LoadLibraryW@4            10154df6 f   kernel32:KERNEL32.dll
 0002:000e2dfc       _HeapFree@12               10154dfc f   kernel32:KERNEL32.dll
 0002:000e2e02       _HeapAlloc@12              10154e02 f   kernel32:KERNEL32.dll
 0002:000e2e08       _GetProcessHeap@0          10154e08 f   kernel32:KERNEL32.dll
 0002:000e2e0e       _VirtualQuery@12           10154e0e f   kernel32:KERNEL32.dll
 0002:000e2e14       _CloseHandle@4             10154e14 f   kernel32:KERNEL32.dll
 0002:000e2e1a       _SetHandleCount@4          10154e1a f   kernel32:KERNEL32.dll
 0002:000e2e20       _GetStartupInfoA@4         10154e20 f   kernel32:KERNEL32.dll
 0002:000e2e26       _SetFilePointer@16         10154e26 f   kernel32:KERNEL32.dll
 0002:000e2e2c       _ReadFile@20               10154e2c f   kernel32:KERNEL32.dll
 0002:000e2e32       _GetConsoleCP@0            10154e32 f   kernel32:KERNEL32.dll
 0002:000e2e38       _GetConsoleMode@8          10154e38 f   kernel32:KERNEL32.dll
 0002:000e2e3e       _HeapSize@12               10154e3e f   kernel32:KERNEL32.dll
 0002:000e2e44       _HeapReAlloc@16            10154e44 f   kernel32:KERNEL32.dll
 0002:000e2e4a       _HeapDestroy@4             10154e4a f   kernel32:KERNEL32.dll
 0002:000e2e50       _HeapCreate@12             10154e50 f   kernel32:KERNEL32.dll
 0002:000e2e56       _VirtualFree@12            10154e56 f   kernel32:KERNEL32.dll
 0002:000e2e5c       _VirtualAlloc@16           10154e5c f   kernel32:KERNEL32.dll
 0002:000e2e62       _FreeEnvironmentStringsA@4 10154e62 f   kernel32:KERNEL32.dll
 0002:000e2e68       _GetEnvironmentStrings@0   10154e68 f   kernel32:KERNEL32.dll
 0002:000e2e6e       _FreeEnvironmentStringsW@4 10154e6e f   kernel32:KERNEL32.dll
 0002:000e2e74       _GetEnvironmentStringsW@0  10154e74 f   kernel32:KERNEL32.dll
 0002:000e2e7a       _QueryPerformanceCounter@4 10154e7a f   kernel32:KERNEL32.dll
 0002:000e2e80       _GetTickCount@0            10154e80 f   kernel32:KERNEL32.dll
 0002:000e2e86       _GetCurrentProcessId@0     10154e86 f   kernel32:KERNEL32.dll
 0002:000e2e8c       _GetSystemTimeAsFileTime@4 10154e8c f   kernel32:KERNEL32.dll
 0002:000e2e92       _FlushFileBuffers@4        10154e92 f   kernel32:KERNEL32.dll
 0002:000e2e98       _LCMapStringA@24           10154e98 f   kernel32:KERNEL32.dll
 0002:000e2e9e       _LCMapStringW@24           10154e9e f   kernel32:KERNEL32.dll
 0002:000e2ea4       _SetStdHandle@8            10154ea4 f   kernel32:KERNEL32.dll
 0002:000e2eaa       _InitializeCriticalSectionAndSpinCount@8 10154eaa f   kernel32:KERNEL32.dll
 0002:000e2eb0       _GetStringTypeA@20         10154eb0 f   kernel32:KERNEL32.dll
 0002:000e2eb6       _GetStringTypeW@16         10154eb6 f   kernel32:KERNEL32.dll
 0002:000e2ebc       _GetTimeFormatA@24         10154ebc f   kernel32:KERNEL32.dll
 0002:000e2ec2       _GetDateFormatA@24         10154ec2 f   kernel32:KERNEL32.dll
 0002:000e2ec8       _GetLocaleInfoA@16         10154ec8 f   kernel32:KERNEL32.dll
 0002:000e2ece       _IsValidLocale@8           10154ece f   kernel32:KERNEL32.dll
 0002:000e2ed4       _EnumSystemLocalesA@8      10154ed4 f   kernel32:KERNEL32.dll
 0002:000e2eda       _GetUserDefaultLCID@0      10154eda f   kernel32:KERNEL32.dll
 0002:000e2ee0       _CreateFileA@28            10154ee0 f   kernel32:KERNEL32.dll
 0002:000e2ee6       _WriteConsoleA@20          10154ee6 f   kernel32:KERNEL32.dll
 0002:000e2eec       _GetConsoleOutputCP@0      10154eec f   kernel32:KERNEL32.dll
 0002:000e2ef2       _GetLocaleInfoW@16         10154ef2 f   kernel32:KERNEL32.dll
 0002:000e2ef8       _GetTimeZoneInformation@4  10154ef8 f   kernel32:KERNEL32.dll
 0002:000e2efe       _SetEndOfFile@4            10154efe f   kernel32:KERNEL32.dll
 0002:000e2f04       _CompareStringA@24         10154f04 f   kernel32:KERNEL32.dll
 0002:000e2f0a       _CompareStringW@24         10154f0a f   kernel32:KERNEL32.dll
 0002:000e2f10       _SetEnvironmentVariableA@8 10154f10 f   kernel32:KERNEL32.dll
 0002:000e2f16       _lstrcpyA@8                10154f16 f   kernel32:KERNEL32.dll
 0002:000e2f1c       _FindNextFileA@8           10154f1c f   kernel32:KERNEL32.dll
 0002:000e2f22       _FindFirstFileA@8          10154f22 f   kernel32:KERNEL32.dll
 0002:000e2f28       _FindClose@4               10154f28 f   kernel32:KERNEL32.dll
 0002:000e2f2e       _RemoveDirectoryA@4        10154f2e f   kernel32:KERNEL32.dll
 0002:000e2f34       _GetSystemDirectoryA@8     10154f34 f   kernel32:KERNEL32.dll
 0002:000e2f3a       _CreateDirectoryA@8        10154f3a f   kernel32:KERNEL32.dll
 0002:000e2f40       _SetFilePointerEx@20       10154f40 f   kernel32:KERNEL32.dll
 0002:000e2f46       _GetFileSizeEx@8           10154f46 f   kernel32:KERNEL32.dll
 0002:000e2f4c       _GetFileInformationByHandle@8 10154f4c f   kernel32:KERNEL32.dll
 0002:000e2f52       _SetFileAttributesA@8      10154f52 f   kernel32:KERNEL32.dll
 0002:000e2f58       _SetFileTime@16            10154f58 f   kernel32:KERNEL32.dll
 0002:000e2f5e       _DeleteFileA@4             10154f5e f   kernel32:KERNEL32.dll
 0002:000e2f64       _MoveFileA@8               10154f64 f   kernel32:KERNEL32.dll
 0002:000e2f6a       _FileTimeToSystemTime@8    10154f6a f   kernel32:KERNEL32.dll
 0002:000e2f70       _FileTimeToLocalFileTime@8 10154f70 f   kernel32:KERNEL32.dll
 0002:000e2f76       _SendMessageA@16           10154f76 f   user32:USER32.dll
 0002:000e2f7c       _wsprintfA                 10154f7c f   user32:USER32.dll
 0002:000e2f90       _ogg_page_version          10154f90 f   ogg_static:framing.obj
 0002:000e2fb0       _ogg_page_continued        10154fb0 f   ogg_static:framing.obj
 0002:000e2fd0       _ogg_page_bos              10154fd0 f   ogg_static:framing.obj
 0002:000e2ff0       _ogg_page_eos              10154ff0 f   ogg_static:framing.obj
 0002:000e3010       _ogg_page_granulepos       10155010 f   ogg_static:framing.obj
 0002:000e3130       _ogg_page_serialno         10155130 f   ogg_static:framing.obj
 0002:000e3170       _ogg_page_pageno           10155170 f   ogg_static:framing.obj
 0002:000e31b0       _ogg_page_packets          101551b0 f   ogg_static:framing.obj
 0002:000e31f0       _ogg_stream_init           101551f0 f   ogg_static:framing.obj
 0002:000e3280       _ogg_stream_clear          10155280 f   ogg_static:framing.obj
 0002:000e32f0       _ogg_stream_destroy        101552f0 f   ogg_static:framing.obj
 0002:000e3320       _ogg_page_checksum_set     10155320 f   ogg_static:framing.obj
 0002:000e3400       _ogg_stream_packetin       10155400 f   ogg_static:framing.obj
 0002:000e3670       _ogg_stream_flush          10155670 f   ogg_static:framing.obj
 0002:000e38f0       _ogg_stream_pageout        101558f0 f   ogg_static:framing.obj
 0002:000e3960       _ogg_stream_eos            10155960 f   ogg_static:framing.obj
 0002:000e3980       _ogg_sync_init             10155980 f   ogg_static:framing.obj
 0002:000e39b0       _ogg_sync_clear            101559b0 f   ogg_static:framing.obj
 0002:000e39f0       _ogg_sync_destroy          101559f0 f   ogg_static:framing.obj
 0002:000e3a20       _ogg_sync_buffer           10155a20 f   ogg_static:framing.obj
 0002:000e3ac0       _ogg_sync_wrote            10155ac0 f   ogg_static:framing.obj
 0002:000e3af0       _ogg_sync_pageseek         10155af0 f   ogg_static:framing.obj
 0002:000e3ca0       _ogg_sync_pageout          10155ca0 f   ogg_static:framing.obj
 0002:000e3cf0       _ogg_stream_pagein         10155cf0 f   ogg_static:framing.obj
 0002:000e40a0       _ogg_sync_reset            101560a0 f   ogg_static:framing.obj
 0002:000e40d0       _ogg_stream_reset          101560d0 f   ogg_static:framing.obj
 0002:000e4140       _ogg_stream_reset_serialno 10156140 f   ogg_static:framing.obj
 0002:000e4170       _ogg_stream_packetout      10156170 f   ogg_static:framing.obj
 0002:000e4320       _ogg_stream_packetpeek     10156320 f   ogg_static:framing.obj
 0002:000e4350       _ogg_packet_clear          10156350 f   ogg_static:framing.obj
 0002:000e4380       _oggpack_writeinit         10156380 f   ogg_static:bitwise.obj
 0002:000e43d0       _oggpackB_writeinit        101563d0 f   ogg_static:bitwise.obj
 0002:000e43f0       _oggpack_writetrunc        101563f0 f   ogg_static:bitwise.obj
 0002:000e4440       _oggpackB_writetrunc       10156440 f   ogg_static:bitwise.obj
 0002:000e4490       _oggpack_write             10156490 f   ogg_static:bitwise.obj
 0002:000e45d0       _oggpackB_write            101565d0 f   ogg_static:bitwise.obj
 0002:000e4700       _oggpack_writealign        10156700 f   ogg_static:bitwise.obj
 0002:000e4730       _oggpackB_writealign       10156730 f   ogg_static:bitwise.obj
 0002:000e4760       _oggpack_writecopy         10156760 f   ogg_static:bitwise.obj
 0002:000e48b0       _oggpackB_writecopy        101568b0 f   ogg_static:bitwise.obj
 0002:000e48e0       _oggpack_reset             101568e0 f   ogg_static:bitwise.obj
 0002:000e4910       _oggpackB_reset            10156910 f   ogg_static:bitwise.obj
 0002:000e4930       _oggpack_writeclear        10156930 f   ogg_static:bitwise.obj
 0002:000e4970       _oggpackB_writeclear       10156970 f   ogg_static:bitwise.obj
 0002:000e4990       _oggpack_readinit          10156990 f   ogg_static:bitwise.obj
 0002:000e49d0       _oggpackB_readinit         101569d0 f   ogg_static:bitwise.obj
 0002:000e4a00       _oggpack_look              10156a00 f   ogg_static:bitwise.obj
 0002:000e4ae0       _oggpackB_look             10156ae0 f   ogg_static:bitwise.obj
 0002:000e4bc0       _oggpack_look1             10156bc0 f   ogg_static:bitwise.obj
 0002:000e4c00       _oggpackB_look1            10156c00 f   ogg_static:bitwise.obj
 0002:000e4c40       _oggpack_adv               10156c40 f   ogg_static:bitwise.obj
 0002:000e4c80       _oggpackB_adv              10156c80 f   ogg_static:bitwise.obj
 0002:000e4cb0       _oggpack_adv1              10156cb0 f   ogg_static:bitwise.obj
 0002:000e4cf0       _oggpackB_adv1             10156cf0 f   ogg_static:bitwise.obj
 0002:000e4d10       _oggpack_read              10156d10 f   ogg_static:bitwise.obj
 0002:000e4e20       _oggpackB_read             10156e20 f   ogg_static:bitwise.obj
 0002:000e4f30       _oggpack_read1             10156f30 f   ogg_static:bitwise.obj
 0002:000e4fa0       _oggpackB_read1            10156fa0 f   ogg_static:bitwise.obj
 0002:000e5010       _oggpack_bytes             10157010 f   ogg_static:bitwise.obj
 0002:000e5040       _oggpack_bits              10157040 f   ogg_static:bitwise.obj
 0002:000e5060       _oggpackB_bytes            10157060 f   ogg_static:bitwise.obj
 0002:000e5080       _oggpackB_bits             10157080 f   ogg_static:bitwise.obj
 0002:000e50a0       _oggpack_get_buffer        101570a0 f   ogg_static:bitwise.obj
 0002:000e50c0       _oggpackB_get_buffer       101570c0 f   ogg_static:bitwise.obj
 0003:00000000       ___xc_a                    1017b000     LIBCMTD:crt0init.obj
 0003:00000348       ___xc_z                    1017b348     LIBCMTD:crt0init.obj
 0003:0000044c       ___xi_a                    1017b44c     LIBCMTD:crt0init.obj
 0003:00000668       ___xi_z                    1017b668     LIBCMTD:crt0init.obj
 0003:0000076c       ___xp_a                    1017b76c     LIBCMTD:crt0init.obj
 0003:00000a80       ___xp_z                    1017ba80     LIBCMTD:crt0init.obj
 0003:00000b84       ___xt_a                    1017bb84     LIBCMTD:crt0init.obj
 0003:00000c88       ___xt_z                    1017bc88     LIBCMTD:crt0init.obj
 0003:00001327       ?_Value@?$_Is_swap_move@U_Swap_move_tag@std@@@std@@2_NB 1017c327     audiostr.obj
 0003:00001328       ?value@?$integral_constant@_N$0A@@tr1@std@@2_NB 1017c328     audiostr.obj
 0003:00001329       ?value@?$integral_constant@_N$00@tr1@std@@2_NB 1017c329     audiostr.obj
 0003:00001330       __real@bff0000000000000    1017c330     audiostr.obj
 0003:0000133c       __real@bf800000            1017c33c     audiostr.obj
 0003:000027d4       _CLSID_DirectSound         1017d7d4     ds.obj
 0003:000027e8       _CLSID_DirectSound8        1017d7e8     ds.obj
 0003:000027fc       _CLSID_DirectSoundCapture  1017d7fc     ds.obj
 0003:00002810       _CLSID_DirectSoundCapture8 1017d810     ds.obj
 0003:00002824       _CLSID_DirectSoundFullDuplex 1017d824     ds.obj
 0003:00002838       _DSDEVID_DefaultPlayback   1017d838     ds.obj
 0003:0000284c       _DSDEVID_DefaultCapture    1017d84c     ds.obj
 0003:00002860       _DSDEVID_DefaultVoicePlayback 1017d860     ds.obj
 0003:00002874       _DSDEVID_DefaultVoiceCapture 1017d874     ds.obj
 0003:00002888       _IID_IReferenceClock       1017d888     ds.obj
 0003:0000289c       _IID_IDirectSound          1017d89c     ds.obj
 0003:000028b0       _IID_IDirectSound8         1017d8b0     ds.obj
 0003:000028c4       _IID_IDirectSoundBuffer    1017d8c4     ds.obj
 0003:000028d8       _IID_IDirectSoundBuffer8   1017d8d8     ds.obj
 0003:000028ec       _GUID_All_Objects          1017d8ec     ds.obj
 0003:00002900       _IID_IDirectSound3DListener 1017d900     ds.obj
 0003:00002914       _IID_IDirectSound3DBuffer  1017d914     ds.obj
 0003:00002928       _IID_IDirectSoundCapture   1017d928     ds.obj
 0003:0000293c       _IID_IDirectSoundCaptureBuffer 1017d93c     ds.obj
 0003:00002950       _IID_IDirectSoundCaptureBuffer8 1017d950     ds.obj
 0003:00002964       _IID_IDirectSoundNotify    1017d964     ds.obj
 0003:00002978       _IID_IKsPropertySet        1017d978     ds.obj
 0003:0000298c       _IID_IDirectSoundFXGargle  1017d98c     ds.obj
 0003:000029a0       _IID_IDirectSoundFXChorus  1017d9a0     ds.obj
 0003:000029b4       _IID_IDirectSoundFXFlanger 1017d9b4     ds.obj
 0003:000029c8       _IID_IDirectSoundFXEcho    1017d9c8     ds.obj
 0003:000029dc       _IID_IDirectSoundFXDistortion 1017d9dc     ds.obj
 0003:000029f0       _IID_IDirectSoundFXCompressor 1017d9f0     ds.obj
 0003:00002a04       _IID_IDirectSoundFXParamEq 1017da04     ds.obj
 0003:00002a18       _IID_IDirectSoundFXI3DL2Reverb 1017da18     ds.obj
 0003:00002a2c       _IID_IDirectSoundFXWavesReverb 1017da2c     ds.obj
 0003:00002a40       _IID_IDirectSoundCaptureFXAec 1017da40     ds.obj
 0003:00002a54       _IID_IDirectSoundCaptureFXNoiseSuppress 1017da54     ds.obj
 0003:00002a68       _IID_IDirectSoundFullDuplex 1017da68     ds.obj
 0003:00002a7c       _DS3DALG_NO_VIRTUALIZATION 1017da7c     ds.obj
 0003:00002a90       _DS3DALG_HRTF_FULL         1017da90     ds.obj
 0003:00002aa4       _DS3DALG_HRTF_LIGHT        1017daa4     ds.obj
 0003:00002ab8       _GUID_DSFX_STANDARD_GARGLE 1017dab8     ds.obj
 0003:00002acc       _GUID_DSFX_STANDARD_CHORUS 1017dacc     ds.obj
 0003:00002ae0       _GUID_DSFX_STANDARD_FLANGER 1017dae0     ds.obj
 0003:00002af4       _GUID_DSFX_STANDARD_ECHO   1017daf4     ds.obj
 0003:00002b08       _GUID_DSFX_STANDARD_DISTORTION 1017db08     ds.obj
 0003:00002b1c       _GUID_DSFX_STANDARD_COMPRESSOR 1017db1c     ds.obj
 0003:00002b30       _GUID_DSFX_STANDARD_PARAMEQ 1017db30     ds.obj
 0003:00002b44       _GUID_DSFX_STANDARD_I3DL2REVERB 1017db44     ds.obj
 0003:00002b58       _GUID_DSFX_WAVES_REVERB    1017db58     ds.obj
 0003:00002b6c       _GUID_DSCFX_CLASS_AEC      1017db6c     ds.obj
 0003:00002b80       _GUID_DSCFX_MS_AEC         1017db80     ds.obj
 0003:00002b94       _GUID_DSCFX_SYSTEM_AEC     1017db94     ds.obj
 0003:00002ba8       _GUID_DSCFX_CLASS_NS       1017dba8     ds.obj
 0003:00002bbc       _GUID_DSCFX_MS_NS          1017dbbc     ds.obj
 0003:00002bd0       _GUID_DSCFX_SYSTEM_NS      1017dbd0     ds.obj
 0003:00002be4       _DSPROPSETID_EAX_ReverbProperties 1017dbe4     ds.obj
 0003:00002bf8       _DSPROPSETID_EAXBUFFER_ReverbProperties 1017dbf8     ds.obj
 0003:00002c10       __real@408f400000000000    1017dc10     ds.obj
 0003:00002c1c       __real@40000000            1017dc1c     ds.obj
 0003:00002c20       __real@4059000000000000    1017dc20     ds.obj
 0003:00002c30       __real@4000000000000000    1017dc30     ds.obj
 0003:00002c3c       ??_C@_1DC@POOIKBAO@?$AAI?$AAT?$AAE?$AAR?$AAA?$AAT?$AAO?$AAR?$AA?5?$AAL?$AAI?$AAS?$AAT?$AA?5?$AAC?$AAO?$AAR?$AAR?$AAU?$AAP?$AAT?$AAE?$AAD?$AA?$CB?$AA?$AA@ 1017dc3c     ds.obj
 0003:00002c78       ??_C@_1IC@LODEOCIN@?$AAC?$AA?3?$AA?2?$AAP?$AAr?$AAo?$AAg?$AAr?$AAa?$AAm?$AA?5?$AAF?$AAi?$AAl?$AAe?$AAs?$AA?2?$AAM?$AAi?$AAc?$AAr?$AAo?$AAs?$AAo?$AAf?$AAt?$AA?5?$AAV?$AAi?$AAs?$AAu?$AAa@ 1017dc78     ds.obj
 0003:00002d14       __real@00000000            1017dd14     ds.obj
 0003:00002d18       __real@3f800000            1017dd18     ds.obj
 0003:00002d1c       __real@3dcccccd            1017dd1c     ds.obj
 0003:00002d20       __real@41a00000            1017dd20     ds.obj
 0003:00002d28       ??_C@_1HM@OJBANLJC@?$AAC?$AA?3?$AA?2?$AAP?$AAr?$AAo?$AAg?$AAr?$AAa?$AAm?$AA?5?$AAF?$AAi?$AAl?$AAe?$AAs?$AA?2?$AAM?$AAi?$AAc?$AAr?$AAo?$AAs?$AAo?$AAf?$AAt?$AA?5?$AAV?$AAi?$AAs?$AAu?$AAa@ 1017dd28     ds.obj
 0003:00002dbc       ??_C@_1CG@JNLFBNGN@?$AA?$CC?$AAi?$AAn?$AAv?$AAa?$AAl?$AAi?$AAd?$AA?5?$AAa?$AAr?$AAg?$AAu?$AAm?$AAe?$AAn?$AAt?$AA?$CC?$AA?$AA@ 1017ddbc     ds.obj
 0003:00002df0       ??_C@_1BGG@LHHKKPG@?$AAs?$AAt?$AAd?$AA?3?$AA?3?$AA_?$AAT?$AAr?$AAe?$AAe?$AA?$DM?$AAc?$AAl?$AAa?$AAs?$AAs?$AA?5?$AAs?$AAt?$AAd?$AA?3?$AA?3?$AA_?$AAT?$AAm?$AAa?$AAp?$AA_?$AAt?$AAr?$AAa?$AAi@ 1017ddf0     ds.obj
 0003:00002fa0       ??_C@_1FO@OCPOOAIA@?$AA?$CI?$AA?$CC?$AAS?$AAt?$AAa?$AAn?$AAd?$AAa?$AAr?$AAd?$AA?5?$AAC?$AA?$CL?$AA?$CL?$AA?5?$AAL?$AAi?$AAb?$AAr?$AAa?$AAr?$AAi?$AAe?$AAs?$AA?5?$AAI?$AAn?$AAv?$AAa?$AAl?$AAi?$AAd@ 1017dfa0     ds.obj
 0003:00003010       ??_C@_1DO@CFEEPGGJ@?$AAm?$AAa?$AAp?$AA?1?$AAs?$AAe?$AAt?$AA?5?$AAi?$AAt?$AAe?$AAr?$AAa?$AAt?$AAo?$AAr?$AAs?$AA?5?$AAi?$AAn?$AAc?$AAo?$AAm?$AAp?$AAa?$AAt?$AAi?$AAb?$AAl?$AAe?$AA?$AA@ 1017e010     ds.obj
 0003:0000305c       ??_C@_1BO@MEPPHOO@?$AA?$CC?$AAo?$AAu?$AAt?$AA?5?$AAo?$AAf?$AA?5?$AAr?$AAa?$AAn?$AAg?$AAe?$AA?$CC?$AA?$AA@ 1017e05c     ds.obj
 0003:00003080       ??_C@_1BGE@GOAIKILD@?$AAs?$AAt?$AAd?$AA?3?$AA?3?$AA_?$AAT?$AAr?$AAe?$AAe?$AA?$DM?$AAc?$AAl?$AAa?$AAs?$AAs?$AA?5?$AAs?$AAt?$AAd?$AA?3?$AA?3?$AA_?$AAT?$AAm?$AAa?$AAp?$AA_?$AAt?$AAr?$AAa?$AAi@ 1017e080     ds.obj
 0003:00003230       ??_C@_1FG@CMLDHNON@?$AA?$CI?$AA?$CC?$AAS?$AAt?$AAa?$AAn?$AAd?$AAa?$AAr?$AAd?$AA?5?$AAC?$AA?$CL?$AA?$CL?$AA?5?$AAL?$AAi?$AAb?$AAr?$AAa?$AAr?$AAi?$AAe?$AAs?$AA?5?$AAO?$AAu?$AAt?$AA?5?$AAo?$AAf?$AA?5@ 1017e230     ds.obj
 0003:00003298       ??_C@_1EI@FHEHNNNM@?$AAm?$AAa?$AAp?$AA?1?$AAs?$AAe?$AAt?$AA?5?$AAi?$AAt?$AAe?$AAr?$AAa?$AAt?$AAo?$AAr?$AA?5?$AAn?$AAo?$AAt?$AA?5?$AAd?$AAe?$AAr?$AAe?$AAf?$AAe?$AAr?$AAe?$AAn?$AAc?$AAa@ 1017e298     ds.obj
 0003:000032f0       ??_C@_1CE@IGJMOCCK@?$AAi?$AAn?$AAv?$AAa?$AAl?$AAi?$AAd?$AA?5?$AAo?$AAp?$AAe?$AAr?$AAa?$AAt?$AAo?$AAr?$AA?$DM?$AA?$AA@ 1017e2f0     ds.obj
 0003:00003598       __real@0000000000000000    1017e598     ds3d.obj
 0003:000039b0       __real@4020000000000000    1017e9b0     sound.obj
 0003:000039c0       __real@4097700000000000    1017e9c0     sound.obj
 0003:000039d0       __real@3fb99999a0000000    1017e9d0     sound.obj
 0003:000039e0       __real@3ff0000000000000    1017e9e0     sound.obj
 0003:000039f0       __real@3fd3333333333333    1017e9f0     sound.obj
 0003:00003a00       __real@3fe0000000000000    1017ea00     sound.obj
 0003:00003a10       ??_C@_1EK@PPDBPCAN@?$AAm?$AAa?$AAp?$AA?1?$AAs?$AAe?$AAt?$AA?5?$AAe?$AAr?$AAa?$AAs?$AAe?$AA?5?$AAi?$AAt?$AAe?$AAr?$AAa?$AAt?$AAo?$AAr?$AA?5?$AAo?$AAu?$AAt?$AAs?$AAi?$AAd?$AAe?$AA?5?$AAr@ 1017ea10     sound.obj
 0003:00003a68       ??_C@_1EM@MHOKKPFH@?$AAm?$AAa?$AAp?$AA?1?$AAs?$AAe?$AAt?$AA?5?$AAi?$AAn?$AAs?$AAe?$AAr?$AAt?$AA?5?$AAi?$AAt?$AAe?$AAr?$AAa?$AAt?$AAo?$AAr?$AA?5?$AAo?$AAu?$AAt?$AAs?$AAi?$AAd?$AAe?$AA?5@ 1017ea68     sound.obj
 0003:00003ac8       ??_C@_1BFK@IPBODIEM@?$AAs?$AAt?$AAd?$AA?3?$AA?3?$AA_?$AAT?$AAr?$AAe?$AAe?$AA?$DM?$AAc?$AAl?$AAa?$AAs?$AAs?$AA?5?$AAs?$AAt?$AAd?$AA?3?$AA?3?$AA_?$AAT?$AAm?$AAa?$AAp?$AA_?$AAt?$AAr?$AAa?$AAi@ 1017eac8     sound.obj
 0003:00003c68       ??_C@_0BE@JONHPENG@map?1set?$DMT?$DO?5too?5long?$AA@ 1017ec68     sound.obj
 0003:00003c84       ??_7length_error@std@@6B@  1017ec84     sound.obj
 0003:00003c94       ??_7logic_error@std@@6B@   1017ec94     sound.obj
 0003:00003ca0       ?npos@?$basic_string@DU?$char_traits@D@std@@V?$allocator@D@2@@std@@2IB 1017eca0     sound.obj
 0003:00003ca8       ??_C@_1BFI@LALOFFFC@?$AAs?$AAt?$AAd?$AA?3?$AA?3?$AA_?$AAT?$AAr?$AAe?$AAe?$AA?$DM?$AAc?$AAl?$AAa?$AAs?$AAs?$AA?5?$AAs?$AAt?$AAd?$AA?3?$AA?3?$AA_?$AAT?$AAm?$AAa?$AAp?$AA_?$AAt?$AAr?$AAa?$AAi@ 1017eca8     sound.obj
 0003:00003e48       ??_C@_1BEM@HGECEAEO@?$AAs?$AAt?$AAd?$AA?3?$AA?3?$AA_?$AAT?$AAr?$AAe?$AAe?$AA?$DM?$AAc?$AAl?$AAa?$AAs?$AAs?$AA?5?$AAs?$AAt?$AAd?$AA?3?$AA?3?$AA_?$AAT?$AAm?$AAa?$AAp?$AA_?$AAt?$AAr?$AAa?$AAi@ 1017ee48     sound.obj
 0003:00003fd8       ??_C@_1EG@EHJFMBHJ@?$AAm?$AAa?$AAp?$AA?1?$AAs?$AAe?$AAt?$AA?5?$AAi?$AAt?$AAe?$AAr?$AAa?$AAt?$AAo?$AAr?$AA?5?$AAn?$AAo?$AAt?$AA?5?$AAi?$AAn?$AAc?$AAr?$AAe?$AAm?$AAe?$AAn?$AAt?$AAa?$AAb@ 1017efd8     sound.obj
 0003:00004030       ??_C@_1BEM@IHIAKFFM@?$AAs?$AAt?$AAd?$AA?3?$AA?3?$AA_?$AAT?$AAr?$AAe?$AAe?$AA?$DM?$AAc?$AAl?$AAa?$AAs?$AAs?$AA?5?$AAs?$AAt?$AAd?$AA?3?$AA?3?$AA_?$AAT?$AAm?$AAa?$AAp?$AA_?$AAt?$AAr?$AAa?$AAi@ 1017f030     sound.obj
 0003:000041c0       ??_C@_1EG@OKCGOALM@?$AAm?$AAa?$AAp?$AA?1?$AAs?$AAe?$AAt?$AA?5?$AAi?$AAt?$AAe?$AAr?$AAa?$AAt?$AAo?$AAr?$AA?5?$AAn?$AAo?$AAt?$AA?5?$AAd?$AAe?$AAc?$AAr?$AAe?$AAm?$AAe?$AAn?$AAt?$AAa?$AAb@ 1017f1c0     sound.obj
 0003:00004218       ??_C@_1IA@IJKDJKBN@?$AAC?$AA?3?$AA?2?$AAP?$AAr?$AAo?$AAg?$AAr?$AAa?$AAm?$AA?5?$AAF?$AAi?$AAl?$AAe?$AAs?$AA?2?$AAM?$AAi?$AAc?$AAr?$AAo?$AAs?$AAo?$AAf?$AAt?$AA?5?$AAV?$AAi?$AAs?$AAu?$AAa@ 1017f218     sound.obj
 0003:000042b4       ??_C@_1CK@EOPGIILJ@?$AAi?$AAn?$AAv?$AAa?$AAl?$AAi?$AAd?$AA?5?$AAn?$AAu?$AAl?$AAl?$AA?5?$AAp?$AAo?$AAi?$AAn?$AAt?$AAe?$AAr?$AA?$AA@ 1017f2b4     sound.obj
 0003:000042ec       ??_7bad_alloc@std@@6B@     1017f2ec     sound.obj
 0003:00004398       ??_C@_1BDG@CFDDHHDG@?$AAs?$AAt?$AAd?$AA?3?$AA?3?$AA_?$AAT?$AAr?$AAe?$AAe?$AA?$DM?$AAc?$AAl?$AAa?$AAs?$AAs?$AA?5?$AAs?$AAt?$AAd?$AA?3?$AA?3?$AA_?$AAT?$AAm?$AAa?$AAp?$AA_?$AAt?$AAr?$AAa?$AAi@ 1017f398     ambientsnd.obj
 0003:00004510       ??_C@_1BGO@DMJJHFDC@?$AAs?$AAt?$AAd?$AA?3?$AA?3?$AA_?$AAT?$AAr?$AAe?$AAe?$AA?$DM?$AAc?$AAl?$AAa?$AAs?$AAs?$AA?5?$AAs?$AAt?$AAd?$AA?3?$AA?3?$AA_?$AAT?$AAm?$AAa?$AAp?$AA_?$AAt?$AAr?$AAa?$AAi@ 1017f510     ambientsnd.obj
 0003:000046c8       ??_C@_1BDE@LBNKJBCD@?$AAs?$AAt?$AAd?$AA?3?$AA?3?$AA_?$AAT?$AAr?$AAe?$AAe?$AA?$DM?$AAc?$AAl?$AAa?$AAs?$AAs?$AA?5?$AAs?$AAt?$AAd?$AA?3?$AA?3?$AA_?$AAT?$AAm?$AAa?$AAp?$AA_?$AAt?$AAr?$AAa?$AAi@ 1017f6c8     ambientsnd.obj
 0003:00004840       ??_C@_1BGM@IJHGLFBJ@?$AAs?$AAt?$AAd?$AA?3?$AA?3?$AA_?$AAT?$AAr?$AAe?$AAe?$AA?$DM?$AAc?$AAl?$AAa?$AAs?$AAs?$AA?5?$AAs?$AAt?$AAd?$AA?3?$AA?3?$AA_?$AAT?$AAm?$AAa?$AAp?$AA_?$AAt?$AAr?$AAa?$AAi@ 1017f840     ambientsnd.obj
 0003:000049f8       ??_C@_1BCI@MMHLBAOK@?$AAs?$AAt?$AAd?$AA?3?$AA?3?$AA_?$AAT?$AAr?$AAe?$AAe?$AA?$DM?$AAc?$AAl?$AAa?$AAs?$AAs?$AA?5?$AAs?$AAt?$AAd?$AA?3?$AA?3?$AA_?$AAT?$AAm?$AAa?$AAp?$AA_?$AAt?$AAr?$AAa?$AAi@ 1017f9f8     ambientsnd.obj
 0003:00004b60       ??_C@_1BCI@DNLJPFPI@?$AAs?$AAt?$AAd?$AA?3?$AA?3?$AA_?$AAT?$AAr?$AAe?$AAe?$AA?$DM?$AAc?$AAl?$AAa?$AAs?$AAs?$AA?5?$AAs?$AAt?$AAd?$AA?3?$AA?3?$AA_?$AAT?$AAm?$AAa?$AAp?$AA_?$AAt?$AAr?$AAa?$AAi@ 1017fb60     ambientsnd.obj
 0003:00004cc8       ??_C@_1BGA@CHDMOGFE@?$AAs?$AAt?$AAd?$AA?3?$AA?3?$AA_?$AAT?$AAr?$AAe?$AAe?$AA?$DM?$AAc?$AAl?$AAa?$AAs?$AAs?$AA?5?$AAs?$AAt?$AAd?$AA?3?$AA?3?$AA_?$AAT?$AAm?$AAa?$AAp?$AA_?$AAt?$AAr?$AAa?$AAi@ 1017fcc8     ambientsnd.obj
 0003:00004e70       ??_C@_1BGA@NGPOADEG@?$AAs?$AAt?$AAd?$AA?3?$AA?3?$AA_?$AAT?$AAr?$AAe?$AAe?$AA?$DM?$AAc?$AAl?$AAa?$AAs?$AAs?$AA?5?$AAs?$AAt?$AAd?$AA?3?$AA?3?$AA_?$AAT?$AAm?$AAa?$AAp?$AA_?$AAt?$AAr?$AAa?$AAi@ 1017fe70     ambientsnd.obj
 0003:00005100       ??_C@_1BFI@HDHNNGBO@?$AAs?$AAt?$AAd?$AA?3?$AA?3?$AA_?$AAT?$AAr?$AAe?$AAe?$AA?$DM?$AAc?$AAl?$AAa?$AAs?$AAs?$AA?5?$AAs?$AAt?$AAd?$AA?3?$AA?3?$AA_?$AAT?$AAm?$AAa?$AAp?$AA_?$AAt?$AAr?$AAa?$AAi@ 10180100     gamesnd.obj
 0003:000058cc       ?collate@?$_Locbase@H@std@@2HB 101808cc     scriptparser.obj
 0003:000058d0       ?ctype@?$_Locbase@H@std@@2HB 101808d0     scriptparser.obj
 0003:000058d4       ?monetary@?$_Locbase@H@std@@2HB 101808d4     scriptparser.obj
 0003:000058d8       ?numeric@?$_Locbase@H@std@@2HB 101808d8     scriptparser.obj
 0003:000058dc       ?time@?$_Locbase@H@std@@2HB 101808dc     scriptparser.obj
 0003:000058e0       ?messages@?$_Locbase@H@std@@2HB 101808e0     scriptparser.obj
 0003:000058e4       ?all@?$_Locbase@H@std@@2HB 101808e4     scriptparser.obj
 0003:000058e8       ?none@?$_Locbase@H@std@@2HB 101808e8     scriptparser.obj
 0003:000058ec       ?table_size@?$ctype@D@std@@2IB 101808ec     scriptparser.obj
 0003:000058f0       ?skipws@?$_Iosb@H@std@@2W4_Fmtflags@12@B 101808f0     scriptparser.obj
 0003:000058f4       ?unitbuf@?$_Iosb@H@std@@2W4_Fmtflags@12@B 101808f4     scriptparser.obj
 0003:000058f8       ?uppercase@?$_Iosb@H@std@@2W4_Fmtflags@12@B 101808f8     scriptparser.obj
 0003:000058fc       ?showbase@?$_Iosb@H@std@@2W4_Fmtflags@12@B 101808fc     scriptparser.obj
 0003:00005900       ?showpoint@?$_Iosb@H@std@@2W4_Fmtflags@12@B 10180900     scriptparser.obj
 0003:00005904       ?showpos@?$_Iosb@H@std@@2W4_Fmtflags@12@B 10180904     scriptparser.obj
 0003:00005908       ?left@?$_Iosb@H@std@@2W4_Fmtflags@12@B 10180908     scriptparser.obj
 0003:0000590c       ?right@?$_Iosb@H@std@@2W4_Fmtflags@12@B 1018090c     scriptparser.obj
 0003:00005910       ?internal@?$_Iosb@H@std@@2W4_Fmtflags@12@B 10180910     scriptparser.obj
 0003:00005914       ?dec@?$_Iosb@H@std@@2W4_Fmtflags@12@B 10180914     scriptparser.obj
 0003:00005918       ?oct@?$_Iosb@H@std@@2W4_Fmtflags@12@B 10180918     scriptparser.obj
 0003:0000591c       ?hex@?$_Iosb@H@std@@2W4_Fmtflags@12@B 1018091c     scriptparser.obj
 0003:00005920       ?scientific@?$_Iosb@H@std@@2W4_Fmtflags@12@B 10180920     scriptparser.obj
 0003:00005924       ?fixed@?$_Iosb@H@std@@2W4_Fmtflags@12@B 10180924     scriptparser.obj
 0003:00005928       ?hexfloat@?$_Iosb@H@std@@2W4_Fmtflags@12@B 10180928     scriptparser.obj
 0003:0000592c       ?boolalpha@?$_Iosb@H@std@@2W4_Fmtflags@12@B 1018092c     scriptparser.obj
 0003:00005930       ?_Stdio@?$_Iosb@H@std@@2W4_Fmtflags@12@B 10180930     scriptparser.obj
 0003:00005934       ?adjustfield@?$_Iosb@H@std@@2W4_Fmtflags@12@B 10180934     scriptparser.obj
 0003:00005938       ?basefield@?$_Iosb@H@std@@2W4_Fmtflags@12@B 10180938     scriptparser.obj
 0003:0000593c       ?floatfield@?$_Iosb@H@std@@2W4_Fmtflags@12@B 1018093c     scriptparser.obj
 0003:00005940       ?goodbit@?$_Iosb@H@std@@2W4_Iostate@12@B 10180940     scriptparser.obj
 0003:00005944       ?eofbit@?$_Iosb@H@std@@2W4_Iostate@12@B 10180944     scriptparser.obj
 0003:00005948       ?failbit@?$_Iosb@H@std@@2W4_Iostate@12@B 10180948     scriptparser.obj
 0003:0000594c       ?badbit@?$_Iosb@H@std@@2W4_Iostate@12@B 1018094c     scriptparser.obj
 0003:00005950       ?_Hardfail@?$_Iosb@H@std@@2W4_Iostate@12@B 10180950     scriptparser.obj
 0003:00005954       ?in@?$_Iosb@H@std@@2W4_Openmode@12@B 10180954     scriptparser.obj
 0003:00005958       ?out@?$_Iosb@H@std@@2W4_Openmode@12@B 10180958     scriptparser.obj
 0003:0000595c       ?ate@?$_Iosb@H@std@@2W4_Openmode@12@B 1018095c     scriptparser.obj
 0003:00005960       ?app@?$_Iosb@H@std@@2W4_Openmode@12@B 10180960     scriptparser.obj
 0003:00005964       ?trunc@?$_Iosb@H@std@@2W4_Openmode@12@B 10180964     scriptparser.obj
 0003:00005968       ?_Nocreate@?$_Iosb@H@std@@2W4_Openmode@12@B 10180968     scriptparser.obj
 0003:0000596c       ?_Noreplace@?$_Iosb@H@std@@2W4_Openmode@12@B 1018096c     scriptparser.obj
 0003:00005970       ?binary@?$_Iosb@H@std@@2W4_Openmode@12@B 10180970     scriptparser.obj
 0003:00005974       ?beg@?$_Iosb@H@std@@2W4_Seekdir@12@B 10180974     scriptparser.obj
 0003:00005978       ?cur@?$_Iosb@H@std@@2W4_Seekdir@12@B 10180978     scriptparser.obj
 0003:0000597c       ?end@?$_Iosb@H@std@@2W4_Seekdir@12@B 1018097c     scriptparser.obj
 0003:00005980       ??_C@_0DP@CCOAGOA@C?3?2Program?5Files?2Microsoft?5Visua@ 10180980     scriptparser.obj
 0003:000059cc       ??_C@_1CK@POGJDOKA@?$AA?$CI?$AA?$CC?$AA_?$AAP?$AAo?$AAs?$AA?5?$AA?$DM?$AA?5?$AAs?$AAi?$AAz?$AAe?$AA?$CI?$AA?$CJ?$AA?$CC?$AA?0?$AA?5?$AA0?$AA?$CJ?$AA?$AA@ 101809cc     scriptparser.obj
 0003:00005a00       ??_C@_1BME@NCIPHHDN@?$AAs?$AAt?$AAd?$AA?3?$AA?3?$AAv?$AAe?$AAc?$AAt?$AAo?$AAr?$AA?$DM?$AAc?$AAl?$AAa?$AAs?$AAs?$AA?5?$AAs?$AAt?$AAd?$AA?3?$AA?3?$AAb?$AAa?$AAs?$AAi?$AAc?$AA_?$AAs?$AAt?$AAr@ 10180a00     scriptparser.obj
 0003:00005c20       ??_C@_1DM@LHGCHCBA@?$AAv?$AAe?$AAc?$AAt?$AAo?$AAr?$AA?5?$AAs?$AAu?$AAb?$AAs?$AAc?$AAr?$AAi?$AAp?$AAt?$AA?5?$AAo?$AAu?$AAt?$AA?5?$AAo?$AAf?$AA?5?$AAr?$AAa?$AAn?$AAg?$AAe?$AA?$AA@ 10180c20     scriptparser.obj
 0003:00005c68       ??_C@_1HO@BGIAGONF@?$AAC?$AA?3?$AA?2?$AAP?$AAr?$AAo?$AAg?$AAr?$AAa?$AAm?$AA?5?$AAF?$AAi?$AAl?$AAe?$AAs?$AA?2?$AAM?$AAi?$AAc?$AAr?$AAo?$AAs?$AAo?$AAf?$AAt?$AA?5?$AAV?$AAi?$AAs?$AAu?$AAa@ 10180c68     scriptparser.obj
 0003:00005d00       ??_C@_1KC@BEMHKPAD@?$AAs?$AAt?$AAd?$AA?3?$AA?3?$AAv?$AAe?$AAc?$AAt?$AAo?$AAr?$AA?$DM?$AAs?$AAt?$AAr?$AAu?$AAc?$AAt?$AA?5?$AAS?$AAT?$AA_?$AAC?$AAE?$AAL?$AAL?$AAS?$AA?0?$AAc?$AAl?$AAa?$AAs@ 10180d00     scriptparser.obj
 0003:00005dc4       ??_C@_0BD@OLBABOEK@vector?$DMT?$DO?5too?5long?$AA@ 10180dc4     scriptparser.obj
 0003:00005de0       ??_C@_1BFI@ICLPDDAM@?$AAs?$AAt?$AAd?$AA?3?$AA?3?$AA_?$AAT?$AAr?$AAe?$AAe?$AA?$DM?$AAc?$AAl?$AAa?$AAs?$AAs?$AA?5?$AAs?$AAt?$AAd?$AA?3?$AA?3?$AA_?$AAT?$AAm?$AAa?$AAp?$AA_?$AAt?$AAr?$AAa?$AAi@ 10180de0     scriptparser.obj
 0003:00005f80       ??_C@_1BGG@JAMMBCCO@?$AAs?$AAt?$AAd?$AA?3?$AA?3?$AA_?$AAT?$AAr?$AAe?$AAe?$AA?$DM?$AAc?$AAl?$AAa?$AAs?$AAs?$AA?5?$AAs?$AAt?$AAd?$AA?3?$AA?3?$AA_?$AAT?$AAm?$AAa?$AAp?$AA_?$AAt?$AAr?$AAa?$AAi@ 10180f80     scriptparser.obj
 0003:00006130       ??_C@_1BFI@GIGMDBID@?$AAs?$AAt?$AAd?$AA?3?$AA?3?$AA_?$AAT?$AAr?$AAe?$AAe?$AA?$DM?$AAc?$AAl?$AAa?$AAs?$AAs?$AA?5?$AAs?$AAt?$AAd?$AA?3?$AA?3?$AA_?$AAT?$AAm?$AAa?$AAp?$AA_?$AAt?$AAr?$AAa?$AAi@ 10181130     scriptparser.obj
 0003:00006700       __real@40dfffc000000000    10181700     floating.obj
 0003:00006780       __real@400921fb60000000    10181780     vecmat.obj
 0003:0000678c       __real@bfc90fdb            1018178c     vecmat.obj
 0003:00006790       __real@3fc90fdb            10181790     vecmat.obj
 0003:00006798       __real@3fd5555560000000    10181798     vecmat.obj
 0003:000067a8       __real@3fd0000000000000    101817a8     vecmat.obj
 0003:000067b8       __real@3fc0000000000000    101817b8     vecmat.obj
 0003:000067c8       __real@3f1a36e2eb1c432d    101817c8     vecmat.obj
 0003:000067d4       __real@42c80000            101817d4     vecmat.obj
 0003:000067d8       __real@3f847ae140000000    101817d8     vecmat.obj
 0003:000067e4       __real@461c3f9a            101817e4     vecmat.obj
 0003:000067e8       __real@3f747ae140000000    101817e8     vecmat.obj
 0003:000067f8       __real@3ea0c6f7a0000000    101817f8     vecmat.obj
 0003:00006808       __real@401921fb60000000    10181808     vecmat.obj
 0003:00006814       __real@40490fdb            10181814     vecmat.obj
 0003:00006818       __real@bfefffffc0000000    10181818     vecmat.obj
 0003:00006828       __real@3fefffffc0000000    10181828     vecmat.obj
 0003:00006838       __real@3ffe666660000000    10181838     vecmat.obj
 0003:00006848       __real@3ff0ccccc0000000    10181848     vecmat.obj
 0003:00006858       __real@4000ccccc0000000    10181858     vecmat.obj
 0003:00006868       __real@3ee4f8b588e368f1    10181868     vecmat.obj
 0003:00006878       __real@3e7ad7f29abcaf48    10181878     vecmat.obj
 0003:00006888       __real@4010000000000000    10181888     vecmat.obj
 0003:00006898       __real@3ee4f8b580000000    10181898     vecmat.obj
 0003:000068a8       __real@3bc79ca10c924223    101818a8     vecmat.obj
 0003:000068b8       __real@3f91df3300000000    101818b8     vecmat.obj
 0003:000068c8       __real@3f50624de0000000    101818c8     vecmat.obj
 0003:000068d4       __real@3f000000            101818d4     vecmat.obj
 0003:000068d8       __real@ccbebc20            101818d8     vecmat.obj
 0003:000068dc       __real@4cbebc20            101818dc     vecmat.obj
 0003:000068e0       __real@4066800000000000    101818e0     vecmat.obj
 0003:000068f0       __real@400921fa00000000    101818f0     vecmat.obj
 0003:000068fc       __real@43b38000            101818fc     vecmat.obj
 0003:00006c20       ??_C@_1EK@EEHFMKDC@?$AAv?$AAe?$AAc?$AAt?$AAo?$AAr?$AA?5?$AAi?$AAn?$AAs?$AAe?$AAr?$AAt?$AA?5?$AAi?$AAt?$AAe?$AAr?$AAa?$AAt?$AAo?$AAr?$AA?5?$AAo?$AAu?$AAt?$AAs?$AAi?$AAd?$AAe?$AA?5?$AAr@ 10181c20     xls.obj
 0003:00006c78       ??_C@_1BPK@MNCDPEOO@?$AAs?$AAt?$AAd?$AA?3?$AA?3?$AA_?$AAV?$AAe?$AAc?$AAt?$AAo?$AAr?$AA_?$AAc?$AAo?$AAn?$AAs?$AAt?$AA_?$AAi?$AAt?$AAe?$AAr?$AAa?$AAt?$AAo?$AAr?$AA?$DM?$AAc?$AAl?$AAa?$AAs@ 10181c78     xls.obj
 0003:00006ed8       ??_C@_1NK@JLHOCNGO@?$AA?$CI?$AA?$CC?$AA_?$AAP?$AAv?$AAe?$AAc?$AAt?$AAo?$AAr?$AA?5?$AA?$DN?$AA?$DN?$AA?5?$AAN?$AAU?$AAL?$AAL?$AA?5?$AA?$HM?$AA?$HM?$AA?5?$AA?$CI?$AA?$CI?$AA?$CI?$AA_?$AAM?$AAy?$AAv?$AAe?$AAc?$AA?5@ 10181ed8     xls.obj
 0003:00006fe0       ??_C@_1BNM@BEDNJHNI@?$AAs?$AAt?$AAd?$AA?3?$AA?3?$AA_?$AAV?$AAe?$AAc?$AAt?$AAo?$AAr?$AA_?$AAc?$AAo?$AAn?$AAs?$AAt?$AA_?$AAi?$AAt?$AAe?$AAr?$AAa?$AAt?$AAo?$AAr?$AA?$DM?$AAc?$AAl?$AAa?$AAs@ 10181fe0     xls.obj
 0003:0000721c       ??_C@_1DM@HINDPMBP@?$AAv?$AAe?$AAc?$AAt?$AAo?$AAr?$AA?5?$AAi?$AAt?$AAe?$AAr?$AAa?$AAt?$AAo?$AAr?$AAs?$AA?5?$AAi?$AAn?$AAc?$AAo?$AAm?$AAp?$AAa?$AAt?$AAi?$AAb?$AAl?$AAe?$AA?$AA@ 1018221c     xls.obj
 0003:00007268       ??_C@_1NI@MIONKKKL@?$AAs?$AAt?$AAd?$AA?3?$AA?3?$AA_?$AAV?$AAe?$AAc?$AAt?$AAo?$AAr?$AA_?$AAc?$AAo?$AAn?$AAs?$AAt?$AA_?$AAi?$AAt?$AAe?$AAr?$AAa?$AAt?$AAo?$AAr?$AA?$DM?$AAs?$AAt?$AAr?$AAu@ 10182268     xls.obj
 0003:00007370       ??_C@_1LK@PCHKJENF@?$AAs?$AAt?$AAd?$AA?3?$AA?3?$AA_?$AAV?$AAe?$AAc?$AAt?$AAo?$AAr?$AA_?$AAc?$AAo?$AAn?$AAs?$AAt?$AA_?$AAi?$AAt?$AAe?$AAr?$AAa?$AAt?$AAo?$AAr?$AA?$DM?$AAs?$AAt?$AAr?$AAu@ 10182370     xls.obj
 0003:00007450       ??_C@_1BAC@KBDNDJPK@?$AA?$CI?$AA?$CC?$AA_?$AAM?$AAy?$AAp?$AAt?$AAr?$AA?5?$AA?$CL?$AA?5?$AA_?$AAO?$AAf?$AAf?$AA?5?$AA?$DM?$AA?$DN?$AA?5?$AA?$CI?$AA?$CI?$AA_?$AAM?$AAy?$AAv?$AAe?$AAc?$AA?5?$AA?$CK?$AA?$CJ?$AA?$CI?$AAt@ 10182450     xls.obj
 0003:00007588       ??_C@_1BOE@HHEDPKGH@?$AAs?$AAt?$AAd?$AA?3?$AA?3?$AA_?$AAV?$AAe?$AAc?$AAt?$AAo?$AAr?$AA_?$AAc?$AAo?$AAn?$AAs?$AAt?$AA_?$AAi?$AAt?$AAe?$AAr?$AAa?$AAt?$AAo?$AAr?$AA?$DM?$AAc?$AAl?$AAa?$AAs@ 10182588     xls.obj
 0003:000077cc       ??_C@_1DM@LBMEEJPP@?$AA?$CI?$AA?$CC?$AAt?$AAh?$AAi?$AAs?$AA?9?$AA?$DO?$AA_?$AAH?$AAa?$AAs?$AA_?$AAc?$AAo?$AAn?$AAt?$AAa?$AAi?$AAn?$AAe?$AAr?$AA?$CI?$AA?$CJ?$AA?$CC?$AA?0?$AA?5?$AA0?$AA?$CJ?$AA?$AA@ 101827cc     xls.obj
 0003:00007818       ??_C@_1MC@GIGHPNIA@?$AAs?$AAt?$AAd?$AA?3?$AA?3?$AA_?$AAV?$AAe?$AAc?$AAt?$AAo?$AAr?$AA_?$AAc?$AAo?$AAn?$AAs?$AAt?$AA_?$AAi?$AAt?$AAe?$AAr?$AAa?$AAt?$AAo?$AAr?$AA?$DM?$AAs?$AAt?$AAr?$AAu@ 10182818     xls.obj
 0003:00007900       ??_C@_1EI@HGIDLLCM@?$AAv?$AAe?$AAc?$AAt?$AAo?$AAr?$AA?5?$AAe?$AAr?$AAa?$AAs?$AAe?$AA?5?$AAi?$AAt?$AAe?$AAr?$AAa?$AAt?$AAo?$AAr?$AA?5?$AAo?$AAu?$AAt?$AAs?$AAi?$AAd?$AAe?$AA?5?$AAr?$AAa@ 10182900     xls.obj
 0003:00007958       ??_C@_1HO@GIFLOCNO@?$AAC?$AA?3?$AA?2?$AAP?$AAr?$AAo?$AAg?$AAr?$AAa?$AAm?$AA?5?$AAF?$AAi?$AAl?$AAe?$AAs?$AA?2?$AAM?$AAi?$AAc?$AAr?$AAo?$AAs?$AAo?$AAf?$AAt?$AA?5?$AAV?$AAi?$AAs?$AAu?$AAa@ 10182958     xls.obj
 0003:000079f0       ??_C@_1BOC@BMIIFNLH@?$AAs?$AAt?$AAd?$AA?3?$AA?3?$AA_?$AAV?$AAe?$AAc?$AAt?$AAo?$AAr?$AA_?$AAc?$AAo?$AAn?$AAs?$AAt?$AA_?$AAi?$AAt?$AAe?$AAr?$AAa?$AAt?$AAo?$AAr?$AA?$DM?$AAc?$AAl?$AAa?$AAs@ 101829f0     xls.obj
 0003:00007c38       ??_C@_1EG@FOHJJHAC@?$AAv?$AAe?$AAc?$AAt?$AAo?$AAr?$AA?5?$AAi?$AAt?$AAe?$AAr?$AAa?$AAt?$AAo?$AAr?$AA?5?$AAn?$AAo?$AAt?$AA?5?$AAd?$AAe?$AAr?$AAe?$AAf?$AAe?$AAr?$AAe?$AAn?$AAc?$AAa?$AAb@ 10182c38     xls.obj
 0003:00007c90       ??_C@_1EE@EJDKCLKB@?$AAv?$AAe?$AAc?$AAt?$AAo?$AAr?$AA?5?$AAi?$AAt?$AAe?$AAr?$AAa?$AAt?$AAo?$AAr?$AA?5?$AAn?$AAo?$AAt?$AA?5?$AAi?$AAn?$AAc?$AAr?$AAe?$AAm?$AAe?$AAn?$AAt?$AAa?$AAb?$AAl@ 10182c90     xls.obj
 0003:00007ce8       ??_C@_1HE@NMBDDEHP@?$AA?$CI?$AA?$CC?$AA_?$AAM?$AAy?$AAp?$AAt?$AAr?$AA?5?$AA?$DM?$AA?5?$AA?$CI?$AA?$CI?$AA_?$AAM?$AAy?$AAv?$AAe?$AAc?$AA?5?$AA?$CK?$AA?$CJ?$AA?$CI?$AAt?$AAh?$AAi?$AAs?$AA?9?$AA?$DO?$AA_?$AAG?$AAe@ 10182ce8     xls.obj
 0003:00007d78       ??_C@_1BOE@CDBPCCE@?$AAs?$AAt?$AAd?$AA?3?$AA?3?$AA_?$AAV?$AAe?$AAc?$AAt?$AAo?$AAr?$AA_?$AAc?$AAo?$AAn?$AAs?$AAt?$AA_?$AAi?$AAt?$AAe?$AAr?$AAa?$AAt?$AAo?$AAr?$AA?$DM?$AAc?$AAl?$AAa?$AAs@ 10182d78     xls.obj
 0003:00007fbc       ??_C@_1CO@DGLIKNHI@?$AAi?$AAn?$AAv?$AAa?$AAl?$AAi?$AAd?$AA?5?$AAi?$AAt?$AAe?$AAr?$AAa?$AAt?$AAo?$AAr?$AA?5?$AAr?$AAa?$AAn?$AAg?$AAe?$AA?$AA@ 10182fbc     xls.obj
 0003:0000b360       __real@40400000            10186360     wzSound.obj
 0003:0000b364       _GUID_NULL                 10186364     uuid:cguid_i.obj
 0003:0000b374       _CATID_MARSHALER           10186374     uuid:cguid_i.obj
 0003:0000b384       _IID_IRpcChannel           10186384     uuid:cguid_i.obj
 0003:0000b394       _IID_IRpcStub              10186394     uuid:cguid_i.obj
 0003:0000b3a4       _IID_IStubManager          101863a4     uuid:cguid_i.obj
 0003:0000b3b4       _IID_IRpcProxy             101863b4     uuid:cguid_i.obj
 0003:0000b3c4       _IID_IProxyManager         101863c4     uuid:cguid_i.obj
 0003:0000b3d4       _IID_IPSFactory            101863d4     uuid:cguid_i.obj
 0003:0000b3e4       _IID_IInternalMoniker      101863e4     uuid:cguid_i.obj
 0003:0000b3f4       _IID_IDfReserved1          101863f4     uuid:cguid_i.obj
 0003:0000b404       _IID_IDfReserved2          10186404     uuid:cguid_i.obj
 0003:0000b414       _IID_IDfReserved3          10186414     uuid:cguid_i.obj
 0003:0000b424       _CLSID_StdMarshal          10186424     uuid:cguid_i.obj
 0003:0000b434       _IID_IStub                 10186434     uuid:cguid_i.obj
 0003:0000b444       _IID_IProxy                10186444     uuid:cguid_i.obj
 0003:0000b454       _IID_IEnumGeneric          10186454     uuid:cguid_i.obj
 0003:0000b464       _IID_IEnumHolder           10186464     uuid:cguid_i.obj
 0003:0000b474       _IID_IEnumCallback         10186474     uuid:cguid_i.obj
 0003:0000b484       _IID_IOleManager           10186484     uuid:cguid_i.obj
 0003:0000b494       _IID_IOlePresObj           10186494     uuid:cguid_i.obj
 0003:0000b4a4       _IID_IDebug                101864a4     uuid:cguid_i.obj
 0003:0000b4b4       _IID_IDebugStream          101864b4     uuid:cguid_i.obj
 0003:0000b4c4       _CLSID_PSGenObject         101864c4     uuid:cguid_i.obj
 0003:0000b4d4       _CLSID_PSClientSite        101864d4     uuid:cguid_i.obj
 0003:0000b4e4       _CLSID_PSClassObject       101864e4     uuid:cguid_i.obj
 0003:0000b4f4       _CLSID_PSInPlaceActive     101864f4     uuid:cguid_i.obj
 0003:0000b504       _CLSID_PSInPlaceFrame      10186504     uuid:cguid_i.obj
 0003:0000b514       _CLSID_PSDragDrop          10186514     uuid:cguid_i.obj
 0003:0000b524       _CLSID_PSBindCtx           10186524     uuid:cguid_i.obj
 0003:0000b534       _CLSID_PSEnumerators       10186534     uuid:cguid_i.obj
 0003:0000b544       _CLSID_StaticMetafile      10186544     uuid:cguid_i.obj
 0003:0000b554       _CLSID_StaticDib           10186554     uuid:cguid_i.obj
 0003:0000b564       _CLSID_Picture_Metafile    10186564     uuid:cguid_i.obj
 0003:0000b574       _CLSID_Picture_EnhMetafile 10186574     uuid:cguid_i.obj
 0003:0000b584       _CLSID_Picture_Dib         10186584     uuid:cguid_i.obj
 0003:0000b594       _CLSID_DCOMAccessControl   10186594     uuid:cguid_i.obj
 0003:0000b5a4       _CLSID_StdGlobalInterfaceTable 101865a4     uuid:cguid_i.obj
 0003:0000b5b4       _CLSID_ManualResetEvent    101865b4     uuid:cguid_i.obj
 0003:0000b5c4       _CLSID_StdEvent            101865c4     uuid:cguid_i.obj
 0003:0000b5d4       _CLSID_SynchronizeContainer 101865d4     uuid:cguid_i.obj
 0003:0000b5e4       _CLSID_ComBinding          101865e4     uuid:cguid_i.obj
 0003:0000b5f4       _CLSID_StdAsyncActManager  101865f4     uuid:cguid_i.obj
 0003:0000b604       _CLSID_InProcFreeMarshaler 10186604     uuid:cguid_i.obj
 0003:0000b614       _CLSID_RemoteUnknownPSFactory 10186614     uuid:cguid_i.obj
 0003:0000b624       _IID_IRichEditOle          10186624     uuid:cguid_i.obj
 0003:0000b634       _IID_IRichEditOleCallback  10186634     uuid:cguid_i.obj
 0003:0000b644       _CLSID_AllClasses          10186644     uuid:cguid_i.obj
 0003:0000b654       _CLSID_LocalMachineClasses 10186654     uuid:cguid_i.obj
 0003:0000b664       _CLSID_CurrentUserClasses  10186664     uuid:cguid_i.obj
 0003:0000b674       _CLSID_AddrControl         10186674     uuid:cguid_i.obj
 0003:0000b684       _CLSID_GlobalOptions       10186684     uuid:cguid_i.obj
 0003:0000b694       _CLSID_SurrogateManager    10186694     uuid:cguid_i.obj
 0003:0000b6a4       _CLSID_ContextSwitcher     101866a4     uuid:cguid_i.obj
 0003:0000b6b4       _IID_IPropertyFrame        101866b4     uuid:cguid_i.obj
 0003:0000b6c4       _CLSID_CFontPropPage       101866c4     uuid:cguid_i.obj
 0003:0000b6d4       _CLSID_CColorPropPage      101866d4     uuid:cguid_i.obj
 0003:0000b6e4       _CLSID_CPicturePropPage    101866e4     uuid:cguid_i.obj
 0003:0000b6f4       _CLSID_StockFontPage       101866f4     uuid:cguid_i.obj
 0003:0000b704       _CLSID_StockColorPage      10186704     uuid:cguid_i.obj
 0003:0000b714       _CLSID_StockPicturePage    10186714     uuid:cguid_i.obj
 0003:0000b724       _CLSID_PersistPropset      10186724     uuid:cguid_i.obj
 0003:0000b734       _CLSID_ConvertVBX          10186734     uuid:cguid_i.obj
 0003:0000b744       _CLSID_StdFont             10186744     uuid:cguid_i.obj
 0003:0000b754       _CLSID_StdPicture          10186754     uuid:cguid_i.obj
 0003:0000b764       _GUID_HIMETRIC             10186764     uuid:cguid_i.obj
 0003:0000b774       _GUID_COLOR                10186774     uuid:cguid_i.obj
 0003:0000b784       _GUID_XPOSPIXEL            10186784     uuid:cguid_i.obj
 0003:0000b794       _GUID_YPOSPIXEL            10186794     uuid:cguid_i.obj
 0003:0000b7a4       _GUID_XSIZEPIXEL           101867a4     uuid:cguid_i.obj
 0003:0000b7b4       _GUID_YSIZEPIXEL           101867b4     uuid:cguid_i.obj
 0003:0000b7c4       _GUID_XPOS                 101867c4     uuid:cguid_i.obj
 0003:0000b7d4       _GUID_YPOS                 101867d4     uuid:cguid_i.obj
 0003:0000b7e4       _GUID_XSIZE                101867e4     uuid:cguid_i.obj
 0003:0000b7f4       _GUID_YSIZE                101867f4     uuid:cguid_i.obj
 0003:0000b804       _GUID_TRISTATE             10186804     uuid:cguid_i.obj
 0003:0000b814       _GUID_OPTIONVALUEEXCLUSIVE 10186814     uuid:cguid_i.obj
 0003:0000b824       _GUID_CHECKVALUEEXCLUSIVE  10186824     uuid:cguid_i.obj
 0003:0000b834       _GUID_FONTNAME             10186834     uuid:cguid_i.obj
 0003:0000b844       _GUID_FONTSIZE             10186844     uuid:cguid_i.obj
 0003:0000b854       _GUID_FONTBOLD             10186854     uuid:cguid_i.obj
 0003:0000b864       _GUID_FONTITALIC           10186864     uuid:cguid_i.obj
 0003:0000b874       _GUID_FONTUNDERSCORE       10186874     uuid:cguid_i.obj
 0003:0000b884       _GUID_FONTSTRIKETHROUGH    10186884     uuid:cguid_i.obj
 0003:0000b894       _GUID_HANDLE               10186894     uuid:cguid_i.obj
 0003:0000b8a4       _IID_StdOle                101868a4     uuid:cguid_i.obj
 0003:0000b8b4       _IID_ICursor               101868b4     uuid:cguid_i.obj
 0003:0000b8c4       _IID_ICursorMove           101868c4     uuid:cguid_i.obj
 0003:0000b8d4       _IID_ICursorScroll         101868d4     uuid:cguid_i.obj
 0003:0000b8e4       _IID_ICursorUpdateARow     101868e4     uuid:cguid_i.obj
 0003:0000b8f4       _IID_INotifyDBEvents       101868f4     uuid:cguid_i.obj
 0003:0000b904       _IID_ICursorFind           10186904     uuid:cguid_i.obj
 0003:0000b914       _IID_IEntryID              10186914     uuid:cguid_i.obj
 0003:0000b924       __GUID_NAMEONLY            10186924     uuid:cguid_i.obj
 0003:0000b934       __DBBMKGUID                10186934     uuid:cguid_i.obj
 0003:0000b944       __DBCIDGUID                10186944     uuid:cguid_i.obj
 0003:0000b954       _IID_IBoundObject          10186954     uuid:cguid_i.obj
 0003:0000b964       _IID_IBoundObjectSite      10186964     uuid:cguid_i.obj
 0003:0000b974       _CLSID_GblComponentCategoriesMgr 10186974     uuid:cguid_i.obj
 0003:0000b984       _CLSID_ThumbnailFCNHandler 10186984     uuid:cguid_i.obj
 0003:0000b994       _CLSID_ThumbnailUpdater    10186994     uuid:cguid_i.obj
 0003:0000b9a4       _GUID_DEVCLASS_1394        101869a4     uuid:cguid_i.obj
 0003:0000b9b4       _GUID_DEVCLASS_1394DEBUG   101869b4     uuid:cguid_i.obj
 0003:0000b9c4       _GUID_DEVCLASS_61883       101869c4     uuid:cguid_i.obj
 0003:0000b9d4       _GUID_DEVCLASS_ADAPTER     101869d4     uuid:cguid_i.obj
 0003:0000b9e4       _GUID_DEVCLASS_APMSUPPORT  101869e4     uuid:cguid_i.obj
 0003:0000b9f4       _GUID_DEVCLASS_AVC         101869f4     uuid:cguid_i.obj
 0003:0000ba04       _GUID_DEVCLASS_BATTERY     10186a04     uuid:cguid_i.obj
 0003:0000ba14       _GUID_DEVCLASS_BIOMETRIC   10186a14     uuid:cguid_i.obj
 0003:0000ba24       _GUID_DEVCLASS_BLUETOOTH   10186a24     uuid:cguid_i.obj
 0003:0000ba34       _GUID_DEVCLASS_CDROM       10186a34     uuid:cguid_i.obj
 0003:0000ba44       _GUID_DEVCLASS_COMPUTER    10186a44     uuid:cguid_i.obj
 0003:0000ba54       _GUID_DEVCLASS_DECODER     10186a54     uuid:cguid_i.obj
 0003:0000ba64       _GUID_DEVCLASS_DISKDRIVE   10186a64     uuid:cguid_i.obj
 0003:0000ba74       _GUID_DEVCLASS_DISPLAY     10186a74     uuid:cguid_i.obj
 0003:0000ba84       _GUID_DEVCLASS_DOT4        10186a84     uuid:cguid_i.obj
 0003:0000ba94       _GUID_DEVCLASS_DOT4PRINT   10186a94     uuid:cguid_i.obj
 0003:0000baa4       _GUID_DEVCLASS_ENUM1394    10186aa4     uuid:cguid_i.obj
 0003:0000bab4       _GUID_DEVCLASS_FDC         10186ab4     uuid:cguid_i.obj
 0003:0000bac4       _GUID_DEVCLASS_FLOPPYDISK  10186ac4     uuid:cguid_i.obj
 0003:0000bad4       _GUID_DEVCLASS_GPS         10186ad4     uuid:cguid_i.obj
 0003:0000bae4       _GUID_DEVCLASS_HDC         10186ae4     uuid:cguid_i.obj
 0003:0000baf4       _GUID_DEVCLASS_HIDCLASS    10186af4     uuid:cguid_i.obj
 0003:0000bb04       _GUID_DEVCLASS_IMAGE       10186b04     uuid:cguid_i.obj
 0003:0000bb14       _GUID_DEVCLASS_INFINIBAND  10186b14     uuid:cguid_i.obj
 0003:0000bb24       _GUID_DEVCLASS_INFRARED    10186b24     uuid:cguid_i.obj
 0003:0000bb34       _GUID_DEVCLASS_KEYBOARD    10186b34     uuid:cguid_i.obj
 0003:0000bb44       _GUID_DEVCLASS_LEGACYDRIVER 10186b44     uuid:cguid_i.obj
 0003:0000bb54       _GUID_DEVCLASS_MEDIA       10186b54     uuid:cguid_i.obj
 0003:0000bb64       _GUID_DEVCLASS_MEDIUM_CHANGER 10186b64     uuid:cguid_i.obj
 0003:0000bb74       _GUID_DEVCLASS_MODEM       10186b74     uuid:cguid_i.obj
 0003:0000bb84       _GUID_DEVCLASS_MONITOR     10186b84     uuid:cguid_i.obj
 0003:0000bb94       _GUID_DEVCLASS_MOUSE       10186b94     uuid:cguid_i.obj
 0003:0000bba4       _GUID_DEVCLASS_MTD         10186ba4     uuid:cguid_i.obj
 0003:0000bbb4       _GUID_DEVCLASS_MULTIFUNCTION 10186bb4     uuid:cguid_i.obj
 0003:0000bbc4       _GUID_DEVCLASS_MULTIPORTSERIAL 10186bc4     uuid:cguid_i.obj
 0003:0000bbd4       _GUID_DEVCLASS_NET         10186bd4     uuid:cguid_i.obj
 0003:0000bbe4       _GUID_DEVCLASS_NETCLIENT   10186be4     uuid:cguid_i.obj
 0003:0000bbf4       _GUID_DEVCLASS_NETSERVICE  10186bf4     uuid:cguid_i.obj
 0003:0000bc04       _GUID_DEVCLASS_NETTRANS    10186c04     uuid:cguid_i.obj
 0003:0000bc14       _GUID_DEVCLASS_NODRIVER    10186c14     uuid:cguid_i.obj
 0003:0000bc24       _GUID_DEVCLASS_PCMCIA      10186c24     uuid:cguid_i.obj
 0003:0000bc34       _GUID_DEVCLASS_PNPPRINTERS 10186c34     uuid:cguid_i.obj
 0003:0000bc44       _GUID_DEVCLASS_PORTS       10186c44     uuid:cguid_i.obj
 0003:0000bc54       _GUID_DEVCLASS_PRINTER     10186c54     uuid:cguid_i.obj
 0003:0000bc64       _GUID_DEVCLASS_PRINTERUPGRADE 10186c64     uuid:cguid_i.obj
 0003:0000bc74       _GUID_DEVCLASS_PROCESSOR   10186c74     uuid:cguid_i.obj
 0003:0000bc84       _GUID_DEVCLASS_SBP2        10186c84     uuid:cguid_i.obj
 0003:0000bc94       _GUID_DEVCLASS_SCSIADAPTER 10186c94     uuid:cguid_i.obj
 0003:0000bca4       _GUID_DEVCLASS_SECURITYACCELERATOR 10186ca4     uuid:cguid_i.obj
 0003:0000bcb4       _GUID_DEVCLASS_SIDESHOW    10186cb4     uuid:cguid_i.obj
 0003:0000bcc4       _GUID_DEVCLASS_SMARTCARDREADER 10186cc4     uuid:cguid_i.obj
 0003:0000bcd4       _GUID_DEVCLASS_SOUND       10186cd4     uuid:cguid_i.obj
 0003:0000bce4       _GUID_DEVCLASS_SYSTEM      10186ce4     uuid:cguid_i.obj
 0003:0000bcf4       _GUID_DEVCLASS_TAPEDRIVE   10186cf4     uuid:cguid_i.obj
 0003:0000bd04       _GUID_DEVCLASS_UNKNOWN     10186d04     uuid:cguid_i.obj
 0003:0000bd14       _GUID_DEVCLASS_USB         10186d14     uuid:cguid_i.obj
 0003:0000bd24       _GUID_DEVCLASS_VOLUME      10186d24     uuid:cguid_i.obj
 0003:0000bd34       _GUID_DEVCLASS_VOLUMESNAPSHOT 10186d34     uuid:cguid_i.obj
 0003:0000bd44       _GUID_DEVCLASS_WCEUSBS     10186d44     uuid:cguid_i.obj
 0003:0000bd54       _GUID_DEVCLASS_WPD         10186d54     uuid:cguid_i.obj
 0003:0000bd64       _GUID_DEVCLASS_FSFILTER_ACTIVITYMONITOR 10186d64     uuid:cguid_i.obj
 0003:0000bd74       _GUID_DEVCLASS_FSFILTER_UNDELETE 10186d74     uuid:cguid_i.obj
 0003:0000bd84       _GUID_DEVCLASS_FSFILTER_ANTIVIRUS 10186d84     uuid:cguid_i.obj
 0003:0000bd94       _GUID_DEVCLASS_FSFILTER_REPLICATION 10186d94     uuid:cguid_i.obj
 0003:0000bda4       _GUID_DEVCLASS_FSFILTER_CONTINUOUSBACKUP 10186da4     uuid:cguid_i.obj
 0003:0000bdb4       _GUID_DEVCLASS_FSFILTER_CONTENTSCREENER 10186db4     uuid:cguid_i.obj
 0003:0000bdc4       _GUID_DEVCLASS_FSFILTER_QUOTAMANAGEMENT 10186dc4     uuid:cguid_i.obj
 0003:0000bdd4       _GUID_DEVCLASS_FSFILTER_SYSTEMRECOVERY 10186dd4     uuid:cguid_i.obj
 0003:0000bde4       _GUID_DEVCLASS_FSFILTER_CFSMETADATASERVER 10186de4     uuid:cguid_i.obj
 0003:0000bdf4       _GUID_DEVCLASS_FSFILTER_HSM 10186df4     uuid:cguid_i.obj
 0003:0000be04       _GUID_DEVCLASS_FSFILTER_COMPRESSION 10186e04     uuid:cguid_i.obj
 0003:0000be14       _GUID_DEVCLASS_FSFILTER_ENCRYPTION 10186e14     uuid:cguid_i.obj
 0003:0000be24       _GUID_DEVCLASS_FSFILTER_PHYSICALQUOTAMANAGEMENT 10186e24     uuid:cguid_i.obj
 0003:0000be34       _GUID_DEVCLASS_FSFILTER_OPENFILEBACKUP 10186e34     uuid:cguid_i.obj
 0003:0000be44       _GUID_DEVCLASS_FSFILTER_SECURITYENHANCER 10186e44     uuid:cguid_i.obj
 0003:0000be54       _GUID_DEVCLASS_FSFILTER_COPYPROTECTION 10186e54     uuid:cguid_i.obj
 0003:0000be64       _GUID_DEVCLASS_FSFILTER_SYSTEM 10186e64     uuid:cguid_i.obj
 0003:0000be74       _GUID_DEVCLASS_FSFILTER_INFRASTRUCTURE 10186e74     uuid:cguid_i.obj
 0003:0000be84       _GUID_DEVINTERFACE_DISK    10186e84     uuid:cguid_i.obj
 0003:0000be94       _GUID_DEVINTERFACE_CDROM   10186e94     uuid:cguid_i.obj
 0003:0000bea4       _GUID_DEVINTERFACE_PARTITION 10186ea4     uuid:cguid_i.obj
 0003:0000beb4       _GUID_DEVINTERFACE_TAPE    10186eb4     uuid:cguid_i.obj
 0003:0000bec4       _GUID_DEVINTERFACE_WRITEONCEDISK 10186ec4     uuid:cguid_i.obj
 0003:0000bed4       _GUID_DEVINTERFACE_VOLUME  10186ed4     uuid:cguid_i.obj
 0003:0000bee4       _GUID_DEVINTERFACE_MEDIUMCHANGER 10186ee4     uuid:cguid_i.obj
 0003:0000bef4       _GUID_DEVINTERFACE_FLOPPY  10186ef4     uuid:cguid_i.obj
 0003:0000bf04       _GUID_DEVINTERFACE_CDCHANGER 10186f04     uuid:cguid_i.obj
 0003:0000bf14       _GUID_DEVINTERFACE_STORAGEPORT 10186f14     uuid:cguid_i.obj
 0003:0000bf24       _GUID_DEVINTERFACE_COMPORT 10186f24     uuid:cguid_i.obj
 0003:0000bf34       _GUID_DEVINTERFACE_SERENUM_BUS_ENUMERATOR 10186f34     uuid:cguid_i.obj
 0003:0000bf44       ??_C@_0P@GHFPNOJB@bad?5allocation?$AA@ 10186f44     libcpmtd:stdthrow.obj
 0003:0000bf54       ??_C@_01EEMJAFIK@?6?$AA@   10186f54     libcpmtd:stdthrow.obj
 0003:0000bf58       ??_C@_07CIFAGBMG@unknown?$AA@ 10186f58     libcpmtd:stdthrow.obj
 0003:0000bf60       ??_C@_0M@LLHBPFNE@exception?3?5?$AA@ 10186f60     libcpmtd:stdthrow.obj
 0003:0000bf6c       ??_C@_0BA@JFNIOLAK@string?5too?5long?$AA@ 10186f6c     libcpmtd:string.obj
 0003:0000bf7c       ??_C@_0BI@CFPLBAOH@invalid?5string?5position?$AA@ 10186f7c     libcpmtd:string.obj
 0003:0000bf98       ??_7out_of_range@std@@6B@  10186f98     libcpmtd:string.obj
 0003:0000bfa0       ??_C@_0BI@ILCMCLF@invalid?5string?5argument?$AA@ 10186fa0     libcpmtd:string.obj
 0003:0000bfbc       ??_7invalid_argument@std@@6B@ 10186fbc     libcpmtd:string.obj
 0003:0000bfc4       ??_C@_0CO@JPCIKGOF@f?3?2dd?2vctools?2crt_bld?2self_x86?2c@ 10186fc4     libcpmtd:string.obj
 0003:0000bff8       ??_C@_1FO@BEGKGBFG@?$AAf?$AA?3?$AA?2?$AAd?$AAd?$AA?2?$AAv?$AAc?$AAt?$AAo?$AAo?$AAl?$AAs?$AA?2?$AAc?$AAr?$AAt?$AA_?$AAb?$AAl?$AAd?$AA?2?$AAs?$AAe?$AAl?$AAf?$AA_?$AAx?$AA8?$AA6?$AA?2?$AAc@ 10186ff8     libcpmtd:string.obj
 0003:0000c060       __real@8@3ffe8000000000000000 10187060     vorbisfile_static:vorbisfile.obj
 0003:0000c068       __real@4@3ffe8000000000000000 10187068     vorbisfile_static:vorbisfile.obj
 0003:0000c070       __real@8@00000000000000000000 10187070     vorbisfile_static:vorbisfile.obj
 0003:0000c078       __real@8@c0068300000000000000 10187078     vorbisfile_static:vorbisfile.obj
 0003:0000c080       __real@4@400e8000000000000000 10187080     vorbisfile_static:vorbisfile.obj
 0003:0000c084       __real@4@40068000000000000000 10187084     vorbisfile_static:vorbisfile.obj
 0003:0000c088       __real@8@3fff8000000000000000 10187088     vorbisfile_static:vorbisfile.obj
 0003:0000c090       __real@8@bfff8000000000000000 10187090     vorbisfile_static:info.obj
 0003:0000c098       __real@4@c0068c00000000000000 10187098     vorbisfile_static:analysis.obj
 0003:0000c0a0       __real@8@3ff283126e978d4fe000 101870a0     vorbisfile_static:analysis.obj
 0003:0000c0a8       __real@8@3ff1d1b7170000000000 101870a8     vorbisfile_static:analysis.obj
 0003:0000c0b0       __real@8@4002d1999a0000000000 101870b0     vorbisfile_static:analysis.obj
 0003:0000c0b8       __real@8@3ff4c1fc8f0000000000 101870b8     vorbisfile_static:analysis.obj
 0003:0000c0c0       __real@8@40008f5c290000000000 101870c0     vorbisfile_static:analysis.obj
 0003:0000c0c8       __real@8@3fe59ee9ee0000000000 101870c8     vorbisfile_static:analysis.obj
 0003:0000c0d0       __real@8@3ffd8000000000000000 101870d0     vorbisfile_static:analysis.obj
 0003:0000c0d8       __real@4@400afa00000000000000 101870d8     vorbisfile_static:analysis.obj
 0003:0000c0dc       __real@4@4008bf115b0000000000 101870dc     vorbisfile_static:analysis.obj
 0003:0000c0e0       __real@4@3feac0a8c10000000000 101870e0     vorbisfile_static:analysis.obj
 0003:0000c0e4       __real@4@40038000000000000000 101870e4     vorbisfile_static:psy.obj
 0003:0000c0e8       __real@4@00000000000000000000 101870e8     vorbisfile_static:psy.obj
 0003:0000c0ec       __real@4@3ff1d1b7170000000000 101870ec     vorbisfile_static:psy.obj
 0003:0000c0f0       __real@4@3ff4c1fc8f0000000000 101870f0     vorbisfile_static:psy.obj
 0003:0000c0f4       __real@4@3fe59ee9ee0000000000 101870f4     vorbisfile_static:psy.obj
 0003:0000c0f8       __real@8@4005c800000000000000 101870f8     vorbisfile_static:psy.obj
 0003:0000c100       __real@8@3ffeb172150000000000 10187100     vorbisfile_static:psy.obj
 0003:0000c108       __real@8@3ffc8000000000000000 10187108     vorbisfile_static:psy.obj
 0003:0000c110       __real@8@4001bee7b40000000000 10187110     vorbisfile_static:psy.obj
 0003:0000c118       __real@8@3fffb8aa3b0000000000 10187118     vorbisfile_static:psy.obj
 0003:0000c120       __real@4@3ffd8000000000000000 10187120     vorbisfile_static:psy.obj
 0003:0000c128       __real@8@40008000000000000000 10187128     vorbisfile_static:psy.obj
 0003:0000c130       __real@4@40028000000000000000 10187130     vorbisfile_static:psy.obj
 0003:0000c134       __real@4@c006c800000000000000 10187134     vorbisfile_static:psy.obj
 0003:0000c138       __real@8@3ffff800000000000000 10187138     vorbisfile_static:psy.obj
 0003:0000c140       __real@8@40008400000000000000 10187140     vorbisfile_static:psy.obj
 0003:0000c148       __real@4@3fff8000000000000000 10187148     vorbisfile_static:psy.obj
 0003:0000c14c       __real@4@4002a000000000000000 1018714c     vorbisfile_static:psy.obj
 0003:0000c150       __real@8@4003f000000000000000 10187150     vorbisfile_static:psy.obj
 0003:0000c158       __real@8@4002a000000000000000 10187158     vorbisfile_static:psy.obj
 0003:0000c160       __real@4@4008f9c0000000000000 10187160     vorbisfile_static:psy.obj
 0003:0000c164       __real@4@4001c000000000000000 10187164     vorbisfile_static:psy.obj
 0003:0000c168       __real@8@3ffbcccccd0000000000 10187168     vorbisfile_static:psy.obj
 0003:0000c170       __real@4@c00c9c3c000000000000 10187170     vorbisfile_static:psy.obj
 0003:0000c178       __real@8@c0008000000000000000 10187178     vorbisfile_static:psy.obj
 0003:0000c180       __real@8@3ffffffcb90000000000 10187180     vorbisfile_static:psy.obj
 0003:0000c188       __real@8@4001f000000000000000 10187188     vorbisfile_static:bitrate.obj
 0003:0000c190       __real@8@4000c90fdb0000000000 10187190     vorbisfile_static:envelope.obj
 0003:0000c198       __real@8@3ff9caa5254a952a5000 10187198     vorbisfile_static:envelope.obj
 0003:0000c1a0       __real@4@400fc34f800000000000 101871a0     vorbisfile_static:envelope.obj
 0003:0000c1a8       __real@8@40028000000000000000 101871a8     vorbisfile_static:envelope.obj
 0003:0000c1b0       __real@8@4002f000000000000000 101871b0     vorbisfile_static:envelope.obj
 0003:0000c1b8       __real@8@3ffb8000000000000000 101871b8     vorbisfile_static:envelope.obj
 0003:0000c1c0       __real@8@3ffeb333333333333000 101871c0     vorbisfile_static:envelope.obj
 0003:0000c1c8       __real@8@3ffcccccccccccccd000 101871c8     vorbisfile_static:envelope.obj
 0003:0000c1d0       __real@4@40018000000000000000 101871d0     vorbisfile_static:mdct.obj
 0003:0000c1d8       __real@8@bffe8000000000000000 101871d8     vorbisfile_static:mdct.obj
 0003:0000c1e0       __real@4@4000c90fdb0000000000 101871e0     vorbisfile_static:mdct.obj
 0003:0000c1e4       __real@4@3ffeb504f30000000000 101871e4     vorbisfile_static:mdct.obj
 0003:0000c1e8       __real@4@3ffdc3ef150000000000 101871e8     vorbisfile_static:mdct.obj
 0003:0000c1ec       __real@4@3ffeec835e0000000000 101871ec     vorbisfile_static:mdct.obj
 0003:0000c1f0       __real@4@4008ffe0000000000000 101871f0     vorbisfile_static:floor1.obj
 0003:0000c1f4       __real@4@4001ea0ea10000000000 101871f4     vorbisfile_static:floor1.obj
 0003:0000c1f8       __real@8@4004a2f9838f1632f000 101871f8     vorbisfile_static:lsp.obj
 0003:0000c200       __real@4@40048000000000000000 10187200     vorbisfile_static:lsp.obj
 0003:0000c204       __real@4@40058000000000000000 10187204     vorbisfile_static:lsp.obj
 0003:0000c208       __real@4@c0028000000000000000 10187208     vorbisfile_static:lsp.obj
 0003:0000c210       __real@8@3fdaafebff0bcb24a800 10187210     vorbisfile_static:lsp.obj
 0003:0000c218       __real@8@bfeb8637bd05af6c6800 10187218     vorbisfile_static:lsp.obj
 0003:0000c220       __real@8@3feb8637bd05af6c6800 10187220     vorbisfile_static:lsp.obj
 0003:0000c228       __real@8@3fbcbce5086492111800 10187228     vorbisfile_static:lsp.obj
 0003:0000c230       ?ProcessDetach@NativeDll@<CrtImplementationDetails>@@0IB 10187230     LIBCMTD:dbgfree.obj
 0003:0000c234       ?ProcessAttach@NativeDll@<CrtImplementationDetails>@@0IB 10187234     LIBCMTD:dbgfree.obj
 0003:0000c238       ?ThreadAttach@NativeDll@<CrtImplementationDetails>@@0IB 10187238     LIBCMTD:dbgfree.obj
 0003:0000c23c       ?ThreadDetach@NativeDll@<CrtImplementationDetails>@@0IB 1018723c     LIBCMTD:dbgfree.obj
 0003:0000c240       ?ProcessVerifier@NativeDll@<CrtImplementationDetails>@@0IB 10187240     LIBCMTD:dbgfree.obj
 0003:0000c244       ??_C@_1BI@DCHLDCPP@?$AAs?$AAr?$AAc?$AA?5?$AA?$CB?$AA?$DN?$AA?5?$AAN?$AAU?$AAL?$AAL?$AA?$AA@ 10187244     LIBCMTD:stricmp.obj
 0003:0000c25c       ??_C@_1BG@GLLONOEH@?$AA_?$AAs?$AAt?$AAr?$AAi?$AAc?$AAm?$AAp?$AA_?$AAl?$AA?$AA@ 1018725c     LIBCMTD:stricmp.obj
 0003:0000c278       ??_C@_1GC@OILHAOLL@?$AAf?$AA?3?$AA?2?$AAd?$AAd?$AA?2?$AAv?$AAc?$AAt?$AAo?$AAo?$AAl?$AAs?$AA?2?$AAc?$AAr?$AAt?$AA_?$AAb?$AAl?$AAd?$AA?2?$AAs?$AAe?$AAl?$AAf?$AA_?$AAx?$AA8?$AA6?$AA?2?$AAc@ 10187278     LIBCMTD:stricmp.obj
 0003:0000c2dc       ??_C@_1BI@GKKCBDMD@?$AAd?$AAs?$AAt?$AA?5?$AA?$CB?$AA?$DN?$AA?5?$AAN?$AAU?$AAL?$AAL?$AA?$AA@ 101872dc     LIBCMTD:stricmp.obj
 0003:0000c2f4       ??_C@_1BC@JLGKKIIG@?$AA_?$AAs?$AAt?$AAr?$AAi?$AAc?$AAm?$AAp?$AA?$AA@ 101872f4     LIBCMTD:stricmp.obj
 0003:0000c308       __FPinit                   10187308     LIBCMTD:_fpinit_.obj
 0003:0000c30c       __FPmtinit                 1018730c     LIBCMTD:_fpinit_.obj
 0003:0000c310       __FPmtterm                 10187310     LIBCMTD:_fpinit_.obj
 0003:0000c314       ??_C@_0DA@HMCPFNKN@f?3?2dd?2vctools?2crt_bld?2self_x86?2c@ 10187314     LIBCMTD:onexit.obj
 0003:0000c344       ??_C@_17LGKOMLJ@?$AA?4?$AA?4?$AA?4?$AA?$AA@ 10187344     LIBCMTD:dbgrptw.obj
 0003:0000c34c       ??_C@_1CC@CGHMNGDG@?$AAA?$AAs?$AAs?$AAe?$AAr?$AAt?$AAi?$AAo?$AAn?$AA?5?$AAF?$AAa?$AAi?$AAl?$AAe?$AAd?$AA?$AA@ 1018734c     LIBCMTD:dbgrptw.obj
 0003:0000c370       ??_C@_1M@ILHOPKA@?$AAE?$AAr?$AAr?$AAo?$AAr?$AA?$AA@ 10187370     LIBCMTD:dbgrptw.obj
 0003:0000c37c       ??_C@_1BA@GLMCNLEM@?$AAW?$AAa?$AAr?$AAn?$AAi?$AAn?$AAg?$AA?$AA@ 1018737c     LIBCMTD:dbgrptw.obj
 0003:0000c398       ??_C@_0DA@PCCBBBID@f?3?2dd?2vctools?2crt_bld?2self_x86?2c@ 10187398     LIBCMTD:dbgrptw.obj
 0003:0000c3c8       ??_C@_1FI@PHIAFFHM@?$AA?$CI?$AA?$CC?$AAT?$AAh?$AAe?$AA?5?$AAh?$AAo?$AAo?$AAk?$AA?5?$AAf?$AAu?$AAn?$AAc?$AAt?$AAi?$AAo?$AAn?$AA?5?$AAi?$AAs?$AA?5?$AAn?$AAo?$AAt?$AA?5?$AAi?$AAn?$AA?5?$AAt?$AAh@ 101873c8     LIBCMTD:dbgrptw.obj
 0003:0000c420       ??_C@_1CG@JBJEFOCM@?$AAp?$AAf?$AAn?$AAN?$AAe?$AAw?$AAH?$AAo?$AAo?$AAk?$AA?5?$AA?$CB?$AA?$DN?$AA?5?$AAN?$AAU?$AAL?$AAL?$AA?$AA@ 10187420     LIBCMTD:dbgrptw.obj
 0003:0000c448       ??_C@_1CI@IIHEAKEI@?$AA_?$AAC?$AAr?$AAt?$AAS?$AAe?$AAt?$AAR?$AAe?$AAp?$AAo?$AAr?$AAt?$AAH?$AAo?$AAo?$AAk?$AAW?$AA2?$AA?$AA@ 10187448     LIBCMTD:dbgrptw.obj
 0003:0000c470       ??_C@_1GA@IBJGKIFE@?$AAf?$AA?3?$AA?2?$AAd?$AAd?$AA?2?$AAv?$AAc?$AAt?$AAo?$AAo?$AAl?$AAs?$AA?2?$AAc?$AAr?$AAt?$AA_?$AAb?$AAl?$AAd?$AA?2?$AAs?$AAe?$AAl?$AAf?$AA_?$AAx?$AA8?$AA6?$AA?2?$AAc@ 10187470     LIBCMTD:dbgrptw.obj
 0003:0000c4d0       ??_C@_1HI@OFEHGPPC@?$AAm?$AAo?$AAd?$AAe?$AA?5?$AA?$DN?$AA?$DN?$AA?5?$AA_?$AAC?$AAR?$AAT?$AA_?$AAR?$AAP?$AAT?$AAH?$AAO?$AAO?$AAK?$AA_?$AAI?$AAN?$AAS?$AAT?$AAA?$AAL?$AAL?$AA?5?$AA?$HM?$AA?$HM?$AA?5@ 101874d0     LIBCMTD:dbgrptw.obj
 0003:0000c548       ??_C@_1EG@PEOEAKBB@?$AAM?$AAi?$AAc?$AAr?$AAo?$AAs?$AAo?$AAf?$AAt?$AA?5?$AAV?$AAi?$AAs?$AAu?$AAa?$AAl?$AA?5?$AAC?$AA?$CL?$AA?$CL?$AA?5?$AAD?$AAe?$AAb?$AAu?$AAg?$AA?5?$AAL?$AAi?$AAb?$AAr?$AAa@ 10187548     LIBCMTD:dbgrptw.obj
 0003:0000c590       ??_C@_1FG@BBOLDHGF@?$AA_?$AAC?$AAr?$AAt?$AAD?$AAb?$AAg?$AAR?$AAe?$AAp?$AAo?$AAr?$AAt?$AA?3?$AA?5?$AAS?$AAt?$AAr?$AAi?$AAn?$AAg?$AA?5?$AAt?$AAo?$AAo?$AA?5?$AAl?$AAo?$AAn?$AAg?$AA?5?$AAo@ 10187590     LIBCMTD:dbgrptw.obj
 0003:0000c5e8       ??_C@_1JI@EACPGHID@?$AAw?$AAc?$AAs?$AAc?$AAp?$AAy?$AA_?$AAs?$AA?$CI?$AAs?$AAz?$AAO?$AAu?$AAt?$AAM?$AAe?$AAs?$AAs?$AAa?$AAg?$AAe?$AA?0?$AA?5?$AA4?$AA0?$AA9?$AA6?$AA?0?$AA?5?$AAL?$AA?$CC?$AA_@ 101875e8     LIBCMTD:dbgrptw.obj
 0003:0000c680       ??_C@_1BI@KALLJECN@?$AA?$CI?$AA?$CK?$AA_?$AAe?$AAr?$AAr?$AAn?$AAo?$AA?$CI?$AA?$CJ?$AA?$CJ?$AA?$AA@ 10187680     LIBCMTD:dbgrptw.obj
 0003:0000c698       ??_C@_1KK@MEFMPOLM@?$AAD?$AAe?$AAb?$AAu?$AAg?$AA?5?$AA?$CF?$AAs?$AA?$CB?$AA?6?$AA?6?$AAP?$AAr?$AAo?$AAg?$AAr?$AAa?$AAm?$AA?3?$AA?5?$AA?$CF?$AAs?$AA?$CF?$AAs?$AA?$CF?$AAs?$AA?$CF?$AAs?$AA?$CF?$AAs?$AA?$CF?$AAs@ 10187698     LIBCMTD:dbgrptw.obj
 0003:0000c744       ??_C@_1BE@CGCJKGHI@?$AA?6?$AAM?$AAo?$AAd?$AAu?$AAl?$AAe?$AA?3?$AA?5?$AA?$AA@ 10187744     LIBCMTD:dbgrptw.obj
 0003:0000c758       ??_C@_1BA@LNHECFIM@?$AA?6?$AAF?$AAi?$AAl?$AAe?$AA?3?$AA?5?$AA?$AA@ 10187758     LIBCMTD:dbgrptw.obj
 0003:0000c768       ??_C@_1BA@GLLGCPCK@?$AA?6?$AAL?$AAi?$AAn?$AAe?$AA?3?$AA?5?$AA?$AA@ 10187768     LIBCMTD:dbgrptw.obj
 0003:0000c778       ??_C@_15IABLJNFO@?$AA?6?$AA?6?$AA?$AA@ 10187778     LIBCMTD:dbgrptw.obj
 0003:0000c780       ??_C@_1BK@PEDCIPMA@?$AAE?$AAx?$AAp?$AAr?$AAe?$AAs?$AAs?$AAi?$AAo?$AAn?$AA?3?$AA?5?$AA?$AA@ 10187780     LIBCMTD:dbgrptw.obj
 0003:0000c79c       ??_C@_11LOCGONAA@?$AA?$AA@ 1018779c     LIBCMTD:dbgrptw.obj
 0003:0000c7a0       ??_C@_1OG@PMPPFHAF@?$AA?6?$AA?6?$AAF?$AAo?$AAr?$AA?5?$AAi?$AAn?$AAf?$AAo?$AAr?$AAm?$AAa?$AAt?$AAi?$AAo?$AAn?$AA?5?$AAo?$AAn?$AA?5?$AAh?$AAo?$AAw?$AA?5?$AAy?$AAo?$AAu?$AAr?$AA?5?$AAp?$AAr@ 101877a0     LIBCMTD:dbgrptw.obj
 0003:0000c888       ??_C@_1NO@LECLLHOL@?$AAm?$AAe?$AAm?$AAc?$AAp?$AAy?$AA_?$AAs?$AA?$CI?$AAs?$AAz?$AAS?$AAh?$AAo?$AAr?$AAt?$AAP?$AAr?$AAo?$AAg?$AAN?$AAa?$AAm?$AAe?$AA?0?$AA?5?$AAs?$AAi?$AAz?$AAe?$AAo?$AAf@ 10187888     LIBCMTD:dbgrptw.obj
 0003:0000c968       ??_C@_1CO@EAEJAADC@?$AA?$DM?$AAp?$AAr?$AAo?$AAg?$AAr?$AAa?$AAm?$AA?5?$AAn?$AAa?$AAm?$AAe?$AA?5?$AAu?$AAn?$AAk?$AAn?$AAo?$AAw?$AAn?$AA?$DO?$AA?$AA@ 10187968     LIBCMTD:dbgrptw.obj
 0003:0000c998       ??_C@_1GI@DEDNNLCI@?$AAw?$AAc?$AAs?$AAc?$AAp?$AAy?$AA_?$AAs?$AA?$CI?$AAs?$AAz?$AAE?$AAx?$AAe?$AAN?$AAa?$AAm?$AAe?$AA?0?$AA?5?$AA2?$AA6?$AA0?$AA?0?$AA?5?$AAL?$AA?$CC?$AA?$DM?$AAp?$AAr?$AAo?$AAg@ 10187998     LIBCMTD:dbgrptw.obj
 0003:0000ca00       ??_C@_1CI@PGJIFDEK@?$AA_?$AA_?$AAc?$AAr?$AAt?$AAM?$AAe?$AAs?$AAs?$AAa?$AAg?$AAe?$AAW?$AAi?$AAn?$AAd?$AAo?$AAw?$AAW?$AA?$AA@ 10187a00     LIBCMTD:dbgrptw.obj
 0003:0000ca28       ??_C@_1GE@BDAODJCD@?$AAf?$AA?3?$AA?2?$AAd?$AAd?$AA?2?$AAv?$AAc?$AAt?$AAo?$AAo?$AAl?$AAs?$AA?2?$AAc?$AAr?$AAt?$AA_?$AAb?$AAl?$AAd?$AA?2?$AAs?$AAe?$AAl?$AAf?$AA_?$AAx?$AA8?$AA6?$AA?2?$AAc@ 10187a28     LIBCMTD:dbgdel.obj
 0003:0000ca90       ??_C@_1EO@LHDAJOCM@?$AA_?$AAB?$AAL?$AAO?$AAC?$AAK?$AA_?$AAT?$AAY?$AAP?$AAE?$AA_?$AAI?$AAS?$AA_?$AAV?$AAA?$AAL?$AAI?$AAD?$AA?$CI?$AAp?$AAH?$AAe?$AAa?$AAd?$AA?9?$AA?$DO?$AAn?$AAB?$AAl?$AAo@ 10187a90     LIBCMTD:dbgdel.obj
 0003:0000cb04       ??_7type_info@@6B@         10187b04     LIBCMTD:typinfo.obj
 0003:0000cb0c       ??_7exception@std@@6B@     10187b0c     LIBCMTD:stdexcpt.obj
 0003:0000cb14       ??_C@_0BC@EOODALEL@Unknown?5exception?$AA@ 10187b14     LIBCMTD:stdexcpt.obj
 0003:0000cb2c       ??_7bad_cast@std@@6B@      10187b2c     LIBCMTD:stdexcpt.obj
 0003:0000cb38       ??_7bad_typeid@std@@6B@    10187b38     LIBCMTD:stdexcpt.obj
 0003:0000cb44       ??_7__non_rtti_object@std@@6B@ 10187b44     LIBCMTD:stdexcpt.obj
 0003:0000cb4c       ??_C@_1CK@DDKKOLAN@?$AAs?$AAi?$AAz?$AAe?$AAI?$AAn?$AAB?$AAy?$AAt?$AAe?$AAs?$AA?5?$AA?$DO?$AA?$DN?$AA?5?$AAc?$AAo?$AAu?$AAn?$AAt?$AA?$AA@ 10187b4c     LIBCMTD:memcpy_s.obj
 0003:0000cb78       ??_C@_1BC@GKHDJMGB@?$AAm?$AAe?$AAm?$AAc?$AAp?$AAy?$AA_?$AAs?$AA?$AA@ 10187b78     LIBCMTD:memcpy_s.obj
 0003:0000cb90       ??_C@_1GE@NEOPGGBM@?$AAf?$AA?3?$AA?2?$AAd?$AAd?$AA?2?$AAv?$AAc?$AAt?$AAo?$AAo?$AAl?$AAs?$AA?2?$AAc?$AAr?$AAt?$AA_?$AAb?$AAl?$AAd?$AA?2?$AAs?$AAe?$AAl?$AAf?$AA_?$AAx?$AA8?$AA6?$AA?2?$AAc@ 10187b90     LIBCMTD:memcpy_s.obj
 0003:0000cbf4       ??_C@_1BE@NMKKBGPA@?$AAm?$AAe?$AAm?$AAm?$AAo?$AAv?$AAe?$AA_?$AAs?$AA?$AA@ 10187bf4     LIBCMTD:memmove_s.obj
 0003:0000cc08       ??_C@_1GG@JKNLCIHH@?$AAf?$AA?3?$AA?2?$AAd?$AAd?$AA?2?$AAv?$AAc?$AAt?$AAo?$AAo?$AAl?$AAs?$AA?2?$AAc?$AAr?$AAt?$AA_?$AAb?$AAl?$AAd?$AA?2?$AAs?$AAe?$AAl?$AAf?$AA_?$AAx?$AA8?$AA6?$AA?2?$AAc@ 10187c08     LIBCMTD:memmove_s.obj
 0003:0000cc70       ??_C@_1CC@OLIJCKA@?$AA?$CI?$AAs?$AAt?$AAr?$AAi?$AAn?$AAg?$AA?5?$AA?$CB?$AA?$DN?$AA?5?$AAN?$AAU?$AAL?$AAL?$AA?$CJ?$AA?$AA@ 10187c70     LIBCMTD:sprintf.obj
 0003:0000cc94       ??_C@_1BA@KBJJGFFE@?$AAs?$AAp?$AAr?$AAi?$AAn?$AAt?$AAf?$AA?$AA@ 10187c94     LIBCMTD:sprintf.obj
 0003:0000cca8       ??_C@_1GC@BMNPEKNN@?$AAf?$AA?3?$AA?2?$AAd?$AAd?$AA?2?$AAv?$AAc?$AAt?$AAo?$AAo?$AAl?$AAs?$AA?2?$AAc?$AAr?$AAt?$AA_?$AAb?$AAl?$AAd?$AA?2?$AAs?$AAe?$AAl?$AAf?$AA_?$AAx?$AA8?$AA6?$AA?2?$AAc@ 10187ca8     LIBCMTD:sprintf.obj
 0003:0000cd0c       ??_C@_1CC@MGIEJOME@?$AA?$CI?$AAf?$AAo?$AAr?$AAm?$AAa?$AAt?$AA?5?$AA?$CB?$AA?$DN?$AA?5?$AAN?$AAU?$AAL?$AAL?$AA?$CJ?$AA?$AA@ 10187d0c     LIBCMTD:sprintf.obj
 0003:0000cd30       ??_C@_0BO@GNIAFIKK@Unknown?5Runtime?5Check?5Error?6?$AN?$AA@ 10187d30     LIBCMTD:_error_.obj
 0003:0000cd50       ??_C@_0CM@NGINOKPC@Stack?5memory?5around?5_alloca?5was?5@ 10187d50     LIBCMTD:_error_.obj
 0003:0000cd7c       ??_C@_0DG@HKJMLLLP@A?5local?5variable?5was?5used?5before@ 10187d7c     LIBCMTD:_error_.obj
 0003:0000cdb4       ??_C@_0BN@FFOINMNJ@Stack?5memory?5was?5corrupted?6?$AN?$AA@ 10187db4     LIBCMTD:_error_.obj
 0003:0000cdd8       ??_C@_0BBN@GPMLNJCF@A?5cast?5to?5a?5smaller?5data?5type?5ha@ 10187dd8     LIBCMTD:_error_.obj
 0003:0000cef8       ??_C@_0NN@NGPKDKPD@The?5value?5of?5ESP?5was?5not?5properl@ 10187ef8     LIBCMTD:_error_.obj
 0003:0000d074       ??_C@_0CA@IODNCDPG@Run?9Time?5Check?5Failure?5?$CD?$CFd?5?9?5?$CFs?$AA@ 10188074     LIBCMTD:_error_.obj
 0003:0000d094       ??_C@_0BE@GNBOBNCK@Unknown?5Module?5Name?$AA@ 10188094     LIBCMTD:_error_.obj
 0003:0000d0a8       ??_C@_0BB@PFFGGCJP@Unknown?5Filename?$AA@ 101880a8     LIBCMTD:_error_.obj
 0003:0000d0c0       ??_C@_1EA@NFKNIFJP@?$AAR?$AAu?$AAn?$AA?9?$AAT?$AAi?$AAm?$AAe?$AA?5?$AAC?$AAh?$AAe?$AAc?$AAk?$AA?5?$AAF?$AAa?$AAi?$AAl?$AAu?$AAr?$AAe?$AA?5?$AA?$CD?$AA?$CF?$AAd?$AA?5?$AA?9?$AA?5?$AA?$CF?$AAs?$AA?$AA@ 101880c0     LIBCMTD:_error_.obj
 0003:0000d100       ??_C@_1GM@OLMCBDMB@?$AAR?$AAu?$AAn?$AAt?$AAi?$AAm?$AAe?$AA?5?$AAC?$AAh?$AAe?$AAc?$AAk?$AA?5?$AAE?$AAr?$AAr?$AAo?$AAr?$AA?4?$AA?6?$AA?$AN?$AA?5?$AAU?$AAn?$AAa?$AAb?$AAl?$AAe?$AA?5?$AAt?$AAo@ 10188100     LIBCMTD:_error_.obj
 0003:0000d16c       ??_C@_0CG@IAFNJNEE@Stack?5corrupted?5near?5unknown?5var@ 1018816c     LIBCMTD:_error_.obj
 0003:0000d198       ??_C@_0EJ@LJKNEOLN@Stack?5area?5around?5_alloca?5memory@ 10188198     LIBCMTD:_error_.obj
 0003:0000d1e4       ??_C@_08KJEDNCKC@?$CFs?$CFs?$CFs?$CFs?$AA@ 101881e4     LIBCMTD:_error_.obj
 0003:0000d1f0       ??_C@_02LLMPMKNF@?$DO?5?$AA@ 101881f0     LIBCMTD:_error_.obj
 0003:0000d1f4       ??_C@_0BC@KIBAILCI@?$CFs?$CFs?$CFp?$CFs?$CFld?$CFs?$CFd?$CFs?$AA@ 101881f4     LIBCMTD:_error_.obj
 0003:0000d208       ??_C@_0EI@CLEPFNGI@Stack?5area?5around?5_alloca?5memory@ 10188208     LIBCMTD:_error_.obj
 0003:0000d250       ??_C@_0N@MHFFIMFG@?6Address?3?50x?$AA@ 10188250     LIBCMTD:_error_.obj
 0003:0000d260       ??_C@_07DFDJCKFN@?6Size?3?5?$AA@ 10188260     LIBCMTD:_error_.obj
 0003:0000d268       ??_C@_0CK@DKGBICFE@?6Allocation?5number?5within?5this?5f@ 10188268     LIBCMTD:_error_.obj
 0003:0000d294       ??_C@_08OMAHNMHJ@?6Data?3?5?$DM?$AA@ 10188294     LIBCMTD:_error_.obj
 0003:0000d2a0       ??_C@_09FOPFMPEJ@wsprintfA?$AA@ 101882a0     LIBCMTD:_error_.obj
 0003:0000d2ac       ??_C@_0L@GMPLCCII@user32?4dll?$AA@ 101882ac     LIBCMTD:_error_.obj
 0003:0000d2b8       ??_C@_05MKKEDADM@?$CF?42X?5?$AA@ 101882b8     LIBCMTD:_error_.obj
 0003:0000d2c0       ??_C@_0DE@OHJBPMBP@A?5variable?5is?5being?5used?5without@ 101882c0     LIBCMTD:_error_.obj
 0003:0000d2f4       ??_C@_1BA@NJCJMLHI@?$AA_?$AAa?$AAt?$AAo?$AAf?$AA_?$AAl?$AA?$AA@ 101882f4     LIBCMTD:atof.obj
 0003:0000d308       ??_C@_1FM@HAAJIFE@?$AAf?$AA?3?$AA?2?$AAd?$AAd?$AA?2?$AAv?$AAc?$AAt?$AAo?$AAo?$AAl?$AAs?$AA?2?$AAc?$AAr?$AAt?$AA_?$AAb?$AAl?$AAd?$AA?2?$AAs?$AAe?$AAl?$AAf?$AA_?$AAx?$AA8?$AA6?$AA?2?$AAc@ 10188308     LIBCMTD:atof.obj
 0003:0000d364       ??_C@_1BK@LAOAACLJ@?$AAn?$AAp?$AAt?$AAr?$AA?5?$AA?$CB?$AA?$DN?$AA?5?$AAN?$AAU?$AAL?$AAL?$AA?$AA@ 10188364     LIBCMTD:atof.obj
 0003:0000d380       ??_C@_1BI@IGILPKD@?$AA_?$AAv?$AAs?$AAp?$AAr?$AAi?$AAn?$AAt?$AAf?$AA_?$AAl?$AA?$AA@ 10188380     LIBCMTD:vsprintf.obj
 0003:0000d398       ??_C@_1GE@DPADKNCG@?$AAf?$AA?3?$AA?2?$AAd?$AAd?$AA?2?$AAv?$AAc?$AAt?$AAo?$AAo?$AAl?$AAs?$AA?2?$AAc?$AAr?$AAt?$AA_?$AAb?$AAl?$AAd?$AA?2?$AAs?$AAe?$AAl?$AAf?$AA_?$AAx?$AA8?$AA6?$AA?2?$AAc@ 10188398     LIBCMTD:vsprintf.obj
 0003:0000d3fc       ??_C@_1CE@HMKDJHB@?$AA_?$AAv?$AAs?$AAc?$AAp?$AAr?$AAi?$AAn?$AAt?$AAf?$AA_?$AAh?$AAe?$AAl?$AAp?$AAe?$AAr?$AA?$AA@ 101883fc     LIBCMTD:vsprintf.obj
 0003:0000d420       ??_C@_1DE@MLEJGPLF@?$AA?$CI?$AAL?$AA?$CC?$AAI?$AAn?$AAv?$AAa?$AAl?$AAi?$AAd?$AA?5?$AAp?$AAa?$AAr?$AAa?$AAm?$AAe?$AAt?$AAe?$AAr?$AA?$CC?$AA?0?$AA?5?$AA0?$AA?$CJ?$AA?$AA@ 10188420     LIBCMTD:splitpat.obj
 0003:0000d454       ??_C@_1CE@DEGFKGOA@?$AA_?$AAs?$AAp?$AAl?$AAi?$AAt?$AAp?$AAa?$AAt?$AAh?$AA_?$AAh?$AAe?$AAl?$AAp?$AAe?$AAr?$AA?$AA@ 10188454     LIBCMTD:splitpat.obj
 0003:0000d478       ??_C@_1HA@GHKPFCBF@?$AAf?$AA?3?$AA?2?$AAd?$AAd?$AA?2?$AAv?$AAc?$AAt?$AAo?$AAo?$AAl?$AAs?$AA?2?$AAc?$AAr?$AAt?$AA_?$AAb?$AAl?$AAd?$AA?2?$AAs?$AAe?$AAl?$AAf?$AA_?$AAx?$AA8?$AA6?$AA?2?$AAc@ 10188478     LIBCMTD:splitpat.obj
 0003:0000d4e8       ??_C@_1CI@MLPLHPBP@?$AA?$CI?$AA?$CI?$AA?$CI?$AA_?$AAP?$AAa?$AAt?$AAh?$AA?$CJ?$AA?$CJ?$AA?$CJ?$AA?5?$AA?$CB?$AA?$DN?$AA?5?$AAN?$AAU?$AAL?$AAL?$AA?$AA@ 101884e8     LIBCMTD:splitpat.obj
 0003:0000d510       ??_C@_1CI@HBNALCBB@?$AA?$CI?$AA?$CK?$AAm?$AAo?$AAd?$AAe?$AA?5?$AA?$CB?$AA?$DN?$AA?5?$AA_?$AAT?$AA?$CI?$AA?8?$AA?2?$AA0?$AA?8?$AA?$CJ?$AA?$CJ?$AA?$AA@ 10188510     LIBCMTD:fopen.obj
 0003:0000d538       ??_C@_1BO@MJMKAKCJ@?$AA?$CI?$AAm?$AAo?$AAd?$AAe?$AA?5?$AA?$CB?$AA?$DN?$AA?5?$AAN?$AAU?$AAL?$AAL?$AA?$CJ?$AA?$AA@ 10188538     LIBCMTD:fopen.obj
 0003:0000d558       ??_C@_1BA@HNEAFMNL@?$AA_?$AAf?$AAs?$AAo?$AAp?$AAe?$AAn?$AA?$AA@ 10188558     LIBCMTD:fopen.obj
 0003:0000d568       ??_C@_1FO@NCADDBOO@?$AAf?$AA?3?$AA?2?$AAd?$AAd?$AA?2?$AAv?$AAc?$AAt?$AAo?$AAo?$AAl?$AAs?$AA?2?$AAc?$AAr?$AAt?$AA_?$AAb?$AAl?$AAd?$AA?2?$AAs?$AAe?$AAl?$AAf?$AA_?$AAx?$AA8?$AA6?$AA?2?$AAc@ 10188568     LIBCMTD:fopen.obj
 0003:0000d5c8       ??_C@_1BO@CLGIAEOJ@?$AA?$CI?$AAf?$AAi?$AAl?$AAe?$AA?5?$AA?$CB?$AA?$DN?$AA?5?$AAN?$AAU?$AAL?$AAL?$AA?$CJ?$AA?$AA@ 101885c8     LIBCMTD:fopen.obj
 0003:0000d5e8       ??_C@_1BA@PBGKCCAP@?$AAf?$AAo?$AAp?$AAe?$AAn?$AA_?$AAs?$AA?$AA@ 101885e8     LIBCMTD:fopen.obj
 0003:0000d5f8       ??_C@_1CA@LLJLFCDN@?$AA?$CI?$AAp?$AAf?$AAi?$AAl?$AAe?$AA?5?$AA?$CB?$AA?$DN?$AA?5?$AAN?$AAU?$AAL?$AAL?$AA?$CJ?$AA?$AA@ 101885f8     LIBCMTD:fopen.obj
 0003:0000d618       ??_C@_1O@EGMJNCOI@?$AAf?$AAc?$AAl?$AAo?$AAs?$AAe?$AA?$AA@ 10188618     LIBCMTD:fclose.obj
 0003:0000d628       ??_C@_1GA@KMIDAPAP@?$AAf?$AA?3?$AA?2?$AAd?$AAd?$AA?2?$AAv?$AAc?$AAt?$AAo?$AAo?$AAl?$AAs?$AA?2?$AAc?$AAr?$AAt?$AA_?$AAb?$AAl?$AAd?$AA?2?$AAs?$AAe?$AAl?$AAf?$AA_?$AAx?$AA8?$AA6?$AA?2?$AAc@ 10188628     LIBCMTD:fclose.obj
 0003:0000d688       ??_C@_1CC@FADMNIL@?$AA?$CI?$AAs?$AAt?$AAr?$AAe?$AAa?$AAm?$AA?5?$AA?$CB?$AA?$DN?$AA?5?$AAN?$AAU?$AAL?$AAL?$AA?$CJ?$AA?$AA@ 10188688     LIBCMTD:fclose.obj
 0003:0000d6ac       ??_C@_1BO@JINCABEC@?$AA_?$AAf?$AAc?$AAl?$AAo?$AAs?$AAe?$AA_?$AAn?$AAo?$AAl?$AAo?$AAc?$AAk?$AA?$AA@ 101886ac     LIBCMTD:fclose.obj
 0003:0000d6cc       ??_C@_1BM@JMKHIAHP@?$AA?$CI?$AAs?$AAt?$AAr?$AA?5?$AA?$CB?$AA?$DN?$AA?5?$AAN?$AAU?$AAL?$AAL?$AA?$CJ?$AA?$AA@ 101886cc     LIBCMTD:fclose.obj
 0003:0000d6e8       ??_C@_1M@CKCKPMNP@?$AAf?$AAt?$AAe?$AAl?$AAl?$AA?$AA@ 101886e8     LIBCMTD:ftell.obj
 0003:0000d6f8       ??_C@_1FO@NBACIADE@?$AAf?$AA?3?$AA?2?$AAd?$AAd?$AA?2?$AAv?$AAc?$AAt?$AAo?$AAo?$AAl?$AAs?$AA?2?$AAc?$AAr?$AAt?$AA_?$AAb?$AAl?$AAd?$AA?2?$AAs?$AAe?$AAl?$AAf?$AA_?$AAx?$AA8?$AA6?$AA?2?$AAc@ 101886f8     LIBCMTD:ftell.obj
 0003:0000d758       ??_C@_1BM@EPIDANEK@?$AA_?$AAf?$AAt?$AAe?$AAl?$AAl?$AA_?$AAn?$AAo?$AAl?$AAo?$AAc?$AAk?$AA?$AA@ 10188758     LIBCMTD:ftell.obj
 0003:0000d778       ??_C@_1IO@PMHBOLJK@?$AA?$CI?$AA?$CI?$AAw?$AAh?$AAe?$AAn?$AAc?$AAe?$AA?5?$AA?$DN?$AA?$DN?$AA?5?$AAS?$AAE?$AAE?$AAK?$AA_?$AAS?$AAE?$AAT?$AA?$CJ?$AA?5?$AA?$HM?$AA?$HM?$AA?5?$AA?$CI?$AAw?$AAh?$AAe?$AAn?$AAc?$AAe@ 10188778     LIBCMTD:fseek.obj
 0003:0000d808       ??_C@_1M@HCCOIONH@?$AAf?$AAs?$AAe?$AAe?$AAk?$AA?$AA@ 10188808     LIBCMTD:fseek.obj
 0003:0000d818       ??_C@_1FO@ECBPAICH@?$AAf?$AA?3?$AA?2?$AAd?$AAd?$AA?2?$AAv?$AAc?$AAt?$AAo?$AAo?$AAl?$AAs?$AA?2?$AAc?$AAr?$AAt?$AA_?$AAb?$AAl?$AAd?$AA?2?$AAs?$AAe?$AAl?$AAf?$AA_?$AAx?$AA8?$AA6?$AA?2?$AAc@ 10188818     LIBCMTD:fseek.obj
 0003:0000d878       ??_C@_1BA@CMLCEIGG@?$AAf?$AAr?$AAe?$AAa?$AAd?$AA_?$AAs?$AA?$AA@ 10188878     LIBCMTD:fread.obj
 0003:0000d888       ??_C@_1FO@PNLFLIH@?$AAf?$AA?3?$AA?2?$AAd?$AAd?$AA?2?$AAv?$AAc?$AAt?$AAo?$AAo?$AAl?$AAs?$AA?2?$AAc?$AAr?$AAt?$AA_?$AAb?$AAl?$AAd?$AA?2?$AAs?$AAe?$AAl?$AAf?$AA_?$AAx?$AA8?$AA6?$AA?2?$AAc@ 10188888     LIBCMTD:fread.obj
 0003:0000d8e8       ??_C@_1DA@DKEFLDMG@?$AA?$CI?$AA?$CC?$AAb?$AAu?$AAf?$AAf?$AAe?$AAr?$AA?5?$AAt?$AAo?$AAo?$AA?5?$AAs?$AAm?$AAa?$AAl?$AAl?$AA?$CC?$AA?0?$AA?5?$AA0?$AA?$CJ?$AA?$AA@ 101888e8     LIBCMTD:fread.obj
 0003:0000d918       ??_C@_1LG@DCNDJCHK@?$AA?$CI?$AA?$CC?$AAI?$AAn?$AAc?$AAo?$AAn?$AAs?$AAi?$AAs?$AAt?$AAe?$AAn?$AAt?$AA?5?$AAS?$AAt?$AAr?$AAe?$AAa?$AAm?$AA?5?$AAC?$AAo?$AAu?$AAn?$AAt?$AA?4?$AA?5?$AAF?$AAl?$AAu@ 10188918     LIBCMTD:fread.obj
 0003:0000d9d0       ??_C@_1EA@FAMECDND@?$AAn?$AAu?$AAm?$AA?5?$AA?$DM?$AA?$DN?$AA?5?$AA?$CI?$AAS?$AAI?$AAZ?$AAE?$AA_?$AAM?$AAA?$AAX?$AA?5?$AA?1?$AA?5?$AAe?$AAl?$AAe?$AAm?$AAe?$AAn?$AAt?$AAS?$AAi?$AAz?$AAe?$AA?$CJ?$AA?$AA@ 101889d0     LIBCMTD:fread.obj
 0003:0000da10       ??_C@_1CA@IDPOGFL@?$AA_?$AAf?$AAr?$AAe?$AAa?$AAd?$AA_?$AAn?$AAo?$AAl?$AAo?$AAc?$AAk?$AA_?$AAs?$AA?$AA@ 10188a10     LIBCMTD:fread.obj
 0003:0000da30       ??_C@_1CC@CGFEEBMC@?$AA?$CI?$AAb?$AAu?$AAf?$AAf?$AAe?$AAr?$AA?5?$AA?$CB?$AA?$DN?$AA?5?$AAN?$AAU?$AAL?$AAL?$AA?$CJ?$AA?$AA@ 10188a30     LIBCMTD:fread.obj
 0003:0000da54       ??_C@_1O@GKDHFACN@?$AAp?$AAr?$AAi?$AAn?$AAt?$AAf?$AA?$AA@ 10188a54     LIBCMTD:printf.obj
 0003:0000da68       ??_C@_1GA@LHEGHOAF@?$AAf?$AA?3?$AA?2?$AAd?$AAd?$AA?2?$AAv?$AAc?$AAt?$AAo?$AAo?$AAl?$AAs?$AA?2?$AAc?$AAr?$AAt?$AA_?$AAb?$AAl?$AAd?$AA?2?$AAs?$AAe?$AAl?$AAf?$AA_?$AAx?$AA8?$AA6?$AA?2?$AAc@ 10188a68     LIBCMTD:printf.obj
 0003:0000dac8       ??_C@_1O@KLNKIMAP@?$AAf?$AAw?$AAr?$AAi?$AAt?$AAe?$AA?$AA@ 10188ac8     LIBCMTD:fwrite.obj
 0003:0000dad8       ??_C@_1GA@DOFNKKGD@?$AAf?$AA?3?$AA?2?$AAd?$AAd?$AA?2?$AAv?$AAc?$AAt?$AAo?$AAo?$AAl?$AAs?$AA?2?$AAc?$AAr?$AAt?$AA_?$AAb?$AAl?$AAd?$AA?2?$AAs?$AAe?$AAl?$AAf?$AA_?$AAx?$AA8?$AA6?$AA?2?$AAc@ 10188ad8     LIBCMTD:fwrite.obj
 0003:0000db38       ??_C@_1DC@FHEPNAPF@?$AAn?$AAu?$AAm?$AA?5?$AA?$DM?$AA?$DN?$AA?5?$AA?$CI?$AAS?$AAI?$AAZ?$AAE?$AA_?$AAM?$AAA?$AAX?$AA?5?$AA?1?$AA?5?$AAs?$AAi?$AAz?$AAe?$AA?$CJ?$AA?$AA@ 10188b38     LIBCMTD:fwrite.obj
 0003:0000db6c       ??_C@_1BO@JGPKCBCE@?$AA_?$AAf?$AAw?$AAr?$AAi?$AAt?$AAe?$AA_?$AAn?$AAo?$AAl?$AAo?$AAc?$AAk?$AA?$AA@ 10188b6c     LIBCMTD:fwrite.obj
 0003:0000db8c       ??_C@_1BG@KCMPBBDK@?$AA_?$AAg?$AAe?$AAt?$AA_?$AAe?$AAr?$AAr?$AAn?$AAo?$AA?$AA@ 10188b8c     LIBCMTD:dosmap.obj
 0003:0000dba8       ??_C@_1GA@MFGIMPNL@?$AAf?$AA?3?$AA?2?$AAd?$AAd?$AA?2?$AAv?$AAc?$AAt?$AAo?$AAo?$AAl?$AAs?$AA?2?$AAc?$AAr?$AAt?$AA_?$AAb?$AAl?$AAd?$AA?2?$AAs?$AAe?$AAl?$AAf?$AA_?$AAx?$AA8?$AA6?$AA?2?$AAc@ 10188ba8     LIBCMTD:dosmap.obj
 0003:0000dc08       ??_C@_1BO@LKEBEKJP@?$AAp?$AAV?$AAa?$AAl?$AAu?$AAe?$AA?5?$AA?$CB?$AA?$DN?$AA?5?$AAN?$AAU?$AAL?$AAL?$AA?$AA@ 10188c08     LIBCMTD:dosmap.obj
 0003:0000dc28       ??_C@_1BM@INIPHHDD@?$AA_?$AAg?$AAe?$AAt?$AA_?$AAd?$AAo?$AAs?$AAe?$AAr?$AAr?$AAn?$AAo?$AA?$AA@ 10188c28     LIBCMTD:dosmap.obj
 0003:0000dc44       ??_C@_06PJIGMIJB@Client?$AA@ 10188c44     LIBCMTD:dbgheap.obj
 0003:0000dc4c       ??_C@_06KMEJCCGM@Ignore?$AA@ 10188c4c     LIBCMTD:dbgheap.obj
 0003:0000dc54       ??_C@_03OGPFLFLO@CRT?$AA@  10188c54     LIBCMTD:dbgheap.obj
 0003:0000dc58       ??_C@_06EFAGIKOH@Normal?$AA@ 10188c58     LIBCMTD:dbgheap.obj
 0003:0000dc60       ??_C@_04HJMOFLDF@Free?$AA@ 10188c60     LIBCMTD:dbgheap.obj
 0003:0000dc7c       ??_C@_0DC@JEMAGEKG@Error?3?5memory?5allocation?3?5bad?5me@ 10188c7c     LIBCMTD:dbgheap.obj
 0003:0000dcb0       ??_C@_0CF@BICKFLAF@Invalid?5allocation?5size?3?5?$CFIu?5byt@ 10188cb0     LIBCMTD:dbgheap.obj
 0003:0000dcd8       ??_C@_02DKCKIIND@?$CFs?$AA@ 10188cd8     LIBCMTD:dbgheap.obj
 0003:0000dcdc       ??_C@_0CB@CCLOLAHO@Client?5hook?5allocation?5failure?4?6@ 10188cdc     LIBCMTD:dbgheap.obj
 0003:0000dd00       ??_C@_0DF@BBEGIFEK@Client?5hook?5allocation?5failure?5a@ 10188d00     LIBCMTD:dbgheap.obj
 0003:0000dd38       ??_C@_1GC@DNJKKEAA@?$AAf?$AA?3?$AA?2?$AAd?$AAd?$AA?2?$AAv?$AAc?$AAt?$AAo?$AAo?$AAl?$AAs?$AA?2?$AAc?$AAr?$AAt?$AA_?$AAb?$AAl?$AAd?$AA?2?$AAs?$AAe?$AAl?$AAf?$AA_?$AAx?$AA8?$AA6?$AA?2?$AAc@ 10188d38     LIBCMTD:dbgheap.obj
 0003:0000dd9c       ??_C@_1CE@LJFEPPMP@?$AA_?$AAC?$AAr?$AAt?$AAC?$AAh?$AAe?$AAc?$AAk?$AAM?$AAe?$AAm?$AAo?$AAr?$AAy?$AA?$CI?$AA?$CJ?$AA?$AA@ 10188d9c     LIBCMTD:dbgheap.obj
 0003:0000ddc0       ??_C@_1CC@CKBDKDFF@?$AA_?$AAc?$AAa?$AAl?$AAl?$AAo?$AAc?$AA_?$AAd?$AAb?$AAg?$AA_?$AAi?$AAm?$AAp?$AAl?$AA?$AA@ 10188dc0     LIBCMTD:dbgheap.obj
 0003:0000dde4       ??_C@_1DO@MEOGCGBN@?$AA?$CI?$AA_?$AAH?$AAE?$AAA?$AAP?$AA_?$AAM?$AAA?$AAX?$AAR?$AAE?$AAQ?$AA?5?$AA?1?$AA?5?$AAn?$AAN?$AAu?$AAm?$AA?$CJ?$AA?5?$AA?$DO?$AA?$DN?$AA?5?$AAn?$AAS?$AAi?$AAz?$AAe?$AA?$AA@ 10188de4     LIBCMTD:dbgheap.obj
 0003:0000de24       ??_C@_1DE@KOOKLFBB@?$AA_?$AAp?$AAF?$AAi?$AAr?$AAs?$AAt?$AAB?$AAl?$AAo?$AAc?$AAk?$AA?5?$AA?$DN?$AA?$DN?$AA?5?$AAp?$AAO?$AAl?$AAd?$AAB?$AAl?$AAo?$AAc?$AAk?$AA?$AA@ 10188e24     LIBCMTD:dbgheap.obj
 0003:0000de58       ??_C@_1DC@GEFKNOOL@?$AA_?$AAp?$AAL?$AAa?$AAs?$AAt?$AAB?$AAl?$AAo?$AAc?$AAk?$AA?5?$AA?$DN?$AA?$DN?$AA?5?$AAp?$AAO?$AAl?$AAd?$AAB?$AAl?$AAo?$AAc?$AAk?$AA?$AA@ 10188e58     LIBCMTD:dbgheap.obj
 0003:0000de90       ??_C@_1GE@PCKLOLAO@?$AAf?$AAR?$AAe?$AAa?$AAl?$AAl?$AAo?$AAc?$AA?5?$AA?$HM?$AA?$HM?$AA?5?$AA?$CI?$AA?$CB?$AAf?$AAR?$AAe?$AAa?$AAl?$AAl?$AAo?$AAc?$AA?5?$AA?$CG?$AA?$CG?$AA?5?$AAp?$AAN?$AAe?$AAw?$AAB?$AAl@ 10188e90     LIBCMTD:dbgheap.obj
 0003:0000def4       ??_C@_0DA@HFBKENN@Error?3?5possible?5heap?5corruption?5@ 10188ef4     LIBCMTD:dbgheap.obj
 0003:0000df28       ??_C@_1IK@DCPKDGNH@?$AAp?$AAO?$AAl?$AAd?$AAB?$AAl?$AAo?$AAc?$AAk?$AA?9?$AA?$DO?$AAn?$AAL?$AAi?$AAn?$AAe?$AA?5?$AA?$DN?$AA?$DN?$AA?5?$AAI?$AAG?$AAN?$AAO?$AAR?$AAE?$AA_?$AAL?$AAI?$AAN?$AAE?$AA?5@ 10188f28     LIBCMTD:dbgheap.obj
 0003:0000dfb8       ??_C@_1EE@GFOPCECE@?$AA_?$AAC?$AAr?$AAt?$AAI?$AAs?$AAV?$AAa?$AAl?$AAi?$AAd?$AAH?$AAe?$AAa?$AAp?$AAP?$AAo?$AAi?$AAn?$AAt?$AAe?$AAr?$AA?$CI?$AAp?$AAU?$AAs?$AAe?$AAr?$AAD?$AAa?$AAt?$AAa@ 10188fb8     LIBCMTD:dbgheap.obj
 0003:0000e000       ??_C@_0EM@LGFLMAGJ@The?5Block?5at?50x?$CFp?5was?5allocated?5@ 10189000     LIBCMTD:dbgheap.obj
 0003:0000e050       ??_C@_0FA@EFEIGJKG@Error?3?5memory?5allocation?3?5bad?5me@ 10189050     LIBCMTD:dbgheap.obj
 0003:0000e0a0       ??_C@_0ED@GPCPBAGP@Invalid?5allocation?5size?3?5?$CFIu?5byt@ 101890a0     LIBCMTD:dbgheap.obj
 0003:0000e0e4       ??_C@_0CE@DOFMDOL@Client?5hook?5re?9allocation?5failur@ 101890e4     LIBCMTD:dbgheap.obj
 0003:0000e108       ??_C@_0DI@KKJPDPGM@Client?5hook?5re?9allocation?5failur@ 10189108     LIBCMTD:dbgheap.obj
 0003:0000e140       ??_C@_1BM@OKFKJCEN@?$AA_?$AAr?$AAe?$AAc?$AAa?$AAl?$AAl?$AAo?$AAc?$AA_?$AAd?$AAb?$AAg?$AA?$AA@ 10189140     LIBCMTD:dbgheap.obj
 0003:0000e15c       ??_C@_1DO@GOKJCEHJ@?$AA?$CI?$AA_?$AAH?$AAE?$AAA?$AAP?$AA_?$AAM?$AAA?$AAX?$AAR?$AAE?$AAQ?$AA?5?$AA?1?$AA?5?$AAc?$AAo?$AAu?$AAn?$AAt?$AA?$CJ?$AA?5?$AA?$DO?$AA?$DN?$AA?5?$AAs?$AAi?$AAz?$AAe?$AA?$AA@ 1018915c     LIBCMTD:dbgheap.obj
 0003:0000e19c       ??_C@_1BI@HAPNGHDP@?$AA_?$AAe?$AAx?$AAp?$AAa?$AAn?$AAd?$AA_?$AAd?$AAb?$AAg?$AA?$AA@ 1018919c     LIBCMTD:dbgheap.obj
 0003:0000e1b4       ??_C@_1CE@CJACEFBA@?$AAp?$AAU?$AAs?$AAe?$AAr?$AAD?$AAa?$AAt?$AAa?$AA?5?$AA?$CB?$AA?$DN?$AA?5?$AAN?$AAU?$AAL?$AAL?$AA?$AA@ 101891b4     LIBCMTD:dbgheap.obj
 0003:0000e1d8       ??_C@_1CM@MMAADDMD@?$AA_?$AAp?$AAF?$AAi?$AAr?$AAs?$AAt?$AAB?$AAl?$AAo?$AAc?$AAk?$AA?5?$AA?$DN?$AA?$DN?$AA?5?$AAp?$AAH?$AAe?$AAa?$AAd?$AA?$AA@ 101891d8     LIBCMTD:dbgheap.obj
 0003:0000e204       ??_C@_1CK@DMAGEMBG@?$AA_?$AAp?$AAL?$AAa?$AAs?$AAt?$AAB?$AAl?$AAo?$AAc?$AAk?$AA?5?$AA?$DN?$AA?$DN?$AA?5?$AAp?$AAH?$AAe?$AAa?$AAd?$AA?$AA@ 10189204     LIBCMTD:dbgheap.obj
 0003:0000e230       ??_C@_1DM@ODCJIDCP@?$AAp?$AAH?$AAe?$AAa?$AAd?$AA?9?$AA?$DO?$AAn?$AAB?$AAl?$AAo?$AAc?$AAk?$AAU?$AAs?$AAe?$AA?5?$AA?$DN?$AA?$DN?$AA?5?$AAn?$AAB?$AAl?$AAo?$AAc?$AAk?$AAU?$AAs?$AAe?$AA?$AA@ 10189230     LIBCMTD:dbgheap.obj
 0003:0000e270       ??_C@_1HK@HPCBMDFG@?$AAp?$AAH?$AAe?$AAa?$AAd?$AA?9?$AA?$DO?$AAn?$AAL?$AAi?$AAn?$AAe?$AA?5?$AA?$DN?$AA?$DN?$AA?5?$AAI?$AAG?$AAN?$AAO?$AAR?$AAE?$AA_?$AAL?$AAI?$AAN?$AAE?$AA?5?$AA?$CG?$AA?$CG?$AA?5?$AAp@ 10189270     LIBCMTD:dbgheap.obj
 0003:0000e2f0       ??_C@_0IG@LEMBDCJK@HEAP?5CORRUPTION?5DETECTED?3?5after?5@ 101892f0     LIBCMTD:dbgheap.obj
 0003:0000e378       ??_C@_0KE@MBMNHHHN@HEAP?5CORRUPTION?5DETECTED?3?5after?5@ 10189378     LIBCMTD:dbgheap.obj
 0003:0000e420       ??_C@_0IK@PJCGLBOB@HEAP?5CORRUPTION?5DETECTED?3?5before@ 10189420     LIBCMTD:dbgheap.obj
 0003:0000e4b0       ??_C@_0KI@JGFOHMEB@HEAP?5CORRUPTION?5DETECTED?3?5before@ 101894b0     LIBCMTD:dbgheap.obj
 0003:0000e558       ??_C@_0BL@KEIPLFAC@Client?5hook?5free?5failure?4?6?$AA@ 10189558     LIBCMTD:dbgheap.obj
 0003:0000e578       ??_C@_0EJ@HEIBCIMJ@The?5Block?5at?50x?$CFp?5was?5allocated?5@ 10189578     LIBCMTD:dbgheap.obj
 0003:0000e5c4       ??_C@_1BG@MBKOGDLD@?$AA_?$AAm?$AAs?$AAi?$AAz?$AAe?$AA_?$AAd?$AAb?$AAg?$AA?$AA@ 101895c4     LIBCMTD:dbgheap.obj
 0003:0000e5dc       ??_C@_0CI@JMLBEDHJ@?$CFhs?5located?5at?50x?$CFp?5is?5?$CFIu?5bytes@ 101895dc     LIBCMTD:dbgheap.obj
 0003:0000e608       ??_C@_0EG@DGJMPDBH@?$CFhs?5located?5at?50x?$CFp?5is?5?$CFIu?5bytes@ 10189608     LIBCMTD:dbgheap.obj
 0003:0000e650       ??_C@_0IC@BBJIOOJH@HEAP?5CORRUPTION?5DETECTED?3?5on?5top@ 10189650     LIBCMTD:dbgheap.obj
 0003:0000e6d8       ??_C@_0KA@IHNJJKPL@HEAP?5CORRUPTION?5DETECTED?3?5on?5top@ 101896d8     LIBCMTD:dbgheap.obj
 0003:0000e778       ??_C@_07OHKEFPKJ@DAMAGED?$AA@ 10189778     LIBCMTD:dbgheap.obj
 0003:0000e780       ??_C@_0CL@HNNNMKMJ@_heapchk?5fails?5with?5unknown?5retu@ 10189780     LIBCMTD:dbgheap.obj
 0003:0000e7ac       ??_C@_0CC@MFFCHFHO@_heapchk?5fails?5with?5_HEAPBADPTR?4@ 101897ac     LIBCMTD:dbgheap.obj
 0003:0000e7d0       ??_C@_0CC@MJGLGBDG@_heapchk?5fails?5with?5_HEAPBADEND?4@ 101897d0     LIBCMTD:dbgheap.obj
 0003:0000e7f4       ??_C@_0CD@CPKEAPBD@_heapchk?5fails?5with?5_HEAPBADNODE@ 101897f4     LIBCMTD:dbgheap.obj
 0003:0000e818       ??_C@_0CE@MKKHMBMK@_heapchk?5fails?5with?5_HEAPBADBEGI@ 10189818     LIBCMTD:dbgheap.obj
 0003:0000e83c       ??_C@_1BO@GJFDNMNF@?$AA_?$AAC?$AAr?$AAt?$AAS?$AAe?$AAt?$AAD?$AAb?$AAg?$AAF?$AAl?$AAa?$AAg?$AA?$AA@ 1018983c     LIBCMTD:dbgheap.obj
 0003:0000e860       ??_C@_1BHO@NNANJNF@?$AA?$CI?$AAf?$AAN?$AAe?$AAw?$AAB?$AAi?$AAt?$AAs?$AA?$DN?$AA?$DN?$AA_?$AAC?$AAR?$AAT?$AAD?$AAB?$AAG?$AA_?$AAR?$AAE?$AAP?$AAO?$AAR?$AAT?$AA_?$AAF?$AAL?$AAA?$AAG?$AA?$CJ?$AA?5@ 10189860     LIBCMTD:dbgheap.obj
 0003:0000e9e0       ??_C@_1DE@GJCKCKEC@?$AA_?$AAC?$AAr?$AAt?$AAD?$AAo?$AAF?$AAo?$AAr?$AAA?$AAl?$AAl?$AAC?$AAl?$AAi?$AAe?$AAn?$AAt?$AAO?$AAb?$AAj?$AAe?$AAc?$AAt?$AAs?$AA?$AA@ 101899e0     LIBCMTD:dbgheap.obj
 0003:0000ea14       ??_C@_1BI@CJGCEEDL@?$AAp?$AAf?$AAn?$AA?5?$AA?$CB?$AA?$DN?$AA?5?$AAN?$AAU?$AAL?$AAL?$AA?$AA@ 10189a14     LIBCMTD:dbgheap.obj
 0003:0000ea2c       ??_C@_0CB@EAAIGELO@Bad?5memory?5block?5found?5at?50x?$CFp?4?6@ 10189a2c     LIBCMTD:dbgheap.obj
 0003:0000ea50       ??_C@_0DP@LEFMFBOD@Bad?5memory?5block?5found?5at?50x?$CFp?4?6@ 10189a50     LIBCMTD:dbgheap.obj
 0003:0000ea90       ??_C@_1CE@NJJKELF@?$AA_?$AAC?$AAr?$AAt?$AAM?$AAe?$AAm?$AAC?$AAh?$AAe?$AAc?$AAk?$AAp?$AAo?$AAi?$AAn?$AAt?$AA?$AA@ 10189a90     LIBCMTD:dbgheap.obj
 0003:0000eab4       ??_C@_1BM@MIMANDHC@?$AAs?$AAt?$AAa?$AAt?$AAe?$AA?5?$AA?$CB?$AA?$DN?$AA?5?$AAN?$AAU?$AAL?$AAL?$AA?$AA@ 10189ab4     LIBCMTD:dbgheap.obj
 0003:0000ead0       ??_C@_1CC@DFPEDFBP@?$AAn?$AAe?$AAw?$AAS?$AAt?$AAa?$AAt?$AAe?$AA?5?$AA?$CB?$AA?$DN?$AA?5?$AAN?$AAU?$AAL?$AAL?$AA?$AA@ 10189ad0     LIBCMTD:dbgheap.obj
 0003:0000eaf4       ??_C@_1CC@DHPFEMMN@?$AAo?$AAl?$AAd?$AAS?$AAt?$AAa?$AAt?$AAe?$AA?5?$AA?$CB?$AA?$DN?$AA?5?$AAN?$AAU?$AAL?$AAL?$AA?$AA@ 10189af4     LIBCMTD:dbgheap.obj
 0003:0000eb18       ??_C@_1CE@PDIENACM@?$AA_?$AAC?$AAr?$AAt?$AAM?$AAe?$AAm?$AAD?$AAi?$AAf?$AAf?$AAe?$AAr?$AAe?$AAn?$AAc?$AAe?$AA?$AA@ 10189b18     LIBCMTD:dbgheap.obj
 0003:0000eb3c       ??_C@_0BH@GFGKJDCO@Object?5dump?5complete?4?6?$AA@ 10189b3c     LIBCMTD:dbgheap.obj
 0003:0000eb54       ??_C@_0DA@MDLBNIBM@crt?5block?5at?50x?$CFp?0?5subtype?5?$CFx?0?5?$CF@ 10189b54     LIBCMTD:dbgheap.obj
 0003:0000eb84       ??_C@_0CH@FAGDDGPN@normal?5block?5at?50x?$CFp?0?5?$CFIu?5bytes?5@ 10189b84     LIBCMTD:dbgheap.obj
 0003:0000ebac       ??_C@_0DD@GHNAAKBB@client?5block?5at?50x?$CFp?0?5subtype?5?$CFx@ 10189bac     LIBCMTD:dbgheap.obj
 0003:0000ebe0       ??_C@_06PKLGBFGM@?$HL?$CFld?$HN?5?$AA@ 10189be0     LIBCMTD:dbgheap.obj
 0003:0000ebe8       ??_C@_0L@JMEFFCCJ@?$CFhs?$CI?$CFd?$CJ?5?3?5?$AA@ 10189be8     LIBCMTD:dbgheap.obj
 0003:0000ebf4       ??_C@_0BE@OIEFNFL@?$CDFile?5Error?$CD?$CI?$CFd?$CJ?5?3?5?$AA@ 10189bf4     LIBCMTD:dbgheap.obj
 0003:0000ec08       ??_C@_0BE@KCIPKCIA@Dumping?5objects?5?9?$DO?6?$AA@ 10189c08     LIBCMTD:dbgheap.obj
 0003:0000ec1c       ??_C@_0BA@HJBKCELP@?5Data?3?5?$DM?$CFs?$DO?5?$CFs?6?$AA@ 10189c1c     LIBCMTD:dbgheap.obj
 0003:0000ec2c       ??_C@_1CG@LPFIACGM@?$AA_?$AAp?$AAr?$AAi?$AAn?$AAt?$AAM?$AAe?$AAm?$AAB?$AAl?$AAo?$AAc?$AAk?$AAD?$AAa?$AAt?$AAa?$AA?$AA@ 10189c2c     LIBCMTD:dbgheap.obj
 0003:0000ec54       ??_C@_0BI@JBFPOEJA@Detected?5memory?5leaks?$CB?6?$AA@ 10189c54     LIBCMTD:dbgheap.obj
 0003:0000ec6c       ??_C@_0BP@DEDHGGGI@Total?5allocations?3?5?$CFId?5bytes?4?6?$AA@ 10189c6c     LIBCMTD:dbgheap.obj
 0003:0000ec8c       ??_C@_0CB@BLHDAFNE@Largest?5number?5used?3?5?$CFId?5bytes?4?6@ 10189c8c     LIBCMTD:dbgheap.obj
 0003:0000ecb0       ??_C@_0BO@DACNIABB@?$CFId?5bytes?5in?5?$CFId?5?$CFhs?5Blocks?4?6?$AA@ 10189cb0     LIBCMTD:dbgheap.obj
 0003:0000ecd0       ??_C@_1CM@MPNIBKGK@?$AA_?$AAC?$AAr?$AAt?$AAM?$AAe?$AAm?$AAD?$AAu?$AAm?$AAp?$AAS?$AAt?$AAa?$AAt?$AAi?$AAs?$AAt?$AAi?$AAc?$AAs?$AA?$AA@ 10189cd0     LIBCMTD:dbgheap.obj
 0003:0000ecfc       ??_C@_1DK@LFLKFPDA@?$AAo?$AAf?$AAf?$AAs?$AAe?$AAt?$AA?5?$AA?$DN?$AA?$DN?$AA?5?$AA0?$AA?5?$AA?$HM?$AA?$HM?$AA?5?$AAo?$AAf?$AAf?$AAs?$AAe?$AAt?$AA?5?$AA?$DM?$AA?5?$AAs?$AAi?$AAz?$AAe?$AA?$AA@ 10189cfc     LIBCMTD:dbgheap.obj
 0003:0000ed38       ??_C@_1DG@DONCJBBJ@?$AA_?$AAa?$AAl?$AAi?$AAg?$AAn?$AAe?$AAd?$AA_?$AAo?$AAf?$AAf?$AAs?$AAe?$AAt?$AA_?$AAm?$AAa?$AAl?$AAl?$AAo?$AAc?$AA_?$AAd?$AAb?$AAg?$AA?$AA@ 10189d38     LIBCMTD:dbgheap.obj
 0003:0000ed70       ??_C@_1CE@NPMGPNNP@?$AAI?$AAS?$AA_?$AA2?$AA_?$AAP?$AAO?$AAW?$AA_?$AAN?$AA?$CI?$AAa?$AAl?$AAi?$AAg?$AAn?$AA?$CJ?$AA?$AA@ 10189d70     LIBCMTD:dbgheap.obj
 0003:0000ed94       ??_C@_1DI@NINIKFFK@?$AA_?$AAa?$AAl?$AAi?$AAg?$AAn?$AAe?$AAd?$AA_?$AAo?$AAf?$AAf?$AAs?$AAe?$AAt?$AA_?$AAr?$AAe?$AAa?$AAl?$AAl?$AAo?$AAc?$AA_?$AAd?$AAb?$AAg?$AA?$AA@ 10189d94     LIBCMTD:dbgheap.obj
 0003:0000edcc       ??_C@_0DL@PGHMMKNE@Damage?5before?50x?$CFp?5which?5was?5all@ 10189dcc     LIBCMTD:dbgheap.obj
 0003:0000ee08       ??_C@_0EI@NDNJMAJK@The?5block?5at?50x?$CFp?5was?5not?5alloca@ 10189e08     LIBCMTD:dbgheap.obj
 0003:0000ee50       ??_C@_1DK@MMLHIFFH@?$AA_?$AAa?$AAl?$AAi?$AAg?$AAn?$AAe?$AAd?$AA_?$AAo?$AAf?$AAf?$AAs?$AAe?$AAt?$AA_?$AAr?$AAe?$AAc?$AAa?$AAl?$AAl?$AAo?$AAc?$AA_?$AAd?$AAb?$AAg?$AA?$AA@ 10189e50     LIBCMTD:dbgheap.obj
 0003:0000ee90       ??_C@_0EF@PGELACII@The?5block?5at?50x?$CFp?5was?5not?5alloca@ 10189e90     LIBCMTD:dbgheap.obj
 0003:0000eed8       ??_C@_1CG@CEGMHIMN@?$AA_?$AAa?$AAl?$AAi?$AAg?$AAn?$AAe?$AAd?$AA_?$AAm?$AAs?$AAi?$AAz?$AAe?$AA_?$AAd?$AAb?$AAg?$AA?$AA@ 10189ed8     LIBCMTD:dbgheap.obj
 0003:0000ef00       ??_C@_1CC@MOBIKHH@?$AAm?$AAe?$AAm?$AAb?$AAl?$AAo?$AAc?$AAk?$AA?5?$AA?$CB?$AA?$DN?$AA?5?$AAN?$AAU?$AAL?$AAL?$AA?$AA@ 10189f00     LIBCMTD:dbgheap.obj
 0003:0000ef24       __pDefaultRawDllMain       10189f24     LIBCMTD:dllcrt0.obj
 0003:0000ef24       __pRawDllMain              10189f24     LIBCMTD:dllcrt0.obj
 0003:0000ef28       ??_C@_0DB@OLNOAEGF@f?3?2dd?2vctools?2crt_bld?2self_x86?2c@ 10189f28     LIBCMTD:dllcrt0.obj
 0003:0000ef60       ??_C@_1BAA@ODEGEDCK@?$AA?$CI?$AA?5?$AA?$CI?$AA_?$AAS?$AAt?$AAr?$AAe?$AAa?$AAm?$AA?9?$AA?$DO?$AA_?$AAf?$AAl?$AAa?$AAg?$AA?5?$AA?$CG?$AA?5?$AA_?$AAI?$AAO?$AAS?$AAT?$AAR?$AAG?$AA?$CJ?$AA?5?$AA?$HM?$AA?$HM?$AA?5@ 10189f60     LIBCMTD:fputs.obj
 0003:0000f060       ??_C@_1M@LIIFKKLB@?$AAf?$AAp?$AAu?$AAt?$AAs?$AA?$AA@ 1018a060     LIBCMTD:fputs.obj
 0003:0000f070       ??_C@_1FO@FFFEAAEI@?$AAf?$AA?3?$AA?2?$AAd?$AAd?$AA?2?$AAv?$AAc?$AAt?$AAo?$AAo?$AAl?$AAs?$AA?2?$AAc?$AAr?$AAt?$AA_?$AAb?$AAl?$AAd?$AA?2?$AAs?$AAe?$AAl?$AAf?$AA_?$AAx?$AA8?$AA6?$AA?2?$AAc@ 1018a070     LIBCMTD:fputs.obj
 0003:0000f0d0       ??_C@_0CP@BNKDODJJ@f?3?2dd?2vctools?2crt_bld?2self_x86?2c@ 1018a0d0     LIBCMTD:_file.obj
 0003:0000f150       ??_C@_1BA@DNOHIGNM@?$AAf?$AAp?$AAr?$AAi?$AAn?$AAt?$AAf?$AA?$AA@ 1018a150     LIBCMTD:fprintf.obj
 0003:0000f160       ??_C@_1GC@NHJDDBOH@?$AAf?$AA?3?$AA?2?$AAd?$AAd?$AA?2?$AAv?$AAc?$AAt?$AAo?$AAo?$AAl?$AAs?$AA?2?$AAc?$AAr?$AAt?$AA_?$AAb?$AAl?$AAd?$AA?2?$AAs?$AAe?$AAl?$AAf?$AA_?$AAx?$AA8?$AA6?$AA?2?$AAc@ 1018a160     LIBCMTD:fprintf.obj
 0003:0000f1c4       ??_C@_02LMMGGCAJ@?3?5?$AA@ 1018a1c4     LIBCMTD:perror.obj
 0003:0000f218       ??_C@_1BK@HJGMBFLF@?$AAc?$AAo?$AAm?$AAp?$AA?5?$AA?$CB?$AA?$DN?$AA?5?$AAN?$AAU?$AAL?$AAL?$AA?$AA@ 1018a218     LIBCMTD:qsort.obj
 0003:0000f234       ??_C@_1BE@NJBEBBME@?$AAw?$AAi?$AAd?$AAt?$AAh?$AA?5?$AA?$DO?$AA?5?$AA0?$AA?$AA@ 1018a234     LIBCMTD:qsort.obj
 0003:0000f248       ??_C@_1M@INMHODIG@?$AAq?$AAs?$AAo?$AAr?$AAt?$AA?$AA@ 1018a248     LIBCMTD:qsort.obj
 0003:0000f258       ??_C@_1FO@NDBPJPLL@?$AAf?$AA?3?$AA?2?$AAd?$AAd?$AA?2?$AAv?$AAc?$AAt?$AAo?$AAo?$AAl?$AAs?$AA?2?$AAc?$AAr?$AAt?$AA_?$AAb?$AAl?$AAd?$AA?2?$AAs?$AAe?$AAl?$AAf?$AA_?$AAx?$AA8?$AA6?$AA?2?$AAc@ 1018a258     LIBCMTD:qsort.obj
 0003:0000f2b8       ??_C@_1DC@HAGCIKOA@?$AAb?$AAa?$AAs?$AAe?$AA?5?$AA?$CB?$AA?$DN?$AA?5?$AAN?$AAU?$AAL?$AAL?$AA?5?$AA?$HM?$AA?$HM?$AA?5?$AAn?$AAu?$AAm?$AA?5?$AA?$DN?$AA?$DN?$AA?5?$AA0?$AA?$AA@ 1018a2b8     LIBCMTD:qsort.obj
 0003:0000f2ec       ??_C@_0P@MIGLKIOC@CorExitProcess?$AA@ 1018a2ec     LIBCMTD:crt0dat.obj
 0003:0000f2fc       ??_C@_1BI@BGOHAHKC@?$AAm?$AAs?$AAc?$AAo?$AAr?$AAe?$AAe?$AA?4?$AAd?$AAl?$AAl?$AA?$AA@ 1018a2fc     LIBCMTD:crt0dat.obj
 0003:0000f314       ??_C@_1CC@CDIPMFPD@?$AA_?$AAw?$AAp?$AAg?$AAm?$AAp?$AAt?$AAr?$AA?5?$AA?$CB?$AA?$DN?$AA?5?$AAN?$AAU?$AAL?$AAL?$AA?$AA@ 1018a314     LIBCMTD:crt0dat.obj
 0003:0000f338       ??_C@_1BK@PNLDCCDP@?$AA_?$AAg?$AAe?$AAt?$AA_?$AAw?$AAp?$AAg?$AAm?$AAp?$AAt?$AAr?$AA?$AA@ 1018a338     LIBCMTD:crt0dat.obj
 0003:0000f358       ??_C@_1GC@DGCPEDNJ@?$AAf?$AA?3?$AA?2?$AAd?$AAd?$AA?2?$AAv?$AAc?$AAt?$AAo?$AAo?$AAl?$AAs?$AA?2?$AAc?$AAr?$AAt?$AA_?$AAb?$AAl?$AAd?$AA?2?$AAs?$AAe?$AAl?$AAf?$AA_?$AAx?$AA8?$AA6?$AA?2?$AAc@ 1018a358     LIBCMTD:crt0dat.obj
 0003:0000f3bc       ??_C@_1CA@BBNAFCKO@?$AA_?$AAp?$AAg?$AAm?$AAp?$AAt?$AAr?$AA?5?$AA?$CB?$AA?$DN?$AA?5?$AAN?$AAU?$AAL?$AAL?$AA?$AA@ 1018a3bc     LIBCMTD:crt0dat.obj
 0003:0000f3dc       ??_C@_1BI@COAAPHJK@?$AA_?$AAg?$AAe?$AAt?$AA_?$AAp?$AAg?$AAm?$AAp?$AAt?$AAr?$AA?$AA@ 1018a3dc     LIBCMTD:crt0dat.obj
 0003:0000f3f4       ??_C@_1M@KFLMCEDC@?$AAf?$AAr?$AAe?$AAx?$AAp?$AA?$AA@ 1018a3f4     LIBCMTD:_frexp_.obj
 0003:0000f400       ??_C@_1HC@HDCMDJF@?$AAf?$AA?3?$AA?2?$AAd?$AAd?$AA?2?$AAv?$AAc?$AAt?$AAo?$AAo?$AAl?$AAs?$AA?2?$AAc?$AAr?$AAt?$AA_?$AAb?$AAl?$AAd?$AA?2?$AAs?$AAe?$AAl?$AAf?$AA_?$AAx?$AA8?$AA6?$AA?2?$AAc@ 1018a400     LIBCMTD:_frexp_.obj
 0003:0000f474       ??_C@_1BO@KGGHBFPG@?$AAe?$AAx?$AAp?$AAp?$AAt?$AAr?$AA?5?$AA?$CB?$AA?$DN?$AA?5?$AAN?$AAU?$AAL?$AAL?$AA?$AA@ 1018a474     LIBCMTD:_frexp_.obj
 0003:0000f494       ??_C@_0BP@OGBCLIBO@Stack?5around?5_alloca?5corrupted?$AA@ 1018a494     LIBCMTD:_userapi_.obj
 0003:0000f4b4       ??_C@_0CK@CNLNOEPB@Local?5variable?5used?5before?5initi@ 1018a4b4     LIBCMTD:_userapi_.obj
 0003:0000f4e0       ??_C@_0BI@CIGMDCBH@Stack?5memory?5corruption?$AA@ 1018a4e0     LIBCMTD:_userapi_.obj
 0003:0000f4f8       ??_C@_0CK@FEGOIOPB@Cast?5to?5smaller?5type?5causing?5los@ 1018a4f8     LIBCMTD:_userapi_.obj
 0003:0000f524       ??_C@_0BJ@HEGAHDFO@Stack?5pointer?5corruption?$AA@ 1018a524     LIBCMTD:_userapi_.obj
 0003:0000f554       ??_C@_0DP@CBBAPGOP@f?3?2dd?2vctools?2crt_bld?2self_x86?2c@ 1018a554     LIBCMTD:chkesp.obj
 0003:0000f593       ??_C@_00CNPNBAHC@?$AA@     1018a593     LIBCMTD:chkesp.obj
 0003:0000f598       ??_C@_0NM@DNEDKLDF@The?5value?5of?5ESP?5was?5not?5properl@ 1018a598     LIBCMTD:chkesp.obj
 0003:0000f674       ??_C@_0DB@MHMEONEC@f?3?2dd?2vctools?2crt_bld?2self_x86?2c@ 1018a674     LIBCMTD:mbctype.obj
 0003:0000f6a8       ??_C@_07LCBHPJJN@LC_TIME?$AA@ 1018a6a8     LIBCMTD:setlocal.obj
 0003:0000f6b0       ??_C@_0L@DLHIECNL@LC_NUMERIC?$AA@ 1018a6b0     LIBCMTD:setlocal.obj
 0003:0000f6bc       ??_C@_0M@MIENIKLA@LC_MONETARY?$AA@ 1018a6bc     LIBCMTD:setlocal.obj
 0003:0000f6c8       ??_C@_08EADHIDAD@LC_CTYPE?$AA@ 1018a6c8     LIBCMTD:setlocal.obj
 0003:0000f6d4       ??_C@_0L@KFJHEKIK@LC_COLLATE?$AA@ 1018a6d4     LIBCMTD:setlocal.obj
 0003:0000f6e0       ??_C@_06NEFDFEKB@LC_ALL?$AA@ 1018a6e0     LIBCMTD:setlocal.obj
 0003:0000f6e8       ___lc_category             1018a6e8     LIBCMTD:setlocal.obj
 0003:0000f7b0       ??_C@_1GE@OLEIGPBJ@?$AAf?$AA?3?$AA?2?$AAd?$AAd?$AA?2?$AAv?$AAc?$AAt?$AAo?$AAo?$AAl?$AAs?$AA?2?$AAc?$AAr?$AAt?$AA_?$AAb?$AAl?$AAd?$AA?2?$AAs?$AAe?$AAl?$AAf?$AA_?$AAx?$AA8?$AA6?$AA?2?$AAc@ 1018a7b0     LIBCMTD:setlocal.obj
 0003:0000f818       ??_C@_1BKC@GGIENNAK@?$AA?$CI?$AA?$CI?$AAp?$AAt?$AAl?$AAo?$AAc?$AAi?$AA?9?$AA?$DO?$AAl?$AAc?$AA_?$AAc?$AAa?$AAt?$AAe?$AAg?$AAo?$AAr?$AAy?$AA?$FL?$AAc?$AAa?$AAt?$AAe?$AAg?$AAo?$AAr?$AAy?$AA?$FN?$AA?4@ 1018a818     LIBCMTD:setlocal.obj
 0003:0000f9bc       ??_C@_1CI@FGIONOJM@?$AA_?$AAc?$AAo?$AAn?$AAf?$AAi?$AAg?$AAt?$AAh?$AAr?$AAe?$AAa?$AAd?$AAl?$AAo?$AAc?$AAa?$AAl?$AAe?$AA?$AA@ 1018a9bc     LIBCMTD:setlocal.obj
 0003:0000f9e8       ??_C@_1GA@LDEGDKD@?$AA?$CI?$AA?$CC?$AAI?$AAn?$AAv?$AAa?$AAl?$AAi?$AAd?$AA?5?$AAp?$AAa?$AAr?$AAa?$AAm?$AAe?$AAt?$AAe?$AAr?$AA?5?$AAf?$AAo?$AAr?$AA?5?$AA_?$AAc?$AAo?$AAn?$AAf?$AAi?$AAg?$AAt@ 1018a9e8     LIBCMTD:setlocal.obj
 0003:0000fa48       ??_C@_0DC@JCPFNMID@f?3?2dd?2vctools?2crt_bld?2self_x86?2c@ 1018aa48     LIBCMTD:setlocal.obj
 0003:0000fa7c       ??_C@_1BE@DBJGBOJC@?$AAs?$AAe?$AAt?$AAl?$AAo?$AAc?$AAa?$AAl?$AAe?$AA?$AA@ 1018aa7c     LIBCMTD:setlocal.obj
 0003:0000fa90       ??_C@_1FG@OHLFEKMC@?$AAL?$AAC?$AA_?$AAM?$AAI?$AAN?$AA?5?$AA?$DM?$AA?$DN?$AA?5?$AA_?$AAc?$AAa?$AAt?$AAe?$AAg?$AAo?$AAr?$AAy?$AA?5?$AA?$CG?$AA?$CG?$AA?5?$AA_?$AAc?$AAa?$AAt?$AAe?$AAg?$AAo?$AAr?$AAy@ 1018aa90     LIBCMTD:setlocal.obj
 0003:0000fae8       ??_C@_1IA@PFIKKKFB@?$AAs?$AAt?$AAr?$AAn?$AAc?$AAp?$AAy?$AA_?$AAs?$AA?$CI?$AAl?$AAc?$AAt?$AAe?$AAm?$AAp?$AA?0?$AA?5?$AA?$CI?$AAs?$AAi?$AAz?$AAe?$AAo?$AAf?$AA?$CI?$AAl?$AAc?$AAt?$AAe?$AAm?$AAp@ 1018aae8     LIBCMTD:setlocal.obj
 0003:0000fb68       ??_C@_1CE@OFNHIOO@?$AA_?$AAs?$AAe?$AAt?$AAl?$AAo?$AAc?$AAa?$AAl?$AAe?$AA_?$AAn?$AAo?$AAl?$AAo?$AAc?$AAk?$AA?$AA@ 1018ab68     LIBCMTD:setlocal.obj
 0003:0000fb8c       ??_C@_01ICJEACDI@?$DL?$AA@ 1018ab8c     LIBCMTD:setlocal.obj
 0003:0000fb90       ??_C@_02BALPLPBG@?$DN?$DL?$AA@ 1018ab90     LIBCMTD:setlocal.obj
 0003:0000fb98       ??_C@_1GO@JALHLJEH@?$AAs?$AAt?$AAr?$AAc?$AAp?$AAy?$AA_?$AAs?$AA?$CI?$AAp?$AAc?$AAh?$AA?5?$AA?$CL?$AA?5?$AAs?$AAi?$AAz?$AAe?$AAo?$AAf?$AA?$CI?$AAi?$AAn?$AAt?$AA?$CJ?$AA?0?$AA?5?$AAc?$AAc?$AAh?$AA?5@ 1018ab98     LIBCMTD:setlocal.obj
 0003:0000fc08       ??_C@_1CG@IEFIICPK@?$AA_?$AAs?$AAe?$AAt?$AAl?$AAo?$AAc?$AAa?$AAl?$AAe?$AA_?$AAs?$AAe?$AAt?$AA_?$AAc?$AAa?$AAt?$AA?$AA@ 1018ac08     LIBCMTD:setlocal.obj
 0003:0000fc30       ??_C@_1DA@GDKKLCLM@?$AAs?$AAt?$AAr?$AAc?$AAa?$AAt?$AA_?$AAs?$AA?$CI?$AAp?$AAc?$AAh?$AA?0?$AA?5?$AAc?$AAc?$AAh?$AA?0?$AA?5?$AA?$CC?$AA?$DL?$AA?$CC?$AA?$CJ?$AA?$AA@ 1018ac30     LIBCMTD:setlocal.obj
 0003:0000fc60       ??_C@_1CG@NNFIJLDA@?$AA_?$AAs?$AAe?$AAt?$AAl?$AAo?$AAc?$AAa?$AAl?$AAe?$AA_?$AAg?$AAe?$AAt?$AA_?$AAa?$AAl?$AAl?$AA?$AA@ 1018ac60     LIBCMTD:setlocal.obj
 0003:0000fc88       ??_C@_01NEMOKFLO@?$DN?$AA@ 1018ac88     LIBCMTD:setlocal.obj
 0003:0000fc90       ??_C@_1FA@MHAOOIBO@?$AAs?$AAt?$AAr?$AAc?$AAp?$AAy?$AA_?$AAs?$AA?$CI?$AAo?$AAu?$AAt?$AAp?$AAu?$AAt?$AA?0?$AA?5?$AAs?$AAi?$AAz?$AAe?$AAI?$AAn?$AAC?$AAh?$AAa?$AAr?$AAs?$AA?0?$AA?5?$AAc?$AAa@ 1018ac90     LIBCMTD:setlocal.obj
 0003:0000fce0       ??_C@_1IA@ONNFOEDA@?$AAs?$AAt?$AAr?$AAn?$AAc?$AAp?$AAy?$AA_?$AAs?$AA?$CI?$AAc?$AAa?$AAc?$AAh?$AAe?$AAi?$AAn?$AA?0?$AA?5?$AAc?$AAa?$AAc?$AAh?$AAe?$AAi?$AAn?$AAS?$AAi?$AAz?$AAe?$AA?0?$AA?5@ 1018ace0     LIBCMTD:setlocal.obj
 0003:0000fd60       ??_C@_01GFHCPBMG@C?$AA@    1018ad60     LIBCMTD:setlocal.obj
 0003:0000fd68       ??_C@_1EG@MOMHKOD@?$AAs?$AAt?$AAr?$AAc?$AAp?$AAy?$AA_?$AAs?$AA?$CI?$AAo?$AAu?$AAt?$AAp?$AAu?$AAt?$AA?0?$AA?5?$AAs?$AAi?$AAz?$AAe?$AAI?$AAn?$AAC?$AAh?$AAa?$AAr?$AAs?$AA?0?$AA?5?$AA?$CC?$AAC@ 1018ad68     LIBCMTD:setlocal.obj
 0003:0000fdb0       ??_C@_1BM@OIIBLEFG@?$AA_?$AAe?$AAx?$AAp?$AAa?$AAn?$AAd?$AAl?$AAo?$AAc?$AAa?$AAl?$AAe?$AA?$AA@ 1018adb0     LIBCMTD:setlocal.obj
 0003:0000fdd0       ??_C@_1BGM@IJDLABMC@?$AAs?$AAt?$AAr?$AAc?$AAa?$AAt?$AA_?$AAs?$AA?$CI?$AAo?$AAu?$AAt?$AAs?$AAt?$AAr?$AA?0?$AA?5?$AAs?$AAi?$AAz?$AAe?$AAI?$AAn?$AAB?$AAy?$AAt?$AAe?$AAs?$AA?0?$AA?5?$AA?$CI?$AA?5@ 1018add0     LIBCMTD:setlocal.obj
 0003:0000ff3c       ??_C@_1BC@PIABMDIP@?$AA_?$AAs?$AAt?$AAr?$AAc?$AAa?$AAt?$AAs?$AA?$AA@ 1018af3c     LIBCMTD:setlocal.obj
 0003:0000ff50       ??_C@_1MM@NOPMGFHF@?$AAs?$AAt?$AAr?$AAn?$AAc?$AAp?$AAy?$AA_?$AAs?$AA?$CI?$AAn?$AAa?$AAm?$AAe?$AAs?$AA?9?$AA?$DO?$AAs?$AAz?$AAC?$AAo?$AAd?$AAe?$AAP?$AAa?$AAg?$AAe?$AA?0?$AA?5?$AA?$CI?$AAs?$AAi@ 1018af50     LIBCMTD:setlocal.obj
 0003:00010020       ??_C@_1MG@PHNILIAG@?$AAs?$AAt?$AAr?$AAn?$AAc?$AAp?$AAy?$AA_?$AAs?$AA?$CI?$AAn?$AAa?$AAm?$AAe?$AAs?$AA?9?$AA?$DO?$AAs?$AAz?$AAC?$AAo?$AAu?$AAn?$AAt?$AAr?$AAy?$AA?0?$AA?5?$AA?$CI?$AAs?$AAi?$AAz@ 1018b020     LIBCMTD:setlocal.obj
 0003:000100e8       ??_C@_1MM@BFEECMAF@?$AAs?$AAt?$AAr?$AAn?$AAc?$AAp?$AAy?$AA_?$AAs?$AA?$CI?$AAn?$AAa?$AAm?$AAe?$AAs?$AA?9?$AA?$DO?$AAs?$AAz?$AAL?$AAa?$AAn?$AAg?$AAu?$AAa?$AAg?$AAe?$AA?0?$AA?5?$AA?$CI?$AAs?$AAi@ 1018b0e8     LIBCMTD:setlocal.obj
 0003:000101b4       ??_C@_03EGDHDPFD@_?4?0?$AA@ 1018b1b4     LIBCMTD:setlocal.obj
 0003:000101b8       ??_C@_1NG@FMOPGKGG@?$AAs?$AAt?$AAr?$AAn?$AAc?$AAp?$AAy?$AA_?$AAs?$AA?$CI?$AAn?$AAa?$AAm?$AAe?$AAs?$AA?9?$AA?$DO?$AAs?$AAz?$AAC?$AAo?$AAd?$AAe?$AAP?$AAa?$AAg?$AAe?$AA?0?$AA?5?$AA?$CI?$AAs?$AAi@ 1018b1b8     LIBCMTD:setlocal.obj
 0003:00010290       ??_C@_1BK@CBMMLAGJ@?$AA_?$AA_?$AAl?$AAc?$AA_?$AAs?$AAt?$AAr?$AAt?$AAo?$AAl?$AAc?$AA?$AA@ 1018b290     LIBCMTD:setlocal.obj
 0003:000102ac       ??_C@_01LFCBOECM@?4?$AA@   1018b2ac     LIBCMTD:setlocal.obj
 0003:000102b0       ??_C@_01IDAFKMJL@_?$AA@    1018b2b0     LIBCMTD:setlocal.obj
 0003:000102b8       ??_C@_1HC@IBDBLKCB@?$AAs?$AAt?$AAr?$AAc?$AAp?$AAy?$AA_?$AAs?$AA?$CI?$AAl?$AAo?$AAc?$AAa?$AAl?$AAe?$AA?0?$AA?5?$AAs?$AAi?$AAz?$AAe?$AAI?$AAn?$AAB?$AAy?$AAt?$AAe?$AAs?$AA?0?$AA?5?$AA?$CI?$AAc@ 1018b2b8     LIBCMTD:setlocal.obj
 0003:0001032c       ??_C@_1BK@FGDJDEPG@?$AA_?$AA_?$AAl?$AAc?$AA_?$AAl?$AAc?$AAt?$AAo?$AAs?$AAt?$AAr?$AA?$AA@ 1018b32c     LIBCMTD:setlocal.obj
 0003:00010348       ??_C@_0O@NLDKAIKN@EncodePointer?$AA@ 1018b348     LIBCMTD:tidtable.obj
 0003:00010358       ??_C@_1BK@DBDEIDLH@?$AAK?$AAE?$AAR?$AAN?$AAE?$AAL?$AA3?$AA2?$AA?4?$AAD?$AAL?$AAL?$AA?$AA@ 1018b358     LIBCMTD:tidtable.obj
 0003:00010374       ??_C@_0O@KBPMFGHI@DecodePointer?$AA@ 1018b374     LIBCMTD:tidtable.obj
 0003:00010384       ??_C@_0DC@LMJHGCKC@f?3?2dd?2vctools?2crt_bld?2self_x86?2c@ 1018b384     LIBCMTD:tidtable.obj
 0003:000103b8       ??_C@_07PEJMOBNF@FlsFree?$AA@ 1018b3b8     LIBCMTD:tidtable.obj
 0003:000103c0       ??_C@_0M@JCPCPOEF@FlsSetValue?$AA@ 1018b3c0     LIBCMTD:tidtable.obj
 0003:000103cc       ??_C@_0M@GDNOONDI@FlsGetValue?$AA@ 1018b3cc     LIBCMTD:tidtable.obj
 0003:000103d8       ??_C@_08KNHFBNJ@FlsAlloc?$AA@ 1018b3d8     LIBCMTD:tidtable.obj
 0003:000103f0       ??_C@_1GE@KOCFNGPB@?$AA_?$AAc?$AAo?$AAn?$AAt?$AAr?$AAo?$AAl?$AAf?$AAp?$AA_?$AAs?$AA?$CI?$AA?$CI?$AA?$CI?$AAv?$AAo?$AAi?$AAd?$AA?5?$AA?$CK?$AA?$CJ?$AA0?$AA?$CJ?$AA?0?$AA?5?$AA0?$AAx?$AA0?$AA0?$AA0?$AA1@ 1018b3f0     LIBCMTD:fp8.obj
 0003:00010454       ??_C@_1CK@JMKHCBEI@?$AA_?$AAs?$AAe?$AAt?$AAd?$AAe?$AAf?$AAa?$AAu?$AAl?$AAt?$AAp?$AAr?$AAe?$AAc?$AAi?$AAs?$AAi?$AAo?$AAn?$AA?$AA@ 1018b454     LIBCMTD:fp8.obj
 0003:00010480       ??_C@_1GG@PHGJJHBC@?$AAf?$AA?3?$AA?2?$AAd?$AAd?$AA?2?$AAv?$AAc?$AAt?$AAo?$AAo?$AAl?$AAs?$AA?2?$AAc?$AAr?$AAt?$AA_?$AAb?$AAl?$AAd?$AA?2?$AAs?$AAe?$AAl?$AAf?$AA_?$AAx?$AA8?$AA6?$AA?2?$AAc@ 1018b480     LIBCMTD:fp8.obj
 0003:000104e8       __real@4150017ec0000000    1018b4e8     LIBCMTD:_testfdiv_.obj
 0003:000104f0       __real@4147ffff80000000    1018b4f0     LIBCMTD:_testfdiv_.obj
 0003:000104f8       ??_C@_0BK@NHEOCAHP@IsProcessorFeaturePresent?$AA@ 1018b4f8     LIBCMTD:_testfdiv_.obj
 0003:00010514       ??_C@_08CPNIBGIE@KERNEL32?$AA@ 1018b514     LIBCMTD:_testfdiv_.obj
 0003:00010520       ??_C@_1CA@CBMNPEO@?$AAs?$AAi?$AAz?$AAe?$AAI?$AAn?$AAB?$AAy?$AAt?$AAe?$AAs?$AA?5?$AA?$DO?$AA?5?$AA0?$AA?$AA@ 1018b520     LIBCMTD:cvt.obj
 0003:00010540       ??_C@_1BC@INKAPMHI@?$AA_?$AAc?$AAf?$AAt?$AAo?$AAe?$AA_?$AAl?$AA?$AA@ 1018b540     LIBCMTD:cvt.obj
 0003:00010558       ??_C@_1GO@NCCGBNKI@?$AAf?$AA?3?$AA?2?$AAd?$AAd?$AA?2?$AAv?$AAc?$AAt?$AAo?$AAo?$AAl?$AAs?$AA?2?$AAc?$AAr?$AAt?$AA_?$AAb?$AAl?$AAd?$AA?2?$AAs?$AAe?$AAl?$AAf?$AA_?$AAx?$AA8?$AA6?$AA?2?$AAc@ 1018b558     LIBCMTD:cvt.obj
 0003:000105c8       ??_C@_1BI@ICGGMGLK@?$AAb?$AAu?$AAf?$AA?5?$AA?$CB?$AA?$DN?$AA?5?$AAN?$AAU?$AAL?$AAL?$AA?$AA@ 1018b5c8     LIBCMTD:cvt.obj
 0003:000105e0       ??_C@_05KLBDPFGC@e?$CL000?$AA@ 1018b5e0     LIBCMTD:cvt.obj
 0003:000105e8       ??_C@_1LE@EOIFGNCJ@?$AAs?$AAt?$AAr?$AAc?$AAp?$AAy?$AA_?$AAs?$AA?$CI?$AAp?$AA?0?$AA?5?$AA?$CI?$AAs?$AAi?$AAz?$AAe?$AAI?$AAn?$AAB?$AAy?$AAt?$AAe?$AAs?$AA?5?$AA?$DN?$AA?$DN?$AA?5?$AA?$CI?$AAs?$AAi?$AAz@ 1018b5e8     LIBCMTD:cvt.obj
 0003:000106a0       ??_C@_1HE@NACBNDPP@?$AAs?$AAi?$AAz?$AAe?$AAI?$AAn?$AAB?$AAy?$AAt?$AAe?$AAs?$AA?5?$AA?$DO?$AA?5?$AA?$CI?$AAs?$AAi?$AAz?$AAe?$AA_?$AAt?$AA?$CJ?$AA?$CI?$AA3?$AA?5?$AA?$CL?$AA?5?$AA?$CI?$AAn?$AAd?$AAe?$AAc@ 1018b6a0     LIBCMTD:cvt.obj
 0003:00010714       ??_C@_1BE@OLBNEILL@?$AA_?$AAc?$AAf?$AAt?$AAo?$AAe?$AA2?$AA_?$AAl?$AA?$AA@ 1018b714     LIBCMTD:cvt.obj
 0003:00010728       ??_C@_1FC@IKIMAMJB@?$AAs?$AAi?$AAz?$AAe?$AAI?$AAn?$AAB?$AAy?$AAt?$AAe?$AAs?$AA?5?$AA?$DO?$AA?5?$AA?$CI?$AAs?$AAi?$AAz?$AAe?$AA_?$AAt?$AA?$CJ?$AA?$CI?$AA1?$AA?5?$AA?$CL?$AA?5?$AA4?$AA?5?$AA?$CL?$AA?5?$AAn@ 1018b728     LIBCMTD:cvt.obj
 0003:0001077c       ??_C@_1BC@JOKPCIC@?$AA_?$AAc?$AAf?$AAt?$AAo?$AAa?$AA_?$AAl?$AA?$AA@ 1018b77c     LIBCMTD:cvt.obj
 0003:00010790       ??_C@_1BC@DCPPLJL@?$AA_?$AAc?$AAf?$AAt?$AAo?$AAf?$AA_?$AAl?$AA?$AA@ 1018b790     LIBCMTD:cvt.obj
 0003:000107a4       ??_C@_1BE@CKPDLI@?$AA_?$AAc?$AAf?$AAt?$AAo?$AAf?$AA2?$AA_?$AAl?$AA?$AA@ 1018b7a4     LIBCMTD:cvt.obj
 0003:000107b8       ??_C@_1BC@MPIFPLAF@?$AA_?$AAc?$AAf?$AAt?$AAo?$AAg?$AA_?$AAl?$AA?$AA@ 1018b7b8     LIBCMTD:cvt.obj
 0003:000110d8       __DEFAULT_CW_in_mem        1018c0d8     LIBCMTD:_common_.obj
 0003:000110da       __pi_by_2_to_61            1018c0da     LIBCMTD:_common_.obj
 0003:00014a60       __pDestructExceptionObject 1018fa60     LIBCMTD:frame.obj
 0003:00014a64       ??_C@_0O@DPKOEFFH@bad?5exception?$AA@ 1018fa64     LIBCMTD:frame.obj
 0003:00014a78       ??_7bad_exception@std@@6B@ 1018fa78     LIBCMTD:frame.obj
 0003:00014a80       ??_C@_0CP@MKONOLCI@f?3?2dd?2vctools?2crt_bld?2self_x86?2c@ 1018fa80     LIBCMTD:mlock.obj
 0003:00014ab0       ??_C@_1NK@LOFHIHFC@?$AAf?$AAM?$AAo?$AAd?$AAe?$AA?5?$AA?$DN?$AA?$DN?$AA?5?$AA_?$AAC?$AAR?$AAT?$AAD?$AAB?$AAG?$AA_?$AAR?$AAE?$AAP?$AAO?$AAR?$AAT?$AA_?$AAM?$AAO?$AAD?$AAE?$AA?5?$AA?$HM?$AA?$HM?$AA?5@ 1018fab0     LIBCMTD:dbgrptt.obj
 0003:00014b8c       ??_C@_1CE@FIHIECNJ@?$AA_?$AAC?$AAr?$AAt?$AAS?$AAe?$AAt?$AAR?$AAe?$AAp?$AAo?$AAr?$AAt?$AAM?$AAo?$AAd?$AAe?$AA?$AA@ 1018fb8c     LIBCMTD:dbgrptt.obj
 0003:00014bb0       ??_C@_1GC@FIGJJMEN@?$AAf?$AA?3?$AA?2?$AAd?$AAd?$AA?2?$AAv?$AAc?$AAt?$AAo?$AAo?$AAl?$AAs?$AA?2?$AAc?$AAr?$AAt?$AA_?$AAb?$AAl?$AAd?$AA?2?$AAs?$AAe?$AAl?$AAf?$AA_?$AAx?$AA8?$AA6?$AA?2?$AAc@ 1018fbb0     LIBCMTD:dbgrptt.obj
 0003:00014c18       ??_C@_1FA@IFFFOLDJ@?$AAn?$AAR?$AAp?$AAt?$AAT?$AAy?$AAp?$AAe?$AA?5?$AA?$DO?$AA?$DN?$AA?5?$AA0?$AA?5?$AA?$CG?$AA?$CG?$AA?5?$AAn?$AAR?$AAp?$AAt?$AAT?$AAy?$AAp?$AAe?$AA?5?$AA?$DM?$AA?5?$AA_?$AAC?$AAR?$AAT@ 1018fc18     LIBCMTD:dbgrptt.obj
 0003:00014c68       ??_C@_1CE@IKKEDCME@?$AA_?$AAC?$AAr?$AAt?$AAS?$AAe?$AAt?$AAR?$AAe?$AAp?$AAo?$AAr?$AAt?$AAF?$AAi?$AAl?$AAe?$AA?$AA@ 1018fc68     LIBCMTD:dbgrptt.obj
 0003:00014c90       ??_C@_1HO@PJOFIKFE@?$AA_?$AAC?$AAr?$AAt?$AAD?$AAb?$AAg?$AAR?$AAe?$AAp?$AAo?$AAr?$AAt?$AA?3?$AA?5?$AAS?$AAt?$AAr?$AAi?$AAn?$AAg?$AA?5?$AAt?$AAo?$AAo?$AA?5?$AAl?$AAo?$AAn?$AAg?$AA?5?$AAo@ 1018fc90     LIBCMTD:dbgrptt.obj
 0003:00014d10       ??_C@_1MC@IGEECMDB@?$AAw?$AAc?$AAs?$AAc?$AAp?$AAy?$AA_?$AAs?$AA?$CI?$AAs?$AAz?$AAO?$AAu?$AAt?$AAM?$AAe?$AAs?$AAs?$AAa?$AAg?$AAe?$AA2?$AA?0?$AA?5?$AA4?$AA0?$AA9?$AA6?$AA?0?$AA?5?$AAL?$AA?$CC@ 1018fd10     LIBCMTD:dbgrptt.obj
 0003:00014dd8       ??_C@_1IM@OOKIFKOH@?$AAe?$AA?5?$AA?$DN?$AA?5?$AAm?$AAb?$AAs?$AAt?$AAo?$AAw?$AAc?$AAs?$AA_?$AAs?$AA?$CI?$AA?$CG?$AAr?$AAe?$AAt?$AA?0?$AA?5?$AAs?$AAz?$AAO?$AAu?$AAt?$AAM?$AAe?$AAs?$AAs?$AAa?$AAg@ 1018fdd8     LIBCMTD:dbgrptt.obj
 0003:00014e68       ??_C@_1FI@IBIOIHEG@?$AAs?$AAt?$AAr?$AAc?$AAp?$AAy?$AA_?$AAs?$AA?$CI?$AAs?$AAz?$AAO?$AAu?$AAt?$AAM?$AAe?$AAs?$AAs?$AAa?$AAg?$AAe?$AA?0?$AA?5?$AA4?$AA0?$AA9?$AA6?$AA?0?$AA?5?$AAs?$AAz?$AAL@ 1018fe68     LIBCMTD:dbgrptt.obj
 0003:00014ec0       ??_C@_1JG@CPKCIOEE@?$AAs?$AAt?$AAr?$AAc?$AAp?$AAy?$AA_?$AAs?$AA?$CI?$AAs?$AAz?$AAO?$AAu?$AAt?$AAM?$AAe?$AAs?$AAs?$AAa?$AAg?$AAe?$AA?0?$AA?5?$AA4?$AA0?$AA9?$AA6?$AA?0?$AA?5?$AA?$CC?$AA_?$AAC@ 1018fec0     LIBCMTD:dbgrptt.obj
 0003:00014f58       ??_C@_0M@IPILFDFN@?$CFs?$CI?$CFd?$CJ?5?3?5?$CFs?$AA@ 1018ff58     LIBCMTD:dbgrptt.obj
 0003:00014f68       ??_C@_1EI@LDHJEDO@?$AAs?$AAt?$AAr?$AAc?$AAa?$AAt?$AA_?$AAs?$AA?$CI?$AAs?$AAz?$AAL?$AAi?$AAn?$AAe?$AAM?$AAe?$AAs?$AAs?$AAa?$AAg?$AAe?$AA?0?$AA?5?$AA4?$AA0?$AA9?$AA6?$AA?0?$AA?5?$AA?$CC?$AA?2@ 1018ff68     LIBCMTD:dbgrptt.obj
 0003:00014fb0       ??_C@_01LIIJDEN@?$AN?$AA@  1018ffb0     LIBCMTD:dbgrptt.obj
 0003:00014fb8       ??_C@_1EI@CACDLAFK@?$AAs?$AAt?$AAr?$AAc?$AAa?$AAt?$AA_?$AAs?$AA?$CI?$AAs?$AAz?$AAL?$AAi?$AAn?$AAe?$AAM?$AAe?$AAs?$AAs?$AAa?$AAg?$AAe?$AA?0?$AA?5?$AA4?$AA0?$AA9?$AA6?$AA?0?$AA?5?$AA?$CC?$AA?2@ 1018ffb8     LIBCMTD:dbgrptt.obj
 0003:00015000       ??_C@_1FK@NPGBPOFO@?$AAs?$AAt?$AAr?$AAc?$AAa?$AAt?$AA_?$AAs?$AA?$CI?$AAs?$AAz?$AAL?$AAi?$AAn?$AAe?$AAM?$AAe?$AAs?$AAs?$AAa?$AAg?$AAe?$AA?0?$AA?5?$AA4?$AA0?$AA9?$AA6?$AA?0?$AA?5?$AAs?$AAz@ 10190000     LIBCMTD:dbgrptt.obj
 0003:00015060       ??_C@_1KK@GIGAEDMO@?$AAs?$AAt?$AAr?$AAc?$AAp?$AAy?$AA_?$AAs?$AA?$CI?$AAs?$AAz?$AAL?$AAi?$AAn?$AAe?$AAM?$AAe?$AAs?$AAs?$AAa?$AAg?$AAe?$AA?0?$AA?5?$AA4?$AA0?$AA9?$AA6?$AA?0?$AA?5?$AAs?$AAz@ 10190060     LIBCMTD:dbgrptt.obj
 0003:0001510c       ??_C@_0BC@LAIDCHCH@Assertion?5failed?$CB?$AA@ 1019010c     LIBCMTD:dbgrptt.obj
 0003:00015120       ??_C@_0BD@CAENFOHP@Assertion?5failed?3?5?$AA@ 10190120     LIBCMTD:dbgrptt.obj
 0003:00015134       ??_C@_0CL@EACFGMNB@_CrtDbgReport?3?5String?5too?5long?5o@ 10190134     LIBCMTD:dbgrptt.obj
 0003:00015160       ??_C@_1JI@GAALPGBM@?$AAs?$AAt?$AAr?$AAc?$AAp?$AAy?$AA_?$AAs?$AA?$CI?$AAs?$AAz?$AAU?$AAs?$AAe?$AAr?$AAM?$AAe?$AAs?$AAs?$AAa?$AAg?$AAe?$AA?0?$AA?5?$AA4?$AA0?$AA9?$AA6?$AA?0?$AA?5?$AA?$CC?$AA_@ 10190160     LIBCMTD:dbgrptt.obj
 0003:000151f8       ??_C@_07BHGABMGB@?0?5Line?5?$AA@ 101901f8     LIBCMTD:dbgrptt.obj
 0003:00015200       ??_C@_0P@DFJNDPOP@?$DMfile?5unknown?$DO?$AA@ 10190200     LIBCMTD:dbgrptt.obj
 0003:00015210       ??_C@_0CG@BNGLOCEO@Second?5Chance?5Assertion?5Failed?3?5@ 10190210     LIBCMTD:dbgrptt.obj
 0003:00015238       ??_C@_1FA@JPHJBHEM@?$AA_?$AAi?$AAt?$AAo?$AAa?$AA_?$AAs?$AA?$CI?$AAn?$AAL?$AAi?$AAn?$AAe?$AA?0?$AA?5?$AAs?$AAz?$AAL?$AAi?$AAn?$AAe?$AAM?$AAe?$AAs?$AAs?$AAa?$AAg?$AAe?$AA?0?$AA?5?$AA4?$AA0@ 10190238     LIBCMTD:dbgrptt.obj
 0003:00015288       ??_C@_1CA@KHJHLKA@?$AA_?$AAV?$AAC?$AAr?$AAt?$AAD?$AAb?$AAg?$AAR?$AAe?$AAp?$AAo?$AAr?$AAt?$AAA?$AA?$AA@ 10190288     LIBCMTD:dbgrptt.obj
 0003:000152a8       ??_C@_1IE@CPGKIAGP@?$AAw?$AAc?$AAs?$AAt?$AAo?$AAm?$AAb?$AAs?$AA_?$AAs?$AA?$CI?$AA?$CG?$AAr?$AAe?$AAt?$AA?0?$AA?5?$AAs?$AAz?$AAa?$AAO?$AAu?$AAt?$AAM?$AAe?$AAs?$AAs?$AAa?$AAg?$AAe?$AA?0?$AA?5@ 101902a8     LIBCMTD:dbgrptt.obj
 0003:0001532c       ??_C@_0DP@GNPEPHJD@_CrtDbgReport?3?5String?5too?5long?5o@ 1019032c     LIBCMTD:dbgrptt.obj
 0003:00015370       ??_C@_1MA@LBAMNNOB@?$AAs?$AAt?$AAr?$AAc?$AAp?$AAy?$AA_?$AAs?$AA?$CI?$AAs?$AAz?$AAO?$AAu?$AAt?$AAM?$AAe?$AAs?$AAs?$AAa?$AAg?$AAe?$AA2?$AA?0?$AA?5?$AA4?$AA0?$AA9?$AA6?$AA?0?$AA?5?$AA?$CC?$AA_@ 10190370     LIBCMTD:dbgrptt.obj
 0003:00015430       ??_C@_1JC@EOAPFDLN@?$AAw?$AAc?$AAs?$AAt?$AAo?$AAm?$AAb?$AAs?$AA_?$AAs?$AA?$CI?$AA?$CI?$AA?$CI?$AAv?$AAo?$AAi?$AAd?$AA?5?$AA?$CK?$AA?$CJ?$AA0?$AA?$CJ?$AA?0?$AA?5?$AAs?$AAz?$AAO?$AAu?$AAt?$AAM?$AAe?$AAs@ 10190430     LIBCMTD:dbgrptt.obj
 0003:000154c8       ??_C@_1FI@DBAIJPJE@?$AAw?$AAc?$AAs?$AAc?$AAp?$AAy?$AA_?$AAs?$AA?$CI?$AAs?$AAz?$AAO?$AAu?$AAt?$AAM?$AAe?$AAs?$AAs?$AAa?$AAg?$AAe?$AA?0?$AA?5?$AA4?$AA0?$AA9?$AA6?$AA?0?$AA?5?$AAs?$AAz?$AAL@ 101904c8     LIBCMTD:dbgrptt.obj
 0003:00015520       ??_C@_1BI@JIDBEPIG@?$AA?$CF?$AAs?$AA?$CI?$AA?$CF?$AAd?$AA?$CJ?$AA?5?$AA?3?$AA?5?$AA?$CF?$AAs?$AA?$AA@ 10190520     LIBCMTD:dbgrptt.obj
 0003:00015538       ??_C@_1EK@PHCBEDKB@?$AAw?$AAc?$AAs?$AAc?$AAa?$AAt?$AA_?$AAs?$AA?$CI?$AAs?$AAz?$AAL?$AAi?$AAn?$AAe?$AAM?$AAe?$AAs?$AAs?$AAa?$AAg?$AAe?$AA?0?$AA?5?$AA4?$AA0?$AA9?$AA6?$AA?0?$AA?5?$AAL?$AA?$CC@ 10190538     LIBCMTD:dbgrptt.obj
 0003:00015584       ??_C@_13CMNBPIDO@?$AA?$AN?$AA?$AA@ 10190584     LIBCMTD:dbgrptt.obj
 0003:00015588       ??_C@_1EK@NMDFGHMF@?$AAw?$AAc?$AAs?$AAc?$AAa?$AAt?$AA_?$AAs?$AA?$CI?$AAs?$AAz?$AAL?$AAi?$AAn?$AAe?$AAM?$AAe?$AAs?$AAs?$AAa?$AAg?$AAe?$AA?0?$AA?5?$AA4?$AA0?$AA9?$AA6?$AA?0?$AA?5?$AAL?$AA?$CC@ 10190588     LIBCMTD:dbgrptt.obj
 0003:000155d8       ??_C@_1FK@HPADHBBD@?$AAw?$AAc?$AAs?$AAc?$AAa?$AAt?$AA_?$AAs?$AA?$CI?$AAs?$AAz?$AAL?$AAi?$AAn?$AAe?$AAM?$AAe?$AAs?$AAs?$AAa?$AAg?$AAe?$AA?0?$AA?5?$AA4?$AA0?$AA9?$AA6?$AA?0?$AA?5?$AAs?$AAz@ 101905d8     LIBCMTD:dbgrptt.obj
 0003:00015638       ??_C@_1KO@DGAHENCH@?$AAw?$AAc?$AAs?$AAc?$AAp?$AAy?$AA_?$AAs?$AA?$CI?$AAs?$AAz?$AAL?$AAi?$AAn?$AAe?$AAM?$AAe?$AAs?$AAs?$AAa?$AAg?$AAe?$AA?0?$AA?5?$AA4?$AA0?$AA9?$AA6?$AA?0?$AA?5?$AAs?$AAz@ 10190638     LIBCMTD:dbgrptt.obj
 0003:000156e8       ??_C@_1CE@OJBNHDMO@?$AAA?$AAs?$AAs?$AAe?$AAr?$AAt?$AAi?$AAo?$AAn?$AA?5?$AAf?$AAa?$AAi?$AAl?$AAe?$AAd?$AA?$CB?$AA?$AA@ 101906e8     LIBCMTD:dbgrptt.obj
 0003:0001570c       ??_C@_1CG@FFFGGODN@?$AAA?$AAs?$AAs?$AAe?$AAr?$AAt?$AAi?$AAo?$AAn?$AA?5?$AAf?$AAa?$AAi?$AAl?$AAe?$AAd?$AA?3?$AA?5?$AA?$AA@ 1019070c     LIBCMTD:dbgrptt.obj
 0003:00015738       ??_C@_1JK@KHFABAEO@?$AAw?$AAc?$AAs?$AAc?$AAp?$AAy?$AA_?$AAs?$AA?$CI?$AAs?$AAz?$AAU?$AAs?$AAe?$AAr?$AAM?$AAe?$AAs?$AAs?$AAa?$AAg?$AAe?$AA?0?$AA?5?$AA4?$AA0?$AA9?$AA6?$AA?0?$AA?5?$AAL?$AA?$CC@ 10190738     LIBCMTD:dbgrptt.obj
 0003:000157d4       ??_C@_13LBAGMAIH@?$AA?6?$AA?$AA@ 101907d4     LIBCMTD:dbgrptt.obj
 0003:000157d8       ??_C@_1BA@ELMMDCFC@?$AA?0?$AA?5?$AAL?$AAi?$AAn?$AAe?$AA?5?$AA?$AA@ 101907d8     LIBCMTD:dbgrptt.obj
 0003:000157e8       ??_C@_1BO@OCHMLCAG@?$AA?$DM?$AAf?$AAi?$AAl?$AAe?$AA?5?$AAu?$AAn?$AAk?$AAn?$AAo?$AAw?$AAn?$AA?$DO?$AA?$AA@ 101907e8     LIBCMTD:dbgrptt.obj
 0003:00015808       ??_C@_1EM@MJFLEDMB@?$AAS?$AAe?$AAc?$AAo?$AAn?$AAd?$AA?5?$AAC?$AAh?$AAa?$AAn?$AAc?$AAe?$AA?5?$AAA?$AAs?$AAs?$AAe?$AAr?$AAt?$AAi?$AAo?$AAn?$AA?5?$AAF?$AAa?$AAi?$AAl?$AAe?$AAd?$AA?3?$AA?5@ 10190808     LIBCMTD:dbgrptt.obj
 0003:00015858       ??_C@_1FA@CNLLOMHI@?$AA_?$AAi?$AAt?$AAo?$AAw?$AA_?$AAs?$AA?$CI?$AAn?$AAL?$AAi?$AAn?$AAe?$AA?0?$AA?5?$AAs?$AAz?$AAL?$AAi?$AAn?$AAe?$AAM?$AAe?$AAs?$AAs?$AAa?$AAg?$AAe?$AA?0?$AA?5?$AA4?$AA0@ 10190858     LIBCMTD:dbgrptt.obj
 0003:000158a8       ??_C@_1CA@HPALHDOD@?$AA_?$AAV?$AAC?$AAr?$AAt?$AAD?$AAb?$AAg?$AAR?$AAe?$AAp?$AAo?$AAr?$AAt?$AAW?$AA?$AA@ 101908a8     LIBCMTD:dbgrptt.obj
 0003:000158c8       ??_C@_1O@EJLDHPPL@?$AAs?$AAi?$AAg?$AAn?$AAa?$AAl?$AA?$AA@ 101908c8     LIBCMTD:winsig.obj
 0003:000158d8       ??_C@_1GA@DBECNFG@?$AAf?$AA?3?$AA?2?$AAd?$AAd?$AA?2?$AAv?$AAc?$AAt?$AAo?$AAo?$AAl?$AAs?$AA?2?$AAc?$AAr?$AAt?$AA_?$AAb?$AAl?$AAd?$AA?2?$AAs?$AAe?$AAl?$AAf?$AA_?$AAx?$AA8?$AA6?$AA?2?$AAc@ 101908d8     LIBCMTD:winsig.obj
 0003:00015938       ??_C@_1DO@MLNEDKGB@?$AA?$CI?$AA?$CC?$AAI?$AAn?$AAv?$AAa?$AAl?$AAi?$AAd?$AA?5?$AAs?$AAi?$AAg?$AAn?$AAa?$AAl?$AA?5?$AAo?$AAr?$AA?5?$AAe?$AAr?$AAr?$AAo?$AAr?$AA?$CC?$AA?0?$AA?5?$AA0?$AA?$CJ?$AA?$AA@ 10190938     LIBCMTD:winsig.obj
 0003:00015978       ??_C@_0DA@ELJOOIJF@f?3?2dd?2vctools?2crt_bld?2self_x86?2c@ 10190978     LIBCMTD:winsig.obj
 0003:000159a8       ??_C@_1M@DMJEIKHL@?$AAr?$AAa?$AAi?$AAs?$AAe?$AA?$AA@ 101909a8     LIBCMTD:winsig.obj
 0003:000159b4       ??_C@_0BI@DFKBFLJE@GetProcessWindowStation?$AA@ 101909b4     LIBCMTD:crtmboxw.obj
 0003:000159cc       ??_C@_0BK@DEKFELLI@GetUserObjectInformationW?$AA@ 101909cc     LIBCMTD:crtmboxw.obj
 0003:000159e8       ??_C@_0BD@HHGDFDBJ@GetLastActivePopup?$AA@ 101909e8     LIBCMTD:crtmboxw.obj
 0003:000159fc       ??_C@_0BA@HNOPNCHB@GetActiveWindow?$AA@ 101909fc     LIBCMTD:crtmboxw.obj
 0003:00015a0c       ??_C@_0M@DLDCCGNP@MessageBoxW?$AA@ 10190a0c     LIBCMTD:crtmboxw.obj
 0003:00015a18       ??_C@_1BG@GOEBHBDC@?$AAU?$AAS?$AAE?$AAR?$AA3?$AA2?$AA?4?$AAD?$AAL?$AAL?$AA?$AA@ 10190a18     LIBCMTD:crtmboxw.obj
 0003:00015a30       ??_C@_1BE@BMIJMLDD@?$AA_?$AAs?$AAw?$AAp?$AAr?$AAi?$AAn?$AAt?$AAf?$AA?$AA@ 10190a30     LIBCMTD:swprintf.obj
 0003:00015a48       ??_C@_1GE@DKGHLBLP@?$AAf?$AA?3?$AA?2?$AAd?$AAd?$AA?2?$AAv?$AAc?$AAt?$AAo?$AAo?$AAl?$AAs?$AA?2?$AAc?$AAr?$AAt?$AA_?$AAb?$AAl?$AAd?$AA?2?$AAs?$AAe?$AAl?$AAf?$AA_?$AAx?$AA8?$AA6?$AA?2?$AAc@ 10190a48     LIBCMTD:swprintf.obj
 0003:00015aac       ??_C@_1DM@MADKGDLO@?$AA?$CI?$AAL?$AA?$CC?$AAB?$AAu?$AAf?$AAf?$AAe?$AAr?$AA?5?$AAi?$AAs?$AA?5?$AAt?$AAo?$AAo?$AA?5?$AAs?$AAm?$AAa?$AAl?$AAl?$AA?$CC?$AA?5?$AA?$CG?$AA?$CG?$AA?5?$AA0?$AA?$CJ?$AA?$AA@ 10190aac     LIBCMTD:wcscpy_s.obj
 0003:00015ae8       ??_C@_1CI@HCPHDDLE@?$AAB?$AAu?$AAf?$AAf?$AAe?$AAr?$AA?5?$AAi?$AAs?$AA?5?$AAt?$AAo?$AAo?$AA?5?$AAs?$AAm?$AAa?$AAl?$AAl?$AA?$AA@ 10190ae8     LIBCMTD:wcscpy_s.obj
 0003:00015b10       ??_C@_1CG@OFBJMIGJ@?$AA?$CI?$AA?$CI?$AA?$CI?$AA_?$AAS?$AAr?$AAc?$AA?$CJ?$AA?$CJ?$AA?$CJ?$AA?5?$AA?$CB?$AA?$DN?$AA?5?$AAN?$AAU?$AAL?$AAL?$AA?$AA@ 10190b10     LIBCMTD:wcscpy_s.obj
 0003:00015b38       ??_C@_1BC@KIONAFPO@?$AAw?$AAc?$AAs?$AAc?$AAp?$AAy?$AA_?$AAs?$AA?$AA@ 10190b38     LIBCMTD:wcscpy_s.obj
 0003:00015b50       ??_C@_1GI@BGBNCIMA@?$AAf?$AA?3?$AA?2?$AAd?$AAd?$AA?2?$AAv?$AAc?$AAt?$AAo?$AAo?$AAl?$AAs?$AA?2?$AAc?$AAr?$AAt?$AA_?$AAb?$AAl?$AAd?$AA?2?$AAs?$AAe?$AAl?$AAf?$AA_?$AAx?$AA8?$AA6?$AA?2?$AAc@ 10190b50     LIBCMTD:wcscpy_s.obj
 0003:00015bb8       ??_C@_1FC@PFMLEHKI@?$AA?$CI?$AA?$CI?$AA_?$AAD?$AAs?$AAt?$AA?$CJ?$AA?$CJ?$AA?5?$AA?$CB?$AA?$DN?$AA?5?$AAN?$AAU?$AAL?$AAL?$AA?5?$AA?$CG?$AA?$CG?$AA?5?$AA?$CI?$AA?$CI?$AA_?$AAS?$AAi?$AAz?$AAe?$AAI?$AAn?$AAW?$AAo?$AAr@ 10190bb8     LIBCMTD:wcscpy_s.obj
 0003:00015c10       ??_C@_1HG@KNCBMCDD@?$AAf?$AA?3?$AA?2?$AAd?$AAd?$AA?2?$AAv?$AAc?$AAt?$AAo?$AAo?$AAl?$AAs?$AA?2?$AAc?$AAr?$AAt?$AA_?$AAb?$AAl?$AAd?$AA?2?$AAs?$AAe?$AAl?$AAf?$AA_?$AAx?$AA8?$AA6?$AA?2?$AAc@ 10190c10     LIBCMTD:typname.obj
 0003:00015c88       ??_C@_1CI@IDCGDBOP@?$AAp?$AAN?$AAo?$AAd?$AAe?$AA?9?$AA?$DO?$AAn?$AAe?$AAx?$AAt?$AA?5?$AA?$CB?$AA?$DN?$AA?5?$AAN?$AAU?$AAL?$AAL?$AA?$AA@ 10190c88     LIBCMTD:typname.obj
 0003:00015cb0       ??_C@_1JK@MLBKHELP@?$AAs?$AAt?$AAr?$AAc?$AAp?$AAy?$AA_?$AAs?$AA?5?$AA?$CI?$AA?$CI?$AAc?$AAh?$AAa?$AAr?$AA?5?$AA?$CK?$AA?$CJ?$AA?$CI?$AA?$CI?$AAt?$AAy?$AAp?$AAe?$AA_?$AAi?$AAn?$AAf?$AAo?$AA?5?$AA?$CK?$AA?$CJ@ 10190cb0     LIBCMTD:typname.obj
 0003:00015d4c       ??_C@_1CM@OOICDMK@?$AAt?$AAy?$AAp?$AAe?$AA_?$AAi?$AAn?$AAf?$AAo?$AA?3?$AA?3?$AA_?$AAN?$AAa?$AAm?$AAe?$AA_?$AAb?$AAa?$AAs?$AAe?$AA?$AA@ 10190d4c     LIBCMTD:typname.obj
 0003:00015d78       ??_C@_1GI@EAJKJPED@?$AAs?$AAt?$AAr?$AAc?$AAp?$AAy?$AA_?$AAs?$AA?5?$AA?$CI?$AAp?$AAT?$AAm?$AAp?$AAT?$AAy?$AAp?$AAe?$AAN?$AAa?$AAm?$AAe?$AA?0?$AA?5?$AAl?$AAe?$AAn?$AA?$CL?$AA2?$AA?0?$AA?5?$AA?$CI@ 10190d78     LIBCMTD:typname.obj
 0003:00015de0       ??_C@_1DO@OJJLFJPE@?$AAt?$AAy?$AAp?$AAe?$AA_?$AAi?$AAn?$AAf?$AAo?$AA?3?$AA?3?$AA_?$AAN?$AAa?$AAm?$AAe?$AA_?$AAb?$AAa?$AAs?$AAe?$AA_?$AAi?$AAn?$AAt?$AAe?$AAr?$AAn?$AAa?$AAl?$AA?$AA@ 10190de0     LIBCMTD:typname.obj
 0003:00015e20       ??_C@_1BC@CFJEPFGF@?$AAs?$AAt?$AAr?$AAc?$AAp?$AAy?$AA_?$AAs?$AA?$AA@ 10190e20     LIBCMTD:strcpy_s.obj
 0003:00015e38       ??_C@_1FC@NCPEPIBI@?$AA?$CI?$AA?$CI?$AA_?$AAD?$AAs?$AAt?$AA?$CJ?$AA?$CJ?$AA?5?$AA?$CB?$AA?$DN?$AA?5?$AAN?$AAU?$AAL?$AAL?$AA?5?$AA?$CG?$AA?$CG?$AA?5?$AA?$CI?$AA?$CI?$AA_?$AAS?$AAi?$AAz?$AAe?$AAI?$AAn?$AAB?$AAy?$AAt@ 10190e38     LIBCMTD:strcpy_s.obj
 0003:00015e90       ??_C@_1GG@CDHAPCGF@?$AAf?$AA?3?$AA?2?$AAd?$AAd?$AA?2?$AAv?$AAc?$AAt?$AAo?$AAo?$AAl?$AAs?$AA?2?$AAc?$AAr?$AAt?$AA_?$AAb?$AAl?$AAd?$AA?2?$AAs?$AAe?$AAl?$AAf?$AA_?$AAx?$AA8?$AA6?$AA?2?$AAc@ 10190e90     LIBCMTD:handler.obj
 0003:00015ef8       ??_C@_1BC@JLLICHIC@?$AAp?$AAn?$AAh?$AA?5?$AA?$DN?$AA?$DN?$AA?5?$AA0?$AA?$AA@ 10190ef8     LIBCMTD:handler.obj
 0003:00015f10       ??_C@_1HO@MLMGPAFH@?$AA?$CI?$AA?$CC?$AAi?$AAn?$AAc?$AAo?$AAn?$AAs?$AAi?$AAs?$AAt?$AAe?$AAn?$AAt?$AA?5?$AAI?$AAO?$AAB?$AA?5?$AAf?$AAi?$AAe?$AAl?$AAd?$AAs?$AA?$CC?$AA?0?$AA?5?$AAs?$AAt?$AAr?$AAe@ 10190f10     LIBCMTD:_flsbuf.obj
 0003:00015f90       ??_C@_1GC@GNCCMPNN@?$AAf?$AA?3?$AA?2?$AAd?$AAd?$AA?2?$AAv?$AAc?$AAt?$AAo?$AAo?$AAl?$AAs?$AA?2?$AAc?$AAr?$AAt?$AA_?$AAb?$AAl?$AAd?$AA?2?$AAs?$AAe?$AAl?$AAf?$AA_?$AAx?$AA8?$AA6?$AA?2?$AAc@ 10190f90     LIBCMTD:_flsbuf.obj
 0003:00015ff4       ??_C@_1BI@MFCLPIBM@?$AAs?$AAt?$AAr?$AA?5?$AA?$CB?$AA?$DN?$AA?5?$AAN?$AAU?$AAL?$AAL?$AA?$AA@ 10190ff4     LIBCMTD:_flsbuf.obj
 0003:0001600c       ??_C@_1O@CEDCILHN@?$AA?$CI?$AAn?$AAu?$AAl?$AAl?$AA?$CJ?$AA?$AA@ 1019100c     LIBCMTD:output.obj
 0003:0001601c       ??_C@_06OJHGLDPL@?$CInull?$CJ?$AA@ 1019101c     LIBCMTD:output.obj
 0003:00016028       ___lookuptable             10191028     LIBCMTD:output.obj
 0003:00016084       ??_C@_0DA@NFBEBPEE@f?3?2dd?2vctools?2crt_bld?2self_x86?2c@ 10191084     LIBCMTD:output.obj
 0003:000160b8       ??_C@_1EK@PNGFDECN@?$AA?$CI?$AA?$CC?$AA?8?$AAn?$AA?8?$AA?5?$AAf?$AAo?$AAr?$AAm?$AAa?$AAt?$AA?5?$AAs?$AAp?$AAe?$AAc?$AAi?$AAf?$AAi?$AAe?$AAr?$AA?5?$AAd?$AAi?$AAs?$AAa?$AAb?$AAl?$AAe?$AAd?$AA?$CC@ 101910b8     LIBCMTD:output.obj
 0003:00016104       ??_C@_1CC@IFFHEMNF@?$AA?$CI?$AAc?$AAh?$AA?5?$AA?$CB?$AA?$DN?$AA?5?$AA_?$AAT?$AA?$CI?$AA?8?$AA?2?$AA0?$AA?8?$AA?$CJ?$AA?$CJ?$AA?$AA@ 10191104     LIBCMTD:output.obj
 0003:00016128       ??_C@_1BE@IONLIDNC@?$AA_?$AAo?$AAu?$AAt?$AAp?$AAu?$AAt?$AA_?$AAl?$AA?$AA@ 10191128     LIBCMTD:output.obj
 0003:00016140       ??_C@_1GA@HHFOFBLN@?$AAf?$AA?3?$AA?2?$AAd?$AAd?$AA?2?$AAv?$AAc?$AAt?$AAo?$AAo?$AAl?$AAs?$AA?2?$AAc?$AAr?$AAt?$AA_?$AAb?$AAl?$AAd?$AA?2?$AAs?$AAe?$AAl?$AAf?$AA_?$AAx?$AA8?$AA6?$AA?2?$AAc@ 10191140     LIBCMTD:output.obj
 0003:000161a0       ??_C@_1EC@FABAOFFO@?$AA?$CI?$AAc?$AAo?$AAu?$AAn?$AAt?$AA?5?$AA?$DN?$AA?$DN?$AA?5?$AA0?$AA?$CJ?$AA?5?$AA?$HM?$AA?$HM?$AA?5?$AA?$CI?$AAs?$AAt?$AAr?$AAi?$AAn?$AAg?$AA?5?$AA?$CB?$AA?$DN?$AA?5?$AAN?$AAU?$AAL?$AAL?$AA?$CJ@ 101911a0     LIBCMTD:vsnprnc.obj
 0003:000161e4       ??_C@_1CE@PCFPEIFI@?$AA_?$AAv?$AAs?$AAn?$AAp?$AAr?$AAi?$AAn?$AAt?$AAf?$AA_?$AAh?$AAe?$AAl?$AAp?$AAe?$AAr?$AA?$AA@ 101911e4     LIBCMTD:vsnprnc.obj
 0003:00016208       ??_C@_1DA@HPBFKMEB@?$AA?$CI?$AA?$CC?$AAB?$AAu?$AAf?$AAf?$AAe?$AAr?$AA?5?$AAt?$AAo?$AAo?$AA?5?$AAs?$AAm?$AAa?$AAl?$AAl?$AA?$CC?$AA?0?$AA?5?$AA0?$AA?$CJ?$AA?$AA@ 10191208     LIBCMTD:vsnprnc.obj
 0003:00016238       ??_C@_1EE@OKCKIGFK@?$AAs?$AAt?$AAr?$AAi?$AAn?$AAg?$AA?5?$AA?$CB?$AA?$DN?$AA?5?$AAN?$AAU?$AAL?$AAL?$AA?5?$AA?$CG?$AA?$CG?$AA?5?$AAs?$AAi?$AAz?$AAe?$AAI?$AAn?$AAB?$AAy?$AAt?$AAe?$AAs?$AA?5?$AA?$DO?$AA?5@ 10191238     LIBCMTD:vsnprnc.obj
 0003:0001627c       ??_C@_1BM@BLJALHEF@?$AA_?$AAv?$AAs?$AAp?$AAr?$AAi?$AAn?$AAt?$AAf?$AA_?$AAs?$AA_?$AAl?$AA?$AA@ 1019127c     LIBCMTD:vsnprnc.obj
 0003:00016298       ??_C@_1BO@MLMCMBKN@?$AAf?$AAo?$AAr?$AAm?$AAa?$AAt?$AA?5?$AA?$CB?$AA?$DN?$AA?5?$AAN?$AAU?$AAL?$AAL?$AA?$AA@ 10191298     LIBCMTD:vsnprnc.obj
 0003:000162b8       ??_C@_1BO@MMPELNIM@?$AA_?$AAv?$AAs?$AAn?$AAp?$AAr?$AAi?$AAn?$AAt?$AAf?$AA_?$AAs?$AA_?$AAl?$AA?$AA@ 101912b8     LIBCMTD:vsnprnc.obj
 0003:000162d8       ??_C@_1FE@CEHLKAHD@?$AAi?$AAb?$AAa?$AAs?$AAe?$AA?5?$AA?$DN?$AA?$DN?$AA?5?$AA0?$AA?5?$AA?$HM?$AA?$HM?$AA?5?$AA?$CI?$AA2?$AA?5?$AA?$DM?$AA?$DN?$AA?5?$AAi?$AAb?$AAa?$AAs?$AAe?$AA?5?$AA?$CG?$AA?$CG?$AA?5?$AAi?$AAb?$AAa@ 101912d8     LIBCMTD:strtol.obj
 0003:0001632c       ??_C@_1BA@LOLAMAJG@?$AAs?$AAt?$AAr?$AAt?$AAo?$AAx?$AAl?$AA?$AA@ 1019132c     LIBCMTD:strtol.obj
 0003:00016340       ??_C@_1GA@IPHKKOEI@?$AAf?$AA?3?$AA?2?$AAd?$AAd?$AA?2?$AAv?$AAc?$AAt?$AAo?$AAo?$AAl?$AAs?$AA?2?$AAc?$AAr?$AAt?$AA_?$AAb?$AAl?$AAd?$AA?2?$AAs?$AAe?$AAl?$AAf?$AA_?$AAx?$AA8?$AA6?$AA?2?$AAc@ 10191340     LIBCMTD:strtol.obj
 0003:000163a0       ??_C@_1BA@BMMDEPNE@?$AAs?$AAt?$AAr?$AAt?$AAo?$AAx?$AAq?$AA?$AA@ 101913a0     LIBCMTD:strtoq.obj
 0003:000163b0       ??_C@_1GA@GIMEIKLC@?$AAf?$AA?3?$AA?2?$AAd?$AAd?$AA?2?$AAv?$AAc?$AAt?$AAo?$AAo?$AAl?$AAs?$AA?2?$AAc?$AAr?$AAt?$AA_?$AAb?$AAl?$AAd?$AA?2?$AAs?$AAe?$AAl?$AAf?$AA_?$AAx?$AA8?$AA6?$AA?2?$AAc@ 101913b0     LIBCMTD:strtoq.obj
 0003:00016410       ??_C@_0M@EKFFODEC@MSPDB80?4DLL?$AA@ 10191410     LIBCMTD:_pdblkup_.obj
 0003:0001641c       ??_C@_01KDCPPGHE@r?$AA@    1019141c     LIBCMTD:_pdblkup_.obj
 0003:00016420       ??_C@_0BB@KCIACLNC@PDBOpenValidate5?$AA@ 10191420     LIBCMTD:_pdblkup_.obj
 0003:00016434       ??_C@_0BF@BMIHBHCA@EnvironmentDirectory?$AA@ 10191434     LIBCMTD:_pdblkup_.obj
 0003:0001644c       ??_C@_0CN@JNNIHDGH@SOFTWARE?2Microsoft?2VisualStudio?2@ 1019144c     LIBCMTD:_pdblkup_.obj
 0003:0001647c       ??_C@_0M@HLOHPNFA@RegCloseKey?$AA@ 1019147c     LIBCMTD:_pdblkup_.obj
 0003:00016488       ??_C@_0BB@HHEIPGME@RegQueryValueExA?$AA@ 10191488     LIBCMTD:_pdblkup_.obj
 0003:0001649c       ??_C@_0O@DCOGKJGG@RegOpenKeyExA?$AA@ 1019149c     LIBCMTD:_pdblkup_.obj
 0003:000164ac       ??_C@_0N@JJPEKNFO@ADVAPI32?4DLL?$AA@ 101914ac     LIBCMTD:_pdblkup_.obj
 0003:000164c0       ??_C@_1GC@CHGJNMHG@?$AAf?$AA?3?$AA?2?$AAd?$AAd?$AA?2?$AAv?$AAc?$AAt?$AAo?$AAo?$AAl?$AAs?$AA?2?$AAc?$AAr?$AAt?$AA_?$AAb?$AAl?$AAd?$AA?2?$AAs?$AAe?$AAl?$AAf?$AA_?$AAx?$AA8?$AA6?$AA?2?$AAc@ 101914c0     LIBCMTD:isctype.obj
 0003:00016524       ??_C@_1DC@BPLPALML@?$AA?$CI?$AAu?$AAn?$AAs?$AAi?$AAg?$AAn?$AAe?$AAd?$AA?$CJ?$AA?$CI?$AAc?$AA?5?$AA?$CL?$AA?5?$AA1?$AA?$CJ?$AA?5?$AA?$DM?$AA?$DN?$AA?5?$AA2?$AA5?$AA6?$AA?$AA@ 10191524     LIBCMTD:isctype.obj
 0003:00016558       ??_C@_1BO@IHLJHOPI@?$AA_?$AA_?$AAs?$AAt?$AAr?$AAg?$AAt?$AAo?$AAl?$AAd?$AA1?$AA2?$AA_?$AAl?$AA?$AA@ 10191558     LIBCMTD:_strgtold_.obj
 0003:00016578       ??_C@_1IG@IGKPPFIM@?$AAf?$AA?3?$AA?2?$AAd?$AAd?$AA?2?$AAv?$AAc?$AAt?$AAo?$AAo?$AAl?$AAs?$AA?2?$AAc?$AAr?$AAt?$AA_?$AAb?$AAl?$AAd?$AA?2?$AAs?$AAe?$AAl?$AAf?$AA_?$AAx?$AA8?$AA6?$AA?2?$AAc@ 10191578     LIBCMTD:_strgtold_.obj
 0003:00016600       ??_C@_1CA@MBDBOHIB@?$AA_?$AAL?$AAo?$AAc?$AAa?$AAl?$AAe?$AA?5?$AA?$CB?$AA?$DN?$AA?5?$AAN?$AAU?$AAL?$AAL?$AA?$AA@ 10191600     LIBCMTD:_strgtold_.obj
 0003:00016620       ??_C@_1FK@BCPANIEK@?$AA?$CI?$AA?$CC?$AAM?$AAi?$AAs?$AAs?$AAi?$AAn?$AAg?$AA?5?$AAp?$AAo?$AAs?$AAi?$AAt?$AAi?$AAo?$AAn?$AA?5?$AAi?$AAn?$AA?5?$AAt?$AAh?$AAe?$AA?5?$AAf?$AAo?$AAr?$AAm?$AAa?$AAt@ 10191620     LIBCMTD:outputp.obj
 0003:00016680       ??_C@_1FK@LNCFKALM@?$AA?$CI?$AA?$CI?$AAs?$AAt?$AAa?$AAt?$AAe?$AA?5?$AA?$DN?$AA?$DN?$AA?5?$AAS?$AAT?$AA_?$AAN?$AAO?$AAR?$AAM?$AAA?$AAL?$AA?$CJ?$AA?5?$AA?$HM?$AA?$HM?$AA?5?$AA?$CI?$AAs?$AAt?$AAa?$AAt?$AAe?$AA?5@ 10191680     LIBCMTD:outputp.obj
 0003:000166e0       ??_C@_1JC@OACKELNN@?$AA_?$AAt?$AAv?$AAa?$AAl?$AAi?$AAd?$AAa?$AAt?$AAe?$AA_?$AAp?$AAa?$AAr?$AAa?$AAm?$AA_?$AAr?$AAe?$AAu?$AAs?$AAe?$AA?$CI?$AA?$CG?$AAp?$AAo?$AAs?$AA_?$AAv?$AAa?$AAl?$AAu@ 101916e0     LIBCMTD:outputp.obj
 0003:00016778       ??_C@_1IK@NBGDDCBN@?$AA_?$AAt?$AAv?$AAa?$AAl?$AAi?$AAd?$AAa?$AAt?$AAe?$AA_?$AAp?$AAa?$AAr?$AAa?$AAm?$AA_?$AAr?$AAe?$AAu?$AAs?$AAe?$AA?$CI?$AA?$CG?$AAp?$AAo?$AAs?$AA_?$AAv?$AAa?$AAl?$AAu@ 10191778     LIBCMTD:outputp.obj
 0003:00016804       ??_C@_1DG@GOHGNKHE@?$AAp?$AAa?$AAs?$AAs?$AA?5?$AA?$DN?$AA?$DN?$AA?5?$AAF?$AAO?$AAR?$AAM?$AAA?$AAT?$AA_?$AAO?$AAU?$AAT?$AAP?$AAU?$AAT?$AA_?$AAP?$AAA?$AAS?$AAS?$AA?$AA@ 10191804     LIBCMTD:outputp.obj
 0003:00016840       ??_C@_1IM@DNGHAPLB@?$AA_?$AAt?$AAv?$AAa?$AAl?$AAi?$AAd?$AAa?$AAt?$AAe?$AA_?$AAp?$AAa?$AAr?$AAa?$AAm?$AA_?$AAr?$AAe?$AAu?$AAs?$AAe?$AA?$CI?$AA?$CG?$AAp?$AAo?$AAs?$AA_?$AAv?$AAa?$AAl?$AAu@ 10191840     LIBCMTD:outputp.obj
 0003:000168d0       ??_C@_1IG@HJIMKDHC@?$AA_?$AAt?$AAv?$AAa?$AAl?$AAi?$AAd?$AAa?$AAt?$AAe?$AA_?$AAp?$AAa?$AAr?$AAa?$AAm?$AA_?$AAr?$AAe?$AAu?$AAs?$AAe?$AA?$CI?$AA?$CG?$AAp?$AAo?$AAs?$AA_?$AAv?$AAa?$AAl?$AAu@ 101918d0     LIBCMTD:outputp.obj
 0003:00016958       ??_C@_1IG@FDCPLALG@?$AA_?$AAt?$AAv?$AAa?$AAl?$AAi?$AAd?$AAa?$AAt?$AAe?$AA_?$AAp?$AAa?$AAr?$AAa?$AAm?$AA_?$AAr?$AAe?$AAu?$AAs?$AAe?$AA?$CI?$AA?$CG?$AAp?$AAo?$AAs?$AA_?$AAv?$AAa?$AAl?$AAu@ 10191958     LIBCMTD:outputp.obj
 0003:000169e0       ??_C@_1IK@MHEDJAMK@?$AA_?$AAt?$AAv?$AAa?$AAl?$AAi?$AAd?$AAa?$AAt?$AAe?$AA_?$AAp?$AAa?$AAr?$AAa?$AAm?$AA_?$AAr?$AAe?$AAu?$AAs?$AAe?$AA?$CI?$AA?$CG?$AAp?$AAo?$AAs?$AA_?$AAv?$AAa?$AAl?$AAu@ 101919e0     LIBCMTD:outputp.obj
 0003:00016a70       ??_C@_1EM@BNPHBBIA@?$AA?$CI?$AA?$CI?$AAt?$AAy?$AAp?$AAe?$AA_?$AAp?$AAo?$AAs?$AA?$DO?$AA?$DN?$AA0?$AA?$CJ?$AA?5?$AA?$CG?$AA?$CG?$AA?5?$AA?$CI?$AAt?$AAy?$AAp?$AAe?$AA_?$AAp?$AAo?$AAs?$AA?$DM?$AA_?$AAA?$AAR?$AAG@ 10191a70     LIBCMTD:outputp.obj
 0003:00016ac0       ??_C@_1IK@EIEPDKHJ@?$AA_?$AAt?$AAv?$AAa?$AAl?$AAi?$AAd?$AAa?$AAt?$AAe?$AA_?$AAp?$AAa?$AAr?$AAa?$AAm?$AA_?$AAr?$AAe?$AAu?$AAs?$AAe?$AA?$CI?$AA?$CG?$AAp?$AAo?$AAs?$AA_?$AAv?$AAa?$AAl?$AAu@ 10191ac0     LIBCMTD:outputp.obj
 0003:00016b50       ??_C@_1JG@JBJBOCFB@?$AA?$CI?$AA?$CI?$AAp?$AAr?$AAe?$AAc?$AAi?$AAs?$AA_?$AAp?$AAo?$AAs?$AA?5?$AA?$DO?$AA?$DN?$AA?5?$AA0?$AA?$CJ?$AA?5?$AA?$CG?$AA?$CG?$AA?5?$AA?$CI?$AA?$CK?$AAe?$AAn?$AAd?$AA_?$AAp?$AAo?$AAs?$AA?5@ 10191b50     LIBCMTD:outputp.obj
 0003:00016be8       ??_C@_1II@PIPIMLPF@?$AA_?$AAt?$AAv?$AAa?$AAl?$AAi?$AAd?$AAa?$AAt?$AAe?$AA_?$AAp?$AAa?$AAr?$AAa?$AAm?$AA_?$AAr?$AAe?$AAu?$AAs?$AAe?$AA?$CI?$AA?$CG?$AAp?$AAo?$AAs?$AA_?$AAv?$AAa?$AAl?$AAu@ 10191be8     LIBCMTD:outputp.obj
 0003:00016c70       ??_C@_1JE@NMBHOLFI@?$AA?$CI?$AA?$CI?$AAw?$AAi?$AAd?$AAt?$AAh?$AA_?$AAp?$AAo?$AAs?$AA?5?$AA?$DO?$AA?$DN?$AA?5?$AA0?$AA?$CJ?$AA?5?$AA?$CG?$AA?$CG?$AA?5?$AA?$CI?$AA?$CK?$AAe?$AAn?$AAd?$AA_?$AAp?$AAo?$AAs?$AA?5?$AA?$DN@ 10191c70     LIBCMTD:outputp.obj
 0003:00016d08       ??_C@_1EE@DMAIGNBG@?$AA?$CI?$AA?$CC?$AAI?$AAn?$AAc?$AAo?$AAr?$AAr?$AAe?$AAc?$AAt?$AA?5?$AAf?$AAo?$AAr?$AAm?$AAa?$AAt?$AA?5?$AAs?$AAp?$AAe?$AAc?$AAi?$AAf?$AAi?$AAe?$AAr?$AA?$CC?$AA?0?$AA?5?$AA0@ 10191d08     LIBCMTD:outputp.obj
 0003:00016d50       ??_C@_1JC@PFJNKEIO@?$AA?$CI?$AA?$CI?$AAt?$AAy?$AAp?$AAe?$AA_?$AAp?$AAo?$AAs?$AA?5?$AA?$DO?$AA?$DN?$AA?5?$AA0?$AA?$CJ?$AA?5?$AA?$CG?$AA?$CG?$AA?5?$AA?$CI?$AA?$CK?$AAe?$AAn?$AAd?$AA_?$AAp?$AAo?$AAs?$AA?5?$AA?$DN?$AA?$DN@ 10191d50     LIBCMTD:outputp.obj
 0003:00016de4       ??_C@_1BI@KANOLAMF@?$AA_?$AAo?$AAu?$AAt?$AAp?$AAu?$AAt?$AA_?$AAp?$AA_?$AAl?$AA?$AA@ 10191de4     LIBCMTD:outputp.obj
 0003:00016dfc       ??_C@_1BI@GEIGEDDA@?$AA_?$AAm?$AAa?$AAk?$AAe?$AAp?$AAa?$AAt?$AAh?$AA_?$AAs?$AA?$AA@ 10191dfc     LIBCMTD:makepath_s.obj
 0003:00016e18       ??_C@_1GO@DHMODCKM@?$AAf?$AA?3?$AA?2?$AAd?$AAd?$AA?2?$AAv?$AAc?$AAt?$AAo?$AAo?$AAl?$AAs?$AA?2?$AAc?$AAr?$AAt?$AA_?$AAb?$AAl?$AAd?$AA?2?$AAs?$AAe?$AAl?$AAf?$AA_?$AAx?$AA8?$AA6?$AA?2?$AAc@ 10191e18     LIBCMTD:makepath_s.obj
 0003:00016ea8       ??_C@_1CI@KEDPFCAL@?$AA?$CI?$AA?$CK?$AAm?$AAo?$AAd?$AAe?$AA?5?$AA?$DN?$AA?$DN?$AA?5?$AA_?$AAT?$AA?$CI?$AA?8?$AA?2?$AA0?$AA?8?$AA?$CJ?$AA?$CJ?$AA?$AA@ 10191ea8     LIBCMTD:_open.obj
 0003:00016ed0       ??_C@_1BE@DONHJJKE@?$AA_?$AAo?$AAp?$AAe?$AAn?$AAf?$AAi?$AAl?$AAe?$AA?$AA@ 10191ed0     LIBCMTD:_open.obj
 0003:00016ee4       ??_C@_1DK@PKMJBLLN@?$AA?$CI?$AA?$CC?$AAI?$AAn?$AAv?$AAa?$AAl?$AAi?$AAd?$AA?5?$AAf?$AAi?$AAl?$AAe?$AA?5?$AAo?$AAp?$AAe?$AAn?$AA?5?$AAm?$AAo?$AAd?$AAe?$AA?$CC?$AA?0?$AA0?$AA?$CJ?$AA?$AA@ 10191ee4     LIBCMTD:_open.obj
 0003:00016f20       ??_C@_1BK@HGLMNMEC@?$AAm?$AAo?$AAd?$AAe?$AA?5?$AA?$CB?$AA?$DN?$AA?5?$AAN?$AAU?$AAL?$AAL?$AA?$AA@ 10191f20     LIBCMTD:_open.obj
 0003:00016f40       ??_C@_1FO@POGAHKND@?$AAf?$AA?3?$AA?2?$AAd?$AAd?$AA?2?$AAv?$AAc?$AAt?$AAo?$AAo?$AAl?$AAs?$AA?2?$AAc?$AAr?$AAt?$AA_?$AAb?$AAl?$AAd?$AA?2?$AAs?$AAe?$AAl?$AAf?$AA_?$AAx?$AA8?$AA6?$AA?2?$AAc@ 10191f40     LIBCMTD:_open.obj
 0003:00016fa0       ??_C@_1CC@JBMDNKJP@?$AAf?$AAi?$AAl?$AAe?$AAn?$AAa?$AAm?$AAe?$AA?5?$AA?$CB?$AA?$DN?$AA?5?$AAN?$AAU?$AAL?$AAL?$AA?$AA@ 10191fa0     LIBCMTD:_open.obj
 0003:00016fc4       ??_C@_0DA@NLPACBPK@f?3?2dd?2vctools?2crt_bld?2self_x86?2c@ 10191fc4     LIBCMTD:stream.obj
 0003:00016ff8       ??_C@_1JE@ECKHFIFP@?$AA?$CI?$AA?$CC?$AAI?$AAn?$AAv?$AAa?$AAl?$AAi?$AAd?$AA?5?$AAf?$AAi?$AAl?$AAe?$AA?5?$AAd?$AAe?$AAs?$AAc?$AAr?$AAi?$AAp?$AAt?$AAo?$AAr?$AA?4?$AA?5?$AAF?$AAi?$AAl?$AAe?$AA?5@ 10191ff8     LIBCMTD:close.obj
 0003:0001708c       ??_C@_1CM@OKGMMMDH@?$AA?$CI?$AA_?$AAo?$AAs?$AAf?$AAi?$AAl?$AAe?$AA?$CI?$AAf?$AAh?$AA?$CJ?$AA?5?$AA?$CG?$AA?5?$AAF?$AAO?$AAP?$AAE?$AAN?$AA?$CJ?$AA?$AA@ 1019208c     LIBCMTD:close.obj
 0003:000170b8       ??_C@_1O@EDEJGJBM@?$AA_?$AAc?$AAl?$AAo?$AAs?$AAe?$AA?$AA@ 101920b8     LIBCMTD:close.obj
 0003:000170c8       ??_C@_1FO@NNGNFGFH@?$AAf?$AA?3?$AA?2?$AAd?$AAd?$AA?2?$AAv?$AAc?$AAt?$AAo?$AAo?$AAl?$AAs?$AA?2?$AAc?$AAr?$AAt?$AA_?$AAb?$AAl?$AAd?$AA?2?$AAs?$AAe?$AAl?$AAf?$AA_?$AAx?$AA8?$AA6?$AA?2?$AAc@ 101920c8     LIBCMTD:close.obj
 0003:00017128       ??_C@_1FO@LPCLHKGE@?$AA?$CI?$AAf?$AAh?$AA?5?$AA?$DO?$AA?$DN?$AA?5?$AA0?$AA?5?$AA?$CG?$AA?$CG?$AA?5?$AA?$CI?$AAu?$AAn?$AAs?$AAi?$AAg?$AAn?$AAe?$AAd?$AA?$CJ?$AAf?$AAh?$AA?5?$AA?$DM?$AA?5?$AA?$CI?$AAu?$AAn?$AAs?$AAi@ 10192128     LIBCMTD:close.obj
 0003:00017188       ??_C@_1BA@JGHIEKKM@?$AA_?$AAf?$AAi?$AAl?$AAe?$AAn?$AAo?$AA?$AA@ 10192188     LIBCMTD:fileno.obj
 0003:00017198       ??_C@_1GA@PBJHELNC@?$AAf?$AA?3?$AA?2?$AAd?$AAd?$AA?2?$AAv?$AAc?$AAt?$AAo?$AAo?$AAl?$AAs?$AA?2?$AAc?$AAr?$AAt?$AA_?$AAb?$AAl?$AAd?$AA?2?$AAs?$AAe?$AAl?$AAf?$AA_?$AAx?$AA8?$AA6?$AA?2?$AAc@ 10192198     LIBCMTD:fileno.obj
 0003:000171f8       ??_C@_1GE@MIMBMOF@?$AAf?$AA?3?$AA?2?$AAd?$AAd?$AA?2?$AAv?$AAc?$AAt?$AAo?$AAo?$AAl?$AAs?$AA?2?$AAc?$AAr?$AAt?$AA_?$AAb?$AAl?$AAd?$AA?2?$AAs?$AAe?$AAl?$AAf?$AA_?$AAx?$AA8?$AA6?$AA?2?$AAc@ 101921f8     LIBCMTD:_freebuf.obj
 0003:0001725c       ??_C@_1BO@KIJENGPH@?$AAs?$AAt?$AAr?$AAe?$AAa?$AAm?$AA?5?$AA?$CB?$AA?$DN?$AA?5?$AAN?$AAU?$AAL?$AAL?$AA?$AA@ 1019225c     LIBCMTD:_freebuf.obj
 0003:0001727c       ??_C@_0DA@NBLAKPEL@f?3?2dd?2vctools?2crt_bld?2self_x86?2c@ 1019227c     LIBCMTD:ioinit.obj
 0003:000172ac       ??_C@_1O@EDOIKGHF@?$AA_?$AAl?$AAs?$AAe?$AAe?$AAk?$AA?$AA@ 101922ac     LIBCMTD:lseek.obj
 0003:000172c0       ??_C@_1FO@LGKMLCAL@?$AAf?$AA?3?$AA?2?$AAd?$AAd?$AA?2?$AAv?$AAc?$AAt?$AAo?$AAo?$AAl?$AAs?$AA?2?$AAc?$AAr?$AAt?$AA_?$AAb?$AAl?$AAd?$AA?2?$AAs?$AAe?$AAl?$AAf?$AA_?$AAx?$AA8?$AA6?$AA?2?$AAc@ 101922c0     LIBCMTD:lseek.obj
 0003:00017320       ??_C@_1DM@LMLOLGJ@?$AA?$CI?$AA?$CC?$AAI?$AAn?$AAv?$AAa?$AAl?$AAi?$AAd?$AA?5?$AAf?$AAi?$AAl?$AAe?$AA?5?$AAd?$AAe?$AAs?$AAc?$AAr?$AAi?$AAp?$AAt?$AAo?$AAr?$AA?$CC?$AA?0?$AA0?$AA?$CJ?$AA?$AA@ 10192320     LIBCMTD:lseek.obj
 0003:0001735c       ??_C@_1BA@IIKEPOGH@?$AA_?$AAf?$AAi?$AAl?$AAb?$AAu?$AAf?$AA?$AA@ 1019235c     LIBCMTD:_filbuf.obj
 0003:00017370       ??_C@_1GC@CHFNJKFB@?$AAf?$AA?3?$AA?2?$AAd?$AAd?$AA?2?$AAv?$AAc?$AAt?$AAo?$AAo?$AAl?$AAs?$AA?2?$AAc?$AAr?$AAt?$AA_?$AAb?$AAl?$AAd?$AA?2?$AAs?$AAe?$AAl?$AAf?$AA_?$AAx?$AA8?$AA6?$AA?2?$AAc@ 10192370     LIBCMTD:_filbuf.obj
 0003:000173d4       ??_C@_1CC@HBLPFNKH@?$AA?$CI?$AAc?$AAn?$AAt?$AA?5?$AA?$DM?$AA?$DN?$AA?5?$AAI?$AAN?$AAT?$AA_?$AAM?$AAA?$AAX?$AA?$CJ?$AA?$AA@ 101923d4     LIBCMTD:read.obj
 0003:000173f8       ??_C@_1M@NHJOLLDM@?$AA_?$AAr?$AAe?$AAa?$AAd?$AA?$AA@ 101923f8     LIBCMTD:read.obj
 0003:00017408       ??_C@_1FM@NGICBHLO@?$AAf?$AA?3?$AA?2?$AAd?$AAd?$AA?2?$AAv?$AAc?$AAt?$AAo?$AAo?$AAl?$AAs?$AA?2?$AAc?$AAr?$AAt?$AA_?$AAb?$AAl?$AAd?$AA?2?$AAs?$AAe?$AAl?$AAf?$AA_?$AAx?$AA8?$AA6?$AA?2?$AAc@ 10192408     LIBCMTD:read.obj
 0003:00017464       ??_C@_0CO@CEGKNHEH@f?3?2dd?2vctools?2crt_bld?2self_x86?2c@ 10192464     LIBCMTD:read.obj
 0003:00017494       ??_C@_1CC@EEOLPHGO@?$AA?$CI?$AA?$CI?$AAc?$AAn?$AAt?$AA?5?$AA?$CG?$AA?5?$AA1?$AA?$CJ?$AA?5?$AA?$DN?$AA?$DN?$AA?5?$AA0?$AA?$CJ?$AA?$AA@ 10192494     LIBCMTD:read.obj
 0003:000174b8       ??_C@_1CG@OHLJHGGK@?$AA?$CI?$AAi?$AAn?$AAp?$AAu?$AAt?$AAb?$AAu?$AAf?$AA?5?$AA?$CB?$AA?$DN?$AA?5?$AAN?$AAU?$AAL?$AAL?$AA?$CJ?$AA?$AA@ 101924b8     LIBCMTD:read.obj
 0003:000174e0       ??_C@_1BK@JJBHNDKJ@?$AA_?$AAr?$AAe?$AAa?$AAd?$AA_?$AAn?$AAo?$AAl?$AAo?$AAc?$AAk?$AA?$AA@ 101924e0     LIBCMTD:read.obj
 0003:00017650       ??_C@_0L@KDOEJCKC@_nextafter?$AA@ 10192650     LIBCMTD:_fpexcept_.obj
 0003:0001765c       ??_C@_05JGDBENOH@_logb?$AA@ 1019265c     LIBCMTD:_fpexcept_.obj
 0003:00017664       ??_C@_03ONILCKOB@_yn?$AA@  10192664     LIBCMTD:_fpexcept_.obj
 0003:00017668       ??_C@_03NAKIGLHK@_y1?$AA@  10192668     LIBCMTD:_fpexcept_.obj
 0003:0001766c       ??_C@_03MJLDFKDL@_y0?$AA@  1019266c     LIBCMTD:_fpexcept_.obj
 0003:00017670       ??_C@_05GKKHEGJL@frexp?$AA@ 10192670     LIBCMTD:_fpexcept_.obj
 0003:00017678       ??_C@_04KEPJIHGP@fmod?$AA@ 10192678     LIBCMTD:_fpexcept_.obj
 0003:00017680       ??_C@_06MEIMCGCF@_hypot?$AA@ 10192680     LIBCMTD:_fpexcept_.obj
 0003:00017688       ??_C@_05KBKMEMPO@_cabs?$AA@ 10192688     LIBCMTD:_fpexcept_.obj
 0003:00017690       ??_C@_05CEJMAHNP@ldexp?$AA@ 10192690     LIBCMTD:_fpexcept_.obj
 0003:00017698       ??_C@_04EHEDPDJG@modf?$AA@ 10192698     LIBCMTD:_fpexcept_.obj
 0003:000176a0       ??_C@_04ODHECPBC@fabs?$AA@ 101926a0     LIBCMTD:_fpexcept_.obj
 0003:000176a8       ??_C@_05PBJFFIGL@floor?$AA@ 101926a8     LIBCMTD:_fpexcept_.obj
 0003:000176b0       ??_C@_04GFPJNGEK@ceil?$AA@ 101926b0     LIBCMTD:_fpexcept_.obj
 0003:000176b8       ??_C@_03IIINPABG@tan?$AA@  101926b8     LIBCMTD:_fpexcept_.obj
 0003:000176bc       ??_C@_03LALBNOCG@cos?$AA@  101926bc     LIBCMTD:_fpexcept_.obj
 0003:000176c0       ??_C@_03BLEJJJBH@sin?$AA@  101926c0     LIBCMTD:_fpexcept_.obj
 0003:000176c4       ??_C@_04EIAKFFMI@sqrt?$AA@ 101926c4     LIBCMTD:_fpexcept_.obj
 0003:000176cc       ??_C@_05KNGEOGJB@atan2?$AA@ 101926cc     LIBCMTD:_fpexcept_.obj
 0003:000176d4       ??_C@_04MLLJIGOK@atan?$AA@ 101926d4     LIBCMTD:_fpexcept_.obj
 0003:000176dc       ??_C@_04PDIFKINK@acos?$AA@ 101926dc     LIBCMTD:_fpexcept_.obj
 0003:000176e4       ??_C@_04FIHNOPOL@asin?$AA@ 101926e4     LIBCMTD:_fpexcept_.obj
 0003:000176ec       ??_C@_04FJHINJAO@tanh?$AA@ 101926ec     LIBCMTD:_fpexcept_.obj
 0003:000176f4       ??_C@_04HPJJNFIM@cosh?$AA@ 101926f4     LIBCMTD:_fpexcept_.obj
 0003:000176fc       ??_C@_04COOMCNPB@sinh?$AA@ 101926fc     LIBCMTD:_fpexcept_.obj
 0003:00017704       ??_C@_05HGHHAHAP@log10?$AA@ 10192704     LIBCMTD:_fpexcept_.obj
 0003:0001770c       ??_C@_03MGHMBJCF@log?$AA@  1019270c     LIBCMTD:_fpexcept_.obj
 0003:00017710       ??_C@_03JGHBODFD@pow?$AA@  10192710     LIBCMTD:_fpexcept_.obj
 0003:00017714       ??_C@_03KHJOGHMM@exp?$AA@  10192714     LIBCMTD:_fpexcept_.obj
 0003:0001b870       ??_C@_0DB@OLNNDFNH@f?3?2dd?2vctools?2crt_bld?2self_x86?2c@ 10196870     LIBCMTD:_sftbuf.obj
 0003:0001b8a8       ??_C@_1GC@DGAFOCMO@?$AAf?$AA?3?$AA?2?$AAd?$AAd?$AA?2?$AAv?$AAc?$AAt?$AAo?$AAo?$AAl?$AAs?$AA?2?$AAc?$AAr?$AAt?$AA_?$AAb?$AAl?$AAd?$AA?2?$AAs?$AAe?$AAl?$AAf?$AA_?$AAx?$AA8?$AA6?$AA?2?$AAc@ 101968a8     LIBCMTD:_sftbuf.obj
 0003:0001b90c       ??_C@_1CO@KCKAACMI@?$AAf?$AAl?$AAa?$AAg?$AA?5?$AA?$DN?$AA?$DN?$AA?5?$AA0?$AA?5?$AA?$HM?$AA?$HM?$AA?5?$AAf?$AAl?$AAa?$AAg?$AA?5?$AA?$DN?$AA?$DN?$AA?5?$AA1?$AA?$AA@ 1019690c     LIBCMTD:_sftbuf.obj
 0003:0001b93c       ??_C@_1BO@JGFPDJCP@?$AAv?$AAp?$AAr?$AAi?$AAn?$AAt?$AAf?$AA_?$AAh?$AAe?$AAl?$AAp?$AAe?$AAr?$AA?$AA@ 1019693c     LIBCMTD:vprintf.obj
 0003:0001b960       ??_C@_1GC@DHFFJKMC@?$AAf?$AA?3?$AA?2?$AAd?$AAd?$AA?2?$AAv?$AAc?$AAt?$AAo?$AAo?$AAl?$AAs?$AA?2?$AAc?$AAr?$AAt?$AA_?$AAb?$AAl?$AAd?$AA?2?$AAs?$AAe?$AAl?$AAf?$AA_?$AAx?$AA8?$AA6?$AA?2?$AAc@ 10196960     LIBCMTD:vprintf.obj
 0003:0001b9c4       ??_C@_1O@KOFKDHPL@?$AA_?$AAw?$AAr?$AAi?$AAt?$AAe?$AA?$AA@ 101969c4     LIBCMTD:write.obj
 0003:0001b9d8       ??_C@_1FO@EPLDPDDL@?$AAf?$AA?3?$AA?2?$AAd?$AAd?$AA?2?$AAv?$AAc?$AAt?$AAo?$AAo?$AAl?$AAs?$AA?2?$AAc?$AAr?$AAt?$AA_?$AAb?$AAl?$AAd?$AA?2?$AAs?$AAe?$AAl?$AAf?$AA_?$AAx?$AA8?$AA6?$AA?2?$AAc@ 101969d8     LIBCMTD:write.obj
 0003:0001ba38       ??_C@_1DI@CNMHHHLG@?$AAi?$AAs?$AAl?$AAe?$AAa?$AAd?$AAb?$AAy?$AAt?$AAe?$AA?$CI?$AA_?$AAd?$AAb?$AAc?$AAs?$AAB?$AAu?$AAf?$AAf?$AAe?$AAr?$AA?$CI?$AAf?$AAh?$AA?$CJ?$AA?$CJ?$AA?$AA@ 10196a38     LIBCMTD:write.obj
 0003:0001ba70       ??_C@_1BM@NCANHCIP@?$AA_?$AAw?$AAr?$AAi?$AAt?$AAe?$AA_?$AAn?$AAo?$AAl?$AAo?$AAc?$AAk?$AA?$AA@ 10196a70     LIBCMTD:write.obj
 0003:0001ba8c       ??_C@_1BM@KFJLMBPG@?$AA?$CI?$AAb?$AAu?$AAf?$AA?5?$AA?$CB?$AA?$DN?$AA?5?$AAN?$AAU?$AAL?$AAL?$AA?$CJ?$AA?$AA@ 10196a8c     LIBCMTD:write.obj
 0003:0001baa8       ??_C@_03KHICJKCI@?4?4?4?$AA@ 10196aa8     LIBCMTD:dbgrpt.obj
 0003:0001baac       ??_C@_0BB@NAGLCMLI@Assertion?5Failed?$AA@ 10196aac     LIBCMTD:dbgrpt.obj
 0003:0001bac0       ??_C@_05NAOIJFC@Error?$AA@ 10196ac0     LIBCMTD:dbgrpt.obj
 0003:0001bac8       ??_C@_07KGMMFLDN@Warning?$AA@ 10196ac8     LIBCMTD:dbgrpt.obj
 0003:0001badc       ??_C@_1CG@GNMJDMIO@?$AA_?$AAC?$AAr?$AAt?$AAS?$AAe?$AAt?$AAR?$AAe?$AAp?$AAo?$AAr?$AAt?$AAH?$AAo?$AAo?$AAk?$AA2?$AA?$AA@ 10196adc     LIBCMTD:dbgrpt.obj
 0003:0001bb04       ??_C@_0CD@EBCGLDDL@Microsoft?5Visual?5C?$CL?$CL?5Debug?5Libra@ 10196b04     LIBCMTD:dbgrpt.obj
 0003:0001bb28       ??_C@_0FF@CCONDJCB@Debug?5?$CFs?$CB?6?6Program?3?5?$CFs?$CFs?$CFs?$CFs?$CFs?$CFs@ 10196b28     LIBCMTD:dbgrpt.obj
 0003:0001bb80       ??_C@_09OFBFHMBK@?6Module?3?5?$AA@ 10196b80     LIBCMTD:dbgrpt.obj
 0003:0001bb8c       ??_C@_07OPHPPLBG@?6File?3?5?$AA@ 10196b8c     LIBCMTD:dbgrpt.obj
 0003:0001bb94       ??_C@_07DBMPPHDI@?6Line?3?5?$AA@ 10196b94     LIBCMTD:dbgrpt.obj
 0003:0001bb9c       ??_C@_02PHMGELLB@?6?6?$AA@ 10196b9c     LIBCMTD:dbgrpt.obj
 0003:0001bba0       ??_C@_0N@MEECIJGN@Expression?3?5?$AA@ 10196ba0     LIBCMTD:dbgrpt.obj
 0003:0001bbb0       ??_C@_0HD@GNBNFCCL@?6?6For?5information?5on?5how?5your?5pr@ 10196bb0     LIBCMTD:dbgrpt.obj
 0003:0001bc24       ??_C@_0BH@DNAGHKFM@?$DMprogram?5name?5unknown?$DO?$AA@ 10196c24     LIBCMTD:dbgrpt.obj
 0003:0001bc40       ??_C@_1GG@DLDHOIGE@?$AAs?$AAt?$AAr?$AAc?$AAp?$AAy?$AA_?$AAs?$AA?$CI?$AAs?$AAz?$AAE?$AAx?$AAe?$AAN?$AAa?$AAm?$AAe?$AA?0?$AA?5?$AA2?$AA6?$AA0?$AA?0?$AA?5?$AA?$CC?$AA?$DM?$AAp?$AAr?$AAo?$AAg?$AAr@ 10196c40     LIBCMTD:dbgrpt.obj
 0003:0001bca8       ??_C@_1CI@IDOKFLAJ@?$AA_?$AA_?$AAc?$AAr?$AAt?$AAM?$AAe?$AAs?$AAs?$AAa?$AAg?$AAe?$AAW?$AAi?$AAn?$AAd?$AAo?$AAw?$AAA?$AA?$AA@ 10196ca8     LIBCMTD:dbgrpt.obj
 0003:0001bcd0       ??_C@_1BK@JMCGJOCC@?$AA_?$AAe?$AAx?$AAp?$AAa?$AAn?$AAd?$AA_?$AAb?$AAa?$AAs?$AAe?$AA?$AA@ 10196cd0     LIBCMTD:expand.obj
 0003:0001bcf0       ??_C@_1GA@EBHFLDNH@?$AAf?$AA?3?$AA?2?$AAd?$AAd?$AA?2?$AAv?$AAc?$AAt?$AAo?$AAo?$AAl?$AAs?$AA?2?$AAc?$AAr?$AAt?$AA_?$AAb?$AAl?$AAd?$AA?2?$AAs?$AAe?$AAl?$AAf?$AA_?$AAx?$AA8?$AA6?$AA?2?$AAc@ 10196cf0     LIBCMTD:expand.obj
 0003:0001bd50       ??_C@_1BO@KFIJIAEA@?$AAp?$AAB?$AAl?$AAo?$AAc?$AAk?$AA?5?$AA?$CB?$AA?$DN?$AA?5?$AAN?$AAU?$AAL?$AAL?$AA?$AA@ 10196d50     LIBCMTD:expand.obj
 0003:0001bd70       ??_C@_0BF@PEEJCKGM@HeapQueryInformation?$AA@ 10196d70     LIBCMTD:expand.obj
 0003:0001bd88       ??_C@_1BK@MGMFAEKH@?$AAk?$AAe?$AAr?$AAn?$AAe?$AAl?$AA3?$AA2?$AA?4?$AAd?$AAl?$AAl?$AA?$AA@ 10196d88     LIBCMTD:expand.obj
 0003:0001bda8       ??_C@_1GE@JDDMFOID@?$AAf?$AA?3?$AA?2?$AAd?$AAd?$AA?2?$AAv?$AAc?$AAt?$AAo?$AAo?$AAl?$AAs?$AA?2?$AAc?$AAr?$AAt?$AA_?$AAb?$AAl?$AAd?$AA?2?$AAs?$AAe?$AAl?$AAf?$AA_?$AAx?$AA8?$AA6?$AA?2?$AAc@ 10196da8     LIBCMTD:heapinit.obj
 0003:0001be0c       ??_C@_1BC@DENNNKIM@?$AA_?$AAc?$AAr?$AAt?$AAh?$AAe?$AAa?$AAp?$AA?$AA@ 10196e0c     LIBCMTD:heapinit.obj
 0003:0001be20       ??_C@_1GA@CMCJKKIB@?$AAf?$AA?3?$AA?2?$AAd?$AAd?$AA?2?$AAv?$AAc?$AAt?$AAo?$AAo?$AAl?$AAs?$AA?2?$AAc?$AAr?$AAt?$AA_?$AAb?$AAl?$AAd?$AA?2?$AAs?$AAe?$AAl?$AAf?$AA_?$AAx?$AA8?$AA6?$AA?2?$AAc@ 10196e20     LIBCMTD:sbheap.obj
 0003:0001be80       ??_C@_1IC@MOGBEBCE@?$AA?$CI?$AAt?$AAh?$AAr?$AAe?$AAs?$AAh?$AAo?$AAl?$AAd?$AA?5?$AA?$DM?$AA?$DN?$AA?5?$AAM?$AAA?$AAX?$AA_?$AAA?$AAL?$AAL?$AAO?$AAC?$AA_?$AAD?$AAA?$AAT?$AAA?$AA_?$AAS?$AAI?$AAZ@ 10196e80     LIBCMTD:sbheap.obj
 0003:0001bf04       ??_C@_1CG@BBFCGKBK@?$AA_?$AAs?$AAe?$AAt?$AA_?$AAs?$AAb?$AAh?$AA_?$AAt?$AAh?$AAr?$AAe?$AAs?$AAh?$AAo?$AAl?$AAd?$AA?$AA@ 10196f04     LIBCMTD:sbheap.obj
 0003:0001bf30       ??_C@_1EC@DACAONFE@?$AAt?$AAh?$AAr?$AAe?$AAs?$AAh?$AAo?$AAl?$AAd?$AA?5?$AA?$DM?$AA?$DN?$AA?5?$AAM?$AAA?$AAX?$AA_?$AAA?$AAL?$AAL?$AAO?$AAC?$AA_?$AAD?$AAA?$AAT?$AAA?$AA_?$AAS?$AAI?$AAZ?$AAE@ 10196f30     LIBCMTD:sbheap.obj
 0003:0001bf74       ??_C@_1BM@GFNECEDD@?$AA_?$AAs?$AAe?$AAt?$AA_?$AAa?$AAm?$AAb?$AAl?$AAk?$AAs?$AAi?$AAz?$AA?$AA@ 10196f74     LIBCMTD:sbheap.obj
 0003:0001bf90       ??_C@_1DK@BKLENMLC@?$AA0?$AA?5?$AA?$DM?$AA?5?$AAs?$AAi?$AAz?$AAe?$AA?5?$AA?$CG?$AA?$CG?$AA?5?$AAs?$AAi?$AAz?$AAe?$AA?5?$AA?$DM?$AA?$DN?$AA?5?$AAU?$AAI?$AAN?$AAT?$AA_?$AAM?$AAA?$AAX?$AA?$AA@ 10196f90     LIBCMTD:sbheap.obj
 0003:0001bfcc       ??_C@_1BM@OFBCOJJF@?$AA_?$AAg?$AAe?$AAt?$AA_?$AAa?$AAm?$AAb?$AAl?$AAk?$AAs?$AAi?$AAz?$AA?$AA@ 10196fcc     LIBCMTD:sbheap.obj
 0003:0001bfe8       ??_C@_1BM@IELHFPPM@?$AAp?$AAS?$AAi?$AAz?$AAe?$AA?5?$AA?$CB?$AA?$DN?$AA?5?$AAN?$AAU?$AAL?$AAL?$AA?$AA@ 10196fe8     LIBCMTD:sbheap.obj
 0003:0001c004       ??_C@_1DE@MMOGFGHF@?$AAs?$AAt?$AAr?$AAc?$AAp?$AAy?$AA_?$AAs?$AA?$CI?$AA?$CK?$AAe?$AAn?$AAv?$AA?0?$AA?5?$AAc?$AAc?$AAh?$AAa?$AAr?$AAs?$AA?0?$AA?5?$AAp?$AA?$CJ?$AA?$AA@ 10197004     LIBCMTD:stdenvp.obj
 0003:0001c038       ??_C@_1BC@GHMCNHHL@?$AA_?$AAs?$AAe?$AAt?$AAe?$AAn?$AAv?$AAp?$AA?$AA@ 10197038     LIBCMTD:stdenvp.obj
 0003:0001c050       ??_C@_1GC@DGBFLDBN@?$AAf?$AA?3?$AA?2?$AAd?$AAd?$AA?2?$AAv?$AAc?$AAt?$AAo?$AAo?$AAl?$AAs?$AA?2?$AAc?$AAr?$AAt?$AA_?$AAb?$AAl?$AAd?$AA?2?$AAs?$AAe?$AAl?$AAf?$AA_?$AAx?$AA8?$AA6?$AA?2?$AAc@ 10197050     LIBCMTD:stdenvp.obj
 0003:0001c0b4       ??_C@_0DB@BMEBJJKP@f?3?2dd?2vctools?2crt_bld?2self_x86?2c@ 101970b4     LIBCMTD:stdenvp.obj
 0003:0001c0e8       ??_C@_0DB@OEPBJOLC@f?3?2dd?2vctools?2crt_bld?2self_x86?2c@ 101970e8     LIBCMTD:stdargv.obj
 0003:0001c11c       ??_C@_0CP@PPLBCJDN@f?3?2dd?2vctools?2crt_bld?2self_x86?2c@ 1019711c     LIBCMTD:a_env.obj
 0003:0001c150       __XcptActTab               10197150     LIBCMTD:winxfltr.obj
 0003:0001c1c8       ??_C@_0P@GGKDKEEG@runtime?5error?5?$AA@ 101971c8     LIBCMTD:crt0msg.obj
 0003:0001c1d8       ??_C@_02PCIJFNDE@?$AN?6?$AA@ 101971d8     LIBCMTD:crt0msg.obj
 0003:0001c1dc       ??_C@_0O@MJNIPGOH@TLOSS?5error?$AN?6?$AA@ 101971dc     LIBCMTD:crt0msg.obj
 0003:0001c1ec       ??_C@_0N@BONNPDHF@SING?5error?$AN?6?$AA@ 101971ec     LIBCMTD:crt0msg.obj
 0003:0001c1fc       ??_C@_0P@MBDAJNE@DOMAIN?5error?$AN?6?$AA@ 101971fc     LIBCMTD:crt0msg.obj
 0003:0001c210       ??_C@_0BFB@HKKMCDOL@R6034?$AN?6An?5application?5has?5made?5a@ 10197210     LIBCMTD:crt0msg.obj
 0003:0001c368       ??_C@_0PH@EPAFIJ@R6033?$AN?6?9?5Attempt?5to?5use?5MSIL?5cod@ 10197368     LIBCMTD:crt0msg.obj
 0003:0001c460       ??_C@_0DD@BKEEABMM@R6032?$AN?6?9?5not?5enough?5space?5for?5lo@ 10197460     LIBCMTD:crt0msg.obj
 0003:0001c498       ??_C@_0GD@OFKILIED@R6031?$AN?6?9?5Attempt?5to?5initialize?5t@ 10197498     LIBCMTD:crt0msg.obj
 0003:0001c4fc       ??_C@_0BP@LPMHJOKI@R6030?$AN?6?9?5CRT?5not?5initialized?$AN?6?$AA@ 101974fc     LIBCMTD:crt0msg.obj
 0003:0001c51c       ??_C@_0CF@KJDAIALP@R6028?$AN?6?9?5unable?5to?5initialize?5he@ 1019751c     LIBCMTD:crt0msg.obj
 0003:0001c544       ??_C@_0DF@GAKBPDFP@R6027?$AN?6?9?5not?5enough?5space?5for?5lo@ 10197544     LIBCMTD:crt0msg.obj
 0003:0001c57c       ??_C@_0DF@IBLNNAIG@R6026?$AN?6?9?5not?5enough?5space?5for?5st@ 1019757c     LIBCMTD:crt0msg.obj
 0003:0001c5b4       ??_C@_0CG@IOHKGFNJ@R6025?$AN?6?9?5pure?5virtual?5function?5c@ 101975b4     LIBCMTD:crt0msg.obj
 0003:0001c5dc       ??_C@_0DF@JIJJFJDC@R6024?$AN?6?9?5not?5enough?5space?5for?5_o@ 101975dc     LIBCMTD:crt0msg.obj
 0003:0001c614       ??_C@_0CJ@EGEJHFME@R6019?$AN?6?9?5unable?5to?5open?5console?5@ 10197614     LIBCMTD:crt0msg.obj
 0003:0001c640       ??_C@_0CB@GNHNIELH@R6018?$AN?6?9?5unexpected?5heap?5error?$AN?6@ 10197640     LIBCMTD:crt0msg.obj
 0003:0001c664       ??_C@_0CN@FOLDKNG@R6017?$AN?6?9?5unexpected?5multithread?5@ 10197664     LIBCMTD:crt0msg.obj
 0003:0001c694       ??_C@_0CM@FAHFJNHO@R6016?$AN?6?9?5not?5enough?5space?5for?5th@ 10197694     LIBCMTD:crt0msg.obj
 0003:0001c6c0       ??_C@_0JG@LBKMGKLD@?$AN?6This?5application?5has?5requested@ 101976c0     LIBCMTD:crt0msg.obj
 0003:0001c758       ??_C@_0CM@FLCNIPKK@R6009?$AN?6?9?5not?5enough?5space?5for?5en@ 10197758     LIBCMTD:crt0msg.obj
 0003:0001c784       ??_C@_0CK@KMMJOAPP@R6008?$AN?6?9?5not?5enough?5space?5for?5ar@ 10197784     LIBCMTD:crt0msg.obj
 0003:0001c7b0       ??_C@_0CN@LEKKICBM@R6002?$AN?6?9?5floating?5point?5support?5@ 101977b0     LIBCMTD:crt0msg.obj
 0003:0001c7e0       ??_C@_0CF@GOGNBNAK@Microsoft?5Visual?5C?$CL?$CL?5Runtime?5Lib@ 101977e0     LIBCMTD:crt0msg.obj
 0003:0001c808       ??_C@_1KC@JBIKIPNF@?$AAs?$AAt?$AAr?$AAc?$AAa?$AAt?$AA_?$AAs?$AA?$CI?$AAo?$AAu?$AAt?$AAm?$AAs?$AAg?$AA?0?$AA?5?$AA?$CI?$AAs?$AAi?$AAz?$AAe?$AAo?$AAf?$AA?$CI?$AAo?$AAu?$AAt?$AAm?$AAs?$AAg?$AA?$CJ@ 10197808     LIBCMTD:crt0msg.obj
 0003:0001c8b0       ??_C@_1HO@POLIDBMF@?$AAs?$AAt?$AAr?$AAc?$AAa?$AAt?$AA_?$AAs?$AA?$CI?$AAo?$AAu?$AAt?$AAm?$AAs?$AAg?$AA?0?$AA?5?$AA?$CI?$AAs?$AAi?$AAz?$AAe?$AAo?$AAf?$AA?$CI?$AAo?$AAu?$AAt?$AAm?$AAs?$AAg?$AA?$CJ@ 101978b0     LIBCMTD:crt0msg.obj
 0003:0001c930       ??_C@_1HG@CJJGKFHK@?$AAs?$AAt?$AAr?$AAn?$AAc?$AAp?$AAy?$AA_?$AAs?$AA?$CI?$AAp?$AAc?$AAh?$AA?0?$AA?5?$AAp?$AAr?$AAo?$AAg?$AAn?$AAa?$AAm?$AAe?$AA_?$AAs?$AAi?$AAz?$AAe?$AA?5?$AA?9?$AA?5?$AA?$CI@ 10197930     LIBCMTD:crt0msg.obj
 0003:0001c9a8       ??_C@_1HI@FOOPEDMH@?$AAs?$AAt?$AAr?$AAc?$AAp?$AAy?$AA_?$AAs?$AA?$CI?$AAp?$AAr?$AAo?$AAg?$AAn?$AAa?$AAm?$AAe?$AA?0?$AA?5?$AAp?$AAr?$AAo?$AAg?$AAn?$AAa?$AAm?$AAe?$AA_?$AAs?$AAi?$AAz?$AAe@ 101979a8     LIBCMTD:crt0msg.obj
 0003:0001ca20       ??_C@_0BK@OFGJDLJJ@Runtime?5Error?$CB?6?6Program?3?5?$AA@ 10197a20     LIBCMTD:crt0msg.obj
 0003:0001ca40       ??_C@_1KM@NKKPELHG@?$AAs?$AAt?$AAr?$AAc?$AAp?$AAy?$AA_?$AAs?$AA?$CI?$AAo?$AAu?$AAt?$AAm?$AAs?$AAg?$AA?0?$AA?5?$AA?$CI?$AAs?$AAi?$AAz?$AAe?$AAo?$AAf?$AA?$CI?$AAo?$AAu?$AAt?$AAm?$AAs?$AAg?$AA?$CJ@ 10197a40     LIBCMTD:crt0msg.obj
 0003:0001caec       ??_C@_1BI@EAHMBMEC@?$AA_?$AAN?$AAM?$AAS?$AAG?$AA_?$AAW?$AAR?$AAI?$AAT?$AAE?$AA?$AA@ 10197aec     LIBCMTD:crt0msg.obj
 0003:0001cb08       ??_C@_1GC@HKOJBOFF@?$AAf?$AA?3?$AA?2?$AAd?$AAd?$AA?2?$AAv?$AAc?$AAt?$AAo?$AAo?$AAl?$AAs?$AA?2?$AAc?$AAr?$AAt?$AA_?$AAb?$AAl?$AAd?$AA?2?$AAs?$AAe?$AAl?$AAf?$AA_?$AAx?$AA8?$AA6?$AA?2?$AAc@ 10197b08     LIBCMTD:crt0msg.obj
 0003:0001cb6c       ??_C@_1DG@LNNHNFHJ@?$AA?$CI?$AA_?$AAo?$AAs?$AAf?$AAi?$AAl?$AAe?$AA?$CI?$AAf?$AAi?$AAl?$AAe?$AAd?$AAe?$AAs?$AA?$CJ?$AA?5?$AA?$CG?$AA?5?$AAF?$AAO?$AAP?$AAE?$AAN?$AA?$CJ?$AA?$AA@ 10197b6c     LIBCMTD:commit.obj
 0003:0001cba4       ??_C@_1BA@FLNMBBIM@?$AA_?$AAc?$AAo?$AAm?$AAm?$AAi?$AAt?$AA?$AA@ 10197ba4     LIBCMTD:commit.obj
 0003:0001cbb8       ??_C@_1GA@BOPCOCFN@?$AAf?$AA?3?$AA?2?$AAd?$AAd?$AA?2?$AAv?$AAc?$AAt?$AAo?$AAo?$AAl?$AAs?$AA?2?$AAc?$AAr?$AAt?$AA_?$AAb?$AAl?$AAd?$AA?2?$AAs?$AAe?$AAl?$AAf?$AA_?$AAx?$AA8?$AA6?$AA?2?$AAc@ 10197bb8     LIBCMTD:commit.obj
 0003:0001cc18       ??_C@_1HC@KFLBHHBC@?$AA?$CI?$AAf?$AAi?$AAl?$AAe?$AAd?$AAe?$AAs?$AA?5?$AA?$DO?$AA?$DN?$AA?5?$AA0?$AA?5?$AA?$CG?$AA?$CG?$AA?5?$AA?$CI?$AAu?$AAn?$AAs?$AAi?$AAg?$AAn?$AAe?$AAd?$AA?$CJ?$AAf?$AAi?$AAl?$AAe?$AAd@ 10197c18     LIBCMTD:commit.obj
 0003:0001ccf8       ??_C@_05EOHGHCHD@exp10?$AA@ 10197cf8     LIBCMTD:_libm_error_.obj
 0003:0001cd00       ??_C@_13NOLLCAOD@?$AA?$AA?$AA?$AA@ 10197d00     LIBCMTD:a_map.obj
 0003:0001cd08       ??_C@_1GA@INJGGEBC@?$AAf?$AA?3?$AA?2?$AAd?$AAd?$AA?2?$AAv?$AAc?$AAt?$AAo?$AAo?$AAl?$AAs?$AA?2?$AAc?$AAr?$AAt?$AA_?$AAb?$AAl?$AAd?$AA?2?$AAs?$AAe?$AAl?$AAf?$AA_?$AAx?$AA8?$AA6?$AA?2?$AAc@ 10197d08     LIBCMTD:a_map.obj
 0003:0001cd68       ??_C@_1FE@KNPCCODH@?$AA?$CI?$AA?$CC?$AAC?$AAo?$AAr?$AAr?$AAu?$AAp?$AAt?$AAe?$AAd?$AA?5?$AAp?$AAo?$AAi?$AAn?$AAt?$AAe?$AAr?$AA?5?$AAp?$AAa?$AAs?$AAs?$AAe?$AAd?$AA?5?$AAt?$AAo?$AA?5?$AA_?$AAf@ 10197d68     LIBCMTD:a_map.obj
 0003:0001cdbc       ??_C@_1CA@OEHMHBJF@?$AAv?$AAf?$AAp?$AAr?$AAi?$AAn?$AAt?$AAf?$AA_?$AAh?$AAe?$AAl?$AAp?$AAe?$AAr?$AA?$AA@ 10197dbc     LIBCMTD:vfprintf.obj
 0003:0001cde0       ??_C@_1GE@PEEPNGBM@?$AAf?$AA?3?$AA?2?$AAd?$AAd?$AA?2?$AAv?$AAc?$AAt?$AAo?$AAo?$AAl?$AAs?$AA?2?$AAc?$AAr?$AAt?$AA_?$AAb?$AAl?$AAd?$AA?2?$AAs?$AAe?$AAl?$AAf?$AA_?$AAx?$AA8?$AA6?$AA?2?$AAc@ 10197de0     LIBCMTD:vfprintf.obj
 0003:0001ce44       ??_C@_0DB@KIKNCIEC@f?3?2dd?2vctools?2crt_bld?2self_x86?2c@ 10197e44     LIBCMTD:osfinfo.obj
 0003:0001ce78       ??_C@_1BO@EMBOBGKE@?$AA_?$AAg?$AAe?$AAt?$AA_?$AAo?$AAs?$AAf?$AAh?$AAa?$AAn?$AAd?$AAl?$AAe?$AA?$AA@ 10197e78     LIBCMTD:osfinfo.obj
 0003:0001ce98       ??_C@_1GC@MLKLDJJG@?$AAf?$AA?3?$AA?2?$AAd?$AAd?$AA?2?$AAv?$AAc?$AAt?$AAo?$AAo?$AAl?$AAs?$AA?2?$AAc?$AAr?$AAt?$AA_?$AAb?$AAl?$AAd?$AA?2?$AAs?$AAe?$AAl?$AAf?$AA_?$AAx?$AA8?$AA6?$AA?2?$AAc@ 10197e98     LIBCMTD:osfinfo.obj
 0003:0001cefc       ??_C@_0BG@KLEAJEFJ@Illegal?5byte?5sequence?$AA@ 10197efc     LIBCMTD:syserr.obj
 0003:0001cf14       ??_C@_0BE@ICMCHPHH@Directory?5not?5empty?$AA@ 10197f14     LIBCMTD:syserr.obj
 0003:0001cf28       ??_C@_0BJ@IHEHINLI@Function?5not?5implemented?$AA@ 10197f28     LIBCMTD:syserr.obj
 0003:0001cf44       ??_C@_0BD@CLHBCGPB@No?5locks?5available?$AA@ 10197f44     LIBCMTD:syserr.obj
 0003:0001cf58       ??_C@_0BC@BEDIHIDK@Filename?5too?5long?$AA@ 10197f58     LIBCMTD:syserr.obj
 0003:0001cf6c       ??_C@_0BK@JAEBMJJM@Resource?5deadlock?5avoided?$AA@ 10197f6c     LIBCMTD:syserr.obj
 0003:0001cf88       ??_C@_0BB@FCBJFCAJ@Result?5too?5large?$AA@ 10197f88     LIBCMTD:syserr.obj
 0003:0001cf9c       ??_C@_0N@MMJPGLJK@Domain?5error?$AA@ 10197f9c     LIBCMTD:syserr.obj
 0003:0001cfac       ??_C@_0M@LHEPIIOM@Broken?5pipe?$AA@ 10197fac     LIBCMTD:syserr.obj
 0003:0001cfb8       ??_C@_0P@PKCJJLLM@Too?5many?5links?$AA@ 10197fb8     LIBCMTD:syserr.obj
 0003:0001cfc8       ??_C@_0BG@DDBFNKBH@Read?9only?5file?5system?$AA@ 10197fc8     LIBCMTD:syserr.obj
 0003:0001cfe0       ??_C@_0N@FEHLOILP@Invalid?5seek?$AA@ 10197fe0     LIBCMTD:syserr.obj
 0003:0001cff0       ??_C@_0BI@FEALHKLD@No?5space?5left?5on?5device?$AA@ 10197ff0     LIBCMTD:syserr.obj
 0003:0001d008       ??_C@_0P@LFMMIPAE@File?5too?5large?$AA@ 10198008     LIBCMTD:syserr.obj
 0003:0001d018       ??_C@_0CE@ONOKNLPF@Inappropriate?5I?1O?5control?5operat@ 10198018     LIBCMTD:syserr.obj
 0003:0001d03c       ??_C@_0BE@INBJMKGG@Too?5many?5open?5files?$AA@ 1019803c     LIBCMTD:syserr.obj
 0003:0001d050       ??_C@_0BO@IIFBODJE@Too?5many?5open?5files?5in?5system?$AA@ 10198050     LIBCMTD:syserr.obj
 0003:0001d070       ??_C@_0BB@HMGGCEBG@Invalid?5argument?$AA@ 10198070     LIBCMTD:syserr.obj
 0003:0001d084       ??_C@_0P@NDHGCGKE@Is?5a?5directory?$AA@ 10198084     LIBCMTD:syserr.obj
 0003:0001d094       ??_C@_0BA@CJBACOOL@Not?5a?5directory?$AA@ 10198094     LIBCMTD:syserr.obj
 0003:0001d0a4       ??_C@_0P@NLEIANHE@No?5such?5device?$AA@ 101980a4     LIBCMTD:syserr.obj
 0003:0001d0b4       ??_C@_0O@OAMDNOCP@Improper?5link?$AA@ 101980b4     LIBCMTD:syserr.obj
 0003:0001d0c4       ??_C@_0M@NAAJNNGH@File?5exists?$AA@ 101980c4     LIBCMTD:syserr.obj
 0003:0001d0d0       ??_C@_0BA@BIBLIOEK@Resource?5device?$AA@ 101980d0     LIBCMTD:syserr.obj
 0003:0001d0e0       ??_C@_0O@NIPGCINC@Unknown?5error?$AA@ 101980e0     LIBCMTD:syserr.obj
 0003:0001d0f0       ??_C@_0M@LOEHLCJD@Bad?5address?$AA@ 101980f0     LIBCMTD:syserr.obj
 0003:0001d0fc       ??_C@_0BC@HFNFNKAI@Permission?5denied?$AA@ 101980fc     LIBCMTD:syserr.obj
 0003:0001d110       ??_C@_0BB@IMDKMPFB@Not?5enough?5space?$AA@ 10198110     LIBCMTD:syserr.obj
 0003:0001d124       ??_C@_0CB@EPFKGNAK@Resource?5temporarily?5unavailable@ 10198124     LIBCMTD:syserr.obj
 0003:0001d148       ??_C@_0BD@LOHELEP@No?5child?5processes?$AA@ 10198148     LIBCMTD:syserr.obj
 0003:0001d15c       ??_C@_0BE@NFGDDCEF@Bad?5file?5descriptor?$AA@ 1019815c     LIBCMTD:syserr.obj
 0003:0001d170       ??_C@_0BC@HKPNECK@Exec?5format?5error?$AA@ 10198170     LIBCMTD:syserr.obj
 0003:0001d184       ??_C@_0BC@MFFGCDFL@Arg?5list?5too?5long?$AA@ 10198184     LIBCMTD:syserr.obj
 0003:0001d198       ??_C@_0BK@DPKMCKJ@No?5such?5device?5or?5address?$AA@ 10198198     LIBCMTD:syserr.obj
 0003:0001d1b4       ??_C@_0BD@KKNFOBBD@Input?1output?5error?$AA@ 101981b4     LIBCMTD:syserr.obj
 0003:0001d1c8       ??_C@_0BK@FJBOAFDK@Interrupted?5function?5call?$AA@ 101981c8     LIBCMTD:syserr.obj
 0003:0001d1e4       ??_C@_0BA@FKIAIBGA@No?5such?5process?$AA@ 101981e4     LIBCMTD:syserr.obj
 0003:0001d1f4       ??_C@_0BK@FMDHKPNF@No?5such?5file?5or?5directory?$AA@ 101981f4     LIBCMTD:syserr.obj
 0003:0001d210       ??_C@_0BI@BJFCGOHL@Operation?5not?5permitted?$AA@ 10198210     LIBCMTD:syserr.obj
 0003:0001d228       ??_C@_08INEPGKHH@No?5error?$AA@ 10198228     LIBCMTD:syserr.obj
 0003:0001d234       ??_C@_0BC@JEAENNKH@SystemFunction036?$AA@ 10198234     LIBCMTD:rand_s.obj
 0003:0001d248       ??_C@_1GA@EBEDGGGB@?$AA?$CI?$AA?$CC?$AAr?$AAa?$AAn?$AAd?$AA_?$AAs?$AA?5?$AAi?$AAs?$AA?5?$AAn?$AAo?$AAt?$AA?5?$AAa?$AAv?$AAa?$AAi?$AAl?$AAa?$AAb?$AAl?$AAe?$AA?5?$AAo?$AAn?$AA?5?$AAt?$AAh?$AAi@ 10198248     LIBCMTD:rand_s.obj
 0003:0001d2a8       ??_C@_1O@IJGPPOGF@?$AAr?$AAa?$AAn?$AAd?$AA_?$AAs?$AA?$AA@ 101982a8     LIBCMTD:rand_s.obj
 0003:0001d2b8       ??_C@_1GA@HBGBBKCD@?$AAf?$AA?3?$AA?2?$AAd?$AAd?$AA?2?$AAv?$AAc?$AAt?$AAo?$AAo?$AAl?$AAs?$AA?2?$AAc?$AAr?$AAt?$AA_?$AAb?$AAl?$AAd?$AA?2?$AAs?$AAe?$AAl?$AAf?$AA_?$AAx?$AA8?$AA6?$AA?2?$AAc@ 101982b8     LIBCMTD:rand_s.obj
 0003:0001d318       ??_C@_1CK@GFDNDKK@?$AA_?$AAR?$AAa?$AAn?$AAd?$AAo?$AAm?$AAV?$AAa?$AAl?$AAu?$AAe?$AA?5?$AA?$CB?$AA?$DN?$AA?5?$AAN?$AAU?$AAL?$AAL?$AA?$AA@ 10198318     LIBCMTD:rand_s.obj
 0003:0001d348       ??_C@_1GO@NGIGJNHH@?$AAs?$AAt?$AAr?$AAn?$AAc?$AAp?$AAy?$AA_?$AAs?$AA?$CI?$AA?$CK?$AAs?$AAt?$AAr?$AAa?$AAd?$AAd?$AAr?$AAe?$AAs?$AAs?$AA?0?$AA?5?$AAo?$AAu?$AAt?$AAs?$AAi?$AAz?$AAe?$AA?0?$AA?5@ 10198348     LIBCMTD:inithelp.obj
 0003:0001d3b8       ??_C@_1CA@KHHCPEI@?$AA_?$AA_?$AAg?$AAe?$AAt?$AAl?$AAo?$AAc?$AAa?$AAl?$AAe?$AAi?$AAn?$AAf?$AAo?$AA?$AA@ 101983b8     LIBCMTD:inithelp.obj
 0003:0001d3d8       ??_C@_1GE@PLPIMDHG@?$AAf?$AA?3?$AA?2?$AAd?$AAd?$AA?2?$AAv?$AAc?$AAt?$AAo?$AAo?$AAl?$AAs?$AA?2?$AAc?$AAr?$AAt?$AA_?$AAb?$AAl?$AAd?$AA?2?$AAs?$AAe?$AAl?$AAf?$AA_?$AAx?$AA8?$AA6?$AA?2?$AAc@ 101983d8     LIBCMTD:inithelp.obj
 0003:0001d43c       ??_C@_0DC@CFDMMFIG@f?3?2dd?2vctools?2crt_bld?2self_x86?2c@ 1019843c     LIBCMTD:inithelp.obj
 0003:0001d470       ___newctype                10198470     LIBCMTD:ctype.obj
 0003:0001d770       __wctype                   10198770     LIBCMTD:ctype.obj
 0003:0001d978       ___newclmap                10198978     LIBCMTD:ctype.obj
 0003:0001daf8       ___newcumap                10198af8     LIBCMTD:ctype.obj
 0003:0001dc78       ??_C@_1GE@GJCMHHMH@?$AAf?$AA?3?$AA?2?$AAd?$AAd?$AA?2?$AAv?$AAc?$AAt?$AAo?$AAo?$AAl?$AAs?$AA?2?$AAc?$AAr?$AAt?$AA_?$AAb?$AAl?$AAd?$AA?2?$AAs?$AAe?$AAl?$AAf?$AA_?$AAx?$AA8?$AA6?$AA?2?$AAc@ 10198c78     LIBCMTD:inittime.obj
 0003:0001dce0       ??_C@_1EE@FDHCFDHN@?$AAp?$AAl?$AAo?$AAc?$AAi?$AA?9?$AA?$DO?$AAl?$AAc?$AA_?$AAt?$AAi?$AAm?$AAe?$AA_?$AAc?$AAu?$AAr?$AAr?$AA?9?$AA?$DO?$AAr?$AAe?$AAf?$AAc?$AAo?$AAu?$AAn?$AAt?$AA?5?$AA?$DO?$AA?5@ 10198ce0     LIBCMTD:inittime.obj
 0003:0001dd24       ??_C@_0DC@KICHHNFK@f?3?2dd?2vctools?2crt_bld?2self_x86?2c@ 10198d24     LIBCMTD:inittime.obj
 0003:0001dd58       ??_C@_1GC@EDJOCBCL@?$AAf?$AA?3?$AA?2?$AAd?$AAd?$AA?2?$AAv?$AAc?$AAt?$AAo?$AAo?$AAl?$AAs?$AA?2?$AAc?$AAr?$AAt?$AA_?$AAb?$AAl?$AAd?$AA?2?$AAs?$AAe?$AAl?$AAf?$AA_?$AAx?$AA8?$AA6?$AA?2?$AAc@ 10198d58     LIBCMTD:initnum.obj
 0003:0001ddbc       ??_C@_1DM@IFKAINNE@?$AAp?$AAl?$AAo?$AAc?$AAi?$AA?9?$AA?$DO?$AAl?$AAc?$AAo?$AAn?$AAv?$AA_?$AAn?$AAu?$AAm?$AA_?$AAr?$AAe?$AAf?$AAc?$AAo?$AAu?$AAn?$AAt?$AA?5?$AA?$DO?$AA?5?$AA0?$AA?$AA@ 10198dbc     LIBCMTD:initnum.obj
 0003:0001ddf8       ??_C@_0DB@KKFMDHFI@f?3?2dd?2vctools?2crt_bld?2self_x86?2c@ 10198df8     LIBCMTD:initnum.obj
 0003:0001de30       ??_C@_1GC@IKADOFBJ@?$AAf?$AA?3?$AA?2?$AAd?$AAd?$AA?2?$AAv?$AAc?$AAt?$AAo?$AAo?$AAl?$AAs?$AA?2?$AAc?$AAr?$AAt?$AA_?$AAb?$AAl?$AAd?$AA?2?$AAs?$AAe?$AAl?$AAf?$AA_?$AAx?$AA8?$AA6?$AA?2?$AAc@ 10198e30     LIBCMTD:initmon.obj
 0003:0001de94       ??_C@_1DM@GKAPAMDO@?$AAp?$AAl?$AAo?$AAc?$AAi?$AA?9?$AA?$DO?$AAl?$AAc?$AAo?$AAn?$AAv?$AA_?$AAm?$AAo?$AAn?$AA_?$AAr?$AAe?$AAf?$AAc?$AAo?$AAu?$AAn?$AAt?$AA?5?$AA?$DO?$AA?5?$AA0?$AA?$AA@ 10198e94     LIBCMTD:initmon.obj
 0003:0001ded0       ??_C@_0DB@BECNGFDL@f?3?2dd?2vctools?2crt_bld?2self_x86?2c@ 10198ed0     LIBCMTD:initmon.obj
 0003:0001df04       ??_C@_1DG@NMBGBDM@?$AAp?$AAl?$AAo?$AAc?$AAi?$AA?9?$AA?$DO?$AAc?$AAt?$AAy?$AAp?$AAe?$AA1?$AA_?$AAr?$AAe?$AAf?$AAc?$AAo?$AAu?$AAn?$AAt?$AA?5?$AA?$DO?$AA?5?$AA0?$AA?$AA@ 10198f04     LIBCMTD:initctyp.obj
 0003:0001df40       ??_C@_1GE@OCPKBDKE@?$AAf?$AA?3?$AA?2?$AAd?$AAd?$AA?2?$AAv?$AAc?$AAt?$AAo?$AAo?$AAl?$AAs?$AA?2?$AAc?$AAr?$AAt?$AA_?$AAb?$AAl?$AAd?$AA?2?$AAs?$AAe?$AAl?$AAf?$AA_?$AAx?$AA8?$AA6?$AA?2?$AAc@ 10198f40     LIBCMTD:initctyp.obj
 0003:0001dfa4       ??_C@_0DC@EHLBFILA@f?3?2dd?2vctools?2crt_bld?2self_x86?2c@ 10198fa4     LIBCMTD:initctyp.obj
 0003:0001dfd8       ??_C@_08JCCMCCIL@HH?3mm?3ss?$AA@ 10198fd8     LIBCMTD:strftime.obj
 0003:0001dfe4       ??_C@_0BE@CKGJFCPC@dddd?0?5MMMM?5dd?0?5yyyy?$AA@ 10198fe4     LIBCMTD:strftime.obj
 0003:0001dff8       ??_C@_08BPBNCDIB@MM?1dd?1yy?$AA@ 10198ff8     LIBCMTD:strftime.obj
 0003:0001e004       ??_C@_02CJNFDJBF@PM?$AA@   10199004     LIBCMTD:strftime.obj
 0003:0001e008       ??_C@_02DEDBPAFC@AM?$AA@   10199008     LIBCMTD:strftime.obj
 0003:0001e00c       ??_C@_08EDHMEBNP@December?$AA@ 1019900c     LIBCMTD:strftime.obj
 0003:0001e018       ??_C@_08HCHEGEOA@November?$AA@ 10199018     LIBCMTD:strftime.obj
 0003:0001e024       ??_C@_07JJNFCEND@October?$AA@ 10199024     LIBCMTD:strftime.obj
 0003:0001e02c       ??_C@_09BHHEALKD@September?$AA@ 1019902c     LIBCMTD:strftime.obj
 0003:0001e038       ??_C@_06LBBHFDDG@August?$AA@ 10199038     LIBCMTD:strftime.obj
 0003:0001e040       ??_C@_04MIEPOIFP@July?$AA@ 10199040     LIBCMTD:strftime.obj
 0003:0001e048       ??_C@_04CNLMGBGM@June?$AA@ 10199048     LIBCMTD:strftime.obj
 0003:0001e050       ??_C@_05DMJDNLEJ@April?$AA@ 10199050     LIBCMTD:strftime.obj
 0003:0001e058       ??_C@_05HPCKOFNC@March?$AA@ 10199058     LIBCMTD:strftime.obj
 0003:0001e060       ??_C@_08GNJGEPFN@February?$AA@ 10199060     LIBCMTD:strftime.obj
 0003:0001e06c       ??_C@_07CGJPFGJA@January?$AA@ 1019906c     LIBCMTD:strftime.obj
 0003:0001e074       ??_C@_03MKABNOCG@Dec?$AA@  10199074     LIBCMTD:strftime.obj
 0003:0001e078       ??_C@_03JPJOFNIA@Nov?$AA@  10199078     LIBCMTD:strftime.obj
 0003:0001e07c       ??_C@_03BMAOKBAD@Oct?$AA@  1019907c     LIBCMTD:strftime.obj
 0003:0001e080       ??_C@_03GGCAPAJC@Sep?$AA@  10199080     LIBCMTD:strftime.obj
 0003:0001e084       ??_C@_03IFJFEIGA@Aug?$AA@  10199084     LIBCMTD:strftime.obj
 0003:0001e088       ??_C@_03LBGABGKK@Jul?$AA@  10199088     LIBCMTD:strftime.obj
 0003:0001e08c       ??_C@_03IDFGHECI@Jun?$AA@  1019908c     LIBCMTD:strftime.obj
 0003:0001e090       ??_C@_03CNMDKL@May?$AA@    10199090     LIBCMTD:strftime.obj
 0003:0001e094       ??_C@_03LEOLGMJP@Apr?$AA@  10199094     LIBCMTD:strftime.obj
 0003:0001e098       ??_C@_03ODNJBKGA@Mar?$AA@  10199098     LIBCMTD:strftime.obj
 0003:0001e09c       ??_C@_03HJBDCHOM@Feb?$AA@  1019909c     LIBCMTD:strftime.obj
 0003:0001e0a0       ??_C@_03JIHJHPIE@Jan?$AA@  101990a0     LIBCMTD:strftime.obj
 0003:0001e0a4       ??_C@_08INBOOONO@Saturday?$AA@ 101990a4     LIBCMTD:strftime.obj
 0003:0001e0b0       ??_C@_06JECMNKMI@Friday?$AA@ 101990b0     LIBCMTD:strftime.obj
 0003:0001e0b8       ??_C@_08HACCIKIA@Thursday?$AA@ 101990b8     LIBCMTD:strftime.obj
 0003:0001e0c4       ??_C@_09DLIGFAKA@Wednesday?$AA@ 101990c4     LIBCMTD:strftime.obj
 0003:0001e0d0       ??_C@_07BAAGCFCM@Tuesday?$AA@ 101990d0     LIBCMTD:strftime.obj
 0003:0001e0d8       ??_C@_06JLEDEDGH@Monday?$AA@ 101990d8     LIBCMTD:strftime.obj
 0003:0001e0e0       ??_C@_06OOPIFAJ@Sunday?$AA@ 101990e0     LIBCMTD:strftime.obj
 0003:0001e0e8       ??_C@_03FEFJNEK@Sat?$AA@   101990e8     LIBCMTD:strftime.obj
 0003:0001e0ec       ??_C@_03IDIOELNC@Fri?$AA@  101990ec     LIBCMTD:strftime.obj
 0003:0001e0f0       ??_C@_03IOFIKPDN@Thu?$AA@  101990f0     LIBCMTD:strftime.obj
 0003:0001e0f4       ??_C@_03MHOMLAJA@Wed?$AA@  101990f4     LIBCMTD:strftime.obj
 0003:0001e0f8       ??_C@_03NAGEINEP@Tue?$AA@  101990f8     LIBCMTD:strftime.obj
 0003:0001e0fc       ??_C@_03PDAGKDH@Mon?$AA@   101990fc     LIBCMTD:strftime.obj
 0003:0001e100       ??_C@_03KOEHGMDN@Sun?$AA@  10199100     LIBCMTD:strftime.obj
 0003:0001e108       ??_C@_1FM@LPEPDBJF@?$AAs?$AAt?$AAr?$AAc?$AAp?$AAy?$AA_?$AAs?$AA?$CI?$AAs?$AA?0?$AA?5?$AA?$CI?$AAl?$AAe?$AAn?$AA?5?$AA?$CL?$AA?5?$AA1?$AA?$CJ?$AA?5?$AA?9?$AA?5?$AA?$CI?$AAs?$AA?5?$AA?9?$AA?5?$AAp?$AA?$CJ?$AA?0@ 10199108     LIBCMTD:strftime.obj
 0003:0001e168       ??_C@_1GG@NAGHPCAA@?$AAs?$AAt?$AAr?$AAc?$AAp?$AAy?$AA_?$AAs?$AA?$CI?$AAs?$AA?0?$AA?5?$AA?$CI?$AAl?$AAe?$AAn?$AA?5?$AA?$CL?$AA?5?$AA1?$AA?$CJ?$AA?5?$AA?9?$AA?5?$AA?$CI?$AAs?$AA?5?$AA?9?$AA?5?$AAp?$AA?$CJ?$AA?0@ 10199168     LIBCMTD:strftime.obj
 0003:0001e1d0       ??_C@_1BG@LGACIFJI@?$AA_?$AAG?$AAe?$AAt?$AAd?$AAa?$AAy?$AAs?$AA_?$AAl?$AA?$AA@ 101991d0     LIBCMTD:strftime.obj
 0003:0001e1e8       ??_C@_1GE@FCOIONJG@?$AAf?$AA?3?$AA?2?$AAd?$AAd?$AA?2?$AAv?$AAc?$AAt?$AAo?$AAo?$AAl?$AAs?$AA?2?$AAc?$AAr?$AAt?$AA_?$AAb?$AAl?$AAd?$AA?2?$AAs?$AAe?$AAl?$AAf?$AA_?$AAx?$AA8?$AA6?$AA?2?$AAc@ 101991e8     LIBCMTD:strftime.obj
 0003:0001e24c       ??_C@_0DC@MEPJBKMO@f?3?2dd?2vctools?2crt_bld?2self_x86?2c@ 1019924c     LIBCMTD:strftime.obj
 0003:0001e280       ??_C@_1FO@IFFKPIEL@?$AAs?$AAt?$AAr?$AAc?$AAp?$AAy?$AA_?$AAs?$AA?$CI?$AAs?$AA?0?$AA?5?$AA?$CI?$AAl?$AAe?$AAn?$AA?5?$AA?$CL?$AA?5?$AA1?$AA?$CJ?$AA?5?$AA?9?$AA?5?$AA?$CI?$AAs?$AA?5?$AA?9?$AA?5?$AAp?$AA?$CJ?$AA?0@ 10199280     LIBCMTD:strftime.obj
 0003:0001e2e0       ??_C@_1GI@LNJDDNLK@?$AAs?$AAt?$AAr?$AAc?$AAp?$AAy?$AA_?$AAs?$AA?$CI?$AAs?$AA?0?$AA?5?$AA?$CI?$AAl?$AAe?$AAn?$AA?5?$AA?$CL?$AA?5?$AA1?$AA?$CJ?$AA?5?$AA?9?$AA?5?$AA?$CI?$AAs?$AA?5?$AA?9?$AA?5?$AAp?$AA?$CJ?$AA?0@ 101992e0     LIBCMTD:strftime.obj
 0003:0001e348       ??_C@_1BK@IDMELNCB@?$AA_?$AAG?$AAe?$AAt?$AAm?$AAo?$AAn?$AAt?$AAh?$AAs?$AA_?$AAl?$AA?$AA@ 10199348     LIBCMTD:strftime.obj
 0003:0001e368       ??_C@_1FG@CJBIADLJ@?$AAs?$AAt?$AAr?$AAc?$AAp?$AAy?$AA_?$AAs?$AA?$CI?$AAs?$AA?0?$AA?5?$AAl?$AAe?$AAn?$AA?5?$AA?9?$AA?5?$AA?$CI?$AAs?$AA?5?$AA?9?$AA?5?$AAp?$AA?$CJ?$AA?0?$AA?5?$AAp?$AAt?$AA?9?$AA?$DO?$AAw@ 10199368     LIBCMTD:strftime.obj
 0003:0001e3c0       ??_C@_1FI@PPIHCJGH@?$AAs?$AAt?$AAr?$AAc?$AAp?$AAy?$AA_?$AAs?$AA?$CI?$AAs?$AA?0?$AA?5?$AAl?$AAe?$AAn?$AA?5?$AA?9?$AA?5?$AA?$CI?$AAs?$AA?5?$AA?9?$AA?5?$AAp?$AA?$CJ?$AA?0?$AA?5?$AAp?$AAt?$AA?9?$AA?$DO?$AAw@ 101993c0     LIBCMTD:strftime.obj
 0003:0001e418       ??_C@_1FI@GDNOPCGD@?$AAs?$AAt?$AAr?$AAc?$AAp?$AAy?$AA_?$AAs?$AA?$CI?$AAs?$AA?0?$AA?5?$AAl?$AAe?$AAn?$AA?5?$AA?9?$AA?5?$AA?$CI?$AAs?$AA?5?$AA?9?$AA?5?$AAp?$AA?$CJ?$AA?0?$AA?5?$AAp?$AAt?$AA?9?$AA?$DO?$AAw@ 10199418     LIBCMTD:strftime.obj
 0003:0001e470       ??_C@_1FA@MEHIJEIL@?$AAs?$AAt?$AAr?$AAc?$AAp?$AAy?$AA_?$AAs?$AA?$CI?$AAs?$AA?0?$AA?5?$AAl?$AAe?$AAn?$AA?5?$AA?9?$AA?5?$AA?$CI?$AAs?$AA?5?$AA?9?$AA?5?$AAp?$AA?$CJ?$AA?0?$AA?5?$AAp?$AAt?$AA?9?$AA?$DO?$AAa@ 10199470     LIBCMTD:strftime.obj
 0003:0001e4c0       ??_C@_1FA@INCJEBF@?$AAs?$AAt?$AAr?$AAc?$AAp?$AAy?$AA_?$AAs?$AA?$CI?$AAs?$AA?0?$AA?5?$AAl?$AAe?$AAn?$AA?5?$AA?9?$AA?5?$AA?$CI?$AAs?$AA?5?$AA?9?$AA?5?$AAp?$AA?$CJ?$AA?0?$AA?5?$AAp?$AAt?$AA?9?$AA?$DO?$AAa@ 101994c0     LIBCMTD:strftime.obj
 0003:0001e510       ??_C@_1FC@BEAPAEGE@?$AAs?$AAt?$AAr?$AAc?$AAp?$AAy?$AA_?$AAs?$AA?$CI?$AAs?$AA?0?$AA?5?$AAl?$AAe?$AAn?$AA?5?$AA?9?$AA?5?$AA?$CI?$AAs?$AA?5?$AA?9?$AA?5?$AAp?$AA?$CJ?$AA?0?$AA?5?$AAp?$AAt?$AA?9?$AA?$DO?$AAm@ 10199510     LIBCMTD:strftime.obj
 0003:0001e568       ??_C@_1FM@CHHONFED@?$AAs?$AAt?$AAr?$AAc?$AAp?$AAy?$AA_?$AAs?$AA?$CI?$AAs?$AA?0?$AA?5?$AAl?$AAe?$AAn?$AA?5?$AA?9?$AA?5?$AA?$CI?$AAs?$AA?5?$AA?9?$AA?5?$AAp?$AA?$CJ?$AA?0?$AA?5?$AAp?$AAt?$AA?9?$AA?$DO?$AAm@ 10199568     LIBCMTD:strftime.obj
 0003:0001e5c8       ??_C@_1FA@EBHJJADL@?$AAs?$AAt?$AAr?$AAc?$AAp?$AAy?$AA_?$AAs?$AA?$CI?$AAs?$AA?0?$AA?5?$AAl?$AAe?$AAn?$AA?5?$AA?9?$AA?5?$AA?$CI?$AAs?$AA?5?$AA?9?$AA?5?$AAp?$AA?$CJ?$AA?0?$AA?5?$AAp?$AAt?$AA?9?$AA?$DO?$AAw@ 101995c8     LIBCMTD:strftime.obj
 0003:0001e618       ??_C@_1FK@ODMKEFLD@?$AAs?$AAt?$AAr?$AAc?$AAp?$AAy?$AA_?$AAs?$AA?$CI?$AAs?$AA?0?$AA?5?$AAl?$AAe?$AAn?$AA?5?$AA?9?$AA?5?$AA?$CI?$AAs?$AA?5?$AA?9?$AA?5?$AAp?$AA?$CJ?$AA?0?$AA?5?$AAp?$AAt?$AA?9?$AA?$DO?$AAw@ 10199618     LIBCMTD:strftime.obj
 0003:0001e674       ??_C@_1BK@MJNHIAGO@?$AA_?$AAG?$AAe?$AAt?$AAt?$AAn?$AAa?$AAm?$AAe?$AAs?$AA_?$AAl?$AA?$AA@ 10199674     LIBCMTD:strftime.obj
 0003:0001e690       ??_C@_1M@HCOOECOK@?$AAF?$AAA?$AAL?$AAS?$AAE?$AA?$AA@ 10199690     LIBCMTD:strftime.obj
 0003:0001e6a0       ??_C@_1HC@JGDOBCNK@?$AA?$CI?$AA?$CC?$AAI?$AAn?$AAv?$AAa?$AAl?$AAi?$AAd?$AA?5?$AAM?$AAB?$AAC?$AAS?$AA?5?$AAc?$AAh?$AAa?$AAr?$AAa?$AAc?$AAt?$AAe?$AAr?$AA?5?$AAs?$AAe?$AAq?$AAu?$AAe?$AAn?$AAc@ 101996a0     LIBCMTD:strftime.obj
 0003:0001e714       ??_C@_1CA@COHOENPC@?$AAt?$AAi?$AAm?$AAe?$AAp?$AAt?$AAr?$AA?5?$AA?$CB?$AA?$DN?$AA?5?$AAN?$AAU?$AAL?$AAL?$AA?$AA@ 10199714     LIBCMTD:strftime.obj
 0003:0001e734       ??_C@_1CG@MHIOFJLE@?$AA?$CI?$AA?5?$AAf?$AAo?$AAr?$AAm?$AAa?$AAt?$AA?5?$AA?$CB?$AA?$DN?$AA?5?$AAN?$AAU?$AAL?$AAL?$AA?5?$AA?$CJ?$AA?$AA@ 10199734     LIBCMTD:strftime.obj
 0003:0001e75c       ??_C@_1CC@IHEJKGMG@?$AA?$CI?$AA?5?$AAm?$AAa?$AAx?$AAs?$AAi?$AAz?$AAe?$AA?5?$AA?$CB?$AA?$DN?$AA?5?$AA0?$AA?5?$AA?$CJ?$AA?$AA@ 1019975c     LIBCMTD:strftime.obj
 0003:0001e780       ??_C@_1BI@ONBMGNNA@?$AA_?$AAS?$AAt?$AAr?$AAf?$AAt?$AAi?$AAm?$AAe?$AA_?$AAl?$AA?$AA@ 10199780     LIBCMTD:strftime.obj
 0003:0001e798       ??_C@_1CG@MPKJHDAA@?$AA?$CI?$AA?5?$AAs?$AAt?$AAr?$AAi?$AAn?$AAg?$AA?5?$AA?$CB?$AA?$DN?$AA?5?$AAN?$AAU?$AAL?$AAL?$AA?5?$AA?$CJ?$AA?$AA@ 10199798     LIBCMTD:strftime.obj
 0003:0001e7c0       ??_C@_1EG@JNJKHKFI@?$AA?$CI?$AA?5?$AA?$CC?$AAI?$AAn?$AAv?$AAa?$AAl?$AAi?$AAd?$AA?5?$AAf?$AAo?$AAr?$AAm?$AAa?$AAt?$AA?5?$AAd?$AAi?$AAr?$AAe?$AAc?$AAt?$AAi?$AAv?$AAe?$AA?$CC?$AA?5?$AA?0?$AA?5?$AA0@ 101997c0     LIBCMTD:strftime.obj
 0003:0001e808       ??_C@_1HM@LBNGKIAD@?$AA?$CI?$AA?5?$AAt?$AAi?$AAm?$AAe?$AAp?$AAt?$AAr?$AA?9?$AA?$DO?$AAt?$AAm?$AA_?$AAy?$AAe?$AAa?$AAr?$AA?5?$AA?$DO?$AA?$DN?$AA?5?$AA?9?$AA1?$AA9?$AA0?$AA0?$AA?5?$AA?$CJ?$AA?5?$AA?$CG?$AA?$CG@ 10199808     LIBCMTD:strftime.obj
 0003:0001e884       ??_C@_1DC@NMCFBMJP@?$AA?$CI?$AA?5?$AAt?$AAi?$AAm?$AAe?$AAp?$AAt?$AAr?$AA?9?$AA?$DO?$AAt?$AAm?$AA_?$AAy?$AAe?$AAa?$AAr?$AA?5?$AA?$DO?$AA?$DN?$AA0?$AA?5?$AA?$CJ?$AA?$AA@ 10199884     LIBCMTD:strftime.obj
 0003:0001e8b8       ??_C@_1HC@HLKHIKOB@?$AA?$CI?$AA?5?$AA?$CI?$AA?5?$AAt?$AAi?$AAm?$AAe?$AAp?$AAt?$AAr?$AA?9?$AA?$DO?$AAt?$AAm?$AA_?$AAs?$AAe?$AAc?$AA?5?$AA?$DO?$AA?$DN?$AA0?$AA?5?$AA?$CJ?$AA?5?$AA?$CG?$AA?$CG?$AA?5?$AA?$CI?$AA?5?$AAt@ 101998b8     LIBCMTD:strftime.obj
 0003:0001e930       ??_C@_1HC@IGKDPPHL@?$AA?$CI?$AA?5?$AA?$CI?$AA?5?$AAt?$AAi?$AAm?$AAe?$AAp?$AAt?$AAr?$AA?9?$AA?$DO?$AAt?$AAm?$AA_?$AAm?$AAi?$AAn?$AA?5?$AA?$DO?$AA?$DN?$AA0?$AA?5?$AA?$CJ?$AA?5?$AA?$CG?$AA?$CG?$AA?5?$AA?$CI?$AA?5?$AAt@ 10199930     LIBCMTD:strftime.obj
 0003:0001e9a8       ??_C@_1HI@HHCJCPE@?$AA?$CI?$AA?5?$AA?$CI?$AA?5?$AAt?$AAi?$AAm?$AAe?$AAp?$AAt?$AAr?$AA?9?$AA?$DO?$AAt?$AAm?$AA_?$AAy?$AAd?$AAa?$AAy?$AA?5?$AA?$DO?$AA?$DN?$AA0?$AA?5?$AA?$CJ?$AA?5?$AA?$CG?$AA?$CG?$AA?5?$AA?$CI?$AA?5@ 101999a8     LIBCMTD:strftime.obj
 0003:0001ea20       ??_C@_1HG@KCGGFLNI@?$AA?$CI?$AA?5?$AA?$CI?$AA?5?$AAt?$AAi?$AAm?$AAe?$AAp?$AAt?$AAr?$AA?9?$AA?$DO?$AAt?$AAm?$AA_?$AAh?$AAo?$AAu?$AAr?$AA?5?$AA?$DO?$AA?$DN?$AA0?$AA?5?$AA?$CJ?$AA?5?$AA?$CG?$AA?$CG?$AA?5?$AA?$CI?$AA?5@ 10199a20     LIBCMTD:strftime.obj
 0003:0001ea98       ??_C@_1HG@NFHHOAD@?$AA?$CI?$AA?5?$AA?$CI?$AA?5?$AAt?$AAi?$AAm?$AAe?$AAp?$AAt?$AAr?$AA?9?$AA?$DO?$AAt?$AAm?$AA_?$AAm?$AAd?$AAa?$AAy?$AA?5?$AA?$DO?$AA?$DN?$AA1?$AA?5?$AA?$CJ?$AA?5?$AA?$CG?$AA?$CG?$AA?5?$AA?$CI?$AA?5@ 10199a98     LIBCMTD:strftime.obj
 0003:0001eb10       ??_C@_1HC@OOAMILFB@?$AA?$CI?$AA?5?$AA?$CI?$AA?5?$AAt?$AAi?$AAm?$AAe?$AAp?$AAt?$AAr?$AA?9?$AA?$DO?$AAt?$AAm?$AA_?$AAm?$AAo?$AAn?$AA?5?$AA?$DO?$AA?$DN?$AA0?$AA?5?$AA?$CJ?$AA?5?$AA?$CG?$AA?$CG?$AA?5?$AA?$CI?$AA?5?$AAt@ 10199b10     LIBCMTD:strftime.obj
 0003:0001eb84       ??_C@_1BI@HBKPAJH@?$AA_?$AAe?$AAx?$AAp?$AAa?$AAn?$AAd?$AAt?$AAi?$AAm?$AAe?$AA?$AA@ 10199b84     LIBCMTD:strftime.obj
 0003:0001eba0       ??_C@_1HE@BFLEOKFO@?$AA?$CI?$AA?5?$AA?$CI?$AA?5?$AAt?$AAi?$AAm?$AAe?$AAp?$AAt?$AAr?$AA?9?$AA?$DO?$AAt?$AAm?$AA_?$AAw?$AAd?$AAa?$AAy?$AA?5?$AA?$DO?$AA?$DN?$AA0?$AA?5?$AA?$CJ?$AA?5?$AA?$CG?$AA?$CG?$AA?5?$AA?$CI?$AA?5@ 10199ba0     LIBCMTD:strftime.obj
 0003:0001ec18       ??_C@_1HG@PAEENAPO@?$AA?$CI?$AA?$CC?$AAI?$AAn?$AAv?$AAa?$AAl?$AAi?$AAd?$AA?5?$AAM?$AAB?$AAC?$AAS?$AA?5?$AAc?$AAh?$AAa?$AAr?$AAa?$AAc?$AAt?$AAe?$AAr?$AA?5?$AAs?$AAe?$AAq?$AAu?$AAe?$AAn?$AAc@ 10199c18     LIBCMTD:strftime.obj
 0003:0001ec90       ??_C@_1IE@EIDABBDG@?$AA?$CI?$AA?$CC?$AAI?$AAn?$AAv?$AAa?$AAl?$AAi?$AAd?$AA?5?$AAM?$AAB?$AAC?$AAS?$AA?5?$AAc?$AAh?$AAa?$AAr?$AAa?$AAc?$AAt?$AAe?$AAr?$AA?5?$AAs?$AAe?$AAq?$AAu?$AAe?$AAn?$AAc@ 10199c90     LIBCMTD:strftime.obj
 0003:0001ed14       ??_C@_03EBAPMIKO@a?1p?$AA@ 10199d14     LIBCMTD:strftime.obj
 0003:0001ed18       ??_C@_05JAMEPDIN@am?1pm?$AA@ 10199d18     LIBCMTD:strftime.obj
 0003:0001ed20       ??_C@_1BE@NDMJHJJG@?$AAs?$AAt?$AAr?$AAn?$AAc?$AAp?$AAy?$AA_?$AAs?$AA?$AA@ 10199d20     LIBCMTD:strncpy_s.obj
 0003:0001ed38       ??_C@_1GK@PAJJBKJF@?$AAf?$AA?3?$AA?2?$AAd?$AAd?$AA?2?$AAv?$AAc?$AAt?$AAo?$AAo?$AAl?$AAs?$AA?2?$AAc?$AAr?$AAt?$AA_?$AAb?$AAl?$AAd?$AA?2?$AAs?$AAe?$AAl?$AAf?$AA_?$AAx?$AA8?$AA6?$AA?2?$AAc@ 10199d38     LIBCMTD:strncpy_s.obj
 0003:0001eda8       ??_C@_1FA@MJKDNFFB@?$AA?$CI?$AAL?$AA?$CC?$AAS?$AAt?$AAr?$AAi?$AAn?$AAg?$AA?5?$AAi?$AAs?$AA?5?$AAn?$AAo?$AAt?$AA?5?$AAn?$AAu?$AAl?$AAl?$AA?5?$AAt?$AAe?$AAr?$AAm?$AAi?$AAn?$AAa?$AAt?$AAe?$AAd@ 10199da8     LIBCMTD:strcat_s.obj
 0003:0001edf8       ??_C@_1DM@FHLMIEG@?$AAS?$AAt?$AAr?$AAi?$AAn?$AAg?$AA?5?$AAi?$AAs?$AA?5?$AAn?$AAo?$AAt?$AA?5?$AAn?$AAu?$AAl?$AAl?$AA?5?$AAt?$AAe?$AAr?$AAm?$AAi?$AAn?$AAa?$AAt?$AAe?$AAd?$AA?$AA@ 10199df8     LIBCMTD:strcat_s.obj
 0003:0001ee34       ??_C@_1BC@HGPNAKGC@?$AAs?$AAt?$AAr?$AAc?$AAa?$AAt?$AA_?$AAs?$AA?$AA@ 10199e34     LIBCMTD:strcat_s.obj
 0003:0001ee48       ??_C@_1GI@NOKGIAGA@?$AAf?$AA?3?$AA?2?$AAd?$AAd?$AA?2?$AAv?$AAc?$AAt?$AAo?$AAo?$AAl?$AAs?$AA?2?$AAc?$AAr?$AAt?$AA_?$AAb?$AAl?$AAd?$AA?2?$AAs?$AAe?$AAl?$AAf?$AA_?$AAx?$AA8?$AA6?$AA?2?$AAc@ 10199e48     LIBCMTD:strcat_s.obj
 0003:0001eeb0       ??_C@_0O@FMJNFNKE@united?9states?$AA@ 10199eb0     LIBCMTD:getqloc.obj
 0003:0001eec0       ??_C@_0P@NDHFFKCA@united?9kingdom?$AA@ 10199ec0     LIBCMTD:getqloc.obj
 0003:0001eed0       ??_C@_0BC@HHDADLGF@trinidad?5?$CG?5tobago?$AA@ 10199ed0     LIBCMTD:getqloc.obj
 0003:0001eee4       ??_C@_0M@IOAEBDAC@south?9korea?$AA@ 10199ee4     LIBCMTD:getqloc.obj
 0003:0001eef0       ??_C@_0N@FIELFKIJ@south?9africa?$AA@ 10199ef0     LIBCMTD:getqloc.obj
 0003:0001ef00       ??_C@_0M@OPNDHCMC@south?5korea?$AA@ 10199f00     LIBCMTD:getqloc.obj
 0003:0001ef0c       ??_C@_0N@MDEOEPFI@south?5africa?$AA@ 10199f0c     LIBCMTD:getqloc.obj
 0003:0001ef1c       ??_C@_06FKAPCJLB@slovak?$AA@ 10199f1c     LIBCMTD:getqloc.obj
 0003:0001ef24       ??_C@_0M@EFJANOAL@puerto?9rico?$AA@ 10199f24     LIBCMTD:getqloc.obj
 0003:0001ef30       ??_C@_08PGOJKDAI@pr?9china?$AA@ 10199f30     LIBCMTD:getqloc.obj
 0003:0001ef3c       ??_C@_08JHDOMCMI@pr?5china?$AA@ 10199f3c     LIBCMTD:getqloc.obj
 0003:0001ef48       ??_C@_02JHCHFBLL@nz?$AA@   10199f48     LIBCMTD:getqloc.obj
 0003:0001ef4c       ??_C@_0M@LINHDHKP@new?9zealand?$AA@ 10199f4c     LIBCMTD:getqloc.obj
 0003:0001ef58       ??_C@_09IIIPPBDB@hong?9kong?$AA@ 10199f58     LIBCMTD:getqloc.obj
 0003:0001ef64       ??_C@_07HJLCKBG@holland?$AA@ 10199f64     LIBCMTD:getqloc.obj
 0003:0001ef6c       ??_C@_0O@LEHGMHAG@great?5britain?$AA@ 10199f6c     LIBCMTD:getqloc.obj
 0003:0001ef7c       ??_C@_07FACOMELA@england?$AA@ 10199f7c     LIBCMTD:getqloc.obj
 0003:0001ef84       ??_C@_05JIHCEICB@czech?$AA@ 10199f84     LIBCMTD:getqloc.obj
 0003:0001ef8c       ??_C@_05BBJOBLGB@china?$AA@ 10199f8c     LIBCMTD:getqloc.obj
 0003:0001ef94       ??_C@_07GPKPHICP@britain?$AA@ 10199f94     LIBCMTD:getqloc.obj
 0003:0001ef9c       ??_C@_07MHIPBHMG@america?$AA@ 10199f9c     LIBCMTD:getqloc.obj
 0003:0001efa4       ??_C@_03KIALPMKC@usa?$AA@  10199fa4     LIBCMTD:getqloc.obj
 0003:0001efa8       ??_C@_02FGJGKGGD@us?$AA@   10199fa8     LIBCMTD:getqloc.obj
 0003:0001efac       ??_C@_02NEINDODK@uk?$AA@   10199fac     LIBCMTD:getqloc.obj
 0003:0001efb0       ??_C@_05JMPCFJFJ@swiss?$AA@ 10199fb0     LIBCMTD:getqloc.obj
 0003:0001efb8       ??_C@_0BA@HLOCPIOD@swedish?9finland?$AA@ 10199fb8     LIBCMTD:getqloc.obj
 0003:0001efc8       ??_C@_0BC@PKCNIABK@spanish?9venezuela?$AA@ 10199fc8     LIBCMTD:getqloc.obj
 0003:0001efdc       ??_C@_0BA@GBHHMIJI@spanish?9uruguay?$AA@ 10199fdc     LIBCMTD:getqloc.obj
 0003:0001efec       ??_C@_0BE@BHDOHPMC@spanish?9puerto?5rico?$AA@ 10199fec     LIBCMTD:getqloc.obj
 0003:0001f000       ??_C@_0N@KMOIDGGN@spanish?9peru?$AA@ 1019a000     LIBCMTD:getqloc.obj
 0003:0001f010       ??_C@_0BB@HMHLPGPH@spanish?9paraguay?$AA@ 1019a010     LIBCMTD:getqloc.obj
 0003:0001f024       ??_C@_0P@MCPKNGFD@spanish?9panama?$AA@ 1019a024     LIBCMTD:getqloc.obj
 0003:0001f034       ??_C@_0BC@IHOHGAIL@spanish?9nicaragua?$AA@ 1019a034     LIBCMTD:getqloc.obj
 0003:0001f048       ??_C@_0P@KLMJDNFJ@spanish?9modern?$AA@ 1019a048     LIBCMTD:getqloc.obj
 0003:0001f058       ??_C@_0BA@BPAPGBCM@spanish?9mexican?$AA@ 1019a058     LIBCMTD:getqloc.obj
 0003:0001f068       ??_C@_0BB@PDECHHHE@spanish?9honduras?$AA@ 1019a068     LIBCMTD:getqloc.obj
 0003:0001f07c       ??_C@_0BC@KLHKFGDB@spanish?9guatemala?$AA@ 1019a07c     LIBCMTD:getqloc.obj
 0003:0001f090       ??_C@_0BE@MFOOKJAI@spanish?9el?5salvador?$AA@ 1019a090     LIBCMTD:getqloc.obj
 0003:0001f0a4       ??_C@_0BA@FCOKFPFC@spanish?9ecuador?$AA@ 1019a0a4     LIBCMTD:getqloc.obj
 0003:0001f0b4       ??_C@_0BL@PLMGIMOO@spanish?9dominican?5republic?$AA@ 1019a0b4     LIBCMTD:getqloc.obj
 0003:0001f0d0       ??_C@_0BD@HLGDNMHB@spanish?9costa?5rica?$AA@ 1019a0d0     LIBCMTD:getqloc.obj
 0003:0001f0e4       ??_C@_0BB@PKCBKCPE@spanish?9colombia?$AA@ 1019a0e4     LIBCMTD:getqloc.obj
 0003:0001f0f8       ??_C@_0O@MCBIJGNE@spanish?9chile?$AA@ 1019a0f8     LIBCMTD:getqloc.obj
 0003:0001f108       ??_C@_0BA@BEFEIGJJ@spanish?9bolivia?$AA@ 1019a108     LIBCMTD:getqloc.obj
 0003:0001f118       ??_C@_0BC@EMECMPD@spanish?9argentina?$AA@ 1019a118     LIBCMTD:getqloc.obj
 0003:0001f12c       ??_C@_0BF@EALFLENP@portuguese?9brazilian?$AA@ 1019a12c     LIBCMTD:getqloc.obj
 0003:0001f144       ??_C@_0BC@HBLEBLNN@norwegian?9nynorsk?$AA@ 1019a144     LIBCMTD:getqloc.obj
 0003:0001f158       ??_C@_0BB@HMACDDCK@norwegian?9bokmal?$AA@ 1019a158     LIBCMTD:getqloc.obj
 0003:0001f16c       ??_C@_09BAFFPPHE@norwegian?$AA@ 1019a16c     LIBCMTD:getqloc.obj
 0003:0001f178       ??_C@_0O@EAJFJDFG@italian?9swiss?$AA@ 1019a178     LIBCMTD:getqloc.obj
 0003:0001f188       ??_C@_0O@CNOMPGD@irish?9english?$AA@ 1019a188     LIBCMTD:getqloc.obj
 0003:0001f198       ??_C@_0N@EDHBGCKG@german?9swiss?$AA@ 1019a198     LIBCMTD:getqloc.obj
 0003:0001f1a8       ??_C@_0BC@JACMHNBP@german?9luxembourg?$AA@ 1019a1a8     LIBCMTD:getqloc.obj
 0003:0001f1bc       ??_C@_0BE@HBGMGFEG@german?9lichtenstein?$AA@ 1019a1bc     LIBCMTD:getqloc.obj
 0003:0001f1d0       ??_C@_0BA@HKKBIBKL@german?9austrian?$AA@ 1019a1d0     LIBCMTD:getqloc.obj
 0003:0001f1e0       ??_C@_0N@GCAEPEBK@french?9swiss?$AA@ 1019a1e0     LIBCMTD:getqloc.obj
 0003:0001f1f0       ??_C@_0BC@DJFJJCK@french?9luxembourg?$AA@ 1019a1f0     LIBCMTD:getqloc.obj
 0003:0001f204       ??_C@_0BA@NNCEDFIC@french?9canadian?$AA@ 1019a204     LIBCMTD:getqloc.obj
 0003:0001f214       ??_C@_0P@CMPOCLM@french?9belgian?$AA@ 1019a214     LIBCMTD:getqloc.obj
 0003:0001f224       ??_C@_0M@GHHDJOK@english?9usa?$AA@ 1019a224     LIBCMTD:getqloc.obj
 0003:0001f230       ??_C@_0L@PLDJKEIL@english?9us?$AA@ 1019a230     LIBCMTD:getqloc.obj
 0003:0001f23c       ??_C@_0L@HJCCDMNC@english?9uk?$AA@ 1019a23c     LIBCMTD:getqloc.obj
 0003:0001f248       ??_C@_0BK@CKLIAGJB@english?9trinidad?5y?5tobago?$AA@ 1019a248     LIBCMTD:getqloc.obj
 0003:0001f264       ??_C@_0BF@JMJMGNNF@english?9south?5africa?$AA@ 1019a264     LIBCMTD:getqloc.obj
 0003:0001f27c       ??_C@_0L@DKIIFDFD@english?9nz?$AA@ 1019a27c     LIBCMTD:getqloc.obj
 0003:0001f288       ??_C@_0BA@ONHGJCLH@english?9jamaica?$AA@ 1019a288     LIBCMTD:getqloc.obj
 0003:0001f298       ??_C@_0M@HJBGHOPO@english?9ire?$AA@ 1019a298     LIBCMTD:getqloc.obj
 0003:0001f2a4       ??_C@_0BC@LFEKMIFB@english?9caribbean?$AA@ 1019a2a4     LIBCMTD:getqloc.obj
 0003:0001f2b8       ??_C@_0M@OLDPFKHI@english?9can?$AA@ 1019a2b8     LIBCMTD:getqloc.obj
 0003:0001f2c4       ??_C@_0P@OMDEHBMP@english?9belize?$AA@ 1019a2c4     LIBCMTD:getqloc.obj
 0003:0001f2d4       ??_C@_0M@KFHFPFED@english?9aus?$AA@ 1019a2d4     LIBCMTD:getqloc.obj
 0003:0001f2e0       ??_C@_0BB@MNMBKDFE@english?9american?$AA@ 1019a2e0     LIBCMTD:getqloc.obj
 0003:0001f2f4       ??_C@_0O@KIDLNNBA@dutch?9belgian?$AA@ 1019a2f4     LIBCMTD:getqloc.obj
 0003:0001f304       ??_C@_0BE@JBKABBMH@chinese?9traditional?$AA@ 1019a304     LIBCMTD:getqloc.obj
 0003:0001f318       ??_C@_0BC@MJJMPKCG@chinese?9singapore?$AA@ 1019a318     LIBCMTD:getqloc.obj
 0003:0001f32c       ??_C@_0BD@FDKADDCP@chinese?9simplified?$AA@ 1019a32c     LIBCMTD:getqloc.obj
 0003:0001f340       ??_C@_0BB@DBEFDDME@chinese?9hongkong?$AA@ 1019a340     LIBCMTD:getqloc.obj
 0003:0001f354       ??_C@_07DHNMFMCI@chinese?$AA@ 1019a354     LIBCMTD:getqloc.obj
 0003:0001f35c       ??_C@_03FNDDCHI@chi?$AA@   1019a35c     LIBCMTD:getqloc.obj
 0003:0001f360       ??_C@_03BMMIADDJ@chh?$AA@  1019a360     LIBCMTD:getqloc.obj
 0003:0001f364       ??_C@_08OAIPJDGI@canadian?$AA@ 1019a364     LIBCMTD:getqloc.obj
 0003:0001f370       ??_C@_07HBPMNPNJ@belgian?$AA@ 1019a370     LIBCMTD:getqloc.obj
 0003:0001f378       ??_C@_0L@OEKOPBEL@australian?$AA@ 1019a378     LIBCMTD:getqloc.obj
 0003:0001f384       ??_C@_0BB@MEIMBEDG@american?9english?$AA@ 1019a384     LIBCMTD:getqloc.obj
 0003:0001f398       ??_C@_0BB@DFMDPDGB@american?5english?$AA@ 1019a398     LIBCMTD:getqloc.obj
 0003:0001f3ac       ??_C@_08IJLOKOLL@american?$AA@ 1019a3ac     LIBCMTD:getqloc.obj
 0003:0001f3b8       ___rg_language             1019a3b8     LIBCMTD:getqloc.obj
 0003:0001f5c0       ___rg_country              1019a5c0     LIBCMTD:getqloc.obj
 0003:0001f678       ___rglangidNotDefault      1019a678     LIBCMTD:getqloc.obj
 0003:0001f68c       ??_C@_0BC@NFIEMBLL@Norwegian?9Nynorsk?$AA@ 1019a68c     LIBCMTD:getqloc.obj
 0003:0001f6a0       ??_C@_1OM@OECHDGCF@?$AAs?$AAt?$AAr?$AAc?$AAp?$AAy?$AA_?$AAs?$AA?$CI?$AAl?$AAp?$AAO?$AAu?$AAt?$AAS?$AAt?$AAr?$AA?9?$AA?$DO?$AAs?$AAz?$AAL?$AAa?$AAn?$AAg?$AAu?$AAa?$AAg?$AAe?$AA?0?$AA?5?$AA?$CI@ 1019a6a0     LIBCMTD:getqloc.obj
 0003:0001f78c       ??_C@_1CO@NJACLALJ@?$AA_?$AA_?$AAg?$AAe?$AAt?$AA_?$AAq?$AAu?$AAa?$AAl?$AAi?$AAf?$AAi?$AAe?$AAd?$AA_?$AAl?$AAo?$AAc?$AAa?$AAl?$AAe?$AA?$AA@ 1019a78c     LIBCMTD:getqloc.obj
 0003:0001f7c0       ??_C@_1GC@FECJGAE@?$AAf?$AA?3?$AA?2?$AAd?$AAd?$AA?2?$AAv?$AAc?$AAt?$AAo?$AAo?$AAl?$AAs?$AA?2?$AAc?$AAr?$AAt?$AA_?$AAb?$AAl?$AAd?$AA?2?$AAs?$AAe?$AAl?$AAf?$AA_?$AAx?$AA8?$AA6?$AA?2?$AAc@ 1019a7c0     LIBCMTD:getqloc.obj
 0003:0001f824       ??_C@_03NFKLAGEF@OCP?$AA@  1019a824     LIBCMTD:getqloc.obj
 0003:0001f828       ??_C@_01GBGANLPD@0?$AA@    1019a828     LIBCMTD:getqloc.obj
 0003:0001f82c       ??_C@_03DFHEHBHG@ACP?$AA@  1019a82c     LIBCMTD:getqloc.obj
 0003:0001f830       ??_C@_1BK@CDOALEA@?$AA_?$AAc?$AAo?$AAn?$AAt?$AAr?$AAo?$AAl?$AAf?$AAp?$AA_?$AAs?$AA?$AA@ 1019a830     LIBCMTD:_contrlfp_.obj
 0003:0001f850       ??_C@_1HI@JIOCECAH@?$AAf?$AA?3?$AA?2?$AAd?$AAd?$AA?2?$AAv?$AAc?$AAt?$AAo?$AAo?$AAl?$AAs?$AA?2?$AAc?$AAr?$AAt?$AA_?$AAb?$AAl?$AAd?$AA?2?$AAs?$AAe?$AAl?$AAf?$AA_?$AAx?$AA8?$AA6?$AA?2?$AAc@ 1019a850     LIBCMTD:_contrlfp_.obj
 0003:0001f8c8       ??_C@_1DG@JNDMIEJL@?$AA?$CI?$AA?$CC?$AAI?$AAn?$AAv?$AAa?$AAl?$AAi?$AAd?$AA?5?$AAi?$AAn?$AAp?$AAu?$AAt?$AA?5?$AAv?$AAa?$AAl?$AAu?$AAe?$AA?$CC?$AA?0?$AA?5?$AA0?$AA?$CJ?$AA?$AA@ 1019a8c8     LIBCMTD:_contrlfp_.obj
 0003:0001f900       ??_C@_1BK@CLIEHFDF@?$AAp?$AAf?$AAl?$AAt?$AA?5?$AA?$CB?$AA?$DN?$AA?5?$AAN?$AAU?$AAL?$AAL?$AA?$AA@ 1019a900     LIBCMTD:_fptostr.obj
 0003:0001f920       ??_C@_1GM@CEDLGDDI@?$AAs?$AAi?$AAz?$AAe?$AAI?$AAn?$AAB?$AAy?$AAt?$AAe?$AAs?$AA?5?$AA?$DO?$AA?5?$AA?$CI?$AAs?$AAi?$AAz?$AAe?$AA_?$AAt?$AA?$CJ?$AA?$CI?$AA?$CI?$AAd?$AAi?$AAg?$AAi?$AAt?$AAs?$AA?5?$AA?$DO@ 1019a920     LIBCMTD:_fptostr.obj
 0003:0001f98c       ??_C@_1BC@OPALLEB@?$AA_?$AAf?$AAp?$AAt?$AAo?$AAs?$AAt?$AAr?$AA?$AA@ 1019a98c     LIBCMTD:_fptostr.obj
 0003:0001f9a0       ??_C@_1GE@BDKOPHIO@?$AAf?$AA?3?$AA?2?$AAd?$AAd?$AA?2?$AAv?$AAc?$AAt?$AAo?$AAo?$AAl?$AAs?$AA?2?$AAc?$AAr?$AAt?$AA_?$AAb?$AAl?$AAd?$AA?2?$AAs?$AAe?$AAl?$AAf?$AA_?$AAx?$AA8?$AA6?$AA?2?$AAc@ 1019a9a0     LIBCMTD:_fptostr.obj
 0003:0001fa08       ??_C@_1FK@KODCOBKF@?$AAs?$AAt?$AAr?$AAc?$AAp?$AAy?$AA_?$AAs?$AA?$CI?$AAr?$AAe?$AAs?$AAu?$AAl?$AAt?$AAs?$AAt?$AAr?$AA?0?$AA?5?$AAr?$AAe?$AAs?$AAu?$AAl?$AAt?$AAs?$AAi?$AAz?$AAe?$AA?0?$AA?5@ 1019aa08     LIBCMTD:_cfout_.obj
 0003:0001fa64       ??_C@_1BC@BPMMEHLK@?$AA_?$AAf?$AAl?$AAt?$AAo?$AAu?$AAt?$AA2?$AA?$AA@ 1019aa64     LIBCMTD:_cfout_.obj
 0003:0001fa78       ??_C@_1HC@PKFDNKN@?$AAf?$AA?3?$AA?2?$AAd?$AAd?$AA?2?$AAv?$AAc?$AAt?$AAo?$AAo?$AAl?$AAs?$AA?2?$AAc?$AAr?$AAt?$AA_?$AAb?$AAl?$AAd?$AA?2?$AAs?$AAe?$AAl?$AAf?$AA_?$AAx?$AA8?$AA6?$AA?2?$AAc@ 1019aa78     LIBCMTD:_cfout_.obj
 0003:0001faec       ??_C@_1CG@EBJECAJM@?$AA_?$AAs?$AAe?$AAt?$AA_?$AAo?$AAu?$AAt?$AAp?$AAu?$AAt?$AA_?$AAf?$AAo?$AAr?$AAm?$AAa?$AAt?$AA?$AA@ 1019aaec     LIBCMTD:outputformat.obj
 0003:0001fb18       ??_C@_1GM@NFGGJJCM@?$AAf?$AA?3?$AA?2?$AAd?$AAd?$AA?2?$AAv?$AAc?$AAt?$AAo?$AAo?$AAl?$AAs?$AA?2?$AAc?$AAr?$AAt?$AA_?$AAb?$AAl?$AAd?$AA?2?$AAs?$AAe?$AAl?$AAf?$AA_?$AAx?$AA8?$AA6?$AA?2?$AAc@ 1019ab18     LIBCMTD:outputformat.obj
 0003:0001fb88       ??_C@_1EM@EGEEBJLG@?$AA?$CI?$AAo?$AAp?$AAt?$AAi?$AAo?$AAn?$AAs?$AA?5?$AA?$CG?$AA?5?$AA?$HO?$AA_?$AAT?$AAW?$AAO?$AA_?$AAD?$AAI?$AAG?$AAI?$AAT?$AA_?$AAE?$AAX?$AAP?$AAO?$AAN?$AAE?$AAN?$AAT?$AA?$CJ@ 1019ab88     LIBCMTD:outputformat.obj
 0003:0001fbd4       ??_C@_1CG@JEHFHLNG@?$AA_?$AAm?$AAb?$AAs?$AAt?$AAo?$AAw?$AAc?$AAs?$AA_?$AAl?$AA_?$AAh?$AAe?$AAl?$AAp?$AAe?$AAr?$AA?$AA@ 1019abd4     LIBCMTD:mbstowcs.obj
 0003:0001fc00       ??_C@_1GE@LCCDHBMH@?$AAf?$AA?3?$AA?2?$AAd?$AAd?$AA?2?$AAv?$AAc?$AAt?$AAo?$AAo?$AAl?$AAs?$AA?2?$AAc?$AAr?$AAt?$AA_?$AAb?$AAl?$AAd?$AA?2?$AAs?$AAe?$AAl?$AAf?$AA_?$AAx?$AA8?$AA6?$AA?2?$AAc@ 1019ac00     LIBCMTD:mbstowcs.obj
 0003:0001fc64       ??_C@_1BE@EEKACIGI@?$AAs?$AA?5?$AA?$CB?$AA?$DN?$AA?5?$AAN?$AAU?$AAL?$AAL?$AA?$AA@ 1019ac64     LIBCMTD:mbstowcs.obj
 0003:0001fc78       ??_C@_1CO@JNPEPJAL@?$AAr?$AAe?$AAt?$AAs?$AAi?$AAz?$AAe?$AA?5?$AA?$DM?$AA?$DN?$AA?5?$AAs?$AAi?$AAz?$AAe?$AAI?$AAn?$AAW?$AAo?$AAr?$AAd?$AAs?$AA?$AA@ 1019ac78     LIBCMTD:mbstowcs.obj
 0003:0001fca8       ??_C@_1CM@LLECFMFH@?$AAb?$AAu?$AAf?$AAf?$AAe?$AAr?$AAS?$AAi?$AAz?$AAe?$AA?5?$AA?$DM?$AA?$DN?$AA?5?$AAI?$AAN?$AAT?$AA_?$AAM?$AAA?$AAX?$AA?$AA@ 1019aca8     LIBCMTD:mbstowcs.obj
 0003:0001fcd4       ??_C@_1BM@PHENIGHD@?$AA_?$AAm?$AAb?$AAs?$AAt?$AAo?$AAw?$AAc?$AAs?$AA_?$AAs?$AA_?$AAl?$AA?$AA@ 1019acd4     LIBCMTD:mbstowcs.obj
 0003:0001fcf0       ??_C@_1JA@JKDFMOPO@?$AA?$CI?$AAp?$AAw?$AAc?$AAs?$AA?5?$AA?$DN?$AA?$DN?$AA?5?$AAN?$AAU?$AAL?$AAL?$AA?5?$AA?$CG?$AA?$CG?$AA?5?$AAs?$AAi?$AAz?$AAe?$AAI?$AAn?$AAW?$AAo?$AAr?$AAd?$AAs?$AA?5?$AA?$DN?$AA?$DN?$AA?5@ 1019acf0     LIBCMTD:mbstowcs.obj
 0003:0001fd80       ??_C@_1CM@HABGDNLJ@?$AAl?$AAe?$AAn?$AAg?$AAt?$AAh?$AA?5?$AA?$DM?$AA?5?$AAs?$AAi?$AAz?$AAe?$AAI?$AAn?$AAT?$AAC?$AAh?$AAa?$AAr?$AAs?$AA?$AA@ 1019ad80     LIBCMTD:xtoas.obj
 0003:0001fdac       ??_C@_1DE@PCJGDBBD@?$AA2?$AA?5?$AA?$DM?$AA?$DN?$AA?5?$AAr?$AAa?$AAd?$AAi?$AAx?$AA?5?$AA?$CG?$AA?$CG?$AA?5?$AAr?$AAa?$AAd?$AAi?$AAx?$AA?5?$AA?$DM?$AA?$DN?$AA?5?$AA3?$AA6?$AA?$AA@ 1019adac     LIBCMTD:xtoas.obj
 0003:0001fde0       ??_C@_1FA@MKGGAGEI@?$AAs?$AAi?$AAz?$AAe?$AAI?$AAn?$AAT?$AAC?$AAh?$AAa?$AAr?$AAs?$AA?5?$AA?$DO?$AA?5?$AA?$CI?$AAs?$AAi?$AAz?$AAe?$AA_?$AAt?$AA?$CJ?$AA?$CI?$AAi?$AAs?$AA_?$AAn?$AAe?$AAg?$AA?5?$AA?$DP@ 1019ade0     LIBCMTD:xtoas.obj
 0003:0001fe30       ??_C@_1CC@JNJFIMGE@?$AAs?$AAi?$AAz?$AAe?$AAI?$AAn?$AAT?$AAC?$AAh?$AAa?$AAr?$AAs?$AA?5?$AA?$DO?$AA?5?$AA0?$AA?$AA@ 1019ae30     LIBCMTD:xtoas.obj
 0003:0001fe54       ??_C@_1O@GIMBNLEI@?$AAx?$AAt?$AAo?$AAa?$AA_?$AAs?$AA?$AA@ 1019ae54     LIBCMTD:xtoas.obj
 0003:0001fe68       ??_C@_1FM@MFCBFCGB@?$AAf?$AA?3?$AA?2?$AAd?$AAd?$AA?2?$AAv?$AAc?$AAt?$AAo?$AAo?$AAl?$AAs?$AA?2?$AAc?$AAr?$AAt?$AA_?$AAb?$AAl?$AAd?$AA?2?$AAs?$AAe?$AAl?$AAf?$AA_?$AAx?$AA8?$AA6?$AA?2?$AAc@ 1019ae68     LIBCMTD:xtoas.obj
 0003:0001fec4       ??_C@_1BC@MJJNBNFN@?$AAx?$AA6?$AA4?$AAt?$AAo?$AAa?$AA_?$AAs?$AA?$AA@ 1019aec4     LIBCMTD:xtoas.obj
 0003:0001fed8       ??_C@_1CG@LLJCAOHF@?$AA_?$AAw?$AAc?$AAs?$AAt?$AAo?$AAm?$AAb?$AAs?$AA_?$AAl?$AA_?$AAh?$AAe?$AAl?$AAp?$AAe?$AAr?$AA?$AA@ 1019aed8     LIBCMTD:wcstombs.obj
 0003:0001ff00       ??_C@_1GE@OAENIBOD@?$AAf?$AA?3?$AA?2?$AAd?$AAd?$AA?2?$AAv?$AAc?$AAt?$AAo?$AAo?$AAl?$AAs?$AA?2?$AAc?$AAr?$AAt?$AA_?$AAb?$AAl?$AAd?$AA?2?$AAs?$AAe?$AAl?$AAf?$AA_?$AAx?$AA8?$AA6?$AA?2?$AAc@ 1019af00     LIBCMTD:wcstombs.obj
 0003:0001ff64       ??_C@_1BK@OIBENBPM@?$AAp?$AAw?$AAc?$AAs?$AA?5?$AA?$CB?$AA?$DN?$AA?5?$AAN?$AAU?$AAL?$AAL?$AA?$AA@ 1019af64     LIBCMTD:wcstombs.obj
 0003:0001ff80       ??_C@_1CM@KEOGBFLI@?$AAs?$AAi?$AAz?$AAe?$AAI?$AAn?$AAB?$AAy?$AAt?$AAe?$AAs?$AA?5?$AA?$DO?$AA?5?$AAr?$AAe?$AAt?$AAs?$AAi?$AAz?$AAe?$AA?$AA@ 1019af80     LIBCMTD:wcstombs.obj
 0003:0001ffac       ??_C@_1BM@BDMCLLDL@?$AA_?$AAw?$AAc?$AAs?$AAt?$AAo?$AAm?$AAb?$AAs?$AA_?$AAs?$AA_?$AAl?$AA?$AA@ 1019afac     LIBCMTD:wcstombs.obj
 0003:0001ffc8       ??_C@_1IM@MFGKHGBP@?$AA?$CI?$AAd?$AAs?$AAt?$AA?5?$AA?$CB?$AA?$DN?$AA?5?$AAN?$AAU?$AAL?$AAL?$AA?5?$AA?$CG?$AA?$CG?$AA?5?$AAs?$AAi?$AAz?$AAe?$AAI?$AAn?$AAB?$AAy?$AAt?$AAe?$AAs?$AA?5?$AA?$DO?$AA?5?$AA0?$AA?$CJ@ 1019afc8     LIBCMTD:wcstombs.obj
 0003:00020054       ??_C@_1BC@PLIEPKPJ@?$AAw?$AAc?$AAs?$AAc?$AAa?$AAt?$AA_?$AAs?$AA?$AA@ 1019b054     LIBCMTD:wcscat_s.obj
 0003:00020068       ??_C@_1CE@IGKFIJFD@?$AA_?$AAv?$AAs?$AAw?$AAp?$AAr?$AAi?$AAn?$AAt?$AAf?$AA_?$AAh?$AAe?$AAl?$AAp?$AAe?$AAr?$AA?$AA@ 1019b068     LIBCMTD:vswprnc.obj
 0003:00020090       ??_C@_1GE@KINELFI@?$AAf?$AA?3?$AA?2?$AAd?$AAd?$AA?2?$AAv?$AAc?$AAt?$AAo?$AAo?$AAl?$AAs?$AA?2?$AAc?$AAr?$AAt?$AA_?$AAb?$AAl?$AAd?$AA?2?$AAs?$AAe?$AAl?$AAf?$AA_?$AAx?$AA8?$AA6?$AA?2?$AAc@ 1019b090     LIBCMTD:vswprnc.obj
 0003:000200f8       ??_C@_1EE@MPCHJFGP@?$AAs?$AAt?$AAr?$AAi?$AAn?$AAg?$AA?5?$AA?$CB?$AA?$DN?$AA?5?$AAN?$AAU?$AAL?$AAL?$AA?5?$AA?$CG?$AA?$CG?$AA?5?$AAs?$AAi?$AAz?$AAe?$AAI?$AAn?$AAW?$AAo?$AAr?$AAd?$AAs?$AA?5?$AA?$DO?$AA?5@ 1019b0f8     LIBCMTD:vswprnc.obj
 0003:0002013c       ??_C@_1BO@OALHJLCI@?$AA_?$AAv?$AAs?$AAw?$AAp?$AAr?$AAi?$AAn?$AAt?$AAf?$AA_?$AAs?$AA_?$AAl?$AA?$AA@ 1019b13c     LIBCMTD:vswprnc.obj
 0003:0002015c       ??_C@_1CA@BKFKMJFF@?$AA_?$AAv?$AAs?$AAn?$AAw?$AAp?$AAr?$AAi?$AAn?$AAt?$AAf?$AA_?$AAs?$AA_?$AAl?$AA?$AA@ 1019b15c     LIBCMTD:vswprnc.obj
 0003:0002017c       ??_C@_1O@NCBFODOE@?$AAx?$AAt?$AAo?$AAw?$AA_?$AAs?$AA?$AA@ 1019b17c     LIBCMTD:xtows.obj
 0003:0002018c       ??_C@_1BC@HDEJCFPB@?$AAx?$AA6?$AA4?$AAt?$AAo?$AAw?$AA_?$AAs?$AA?$AA@ 1019b18c     LIBCMTD:xtows.obj
 0003:000201a0       ??_C@_1BG@BBCDFOMA@?$AA_?$AAw?$AAo?$AAu?$AAt?$AAp?$AAu?$AAt?$AA_?$AAl?$AA?$AA@ 1019b1a0     LIBCMTD:woutput.obj
 0003:000201b8       ??_C@_1BK@EPLNBKAK@?$AA_?$AAv?$AAs?$AAw?$AAp?$AAr?$AAi?$AAn?$AAt?$AAf?$AA_?$AAl?$AA?$AA@ 1019b1b8     LIBCMTD:vswprint.obj
 0003:000201d4       ??_C@_1CG@IMMIEPNA@?$AA_?$AAv?$AAs?$AAc?$AAw?$AAp?$AAr?$AAi?$AAn?$AAt?$AAf?$AA_?$AAh?$AAe?$AAl?$AAp?$AAe?$AAr?$AA?$AA@ 1019b1d4     LIBCMTD:vswprint.obj
 0003:000201fc       ??_C@_0BK@CFCOFLF@?5Complete?5Object?5Locator?8?$AA@ 1019b1fc     LIBCMTD:undname.obj
 0003:00020218       ??_C@_0BN@MECKDCOJ@?5Class?5Hierarchy?5Descriptor?8?$AA@ 1019b218     LIBCMTD:undname.obj
 0003:00020238       ??_C@_0BD@LGICGFMM@?5Base?5Class?5Array?8?$AA@ 1019b238     LIBCMTD:undname.obj
 0003:0002024c       ??_C@_0BM@LDKODKLH@?5Base?5Class?5Descriptor?5at?5?$CI?$AA@ 1019b24c     LIBCMTD:undname.obj
 0003:00020268       ??_C@_0BC@DAFEJGAK@?5Type?5Descriptor?8?$AA@ 1019b268     LIBCMTD:undname.obj
 0003:0002027c       ??_C@_0BM@PMGGMLDN@?$GAlocal?5static?5thread?5guard?8?$AA@ 1019b27c     LIBCMTD:undname.obj
 0003:00020298       ??_C@_0CL@FGIJHLCE@?$GAmanaged?5vector?5copy?5constructor@ 1019b298     LIBCMTD:undname.obj
 0003:000202c4       ??_C@_0CJ@GJELGAMM@?$GAvector?5vbase?5copy?5constructor?5i@ 1019b2c4     LIBCMTD:undname.obj
 0003:000202f0       ??_C@_0CD@CGAJBKEJ@?$GAvector?5copy?5constructor?5iterato@ 1019b2f0     LIBCMTD:undname.obj
 0003:00020314       ??_C@_0CB@PDBIFEP@?$GAdynamic?5atexit?5destructor?5for?5?8@ 1019b314     LIBCMTD:undname.obj
 0003:00020338       ??_C@_0BL@CLIPGLGB@?$GAdynamic?5initializer?5for?5?8?$AA@ 1019b338     LIBCMTD:undname.obj
 0003:00020354       ??_C@_0CM@FCBBDIGB@?$GAeh?5vector?5vbase?5copy?5constructo@ 1019b354     LIBCMTD:undname.obj
 0003:00020380       ??_C@_0CG@HLDDJMAG@?$GAeh?5vector?5copy?5constructor?5iter@ 1019b380     LIBCMTD:undname.obj
 0003:000203a8       ??_C@_0CF@IMGKMJNO@?$GAmanaged?5vector?5destructor?5itera@ 1019b3a8     LIBCMTD:undname.obj
 0003:000203d0       ??_C@_0CG@CFDHKGGD@?$GAmanaged?5vector?5constructor?5iter@ 1019b3d0     LIBCMTD:undname.obj
 0003:000203f8       ??_C@_0BN@CKNJLHMB@?$GAplacement?5delete?$FL?$FN?5closure?8?$AA@ 1019b3f8     LIBCMTD:undname.obj
 0003:00020418       ??_C@_0BL@CNOONJFP@?$GAplacement?5delete?5closure?8?$AA@ 1019b418     LIBCMTD:undname.obj
 0003:00020434       ??_C@_0P@HJKNJFNN@?$GAomni?5callsig?8?$AA@ 1019b434     LIBCMTD:undname.obj
 0003:00020444       ??_C@_09LBNFPBCA@?5delete?$FL?$FN?$AA@ 1019b444     LIBCMTD:undname.obj
 0003:00020450       ??_C@_06FHBGPFGH@?5new?$FL?$FN?$AA@ 1019b450     LIBCMTD:undname.obj
 0003:00020458       ??_C@_0CE@IIHCMGGL@?$GAlocal?5vftable?5constructor?5closu@ 1019b458     LIBCMTD:undname.obj
 0003:0002047c       ??_C@_0BA@KKLDJDLB@?$GAlocal?5vftable?8?$AA@ 1019b47c     LIBCMTD:undname.obj
 0003:0002048c       ??_C@_05KHLCHHI@?$GARTTI?$AA@ 1019b48c     LIBCMTD:undname.obj
 0003:00020494       ??_C@_03KLGMFNMG@?$GAEH?$AA@ 1019b494     LIBCMTD:undname.obj
 0003:00020498       ??_C@_0BA@KBCDOMBN@?$GAudt?5returning?8?$AA@ 1019b498     LIBCMTD:undname.obj
 0003:000204a8       ??_C@_0BL@LLKPOHJI@?$GAcopy?5constructor?5closure?8?$AA@ 1019b4a8     LIBCMTD:undname.obj
 0003:000204c4       ??_C@_0CH@OOJPLCPH@?$GAeh?5vector?5vbase?5constructor?5ite@ 1019b4c4     LIBCMTD:undname.obj
 0003:000204ec       ??_C@_0CA@GCEOPDGL@?$GAeh?5vector?5destructor?5iterator?8?$AA@ 1019b4ec     LIBCMTD:undname.obj
 0003:0002050c       ??_C@_0CB@JONCMFFK@?$GAeh?5vector?5constructor?5iterator?8@ 1019b50c     LIBCMTD:undname.obj
 0003:00020530       ??_C@_0BL@NILFHHPC@?$GAvirtual?5displacement?5map?8?$AA@ 1019b530     LIBCMTD:undname.obj
 0003:0002054c       ??_C@_0CE@IKBNEHA@?$GAvector?5vbase?5constructor?5iterat@ 1019b54c     LIBCMTD:undname.obj
 0003:00020570       ??_C@_0BN@LFPFMEDL@?$GAvector?5destructor?5iterator?8?$AA@ 1019b570     LIBCMTD:undname.obj
 0003:00020590       ??_C@_0BO@PFGOCPJJ@?$GAvector?5constructor?5iterator?8?$AA@ 1019b590     LIBCMTD:undname.obj
 0003:000205b0       ??_C@_0BN@IMDCHIKM@?$GAscalar?5deleting?5destructor?8?$AA@ 1019b5b0     LIBCMTD:undname.obj
 0003:000205d0       ??_C@_0BO@OBMKPJIG@?$GAdefault?5constructor?5closure?8?$AA@ 1019b5d0     LIBCMTD:undname.obj
 0003:000205f0       ??_C@_0BN@DEGPLNFK@?$GAvector?5deleting?5destructor?8?$AA@ 1019b5f0     LIBCMTD:undname.obj
 0003:00020610       ??_C@_0BD@JDLKDPAB@?$GAvbase?5destructor?8?$AA@ 1019b610     LIBCMTD:undname.obj
 0003:00020624       ??_C@_08OBABFOLI@?$GAstring?8?$AA@ 1019b624     LIBCMTD:undname.obj
 0003:00020630       ??_C@_0BF@KDPPACIK@?$GAlocal?5static?5guard?8?$AA@ 1019b630     LIBCMTD:undname.obj
 0003:00020648       ??_C@_08LLFFHHDJ@?$GAtypeof?8?$AA@ 1019b648     LIBCMTD:undname.obj
 0003:00020654       ??_C@_07FEEIOKP@?$GAvcall?8?$AA@ 1019b654     LIBCMTD:undname.obj
 0003:0002065c       ??_C@_09BLBHBJP@?$GAvbtable?8?$AA@ 1019b65c     LIBCMTD:undname.obj
 0003:00020668       ??_C@_09IFPLHPGF@?$GAvftable?8?$AA@ 1019b668     LIBCMTD:undname.obj
 0003:00020674       ??_C@_02MHEGNOJ@?$FO?$DN?$AA@ 1019b674     LIBCMTD:undname.obj
 0003:00020678       ??_C@_02DHLNPPGH@?$HM?$DN?$AA@ 1019b678     LIBCMTD:undname.obj
 0003:0002067c       ??_C@_02FGJGFEAB@?$CG?$DN?$AA@ 1019b67c     LIBCMTD:undname.obj
 0003:00020680       ??_C@_03CDNPDDLA@?$DM?$DM?$DN?$AA@ 1019b680     LIBCMTD:undname.obj
 0003:00020684       ??_C@_03IKFCCPFF@?$DO?$DO?$DN?$AA@ 1019b684     LIBCMTD:undname.obj
 0003:00020688       ??_C@_02FENAOKFI@?$CF?$DN?$AA@ 1019b688     LIBCMTD:undname.obj
 0003:0002068c       ??_C@_02FJEHGPIO@?1?$DN?$AA@ 1019b68c     LIBCMTD:undname.obj
 0003:00020690       ??_C@_02FKMDLLOA@?9?$DN?$AA@ 1019b690     LIBCMTD:undname.obj
 0003:00020694       ??_C@_02FOEOMHFC@?$CL?$DN?$AA@ 1019b694     LIBCMTD:undname.obj
 0003:00020698       ??_C@_02FPIMKNGF@?$CK?$DN?$AA@ 1019b698     LIBCMTD:undname.obj
 0003:0002069c       ??_C@_02NONPIBCD@?$HM?$HM?$AA@ 1019b69c     LIBCMTD:undname.obj
 0003:000206a0       ??_C@_02PPKAJPJL@?$CG?$CG?$AA@ 1019b6a0     LIBCMTD:undname.obj
 0003:000206a4       ??_C@_01DNKMNLPK@?$HM?$AA@ 1019b6a4     LIBCMTD:undname.obj
 0003:000206a8       ??_C@_01JKBOJNNK@?$FO?$AA@ 1019b6a8     LIBCMTD:undname.obj
 0003:000206ac       ??_C@_01PJKLJHI@?$HO?$AA@  1019b6ac     LIBCMTD:undname.obj
 0003:000206b0       ??_C@_02HCKGKOFO@?$CI?$CJ?$AA@ 1019b6b0     LIBCMTD:undname.obj
 0003:000206b4       ??_C@_01IHBHIGKO@?0?$AA@   1019b6b4     LIBCMTD:undname.obj
 0003:000206b8       ??_C@_02EEKDKGMJ@?$DO?$DN?$AA@ 1019b6b8     LIBCMTD:undname.obj
 0003:000206bc       ??_C@_01PPODPGHN@?$DO?$AA@ 1019b6bc     LIBCMTD:undname.obj
 0003:000206c0       ??_C@_02EHCHHCKH@?$DM?$DN?$AA@ 1019b6c0     LIBCMTD:undname.obj
 0003:000206c4       ??_C@_01MNNFJEPP@?$DM?$AA@ 1019b6c4     LIBCMTD:undname.obj
 0003:000206c8       ??_C@_01FGNFDNOH@?$CF?$AA@ 1019b6c8     LIBCMTD:undname.obj
 0003:000206cc       ??_C@_01KMDKNFGN@?1?$AA@   1019b6cc     LIBCMTD:undname.obj
 0003:000206d0       ??_C@_03MNHNFDLC@?9?$DO?$CK?$AA@ 1019b6d0     LIBCMTD:undname.obj
 0003:000206d4       ??_C@_01HNPIGOCE@?$CG?$AA@ 1019b6d4     LIBCMTD:undname.obj
 0003:000206d8       ??_C@_01MIFGBAGJ@?$CL?$AA@ 1019b6d8     LIBCMTD:undname.obj
 0003:000206dc       ??_C@_01JOAMLHOP@?9?$AA@   1019b6dc     LIBCMTD:undname.obj
 0003:000206e0       ??_C@_02BAABKJLB@?9?9?$AA@ 1019b6e0     LIBCMTD:undname.obj
 0003:000206e4       ??_C@_02ECNGHCIF@?$CL?$CL?$AA@ 1019b6e4     LIBCMTD:undname.obj
 0003:000206e8       ??_C@_01NBENCBCI@?$CK?$AA@ 1019b6e8     LIBCMTD:undname.obj
 0003:000206ec       ??_C@_02HBOOOICD@?9?$DO?$AA@ 1019b6ec     LIBCMTD:undname.obj
 0003:000206f0       ??_C@_08LHJFAFGD@operator?$AA@ 1019b6f0     LIBCMTD:undname.obj
 0003:000206fc       ??_C@_02GPECMEKF@?$FL?$FN?$AA@ 1019b6fc     LIBCMTD:undname.obj
 0003:00020700       ??_C@_02FDNJECIE@?$CB?$DN?$AA@ 1019b700     LIBCMTD:undname.obj
 0003:00020704       ??_C@_02EGOFBIJA@?$DN?$DN?$AA@ 1019b704     LIBCMTD:undname.obj
 0003:00020708       ??_C@_01DCLJPIOD@?$CB?$AA@ 1019b708     LIBCMTD:undname.obj
 0003:0002070c       ??_C@_02FODMEDOG@?$DM?$DM?$AA@ 1019b70c     LIBCMTD:undname.obj
 0003:00020710       ??_C@_02GPIOPFAK@?$DO?$DO?$AA@ 1019b710     LIBCMTD:undname.obj
 0003:00020714       ??_C@_07FPCDHGMM@?5delete?$AA@ 1019b714     LIBCMTD:undname.obj
 0003:0002071c       ??_C@_04NIHEBCM@?5new?$AA@ 1019b71c     LIBCMTD:undname.obj
 0003:00020724       ??_C@_0M@GFIIJFMG@__unaligned?$AA@ 1019b724     LIBCMTD:undname.obj
 0003:00020730       ??_C@_0L@PILCLIHE@__restrict?$AA@ 1019b730     LIBCMTD:undname.obj
 0003:0002073c       ??_C@_07JOMMBBKO@__ptr64?$AA@ 1019b73c     LIBCMTD:undname.obj
 0003:00020744       ??_C@_09HIJEGCPM@__clrcall?$AA@ 1019b744     LIBCMTD:undname.obj
 0003:00020750       ??_C@_0L@JMKHOMEK@__fastcall?$AA@ 1019b750     LIBCMTD:undname.obj
 0003:0002075c       ??_C@_0L@NPHFGOKO@__thiscall?$AA@ 1019b75c     LIBCMTD:undname.obj
 0003:00020768       ??_C@_09IFJBGAPI@__stdcall?$AA@ 1019b768     LIBCMTD:undname.obj
 0003:00020774       ??_C@_08GHMPAG@__pascal?$AA@ 1019b774     LIBCMTD:undname.obj
 0003:00020780       ??_C@_07KOLFKCDI@__cdecl?$AA@ 1019b780     LIBCMTD:undname.obj
 0003:00020788       ??_C@_08EHJDFFNH@__based?$CI?$AA@ 1019b788     LIBCMTD:undname.obj
 0003:00020918       ??_C@_04HEJADOOB@CV?3?5?$AA@ 1019b918     LIBCMTD:undname.obj
 0003:00020920       ??_C@_02MOLJINC@?3?3?$AA@  1019b920     LIBCMTD:undname.obj
 0003:00020924       ??_C@_01GEODFPGF@?8?$AA@   1019b924     LIBCMTD:undname.obj
 0003:00020928       ??_C@_01NLNLIGKH@?$GA?$AA@ 1019b928     LIBCMTD:undname.obj
 0003:0002092c       ??_C@_0O@KHGCOMHP@generic?9type?9?$AA@ 1019b92c     LIBCMTD:undname.obj
 0003:0002093c       ??_C@_0BE@JAEOCHPE@template?9parameter?9?$AA@ 1019b93c     LIBCMTD:undname.obj
 0003:00020950       ??_C@_02OHHJMEON@?8?8?$AA@ 1019b950     LIBCMTD:undname.obj
 0003:00020954       ??_C@_0BG@JNJLAMPM@?$GAanonymous?5namespace?8?$AA@ 1019b954     LIBCMTD:undname.obj
 0003:0002096c       ??_C@_0BN@IBLMMFAP@?$GAnon?9type?9template?9parameter?$AA@ 1019b96c     LIBCMTD:undname.obj
 0003:0002098c       ??_C@_0BE@EODMJLIF@?$GAtemplate?9parameter?$AA@ 1019b98c     LIBCMTD:undname.obj
 0003:000209a0       ??_C@_04GKJNKENE@void?$AA@ 1019b9a0     LIBCMTD:undname.obj
 0003:000209a8       ??_C@_04HIBGFPH@NULL?$AA@  1019b9a8     LIBCMTD:undname.obj
 0003:000209b0       ??_C@_0M@DHNBOJMP@extern?5?$CCC?$CC?5?$AA@ 1019b9b0     LIBCMTD:undname.obj
 0003:000209bc       ??_C@_08KJLFOPNE@?$FLthunk?$FN?3?$AA@ 1019b9bc     LIBCMTD:undname.obj
 0003:000209c8       ??_C@_08GPDDCMKI@public?3?5?$AA@ 1019b9c8     LIBCMTD:undname.obj
 0003:000209d4       ??_C@_0M@GAIFPFIP@protected?3?5?$AA@ 1019b9d4     LIBCMTD:undname.obj
 0003:000209e0       ??_C@_09LAPHOOG@private?3?5?$AA@ 1019b9e0     LIBCMTD:undname.obj
 0003:000209ec       ??_C@_08NIEOINHE@virtual?5?$AA@ 1019b9ec     LIBCMTD:undname.obj
 0003:000209f8       ??_C@_07PGOEDBHP@static?5?$AA@ 1019b9f8     LIBCMTD:undname.obj
 0003:00020a00       ??_C@_0DA@HGFJFBBE@?$GAtemplate?5static?5data?5member?5des@ 1019ba00     LIBCMTD:undname.obj
 0003:00020a30       ??_C@_0DB@ILEFOCIJ@?$GAtemplate?5static?5data?5member?5con@ 1019ba30     LIBCMTD:undname.obj
 0003:00020a64       ??_C@_0CB@KJDOOODE@?$GAlocal?5static?5destructor?5helper?8@ 1019ba64     LIBCMTD:undname.obj
 0003:00020a88       ??_C@_0L@HNGCOGAE@?$GAadjustor?$HL?$AA@ 1019ba88     LIBCMTD:undname.obj
 0003:00020a94       ??_C@_0L@GHPFDFH@?$GAvtordisp?$HL?$AA@ 1019ba94     LIBCMTD:undname.obj
 0003:00020aa0       ??_C@_0N@CBHHHENL@?$GAvtordispex?$HL?$AA@ 1019baa0     LIBCMTD:undname.obj
 0003:00020ab0       ??_C@_01CLKCMJKC@?5?$AA@   1019bab0     LIBCMTD:undname.obj
 0003:00020ab4       ??_C@_02IGFCGPIL@?$HN?8?$AA@ 1019bab4     LIBCMTD:undname.obj
 0003:00020ab8       ??_C@_03OPGICMGF@?$HN?8?5?$AA@ 1019bab8     LIBCMTD:undname.obj
 0003:00020abc       ??_C@_02KCKGHPCA@?$CJ?5?$AA@ 1019babc     LIBCMTD:undname.obj
 0003:00020ac0       ??_C@_05BEFAKPML@void?5?$AA@ 1019bac0     LIBCMTD:undname.obj
 0003:00020ac8       ??_C@_08PABEKFH@volatile?$AA@ 1019bac8     LIBCMTD:undname.obj
 0003:00020ad4       ??_C@_0M@ELJOJFFH@?0?$DMellipsis?$DO?$AA@ 1019bad4     LIBCMTD:undname.obj
 0003:00020ae0       ??_C@_04EENFHACM@?0?4?4?4?$AA@ 1019bae0     LIBCMTD:undname.obj
 0003:00020ae8       ??_C@_0L@EGPHHEKN@?$DMellipsis?$DO?$AA@ 1019bae8     LIBCMTD:undname.obj
 0003:00020af4       ??_C@_07HDJPLPEK@?5throw?$CI?$AA@ 1019baf4     LIBCMTD:undname.obj
 0003:00020afc       ??_C@_09EFNPDFFP@?5volatile?$AA@ 1019bafc     LIBCMTD:undname.obj
 0003:00020b08       ??_C@_05BNCCCJPP@const?$AA@ 1019bb08     LIBCMTD:undname.obj
 0003:00020b10       ??_C@_07EDHNAJHC@signed?5?$AA@ 1019bb10     LIBCMTD:undname.obj
 0003:00020b18       ??_C@_09EBBEKKIH@unsigned?5?$AA@ 1019bb18     LIBCMTD:undname.obj
 0003:00020b24       ??_C@_07NFANNNEC@UNKNOWN?$AA@ 1019bb24     LIBCMTD:undname.obj
 0003:00020b2c       ??_C@_06GCICPBLB@__w64?5?$AA@ 1019bb2c     LIBCMTD:undname.obj
 0003:00020b34       ??_C@_07CLGGIAMF@wchar_t?$AA@ 1019bb34     LIBCMTD:undname.obj
 0003:00020b3c       ??_C@_08GAHOLHEO@__int128?$AA@ 1019bb3c     LIBCMTD:undname.obj
 0003:00020b48       ??_C@_07LFCOJCAC@__int64?$AA@ 1019bb48     LIBCMTD:undname.obj
 0003:00020b50       ??_C@_07OFLPPHGP@__int32?$AA@ 1019bb50     LIBCMTD:undname.obj
 0003:00020b58       ??_C@_07ICFHOGAF@__int16?$AA@ 1019bb58     LIBCMTD:undname.obj
 0003:00020b60       ??_C@_06EBGKOKIG@__int8?$AA@ 1019bb60     LIBCMTD:undname.obj
 0003:00020b68       ??_C@_04DDKJGDCM@bool?$AA@ 1019bb68     LIBCMTD:undname.obj
 0003:00020b70       ??_C@_06BNJCAIGJ@double?$AA@ 1019bb70     LIBCMTD:undname.obj
 0003:00020b78       ??_C@_05CJIMAING@long?5?$AA@ 1019bb78     LIBCMTD:undname.obj
 0003:00020b80       ??_C@_05KNFBNCOH@float?$AA@ 1019bb80     LIBCMTD:undname.obj
 0003:00020b88       ??_C@_04GOKPGOLB@long?$AA@ 1019bb88     LIBCMTD:undname.obj
 0003:00020b90       ??_C@_03JBIPMCLC@int?$AA@  1019bb90     LIBCMTD:undname.obj
 0003:00020b94       ??_C@_05BFKKPKCG@short?$AA@ 1019bb94     LIBCMTD:undname.obj
 0003:00020b9c       ??_C@_04ENMBGAPA@char?$AA@ 1019bb9c     LIBCMTD:undname.obj
 0003:00020ba4       ??_C@_05LJGMCFOG@enum?5?$AA@ 1019bba4     LIBCMTD:undname.obj
 0003:00020bac       ??_C@_0N@DLIEFKNA@cointerface?5?$AA@ 1019bbac     LIBCMTD:undname.obj
 0003:00020bbc       ??_C@_08KOFANOFK@coclass?5?$AA@ 1019bbbc     LIBCMTD:undname.obj
 0003:00020bc8       ??_C@_06LJBABKPM@class?5?$AA@ 1019bbc8     LIBCMTD:undname.obj
 0003:00020bd0       ??_C@_07DIBCDNGL@struct?5?$AA@ 1019bbd0     LIBCMTD:undname.obj
 0003:00020bd8       ??_C@_06MOJHIBMG@union?5?$AA@ 1019bbd8     LIBCMTD:undname.obj
 0003:00020be0       ??_C@_0P@GCIFDJCJ@?$GAunknown?5ecsu?8?$AA@ 1019bbe0     LIBCMTD:undname.obj
 0003:00020bf0       ??_C@_04LAHKHJMA@int?5?$AA@ 1019bbf0     LIBCMTD:undname.obj
 0003:00020bf8       ??_C@_06EHJMALKF@short?5?$AA@ 1019bbf8     LIBCMTD:undname.obj
 0003:00020c00       ??_C@_05CIHEBHNO@char?5?$AA@ 1019bc00     LIBCMTD:undname.obj
 0003:00020c08       ??_C@_06LIJLOJAG@const?5?$AA@ 1019bc08     LIBCMTD:undname.obj
 0003:00020c10       ??_C@_09GAIEOBLP@volatile?5?$AA@ 1019bc10     LIBCMTD:undname.obj
 0003:00020c1c       ??_C@_0O@GKABPPIF@cli?3?3pin_ptr?$DM?$AA@ 1019bc1c     LIBCMTD:undname.obj
 0003:00020c2c       ??_C@_0M@EALIELKG@cli?3?3array?$DM?$AA@ 1019bc2c     LIBCMTD:undname.obj
 0003:00020c38       ??_C@_02GOGNNPBN@?$CJ?$FL?$AA@ 1019bc38     LIBCMTD:undname.obj
 0003:00020c3c       ??_C@_06EEGAIFAK@?$HLflat?$HN?$AA@ 1019bc3c     LIBCMTD:undname.obj
 0003:00020c44       ??_C@_02MDINNEEG@s?5?$AA@  1019bc44     LIBCMTD:undname.obj
 0003:00020c48       ??_C@_05JIBOFOHK@?$HLfor?5?$AA@ 1019bc48     LIBCMTD:undname.obj
 0003:00020c50       ??_7DNameNode@@6B@         1019bc50     LIBCMTD:undname.obj
 0003:00020c5c       ??_7charNode@@6B@          1019bc5c     LIBCMTD:undname.obj
 0003:00020c68       ??_7pcharNode@@6B@         1019bc68     LIBCMTD:undname.obj
 0003:00020c74       ??_7pDNameNode@@6B@        1019bc74     LIBCMTD:undname.obj
 0003:00020c80       ??_7DNameStatusNode@@6B@   1019bc80     LIBCMTD:undname.obj
 0003:00020c8c       ??_C@_04OKOHEJBO@?5?$DP?$DP?5?$AA@ 1019bc8c     LIBCMTD:undname.obj
 0003:00020c94       ??_7pairNode@@6B@          1019bc94     LIBCMTD:undname.obj
 0003:00020ca0       ??_C@_1BE@KHFBJMNM@?$AA_?$AAl?$AAs?$AAe?$AAe?$AAk?$AAi?$AA6?$AA4?$AA?$AA@ 1019bca0     LIBCMTD:lseeki64.obj
 0003:00020cb8       ??_C@_1GE@MINKPNPH@?$AAf?$AA?3?$AA?2?$AAd?$AAd?$AA?2?$AAv?$AAc?$AAt?$AAo?$AAo?$AAl?$AAs?$AA?2?$AAc?$AAr?$AAt?$AA_?$AAb?$AAl?$AAd?$AA?2?$AAs?$AAe?$AAl?$AAf?$AA_?$AAx?$AA8?$AA6?$AA?2?$AAc@ 1019bcb8     LIBCMTD:lseeki64.obj
 0003:00020d1c       ??_C@_0DB@JEHOCBEJ@f?3?2dd?2vctools?2crt_bld?2self_x86?2c@ 1019bd1c     LIBCMTD:_getbuf.obj
 0003:00020d50       ??_C@_1GC@DKMGNNCC@?$AAf?$AA?3?$AA?2?$AAd?$AAd?$AA?2?$AAv?$AAc?$AAt?$AAo?$AAo?$AAl?$AAs?$AA?2?$AAc?$AAr?$AAt?$AA_?$AAb?$AAl?$AAd?$AA?2?$AAs?$AAe?$AAl?$AAf?$AA_?$AAx?$AA8?$AA6?$AA?2?$AAc@ 1019bd50     LIBCMTD:_getbuf.obj
 0003:00020db4       ??_C@_1BA@LEBDGIHM@?$AA_?$AAi?$AAs?$AAa?$AAt?$AAt?$AAy?$AA?$AA@ 1019bdb4     LIBCMTD:isatty.obj
 0003:00020dc8       ??_C@_1GA@LPGDJDEN@?$AAf?$AA?3?$AA?2?$AAd?$AAd?$AA?2?$AAv?$AAc?$AAt?$AAo?$AAo?$AAl?$AAs?$AA?2?$AAc?$AAr?$AAt?$AA_?$AAb?$AAl?$AAd?$AA?2?$AAs?$AAe?$AAl?$AAf?$AA_?$AAx?$AA8?$AA6?$AA?2?$AAc@ 1019bdc8     LIBCMTD:isatty.obj
 0003:00020e28       ??_C@_1BI@IEADNOHF@?$AA_?$AAw?$AAc?$AAt?$AAo?$AAm?$AAb?$AA_?$AAs?$AA_?$AAl?$AA?$AA@ 1019be28     LIBCMTD:wctomb.obj
 0003:00020e40       ??_C@_1GA@LDLHPOO@?$AAf?$AA?3?$AA?2?$AAd?$AAd?$AA?2?$AAv?$AAc?$AAt?$AAo?$AAo?$AAl?$AAs?$AA?2?$AAc?$AAr?$AAt?$AA_?$AAb?$AAl?$AAd?$AA?2?$AAs?$AAe?$AAl?$AAf?$AA_?$AAx?$AA8?$AA6?$AA?2?$AAc@ 1019be40     LIBCMTD:wctomb.obj
 0003:00020ea0       ??_C@_1CO@HFMIILNF@?$AAs?$AAi?$AAz?$AAe?$AAI?$AAn?$AAB?$AAy?$AAt?$AAe?$AAs?$AA?5?$AA?$DM?$AA?$DN?$AA?5?$AAI?$AAN?$AAT?$AA_?$AAM?$AAA?$AAX?$AA?$AA@ 1019bea0     LIBCMTD:wctomb.obj
 0003:00020ed0       ___lookuptable_s           1019bed0     LIBCMTD:outputs.obj
 0003:00020f2c       ??_C@_1BI@COFBLHCG@?$AA_?$AAo?$AAu?$AAt?$AAp?$AAu?$AAt?$AA_?$AAs?$AA_?$AAl?$AA?$AA@ 1019bf2c     LIBCMTD:outputs.obj
 0003:00020f44       ??_C@_1BM@HBMHMBEM@?$AA_?$AAm?$AAb?$AAs?$AAn?$AAb?$AAc?$AAp?$AAy?$AA_?$AAs?$AA_?$AAl?$AA?$AA@ 1019bf44     LIBCMTD:mbsnbcpy_s_l.obj
 0003:00020f60       ??_C@_1GK@MBHICH@?$AAf?$AA?3?$AA?2?$AAd?$AAd?$AA?2?$AAv?$AAc?$AAt?$AAo?$AAo?$AAl?$AAs?$AA?2?$AAc?$AAr?$AAt?$AA_?$AAb?$AAl?$AAd?$AA?2?$AAs?$AAe?$AAl?$AAf?$AA_?$AAx?$AA8?$AA6?$AA?2?$AAc@ 1019bf60     LIBCMTD:mbsnbcpy_s_l.obj
 0003:00020fcc       ??_C@_1CA@HPEMMJMJ@?$AAc?$AAu?$AAr?$AAr?$AAe?$AAn?$AAt?$AA?5?$AA?$CB?$AA?$DN?$AA?5?$AAN?$AAU?$AAL?$AAL?$AA?$AA@ 1019bfcc     LIBCMTD:mbsdec.obj
 0003:00020fec       ??_C@_1BE@KLNCOLCD@?$AA_?$AAm?$AAb?$AAs?$AAd?$AAe?$AAc?$AA_?$AAl?$AA?$AA@ 1019bfec     LIBCMTD:mbsdec.obj
 0003:00021000       ??_C@_1GA@FCFHDJEM@?$AAf?$AA?3?$AA?2?$AAd?$AAd?$AA?2?$AAv?$AAc?$AAt?$AAo?$AAo?$AAl?$AAs?$AA?2?$AAc?$AAr?$AAt?$AA_?$AAb?$AAl?$AAd?$AA?2?$AAs?$AAe?$AAl?$AAf?$AA_?$AAx?$AA8?$AA6?$AA?2?$AAc@ 1019c000     LIBCMTD:mbsdec.obj
 0003:00021060       ??_C@_1BO@JIBAMMGI@?$AAs?$AAt?$AAr?$AAi?$AAn?$AAg?$AA?5?$AA?$CB?$AA?$DN?$AA?5?$AAN?$AAU?$AAL?$AAL?$AA?$AA@ 1019c060     LIBCMTD:mbsdec.obj
 0003:00021080       ??_C@_1M@MFLJCMFJ@?$AA_?$AAo?$AAp?$AAe?$AAn?$AA?$AA@ 1019c080     LIBCMTD:open.obj
 0003:00021090       ??_C@_1FM@LFKHNNH@?$AAf?$AA?3?$AA?2?$AAd?$AAd?$AA?2?$AAv?$AAc?$AAt?$AAo?$AAo?$AAl?$AAs?$AA?2?$AAc?$AAr?$AAt?$AA_?$AAb?$AAl?$AAd?$AA?2?$AAs?$AAe?$AAl?$AAf?$AA_?$AAx?$AA8?$AA6?$AA?2?$AAc@ 1019c090     LIBCMTD:open.obj
 0003:000210ec       ??_C@_1BO@DPAOGEII@?$AA?$CI?$AAp?$AAa?$AAt?$AAh?$AA?5?$AA?$CB?$AA?$DN?$AA?5?$AAN?$AAU?$AAL?$AAL?$AA?$CJ?$AA?$AA@ 1019c0ec     LIBCMTD:open.obj
 0003:00021110       ??_C@_1FG@NFINBJCM@?$AA?$CI?$AA?$CI?$AAp?$AAm?$AAo?$AAd?$AAe?$AA?5?$AA?$CG?$AA?5?$AA?$CI?$AA?$HO?$AA?$CI?$AA_?$AAS?$AA_?$AAI?$AAR?$AAE?$AAA?$AAD?$AA?5?$AA?$HM?$AA?5?$AA_?$AAS?$AA_?$AAI?$AAW?$AAR?$AAI?$AAT@ 1019c110     LIBCMTD:open.obj
 0003:00021168       ??_C@_1BM@IOBAMMHO@?$AA_?$AAs?$AAo?$AAp?$AAe?$AAn?$AA_?$AAh?$AAe?$AAl?$AAp?$AAe?$AAr?$AA?$AA@ 1019c168     LIBCMTD:open.obj
 0003:00021184       ??_C@_1BM@PGEEHLHE@?$AA?$CI?$AAp?$AAf?$AAh?$AA?5?$AA?$CB?$AA?$DN?$AA?5?$AAN?$AAU?$AAL?$AAL?$AA?$CJ?$AA?$AA@ 1019c184     LIBCMTD:open.obj
 0003:000211a0       ??_C@_1IA@IENOJNJF@?$AA0?$AA?5?$AA?$CG?$AA?$CG?$AA?5?$AA?$CC?$AAO?$AAn?$AAl?$AAy?$AA?5?$AAU?$AAT?$AAF?$AA?9?$AA1?$AA6?$AA?5?$AAl?$AAi?$AAt?$AAt?$AAl?$AAe?$AA?5?$AAe?$AAn?$AAd?$AAi?$AAa?$AAn?$AA?5@ 1019c1a0     LIBCMTD:open.obj
 0003:00021220       ??_C@_1CM@IDLMKMPG@?$AA0?$AA?5?$AA?$CG?$AA?$CG?$AA?5?$AA?$CC?$AAI?$AAn?$AAt?$AAe?$AAr?$AAn?$AAa?$AAl?$AA?5?$AAE?$AAr?$AAr?$AAo?$AAr?$AA?$CC?$AA?$AA@ 1019c220     LIBCMTD:open.obj
 0003:00021250       ??_C@_1HM@GJANBLHJ@?$AA?$CI?$AAo?$AAf?$AAl?$AAa?$AAg?$AA?5?$AA?$CG?$AA?5?$AA?$CI?$AA_?$AAO?$AA_?$AAT?$AAE?$AAX?$AAT?$AA?5?$AA?$HM?$AA?5?$AA_?$AAO?$AA_?$AAW?$AAT?$AAE?$AAX?$AAT?$AA?5?$AA?$HM?$AA?5?$AA_@ 1019c250     LIBCMTD:open.obj
 0003:000212cc       ??_C@_1DO@PJLMOANO@?$AA?$CI?$AA?5?$AA?$CC?$AAI?$AAn?$AAv?$AAa?$AAl?$AAi?$AAd?$AA?5?$AAs?$AAh?$AAa?$AAr?$AAi?$AAn?$AAg?$AA?5?$AAf?$AAl?$AAa?$AAg?$AA?$CC?$AA?5?$AA?0?$AA?5?$AA0?$AA?5?$AA?$CJ?$AA?$AA@ 1019c2cc     LIBCMTD:open.obj
 0003:0002130c       ??_C@_1DI@DGKIFCCE@?$AA?$CI?$AA?5?$AA?$CC?$AAI?$AAn?$AAv?$AAa?$AAl?$AAi?$AAd?$AA?5?$AAo?$AAp?$AAe?$AAn?$AA?5?$AAf?$AAl?$AAa?$AAg?$AA?$CC?$AA?5?$AA?0?$AA?5?$AA0?$AA?5?$AA?$CJ?$AA?$AA@ 1019c30c     LIBCMTD:open.obj
 0003:00021344       ??_C@_1CG@ICBEBDJJ@?$AA_?$AAg?$AAe?$AAt?$AA_?$AAf?$AAm?$AAo?$AAd?$AAe?$AA?$CI?$AA?$CG?$AAf?$AAm?$AAo?$AAd?$AAe?$AA?$CJ?$AA?$AA@ 1019c344     LIBCMTD:open.obj
 0003:0002136c       ??_C@_1BO@JOPFMPGH@?$AA_?$AAt?$AAs?$AAo?$AAp?$AAe?$AAn?$AA_?$AAn?$AAo?$AAl?$AAo?$AAc?$AAk?$AA?$AA@ 1019c36c     LIBCMTD:open.obj
 0003:0002138c       ??_C@_1BG@GBJNMPFA@?$AAs?$AA2?$AA?5?$AA?$CB?$AA?$DN?$AA?5?$AAN?$AAU?$AAL?$AAL?$AA?$AA@ 1019c38c     LIBCMTD:mbsnbicm.obj
 0003:000213a4       ??_C@_1BK@GEJONGBG@?$AA_?$AAm?$AAb?$AAs?$AAn?$AAb?$AAi?$AAc?$AAm?$AAp?$AA_?$AAl?$AA?$AA@ 1019c3a4     LIBCMTD:mbsnbicm.obj
 0003:000213c0       ??_C@_1GE@JLFFJINF@?$AAf?$AA?3?$AA?2?$AAd?$AAd?$AA?2?$AAv?$AAc?$AAt?$AAo?$AAo?$AAl?$AAs?$AA?2?$AAc?$AAr?$AAt?$AA_?$AAb?$AAl?$AAd?$AA?2?$AAs?$AAe?$AAl?$AAf?$AA_?$AAx?$AA8?$AA6?$AA?2?$AAc@ 1019c3c0     LIBCMTD:mbsnbicm.obj
 0003:00021424       ??_C@_1BG@MODEICJK@?$AAs?$AA1?$AA?5?$AA?$CB?$AA?$DN?$AA?5?$AAN?$AAU?$AAL?$AAL?$AA?$AA@ 1019c424     LIBCMTD:mbsnbicm.obj
 0003:0002143c       ??_C@_1BI@LPHOHGHI@?$AA_?$AAm?$AAb?$AAs?$AAn?$AAb?$AAc?$AAm?$AAp?$AA_?$AAl?$AA?$AA@ 1019c43c     LIBCMTD:mbsnbcmp.obj
 0003:00021458       ??_C@_1GE@IIBFGEPN@?$AAf?$AA?3?$AA?2?$AAd?$AAd?$AA?2?$AAv?$AAc?$AAt?$AAo?$AAo?$AAl?$AAs?$AA?2?$AAc?$AAr?$AAt?$AA_?$AAb?$AAl?$AAd?$AA?2?$AAs?$AAe?$AAl?$AAf?$AA_?$AAx?$AA8?$AA6?$AA?2?$AAc@ 1019c458     LIBCMTD:mbsnbcmp.obj
 0003:000214c0       __atan_table               1019c4c0     LIBCMTD:_atan_table_.obj
 0003:00022cd0       ??_C@_1BA@NGNGNDEP@?$AA_?$AAc?$AAp?$AAu?$AAt?$AAw?$AAs?$AA?$AA@ 1019dcd0     LIBCMTD:putwch.obj
 0003:00022ce0       ??_C@_1GA@NKLOJFIJ@?$AAf?$AA?3?$AA?2?$AAd?$AAd?$AA?2?$AAv?$AAc?$AAt?$AAo?$AAo?$AAl?$AAs?$AA?2?$AAc?$AAr?$AAt?$AA_?$AAb?$AAl?$AAd?$AA?2?$AAs?$AAe?$AAl?$AAf?$AA_?$AAx?$AA8?$AA6?$AA?2?$AAc@ 1019dce0     LIBCMTD:putwch.obj
 0003:00022d40       ??_C@_1GA@GFFDGGFH@?$AAf?$AA?3?$AA?2?$AAd?$AAd?$AA?2?$AAv?$AAc?$AAt?$AAo?$AAo?$AAl?$AAs?$AA?2?$AAc?$AAr?$AAt?$AA_?$AAb?$AAl?$AAd?$AA?2?$AAs?$AAe?$AAl?$AAf?$AA_?$AAx?$AA8?$AA6?$AA?2?$AAc@ 1019dd40     LIBCMTD:mbtowc.obj
 0003:00022da0       ??_C@_1NC@EINCOKCO@?$AA_?$AAl?$AAo?$AAc?$AA_?$AAu?$AAp?$AAd?$AAa?$AAt?$AAe?$AA?4?$AAG?$AAe?$AAt?$AAL?$AAo?$AAc?$AAa?$AAl?$AAe?$AAT?$AA?$CI?$AA?$CJ?$AA?9?$AA?$DO?$AAl?$AAo?$AAc?$AAi?$AAn?$AAf@ 1019dda0     LIBCMTD:mbtowc.obj
 0003:00022e74       ??_C@_0BK@CIDNPOGP@GetUserObjectInformationA?$AA@ 1019de74     LIBCMTD:crtmbox.obj
 0003:00022e90       ??_C@_0M@CHKKJDAI@MessageBoxA?$AA@ 1019de90     LIBCMTD:crtmbox.obj
 0003:00022e9c       ??_C@_0L@NDEGIDAG@USER32?4DLL?$AA@ 1019de9c     LIBCMTD:crtmbox.obj
 0003:00022ea8       ??_C@_1CA@LFDHAMEM@?$AA_?$AAs?$AAe?$AAt?$AA_?$AAe?$AAr?$AAr?$AAo?$AAr?$AA_?$AAm?$AAo?$AAd?$AAe?$AA?$AA@ 1019dea8     LIBCMTD:errmode.obj
 0003:00022ec8       ??_C@_1GC@FGMGFCNB@?$AAf?$AA?3?$AA?2?$AAd?$AAd?$AA?2?$AAv?$AAc?$AAt?$AAo?$AAo?$AAl?$AAs?$AA?2?$AAc?$AAr?$AAt?$AA_?$AAb?$AAl?$AAd?$AA?2?$AAs?$AAe?$AAl?$AAf?$AA_?$AAx?$AA8?$AA6?$AA?2?$AAc@ 1019dec8     LIBCMTD:errmode.obj
 0003:00022f2c       ??_C@_1DE@BCNCAIK@?$AA?$CI?$AA?$CC?$AAI?$AAn?$AAv?$AAa?$AAl?$AAi?$AAd?$AA?5?$AAe?$AAr?$AAr?$AAo?$AAr?$AA_?$AAm?$AAo?$AAd?$AAe?$AA?$CC?$AA?0?$AA?5?$AA0?$AA?$CJ?$AA?$AA@ 1019df2c     LIBCMTD:errmode.obj
 0003:00022f60       ??_C@_0DC@IHGBBJOH@f?3?2dd?2vctools?2crt_bld?2self_x86?2c@ 1019df60     LIBCMTD:convrtcp.obj
 0003:00022f94       ___dnames                  1019df94     LIBCMTD:timeset.obj
 0003:00022fac       ___mnames                  1019dfac     LIBCMTD:timeset.obj
 0003:00022fd4       ??_C@_1BM@FIMHBHEB@?$AA_?$AAg?$AAe?$AAt?$AA_?$AAd?$AAa?$AAy?$AAl?$AAi?$AAg?$AAh?$AAt?$AA?$AA@ 1019dfd4     LIBCMTD:timeset.obj
 0003:00022ff0       ??_C@_1GC@NEGFAKA@?$AAf?$AA?3?$AA?2?$AAd?$AAd?$AA?2?$AAv?$AAc?$AAt?$AAo?$AAo?$AAl?$AAs?$AA?2?$AAc?$AAr?$AAt?$AA_?$AAb?$AAl?$AAd?$AA?2?$AAs?$AAe?$AAl?$AAf?$AA_?$AAx?$AA8?$AA6?$AA?2?$AAc@ 1019dff0     LIBCMTD:timeset.obj
 0003:00023054       ??_C@_1CI@MKJEHFPG@?$AA?$CI?$AA_?$AAD?$AAa?$AAy?$AAl?$AAi?$AAg?$AAh?$AAt?$AA?5?$AA?$CB?$AA?$DN?$AA?5?$AAN?$AAU?$AAL?$AAL?$AA?$CJ?$AA?$AA@ 1019e054     LIBCMTD:timeset.obj
 0003:0002307c       ??_C@_1BK@EMODDHEE@?$AA_?$AAg?$AAe?$AAt?$AA_?$AAd?$AAs?$AAt?$AAb?$AAi?$AAa?$AAs?$AA?$AA@ 1019e07c     LIBCMTD:timeset.obj
 0003:00023098       ??_C@_1EC@PKDJPAAB@?$AA?$CI?$AA_?$AAD?$AAa?$AAy?$AAl?$AAi?$AAg?$AAh?$AAt?$AA_?$AAs?$AAa?$AAv?$AAi?$AAn?$AAg?$AAs?$AA_?$AAb?$AAi?$AAa?$AAs?$AA?5?$AA?$CB?$AA?$DN?$AA?5?$AAN?$AAU?$AAL?$AAL?$AA?$CJ@ 1019e098     LIBCMTD:timeset.obj
 0003:000230dc       ??_C@_1BM@MGEAKPEJ@?$AA_?$AAg?$AAe?$AAt?$AA_?$AAt?$AAi?$AAm?$AAe?$AAz?$AAo?$AAn?$AAe?$AA?$AA@ 1019e0dc     LIBCMTD:timeset.obj
 0003:000230f8       ??_C@_1CI@PODJJGAL@?$AA?$CI?$AA_?$AAT?$AAi?$AAm?$AAe?$AAz?$AAo?$AAn?$AAe?$AA?5?$AA?$CB?$AA?$DN?$AA?5?$AAN?$AAU?$AAL?$AAL?$AA?$CJ?$AA?$AA@ 1019e0f8     LIBCMTD:timeset.obj
 0003:00023120       ??_C@_1DG@HLGKANIP@?$AA_?$AAI?$AAn?$AAd?$AAe?$AAx?$AA?5?$AA?$DN?$AA?$DN?$AA?5?$AA0?$AA?5?$AA?$HM?$AA?$HM?$AA?5?$AA_?$AAI?$AAn?$AAd?$AAe?$AAx?$AA?5?$AA?$DN?$AA?$DN?$AA?5?$AA1?$AA?$AA@ 1019e120     LIBCMTD:timeset.obj
 0003:00023158       ??_C@_1CK@GBKHKEI@?$AA_?$AAR?$AAe?$AAt?$AAu?$AAr?$AAn?$AAV?$AAa?$AAl?$AAu?$AAe?$AA?5?$AA?$CB?$AA?$DN?$AA?5?$AAN?$AAU?$AAL?$AAL?$AA?$AA@ 1019e158     LIBCMTD:timeset.obj
 0003:00023184       ??_C@_1BI@BHCKCCFA@?$AA_?$AAg?$AAe?$AAt?$AA_?$AAt?$AAz?$AAn?$AAa?$AAm?$AAe?$AA?$AA@ 1019e184     LIBCMTD:timeset.obj
 0003:000231a0       ??_C@_1KA@POFLNEC@?$AA?$CI?$AA_?$AAB?$AAu?$AAf?$AAf?$AAe?$AAr?$AA?5?$AA?$CB?$AA?$DN?$AA?5?$AAN?$AAU?$AAL?$AAL?$AA?5?$AA?$CG?$AA?$CG?$AA?5?$AA_?$AAS?$AAi?$AAz?$AAe?$AAI?$AAn?$AAB?$AAy?$AAt?$AAe?$AAs@ 1019e1a0     LIBCMTD:timeset.obj
 0003:00023240       ??_C@_1EA@GEPBEDLJ@?$AAs?$AAt?$AAr?$AAn?$AAc?$AAp?$AAy?$AA_?$AAs?$AA?$CI?$AAt?$AAz?$AAn?$AAa?$AAm?$AAe?$AA?$FL?$AA1?$AA?$FN?$AA?0?$AA?5?$AA6?$AA4?$AA?0?$AA?5?$AAT?$AAZ?$AA?0?$AA?5?$AA3?$AA?$CJ?$AA?$AA@ 1019e240     LIBCMTD:tzset.obj
 0003:00023280       ??_C@_1EA@FIJBKALB@?$AAs?$AAt?$AAr?$AAn?$AAc?$AAp?$AAy?$AA_?$AAs?$AA?$CI?$AAt?$AAz?$AAn?$AAa?$AAm?$AAe?$AA?$FL?$AA0?$AA?$FN?$AA?0?$AA?5?$AA6?$AA4?$AA?0?$AA?5?$AAT?$AAZ?$AA?0?$AA?5?$AA3?$AA?$CJ?$AA?$AA@ 1019e280     LIBCMTD:tzset.obj
 0003:000232c0       ??_C@_1EK@MCAIMDPB@?$AAs?$AAt?$AAr?$AAc?$AAp?$AAy?$AA_?$AAs?$AA?$CI?$AAl?$AAa?$AAs?$AAt?$AAT?$AAZ?$AA?0?$AA?5?$AAs?$AAt?$AAr?$AAl?$AAe?$AAn?$AA?$CI?$AAT?$AAZ?$AA?$CJ?$AA?5?$AA?$CL?$AA?5?$AA1?$AA?0@ 1019e2c0     LIBCMTD:tzset.obj
 0003:0002330c       ??_C@_0CP@FODJBIFF@f?3?2dd?2vctools?2crt_bld?2self_x86?2c@ 1019e30c     LIBCMTD:tzset.obj
 0003:0002333c       ??_C@_02CLFPBFFP@TZ?$AA@   1019e33c     LIBCMTD:tzset.obj
 0003:00023340       ??_C@_1CO@IMMOMMCB@?$AA_?$AAg?$AAe?$AAt?$AA_?$AAd?$AAs?$AAt?$AAb?$AAi?$AAa?$AAs?$AA?$CI?$AA?$CG?$AAd?$AAs?$AAt?$AAb?$AAi?$AAa?$AAs?$AA?$CJ?$AA?$AA@ 1019e340     LIBCMTD:tzset.obj
 0003:00023370       ??_C@_1DC@MEHEMOPB@?$AA_?$AAg?$AAe?$AAt?$AA_?$AAd?$AAa?$AAy?$AAl?$AAi?$AAg?$AAh?$AAt?$AA?$CI?$AA?$CG?$AAd?$AAa?$AAy?$AAl?$AAi?$AAg?$AAh?$AAt?$AA?$CJ?$AA?$AA@ 1019e370     LIBCMTD:tzset.obj
 0003:000233a4       ??_C@_1DC@CMKCHHFC@?$AA_?$AAg?$AAe?$AAt?$AA_?$AAt?$AAi?$AAm?$AAe?$AAz?$AAo?$AAn?$AAe?$AA?$CI?$AA?$CG?$AAt?$AAi?$AAm?$AAe?$AAz?$AAo?$AAn?$AAe?$AA?$CJ?$AA?$AA@ 1019e3a4     LIBCMTD:tzset.obj
 0003:000233d8       ??_C@_1BM@IIODHMJC@?$AA_?$AAt?$AAz?$AAs?$AAe?$AAt?$AA_?$AAn?$AAo?$AAl?$AAo?$AAc?$AAk?$AA?$AA@ 1019e3d8     LIBCMTD:tzset.obj
 0003:000233f8       ??_C@_1FO@MLHAIHAB@?$AAf?$AA?3?$AA?2?$AAd?$AAd?$AA?2?$AAv?$AAc?$AAt?$AAo?$AAo?$AAl?$AAs?$AA?2?$AAc?$AAr?$AAt?$AA_?$AAb?$AAl?$AAd?$AA?2?$AAs?$AAe?$AAl?$AAf?$AA_?$AAx?$AA8?$AA6?$AA?2?$AAc@ 1019e3f8     LIBCMTD:tzset.obj
 0003:00023458       ??_C@_1CA@GOLIIEDM@?$AA_?$AAi?$AAs?$AAi?$AAn?$AAd?$AAs?$AAt?$AA_?$AAn?$AAo?$AAl?$AAo?$AAc?$AAk?$AA?$AA@ 1019e458     LIBCMTD:tzset.obj
 0003:00023478       ??_C@_1BA@GOCKIDGO@?$AAc?$AAv?$AAt?$AAd?$AAa?$AAt?$AAe?$AA?$AA@ 1019e478     LIBCMTD:tzset.obj
 0003:00023488       ??_C@_1CC@JLPHKJPH@?$AAc?$AAo?$AAu?$AAn?$AAt?$AA?5?$AA?$DM?$AA?$DN?$AA?5?$AAI?$AAN?$AAT?$AA_?$AAM?$AAA?$AAX?$AA?$AA@ 1019e488     LIBCMTD:strnicmp.obj
 0003:000234ac       ??_C@_1BI@BJLEPLEF@?$AA_?$AAs?$AAt?$AAr?$AAn?$AAi?$AAc?$AAm?$AAp?$AA_?$AAl?$AA?$AA@ 1019e4ac     LIBCMTD:strnicmp.obj
 0003:000234c8       ??_C@_1GE@CONPOJMA@?$AAf?$AA?3?$AA?2?$AAd?$AAd?$AA?2?$AAv?$AAc?$AAt?$AAo?$AAo?$AAl?$AAs?$AA?2?$AAc?$AAr?$AAt?$AA_?$AAb?$AAl?$AAd?$AA?2?$AAs?$AAe?$AAl?$AAf?$AA_?$AAx?$AA8?$AA6?$AA?2?$AAc@ 1019e4c8     LIBCMTD:strnicmp.obj
 0003:0002352c       ??_C@_1BE@BHJDFFNA@?$AA_?$AAs?$AAt?$AAr?$AAn?$AAi?$AAc?$AAm?$AAp?$AA?$AA@ 1019e52c     LIBCMTD:strnicmp.obj
 0003:00023540       ?commonFlags@?1??_control87@@9@9 1019e540     LIBCMTD:_ieee87_.obj
 0003:00023548       ??_C@_1GO@OKJGOMCB@?$AA_?$AAc?$AAo?$AAn?$AAt?$AAr?$AAo?$AAl?$AAf?$AAp?$AA_?$AAs?$AA?$CI?$AA?$CI?$AA?$CI?$AAv?$AAo?$AAi?$AAd?$AA?5?$AA?$CK?$AA?$CJ?$AA0?$AA?$CJ?$AA?0?$AA?5?$AAn?$AAe?$AAw?$AAc?$AAt?$AAr@ 1019e548     LIBCMTD:_ieee87_.obj
 0003:000235b8       ??_C@_1BO@OFDNCLL@?$AA_?$AAs?$AAe?$AAt?$AA_?$AAc?$AAo?$AAn?$AAt?$AAr?$AAo?$AAl?$AAf?$AAp?$AA?$AA@ 1019e5b8     LIBCMTD:_ieee87_.obj
 0003:000235d8       ??_C@_1HO@BFDKGHOI@?$AAf?$AA?3?$AA?2?$AAd?$AAd?$AA?2?$AAv?$AAc?$AAt?$AAo?$AAo?$AAl?$AAs?$AA?2?$AAc?$AAr?$AAt?$AA_?$AAb?$AAl?$AAd?$AA?2?$AAs?$AAe?$AAl?$AAf?$AA_?$AAx?$AA8?$AA6?$AA?2?$AAc@ 1019e5d8     LIBCMTD:_ieee87_.obj
 0003:00023658       ??_C@_06IMKFLFPG@1?$CDQNAN?$AA@ 1019e658     LIBCMTD:_x10fout_.obj
 0003:00023660       ??_C@_1EG@MCFPJJEM@?$AAs?$AAt?$AAr?$AAc?$AAp?$AAy?$AA_?$AAs?$AA?$CI?$AAf?$AAo?$AAs?$AA?9?$AA?$DO?$AAm?$AAa?$AAn?$AA?0?$AA?5?$AA2?$AA1?$AA?$CL?$AA1?$AA?0?$AA?5?$AA?$CC?$AA1?$AA?$CD?$AAQ?$AAN?$AAA?$AAN@ 1019e660     LIBCMTD:_x10fout_.obj
 0003:000236a8       ??_C@_05DNEBIAHO@1?$CDINF?$AA@ 1019e6a8     LIBCMTD:_x10fout_.obj
 0003:000236b0       ??_C@_1EE@ICBBBPAI@?$AAs?$AAt?$AAr?$AAc?$AAp?$AAy?$AA_?$AAs?$AA?$CI?$AAf?$AAo?$AAs?$AA?9?$AA?$DO?$AAm?$AAa?$AAn?$AA?0?$AA?5?$AA2?$AA1?$AA?$CL?$AA1?$AA?0?$AA?5?$AA?$CC?$AA1?$AA?$CD?$AAI?$AAN?$AAF?$AA?$CC@ 1019e6b0     LIBCMTD:_x10fout_.obj
 0003:000236f4       ??_C@_05PHHOCPM@1?$CDIND?$AA@ 1019e6f4     LIBCMTD:_x10fout_.obj
 0003:00023700       ??_C@_1EE@MADEBIHF@?$AAs?$AAt?$AAr?$AAc?$AAp?$AAy?$AA_?$AAs?$AA?$CI?$AAf?$AAo?$AAs?$AA?9?$AA?$DO?$AAm?$AAa?$AAn?$AA?0?$AA?5?$AA2?$AA1?$AA?$CL?$AA1?$AA?0?$AA?5?$AA?$CC?$AA1?$AA?$CD?$AAI?$AAN?$AAD?$AA?$CC@ 1019e700     LIBCMTD:_x10fout_.obj
 0003:00023744       ??_C@_06PGGFOGJG@1?$CDSNAN?$AA@ 1019e744     LIBCMTD:_x10fout_.obj
 0003:00023750       ??_C@_1EG@CDDBFNOB@?$AAs?$AAt?$AAr?$AAc?$AAp?$AAy?$AA_?$AAs?$AA?$CI?$AAf?$AAo?$AAs?$AA?9?$AA?$DO?$AAm?$AAa?$AAn?$AA?0?$AA?5?$AA2?$AA1?$AA?$CL?$AA1?$AA?0?$AA?5?$AA?$CC?$AA1?$AA?$CD?$AAS?$AAN?$AAA?$AAN@ 1019e750     LIBCMTD:_x10fout_.obj
 0003:00023798       ??_C@_1BI@ELMAAFLN@?$AA$?$AAI?$AA1?$AA0?$AA_?$AAO?$AAU?$AAT?$AAP?$AAU?$AAT?$AA?$AA@ 1019e798     LIBCMTD:_x10fout_.obj
 0003:000237b0       ??_C@_1HG@HFJMHCFK@?$AAf?$AA?3?$AA?2?$AAd?$AAd?$AA?2?$AAv?$AAc?$AAt?$AAo?$AAo?$AAl?$AAs?$AA?2?$AAc?$AAr?$AAt?$AA_?$AAb?$AAl?$AAd?$AA?2?$AAs?$AAe?$AAl?$AAf?$AA_?$AAx?$AA8?$AA6?$AA?2?$AAc@ 1019e7b0     LIBCMTD:_x10fout_.obj
 0003:00023828       ??_C@_1BK@ONMFGLDB@?$AA_?$AAw?$AAo?$AAu?$AAt?$AAp?$AAu?$AAt?$AA_?$AAs?$AA_?$AAl?$AA?$AA@ 1019e828     LIBCMTD:woutputs.obj
 0003:00023844       ??_C@_1BK@GDEKGMNC@?$AA_?$AAw?$AAo?$AAu?$AAt?$AAp?$AAu?$AAt?$AA_?$AAp?$AA_?$AAl?$AA?$AA@ 1019e844     LIBCMTD:woutputp.obj
 0003:00023860       ??_C@_1O@HJNPHHHB@?$AAf?$AAp?$AAu?$AAt?$AAw?$AAc?$AA?$AA@ 1019e860     LIBCMTD:fputwc.obj
 0003:00023870       ??_C@_1GA@BJIGKGEA@?$AAf?$AA?3?$AA?2?$AAd?$AAd?$AA?2?$AAv?$AAc?$AAt?$AAo?$AAo?$AAl?$AAs?$AA?2?$AAc?$AAr?$AAt?$AA_?$AAb?$AAl?$AAd?$AA?2?$AAs?$AAe?$AAl?$AAf?$AA_?$AAx?$AA8?$AA6?$AA?2?$AAc@ 1019e870     LIBCMTD:fputwc.obj
 0003:000238d0       ??_C@_1BI@GALBKMKE@?$AA?$CI?$AAs?$AAi?$AAz?$AAe?$AA?5?$AA?$DO?$AA?$DN?$AA?5?$AA0?$AA?$CJ?$AA?$AA@ 1019e8d0     LIBCMTD:chsize.obj
 0003:000238e8       ??_C@_1BE@MAFDNGED@?$AA_?$AAc?$AAh?$AAs?$AAi?$AAz?$AAe?$AA_?$AAs?$AA?$AA@ 1019e8e8     LIBCMTD:chsize.obj
 0003:00023900       ??_C@_1GA@DBKMEDOF@?$AAf?$AA?3?$AA?2?$AAd?$AAd?$AA?2?$AAv?$AAc?$AAt?$AAo?$AAo?$AAl?$AAs?$AA?2?$AAc?$AAr?$AAt?$AA_?$AAb?$AAl?$AAd?$AA?2?$AAs?$AAe?$AAl?$AAf?$AA_?$AAx?$AA8?$AA6?$AA?2?$AAc@ 1019e900     LIBCMTD:chsize.obj
 0003:00023960       ??_C@_1BC@JBGGJDCM@?$AA_?$AAs?$AAe?$AAt?$AAm?$AAo?$AAd?$AAe?$AA?$AA@ 1019e960     LIBCMTD:setmode.obj
 0003:00023978       ??_C@_1GC@KODPFLLJ@?$AAf?$AA?3?$AA?2?$AAd?$AAd?$AA?2?$AAv?$AAc?$AAt?$AAo?$AAo?$AAl?$AAs?$AA?2?$AAc?$AAr?$AAt?$AA_?$AAb?$AAl?$AAd?$AA?2?$AAs?$AAe?$AAl?$AAf?$AA_?$AAx?$AA8?$AA6?$AA?2?$AAc@ 1019e978     LIBCMTD:setmode.obj
 0003:000239e0       ??_C@_1OA@HGPJIFPM@?$AA?$CI?$AA?$CI?$AAm?$AAo?$AAd?$AAe?$AA?5?$AA?$DN?$AA?$DN?$AA?5?$AA_?$AAO?$AA_?$AAT?$AAE?$AAX?$AAT?$AA?$CJ?$AA?5?$AA?$HM?$AA?$HM?$AA?5?$AA?$CI?$AAm?$AAo?$AAd?$AAe?$AA?5?$AA?$DN?$AA?$DN?$AA?5?$AA_@ 1019e9e0     LIBCMTD:setmode.obj
 0003:00023ac0       ??_C@_1BG@IEEHLOCL@?$AA_?$AAs?$AAe?$AAt?$AA_?$AAf?$AAm?$AAo?$AAd?$AAe?$AA?$AA@ 1019eac0     LIBCMTD:setmode.obj
 0003:00023ad8       ??_C@_1IC@NDCJMLB@?$AA?$CI?$AA?$CI?$AAm?$AAo?$AAd?$AAe?$AA?5?$AA?$DN?$AA?$DN?$AA?5?$AA_?$AAO?$AA_?$AAT?$AAE?$AAX?$AAT?$AA?$CJ?$AA?5?$AA?$HM?$AA?$HM?$AA?5?$AA?$CI?$AAm?$AAo?$AAd?$AAe?$AA?5?$AA?$DN?$AA?$DN?$AA?5?$AA_@ 1019ead8     LIBCMTD:setmode.obj
 0003:00023b5c       ??_C@_1BG@CKGMPOFH@?$AA_?$AAg?$AAe?$AAt?$AA_?$AAf?$AAm?$AAo?$AAd?$AAe?$AA?$AA@ 1019eb5c     LIBCMTD:setmode.obj
 0003:00023b74       ??_C@_1CA@GPIGPPFN@?$AA?$CI?$AAp?$AAM?$AAo?$AAd?$AAe?$AA?5?$AA?$CB?$AA?$DN?$AA?5?$AAN?$AAU?$AAL?$AAL?$AA?$CJ?$AA?$AA@ 1019eb74     LIBCMTD:setmode.obj
 0003:00023b94       ??_C@_06GDENEHCP@CONIN$?$AA@ 1019eb94     LIBCMTD:initcon.obj
 0003:00023b9c       ??_C@_07GPDNMNG@CONOUT$?$AA@ 1019eb9c     LIBCMTD:initcon.obj
 0003:00023ba8       ??_C@_1FA@HILOOCMA@?$AA?$CI?$AA_?$AAt?$AAc?$AAs?$AAn?$AAl?$AAe?$AAn?$AA?$CI?$AAo?$AAp?$AAt?$AAi?$AAo?$AAn?$AA?0?$AA?5?$AA_?$AAM?$AAA?$AAX?$AA_?$AAE?$AAN?$AAV?$AA?$CJ?$AA?5?$AA?$DM?$AA?5?$AA_?$AAM@ 1019eba8     LIBCMTD:getenv.obj
 0003:00023bf8       ??_C@_1O@GMKGKCJO@?$AAg?$AAe?$AAt?$AAe?$AAn?$AAv?$AA?$AA@ 1019ebf8     LIBCMTD:getenv.obj
 0003:00023c08       ??_C@_1GA@IPPICGKB@?$AAf?$AA?3?$AA?2?$AAd?$AAd?$AA?2?$AAv?$AAc?$AAt?$AAo?$AAo?$AAl?$AAs?$AA?2?$AAc?$AAr?$AAt?$AA_?$AAb?$AAl?$AAd?$AA?2?$AAs?$AAe?$AAl?$AAf?$AA_?$AAx?$AA8?$AA6?$AA?2?$AAc@ 1019ec08     LIBCMTD:getenv.obj
 0003:00023c68       ??_C@_1CC@FKAOHHLO@?$AA?$CI?$AAo?$AAp?$AAt?$AAi?$AAo?$AAn?$AA?5?$AA?$CB?$AA?$DN?$AA?5?$AAN?$AAU?$AAL?$AAL?$AA?$CJ?$AA?$AA@ 1019ec68     LIBCMTD:getenv.obj
 0003:00023c90       ??_C@_1GI@JBIFPFJH@?$AA_?$AAt?$AAc?$AAs?$AAn?$AAl?$AAe?$AAn?$AA?$CI?$AA?$CK?$AAs?$AAe?$AAa?$AAr?$AAc?$AAh?$AA?5?$AA?$CL?$AA?5?$AAl?$AAe?$AAn?$AAg?$AAt?$AAh?$AA?5?$AA?$CL?$AA?5?$AA1?$AA?0?$AA?5?$AA_@ 1019ec90     LIBCMTD:getenv.obj
 0003:00023cf8       ??_C@_1EI@HHOBPCFK@?$AAs?$AAt?$AAr?$AAc?$AAp?$AAy?$AA_?$AAs?$AA?$CI?$AAb?$AAu?$AAf?$AAf?$AAe?$AAr?$AA?0?$AA?5?$AAs?$AAi?$AAz?$AAe?$AAI?$AAn?$AAT?$AAC?$AAh?$AAa?$AAr?$AAs?$AA?0?$AA?5?$AAs@ 1019ecf8     LIBCMTD:getenv.obj
 0003:00023d40       ??_C@_1JM@NLPGJJPH@?$AA?$CI?$AAb?$AAu?$AAf?$AAf?$AAe?$AAr?$AA?5?$AA?$CB?$AA?$DN?$AA?5?$AAN?$AAU?$AAL?$AAL?$AA?5?$AA?$CG?$AA?$CG?$AA?5?$AAs?$AAi?$AAz?$AAe?$AAI?$AAn?$AAT?$AAC?$AAh?$AAa?$AAr?$AAs?$AA?5@ 1019ed40     LIBCMTD:getenv.obj
 0003:00023ddc       ??_C@_1CC@BAJKDIIF@?$AA_?$AAg?$AAe?$AAt?$AAe?$AAn?$AAv?$AA_?$AAs?$AA_?$AAh?$AAe?$AAl?$AAp?$AAe?$AAr?$AA?$AA@ 1019eddc     LIBCMTD:getenv.obj
 0003:00023e00       ??_C@_1CK@PIKDAOCL@?$AAp?$AAR?$AAe?$AAt?$AAu?$AAr?$AAn?$AAV?$AAa?$AAl?$AAu?$AAe?$AA?5?$AA?$CB?$AA?$DN?$AA?5?$AAN?$AAU?$AAL?$AAL?$AA?$AA@ 1019ee00     LIBCMTD:getenv.obj
 0003:00023e2c       ??_C@_1DM@GNKNEGJO@?$AAs?$AAt?$AAr?$AAc?$AAp?$AAy?$AA_?$AAs?$AA?$CI?$AA?$CK?$AAp?$AAB?$AAu?$AAf?$AAf?$AAe?$AAr?$AA?0?$AA?5?$AAs?$AAi?$AAz?$AAe?$AA?0?$AA?5?$AAs?$AAt?$AAr?$AA?$CJ?$AA?$AA@ 1019ee2c     LIBCMTD:getenv.obj
 0003:00023e68       ??_C@_1CA@GDBKELOE@?$AAv?$AAa?$AAr?$AAn?$AAa?$AAm?$AAe?$AA?5?$AA?$CB?$AA?$DN?$AA?5?$AAN?$AAU?$AAL?$AAL?$AA?$AA@ 1019ee68     LIBCMTD:getenv.obj
 0003:00023e88       ??_C@_1CC@KPLOPIEM@?$AA_?$AAd?$AAu?$AAp?$AAe?$AAn?$AAv?$AA_?$AAs?$AA_?$AAh?$AAe?$AAl?$AAp?$AAe?$AAr?$AA?$AA@ 1019ee88     LIBCMTD:getenv.obj
 0003:00023eac       ??_C@_1CA@FHNFMDOJ@?$AAp?$AAB?$AAu?$AAf?$AAf?$AAe?$AAr?$AA?5?$AA?$CB?$AA?$DN?$AA?5?$AAN?$AAU?$AAL?$AAL?$AA?$AA@ 1019eeac     LIBCMTD:getenv.obj
 0003:00023ecc       ??_C@_1BA@PCFLFGNC@?$AAw?$AAc?$AAs?$AAt?$AAo?$AAx?$AAl?$AA?$AA@ 1019eecc     LIBCMTD:wcstol.obj
 0003:00023ee0       ??_C@_1GA@CADFOND@?$AAf?$AA?3?$AA?2?$AAd?$AAd?$AA?2?$AAv?$AAc?$AAt?$AAo?$AAo?$AAl?$AAs?$AA?2?$AAc?$AAr?$AAt?$AA_?$AAb?$AAl?$AAd?$AA?2?$AAs?$AAe?$AAl?$AAf?$AA_?$AAx?$AA8?$AA6?$AA?2?$AAc@ 1019eee0     LIBCMTD:wcstol.obj
 0003:00023f40       ??_C@_1BK@CMPKHPEC@?$AAn?$AA?5?$AA?$DM?$AA?$DN?$AA?5?$AAI?$AAN?$AAT?$AA_?$AAM?$AAA?$AAX?$AA?$AA@ 1019ef40     LIBCMTD:mbsnbico.obj
 0003:00023f5c       ??_C@_1BM@FKNNDAHH@?$AA_?$AAm?$AAb?$AAs?$AAn?$AAb?$AAi?$AAc?$AAo?$AAl?$AAl?$AA_?$AAl?$AA?$AA@ 1019ef5c     LIBCMTD:mbsnbico.obj
 0003:00023f78       ??_C@_1GE@NJHAJPKI@?$AAf?$AA?3?$AA?2?$AAd?$AAd?$AA?2?$AAv?$AAc?$AAt?$AAo?$AAo?$AAl?$AAs?$AA?2?$AAc?$AAr?$AAt?$AA_?$AAb?$AAl?$AAd?$AA?2?$AAs?$AAe?$AAl?$AAf?$AA_?$AAx?$AA8?$AA6?$AA?2?$AAc@ 1019ef78     LIBCMTD:mbsnbico.obj
 0003:00023fdc       ??_C@_0DC@CAFDLBC@f?3?2dd?2vctools?2crt_bld?2self_x86?2c@ 1019efdc     LIBCMTD:wtombenv.obj
 0003:00024010       ??_C@_1FO@IFEMNBMO@?$AAf?$AA?3?$AA?2?$AAd?$AAd?$AA?2?$AAv?$AAc?$AAt?$AAo?$AAo?$AAl?$AAs?$AA?2?$AAc?$AAr?$AAt?$AA_?$AAb?$AAl?$AAd?$AA?2?$AAs?$AAe?$AAl?$AAf?$AA_?$AAx?$AA8?$AA6?$AA?2?$AAc@ 1019f010     LIBCMTD:a_cmp.obj
 0003:00024070       ??_C@_1HK@ELDMAMK@?$AAc?$AAc?$AAh?$AAC?$AAo?$AAu?$AAn?$AAt?$AA1?$AA?$DN?$AA?$DN?$AA0?$AA?5?$AA?$CG?$AA?$CG?$AA?5?$AAc?$AAc?$AAh?$AAC?$AAo?$AAu?$AAn?$AAt?$AA2?$AA?$DN?$AA?$DN?$AA1?$AA?5?$AA?$HM?$AA?$HM?$AA?5@ 1019f070     LIBCMTD:a_cmp.obj
 0003:000240ec       ??_C@_1CC@CNADELFK@?$AA_?$AAs?$AAt?$AAr?$AAi?$AAn?$AAg?$AA2?$AA?5?$AA?$CB?$AA?$DN?$AA?5?$AAN?$AAU?$AAL?$AAL?$AA?$AA@ 1019f0ec     LIBCMTD:strnicol.obj
 0003:00024110       ??_C@_1BK@IOJEBPLP@?$AA_?$AAs?$AAt?$AAr?$AAn?$AAi?$AAc?$AAo?$AAl?$AAl?$AA_?$AAl?$AA?$AA@ 1019f110     LIBCMTD:strnicol.obj
 0003:00024130       ??_C@_1GE@BDOBNJJ@?$AAf?$AA?3?$AA?2?$AAd?$AAd?$AA?2?$AAv?$AAc?$AAt?$AAo?$AAo?$AAl?$AAs?$AA?2?$AAc?$AAr?$AAt?$AA_?$AAb?$AAl?$AAd?$AA?2?$AAs?$AAe?$AAl?$AAf?$AA_?$AAx?$AA8?$AA6?$AA?2?$AAc@ 1019f130     LIBCMTD:strnicol.obj
 0003:00024194       ??_C@_1CC@ICKKAGJA@?$AA_?$AAs?$AAt?$AAr?$AAi?$AAn?$AAg?$AA1?$AA?5?$AA?$CB?$AA?$DN?$AA?5?$AAN?$AAU?$AAL?$AAL?$AA?$AA@ 1019f194     LIBCMTD:strnicol.obj
 0003:000241b8       ??_C@_1FG@OKIAKKPK@?$AAs?$AAt?$AAr?$AAc?$AAp?$AAy?$AA_?$AAs?$AA?$CI?$AAn?$AAa?$AAm?$AAe?$AA?0?$AA?5?$AAs?$AAt?$AAr?$AAl?$AAe?$AAn?$AA?$CI?$AAo?$AAp?$AAt?$AAi?$AAo?$AAn?$AA?$CJ?$AA?5?$AA?$CL?$AA?5@ 1019f1b8     LIBCMTD:setenv.obj
 0003:00024210       ??_C@_1EI@GHDNAPMG@?$AA?$CI?$AA?$CC?$AAC?$AAR?$AAT?$AA?5?$AAL?$AAo?$AAg?$AAi?$AAc?$AA?5?$AAe?$AAr?$AAr?$AAo?$AAr?$AA?5?$AAd?$AAu?$AAr?$AAi?$AAn?$AAg?$AA?5?$AAs?$AAe?$AAt?$AAe?$AAn?$AAv?$AA?$CC@ 1019f210     LIBCMTD:setenv.obj
 0003:00024258       ??_C@_0DA@NHJGCDK@f?3?2dd?2vctools?2crt_bld?2self_x86?2c@ 1019f258     LIBCMTD:setenv.obj
 0003:00024288       ??_C@_1FC@EEJIEIDF@?$AA_?$AAt?$AAc?$AAs?$AAn?$AAl?$AAe?$AAn?$AA?$CI?$AAe?$AAq?$AAu?$AAa?$AAl?$AA?5?$AA?$CL?$AA?5?$AA1?$AA?0?$AA?5?$AA_?$AAM?$AAA?$AAX?$AA_?$AAE?$AAN?$AAV?$AA?$CJ?$AA?5?$AA?$DM?$AA?5@ 1019f288     LIBCMTD:setenv.obj
 0003:000242dc       ??_C@_1DE@EEHFNNGH@?$AAe?$AAq?$AAu?$AAa?$AAl?$AA?5?$AA?9?$AA?5?$AAo?$AAp?$AAt?$AAi?$AAo?$AAn?$AA?5?$AA?$DM?$AA?5?$AA_?$AAM?$AAA?$AAX?$AA_?$AAE?$AAN?$AAV?$AA?$AA@ 1019f2dc     LIBCMTD:setenv.obj
 0003:00024310       ??_C@_1BI@CDAFOAAL@?$AA_?$AA_?$AAc?$AAr?$AAt?$AAs?$AAe?$AAt?$AAe?$AAn?$AAv?$AA?$AA@ 1019f310     LIBCMTD:setenv.obj
 0003:00024328       ??_C@_1GA@KKPDKNLP@?$AAf?$AA?3?$AA?2?$AAd?$AAd?$AA?2?$AAv?$AAc?$AAt?$AAo?$AAo?$AAl?$AAs?$AA?2?$AAc?$AAr?$AAt?$AA_?$AAb?$AAl?$AAd?$AA?2?$AAs?$AAe?$AAl?$AAf?$AA_?$AAx?$AA8?$AA6?$AA?2?$AAc@ 1019f328     LIBCMTD:setenv.obj
 0003:00024388       ??_C@_1CA@LMBEKBDN@?$AAp?$AAo?$AAp?$AAt?$AAi?$AAo?$AAn?$AA?5?$AA?$CB?$AA?$DN?$AA?5?$AAN?$AAU?$AAL?$AAL?$AA?$AA@ 1019f388     LIBCMTD:setenv.obj
 0003:000243a8       ??_C@_1FK@DNFLNPD@?$AAs?$AAt?$AAr?$AAc?$AAp?$AAy?$AA_?$AAs?$AA?$CI?$AA?$CK?$AAn?$AAe?$AAw?$AAe?$AAn?$AAv?$AAp?$AAt?$AAr?$AA?0?$AA?5?$AAe?$AAn?$AAv?$AAp?$AAt?$AAr?$AAS?$AAi?$AAz?$AAe?$AA?0@ 1019f3a8     LIBCMTD:setenv.obj
 0003:00024404       ??_C@_1BK@ECKIJLPM@?$AAc?$AAo?$AAp?$AAy?$AA_?$AAe?$AAn?$AAv?$AAi?$AAr?$AAo?$AAn?$AA?$AA@ 1019f404     LIBCMTD:setenv.obj
 0003:00024420       ??_C@_1BE@JKKFLIKJ@?$AA_?$AAm?$AAb?$AAs?$AAc?$AAh?$AAr?$AA_?$AAl?$AA?$AA@ 1019f420     LIBCMTD:mbschr.obj
 0003:00024438       ??_C@_1GA@GDCAGKMG@?$AAf?$AA?3?$AA?2?$AAd?$AAd?$AA?2?$AAv?$AAc?$AAt?$AAo?$AAo?$AAl?$AAs?$AA?2?$AAc?$AAr?$AAt?$AA_?$AAb?$AAl?$AAd?$AA?2?$AAs?$AAe?$AAl?$AAf?$AA_?$AAx?$AA8?$AA6?$AA?2?$AAc@ 1019f438     LIBCMTD:mbschr.obj
 0003:000ebf14       ??_C@_04FGAJMCLA@?2?$CK?4?$CK?$AA@ 10266f14     wzFilePacker_static_d:wzFilePacker.obj
 0003:000ebf1c       ??_C@_01KICIPPFI@?2?$AA@   10266f1c     wzFilePacker_static_d:wzFilePacker.obj
 0003:000ebf20       ??_C@_05BMGBEOOC@?$CFs?2?$CFs?$AA@ 10266f20     wzFilePacker_static_d:wzFilePacker.obj
 0003:000ebf28       ??_C@_05LCOLKLHA@?$CK?4wpk?$AA@ 10266f28     wzFilePacker_static_d:wzFilePacker.obj
 0003:000ebf30       ??_C@_02GMLFBBN@wb?$AA@    10266f30     wzFilePacker_static_d:wzFilePacker.obj
 0003:000ebf34       ??_C@_03EMIMMIHL@?$CK?4?$CK?$AA@ 10266f34     wzFilePacker_static_d:wzFilePacker.obj
 0003:000ebf38       ??_C@_1IC@MEADOCIB@?$AAc?$AA?3?$AA?2?$AAp?$AAr?$AAo?$AAg?$AAr?$AAa?$AAm?$AA?5?$AAf?$AAi?$AAl?$AAe?$AAs?$AA?2?$AAm?$AAi?$AAc?$AAr?$AAo?$AAs?$AAo?$AAf?$AAt?$AA?5?$AAv?$AAi?$AAs?$AAu?$AAa@ 10266f38     wzFilePacker_static_d:wzFilePacker.obj
 0003:000ebfd4       ??_C@_03HMFOOINA@r?$CLb?$AA@ 10266fd4     wzFilePacker_static_d:wzFilePacker.obj
 0003:000ebfd8       ??_C@_1IA@LLBMBDOH@?$AAc?$AA?3?$AA?2?$AAp?$AAr?$AAo?$AAg?$AAr?$AAa?$AAm?$AA?5?$AAf?$AAi?$AAl?$AAe?$AAs?$AA?2?$AAm?$AAi?$AAc?$AAr?$AAo?$AAs?$AAo?$AAf?$AAt?$AA?5?$AAv?$AAi?$AAs?$AAu?$AAa@ 10266fd8     wzFilePacker_static_d:wzFilePacker.obj
 0003:000ec074       ??_C@_0DP@DDGDHHOD@c?3?2program?5files?2microsoft?5visua@ 10267074     wzFilePacker_static_d:wzFilePacker.obj
 0003:000ec0c0       ??_C@_1HO@CONDIOEO@?$AAc?$AA?3?$AA?2?$AAp?$AAr?$AAo?$AAg?$AAr?$AAa?$AAm?$AA?5?$AAf?$AAi?$AAl?$AAe?$AAs?$AA?2?$AAm?$AAi?$AAc?$AAr?$AAo?$AAs?$AAo?$AAf?$AAt?$AA?5?$AAv?$AAi?$AAs?$AAu?$AAa@ 102670c0     wzFilePacker_static_d:wzFilePacker.obj
 0003:000ec158       ??_C@_1HO@FAAIACEF@?$AAc?$AA?3?$AA?2?$AAp?$AAr?$AAo?$AAg?$AAr?$AAa?$AAm?$AA?5?$AAf?$AAi?$AAl?$AAe?$AAs?$AA?2?$AAm?$AAi?$AAc?$AAr?$AAo?$AAs?$AAo?$AAf?$AAt?$AA?5?$AAv?$AAi?$AAs?$AAu?$AAa@ 10267158     wzFilePacker_static_d:wzFilePacker.obj
 0003:000ec474       ??_C@_19BIEPDBPA@?$AAT?$AAy?$AAp?$AAe?$AA?$AA@ 10267474     wzFilePacker_static_d:vfile.obj
 0003:000ec480       ??_C@_19GJPGFMAH@?$AAA?$AAP?$AAI?$AAs?$AA?$AA@ 10267480     wzFilePacker_static_d:vfile.obj
 0003:000ec490       ??_C@_1IO@BKKINILL@?$AAd?$AA?3?$AA?2?$AAs?$AAu?$AAn?$AAe?$AAn?$AAg?$AAi?$AAn?$AAe?$AA?2?$AAp?$AAu?$AAb?$AAl?$AAi?$AAc?$AA?2?$AAw?$AAz?$AAf?$AAi?$AAl?$AAe?$AAp?$AAa?$AAc?$AAk?$AAe?$AAr@ 10267490     wzFilePacker_static_d:vfile.obj
 0003:000ec540       ??_C@_0EH@HGEJNNNJ@d?3?2sunengine?2public?2wzfilepacker@ 10267540     wzFilePacker_static_d:vfile.obj
 0003:000ec598       ??_C@_19DINFBLAK@?$AAN?$AAa?$AAm?$AAe?$AA?$AA@ 10267598     wzFilePacker_static_d:vfile.obj
 0003:000ec5a4       ??_C@_1BM@PGGFJAOG@?$AA?$CB?$AA?$CC?$AAC?$AAa?$AAn?$AA?8?$AAt?$AA?5?$AAf?$AAa?$AAi?$AAl?$AA?$CC?$AA?$AA@ 102675a4     wzFilePacker_static_d:vfile.obj
 0003:000ec5c8       ??_C@_0L@IGMIFIEL@Can?8t?5fail?$AA@ 102675c8     wzFilePacker_static_d:vfile.obj
 0003:000ec5d8       ??_C@_1BA@GLFNEBDB@?$AAC?$AAo?$AAn?$AAt?$AAe?$AAx?$AAt?$AA?$AA@ 102675d8     wzFilePacker_static_d:vfile.obj
 0003:000ec5ec       ??_C@_15EOIEBHGB@?$AAF?$AAS?$AA?$AA@ 102675ec     wzFilePacker_static_d:vfile.obj
 0003:000ec5f4       ??_C@_1CK@EAOENIFE@?$AAS?$AAe?$AAa?$AAr?$AAc?$AAh?$AAL?$AAi?$AAs?$AAt?$AA?9?$AA?$DO?$AAF?$AAS?$AA?5?$AA?$DN?$AA?$DN?$AA?5?$AAF?$AAS?$AA?$AA@ 102675f4     wzFilePacker_static_d:vfile.obj
 0003:000ec628       ??_C@_1BG@KFONOGAO@?$AAS?$AAe?$AAa?$AAr?$AAc?$AAh?$AAL?$AAi?$AAs?$AAt?$AA?$AA@ 10267628     wzFilePacker_static_d:vfile.obj
 0003:000ec644       ??_C@_19DDLLJDOO@?$AAF?$AAi?$AAl?$AAe?$AA?$AA@ 10267644     wzFilePacker_static_d:vfile.obj
 0003:000ec650       ??_C@_17KFBHKBIP@?$AAF?$AAS?$AA2?$AA?$AA@ 10267650     wzFilePacker_static_d:vfile.obj
 0003:000ec65c       ??_C@_17LHKCAOGB@?$AAF?$AAS?$AA1?$AA?$AA@ 1026765c     wzFilePacker_static_d:vfile.obj
 0003:000ec668       ??_C@_1BC@FOGJKDBH@?$AA?$CB?$AAN?$AAe?$AAw?$AAL?$AAi?$AAs?$AAt?$AA?$AA@ 10267668     wzFilePacker_static_d:vfile.obj
 0003:000ec680       ??_C@_1BC@PKFGPGJB@?$AAF?$AAi?$AAl?$AAe?$AAN?$AAa?$AAm?$AAe?$AA?$AA@ 10267680     wzFilePacker_static_d:vfile.obj
 0003:000ec698       ??_C@_1BA@GBLELBEH@?$AAN?$AAe?$AAw?$AAN?$AAa?$AAm?$AAe?$AA?$AA@ 10267698     wzFilePacker_static_d:vfile.obj
 0003:000ec6ac       ??_C@_19KCGKJLHI@?$AAB?$AAu?$AAf?$AAf?$AA?$AA@ 102676ac     wzFilePacker_static_d:vfile.obj
 0003:000ec6b8       ??_C@_1O@FDFOMCPN@?$AAF?$AAo?$AAr?$AAm?$AAa?$AAt?$AA?$AA@ 102676b8     wzFilePacker_static_d:vfile.obj
 0003:000ec6c8       ??_C@_1BC@FBCPBAMN@?$AAF?$AAi?$AAl?$AAe?$AAS?$AAp?$AAe?$AAc?$AA?$AA@ 102676c8     wzFilePacker_static_d:vfile.obj
 0003:000ec6e0       ??_C@_1BG@MGGDIOJP@?$AAF?$AAi?$AAl?$AAe?$AAS?$AAy?$AAs?$AAt?$AAe?$AAm?$AA?$AA@ 102676e0     wzFilePacker_static_d:vfile.obj
 0003:000ec6fc       ??_C@_1BK@GBENGJBD@?$AAF?$AAi?$AAn?$AAd?$AAe?$AAr?$AA?9?$AA?$DO?$AAA?$AAP?$AAI?$AAs?$AA?$AA@ 102676fc     wzFilePacker_static_d:vfile.obj
 0003:000ec71c       ??_C@_1O@CAEEAAJK@?$AAF?$AAi?$AAn?$AAd?$AAe?$AAr?$AA?$AA@ 1026771c     wzFilePacker_static_d:vfile.obj
 0003:000ec72c       ??_C@_1BK@IMPHHKND@?$AAF?$AAi?$AAn?$AAd?$AAe?$AAr?$AA?9?$AA?$DO?$AAD?$AAa?$AAt?$AAa?$AA?$AA@ 1026772c     wzFilePacker_static_d:vfile.obj
 0003:000ec9d4       ??_C@_02DJGKEECL@?4?4?$AA@ 102679d4     wzFilePacker_static_d:vFile_util.obj
 0003:000ec9d8       ??_C@_0L@IMPLNOCC@?2wz_sound?2?$AA@ 102679d8     wzFilePacker_static_d:vFile_util.obj
 0003:000ecc78       ??_C@_0EF@HMECDIBN@d?3?2sunengine?2public?2wzfilepacker@ 10267c78     wzFilePacker_static_d:Ram.obj
 0003:000eccd0       ??_C@_1IK@HKJMDEGJ@?$AA?$CI?$AAg?$AAe?$AAR?$AAa?$AAm?$AA_?$AAC?$AAu?$AAr?$AAr?$AAe?$AAn?$AAt?$AAl?$AAy?$AAU?$AAs?$AAe?$AAd?$AA?5?$AA?$DO?$AA?$DN?$AA?5?$AA0?$AA?$CJ?$AA?5?$AA?$CG?$AA?$CG?$AA?5?$AA?$CC?$AAf@ 10267cd0     wzFilePacker_static_d:Ram.obj
 0003:000ecd78       ??_C@_1JG@KFPGBALC@?$AA?$CI?$AAg?$AAe?$AAR?$AAa?$AAm?$AA_?$AAN?$AAu?$AAm?$AAb?$AAe?$AAr?$AAO?$AAf?$AAA?$AAl?$AAl?$AAo?$AAc?$AAa?$AAt?$AAi?$AAo?$AAn?$AAs?$AA?5?$AA?$DO?$AA?$DN?$AA?5?$AA0?$AA?$CJ@ 10267d78     wzFilePacker_static_d:Ram.obj
 0003:000ece30       ??_C@_1IK@CNNBLEID@?$AAd?$AA?3?$AA?2?$AAs?$AAu?$AAn?$AAe?$AAn?$AAg?$AAi?$AAn?$AAe?$AA?2?$AAp?$AAu?$AAb?$AAl?$AAi?$AAc?$AA?2?$AAw?$AAz?$AAf?$AAi?$AAl?$AAe?$AAp?$AAa?$AAc?$AAk?$AAe?$AAr@ 10267e30     wzFilePacker_static_d:Ram.obj
 0003:000eced8       ??_C@_0CF@OFBKHJLE@free?$CI?$CJd?5more?5ram?5than?5you?5alloca@ 10267ed8     wzFilePacker_static_d:Ram.obj
 0003:000ecf08       ??_C@_1HC@KPONICKC@?$AA0?$AA?5?$AA?$CG?$AA?$CG?$AA?5?$AA?$CC?$AAr?$AAa?$AAm?$AA_?$AAv?$AAe?$AAr?$AAi?$AAf?$AAy?$AA_?$AAb?$AAl?$AAo?$AAc?$AAk?$AA?3?$AA?5?$AA?5?$AAM?$AAe?$AAm?$AAo?$AAr?$AAy?$AA?5@ 10267f08     wzFilePacker_static_d:Ram.obj
 0003:000ecf90       ??_C@_1HE@PMAKKPCC@?$AA0?$AA?5?$AA?$CG?$AA?$CG?$AA?5?$AA?$CC?$AAr?$AAa?$AAm?$AA_?$AAv?$AAe?$AAr?$AAi?$AAf?$AAy?$AA_?$AAb?$AAl?$AAo?$AAc?$AAk?$AA?3?$AA?5?$AA?5?$AAM?$AAe?$AAm?$AAo?$AAr?$AAy?$AA?5@ 10267f90     wzFilePacker_static_d:Ram.obj
 0003:000ed01c       ??_C@_1CI@LKMCKOAH@?$AA0?$AA?5?$AA?$CG?$AA?$CG?$AA?5?$AA?$CC?$AAf?$AAr?$AAe?$AAe?$AAi?$AAn?$AAg?$AA?5?$AAN?$AAU?$AAL?$AAL?$AA?$CC?$AA?$AA@ 1026801c     wzFilePacker_static_d:Ram.obj
 0003:000ed2d8       ??_C@_0EH@PCFGPPDH@d?3?2sunengine?2public?2wzfilepacker@ 102682d8     wzFilePacker_static_d:fsvfs.obj
 0003:000ed330       ??_C@_1EK@CJFFBGHJ@?$AAF?$AAi?$AAl?$AAe?$AA?9?$AA?$DO?$AAS?$AAi?$AAg?$AAn?$AAa?$AAt?$AAu?$AAr?$AAe?$AA?5?$AA?$DN?$AA?$DN?$AA?5?$AAV?$AAF?$AAS?$AAF?$AAI?$AAL?$AAE?$AA_?$AAS?$AAI?$AAG?$AAN?$AAA@ 10268330     wzFilePacker_static_d:fsvfs.obj
 0003:000ed388       ??_C@_1CC@KEKGLOCK@?$AAF?$AAi?$AAl?$AAe?$AAS?$AAp?$AAe?$AAc?$AA?5?$AA?$CB?$AA?$DN?$AA?5?$AAN?$AAU?$AAL?$AAL?$AA?$AA@ 10268388     wzFilePacker_static_d:fsvfs.obj
 0003:000ed3b0       ??_C@_1IO@MNOEGOMM@?$AAd?$AA?3?$AA?2?$AAs?$AAu?$AAn?$AAe?$AAn?$AAg?$AAi?$AAn?$AAe?$AA?2?$AAp?$AAu?$AAb?$AAl?$AAi?$AAc?$AA?2?$AAw?$AAz?$AAf?$AAi?$AAl?$AAe?$AAp?$AAa?$AAc?$AAk?$AAe?$AAr@ 102683b0     wzFilePacker_static_d:fsvfs.obj
 0003:000ed460       ??_C@_1FC@KDLLCPBF@?$AAF?$AAi?$AAn?$AAd?$AAe?$AAr?$AA?9?$AA?$DO?$AAS?$AAi?$AAg?$AAn?$AAa?$AAt?$AAu?$AAr?$AAe?$AA?5?$AA?$DN?$AA?$DN?$AA?5?$AAV?$AAF?$AAS?$AAF?$AAI?$AAN?$AAD?$AAE?$AAR?$AA_?$AAS@ 10268460     wzFilePacker_static_d:fsvfs.obj
 0003:000ed4c4       ??_C@_1BG@COALCEMK@?$AAP?$AAr?$AAo?$AAp?$AAe?$AAr?$AAt?$AAi?$AAe?$AAs?$AA?$AA@ 102684c4     wzFilePacker_static_d:fsvfs.obj
 0003:000ed4e0       ??_C@_1BO@NEHFBIGI@?$AAF?$AAi?$AAn?$AAd?$AAe?$AAr?$AA?9?$AA?$DO?$AAF?$AAi?$AAn?$AAd?$AAe?$AAr?$AA?$AA@ 102684e0     wzFilePacker_static_d:fsvfs.obj
 0003:000ed508       ??_C@_1FA@OBJEELMH@?$AA?$CB?$AA?$CI?$AAO?$AAp?$AAe?$AAn?$AAM?$AAo?$AAd?$AAe?$AAF?$AAl?$AAa?$AAg?$AAs?$AA?5?$AA?$CG?$AA?5?$AAG?$AAE?$AA_?$AAV?$AAF?$AAI?$AAL?$AAE?$AA_?$AAO?$AAP?$AAE?$AAN?$AA_@ 10268508     wzFilePacker_static_d:fsvfs.obj
 0003:000ed568       ??_C@_1FA@FECNGHMB@?$AAC?$AAo?$AAn?$AAt?$AAe?$AAx?$AAt?$AA?9?$AA?$DO?$AAS?$AAi?$AAg?$AAn?$AAa?$AAt?$AAu?$AAr?$AAe?$AA?5?$AA?$DN?$AA?$DN?$AA?5?$AAV?$AAF?$AAS?$AAF?$AAI?$AAL?$AAE?$AA_?$AAS?$AAI@ 10268568     wzFilePacker_static_d:fsvfs.obj
 0003:000ed5c8       ??_C@_1CG@FCALPGOK@?$AA?$CB?$AA?$CC?$AAN?$AAo?$AAt?$AA?5?$AAi?$AAm?$AAp?$AAl?$AAe?$AAm?$AAe?$AAn?$AAt?$AAe?$AAd?$AA?$CC?$AA?$AA@ 102685c8     wzFilePacker_static_d:fsvfs.obj
 0003:000ed5f8       ??_C@_0BA@IOJHHLDM@Not?5implemented?$AA@ 102685f8     wzFilePacker_static_d:fsvfs.obj
 0003:000ed60c       ??_C@_0BI@LCBABOGN@header?5is?5Final?5Version?$AA@ 1026860c     wzFilePacker_static_d:fsvfs.obj
 0003:000ed628       ??_C@_0P@FOHJAHFG@header?5invalid?$AA@ 10268628     wzFilePacker_static_d:fsvfs.obj
 0003:000ed63c       ??_C@_0DM@MLIJDPNB@Now?5Packing?5File?5Version?5?3?5?$CFd?0?5P@ 1026863c     wzFilePacker_static_d:fsvfs.obj
 0003:000ed684       ??_C@_1BK@IGGAEAHD@?$AAN?$AAa?$AAm?$AAe?$AA?5?$AA?$DN?$AA?$DN?$AA?5?$AAN?$AAU?$AAL?$AAL?$AA?$AA@ 10268684     wzFilePacker_static_d:fsvfs.obj
 0003:000ed6a4       ??_C@_1BM@CGOKOFOC@?$AAR?$AAW?$AAO?$AAp?$AAs?$AA?5?$AA?$CB?$AA?$DN?$AA?5?$AAN?$AAU?$AAL?$AAL?$AA?$AA@ 102686a4     wzFilePacker_static_d:fsvfs.obj
 0003:000ed6c8       ??_C@_1BK@LKGHADHJ@?$AAF?$AAi?$AAl?$AAe?$AA?9?$AA?$DO?$AAS?$AAy?$AAs?$AAt?$AAe?$AAm?$AA?$AA@ 102686c8     wzFilePacker_static_d:fsvfs.obj
 0003:000ed6e8       ??_C@_1CK@HCMIOBIP@?$AAF?$AAi?$AAl?$AAe?$AA?5?$AA?$DN?$AA?$DN?$AA?5?$AAF?$AAi?$AAl?$AAe?$AA?9?$AA?$DO?$AAS?$AAy?$AAs?$AAt?$AAe?$AAm?$AA?$AA@ 102686e8     wzFilePacker_static_d:fsvfs.obj
 0003:000ed720       ??_C@_1EI@PJPCOCGF@?$AAF?$AAi?$AAl?$AAe?$AA?9?$AA?$DO?$AAC?$AAu?$AAr?$AAr?$AAe?$AAn?$AAt?$AAR?$AAe?$AAl?$AAP?$AAo?$AAs?$AA?5?$AA?$DM?$AA?$DN?$AA?5?$AAF?$AAi?$AAl?$AAe?$AA?9?$AA?$DO?$AAL?$AAe?$AAn@ 10268720     wzFilePacker_static_d:fsvfs.obj
 0003:000ed778       ??_C@_1DC@JELMDHOG@?$AAF?$AAi?$AAl?$AAe?$AA?9?$AA?$DO?$AAC?$AAu?$AAr?$AAr?$AAe?$AAn?$AAt?$AAR?$AAe?$AAl?$AAP?$AAo?$AAs?$AA?5?$AA?$DO?$AA?$DN?$AA?5?$AA0?$AA?$AA@ 10268778     wzFilePacker_static_d:fsvfs.obj
 0003:000ed7b4       ??_C@_1BI@LEOHNLJN@?$AAM?$AAa?$AAx?$AAL?$AAe?$AAn?$AA?5?$AA?$CB?$AA?$DN?$AA?5?$AA0?$AA?$AA@ 102687b4     wzFilePacker_static_d:fsvfs.obj
 0003:000ed7d0       ??_C@_1CC@CFEECKHO@?$AA?$CB?$AAF?$AAi?$AAl?$AAe?$AA?9?$AA?$DO?$AAD?$AAi?$AAr?$AAe?$AAc?$AAt?$AAo?$AAr?$AAy?$AA?$AA@ 102687d0     wzFilePacker_static_d:fsvfs.obj
 0003:000ed7f8       ??_C@_1BI@KOMDKJPP@?$AAF?$AAi?$AAl?$AAe?$AA?9?$AA?$DO?$AAR?$AAW?$AAO?$AAp?$AAs?$AA?$AA@ 102687f8     wzFilePacker_static_d:fsvfs.obj
 0003:000ed814       ??_C@_0DA@JPDHOIDD@?$CK?$CK?$CK?$CK?$CK?$CK?$CK?$CK?$CK?$CK?$CK?$CK?$CK?$CK?$CK?$CK?5N2_UpdateFilePo@ 10268814     wzFilePacker_static_d:fsvfs.obj
 0003:000ed850       ??_C@_1BM@MAMEDNBJ@?$AAR?$AAW?$AAO?$AAp?$AAs?$AAP?$AAo?$AAs?$AA?5?$AA?$DO?$AA?$DN?$AA?5?$AA0?$AA?$AA@ 10268850     wzFilePacker_static_d:fsvfs.obj
 0003:000ed874       ??_C@_0CO@LGMGIONK@?$CK?$CK?$CK?$CK?$CK?$CK?$CK?$CK?$CK?$CK?$CK?$CK?$CK?$CK?$CK?$CK?5N2_SetFilePoint@ 10268874     wzFilePacker_static_d:fsvfs.obj
 0003:000ed8ac       ??_C@_0DF@IHAPMOPK@?$CL?$CL?$CL?$CL?$CL?$CL?$CL?$CL?$CL?$CL?5ReadFail_4_Error?5?3?5?G?O@ 102688ac     wzFilePacker_static_d:fsvfs.obj
 0003:000ed8ec       ??_C@_0DH@HABJGGNC@?$CL?$CL?$CL?$CL?$CL?$CL?$CL?$CL?$CL?$CL?5ReadFail_3_Error?5?3?5?$MA?P@ 102688ec     wzFilePacker_static_d:fsvfs.obj
 0003:000ed930       ??_C@_0DG@LCJJILDN@?$CL?$CL?$CL?$CL?$CL?$CL?$CL?$CL?$CL?$CL?5ReadFail_2_Error?5?3?5?$LP?$MA@ 10268930     wzFilePacker_static_d:fsvfs.obj
 0003:000ed970       ??_C@_0CG@GENKINJN@?$CL?$CL?$CL?$CL?$CL?$CL?$CL?$CL?$CL?$CL?5ReadFail_1_ErrorCode?5@ 10268970     wzFilePacker_static_d:fsvfs.obj
 0003:000ed9a0       ??_C@_1BG@GBAIPKFE@?$AAC?$AAo?$AAu?$AAn?$AAt?$AA?5?$AA?$CB?$AA?$DN?$AA?5?$AA0?$AA?$AA@ 102689a0     wzFilePacker_static_d:fsvfs.obj
 0003:000ed9bc       ??_C@_1CK@BIPDICJ@?$AA?$CB?$AA?$CC?$AAI?$AAl?$AAl?$AAe?$AAg?$AAa?$AAl?$AA?5?$AAs?$AAe?$AAe?$AAk?$AA?5?$AAc?$AAa?$AAs?$AAe?$AA?$CC?$AA?$AA@ 102689bc     wzFilePacker_static_d:fsvfs.obj
 0003:000ed9f0       ??_C@_0BC@EMFFNHLN@Illegal?5seek?5case?$AA@ 102689f0     wzFilePacker_static_d:fsvfs.obj
 0003:000eda08       ??_C@_1BO@OFJJJHGJ@?$AAF?$AAi?$AAl?$AAe?$AA?9?$AA?$DO?$AAD?$AAi?$AAr?$AAE?$AAn?$AAt?$AAr?$AAy?$AA?$AA@ 10268a08     wzFilePacker_static_d:fsvfs.obj
 0003:000eda2c       ??_C@_0BH@MMBDGEON@Remove?5Fsvfs?5Tree?5Fail?$AA@ 10268a2c     wzFilePacker_static_d:fsvfs.obj
 0003:000eda48       ??_C@_0BK@PKGCLKLI@Remove?5Fsvfs?5Tree?5SUCCESS?$AA@ 10268a48     wzFilePacker_static_d:fsvfs.obj
 0003:000eda68       ??_C@_0BM@OPDJPMGP@Not?5File?5SameName?5Tree?9Node?$AA@ 10268a68     wzFilePacker_static_d:fsvfs.obj
 0003:000edd14       ??_C@_1BA@IDEFMFHE@?$AA?$CB?$AAH?$AAa?$AAn?$AAd?$AAl?$AAe?$AA?$AA@ 10268d14     wzFilePacker_static_d:FSMEMORY.obj
 0003:000edd28       ??_C@_1JE@BDFHJBKO@?$AAd?$AA?3?$AA?2?$AAs?$AAu?$AAn?$AAe?$AAn?$AAg?$AAi?$AAn?$AAe?$AA?2?$AAp?$AAu?$AAb?$AAl?$AAi?$AAc?$AA?2?$AAw?$AAz?$AAf?$AAi?$AAl?$AAe?$AAp?$AAa?$AAc?$AAk?$AAe?$AAr@ 10268d28     wzFilePacker_static_d:FSMEMORY.obj
 0003:000edde0       ??_C@_0EK@FEEDBNOL@d?3?2sunengine?2public?2wzfilepacker@ 10268de0     wzFilePacker_static_d:FSMEMORY.obj
 0003:000ede38       ??_C@_1FA@GECHDMDP@?$AAF?$AAi?$AAl?$AAe?$AA?9?$AA?$DO?$AAS?$AAi?$AAg?$AAn?$AAa?$AAt?$AAu?$AAr?$AAe?$AA?5?$AA?$DN?$AA?$DN?$AA?5?$AAM?$AAE?$AAM?$AAO?$AAR?$AAY?$AAF?$AAI?$AAL?$AAE?$AA_?$AAS?$AAI@ 10268e38     wzFilePacker_static_d:FSMEMORY.obj
 0003:000ede98       ??_C@_1EE@KCGPABBO@?$AAF?$AAi?$AAl?$AAe?$AA?9?$AA?$DO?$AAS?$AAi?$AAz?$AAe?$AA?5?$AA?$DM?$AA?$DN?$AA?5?$AAF?$AAi?$AAl?$AAe?$AA?9?$AA?$DO?$AAA?$AAl?$AAl?$AAo?$AAc?$AAa?$AAt?$AAe?$AAd?$AAS?$AAi?$AAz@ 10268e98     wzFilePacker_static_d:FSMEMORY.obj
 0003:000edeec       ??_C@_1DK@FPEDPJEN@?$AAF?$AAi?$AAl?$AAe?$AA?9?$AA?$DO?$AAP?$AAo?$AAs?$AAi?$AAt?$AAi?$AAo?$AAn?$AA?5?$AA?$DM?$AA?$DN?$AA?5?$AAF?$AAi?$AAl?$AAe?$AA?9?$AA?$DO?$AAS?$AAi?$AAz?$AAe?$AA?$AA@ 10268eec     wzFilePacker_static_d:FSMEMORY.obj
 0003:000edf38       ??_C@_1EM@HHFIOAPB@?$AAF?$AAi?$AAl?$AAe?$AA?9?$AA?$DO?$AAA?$AAl?$AAl?$AAo?$AAc?$AAa?$AAt?$AAe?$AAd?$AAS?$AAi?$AAz?$AAe?$AA?5?$AA?$DO?$AA?$DN?$AA?5?$AAF?$AAi?$AAl?$AAe?$AA?9?$AA?$DO?$AAP?$AAo?$AAs@ 10268f38     wzFilePacker_static_d:FSMEMORY.obj
 0003:000edf98       ??_C@_1EE@LHFODDMA@?$AAF?$AAi?$AAl?$AAe?$AA?9?$AA?$DO?$AAA?$AAl?$AAl?$AAo?$AAc?$AAa?$AAt?$AAe?$AAd?$AAS?$AAi?$AAz?$AAe?$AA?5?$AA?$DO?$AA?$DN?$AA?5?$AAF?$AAi?$AAl?$AAe?$AA?9?$AA?$DO?$AAS?$AAi?$AAz@ 10268f98     wzFilePacker_static_d:FSMEMORY.obj
 0003:000edfec       ??_C@_1DK@PENJNLK@?$AAF?$AAi?$AAl?$AAe?$AA?9?$AA?$DO?$AAW?$AAe?$AAO?$AAw?$AAn?$AAM?$AAe?$AAm?$AAo?$AAr?$AAy?$AA?5?$AA?$DN?$AA?$DN?$AA?5?$AAG?$AAE?$AA_?$AAT?$AAR?$AAU?$AAE?$AA?$AA@ 10268fec     wzFilePacker_static_d:FSMEMORY.obj
 0003:000ee034       ??_C@_1DG@MDKGLFJA@?$AAF?$AAi?$AAl?$AAe?$AA?9?$AA?$DO?$AAR?$AAe?$AAa?$AAd?$AAO?$AAn?$AAl?$AAy?$AA?5?$AA?$DN?$AA?$DN?$AA?5?$AAG?$AAE?$AA_?$AAF?$AAA?$AAL?$AAS?$AAE?$AA?$AA@ 10269034     wzFilePacker_static_d:FSMEMORY.obj
 0003:000ee078       ??_C@_1EM@DNHIKHKC@?$AAF?$AAi?$AAl?$AAe?$AA?9?$AA?$DO?$AAP?$AAo?$AAs?$AAi?$AAt?$AAi?$AAo?$AAn?$AA?5?$AA?$DM?$AA?$DN?$AA?5?$AAF?$AAi?$AAl?$AAe?$AA?9?$AA?$DO?$AAA?$AAl?$AAl?$AAo?$AAc?$AAa?$AAt?$AAe@ 10269078     wzFilePacker_static_d:FSMEMORY.obj
 0003:000ee0d4       ??_C@_1CK@HGBOKDDO@?$AA?$CB?$AA?$CC?$AAU?$AAn?$AAk?$AAn?$AAo?$AAw?$AAn?$AA?5?$AAs?$AAe?$AAe?$AAk?$AA?5?$AAk?$AAi?$AAn?$AAd?$AA?$CC?$AA?$AA@ 102690d4     wzFilePacker_static_d:FSMEMORY.obj
 0003:000ee108       ??_C@_0BC@LKJPKHAB@Unknown?5seek?5kind?$AA@ 10269108     wzFilePacker_static_d:FSMEMORY.obj
 0003:000ee3a8       ??_C@_0EH@LBFIDONG@d?3?2sunengine?2public?2wzfilepacker@ 102693a8     wzFilePacker_static_d:fsdos.obj
 0003:000ee400       ??_C@_1EK@OCGFAFIJ@?$AAF?$AAi?$AAl?$AAe?$AA?9?$AA?$DO?$AAS?$AAi?$AAg?$AAn?$AAa?$AAt?$AAu?$AAr?$AAe?$AA?5?$AA?$DN?$AA?$DN?$AA?5?$AAD?$AAO?$AAS?$AAF?$AAI?$AAL?$AAE?$AA_?$AAS?$AAI?$AAG?$AAN?$AAA@ 10269400     wzFilePacker_static_d:fsdos.obj
 0003:000ee458       ??_C@_1IO@NBNCDGGF@?$AAd?$AA?3?$AA?2?$AAs?$AAu?$AAn?$AAe?$AAn?$AAg?$AAi?$AAn?$AAe?$AA?2?$AAp?$AAu?$AAb?$AAl?$AAi?$AAc?$AA?2?$AAw?$AAz?$AAf?$AAi?$AAl?$AAe?$AAp?$AAa?$AAc?$AAk?$AAe?$AAr@ 10269458     wzFilePacker_static_d:fsdos.obj
 0003:000ee504       ??_C@_02CEGDFPFP@?4?2?$AA@ 10269504     wzFilePacker_static_d:fsdos.obj
 0003:000ee508       ??_C@_1BO@PFGEMHBK@?$AAF?$AAi?$AAl?$AAe?$AA?9?$AA?$DO?$AAF?$AAu?$AAl?$AAl?$AAP?$AAa?$AAt?$AAh?$AA?$AA@ 10269508     wzFilePacker_static_d:fsdos.obj
 0003:000ee530       ??_C@_1FC@OIENAJFA@?$AAF?$AAi?$AAn?$AAd?$AAe?$AAr?$AA?9?$AA?$DO?$AAS?$AAi?$AAg?$AAn?$AAa?$AAt?$AAu?$AAr?$AAe?$AA?5?$AA?$DN?$AA?$DN?$AA?5?$AAD?$AAO?$AAS?$AAF?$AAI?$AAN?$AAD?$AAE?$AAR?$AA_?$AAS@ 10269530     wzFilePacker_static_d:fsdos.obj
 0003:000ee594       ??_C@_1M@DBIOIGJN@?$AAP?$AAr?$AAo?$AAp?$AAs?$AA?$AA@ 10269594     wzFilePacker_static_d:fsdos.obj
 0003:000ee5a4       ??_C@_1DG@NAJCKGOO@?$AA?$CB?$AA?$CC?$AAI?$AAl?$AAl?$AAe?$AAg?$AAa?$AAl?$AA?5?$AAo?$AAp?$AAe?$AAn?$AA?5?$AAm?$AAo?$AAd?$AAe?$AA?5?$AAf?$AAl?$AAa?$AAg?$AAs?$AA?$CC?$AA?$AA@ 102695a4     wzFilePacker_static_d:fsdos.obj
 0003:000ee5e4       ??_C@_0BI@DAMBELDL@Illegal?5open?5mode?5flags?$AA@ 102695e4     wzFilePacker_static_d:fsdos.obj
 0003:000ee600       ??_C@_1FA@HGKPAJKJ@?$AA?$CB?$AAD?$AAo?$AAs?$AAF?$AAS?$AA?5?$AA?$HM?$AA?$HM?$AA?5?$AAD?$AAo?$AAs?$AAF?$AAS?$AA?9?$AA?$DO?$AAI?$AAs?$AAD?$AAi?$AAr?$AAe?$AAc?$AAt?$AAo?$AAr?$AAy?$AA?5?$AA?$DN?$AA?$DN?$AA?5@ 10269600     wzFilePacker_static_d:fsdos.obj
 0003:000ee660       ??_C@_1FC@NINBKEFI@?$AAF?$AAi?$AAl?$AAe?$AA?9?$AA?$DO?$AAF?$AAi?$AAl?$AAe?$AAH?$AAa?$AAn?$AAd?$AAl?$AAe?$AA?5?$AA?$CB?$AA?$DN?$AA?5?$AAI?$AAN?$AAV?$AAA?$AAL?$AAI?$AAD?$AA_?$AAH?$AAA?$AAN?$AAD@ 10269660     wzFilePacker_static_d:fsdos.obj
 0003:000ee6c4       ??_C@_1DG@CEDIGOFF@?$AAp?$AA?5?$AA?9?$AA?5?$AA?$CI?$AAc?$AAh?$AAa?$AAr?$AA?5?$AA?$CK?$AA?$CJ?$AAB?$AAu?$AAf?$AAf?$AA?5?$AA?$DM?$AA?$DN?$AA?5?$AAM?$AAa?$AAx?$AAL?$AAe?$AAn?$AA?$AA@ 102696c4     wzFilePacker_static_d:fsdos.obj
 0003:000ee704       ??_C@_0BP@PFJFMKGH@Win32_SetFilePointer_Error?3?$CFd?6?$AA@ 10269704     wzFilePacker_static_d:fsdos.obj
 0003:000ee730       ??_C@_1EG@IHBDOBEB@?$AAC?$AAu?$AAr?$AAP?$AAo?$AAs?$AA?5?$AA?$CB?$AA?$DN?$AA?5?$AAI?$AAN?$AAV?$AAA?$AAL?$AAI?$AAD?$AA_?$AAS?$AAE?$AAT?$AA_?$AAF?$AAI?$AAL?$AAE?$AA_?$AAP?$AAO?$AAI?$AAN?$AAT@ 10269730     wzFilePacker_static_d:fsdos.obj
 0003:000eea10       ??_C@_0EJ@EJACJAIP@d?3?2sunengine?2public?2wzfilepacker@ 10269a10     wzFilePacker_static_d:dirtree.obj
 0003:000eea68       ??_C@_1BG@IOMNABBB@?$AAT?$AAr?$AAe?$AAe?$AA?9?$AA?$DO?$AAN?$AAa?$AAm?$AAe?$AA?$AA@ 10269a68     wzFilePacker_static_d:dirtree.obj
 0003:000eea84       ??_C@_19BGDOLOIO@?$AAT?$AAr?$AAe?$AAe?$AA?$AA@ 10269a84     wzFilePacker_static_d:dirtree.obj
 0003:000eea90       ??_C@_1JC@CLLFOBDI@?$AAd?$AA?3?$AA?2?$AAs?$AAu?$AAn?$AAe?$AAn?$AAg?$AAi?$AAn?$AAe?$AA?2?$AAp?$AAu?$AAb?$AAl?$AAi?$AAc?$AA?2?$AAw?$AAz?$AAf?$AAi?$AAl?$AAe?$AAp?$AAa?$AAc?$AAk?$AAe?$AAr@ 10269a90     wzFilePacker_static_d:dirtree.obj
 0003:000eeb40       ??_C@_1BG@LDKKMOFB@?$AAL?$AAe?$AAn?$AAg?$AAt?$AAh?$AA?5?$AA?$DO?$AA?5?$AA0?$AA?$AA@ 10269b40     wzFilePacker_static_d:dirtree.obj
 0003:000eeb5c       ??_C@_19NHABCBNP@?$AAP?$AAa?$AAt?$AAh?$AA?$AA@ 10269b5c     wzFilePacker_static_d:dirtree.obj
 0003:000eeb68       ??_C@_1CC@GAJDMOCL@?$AAs?$AAt?$AAr?$AAl?$AAe?$AAn?$AA?$CI?$AAP?$AAa?$AAt?$AAh?$AA?$CJ?$AA?5?$AA?$DO?$AA?5?$AA0?$AA?$AA@ 10269b68     wzFilePacker_static_d:dirtree.obj
 0003:000eeb90       ??_C@_1GE@PIENNMDG@?$AAI?$AAs?$AAD?$AAi?$AAr?$AAe?$AAc?$AAt?$AAo?$AAr?$AAy?$AA?5?$AA?$DN?$AA?$DN?$AA?5?$AAG?$AAE?$AA_?$AAT?$AAR?$AAU?$AAE?$AA?5?$AA?$HM?$AA?$HM?$AA?5?$AAI?$AAs?$AAD?$AAi?$AAr?$AAe@ 10269b90     wzFilePacker_static_d:dirtree.obj
 0003:000eec08       ??_C@_1EE@FKBHHKMM@?$AA?$CB?$AA?$CC?$AAS?$AAh?$AAo?$AAu?$AAl?$AAd?$AAn?$AA?8?$AAt?$AA?5?$AAb?$AAe?$AA?5?$AAa?$AA?5?$AAw?$AAa?$AAy?$AA?5?$AAt?$AAo?$AA?5?$AAg?$AAe?$AAt?$AA?5?$AAh?$AAe?$AAr?$AAe@ 10269c08     wzFilePacker_static_d:dirtree.obj
 0003:000eec5c       ??_C@_0BP@JMGKAOCP@Shouldn?8t?5be?5a?5way?5to?5get?5here?$AA@ 10269c5c     wzFilePacker_static_d:dirtree.obj
 0003:000eec84       ??_C@_1CE@HCFPDAMO@?$AAS?$AAi?$AAb?$AAl?$AAi?$AAn?$AAg?$AAs?$AA?4?$AAS?$AAi?$AAb?$AAl?$AAi?$AAn?$AAg?$AAs?$AA?$AA@ 10269c84     wzFilePacker_static_d:dirtree.obj
 0003:000eecb0       ??_C@_1O@GKMMPFJ@?$AAP?$AAa?$AAr?$AAe?$AAn?$AAt?$AA?$AA@ 10269cb0     wzFilePacker_static_d:dirtree.obj
 0003:000eecc0       ??_C@_1BA@FCDLMOIE@?$AAS?$AAu?$AAb?$AAT?$AAr?$AAe?$AAe?$AA?$AA@ 10269cc0     wzFilePacker_static_d:dirtree.obj
 0003:000eecd8       ??_C@_1GI@FNGBJDNK@?$AA?$CB?$AA?$CI?$AAT?$AAr?$AAe?$AAe?$AA?9?$AA?$DO?$AAA?$AAt?$AAt?$AAr?$AAi?$AAb?$AAu?$AAt?$AAe?$AAF?$AAl?$AAa?$AAg?$AAs?$AA?5?$AA?$CG?$AA?5?$AAG?$AAE?$AA_?$AAV?$AAF?$AAI?$AAL@ 10269cd8     wzFilePacker_static_d:dirtree.obj
 0003:000eed58       ??_C@_1FE@HJFHFMKE@?$AA?$CB?$AA?$CI?$AAA?$AAt?$AAt?$AAr?$AAi?$AAb?$AAu?$AAt?$AAe?$AAs?$AA?5?$AA?$CG?$AA?5?$AA?$HO?$AAG?$AAE?$AA_?$AAV?$AAF?$AAI?$AAL?$AAE?$AA_?$AAA?$AAT?$AAT?$AAR?$AAI?$AAB?$AA_@ 10269d58     wzFilePacker_static_d:dirtree.obj
 0003:000eedbc       ??_C@_1BG@GOLCKOJO@?$AAA?$AAt?$AAt?$AAr?$AAi?$AAb?$AAu?$AAt?$AAe?$AAs?$AA?$AA@ 10269dbc     wzFilePacker_static_d:dirtree.obj
 0003:000eedd8       ??_C@_1GI@MADGONFB@?$AA?$CB?$AA?$CI?$AAL?$AAe?$AAa?$AAf?$AA?9?$AA?$DO?$AAA?$AAt?$AAt?$AAr?$AAi?$AAb?$AAu?$AAt?$AAe?$AAF?$AAl?$AAa?$AAg?$AAs?$AA?5?$AA?$CG?$AA?5?$AAG?$AAE?$AA_?$AAV?$AAF?$AAI?$AAL@ 10269dd8     wzFilePacker_static_d:dirtree.obj
 0003:000eee54       ??_C@_19NNBNKKFI@?$AAL?$AAe?$AAa?$AAf?$AA?$AA@ 10269e54     wzFilePacker_static_d:dirtree.obj
 0003:000eee60       ??_C@_1BG@JDNEIJGP@?$AAM?$AAa?$AAx?$AAL?$AAe?$AAn?$AA?5?$AA?$DO?$AA?5?$AA0?$AA?$AA@ 10269e60     wzFilePacker_static_d:dirtree.obj
 0003:000eee7c       ??_C@_1CC@IFCDMLA@?$AAF?$AAi?$AAn?$AAd?$AAe?$AAr?$AA?9?$AA?$DO?$AAM?$AAa?$AAt?$AAc?$AAh?$AAE?$AAx?$AAt?$AA?$AA@ 10269e7c     wzFilePacker_static_d:dirtree.obj
 0003:000eeea4       ??_C@_1CE@HIJPFPPI@?$AAF?$AAi?$AAn?$AAd?$AAe?$AAr?$AA?9?$AA?$DO?$AAM?$AAa?$AAt?$AAc?$AAh?$AAN?$AAa?$AAm?$AAe?$AA?$AA@ 10269ea4     wzFilePacker_static_d:dirtree.obj
 0003:000ef158       ??_C@_0FA@PPILMDBI@d?3?2sunengine?2public?2wzfilepacker@ 1026a158     wzFilePacker_static_d:dirtree-common.obj
 0003:000ef1b8       ??_C@_1BA@BHDJAPNN@?$AAP?$AAa?$AAt?$AAt?$AAe?$AAr?$AAn?$AA?$AA@ 1026a1b8     wzFilePacker_static_d:dirtree-common.obj
 0003:000ef1cc       ??_C@_1O@FDGFDJPD@?$AAS?$AAo?$AAu?$AAr?$AAc?$AAe?$AA?$AA@ 1026a1cc     wzFilePacker_static_d:dirtree-common.obj
 0003:000ef1e0       ??_C@_1KA@MGBALOBF@?$AAd?$AA?3?$AA?2?$AAs?$AAu?$AAn?$AAe?$AAn?$AAg?$AAi?$AAn?$AAe?$AA?2?$AAp?$AAu?$AAb?$AAl?$AAi?$AAc?$AA?2?$AAw?$AAz?$AAf?$AAi?$AAl?$AAe?$AAp?$AAa?$AAc?$AAk?$AAe?$AAr@ 1026a1e0     wzFilePacker_static_d:dirtree-common.obj
 0003:000ef2a0       ??_C@_1EK@MBDPDCGA@?$AAM?$AAi?$AAc?$AAr?$AAo?$AAs?$AAo?$AAf?$AAt?$AA?5?$AAV?$AAi?$AAs?$AAu?$AAa?$AAl?$AA?5?$AAC?$AA?$CL?$AA?$CL?$AA?5?$AAR?$AAu?$AAn?$AAt?$AAi?$AAm?$AAe?$AA?5?$AAL?$AAi?$AAb@ 1026a2a0     libcmt:wassert.obj
 0003:000ef2f8       ??_C@_1HK@POCJMFGK@?$AA?$CI?$AAP?$AAr?$AAe?$AAs?$AAs?$AA?5?$AAR?$AAe?$AAt?$AAr?$AAy?$AA?5?$AAt?$AAo?$AA?5?$AAd?$AAe?$AAb?$AAu?$AAg?$AA?5?$AAt?$AAh?$AAe?$AA?5?$AAa?$AAp?$AAp?$AAl?$AAi?$AAc@ 1026a2f8     libcmt:wassert.obj
 0003:000ef390       ??_C@_1OA@EGMLFBHJ@?$AAF?$AAo?$AAr?$AA?5?$AAi?$AAn?$AAf?$AAo?$AAr?$AAm?$AAa?$AAt?$AAi?$AAo?$AAn?$AA?5?$AAo?$AAn?$AA?5?$AAh?$AAo?$AAw?$AA?5?$AAy?$AAo?$AAu?$AAr?$AA?5?$AAp?$AAr?$AAo?$AAg@ 1026a390     libcmt:wassert.obj
 0003:000ef49c       ??_C@_1O@KCAFKHJE@?$AAL?$AAi?$AAn?$AAe?$AA?3?$AA?5?$AA?$AA@ 1026a49c     libcmt:wassert.obj
 0003:000ef4ac       ??_C@_1O@HEMHKNDC@?$AAF?$AAi?$AAl?$AAe?$AA?3?$AA?5?$AA?$AA@ 1026a4ac     libcmt:wassert.obj
 0003:000ef4bc       ??_C@_1BE@PHKBBGE@?$AAP?$AAr?$AAo?$AAg?$AAr?$AAa?$AAm?$AA?3?$AA?5?$AA?$AA@ 1026a4bc     libcmt:wassert.obj
 0003:0011c738       ??_R4length_error@std@@6B@ 10297738     sound.obj
 0003:0011c750       ??_R3length_error@std@@8   10297750     sound.obj
 0003:0011c764       ??_R2length_error@std@@8   10297764     sound.obj
 0003:0011c774       ??_R1A@?0A@EA@length_error@std@@8 10297774     sound.obj
 0003:0011c798       ??_R1A@?0A@EA@logic_error@std@@8 10297798     sound.obj
 0003:0011c7bc       ??_R3logic_error@std@@8    102977bc     sound.obj
 0003:0011c7d0       ??_R2logic_error@std@@8    102977d0     sound.obj
 0003:0011c7dc       ??_R1A@?0A@EA@exception@std@@8 102977dc     sound.obj
 0003:0011c800       ??_R3exception@std@@8      10297800     sound.obj
 0003:0011c814       ??_R2exception@std@@8      10297814     sound.obj
 0003:0011c81c       ??_R4logic_error@std@@6B@  1029781c     sound.obj
 0003:0011c834       ??_R4bad_alloc@std@@6B@    10297834     sound.obj
 0003:0011c84c       ??_R3bad_alloc@std@@8      1029784c     sound.obj
 0003:0011c860       ??_R2bad_alloc@std@@8      10297860     sound.obj
 0003:0011c86c       ??_R1A@?0A@EA@bad_alloc@std@@8 1029786c     sound.obj
 0003:0011c890       ??_R4out_of_range@std@@6B@ 10297890     libcpmtd:string.obj
 0003:0011c8a4       ??_R3out_of_range@std@@8   102978a4     libcpmtd:string.obj
 0003:0011c8b4       ??_R2out_of_range@std@@8   102978b4     libcpmtd:string.obj
 0003:0011c8c4       ??_R1A@?0A@EA@out_of_range@std@@8 102978c4     libcpmtd:string.obj
 0003:0011c8e0       ??_R4invalid_argument@std@@6B@ 102978e0     libcpmtd:string.obj
 0003:0011c8f4       ??_R3invalid_argument@std@@8 102978f4     libcpmtd:string.obj
 0003:0011c904       ??_R2invalid_argument@std@@8 10297904     libcpmtd:string.obj
 0003:0011c914       ??_R1A@?0A@EA@invalid_argument@std@@8 10297914     libcpmtd:string.obj
 0003:0011c930       ??_R4type_info@@6B@        10297930     LIBCMTD:typinfo.obj
 0003:0011c944       ??_R3type_info@@8          10297944     LIBCMTD:typinfo.obj
 0003:0011c954       ??_R2type_info@@8          10297954     LIBCMTD:typinfo.obj
 0003:0011c95c       ??_R1A@?0A@EA@type_info@@8 1029795c     LIBCMTD:typinfo.obj
 0003:0011c978       ??_R4exception@std@@6B@    10297978     LIBCMTD:stdexcpt.obj
 0003:0011c98c       ??_R4bad_cast@std@@6B@     1029798c     LIBCMTD:stdexcpt.obj
 0003:0011c9a0       ??_R3bad_cast@std@@8       102979a0     LIBCMTD:stdexcpt.obj
 0003:0011c9b0       ??_R2bad_cast@std@@8       102979b0     LIBCMTD:stdexcpt.obj
 0003:0011c9bc       ??_R1A@?0A@EA@bad_cast@std@@8 102979bc     LIBCMTD:stdexcpt.obj
 0003:0011c9d8       ??_R4bad_typeid@std@@6B@   102979d8     LIBCMTD:stdexcpt.obj
 0003:0011c9ec       ??_R3bad_typeid@std@@8     102979ec     LIBCMTD:stdexcpt.obj
 0003:0011c9fc       ??_R2bad_typeid@std@@8     102979fc     LIBCMTD:stdexcpt.obj
 0003:0011ca08       ??_R1A@?0A@EA@bad_typeid@std@@8 10297a08     LIBCMTD:stdexcpt.obj
 0003:0011ca24       ??_R4__non_rtti_object@std@@6B@ 10297a24     LIBCMTD:stdexcpt.obj
 0003:0011ca38       ??_R3__non_rtti_object@std@@8 10297a38     LIBCMTD:stdexcpt.obj
 0003:0011ca48       ??_R2__non_rtti_object@std@@8 10297a48     LIBCMTD:stdexcpt.obj
 0003:0011ca58       ??_R1A@?0A@EA@__non_rtti_object@std@@8 10297a58     LIBCMTD:stdexcpt.obj
 0003:0011ca74       ??_R4bad_exception@std@@6B@ 10297a74     LIBCMTD:frame.obj
 0003:0011ca88       ??_R3bad_exception@std@@8  10297a88     LIBCMTD:frame.obj
 0003:0011ca98       ??_R2bad_exception@std@@8  10297a98     LIBCMTD:frame.obj
 0003:0011caa4       ??_R1A@?0A@EA@bad_exception@std@@8 10297aa4     LIBCMTD:frame.obj
 0003:0011cc3c       ___rtc_iaa                 10297c3c     LIBCMTD:_initsect_.obj
 0003:0011cee0       ___rtc_izz                 10297ee0     LIBCMTD:_initsect_.obj
 0003:0011cfe4       ___rtc_taa                 10297fe4     LIBCMTD:_initsect_.obj
 0003:0011d288       ___rtc_tzz                 10298288     LIBCMTD:_initsect_.obj
 0003:0011d8c8       __TI3?AVlength_error@std@@ 102988c8     sound.obj
 0003:0011d90c       __CTA3?AVlength_error@std@@ 1029890c     sound.obj
 0003:0011d920       __CT??_R0?AVlength_error@std@@@8??0length_error@std@@QAE@ABV01@@Z44 10298920     sound.obj
 0003:0011d940       __CT??_R0?AVlogic_error@std@@@8??0logic_error@std@@QAE@ABV01@@Z44 10298940     sound.obj
 0003:0011d960       __CT??_R0?AVexception@std@@@8??0exception@std@@QAE@ABV01@@Z12 10298960     sound.obj
 0003:0011dc58       __TI2?AVbad_alloc@std@@    10298c58     sound.obj
 0003:0011dc6c       __CTA2?AVbad_alloc@std@@   10298c6c     sound.obj
 0003:0011dc7c       __CT??_R0?AVbad_alloc@std@@@8??0bad_alloc@std@@QAE@ABV01@@Z12 10298c7c     sound.obj
 0003:0011fc48       __TI3?AVout_of_range@std@@ 1029ac48     libcpmtd:string.obj
 0003:0011fc84       __CTA3?AVout_of_range@std@@ 1029ac84     libcpmtd:string.obj
 0003:0011fc94       __CT??_R0?AVout_of_range@std@@@8??0out_of_range@std@@QAE@ABV01@@Z44 1029ac94     libcpmtd:string.obj
 0003:0011fcb0       __TI3?AVinvalid_argument@std@@ 1029acb0     libcpmtd:string.obj
 0003:0011fcec       __CTA3?AVinvalid_argument@std@@ 1029acec     libcpmtd:string.obj
 0003:0011fcfc       __CT??_R0?AVinvalid_argument@std@@@8??0invalid_argument@std@@QAE@ABV01@@Z44 1029acfc     libcpmtd:string.obj
 0003:0012033c       __TI2?AVbad_exception@std@@ 1029b33c     LIBCMTD:frame.obj
 0003:0012034c       __CTA2?AVbad_exception@std@@ 1029b34c     LIBCMTD:frame.obj
 0003:00120358       __CT??_R0?AVbad_exception@std@@@8??0bad_exception@std@@QAE@ABV01@@Z12 1029b358     LIBCMTD:frame.obj
 0004:0000000c       ?MAX_CHANNELS@@3HA         1029e00c     ds.obj
 0004:00000018       ?Ds_eax_presets@@3PAUEAX_REVERBPROPERTIES@@A 1029e018     ds.obj
 0004:000001b8       ?DSPROPSETID_EAX_ReverbProperties_Def@@3U_GUID@@A 1029e1b8     ds.obj
 0004:000001c8       ?DSPROPSETID_EAXBUFFER_ReverbProperties_Def@@3U_GUID@@A 1029e1c8     ds.obj
 0004:00000238       ?DSPROPSETID_VoiceManager_Def@@3U_GUID@@A 1029e238     ds3d.obj
 0004:00000250       ?Sound_enabled@@3HA        1029e250     sound.obj
 0004:00000254       ?Master_sound_volume@@3MA  1029e254     sound.obj
 0004:00000258       ?Master_voice_volume@@3MA  1029e258     sound.obj
 0004:0000025c       ?Sound_cache_maintain_milliseconds@@3HA 1029e25c     sound.obj
 0004:00000264       ??_R0?AVlength_error@std@@@8 1029e264     sound.obj
 0004:0000028c       ??_R0?AVlogic_error@std@@@8 1029e28c     sound.obj
 0004:000002b0       ??_R0?AVexception@std@@@8  1029e2b0     sound.obj
 0004:000002d4       ??_R0?AVbad_alloc@std@@@8  1029e2d4     sound.obj
 0004:0000031c       ?timestamp_ticker@@3HA     1029e31c     timer.obj
 0004:00000344       ?fl_magic@@3HA             1029e344     floating.obj
 0004:00000348       ?p_fl_magic@@3PBMB         1029e348     floating.obj
 0004:00000354       ?vmd_x_vector@@3Uvector@@A 1029e354     vecmat.obj
 0004:00000360       ?vmd_y_vector@@3Uvector@@A 1029e360     vecmat.obj
 0004:0000036c       ?vmd_z_vector@@3Uvector@@A 1029e36c     vecmat.obj
 0004:00000378       ?vmd_identity_matrix@@3Umatrix@@A 1029e378     vecmat.obj
 0004:000003b4       ?libxls_major_version@@3HA 1029e3b4     version.obj
 0004:000003c8       ?brdb@@3PAUstr_brdb@@A     1029e3c8     xlstool.obj
 0004:00000dc0       ?nMixerControlID_master_vol@@3HA 1029edc0     wzSound.obj
 0004:00000dc4       ?nMixerControlID_master_pan@@3HA 1029edc4     wzSound.obj
 0004:00000dc8       ?nMixerControlID_master_mute@@3HA 1029edc8     wzSound.obj
 0004:00000dcc       ?nMixerControlID_wav_vol@@3HA 1029edcc     wzSound.obj
 0004:00000dd0       ?nMixerControlID_wav_pan@@3HA 1029edd0     wzSound.obj
 0004:00000dd4       ?nMixerControlID_wav_mute@@3HA 1029edd4     wzSound.obj
 0004:00000dd8       ?nMixerControlID_mic_input_vol@@3PAHA 1029edd8     wzSound.obj
 0004:00000dec       ?nMixerControlID_mic_output_vol@@3HA 1029edec     wzSound.obj
 0004:00000df0       ?nMixerControlID_mic_output_mute@@3HA 1029edf0     wzSound.obj
 0004:00000df4       ?_rolloff_factor@@3MA      1029edf4     wzSound.obj
 0004:00000e10       ??_R0?AVout_of_range@std@@@8 1029ee10     libcpmtd:string.obj
 0004:00000e30       ??_R0?AVinvalid_argument@std@@@8 1029ee30     libcpmtd:string.obj
 0004:00000e58       ??_C@_04EFJP@pcmR?$AA@     1029ee58     vorbisfile_static:vorbisfile.obj
 0004:00000e60       ??_C@_04EHCF@pcmL?$AA@     1029ee60     vorbisfile_static:vorbisfile.obj
 0004:00000e68       ??_C@_01KPOD@?$DN?$AA@     1029ee68     vorbisfile_static:info.obj
 0004:00000e6c       ??_C@_06GIBB@vorbis?$AA@   1029ee6c     vorbisfile_static:info.obj
 0004:00000e74       ??_C@_0BO@KFNF@Xiph?4Org?5libVorbis?5I?520030909?$AA@ 1029ee74     vorbisfile_static:info.obj
 0004:00000e94       _analysis_noisy            1029ee94     vorbisfile_static:analysis.obj
 0004:00000e98       ??_C@_03FBAH@?$CFf?6?$AA@  1029ee98     vorbisfile_static:analysis.obj
 0004:00000e9c       ??_C@_03CHB@?$CFf?5?$AA@   1029ee9c     vorbisfile_static:analysis.obj
 0004:00000ea0       ??_C@_0BO@NFHP@failed?5to?5open?5data?5dump?5file?$AA@ 1029eea0     vorbisfile_static:analysis.obj
 0004:00000ec0       ??_C@_01LLF@w?$AA@         1029eec0     vorbisfile_static:analysis.obj
 0004:00000ec4       ??_C@_07DFJO@?$CFs_?$CFd?4m?$AA@ 1029eec4     vorbisfile_static:analysis.obj
 0004:00006e38       __floor_P                  102a4e38     vorbisfile_static:registry.obj
 0004:00006e40       __residue_P                102a4e40     vorbisfile_static:registry.obj
 0004:00006e4c       __mapping_P                102a4e4c     vorbisfile_static:registry.obj
 0004:0000ee20       _mapping0_exportbundle     102ace20     vorbisfile_static:mapping0.obj
 0004:0000ee38       _residue0_exportbundle     102ace38     vorbisfile_static:res0.obj
 0004:0000ee58       _residue1_exportbundle     102ace58     vorbisfile_static:res0.obj
 0004:0000ee78       _residue2_exportbundle     102ace78     vorbisfile_static:res0.obj
 0004:0000f298       _floor1_exportbundle       102ad298     vorbisfile_static:floor1.obj
 0004:0000f2b8       _floor0_exportbundle       102ad2b8     vorbisfile_static:floor0.obj
 0004:0000f770       ___security_cookie         102ad770     LIBCMTD:gs_cookie.obj
 0004:0000f774       ___security_cookie_complement 102ad774     LIBCMTD:gs_cookie.obj
 0004:0000f778       __fltused                  102ad778     LIBCMTD:_fpinit_.obj
 0004:0000f77c       __ldused                   102ad77c     LIBCMTD:_fpinit_.obj
 0004:0000f790       __half                     102ad790     LIBCMTD:_pow_.obj
 0004:0000f7a4       ??_R0?AVtype_info@@@8      102ad7a4     LIBCMTD:typinfo.obj
 0004:0000f7c0       ??_R0?AVbad_cast@std@@@8   102ad7c0     LIBCMTD:stdexcpt.obj
 0004:0000f7dc       ??_R0?AVbad_typeid@std@@@8 102ad7dc     LIBCMTD:stdexcpt.obj
 0004:0000f7fc       ??_R0?AV__non_rtti_object@std@@@8 102ad7fc     LIBCMTD:stdexcpt.obj
 0004:0000f824       ?_RTC_ErrorLevels@@3PAHA   102ad824     LIBCMTD:_error_.obj
 0004:0000fa10       __crtDbgFlag               102ada10     LIBCMTD:dbgheap.obj
 0004:0000fa14       ___crtDebugFillThreshold   102ada14     LIBCMTD:dbgheap.obj
 0004:0000fa1c       __crtBreakAlloc            102ada1c     LIBCMTD:dbgheap.obj
 0004:0000fa24       ___abort_behavior          102ada24     LIBCMTD:abort.obj
 0004:0000fa28       __iob                      102ada28     LIBCMTD:_file.obj
 0004:0000fcb0       __aexit_rtn                102adcb0     LIBCMTD:crt0dat.obj
 0004:0000fcb8       ___initialmbcinfo          102adcb8     LIBCMTD:mbctype.obj
 0004:0000fed8       __mbctype                  102aded8     LIBCMTD:mbctype.obj
 0004:0000ffe0       __mbcasemap                102adfe0     LIBCMTD:mbctype.obj
 0004:000100e0       ___ptmbcinfo               102ae0e0     LIBCMTD:mbctype.obj
 0004:000101dc       ___globallocalestatus      102ae1dc     LIBCMTD:glstatus.obj
 0004:000101e0       ___clocalestr              102ae1e0     LIBCMTD:nlsdata2.obj
 0004:000101e8       ___initiallocinfo          102ae1e8     LIBCMTD:nlsdata2.obj
 0004:000102c0       ___ptlocinfo               102ae2c0     LIBCMTD:nlsdata2.obj
 0004:000102c4       ___lc_clike                102ae2c4     LIBCMTD:nlsdata2.obj
 0004:000102c8       ___initiallocalestructinfo 102ae2c8     LIBCMTD:nlsdata2.obj
 0004:000102d0       ___flsindex                102ae2d0     LIBCMTD:tidtable.obj
 0004:000102d4       ___getvalueindex           102ae2d4     LIBCMTD:tidtable.obj
 0004:000102d8       __cfltcvt_tab              102ae2d8     LIBCMTD:cmiscdat.obj
 0004:00010300       __infinity                 102ae300     LIBCMTD:_87tran_.obj
 0004:0001030a       __minfinity                102ae30a     LIBCMTD:_87tran_.obj
 0004:00010314       __logemax                  102ae314     LIBCMTD:_87tran_.obj
 0004:0001033a       __OP_EXPjmptab             102ae33a     LIBCMTD:_87tran_.obj
 0004:00010360       __indefinite               102ae360     LIBCMTD:_87disp_.obj
 0004:0001036a       __piby2                    102ae36a     LIBCMTD:_87disp_.obj
 0004:00010394       ??_R0?AVbad_exception@std@@@8 102ae394     LIBCMTD:frame.obj
 0004:000103c0       __pfnAllocHook             102ae3c0     LIBCMTD:dbghook.obj
 0004:000104e8       __crtAssertBusy            102ae4e8     LIBCMTD:dbgrptt.obj
 0004:000104ec       __CrtDbgMode               102ae4ec     LIBCMTD:dbgrptt.obj
 0004:000104f8       __CrtDbgFile               102ae4f8     LIBCMTD:dbgrptt.obj
 0004:00010508       ___nullstring              102ae508     LIBCMTD:output.obj
 0004:0001050c       ___wnullstring             102ae50c     LIBCMTD:output.obj
 0004:00010518       ___badioinfo               102ae518     LIBCMTD:ioinit.obj
 0004:00010558       __lookuptrailbytes         102ae558     LIBCMTD:read.obj
 0004:00010748       __d_inf                    102ae748     LIBCMTD:_util_.obj
 0004:00010750       __d_ind                    102ae750     LIBCMTD:_util_.obj
 0004:00010758       __d_max                    102ae758     LIBCMTD:_util_.obj
 0004:00010760       __d_min                    102ae760     LIBCMTD:_util_.obj
 0004:00010768       __d_mzero                  102ae768     LIBCMTD:_util_.obj
 0004:00010794       __amblksiz                 102ae794     LIBCMTD:heapinit.obj
 0004:00010798       __First_FPE_Indx           102ae798     LIBCMTD:winxfltr.obj
 0004:0001079c       __Num_FPE                  102ae79c     LIBCMTD:winxfltr.obj
 0004:000107a0       __XcptActTabSize           102ae7a0     LIBCMTD:winxfltr.obj
 0004:000107a4       __XcptActTabCount          102ae7a4     LIBCMTD:winxfltr.obj
 0004:00010868       __sys_errlist              102ae868     LIBCMTD:syserr.obj
 0004:00010918       __sys_nerr                 102ae918     LIBCMTD:syserr.obj
 0004:00010920       __pctype                   102ae920     LIBCMTD:ctype.obj
 0004:00010924       __pwctype                  102ae924     LIBCMTD:ctype.obj
 0004:00010928       ___lc_time_c               102ae928     LIBCMTD:strftime.obj
 0004:000109e0       ___lc_time_curr            102ae9e0     LIBCMTD:strftime.obj
 0004:000109e4       ___lconv_static_decimal    102ae9e4     LIBCMTD:lconv.obj
 0004:000109e8       ___lconv_c                 102ae9e8     LIBCMTD:lconv.obj
 0004:00010a18       ___lconv                   102aea18     LIBCMTD:lconv.obj
 0004:00010a1c       ___mb_cur_max              102aea1c     LIBCMTD:nlsdata1.obj
 0004:00010a20       ___decimal_point           102aea20     LIBCMTD:nlsdata1.obj
 0004:00010a24       ___decimal_point_length    102aea24     LIBCMTD:nlsdata1.obj
 0004:00010b90       __NLG_Destination          102aeb90     LIBCMTD:exsup.obj
 0004:00010be0       __pow10pos                 102aebe0     LIBCMTD:_constpow_.obj
 0004:00010d40       __pow10neg                 102aed40     LIBCMTD:_constpow_.obj
 0004:00010e9c       __matherr_flag             102aee9c     LIBCMTD:_matherr_.obj
 0004:00010ea8       __timezone                 102aeea8     LIBCMTD:timeset.obj
 0004:00010eac       __daylight                 102aeeac     LIBCMTD:timeset.obj
 0004:00010eb0       __dstbias                  102aeeb0     LIBCMTD:timeset.obj
 0004:00010f38       __tzname                   102aef38     LIBCMTD:timeset.obj
 0004:00010f58       __coninpfh                 102aef58     LIBCMTD:initcon.obj
 0004:00010f5c       __confh                    102aef5c     LIBCMTD:initcon.obj
 0004:00010f60       __lpdays                   102aef60     LIBCMTD:days.obj
 0004:00010f94       __days                     102aef94     LIBCMTD:days.obj
 0004:00010fd0       __libiconv_version         102aefd0     iconv:iconv.obj
 0004:00010fd4       ??_C@_08KIEN@?1?1IGNORE?$AA@ 102aefd4     iconv:iconv.obj
 0004:00010fe0       ??_C@_0L@CMOP@?1?1TRANSLIT?$AA@ 102aefe0     iconv:iconv.obj
 0004:00010fec       ??_C@_05OGAG@ASCII?$AA@    102aefec     iconv:localcharset.obj
 0004:00010ff4       ??_C@_04FIHK@CP?$CFu?$AA@  102aeff4     iconv:localcharset.obj
 0004:00010ffc       ??_C@_0BAE@GMIJ@CP936?$AAGBK?$AACP1361?$AAJOHAB?$AACP20127?$AAA@ 102aeffc     iconv:localcharset.obj
 0004:0001111c       ?__LINE__Var@?1??geVFile_RegisterFileSystem@@9@9 102af11c     wzFilePacker_static_d:vfile.obj
 0004:00011120       ?__LINE__Var@?1??geVFile_RegisterFileSystemInternal@@9@9@959c4940 102af120     wzFilePacker_static_d:vfile.obj
 0004:00011124       ?__LINE__Var@?1??geVFile_OpenNewSystem@@9@9 102af124     wzFilePacker_static_d:vfile.obj
 0004:00011128       ?__LINE__Var@?1??geVFile_UpdateSystem@@9@9 102af128     wzFilePacker_static_d:vfile.obj
 0004:0001112c       ?__LINE__Var@?1??geVFile_UpdateContext@@9@9 102af12c     wzFilePacker_static_d:vfile.obj
 0004:00011130       ?__LINE__Var@?1??geVFile_Open_Detail@@9@9 102af130     wzFilePacker_static_d:vfile.obj
 0004:00011134       ?__LINE__Var@?1??geVFile_Open@@9@9 102af134     wzFilePacker_static_d:vfile.obj
 0004:00011138       ?__LINE__Var@?1??geVFile_GetContext@@9@9 102af138     wzFilePacker_static_d:vfile.obj
 0004:0001113c       ?__LINE__Var@?1??geVFile_AddPath@@9@9 102af13c     wzFilePacker_static_d:vfile.obj
 0004:00011140       ?__LINE__Var@?1??CopySearchList@@9@9@959c4940 102af140     wzFilePacker_static_d:vfile.obj
 0004:00011144       ?__LINE__Var@?1??geVFile_DeleteFile@@9@9 102af144     wzFilePacker_static_d:vfile.obj
 0004:00011148       ?__LINE__Var@?1??geVFile_RenameFile@@9@9 102af148     wzFilePacker_static_d:vfile.obj
 0004:0001114c       ?__LINE__Var@?1??geVFile_Close@@9@9 102af14c     wzFilePacker_static_d:vfile.obj
 0004:00011150       ?__LINE__Var@?1??geVFile_GetS@@9@9 102af150     wzFilePacker_static_d:vfile.obj
 0004:00011154       ?__LINE__Var@?1??geVFile_Read@@9@9 102af154     wzFilePacker_static_d:vfile.obj
 0004:00011158       ?__LINE__Var@?1??geVFile_Write@@9@9 102af158     wzFilePacker_static_d:vfile.obj
 0004:0001115c       ?__LINE__Var@?1??geVFile_Seek@@9@9 102af15c     wzFilePacker_static_d:vfile.obj
 0004:00011160       ?__LINE__Var@?1??geVFile_Printf@@9@9 102af160     wzFilePacker_static_d:vfile.obj
 0004:00011164       ?__LINE__Var@?1??geVFile_EOF@@9@9 102af164     wzFilePacker_static_d:vfile.obj
 0004:00011168       ?__LINE__Var@?1??geVFile_Tell@@9@9 102af168     wzFilePacker_static_d:vfile.obj
 0004:0001116c       ?__LINE__Var@?1??geVFile_Size@@9@9 102af16c     wzFilePacker_static_d:vfile.obj
 0004:00011170       ?__LINE__Var@?1??geVFile_GetProperties@@9@9 102af170     wzFilePacker_static_d:vfile.obj
 0004:00011174       ?__LINE__Var@?1??geVFile_SetSize@@9@9 102af174     wzFilePacker_static_d:vfile.obj
 0004:00011178       ?__LINE__Var@?1??geVFile_SetAttributes@@9@9 102af178     wzFilePacker_static_d:vfile.obj
 0004:0001117c       ?__LINE__Var@?1??geVFile_SetTime@@9@9 102af17c     wzFilePacker_static_d:vfile.obj
 0004:00011180       ?__LINE__Var@?1??geVFile_SetHints@@9@9 102af180     wzFilePacker_static_d:vfile.obj
 0004:00011184       ?__LINE__Var@?1??geVFile_EnlargeDirectorySize@@9@9 102af184     wzFilePacker_static_d:vfile.obj
 0004:00011188       ?__LINE__Var@?1??geVFile_CreateFinder@@9@9 102af188     wzFilePacker_static_d:vfile.obj
 0004:0001118c       ?__LINE__Var@?1??geVFile_DestroyFinder@@9@9 102af18c     wzFilePacker_static_d:vfile.obj
 0004:00011190       ?__LINE__Var@?1??geVFile_FinderGetNextFile@@9@9 102af190     wzFilePacker_static_d:vfile.obj
 0004:00011194       ?__LINE__Var@?1??geVFile_FinderGetProperties@@9@9 102af194     wzFilePacker_static_d:vfile.obj
 0004:00011198       _cchCurDir                 102af198     wzFilePacker_static_d:vFile_util.obj
 0004:000111a8       ?__LINE__Var@?1??geRam_AllocateClear@@9@9 102af1a8     wzFilePacker_static_d:Ram.obj
 0004:000111ac       ?__LINE__Var@?1??geRam_Free_@@9@9 102af1ac     wzFilePacker_static_d:Ram.obj
 0004:000111b0       ?__LINE__Var@?1??ram_verify_block@@9@9@9ed7aace 102af1b0     wzFilePacker_static_d:Ram.obj
 0004:000111b4       ?__LINE__Var@?1??_geRam_DebugRealloc@@9@9 102af1b4     wzFilePacker_static_d:Ram.obj
 0004:0001123c       ?__LINE__Var@?1??FSVFS_FinderCreate@@9@9@34ff7953 102af23c     wzFilePacker_static_d:fsvfs.obj
 0004:00011240       ?__LINE__Var@?1??FSVFS_FinderGetNextFile@@9@9@34ff7953 102af240     wzFilePacker_static_d:fsvfs.obj
 0004:00011244       ?__LINE__Var@?1??FSVFS_FinderGetProperties@@9@9@34ff7953 102af244     wzFilePacker_static_d:fsvfs.obj
 0004:00011248       ?__LINE__Var@?1??FSVFS_FinderDestroy@@9@9@34ff7953 102af248     wzFilePacker_static_d:fsvfs.obj
 0004:0001124c       ?__LINE__Var@?1??FSVFS_Open@@9@9@34ff7953 102af24c     wzFilePacker_static_d:fsvfs.obj
 0004:00011250       ?__LINE__Var@?1??FSVFS_OpenNewSystem@@9@9@34ff7953 102af250     wzFilePacker_static_d:fsvfs.obj
 0004:00011254       ?__LINE__Var@?1??FSVFS_Close@@9@9@34ff7953 102af254     wzFilePacker_static_d:fsvfs.obj
 0004:00011258       ?__LINE__Var@?1??FSVFS_GetS@@9@9@34ff7953 102af258     wzFilePacker_static_d:fsvfs.obj
 0004:0001125c       ?__LINE__Var@?1??ForceFilePos@@9@9@34ff7953 102af25c     wzFilePacker_static_d:fsvfs.obj
 0004:00011260       ?__LINE__Var@?1??ClampOperationSize@@9@9@34ff7953 102af260     wzFilePacker_static_d:fsvfs.obj
 0004:00011264       ?__LINE__Var@?1??UpdateFilePos@@9@9@34ff7953 102af264     wzFilePacker_static_d:fsvfs.obj
 0004:00011268       ?__LINE__Var@?1??FSVFS_Read@@9@9@34ff7953 102af268     wzFilePacker_static_d:fsvfs.obj
 0004:0001126c       ?__LINE__Var@?1??FSVFS_Write@@9@9@34ff7953 102af26c     wzFilePacker_static_d:fsvfs.obj
 0004:00011270       ?__LINE__Var@?1??FSVFS_Seek@@9@9@34ff7953 102af270     wzFilePacker_static_d:fsvfs.obj
 0004:00011274       ?__LINE__Var@?1??FSVFS_EOF@@9@9@34ff7953 102af274     wzFilePacker_static_d:fsvfs.obj
 0004:00011278       ?__LINE__Var@?1??FSVFS_Tell@@9@9@34ff7953 102af278     wzFilePacker_static_d:fsvfs.obj
 0004:0001127c       ?__LINE__Var@?1??FSVFS_Size@@9@9@34ff7953 102af27c     wzFilePacker_static_d:fsvfs.obj
 0004:00011280       ?__LINE__Var@?1??FSVFS_GetProperties@@9@9@34ff7953 102af280     wzFilePacker_static_d:fsvfs.obj
 0004:00011284       ?__LINE__Var@?1??FSVFS_SetSize@@9@9@34ff7953 102af284     wzFilePacker_static_d:fsvfs.obj
 0004:00011288       ?__LINE__Var@?1??FSVFS_SetAttributes@@9@9@34ff7953 102af288     wzFilePacker_static_d:fsvfs.obj
 0004:0001128c       ?__LINE__Var@?1??FSVFS_SetTime@@9@9@34ff7953 102af28c     wzFilePacker_static_d:fsvfs.obj
 0004:00011290       ?__LINE__Var@?1??FSVFS_SetHints@@9@9@34ff7953 102af290     wzFilePacker_static_d:fsvfs.obj
 0004:00011294       ?__LINE__Var@?1??FSVFS_FileExists@@9@9@34ff7953 102af294     wzFilePacker_static_d:fsvfs.obj
 0004:00011298       ?__LINE__Var@?1??FSVFS_Disperse@@9@9@34ff7953 102af298     wzFilePacker_static_d:fsvfs.obj
 0004:0001129c       ?__LINE__Var@?1??FSVFS_RenameFile@@9@9@34ff7953 102af29c     wzFilePacker_static_d:fsvfs.obj
 0004:00011318       ?__LINE__Var@?1??FSMemory_FinderGetNextFile@@9@9@9d4ac2f6 102af318     wzFilePacker_static_d:FSMEMORY.obj
 0004:0001131c       ?__LINE__Var@?1??FSMemory_FinderGetProperties@@9@9@9d4ac2f6 102af31c     wzFilePacker_static_d:FSMEMORY.obj
 0004:00011320       ?__LINE__Var@?1??FSMemory_FinderDestroy@@9@9@9d4ac2f6 102af320     wzFilePacker_static_d:FSMEMORY.obj
 0004:00011324       ?__LINE__Var@?1??FSMemory_OpenNewSystem@@9@9@9d4ac2f6 102af324     wzFilePacker_static_d:FSMEMORY.obj
 0004:00011328       ?__LINE__Var@?1??FSMemory_UpdateContext@@9@9@9d4ac2f6 102af328     wzFilePacker_static_d:FSMEMORY.obj
 0004:0001132c       ?__LINE__Var@?1??FSMemory_Close@@9@9@9d4ac2f6 102af32c     wzFilePacker_static_d:FSMEMORY.obj
 0004:00011330       ?__LINE__Var@?1??FSMemory_GetS@@9@9@9d4ac2f6 102af330     wzFilePacker_static_d:FSMEMORY.obj
 0004:00011334       ?__LINE__Var@?1??FSMemory_Read@@9@9@9d4ac2f6 102af334     wzFilePacker_static_d:FSMEMORY.obj
 0004:00011338       ?__LINE__Var@?1??FSMemory_Write@@9@9@9d4ac2f6 102af338     wzFilePacker_static_d:FSMEMORY.obj
 0004:0001133c       ?__LINE__Var@?1??TestForExpansion@@9@9@9d4ac2f6 102af33c     wzFilePacker_static_d:FSMEMORY.obj
 0004:00011340       ?__LINE__Var@?1??FSMemory_Seek@@9@9@9d4ac2f6 102af340     wzFilePacker_static_d:FSMEMORY.obj
 0004:00011344       ?__LINE__Var@?1??FSMemory_EOF@@9@9@9d4ac2f6 102af344     wzFilePacker_static_d:FSMEMORY.obj
 0004:00011348       ?__LINE__Var@?1??FSMemory_Tell@@9@9@9d4ac2f6 102af348     wzFilePacker_static_d:FSMEMORY.obj
 0004:0001134c       ?__LINE__Var@?1??FSMemory_Size@@9@9@9d4ac2f6 102af34c     wzFilePacker_static_d:FSMEMORY.obj
 0004:00011350       ?__LINE__Var@?1??FSMemory_GetProperties@@9@9@9d4ac2f6 102af350     wzFilePacker_static_d:FSMEMORY.obj
 0004:00011354       ?__LINE__Var@?1??FSMemory_SetSize@@9@9@9d4ac2f6 102af354     wzFilePacker_static_d:FSMEMORY.obj
 0004:00011358       ?__LINE__Var@?1??FSMemory_SetAttributes@@9@9@9d4ac2f6 102af358     wzFilePacker_static_d:FSMEMORY.obj
 0004:0001135c       ?__LINE__Var@?1??FSMemory_SetTime@@9@9@9d4ac2f6 102af35c     wzFilePacker_static_d:FSMEMORY.obj
 0004:00011360       ?__LINE__Var@?1??FSMemory_SetHints@@9@9@9d4ac2f6 102af360     wzFilePacker_static_d:FSMEMORY.obj
 0004:000113e0       ?__LINE__Var@?1??FSDos_FinderCreate@@9@9@53d7f23b 102af3e0     wzFilePacker_static_d:fsdos.obj
 0004:000113e4       ?__LINE__Var@?1??BuildFileName@@9@9@53d7f23b 102af3e4     wzFilePacker_static_d:fsdos.obj
 0004:000113e8       ?__LINE__Var@?1??FSDos_FinderGetNextFile@@9@9@53d7f23b 102af3e8     wzFilePacker_static_d:fsdos.obj
 0004:000113ec       ?__LINE__Var@?1??FSDos_FinderGetProperties@@9@9@53d7f23b 102af3ec     wzFilePacker_static_d:fsdos.obj
 0004:000113f0       ?__LINE__Var@?1??FSDos_FinderDestroy@@9@9@53d7f23b 102af3f0     wzFilePacker_static_d:fsdos.obj
 0004:000113f4       ?__LINE__Var@?1??FSDos_Open@@9@9@53d7f23b 102af3f4     wzFilePacker_static_d:fsdos.obj
 0004:000113f8       ?__LINE__Var@?1??FSDos_Close@@9@9@53d7f23b 102af3f8     wzFilePacker_static_d:fsdos.obj
 0004:000113fc       ?__LINE__Var@?1??FSDos_GetS@@9@9@53d7f23b 102af3fc     wzFilePacker_static_d:fsdos.obj
 0004:00011400       ?__LINE__Var@?1??FSDos_Read@@9@9@53d7f23b 102af400     wzFilePacker_static_d:fsdos.obj
 0004:00011404       ?__LINE__Var@?1??FSDos_Write@@9@9@53d7f23b 102af404     wzFilePacker_static_d:fsdos.obj
 0004:00011408       ?__LINE__Var@?1??FSDos_Seek@@9@9@53d7f23b 102af408     wzFilePacker_static_d:fsdos.obj
 0004:0001140c       ?__LINE__Var@?1??FSDos_EOF@@9@9@53d7f23b 102af40c     wzFilePacker_static_d:fsdos.obj
 0004:00011410       ?__LINE__Var@?1??FSDos_Tell@@9@9@53d7f23b 102af410     wzFilePacker_static_d:fsdos.obj
 0004:00011414       ?__LINE__Var@?1??FSDos_Size@@9@9@53d7f23b 102af414     wzFilePacker_static_d:fsdos.obj
 0004:00011418       ?__LINE__Var@?1??FSDos_GetProperties@@9@9@53d7f23b 102af418     wzFilePacker_static_d:fsdos.obj
 0004:0001141c       ?__LINE__Var@?1??FSDos_SetSize@@9@9@53d7f23b 102af41c     wzFilePacker_static_d:fsdos.obj
 0004:00011420       ?__LINE__Var@?1??FSDos_SetAttributes@@9@9@53d7f23b 102af420     wzFilePacker_static_d:fsdos.obj
 0004:00011424       ?__LINE__Var@?1??FSDos_SetTime@@9@9@53d7f23b 102af424     wzFilePacker_static_d:fsdos.obj
 0004:00011428       ?__LINE__Var@?1??FSDos_SetHints@@9@9@53d7f23b 102af428     wzFilePacker_static_d:fsdos.obj
 0004:00011438       ?__LINE__Var@?1??DirTree_Create@@9@9 102af438     wzFilePacker_static_d:dirtree.obj
 0004:0001143c       ?__LINE__Var@?1??DirTree_Destroy@@9@9 102af43c     wzFilePacker_static_d:dirtree.obj
 0004:00011440       ?__LINE__Var@?1??DirTree_SetFileSize@@9@9 102af440     wzFilePacker_static_d:dirtree.obj
 0004:00011444       ?__LINE__Var@?1??DirTree_GetFileSize@@9@9 102af444     wzFilePacker_static_d:dirtree.obj
 0004:00011448       ?__LINE__Var@?1??WriteTree@@9@9@6bd7c2e6 102af448     wzFilePacker_static_d:dirtree.obj
 0004:0001144c       ?__LINE__Var@?1??DirTree_CreateFromFile@@9@9 102af44c     wzFilePacker_static_d:dirtree.obj
 0004:00011450       ?__LINE__Var@?1??ReadTree@@9@9@6bd7c2e6 102af450     wzFilePacker_static_d:dirtree.obj
 0004:00011454       ?__LINE__Var@?1??ReadTreeCount@@9@9@6bd7c2e6 102af454     wzFilePacker_static_d:dirtree.obj
 0004:00011458       ?__LINE__Var@?1??DirTree_FindExact@@9@9 102af458     wzFilePacker_static_d:dirtree.obj
 0004:0001145c       ?__LINE__Var@?1??DirTree_FindPartial@@9@9 102af45c     wzFilePacker_static_d:dirtree.obj
 0004:00011460       ?__LINE__Var@?1??DirTree_AddFile@@9@9 102af460     wzFilePacker_static_d:dirtree.obj
 0004:00011464       ?__LINE__Var@?1??DirTree_Remove@@9@9 102af464     wzFilePacker_static_d:dirtree.obj
 0004:00011468       ?__LINE__Var@?1??DirTree_SetFileAttributes@@9@9 102af468     wzFilePacker_static_d:dirtree.obj
 0004:0001146c       ?__LINE__Var@?1??DirTree_GetFileAttributes@@9@9 102af46c     wzFilePacker_static_d:dirtree.obj
 0004:00011470       ?__LINE__Var@?1??DirTree_SetFileOffset@@9@9 102af470     wzFilePacker_static_d:dirtree.obj
 0004:00011474       ?__LINE__Var@?1??DirTree_GetFileOffset@@9@9 102af474     wzFilePacker_static_d:dirtree.obj
 0004:00011478       ?__LINE__Var@?1??DirTree_SetFileTime@@9@9 102af478     wzFilePacker_static_d:dirtree.obj
 0004:0001147c       ?__LINE__Var@?1??DirTree_GetFileTime@@9@9 102af47c     wzFilePacker_static_d:dirtree.obj
 0004:00011480       ?__LINE__Var@?1??DirTree_SetFileHints@@9@9 102af480     wzFilePacker_static_d:dirtree.obj
 0004:00011484       ?__LINE__Var@?1??DirTree_GetName@@9@9 102af484     wzFilePacker_static_d:dirtree.obj
 0004:00011488       ?__LINE__Var@?1??DirTree_CreateFinder@@9@9 102af488     wzFilePacker_static_d:dirtree.obj
 0004:0001148c       ?__LINE__Var@?1??DirTree_DestroyFinder@@9@9 102af48c     wzFilePacker_static_d:dirtree.obj
 0004:00011490       ?__LINE__Var@?1??DirTree_FinderGetNextFile@@9@9 102af490     wzFilePacker_static_d:dirtree.obj
 0004:00011494       ?__LINE__Var@?1??DuplicateString@@9@9 102af494     wzFilePacker_static_d:dirtree-common.obj
 0004:00011498       ?__LINE__Var@?1??MatchPattern@@9@9 102af498     wzFilePacker_static_d:dirtree-common.obj
 0004:000119dc       ??_C@_04BABO@OggS?$AA@     102af9dc     ogg_static:framing.obj
 0004:00015000       ?Compressed_buffer@@3PAEA  102b3000     audiostr.obj
 0004:0002a8ec       ?Global_service_lock@@3U_RTL_CRITICAL_SECTION@@A 102c88ec     audiostr.obj
 0004:0002a904       ?m_ass@@3VAudioStreamServices@@A 102c8904     audiostr.obj
 0004:0002a908       ?Wavedata_service_buffer@@3PAEA 102c8908     audiostr.obj
 0004:00056828       ?Compressed_service_buffer@@3PAEA 102f4828     audiostr.obj
 0004:0006c118       ?Wavedata_load_buffer@@3PAEA 1030a118     audiostr.obj
 0004:00098038       ?Audiostream_inited@@3HA   10336038     audiostr.obj
 0004:00098040       ?Audio_streams@@3PAVAudioStream@@A 10336040     audiostr.obj
 0004:000b3e88       ?ds_hardware_buffers@@3PAUds_sound_buffer@@A 10351e88     ds.obj
 0004:000b4608       ?ds_software_buffers@@3PAUds_sound_buffer@@A 10352608     ds.obj
 0004:000c3608       ?ds_vol_lookup@@3PAHA      10361608     ds.obj
 0004:000c3800       ?pfn_DirectSoundCreate8@@3P6GJPAU_GUID@@PAPAUIDirectSound8@@PAUIUnknown@@@ZA 10361800     ds.obj
 0004:000c3804       ?Ds_dll_loaded@@3HA        10361804     ds.obj
 0004:000c3808       ?Ds_dll_handle@@3PAUHINSTANCE__@@A 10361808     ds.obj
 0004:000c380c       ?pDirectSound8@@3PAUIDirectSound8@@A 1036180c     ds.obj
 0004:000c3810       ?pPrimaryBuffer@@3PAUIDirectSoundBuffer@@A 10361810     ds.obj
 0004:000c3824       ?Channels@@3PAUchannel@@A  10361824     ds.obj
 0004:000c383c       ?ds_initialized@@3HA       1036183c     ds.obj
 0004:000c6a38       ?DS3D_inited@@3HA          10364a38     ds3d.obj
 0004:000c6a3c       ?pDS3D_listener@@3PAUIDirectSound3DListener@@A 10364a3c     ds3d.obj
 0004:000c6a44       ?UserSampleBits@@3GA       10364a44     sound.obj
 0004:000c6a4c       ?UserSampleRate@@3GA       10364a4c     sound.obj
 0004:000c6a54       ?View_matrix@@3Umatrix@@A  10364a54     sound.obj
 0004:000c6a78       ?Snd_hram@@3HA             10364a78     sound.obj
 0004:000c6a7c       ?Snd_sram@@3HA             10364a7c     sound.obj
 0004:000c6a80       ?View_position@@3Uvector@@A 10364a80     sound.obj
 0004:000c6a94       ?Is_sound_cache@@3_NA      10364a94     sound.obj
 0004:000c6a98       ?map_sounds@@3V?$map@HUsound@@U?$less@H@std@@V?$allocator@U?$pair@$$CBHUsound@@@std@@@3@@std@@A 10364a98     sound.obj
 0004:000c6acc       ?cfile_callbacks@@3Uov_callbacks@@A 10364acc     ogg.obj
 0004:000c6adc       ?mmio_callbacks@@3Uov_callbacks@@A 10364adc     ogg.obj
 0004:000c6aec       ?ogg_inited@@3HA           10364aec     ogg.obj
 0004:000c6af8       ?ambi_handles@@3V?$map@HHU?$less@H@std@@V?$allocator@U?$pair@$$CBHH@std@@@2@@std@@A 10364af8     ambientsnd.obj
 0004:000c6b20       ?Event_music@@3PAUEventMusic@@A 10364b20     eventmusic.obj
 0004:000cd3d0       ?Num_music_files@@3HA      1036b3d0     eventmusic.obj
 0004:000cd3d4       ?music_handles@@3V?$map@HHU?$less@H@std@@V?$allocator@U?$pair@$$CBHH@std@@@2@@std@@A 1036b3d4     eventmusic.obj
 0004:000ce8ec       ?index_table_event_music@@3V?$map@HHU?$less@H@std@@V?$allocator@U?$pair@$$CBHH@std@@@2@@std@@A 1036c8ec     scriptparser.obj
 0004:000ce908       ?Snds@@3V?$map@HUgame_snd@@U?$less@H@std@@V?$allocator@U?$pair@$$CBHUgame_snd@@@std@@@3@@std@@A 1036c908     scriptparser.obj
 0004:000ce924       ?index_table_voice_sound@@3V?$map@HHU?$less@H@std@@V?$allocator@U?$pair@$$CBHH@std@@@2@@std@@A 1036c924     scriptparser.obj
 0004:000ce940       ?Snds_iface@@3V?$map@HUgame_snd@@U?$less@H@std@@V?$allocator@U?$pair@$$CBHUgame_snd@@@std@@@3@@std@@A 1036c940     scriptparser.obj
 0004:000ce95c       ?VoiceTbl@@3V?$map@HUVoiceSnd@@U?$less@H@std@@V?$allocator@U?$pair@$$CBHUVoiceSnd@@@std@@@3@@std@@A 1036c95c     scriptparser.obj
 0004:000ce978       ?AmbientTbl@@3V?$map@HUAmbientSnd@@U?$less@H@std@@V?$allocator@U?$pair@$$CBHUAmbientSnd@@@std@@@3@@std@@A 1036c978     scriptparser.obj
 0004:000ce9b8       ?voice_snd@@3PAUVoiceSnd@@A 1036c9b8     voicesnd.obj
 0004:001119b8       ?Num_voice_files@@3HA      103af9b8     voicesnd.obj
 0004:001119bc       ?voice_handles@@3V?$map@HHU?$less@H@std@@V?$allocator@U?$pair@$$CBHH@std@@@2@@std@@A 103af9bc     voicesnd.obj
 0004:0011f048       ?Timing_frame@@3Utiming@@A 103bd048     timer.obj
 0004:0011f0b0       ?Timing_events@@3PAUtiming@@A 103bd0b0     timer.obj
 0004:0011f540       ?Timing_event_count@@3HA   103bd540     timer.obj
 0004:0011f644       _enable_debugLog           103bd644     util_debug.obj
 0004:0011f648       ?hVFS@@3PAXA               103bd648     util_packfile.obj
 0004:0011f650       ?packFile@@3VCPackFile@@A  103bd650     util_packfile.obj
 0004:0011fb28       ?Cfile_list@@3PAUCFILE@@A  103bdb28     cfile.obj
 0004:00120128       ?cfile_inited@@3HA         103be128     cfile.obj
 0004:00120260       ?fi@@3T_flint@@A           103be260     floating.obj
 0004:00120264       ?fo@@3T_flint@@A           103be264     floating.obj
 0004:00120270       ?vmd_zero_vector@@3Uvector@@A 103be270     vecmat.obj
 0004:00120284       ?Rand_count@@3HA           103be284     systemvars.obj
 0004:0012028c       ?libxls_minor_version@@3HA 103be28c     version.obj
 0004:00120290       ?libxls_micro_version@@3HA 103be290     version.obj
 0004:001202a0       ?dwMaxMicVol_output@@3KA   103be2a0     wzSound.obj
 0004:001202a4       ?dwMinMicVol_output@@3KA   103be2a4     wzSound.obj
 0004:001202a8       ?isInitialized@@3HA        103be2a8     wzSound.obj
 0004:001202ac       ?g_mixer_speaker@@3PAUHMIXER__@@A 103be2ac     wzSound.obj
 0004:001202b0       ?g_mixer_microphone@@3PAUHMIXER__@@A 103be2b0     wzSound.obj
 0004:001202b4       ?dwMinMasterVol@@3KA       103be2b4     wzSound.obj
 0004:001202b8       ?dwMaxMasterVol@@3KA       103be2b8     wzSound.obj
 0004:001202bc       ?lMinMasterPan@@3JA        103be2bc     wzSound.obj
 0004:001202c0       ?lMaxMasterPan@@3JA        103be2c0     wzSound.obj
 0004:001202c4       ?dwMinWavVol@@3KA          103be2c4     wzSound.obj
 0004:001202c8       ?dwMaxWavVol@@3KA          103be2c8     wzSound.obj
 0004:001202cc       ?lMinWavPan@@3JA           103be2cc     wzSound.obj
 0004:001202d0       ?lMaxWavPan@@3JA           103be2d0     wzSound.obj
 0004:001202d4       ?dwMinMicVol_input@@3PAKA  103be2d4     wzSound.obj
 0004:001202e8       ?dwMaxMicVol_input@@3PAKA  103be2e8     wzSound.obj
 0004:001202fc       ?dwMicCount_input@@3KA     103be2fc     wzSound.obj
 0004:00120300       ?lMinMicPan@@3JA           103be300     wzSound.obj
 0004:00120304       ?lMaxMicPan@@3JA           103be304     wzSound.obj
 0004:00120308       ?psz_ConfigFile@@3PADA     103be308     wzSound.obj
 0004:0012040c       ?use_secure_filesystem@@3HA 103be40c     wzSound.obj
 0004:00120410       ?psz_VoiceFile@@3PADA      103be410     wzSound.obj
 0004:00120514       ?_doppler_factor@@3MA      103be514     wzSound.obj
 0004:00120518       ?psz_MusicFile@@3PADA      103be518     wzSound.obj
 0004:0012061c       ?_3DQuality@@3KA           103be61c     wzSound.obj
 0004:00120620       ?psz_SoundFile@@3PADA      103be620     wzSound.obj
 0004:00120728       ?psz_secure_filesystem@@3PADA 103be728     wzSound.obj
 0004:00120830       ?psz_local_filesystem@@3PADA 103be830     wzSound.obj
 0004:00120b08       ___fastflag                103beb08     LIBCMTD:_fpinit_.obj
 0004:00120b0c       __adjust_fdiv              103beb0c     LIBCMTD:_fpinit_.obj
 0004:00120b10       ___pInvalidArgHandler      103beb10     LIBCMTD:invarg.obj
 0004:00120b24       ?wsprintffp@@3P6AHPADPBDZZA 103beb24     LIBCMTD:_error_.obj
 0004:00120b40       ?_pfnDumpClient@@3P6AXPAXI@ZA 103beb40     LIBCMTD:dbgheap.obj
 0004:00120b48       ___crtDebugCheckCount      103beb48     LIBCMTD:dbgheap.obj
 0004:00120b54       __aenvptr                  103beb54     LIBCMTD:dllcrt0.obj
 0004:00120b58       __wenvptr                  103beb58     LIBCMTD:dllcrt0.obj
 0004:00120b5c       ___error_mode              103beb5c     LIBCMTD:dllcrt0.obj
 0004:00120b60       ___app_type                103beb60     LIBCMTD:dllcrt0.obj
 0004:00120b64       __cflush                   103beb64     LIBCMTD:_file.obj
 0004:00120b68       __umaskval                 103beb68     LIBCMTD:crt0dat.obj
 0004:00120b6c       ___argc                    103beb6c     LIBCMTD:crt0dat.obj
 0004:00120b70       ___argv                    103beb70     LIBCMTD:crt0dat.obj
 0004:00120b74       ___wargv                   103beb74     LIBCMTD:crt0dat.obj
 0004:00120b78       __environ                  103beb78     LIBCMTD:crt0dat.obj
 0004:00120b7c       ___initenv                 103beb7c     LIBCMTD:crt0dat.obj
 0004:00120b80       __wenviron                 103beb80     LIBCMTD:crt0dat.obj
 0004:00120b84       ___winitenv                103beb84     LIBCMTD:crt0dat.obj
 0004:00120b88       __pgmptr                   103beb88     LIBCMTD:crt0dat.obj
 0004:00120b8c       __wpgmptr                  103beb8c     LIBCMTD:crt0dat.obj
 0004:00120b90       __exitflag                 103beb90     LIBCMTD:crt0dat.obj
 0004:00120b94       __C_Termination_Done       103beb94     LIBCMTD:crt0dat.obj
 0004:00120b98       __C_Exit_Done              103beb98     LIBCMTD:crt0dat.obj
 0004:00120ba8       __newmode                  103beba8     LIBCMTD:_newmode.obj
 0004:00120bb0       ___mbulinfo                103bebb0     LIBCMTD:mbctype.obj
 0004:00120bbc       ___mbcodepage              103bebbc     LIBCMTD:mbctype.obj
 0004:00120bc0       ___ismbcodepage            103bebc0     LIBCMTD:mbctype.obj
 0004:00120bc4       ___mblcid                  103bebc4     LIBCMTD:mbctype.obj
 0004:00120bc8       ___locale_changed          103bebc8     LIBCMTD:setlocal.obj
 0004:00120bcc       ___lc_handle               103bebcc     LIBCMTD:nlsdata2.obj
 0004:00120be4       ___lc_codepage             103bebe4     LIBCMTD:nlsdata2.obj
 0004:00120be8       ___lc_collate_cp           103bebe8     LIBCMTD:nlsdata2.obj
 0004:00120bec       _gpFlsAlloc                103bebec     LIBCMTD:tidtable.obj
 0004:00120bf0       _gpFlsGetValue             103bebf0     LIBCMTD:tidtable.obj
 0004:00120bf4       _gpFlsSetValue             103bebf4     LIBCMTD:tidtable.obj
 0004:00120bf8       _gpFlsFree                 103bebf8     LIBCMTD:tidtable.obj
 0004:00120f24       ?__pInconsistency@@3P6AXXZA 103bef24     LIBCMTD:hooks.obj
 0004:001210c0       ?_pnhHeap@@3P6AHI@ZA       103bf0c0     LIBCMTD:handler.obj
 0004:001210d0       __stdbuf                   103bf0d0     LIBCMTD:_sftbuf.obj
 0004:001210e0       __crtheap                  103bf0e0     LIBCMTD:heapinit.obj
 0004:001210e4       ___sbh_pHeaderDefer        103bf0e4     LIBCMTD:sbheap.obj
 0004:00121520       ___pPurecall               103bf520     LIBCMTD:inithelp.obj
 0004:0012152c       ___lconv_static_null       103bf52c     LIBCMTD:lconv.obj
 0004:00121530       __outputformat             103bf530     LIBCMTD:outputformat.obj
 0004:00121548       ?pArgList@UnDecorator@@0PAVReplicator@@A 103bf548     LIBCMTD:undname.obj
 0004:0012154c       ?pZNameList@UnDecorator@@0PAVReplicator@@A 103bf54c     LIBCMTD:undname.obj
 0004:00121550       ?pTemplateArgList@UnDecorator@@0PAVReplicator@@A 103bf550     LIBCMTD:undname.obj
 0004:00121554       ?gName@UnDecorator@@0PBDB  103bf554     LIBCMTD:undname.obj
 0004:00121558       ?name@UnDecorator@@0PBDB   103bf558     LIBCMTD:undname.obj
 0004:0012155c       ?outputString@UnDecorator@@0PADA 103bf55c     LIBCMTD:undname.obj
 0004:00121560       ?maxStringLength@UnDecorator@@0HA 103bf560     LIBCMTD:undname.obj
 0004:00121564       ?disableFlags@UnDecorator@@0KA 103bf564     LIBCMTD:undname.obj
 0004:00121568       ?m_pGetParameter@UnDecorator@@0P6APADJ@ZA 103bf568     LIBCMTD:undname.obj
 0004:0012156c       ?fExplicitTemplateParams@UnDecorator@@0_NA 103bf56c     LIBCMTD:undname.obj
 0004:0012156d       ?fGetTemplateArgumentList@UnDecorator@@0_NA 103bf56d     LIBCMTD:undname.obj
 0004:001215c0       ?nodes@?1??make@DNameStatusNode@@SAPAV2@W4DNameStatus@@@Z@4PAV2@A 103bf5c0     LIBCMTD:undname.obj
 0004:001215f0       ??_B?1??make@DNameStatusNode@@SAPAV1@W4DNameStatus@@@Z@51 103bf5f0     LIBCMTD:undname.obj
 0004:001215f4       __commode                  103bf5f4     LIBCMTD:ncommode.obj
 0004:001216c8       __fmode                    103bf6c8     LIBCMTD:txtmode.obj
 0004:001216d0       ??_C@_00A@?$AA@            103bf6d0     iconv:localcharset.obj
 0004:001216e8       ?autofree@@3VCAutoFree@@A  103bf6e8     wzFilePacker_static_d:wzFilePacker.obj
 0004:001216f8       _dwTreeCount               103bf6f8     wzFilePacker_static_d:vfile.obj
 0004:001216fc       _g_nTreeArrayCount         103bf6fc     wzFilePacker_static_d:vfile.obj
 0004:00121700       _g_ulStartBinaryOffset     103bf700     wzFilePacker_static_d:vfile.obj
 0004:00121708       _g_ulTatalBinarySize       103bf708     wzFilePacker_static_d:vfile.obj
 0004:00121720       _bCurDirCreated            103bf720     wzFilePacker_static_d:vFile_util.obj
 0004:0012172c       _geRam_CurrentlyUsed       103bf72c     wzFilePacker_static_d:Ram.obj
 0004:00121730       _geRam_MaximumUsed         103bf730     wzFilePacker_static_d:Ram.obj
 0004:00121734       _geRam_NumberOfAllocations 103bf734     wzFilePacker_static_d:Ram.obj
 0004:00121738       _geRam_MaximumNumberOfAllocations 103bf738     wzFilePacker_static_d:Ram.obj
 0004:00122214       __maxwait                  103c0214     libcmt:crtheap.obj
 0004:00122218       __pmatherr                 103c0218     <common>
 0004:00122224       ___sbh_initialized         103c0224     <common>
 0004:00122238       ___sbh_cntHeaderList       103c0238     <common>
 0004:0012223c       ___sbh_pHeaderList         103c023c     <common>
 0004:00122240       ___sbh_threshold           103c0240     <common>
 0004:00122244       ___sbh_pHeaderScan         103c0244     <common>
 0004:00122248       ___sbh_sizeHeaderList      103c0248     <common>
 0004:0012224c       ___sbh_indGroupDefer       103c024c     <common>
 0004:00122250       ___active_heap             103c0250     <common>
 0004:0012225c       __nhandle                  103c025c     <common>
 0004:001222a0       ___pioinfo                 103c02a0     <common>
 0004:001223a0       __pfnReportHook            103c03a0     <common>
 0004:001223b0       __pReportHookListW         103c03b0     <common>
 0004:001223b4       __pReportHookList          103c03b4     <common>
 0004:001223b8       __debugger_hook_dummy      103c03b8     <common>
 0004:001223c4       ___use_sse2_mathfcns       103c03c4     <common>
 0004:001223d0       ___setlc_active            103c03d0     <common>
 0004:001223e0       ___unguarded_readlc_active 103c03e0     <common>
 0004:001223e4       ___sse2_available          103c03e4     <common>
 0004:001223f0       ___env_initialized         103c03f0     <common>
 0004:00122400       ___onexitend               103c0400     <common>
 0004:00122404       ___onexitbegin             103c0404     <common>
 0004:00122408       ___mbctype_initialized     103c0408     <common>
 0004:0012240c       ___dyn_tls_init_callback   103c040c     <common>
 0004:00122410       ___piob                    103c0410     <common>
 0004:00122760       __bufin                    103c0760     <common>
 0004:00123760       __nstream                  103c1760     <common>
 0004:00123764       __acmdln                   103c1764     <common>
 0004:00123770       _StupidUnusedPointer       103c1770     <common>
 0004:00123780       _lpszCurDir                103c1780     <common>
 0004:00123c60       _g_TreeList                103c1c60     <common>
 0005:00000000       __IMPORT_DESCRIPTOR_KERNEL32 103c3000     kernel32:KERNEL32.dll
 0005:00000014       __IMPORT_DESCRIPTOR_USER32 103c3014     user32:USER32.dll
 0005:00000028       __IMPORT_DESCRIPTOR_ole32  103c3028     ole32:ole32.dll
 0005:0000003c       __IMPORT_DESCRIPTOR_WINMM  103c303c     winmm:WINMM.dll
 0005:00000050       __IMPORT_DESCRIPTOR_dbghelp 103c3050     Dbghelp:dbghelp.dll
 0005:00000064       __NULL_IMPORT_DESCRIPTOR   103c3064     kernel32:KERNEL32.dll
 0005:000003f8       __imp__InitializeCriticalSection@4 103c33f8     kernel32:KERNEL32.dll
 0005:000003fc       __imp__DeleteCriticalSection@4 103c33fc     kernel32:KERNEL32.dll
 0005:00000400       __imp__LeaveCriticalSection@4 103c3400     kernel32:KERNEL32.dll
 0005:00000404       __imp__EnterCriticalSection@4 103c3404     kernel32:KERNEL32.dll
 0005:00000408       __imp__InterlockedExchange@8 103c3408     kernel32:KERNEL32.dll
 0005:0000040c       __imp__GetCurrentDirectoryA@8 103c340c     kernel32:KERNEL32.dll
 0005:00000410       __imp__GetProcAddress@8    103c3410     kernel32:KERNEL32.dll
 0005:00000414       __imp__LoadLibraryA@4      103c3414     kernel32:KERNEL32.dll
 0005:00000418       __imp__FreeLibrary@4       103c3418     kernel32:KERNEL32.dll
 0005:0000041c       __imp__Sleep@4             103c341c     kernel32:KERNEL32.dll
 0005:00000420       __imp__GetLastError@0      103c3420     kernel32:KERNEL32.dll
 0005:00000424       __imp__LocalFree@4         103c3424     kernel32:KERNEL32.dll
 0005:00000428       __imp__LocalAlloc@8        103c3428     kernel32:KERNEL32.dll
 0005:0000042c       __imp__OutputDebugStringA@4 103c342c     kernel32:KERNEL32.dll
 0005:00000430       __imp__GetFileAttributesA@4 103c3430     kernel32:KERNEL32.dll
 0005:00000434       __imp__GetModuleFileNameA@12 103c3434     kernel32:KERNEL32.dll
 0005:00000438       __imp__GetDriveTypeA@4     103c3438     kernel32:KERNEL32.dll
 0005:0000043c       __imp__MulDiv@12           103c343c     kernel32:KERNEL32.dll
 0005:00000440       __imp__FileTimeToLocalFileTime@8 103c3440     kernel32:KERNEL32.dll
 0005:00000444       __imp__FileTimeToSystemTime@8 103c3444     kernel32:KERNEL32.dll
 0005:00000448       __imp__MoveFileA@8         103c3448     kernel32:KERNEL32.dll
 0005:0000044c       __imp__DeleteFileA@4       103c344c     kernel32:KERNEL32.dll
 0005:00000450       __imp__SetFileTime@16      103c3450     kernel32:KERNEL32.dll
 0005:00000454       __imp__SetFileAttributesA@8 103c3454     kernel32:KERNEL32.dll
 0005:00000458       __imp__GetFileInformationByHandle@8 103c3458     kernel32:KERNEL32.dll
 0005:0000045c       __imp__GetFileSizeEx@8     103c345c     kernel32:KERNEL32.dll
 0005:00000460       __imp__SetFilePointerEx@20 103c3460     kernel32:KERNEL32.dll
 0005:00000464       __imp__CreateDirectoryA@8  103c3464     kernel32:KERNEL32.dll
 0005:00000468       __imp__GetSystemDirectoryA@8 103c3468     kernel32:KERNEL32.dll
 0005:0000046c       __imp__RemoveDirectoryA@4  103c346c     kernel32:KERNEL32.dll
 0005:00000470       __imp__FindClose@4         103c3470     kernel32:KERNEL32.dll
 0005:00000474       __imp__FindFirstFileA@8    103c3474     kernel32:KERNEL32.dll
 0005:00000478       __imp__FindNextFileA@8     103c3478     kernel32:KERNEL32.dll
 0005:0000047c       __imp__lstrcpyA@8          103c347c     kernel32:KERNEL32.dll
 0005:00000480       __imp__SetEnvironmentVariableA@8 103c3480     kernel32:KERNEL32.dll
 0005:00000484       __imp__CompareStringW@24   103c3484     kernel32:KERNEL32.dll
 0005:00000488       __imp__CompareStringA@24   103c3488     kernel32:KERNEL32.dll
 0005:0000048c       __imp__SetEndOfFile@4      103c348c     kernel32:KERNEL32.dll
 0005:00000490       __imp__GetTimeZoneInformation@4 103c3490     kernel32:KERNEL32.dll
 0005:00000494       __imp__GetLocaleInfoW@16   103c3494     kernel32:KERNEL32.dll
 0005:00000498       __imp__GetConsoleOutputCP@0 103c3498     kernel32:KERNEL32.dll
 0005:0000049c       __imp__WriteConsoleA@20    103c349c     kernel32:KERNEL32.dll
 0005:000004a0       __imp__InterlockedIncrement@4 103c34a0     kernel32:KERNEL32.dll
 0005:000004a4       __imp__InterlockedDecrement@4 103c34a4     kernel32:KERNEL32.dll
 0005:000004a8       __imp__RtlUnwind@16        103c34a8     kernel32:KERNEL32.dll
 0005:000004ac       __imp__TerminateProcess@8  103c34ac     kernel32:KERNEL32.dll
 0005:000004b0       __imp__GetCurrentProcess@0 103c34b0     kernel32:KERNEL32.dll
 0005:000004b4       __imp__UnhandledExceptionFilter@4 103c34b4     kernel32:KERNEL32.dll
 0005:000004b8       __imp__SetUnhandledExceptionFilter@4 103c34b8     kernel32:KERNEL32.dll
 0005:000004bc       __imp__IsDebuggerPresent@0 103c34bc     kernel32:KERNEL32.dll
 0005:000004c0       __imp__GetModuleFileNameW@12 103c34c0     kernel32:KERNEL32.dll
 0005:000004c4       __imp__RaiseException@16   103c34c4     kernel32:KERNEL32.dll
 0005:000004c8       __imp__DebugBreak@0        103c34c8     kernel32:KERNEL32.dll
 0005:000004cc       __imp__WideCharToMultiByte@32 103c34cc     kernel32:KERNEL32.dll
 0005:000004d0       __imp__MultiByteToWideChar@24 103c34d0     kernel32:KERNEL32.dll
 0005:000004d4       __imp__lstrlenA@4          103c34d4     kernel32:KERNEL32.dll
 0005:000004d8       __imp__HeapValidate@12     103c34d8     kernel32:KERNEL32.dll
 0005:000004dc       __imp__IsBadReadPtr@8      103c34dc     kernel32:KERNEL32.dll
 0005:000004e0       __imp__GetCurrentThreadId@0 103c34e0     kernel32:KERNEL32.dll
 0005:000004e4       __imp__GetCommandLineA@0   103c34e4     kernel32:KERNEL32.dll
 0005:000004e8       __imp__GetModuleHandleW@4  103c34e8     kernel32:KERNEL32.dll
 0005:000004ec       __imp__ExitProcess@4       103c34ec     kernel32:KERNEL32.dll
 0005:000004f0       __imp__GetACP@0            103c34f0     kernel32:KERNEL32.dll
 0005:000004f4       __imp__GetOEMCP@0          103c34f4     kernel32:KERNEL32.dll
 0005:000004f8       __imp__GetCPInfo@8         103c34f8     kernel32:KERNEL32.dll
 0005:000004fc       __imp__IsValidCodePage@4   103c34fc     kernel32:KERNEL32.dll
 0005:00000500       __imp__TlsGetValue@4       103c3500     kernel32:KERNEL32.dll
 0005:00000504       __imp__TlsAlloc@0          103c3504     kernel32:KERNEL32.dll
 0005:00000508       __imp__TlsSetValue@8       103c3508     kernel32:KERNEL32.dll
 0005:0000050c       __imp__TlsFree@4           103c350c     kernel32:KERNEL32.dll
 0005:00000510       __imp__SetLastError@4      103c3510     kernel32:KERNEL32.dll
 0005:00000514       __imp__GetCurrentThread@0  103c3514     kernel32:KERNEL32.dll
 0005:00000518       __imp__GetModuleHandleA@4  103c3518     kernel32:KERNEL32.dll
 0005:0000051c       __imp__FatalAppExitA@8     103c351c     kernel32:KERNEL32.dll
 0005:00000520       __imp__GetStdHandle@4      103c3520     kernel32:KERNEL32.dll
 0005:00000524       __imp__WriteFile@20        103c3524     kernel32:KERNEL32.dll
 0005:00000528       __imp__WriteConsoleW@20    103c3528     kernel32:KERNEL32.dll
 0005:0000052c       __imp__GetFileType@4       103c352c     kernel32:KERNEL32.dll
 0005:00000530       __imp__OutputDebugStringW@4 103c3530     kernel32:KERNEL32.dll
 0005:00000534       __imp__SetConsoleCtrlHandler@8 103c3534     kernel32:KERNEL32.dll
 0005:00000538       __imp__LoadLibraryW@4      103c3538     kernel32:KERNEL32.dll
 0005:0000053c       __imp__HeapFree@12         103c353c     kernel32:KERNEL32.dll
 0005:00000540       __imp__HeapAlloc@12        103c3540     kernel32:KERNEL32.dll
 0005:00000544       __imp__GetProcessHeap@0    103c3544     kernel32:KERNEL32.dll
 0005:00000548       __imp__VirtualQuery@12     103c3548     kernel32:KERNEL32.dll
 0005:0000054c       __imp__CloseHandle@4       103c354c     kernel32:KERNEL32.dll
 0005:00000550       __imp__SetHandleCount@4    103c3550     kernel32:KERNEL32.dll
 0005:00000554       __imp__GetStartupInfoA@4   103c3554     kernel32:KERNEL32.dll
 0005:00000558       __imp__SetFilePointer@16   103c3558     kernel32:KERNEL32.dll
 0005:0000055c       __imp__ReadFile@20         103c355c     kernel32:KERNEL32.dll
 0005:00000560       __imp__GetConsoleCP@0      103c3560     kernel32:KERNEL32.dll
 0005:00000564       __imp__GetConsoleMode@8    103c3564     kernel32:KERNEL32.dll
 0005:00000568       __imp__HeapSize@12         103c3568     kernel32:KERNEL32.dll
 0005:0000056c       __imp__HeapReAlloc@16      103c356c     kernel32:KERNEL32.dll
 0005:00000570       __imp__HeapDestroy@4       103c3570     kernel32:KERNEL32.dll
 0005:00000574       __imp__HeapCreate@12       103c3574     kernel32:KERNEL32.dll
 0005:00000578       __imp__VirtualFree@12      103c3578     kernel32:KERNEL32.dll
 0005:0000057c       __imp__VirtualAlloc@16     103c357c     kernel32:KERNEL32.dll
 0005:00000580       __imp__FreeEnvironmentStringsA@4 103c3580     kernel32:KERNEL32.dll
 0005:00000584       __imp__GetEnvironmentStrings@0 103c3584     kernel32:KERNEL32.dll
 0005:00000588       __imp__FreeEnvironmentStringsW@4 103c3588     kernel32:KERNEL32.dll
 0005:0000058c       __imp__GetEnvironmentStringsW@0 103c358c     kernel32:KERNEL32.dll
 0005:00000590       __imp__QueryPerformanceCounter@4 103c3590     kernel32:KERNEL32.dll
 0005:00000594       __imp__GetTickCount@0      103c3594     kernel32:KERNEL32.dll
 0005:00000598       __imp__GetCurrentProcessId@0 103c3598     kernel32:KERNEL32.dll
 0005:0000059c       __imp__GetSystemTimeAsFileTime@4 103c359c     kernel32:KERNEL32.dll
 0005:000005a0       __imp__FlushFileBuffers@4  103c35a0     kernel32:KERNEL32.dll
 0005:000005a4       __imp__LCMapStringA@24     103c35a4     kernel32:KERNEL32.dll
 0005:000005a8       __imp__LCMapStringW@24     103c35a8     kernel32:KERNEL32.dll
 0005:000005ac       __imp__SetStdHandle@8      103c35ac     kernel32:KERNEL32.dll
 0005:000005b0       __imp__InitializeCriticalSectionAndSpinCount@8 103c35b0     kernel32:KERNEL32.dll
 0005:000005b4       __imp__GetStringTypeA@20   103c35b4     kernel32:KERNEL32.dll
 0005:000005b8       __imp__GetStringTypeW@16   103c35b8     kernel32:KERNEL32.dll
 0005:000005bc       __imp__GetTimeFormatA@24   103c35bc     kernel32:KERNEL32.dll
 0005:000005c0       __imp__GetDateFormatA@24   103c35c0     kernel32:KERNEL32.dll
 0005:000005c4       __imp__GetLocaleInfoA@16   103c35c4     kernel32:KERNEL32.dll
 0005:000005c8       __imp__IsValidLocale@8     103c35c8     kernel32:KERNEL32.dll
 0005:000005cc       __imp__EnumSystemLocalesA@8 103c35cc     kernel32:KERNEL32.dll
 0005:000005d0       __imp__GetUserDefaultLCID@0 103c35d0     kernel32:KERNEL32.dll
 0005:000005d4       __imp__CreateFileA@28      103c35d4     kernel32:KERNEL32.dll
 0005:000005d8       \177KERNEL32_NULL_THUNK_DATA 103c35d8     kernel32:KERNEL32.dll
 0005:00000664       __imp__wsprintfA           103c3664     user32:USER32.dll
 0005:00000668       __imp__SendMessageA@16     103c3668     user32:USER32.dll
 0005:0000066c       __imp__GetDesktopWindow@0  103c366c     user32:USER32.dll
 0005:00000670       \177USER32_NULL_THUNK_DATA 103c3670     user32:USER32.dll
 0005:0000069c       __imp__mixerGetControlDetailsA@12 103c369c     winmm:WINMM.dll
 0005:000006a0       __imp__mixerGetLineControlsA@12 103c36a0     winmm:WINMM.dll
 0005:000006a4       __imp__mixerGetLineInfoA@12 103c36a4     winmm:WINMM.dll
 0005:000006a8       __imp__mixerGetNumDevs@0   103c36a8     winmm:WINMM.dll
 0005:000006ac       __imp__mixerOpen@20        103c36ac     winmm:WINMM.dll
 0005:000006b0       __imp__mixerGetDevCapsA@12 103c36b0     winmm:WINMM.dll
 0005:000006b4       __imp__mixerSetControlDetails@12 103c36b4     winmm:WINMM.dll
 0005:000006b8       __imp__timeBeginPeriod@4   103c36b8     winmm:WINMM.dll
 0005:000006bc       __imp__timeGetTime@0       103c36bc     winmm:WINMM.dll
 0005:000006c0       __imp__timeEndPeriod@4     103c36c0     winmm:WINMM.dll
 0005:000006c4       __imp__mmioRead@12         103c36c4     winmm:WINMM.dll
 0005:000006c8       __imp__mmioSeek@12         103c36c8     winmm:WINMM.dll
 0005:000006cc       __imp__mmioClose@8         103c36cc     winmm:WINMM.dll
 0005:000006d0       __imp__timeSetEvent@20     103c36d0     winmm:WINMM.dll
 0005:000006d4       __imp__timeKillEvent@4     103c36d4     winmm:WINMM.dll
 0005:000006d8       __imp__mixerClose@4        103c36d8     winmm:WINMM.dll
 0005:000006dc       \177WINMM_NULL_THUNK_DATA  103c36dc     winmm:WINMM.dll
 0005:00000714       __imp__MakeSureDirectoryPathExists@4 103c3714     Dbghelp:dbghelp.dll
 0005:00000718       \177dbghelp_NULL_THUNK_DATA 103c3718     Dbghelp:dbghelp.dll
 0005:00000744       __imp__CoInitialize@4      103c3744     ole32:ole32.dll
 0005:00000748       __imp__CoUninitialize@0    103c3748     ole32:ole32.dll
 0005:0000074c       \177ole32_NULL_THUNK_DATA  103c374c     ole32:ole32.dll

 entry point at        0002:000010bd

